Archive member included because of file (symbol)

c:/program files (x86)/microchip/xc32/v1.21/bin/../lib/gcc/pic32mx/4.5.2/../../../../pic32mx/lib/size\libmchp_peripheral.a(open_core_timer_lib.o)
                              build/default/production/_ext/365611741/system_services.o (OpenCoreTimer)
c:/program files (x86)/microchip/xc32/v1.21/bin/../lib/gcc/pic32mx/4.5.2/../../../../pic32mx/lib/size\libmchp_peripheral_32MX795F512L.a(soft_reset_lib.o)
                              build/default/production/_ext/365611741/system_services.o (SoftReset)
c:/program files (x86)/microchip/xc32/v1.21/bin/../lib/gcc/pic32mx/4.5.2/../../../../pic32mx/lib/size\libmchp_peripheral_32MX795F512L.a(pcache.o)
                              build/default/production/_ext/365611741/system_services.o (CheKseg0CacheOn)
c:/program files (x86)/microchip/xc32/v1.21/bin/../lib/gcc/pic32mx/4.5.2/../../../../pic32mx/lib/size\libmchp_peripheral_32MX795F512L.a(int_disable_interrupts_lib.o)
                              build/default/production/_ext/365611741/system_services.o (INTDisableInterrupts)
c:/program files (x86)/microchip/xc32/v1.21/bin/../lib/gcc/pic32mx/4.5.2/../../../../pic32mx/lib/size\libmchp_peripheral_32MX795F512L.a(int_restore_interrupts_lib.o)
                              build/default/production/_ext/365611741/system_services.o (INTRestoreInterrupts)
c:/program files (x86)/microchip/xc32/v1.21/bin/../lib/gcc/pic32mx/4.5.2/../../../../pic32mx/lib/size\libmchp_peripheral_32MX795F512L.a(int_enable_mv_int_lib.o)
                              build/default/production/_ext/365611741/system_services.o (INTEnableSystemMultiVectoredInt)
c:/program files (x86)/microchip/xc32/v1.21/bin/../lib/gcc/pic32mx/4.5.2/../../../../pic32mx/lib/size\libmchp_peripheral_32MX795F512L.a(int_tbl_lib.o)
                              build/default/production/_ext/365611741/system_services.o (INTClearFlag)
c:/program files (x86)/microchip/xc32/v1.21/bin/../lib/gcc/pic32mx/4.5.2/../../../../pic32mx/lib/size\libmchp_peripheral_32MX795F512L.a(rtcc_init_lib.o)
                              build/default/production/_ext/365611741/system_services.o (RtccInit)
c:/program files (x86)/microchip/xc32/v1.21/bin/../lib/gcc/pic32mx/4.5.2/../../../../pic32mx/lib/size\libmchp_peripheral_32MX795F512L.a(rtcc_open_lib.o)
                              build/default/production/_ext/365611741/system_services.o (RtccOpen)
c:/program files (x86)/microchip/xc32/v1.21/bin/../lib/gcc/pic32mx/4.5.2/../../../../pic32mx/lib/size\libmchp_peripheral_32MX795F512L.a(spi_chn_data_rdy_lib.o)
                              build/default/production/_ext/792872985/drv_spi.o (SpiChnDataRdy)
c:/program files (x86)/microchip/xc32/v1.21/bin/../lib/gcc/pic32mx/4.5.2/../../../../pic32mx/lib/size\libmchp_peripheral_32MX795F512L.a(spi_chn_getc_lib.o)
                              build/default/production/_ext/792872985/drv_spi.o (SpiChnReadC)
c:/program files (x86)/microchip/xc32/v1.21/bin/../lib/gcc/pic32mx/4.5.2/../../../../pic32mx/lib/size\libmchp_peripheral_32MX795F512L.a(spi_chn_open_lib.o)
                              build/default/production/_ext/792872985/drv_spi.o (SpiChnOpen)
c:/program files (x86)/microchip/xc32/v1.21/bin/../lib/gcc/pic32mx/4.5.2/../../../../pic32mx/lib/size\libmchp_peripheral_32MX795F512L.a(spi_chn_putc_lib.o)
                              build/default/production/_ext/792872985/drv_spi.o (SpiChnWriteC)
c:/program files (x86)/microchip/xc32/v1.21/bin/../lib/gcc/pic32mx/4.5.2/../../../../pic32mx/lib/size\libmchp_peripheral_32MX795F512L.a(spi_chn_tx_buff_empty_lib.o)
                              build/default/production/_ext/792872985/drv_spi.o (SpiChnTxBuffEmpty)
c:/program files (x86)/microchip/xc32/v1.21/bin/../lib/gcc/pic32mx/4.5.2/../../../../pic32mx/lib/size\libmchp_peripheral_32MX795F512L.a(spi_io_tbl_libp.o)
                              c:/program files (x86)/microchip/xc32/v1.21/bin/../lib/gcc/pic32mx/4.5.2/../../../../pic32mx/lib/size\libmchp_peripheral_32MX795F512L.a(spi_chn_open_lib.o) (_SpiIoTbl)
c:/program files (x86)/microchip/xc32/v1.21/bin/../lib/gcc/pic32mx/4.5.2/../../../../pic32mx/lib/size\libmchp_peripheral_32MX795F512L.a(spi_map_tbl_libp.o)
                              c:/program files (x86)/microchip/xc32/v1.21/bin/../lib/gcc/pic32mx/4.5.2/../../../../pic32mx/lib/size\libmchp_peripheral_32MX795F512L.a(spi_chn_data_rdy_lib.o) (_SpiMapTbl)
c:/program files (x86)/microchip/xc32/v1.21/bin/../lib/gcc/pic32mx/4.5.2/../../../../pic32mx/lib/size\libmchp_peripheral_32MX795F512L.a(port_set_pins_digital_in_lib.o)
                              c:/program files (x86)/microchip/xc32/v1.21/bin/../lib/gcc/pic32mx/4.5.2/../../../../pic32mx/lib/size\libmchp_peripheral_32MX795F512L.a(spi_chn_open_lib.o) (PORTSetPinsDigitalIn)
c:/program files (x86)/microchip/xc32/v1.21/bin/../lib/gcc/pic32mx/4.5.2/../../../../pic32mx/lib/size\libmchp_peripheral_32MX795F512L.a(port_set_pins_digital_out_lib.o)
                              c:/program files (x86)/microchip/xc32/v1.21/bin/../lib/gcc/pic32mx/4.5.2/../../../../pic32mx/lib/size\libmchp_peripheral_32MX795F512L.a(spi_chn_open_lib.o) (PORTSetPinsDigitalOut)
c:/program files (x86)/microchip/xc32/v1.21/bin/../lib/gcc/pic32mx/4.5.2/../../../../pic32mx/lib/size\libmchp_peripheral_32MX795F512L.a(_ports_tbl_libp.o)
                              c:/program files (x86)/microchip/xc32/v1.21/bin/../lib/gcc/pic32mx/4.5.2/../../../../pic32mx/lib/size\libmchp_peripheral_32MX795F512L.a(port_set_pins_digital_in_lib.o) (PortRegTbl)
c:/program files (x86)/microchip/xc32/v1.21/bin/../lib/gcc/pic32mx/4.5.2/../../../../pic32mx/lib/size\libmchp_peripheral_32MX795F512L.a(int_enable_interrupts_lib.o)
                              c:/program files (x86)/microchip/xc32/v1.21/bin/../lib/gcc/pic32mx/4.5.2/../../../../pic32mx/lib/size\libmchp_peripheral_32MX795F512L.a(int_enable_mv_int_lib.o) (INTEnableInterrupts)
c:/program files (x86)/microchip/xc32/v1.21/bin/../lib/gcc/pic32mx/4.5.2/../../../../pic32mx/lib/size\libmchp_peripheral_32MX795F512L.a(_rtcc_wait_clock_off_lib.o)
                              c:/program files (x86)/microchip/xc32/v1.21/bin/../lib/gcc/pic32mx/4.5.2/../../../../pic32mx/lib/size\libmchp_peripheral_32MX795F512L.a(rtcc_init_lib.o) (_RtccWaitClockOff)
c:/program files (x86)/microchip/xc32/v1.21/bin/../lib/gcc/pic32mx/4.5.2/../../../../pic32mx/lib/size\libmchp_peripheral_32MX795F512L.a(read_core_timer_lib.o)
                              c:/program files (x86)/microchip/xc32/v1.21/bin/../lib/gcc/pic32mx/4.5.2/../../../../pic32mx/lib/size\libmchp_peripheral_32MX795F512L.a(_rtcc_wait_clock_off_lib.o) (ReadCoreTimer)
c:/program files (x86)/microchip/xc32/v1.21/bin/../lib/gcc/pic32mx/4.5.2/size\libgcc.a(_udivdi3.o)
                              build/default/production/_ext/101875047/big_int.o (__udivdi3)
c:/program files (x86)/microchip/xc32/v1.21/bin/../lib/gcc/pic32mx/4.5.2/../../../../pic32mx/lib/size\libpic32.a(memcmp.o)
                              build/default/production/_ext/97638081/mpfs2.o (memcmp)
c:/program files (x86)/microchip/xc32/v1.21/bin/../lib/gcc/pic32mx/4.5.2/../../../../pic32mx/lib/size\libpic32.a(memcpy.o)
                              build/default/production/_ext/101875047/hashes.o (memcpy)
c:/program files (x86)/microchip/xc32/v1.21/bin/../lib/gcc/pic32mx/4.5.2/../../../../pic32mx/lib/size\libpic32.a(memset.o)
                              build/default/production/_ext/365611741/system_services.o (memset)
c:/program files (x86)/microchip/xc32/v1.21/bin/../lib/gcc/pic32mx/4.5.2/../../../../pic32mx/lib/size\libpic32.a(strcmp.o)
                              build/default/production/_ext/365611741/system_command.o (strcmp)
c:/program files (x86)/microchip/xc32/v1.21/bin/../lib/gcc/pic32mx/4.5.2/../../../../pic32mx/lib/size\libpic32.a(strcpy.o)
                              build/default/production/_ext/365611741/system_command.o (strcpy)
c:/program files (x86)/microchip/xc32/v1.21/bin/../lib/gcc/pic32mx/4.5.2/../../../../pic32mx/lib/size\libpic32.a(strlen.o)
                              build/default/production/_ext/101875047/helpers.o (strlen)
c:/program files (x86)/microchip/xc32/v1.21/bin/../lib/gcc/pic32mx/4.5.2/../../../../pic32mx/lib/size\libpic32.a(default-bootstrap-exception-handler.o)
                              c:/program files (x86)/microchip/xc32/v1.21/bin/../lib/gcc/pic32mx/4.5.2/../../../../pic32mx/lib/size/crt0.o (_bootstrap_exception_handler)
c:/program files (x86)/microchip/xc32/v1.21/bin/../lib/gcc/pic32mx/4.5.2/../../../../pic32mx/lib/size\libpic32.a(default-on-reset.o)
                              c:/program files (x86)/microchip/xc32/v1.21/bin/../lib/gcc/pic32mx/4.5.2/../../../../pic32mx/lib/size/crt0.o (_on_reset)
c:/program files (x86)/microchip/xc32/v1.21/bin/../lib/gcc/pic32mx/4.5.2/../../../../pic32mx/lib/size\libpic32.a(default-on-bootstrap.o)
                              c:/program files (x86)/microchip/xc32/v1.21/bin/../lib/gcc/pic32mx/4.5.2/../../../../pic32mx/lib/size/crt0.o (_on_bootstrap)
c:/program files (x86)/microchip/xc32/v1.21/bin/../lib/gcc/pic32mx/4.5.2/../../../../pic32mx/lib/size\libpic32.a(default-nmi-handler.o)
                              c:/program files (x86)/microchip/xc32/v1.21/bin/../lib/gcc/pic32mx/4.5.2/../../../../pic32mx/lib/size/crt0.o (_nmi_handler)
c:/program files (x86)/microchip/xc32/v1.21/bin/../lib/gcc/pic32mx/4.5.2/../../../../pic32mx/lib/size\libpic32.a(errno.o)
                              build/default/production/_ext/97638081/sys_fs.o (errno)
c:/program files (x86)/microchip/xc32/v1.21/bin/../lib/gcc/pic32mx/4.5.2/../../../../pic32mx/lib/size\libpic32.a(general-exception.o)
                              c:/program files (x86)/microchip/xc32/v1.21/bin/../lib/gcc/pic32mx/4.5.2/../../../../pic32mx/lib/size/crt0.o (_general_exception_context)
c:/program files (x86)/microchip/xc32/v1.21/bin/../lib/gcc/pic32mx/4.5.2/../../../../pic32mx/lib/size\libpic32.a(vector1.o)
                              c:/program files (x86)/microchip/xc32/v1.21/bin/../lib/gcc/pic32mx/4.5.2/../../../../pic32mx/lib/./proc/32MX795F512L\default_isr_vectors.o (__vector_dispatch_1)
c:/program files (x86)/microchip/xc32/v1.21/bin/../lib/gcc/pic32mx/4.5.2/../../../../pic32mx/lib/size\libpic32.a(vector2.o)
                              c:/program files (x86)/microchip/xc32/v1.21/bin/../lib/gcc/pic32mx/4.5.2/../../../../pic32mx/lib/./proc/32MX795F512L\default_isr_vectors.o (__vector_dispatch_2)
c:/program files (x86)/microchip/xc32/v1.21/bin/../lib/gcc/pic32mx/4.5.2/../../../../pic32mx/lib/size\libpic32.a(vector3.o)
                              c:/program files (x86)/microchip/xc32/v1.21/bin/../lib/gcc/pic32mx/4.5.2/../../../../pic32mx/lib/./proc/32MX795F512L\default_isr_vectors.o (__vector_dispatch_3)
c:/program files (x86)/microchip/xc32/v1.21/bin/../lib/gcc/pic32mx/4.5.2/../../../../pic32mx/lib/size\libpic32.a(vector4.o)
                              c:/program files (x86)/microchip/xc32/v1.21/bin/../lib/gcc/pic32mx/4.5.2/../../../../pic32mx/lib/./proc/32MX795F512L\default_isr_vectors.o (__vector_dispatch_4)
c:/program files (x86)/microchip/xc32/v1.21/bin/../lib/gcc/pic32mx/4.5.2/../../../../pic32mx/lib/size\libpic32.a(vector5.o)
                              c:/program files (x86)/microchip/xc32/v1.21/bin/../lib/gcc/pic32mx/4.5.2/../../../../pic32mx/lib/./proc/32MX795F512L\default_isr_vectors.o (__vector_dispatch_5)
c:/program files (x86)/microchip/xc32/v1.21/bin/../lib/gcc/pic32mx/4.5.2/../../../../pic32mx/lib/size\libpic32.a(vector6.o)
                              c:/program files (x86)/microchip/xc32/v1.21/bin/../lib/gcc/pic32mx/4.5.2/../../../../pic32mx/lib/./proc/32MX795F512L\default_isr_vectors.o (__vector_dispatch_6)
c:/program files (x86)/microchip/xc32/v1.21/bin/../lib/gcc/pic32mx/4.5.2/../../../../pic32mx/lib/size\libpic32.a(vector8.o)
                              c:/program files (x86)/microchip/xc32/v1.21/bin/../lib/gcc/pic32mx/4.5.2/../../../../pic32mx/lib/./proc/32MX795F512L\default_isr_vectors.o (__vector_dispatch_8)
c:/program files (x86)/microchip/xc32/v1.21/bin/../lib/gcc/pic32mx/4.5.2/../../../../pic32mx/lib/size\libpic32.a(vector9.o)
                              c:/program files (x86)/microchip/xc32/v1.21/bin/../lib/gcc/pic32mx/4.5.2/../../../../pic32mx/lib/./proc/32MX795F512L\default_isr_vectors.o (__vector_dispatch_9)
c:/program files (x86)/microchip/xc32/v1.21/bin/../lib/gcc/pic32mx/4.5.2/../../../../pic32mx/lib/size\libpic32.a(vector10.o)
                              c:/program files (x86)/microchip/xc32/v1.21/bin/../lib/gcc/pic32mx/4.5.2/../../../../pic32mx/lib/./proc/32MX795F512L\default_isr_vectors.o (__vector_dispatch_10)
c:/program files (x86)/microchip/xc32/v1.21/bin/../lib/gcc/pic32mx/4.5.2/../../../../pic32mx/lib/size\libpic32.a(vector11.o)
                              c:/program files (x86)/microchip/xc32/v1.21/bin/../lib/gcc/pic32mx/4.5.2/../../../../pic32mx/lib/./proc/32MX795F512L\default_isr_vectors.o (__vector_dispatch_11)
c:/program files (x86)/microchip/xc32/v1.21/bin/../lib/gcc/pic32mx/4.5.2/../../../../pic32mx/lib/size\libpic32.a(vector12.o)
                              c:/program files (x86)/microchip/xc32/v1.21/bin/../lib/gcc/pic32mx/4.5.2/../../../../pic32mx/lib/./proc/32MX795F512L\default_isr_vectors.o (__vector_dispatch_12)
c:/program files (x86)/microchip/xc32/v1.21/bin/../lib/gcc/pic32mx/4.5.2/../../../../pic32mx/lib/size\libpic32.a(vector13.o)
                              c:/program files (x86)/microchip/xc32/v1.21/bin/../lib/gcc/pic32mx/4.5.2/../../../../pic32mx/lib/./proc/32MX795F512L\default_isr_vectors.o (__vector_dispatch_13)
c:/program files (x86)/microchip/xc32/v1.21/bin/../lib/gcc/pic32mx/4.5.2/../../../../pic32mx/lib/size\libpic32.a(vector14.o)
                              c:/program files (x86)/microchip/xc32/v1.21/bin/../lib/gcc/pic32mx/4.5.2/../../../../pic32mx/lib/./proc/32MX795F512L\default_isr_vectors.o (__vector_dispatch_14)
c:/program files (x86)/microchip/xc32/v1.21/bin/../lib/gcc/pic32mx/4.5.2/../../../../pic32mx/lib/size\libpic32.a(vector16.o)
                              c:/program files (x86)/microchip/xc32/v1.21/bin/../lib/gcc/pic32mx/4.5.2/../../../../pic32mx/lib/./proc/32MX795F512L\default_isr_vectors.o (__vector_dispatch_16)
c:/program files (x86)/microchip/xc32/v1.21/bin/../lib/gcc/pic32mx/4.5.2/../../../../pic32mx/lib/size\libpic32.a(vector17.o)
                              c:/program files (x86)/microchip/xc32/v1.21/bin/../lib/gcc/pic32mx/4.5.2/../../../../pic32mx/lib/./proc/32MX795F512L\default_isr_vectors.o (__vector_dispatch_17)
c:/program files (x86)/microchip/xc32/v1.21/bin/../lib/gcc/pic32mx/4.5.2/../../../../pic32mx/lib/size\libpic32.a(vector18.o)
                              c:/program files (x86)/microchip/xc32/v1.21/bin/../lib/gcc/pic32mx/4.5.2/../../../../pic32mx/lib/./proc/32MX795F512L\default_isr_vectors.o (__vector_dispatch_18)
c:/program files (x86)/microchip/xc32/v1.21/bin/../lib/gcc/pic32mx/4.5.2/../../../../pic32mx/lib/size\libpic32.a(vector19.o)
                              c:/program files (x86)/microchip/xc32/v1.21/bin/../lib/gcc/pic32mx/4.5.2/../../../../pic32mx/lib/./proc/32MX795F512L\default_isr_vectors.o (__vector_dispatch_19)
c:/program files (x86)/microchip/xc32/v1.21/bin/../lib/gcc/pic32mx/4.5.2/../../../../pic32mx/lib/size\libpic32.a(vector20.o)
                              c:/program files (x86)/microchip/xc32/v1.21/bin/../lib/gcc/pic32mx/4.5.2/../../../../pic32mx/lib/./proc/32MX795F512L\default_isr_vectors.o (__vector_dispatch_20)
c:/program files (x86)/microchip/xc32/v1.21/bin/../lib/gcc/pic32mx/4.5.2/../../../../pic32mx/lib/size\libpic32.a(vector21.o)
                              c:/program files (x86)/microchip/xc32/v1.21/bin/../lib/gcc/pic32mx/4.5.2/../../../../pic32mx/lib/./proc/32MX795F512L\default_isr_vectors.o (__vector_dispatch_21)
c:/program files (x86)/microchip/xc32/v1.21/bin/../lib/gcc/pic32mx/4.5.2/../../../../pic32mx/lib/size\libpic32.a(vector22.o)
                              c:/program files (x86)/microchip/xc32/v1.21/bin/../lib/gcc/pic32mx/4.5.2/../../../../pic32mx/lib/./proc/32MX795F512L\default_isr_vectors.o (__vector_dispatch_22)
c:/program files (x86)/microchip/xc32/v1.21/bin/../lib/gcc/pic32mx/4.5.2/../../../../pic32mx/lib/size\libpic32.a(vector23.o)
                              c:/program files (x86)/microchip/xc32/v1.21/bin/../lib/gcc/pic32mx/4.5.2/../../../../pic32mx/lib/./proc/32MX795F512L\default_isr_vectors.o (__vector_dispatch_23)
c:/program files (x86)/microchip/xc32/v1.21/bin/../lib/gcc/pic32mx/4.5.2/../../../../pic32mx/lib/size\libpic32.a(vector24.o)
                              c:/program files (x86)/microchip/xc32/v1.21/bin/../lib/gcc/pic32mx/4.5.2/../../../../pic32mx/lib/./proc/32MX795F512L\default_isr_vectors.o (__vector_dispatch_24)
c:/program files (x86)/microchip/xc32/v1.21/bin/../lib/gcc/pic32mx/4.5.2/../../../../pic32mx/lib/size\libpic32.a(vector25.o)
                              c:/program files (x86)/microchip/xc32/v1.21/bin/../lib/gcc/pic32mx/4.5.2/../../../../pic32mx/lib/./proc/32MX795F512L\default_isr_vectors.o (__vector_dispatch_25)
c:/program files (x86)/microchip/xc32/v1.21/bin/../lib/gcc/pic32mx/4.5.2/../../../../pic32mx/lib/size\libpic32.a(vector27.o)
                              c:/program files (x86)/microchip/xc32/v1.21/bin/../lib/gcc/pic32mx/4.5.2/../../../../pic32mx/lib/./proc/32MX795F512L\default_isr_vectors.o (__vector_dispatch_27)
c:/program files (x86)/microchip/xc32/v1.21/bin/../lib/gcc/pic32mx/4.5.2/../../../../pic32mx/lib/size\libpic32.a(vector28.o)
                              c:/program files (x86)/microchip/xc32/v1.21/bin/../lib/gcc/pic32mx/4.5.2/../../../../pic32mx/lib/./proc/32MX795F512L\default_isr_vectors.o (__vector_dispatch_28)
c:/program files (x86)/microchip/xc32/v1.21/bin/../lib/gcc/pic32mx/4.5.2/../../../../pic32mx/lib/size\libpic32.a(vector29.o)
                              c:/program files (x86)/microchip/xc32/v1.21/bin/../lib/gcc/pic32mx/4.5.2/../../../../pic32mx/lib/./proc/32MX795F512L\default_isr_vectors.o (__vector_dispatch_29)
c:/program files (x86)/microchip/xc32/v1.21/bin/../lib/gcc/pic32mx/4.5.2/../../../../pic32mx/lib/size\libpic32.a(vector30.o)
                              c:/program files (x86)/microchip/xc32/v1.21/bin/../lib/gcc/pic32mx/4.5.2/../../../../pic32mx/lib/./proc/32MX795F512L\default_isr_vectors.o (__vector_dispatch_30)
c:/program files (x86)/microchip/xc32/v1.21/bin/../lib/gcc/pic32mx/4.5.2/../../../../pic32mx/lib/size\libpic32.a(vector31.o)
                              c:/program files (x86)/microchip/xc32/v1.21/bin/../lib/gcc/pic32mx/4.5.2/../../../../pic32mx/lib/./proc/32MX795F512L\default_isr_vectors.o (__vector_dispatch_31)
c:/program files (x86)/microchip/xc32/v1.21/bin/../lib/gcc/pic32mx/4.5.2/../../../../pic32mx/lib/size\libpic32.a(vector32.o)
                              c:/program files (x86)/microchip/xc32/v1.21/bin/../lib/gcc/pic32mx/4.5.2/../../../../pic32mx/lib/./proc/32MX795F512L\default_isr_vectors.o (__vector_dispatch_32)
c:/program files (x86)/microchip/xc32/v1.21/bin/../lib/gcc/pic32mx/4.5.2/../../../../pic32mx/lib/size\libpic32.a(vector33.o)
                              c:/program files (x86)/microchip/xc32/v1.21/bin/../lib/gcc/pic32mx/4.5.2/../../../../pic32mx/lib/./proc/32MX795F512L\default_isr_vectors.o (__vector_dispatch_33)
c:/program files (x86)/microchip/xc32/v1.21/bin/../lib/gcc/pic32mx/4.5.2/../../../../pic32mx/lib/size\libpic32.a(vector34.o)
                              c:/program files (x86)/microchip/xc32/v1.21/bin/../lib/gcc/pic32mx/4.5.2/../../../../pic32mx/lib/./proc/32MX795F512L\default_isr_vectors.o (__vector_dispatch_34)
c:/program files (x86)/microchip/xc32/v1.21/bin/../lib/gcc/pic32mx/4.5.2/../../../../pic32mx/lib/size\libpic32.a(vector35.o)
                              c:/program files (x86)/microchip/xc32/v1.21/bin/../lib/gcc/pic32mx/4.5.2/../../../../pic32mx/lib/./proc/32MX795F512L\default_isr_vectors.o (__vector_dispatch_35)
c:/program files (x86)/microchip/xc32/v1.21/bin/../lib/gcc/pic32mx/4.5.2/../../../../pic32mx/lib/size\libpic32.a(vector36.o)
                              c:/program files (x86)/microchip/xc32/v1.21/bin/../lib/gcc/pic32mx/4.5.2/../../../../pic32mx/lib/./proc/32MX795F512L\default_isr_vectors.o (__vector_dispatch_36)
c:/program files (x86)/microchip/xc32/v1.21/bin/../lib/gcc/pic32mx/4.5.2/../../../../pic32mx/lib/size\libpic32.a(vector37.o)
                              c:/program files (x86)/microchip/xc32/v1.21/bin/../lib/gcc/pic32mx/4.5.2/../../../../pic32mx/lib/./proc/32MX795F512L\default_isr_vectors.o (__vector_dispatch_37)
c:/program files (x86)/microchip/xc32/v1.21/bin/../lib/gcc/pic32mx/4.5.2/../../../../pic32mx/lib/size\libpic32.a(vector38.o)
                              c:/program files (x86)/microchip/xc32/v1.21/bin/../lib/gcc/pic32mx/4.5.2/../../../../pic32mx/lib/./proc/32MX795F512L\default_isr_vectors.o (__vector_dispatch_38)
c:/program files (x86)/microchip/xc32/v1.21/bin/../lib/gcc/pic32mx/4.5.2/../../../../pic32mx/lib/size\libpic32.a(vector39.o)
                              c:/program files (x86)/microchip/xc32/v1.21/bin/../lib/gcc/pic32mx/4.5.2/../../../../pic32mx/lib/./proc/32MX795F512L\default_isr_vectors.o (__vector_dispatch_39)
c:/program files (x86)/microchip/xc32/v1.21/bin/../lib/gcc/pic32mx/4.5.2/../../../../pic32mx/lib/size\libpic32.a(vector40.o)
                              c:/program files (x86)/microchip/xc32/v1.21/bin/../lib/gcc/pic32mx/4.5.2/../../../../pic32mx/lib/./proc/32MX795F512L\default_isr_vectors.o (__vector_dispatch_40)
c:/program files (x86)/microchip/xc32/v1.21/bin/../lib/gcc/pic32mx/4.5.2/../../../../pic32mx/lib/size\libpic32.a(vector41.o)
                              c:/program files (x86)/microchip/xc32/v1.21/bin/../lib/gcc/pic32mx/4.5.2/../../../../pic32mx/lib/./proc/32MX795F512L\default_isr_vectors.o (__vector_dispatch_41)
c:/program files (x86)/microchip/xc32/v1.21/bin/../lib/gcc/pic32mx/4.5.2/../../../../pic32mx/lib/size\libpic32.a(vector42.o)
                              c:/program files (x86)/microchip/xc32/v1.21/bin/../lib/gcc/pic32mx/4.5.2/../../../../pic32mx/lib/./proc/32MX795F512L\default_isr_vectors.o (__vector_dispatch_42)
c:/program files (x86)/microchip/xc32/v1.21/bin/../lib/gcc/pic32mx/4.5.2/../../../../pic32mx/lib/size\libpic32.a(vector43.o)
                              c:/program files (x86)/microchip/xc32/v1.21/bin/../lib/gcc/pic32mx/4.5.2/../../../../pic32mx/lib/./proc/32MX795F512L\default_isr_vectors.o (__vector_dispatch_43)
c:/program files (x86)/microchip/xc32/v1.21/bin/../lib/gcc/pic32mx/4.5.2/../../../../pic32mx/lib/size\libpic32.a(vector44.o)
                              c:/program files (x86)/microchip/xc32/v1.21/bin/../lib/gcc/pic32mx/4.5.2/../../../../pic32mx/lib/./proc/32MX795F512L\default_isr_vectors.o (__vector_dispatch_44)
c:/program files (x86)/microchip/xc32/v1.21/bin/../lib/gcc/pic32mx/4.5.2/../../../../pic32mx/lib/size\libpic32.a(vector45.o)
                              c:/program files (x86)/microchip/xc32/v1.21/bin/../lib/gcc/pic32mx/4.5.2/../../../../pic32mx/lib/./proc/32MX795F512L\default_isr_vectors.o (__vector_dispatch_45)
c:/program files (x86)/microchip/xc32/v1.21/bin/../lib/gcc/pic32mx/4.5.2/../../../../pic32mx/lib/size\libpic32.a(vector46.o)
                              c:/program files (x86)/microchip/xc32/v1.21/bin/../lib/gcc/pic32mx/4.5.2/../../../../pic32mx/lib/./proc/32MX795F512L\default_isr_vectors.o (__vector_dispatch_46)
c:/program files (x86)/microchip/xc32/v1.21/bin/../lib/gcc/pic32mx/4.5.2/../../../../pic32mx/lib/size\libpic32.a(vector47.o)
                              c:/program files (x86)/microchip/xc32/v1.21/bin/../lib/gcc/pic32mx/4.5.2/../../../../pic32mx/lib/./proc/32MX795F512L\default_isr_vectors.o (__vector_dispatch_47)
c:/program files (x86)/microchip/xc32/v1.21/bin/../lib/gcc/pic32mx/4.5.2/../../../../pic32mx/lib/size\libpic32.a(vector48.o)
                              c:/program files (x86)/microchip/xc32/v1.21/bin/../lib/gcc/pic32mx/4.5.2/../../../../pic32mx/lib/./proc/32MX795F512L\default_isr_vectors.o (__vector_dispatch_48)
c:/program files (x86)/microchip/xc32/v1.21/bin/../lib/gcc/pic32mx/4.5.2/../../../../pic32mx/lib/size\libpic32.a(vector49.o)
                              c:/program files (x86)/microchip/xc32/v1.21/bin/../lib/gcc/pic32mx/4.5.2/../../../../pic32mx/lib/./proc/32MX795F512L\default_isr_vectors.o (__vector_dispatch_49)
c:/program files (x86)/microchip/xc32/v1.21/bin/../lib/gcc/pic32mx/4.5.2/../../../../pic32mx/lib/size\libpic32.a(vector50.o)
                              c:/program files (x86)/microchip/xc32/v1.21/bin/../lib/gcc/pic32mx/4.5.2/../../../../pic32mx/lib/./proc/32MX795F512L\default_isr_vectors.o (__vector_dispatch_50)
c:/program files (x86)/microchip/xc32/v1.21/bin/../lib/gcc/pic32mx/4.5.2/../../../../pic32mx/lib/size\libpic32.a(vector51.o)
                              c:/program files (x86)/microchip/xc32/v1.21/bin/../lib/gcc/pic32mx/4.5.2/../../../../pic32mx/lib/./proc/32MX795F512L\default_isr_vectors.o (__vector_dispatch_51)
c:/program files (x86)/microchip/xc32/v1.21/bin/../lib/gcc/pic32mx/4.5.2/../../../../pic32mx/lib/size\libpic32.a(vector52.o)
                              c:/program files (x86)/microchip/xc32/v1.21/bin/../lib/gcc/pic32mx/4.5.2/../../../../pic32mx/lib/./proc/32MX795F512L\default_isr_vectors.o (__vector_dispatch_52)
c:/program files (x86)/microchip/xc32/v1.21/bin/../lib/gcc/pic32mx/4.5.2/../../../../pic32mx/lib/size\libpic32.a(vector53.o)
                              c:/program files (x86)/microchip/xc32/v1.21/bin/../lib/gcc/pic32mx/4.5.2/../../../../pic32mx/lib/./proc/32MX795F512L\default_isr_vectors.o (__vector_dispatch_53)
c:/program files (x86)/microchip/xc32/v1.21/bin/../lib/gcc/pic32mx/4.5.2/../../../../pic32mx/lib/size\libpic32.a(vector54.o)
                              c:/program files (x86)/microchip/xc32/v1.21/bin/../lib/gcc/pic32mx/4.5.2/../../../../pic32mx/lib/./proc/32MX795F512L\default_isr_vectors.o (__vector_dispatch_54)
c:/program files (x86)/microchip/xc32/v1.21/bin/../lib/gcc/pic32mx/4.5.2/../../../../pic32mx/lib/size\libpic32.a(vector55.o)
                              c:/program files (x86)/microchip/xc32/v1.21/bin/../lib/gcc/pic32mx/4.5.2/../../../../pic32mx/lib/./proc/32MX795F512L\default_isr_vectors.o (__vector_dispatch_55)
c:/program files (x86)/microchip/xc32/v1.21/bin/../lib/gcc/pic32mx/4.5.2/../../../../pic32mx/lib/size\libpic32.a(vector56.o)
                              c:/program files (x86)/microchip/xc32/v1.21/bin/../lib/gcc/pic32mx/4.5.2/../../../../pic32mx/lib/./proc/32MX795F512L\default_isr_vectors.o (__vector_dispatch_56)
c:/program files (x86)/microchip/xc32/v1.21/bin/../lib/gcc/pic32mx/4.5.2/../../../../pic32mx/lib/size\libpic32.a(vector57.o)
                              c:/program files (x86)/microchip/xc32/v1.21/bin/../lib/gcc/pic32mx/4.5.2/../../../../pic32mx/lib/./proc/32MX795F512L\default_isr_vectors.o (__vector_dispatch_57)
c:/program files (x86)/microchip/xc32/v1.21/bin/../lib/gcc/pic32mx/4.5.2/../../../../pic32mx/lib/size\libpic32.a(vector58.o)
                              c:/program files (x86)/microchip/xc32/v1.21/bin/../lib/gcc/pic32mx/4.5.2/../../../../pic32mx/lib/./proc/32MX795F512L\default_isr_vectors.o (__vector_dispatch_58)
c:/program files (x86)/microchip/xc32/v1.21/bin/../lib/gcc/pic32mx/4.5.2/../../../../pic32mx/lib/size\libpic32.a(vector59.o)
                              c:/program files (x86)/microchip/xc32/v1.21/bin/../lib/gcc/pic32mx/4.5.2/../../../../pic32mx/lib/./proc/32MX795F512L\default_isr_vectors.o (__vector_dispatch_59)
c:/program files (x86)/microchip/xc32/v1.21/bin/../lib/gcc/pic32mx/4.5.2/../../../../pic32mx/lib/size\libpic32.a(vector60.o)
                              c:/program files (x86)/microchip/xc32/v1.21/bin/../lib/gcc/pic32mx/4.5.2/../../../../pic32mx/lib/./proc/32MX795F512L\default_isr_vectors.o (__vector_dispatch_60)
c:/program files (x86)/microchip/xc32/v1.21/bin/../lib/gcc/pic32mx/4.5.2/../../../../pic32mx/lib/size\libpic32.a(vector61.o)
                              c:/program files (x86)/microchip/xc32/v1.21/bin/../lib/gcc/pic32mx/4.5.2/../../../../pic32mx/lib/./proc/32MX795F512L\default_isr_vectors.o (__vector_dispatch_61)
c:/program files (x86)/microchip/xc32/v1.21/bin/../lib/gcc/pic32mx/4.5.2/../../../../pic32mx/lib/size\libpic32.a(vector62.o)
                              c:/program files (x86)/microchip/xc32/v1.21/bin/../lib/gcc/pic32mx/4.5.2/../../../../pic32mx/lib/./proc/32MX795F512L\default_isr_vectors.o (__vector_dispatch_62)
c:/program files (x86)/microchip/xc32/v1.21/bin/../lib/gcc/pic32mx/4.5.2/../../../../pic32mx/lib/size\libpic32.a(vector63.o)
                              c:/program files (x86)/microchip/xc32/v1.21/bin/../lib/gcc/pic32mx/4.5.2/../../../../pic32mx/lib/./proc/32MX795F512L\default_isr_vectors.o (__vector_dispatch_63)
c:/program files (x86)/microchip/xc32/v1.21/bin/../lib/gcc/pic32mx/4.5.2/../../../../pic32mx/lib/size\libpic32.a(defaultinterrupt.o)
                              c:/program files (x86)/microchip/xc32/v1.21/bin/../lib/gcc/pic32mx/4.5.2/../../../../pic32mx/lib/size\libpic32.a(vector1.o) (_DefaultInterrupt)
c:/program files (x86)/microchip/xc32/v1.21/bin/../lib/gcc/pic32mx/4.5.2/../../../../pic32mx/lib/size\libc.a(atoi.o)
                              build/default/production/_ext/1472/tcp6_demo_app.o (atoi)
c:/program files (x86)/microchip/xc32/v1.21/bin/../lib/gcc/pic32mx/4.5.2/../../../../pic32mx/lib/size\libc.a(atol.o)
                              build/default/production/_ext/427700826/http2.o (atol)
c:/program files (x86)/microchip/xc32/v1.21/bin/../lib/gcc/pic32mx/4.5.2/../../../../pic32mx/lib/size\libc.a(ctype.o)
                              build/default/production/_ext/427700826/tcpip_helpers.o (_ctype)
c:/program files (x86)/microchip/xc32/v1.21/bin/../lib/gcc/pic32mx/4.5.2/../../../../pic32mx/lib/size\libc.a(malloc.o)
                              build/default/production/_ext/365611741/system_services.o (malloc)
c:/program files (x86)/microchip/xc32/v1.21/bin/../lib/gcc/pic32mx/4.5.2/../../../../pic32mx/lib/size\libc.a(rand.o)
                              build/default/production/_ext/427700826/dhcp.o (rand)
c:/program files (x86)/microchip/xc32/v1.21/bin/../lib/gcc/pic32mx/4.5.2/../../../../pic32mx/lib/size\libc.a(strcat.o)
                              build/default/production/_ext/1472/ping_demo.o (strcat)
c:/program files (x86)/microchip/xc32/v1.21/bin/../lib/gcc/pic32mx/4.5.2/../../../../pic32mx/lib/size\libc.a(strchr.o)
                              build/default/production/_ext/97638081/sys_fs.o (strchr)
c:/program files (x86)/microchip/xc32/v1.21/bin/../lib/gcc/pic32mx/4.5.2/../../../../pic32mx/lib/size\libc.a(strncat.o)
                              build/default/production/_ext/1472/tcp6_demo_app.o (strncat)
c:/program files (x86)/microchip/xc32/v1.21/bin/../lib/gcc/pic32mx/4.5.2/../../../../pic32mx/lib/size\libc.a(strncmp.o)
                              build/default/production/_ext/97638081/sys_fs.o (strncmp)
c:/program files (x86)/microchip/xc32/v1.21/bin/../lib/gcc/pic32mx/4.5.2/../../../../pic32mx/lib/size\libc.a(strncpy.o)
                              build/default/production/_ext/101875047/helpers.o (strncpy)
c:/program files (x86)/microchip/xc32/v1.21/bin/../lib/gcc/pic32mx/4.5.2/../../../../pic32mx/lib/size\libc.a(strrchr.o)
                              build/default/production/_ext/97638081/sys_fs.o (strrchr)
c:/program files (x86)/microchip/xc32/v1.21/bin/../lib/gcc/pic32mx/4.5.2/../../../../pic32mx/lib/size\libc.a(strstr.o)
                              build/default/production/_ext/97638081/sys_fs.o (strstr)
c:/program files (x86)/microchip/xc32/v1.21/bin/../lib/gcc/pic32mx/4.5.2/../../../../pic32mx/lib/size\libc.a(strtol.o)
                              build/default/production/_ext/1472/tcp6_demo_app.o (strtol)
c:/program files (x86)/microchip/xc32/v1.21/bin/../lib/gcc/pic32mx/4.5.2/../../../../pic32mx/lib/size\libc.a(snprintf_cdnopsuxX.eo)
                              build/default/production/_ext/365611741/system_debug.o (_snprintf_cdnopsuxX)
c:/program files (x86)/microchip/xc32/v1.21/bin/../lib/gcc/pic32mx/4.5.2/../../../../pic32mx/lib/size\libc.a(sprintf_cdnopsuxX.eo)
                              build/default/production/_ext/1472/tcp6_demo_app.o (_sprintf_cdnopsuxX)
c:/program files (x86)/microchip/xc32/v1.21/bin/../lib/gcc/pic32mx/4.5.2/../../../../pic32mx/lib/size\libc.a(sprintf_cdnopuxX.eo)
                              build/default/production/_ext/427700826/tcpip_helpers.o (_sprintf_cdnopuxX)
c:/program files (x86)/microchip/xc32/v1.21/bin/../lib/gcc/pic32mx/4.5.2/../../../../pic32mx/lib/size\libc.a(vsnprintf_cdnopsuxX.eo)
                              c:/program files (x86)/microchip/xc32/v1.21/bin/../lib/gcc/pic32mx/4.5.2/../../../../pic32mx/lib/size\libc.a(snprintf_cdnopsuxX.eo) (_vsnprintf_cdnopsuxX)
c:/program files (x86)/microchip/xc32/v1.21/bin/../lib/gcc/pic32mx/4.5.2/../../../../pic32mx/lib/size\libc.a(vsnprintf.o)
                              build/default/production/_ext/365611741/system_debug.o (vsnprintf)
c:/program files (x86)/microchip/xc32/v1.21/bin/../lib/gcc/pic32mx/4.5.2/../../../../pic32mx/lib/size\libc.a(ctypef.o)
                              c:/program files (x86)/microchip/xc32/v1.21/bin/../lib/gcc/pic32mx/4.5.2/../../../../pic32mx/lib/size\libc.a(strtol.o) (toupper)
c:/program files (x86)/microchip/xc32/v1.21/bin/../lib/gcc/pic32mx/4.5.2/../../../../pic32mx/lib/size\libc.a(doprnt_cdnopsuxX.eo)
                              c:/program files (x86)/microchip/xc32/v1.21/bin/../lib/gcc/pic32mx/4.5.2/../../../../pic32mx/lib/size\libc.a(sprintf_cdnopsuxX.eo) (_vfprintf_cdnopsuxX)
c:/program files (x86)/microchip/xc32/v1.21/bin/../lib/gcc/pic32mx/4.5.2/../../../../pic32mx/lib/size\libc.a(doprnt_cdnopuxX.eo)
                              c:/program files (x86)/microchip/xc32/v1.21/bin/../lib/gcc/pic32mx/4.5.2/../../../../pic32mx/lib/size\libc.a(sprintf_cdnopuxX.eo) (_vfprintf_cdnopuxX)
c:/program files (x86)/microchip/xc32/v1.21/bin/../lib/gcc/pic32mx/4.5.2/../../../../pic32mx/lib/size\libc.a(doprnt.o)
                              c:/program files (x86)/microchip/xc32/v1.21/bin/../lib/gcc/pic32mx/4.5.2/../../../../pic32mx/lib/size\libc.a(vsnprintf.o) (vfprintf)
c:/program files (x86)/microchip/xc32/v1.21/bin/../lib/gcc/pic32mx/4.5.2/../../../../pic32mx/lib/size\libc.a(_fputc_simple.o)
                              c:/program files (x86)/microchip/xc32/v1.21/bin/../lib/gcc/pic32mx/4.5.2/../../../../pic32mx/lib/size\libc.a(doprnt_cdnopsuxX.eo) (fputc)
c:/program files (x86)/microchip/xc32/v1.21/bin/../lib/gcc/pic32mx/4.5.2/../../../../pic32mx/lib/size\libc.a(powersf.o)
                              c:/program files (x86)/microchip/xc32/v1.21/bin/../lib/gcc/pic32mx/4.5.2/../../../../pic32mx/lib/size\libc.a(doprnt.o) (_powers_f)
c:/program files (x86)/microchip/xc32/v1.21/bin/../lib/gcc/pic32mx/4.5.2/../../../../pic32mx/lib/size\libc.a(_iob.o)
                              c:/program files (x86)/microchip/xc32/v1.21/bin/../lib/gcc/pic32mx/4.5.2/../../../../pic32mx/lib/size\libc.a(_fputc_simple.o) (_outdone)
c:/program files (x86)/microchip/xc32/v1.21/bin/../lib/gcc/pic32mx/4.5.2/../../../../pic32mx/lib/size\libc.a(_flsbuf_simple.o)
                              c:/program files (x86)/microchip/xc32/v1.21/bin/../lib/gcc/pic32mx/4.5.2/../../../../pic32mx/lib/size\libc.a(_fputc_simple.o) (_flsbuf)
c:/program files (x86)/microchip/xc32/v1.21/bin/../lib/gcc/pic32mx/4.5.2/../../../../pic32mx/lib/size\libpic32.a(sbrk.o)
                              c:/program files (x86)/microchip/xc32/v1.21/bin/../lib/gcc/pic32mx/4.5.2/../../../../pic32mx/lib/size\libc.a(malloc.o) (sbrk)
c:/program files (x86)/microchip/xc32/v1.21/bin/../lib/gcc/pic32mx/4.5.2/../../../../pic32mx/lib/size\libpic32.a(write.o)
                              c:/program files (x86)/microchip/xc32/v1.21/bin/../lib/gcc/pic32mx/4.5.2/../../../../pic32mx/lib/size\libc.a(_fputc_simple.o) (write)
c:/program files (x86)/microchip/xc32/v1.21/bin/../lib/gcc/pic32mx/4.5.2/../../../../pic32mx/lib/size\libpic32.a(_mon_putc.o)
                              c:/program files (x86)/microchip/xc32/v1.21/bin/../lib/gcc/pic32mx/4.5.2/../../../../pic32mx/lib/size\libpic32.a(write.o) (_mon_putc)
c:/program files (x86)/microchip/xc32/v1.21/bin/../lib/gcc/pic32mx/4.5.2/../../../../pic32mx/lib/size\libpic32.a(xc32_uart.o)
                              c:/program files (x86)/microchip/xc32/v1.21/bin/../lib/gcc/pic32mx/4.5.2/../../../../pic32mx/lib/size\libpic32.a(_mon_putc.o) (__XC_UART)
c:/program files (x86)/microchip/xc32/v1.21/bin/../lib/gcc/pic32mx/4.5.2/../../../../pic32mx/lib/size\libm.a(fpmod32.o)
                              c:/program files (x86)/microchip/xc32/v1.21/bin/../lib/gcc/pic32mx/4.5.2/../../../../pic32mx/lib/size\libc.a(doprnt.o) (frexpf)
c:/program files (x86)/microchip/xc32/v1.21/bin/../lib/gcc/pic32mx/4.5.2/../../../../pic32mx/lib/size\libm.a(fp32.o)
                              c:/program files (x86)/microchip/xc32/v1.21/bin/../lib/gcc/pic32mx/4.5.2/../../../../pic32mx/lib/size\libc.a(doprnt.o) (fpsub)
c:/program files (x86)/microchip/xc32/v1.21/bin/../lib/gcc/pic32mx/4.5.2/../../../../pic32mx/lib/size\libe.a(_floatdisf.o)
                              c:/program files (x86)/microchip/xc32/v1.21/bin/../lib/gcc/pic32mx/4.5.2/../../../../pic32mx/lib/size\libc.a(doprnt.o) (__floatdisf)
c:/program files (x86)/microchip/xc32/v1.21/bin/../lib/gcc/pic32mx/4.5.2/size\libgcc.a(_lshrdi3.o)
                              c:/program files (x86)/microchip/xc32/v1.21/bin/../lib/gcc/pic32mx/4.5.2/../../../../pic32mx/lib/size\libc.a(doprnt_cdnopsuxX.eo) (__lshrdi3)
c:/program files (x86)/microchip/xc32/v1.21/bin/../lib/gcc/pic32mx/4.5.2/size\libgcc.a(_floatundisf.o)
                              c:/program files (x86)/microchip/xc32/v1.21/bin/../lib/gcc/pic32mx/4.5.2/../../../../pic32mx/lib/size\libc.a(doprnt.o) (__floatundisf)
c:/program files (x86)/microchip/xc32/v1.21/bin/../lib/gcc/pic32mx/4.5.2/size\libgcc.a(_umoddi3.o)
                              c:/program files (x86)/microchip/xc32/v1.21/bin/../lib/gcc/pic32mx/4.5.2/../../../../pic32mx/lib/size\libc.a(doprnt_cdnopsuxX.eo) (__umoddi3)
c:/program files (x86)/microchip/xc32/v1.21/bin/../lib/gcc/pic32mx/4.5.2/size\libgcc.a(floatunsisf.o)
                              c:/program files (x86)/microchip/xc32/v1.21/bin/../lib/gcc/pic32mx/4.5.2/../../../../pic32mx/lib/size\libc.a(doprnt.o) (__floatunsisf)

Allocating common symbols
Common symbol       size              file

myb64               0x80              build/default/production/_ext/1472/tcp6_demo_app.o
mySocketInfo        0x28              build/default/production/_ext/1472/tcp6_demo_app.o
pNetIf              0x4               build/default/production/_ext/1472/ping_demo.o
httpTransaction     0x4b0             build/default/production/_ext/1472/tcp6_demo_app.o
pingCount           0x1               build/default/production/_ext/1472/ping_demo.o
myNetHandle         0x4               build/default/production/_ext/1472/tcp6_demo_app.o
mac_addr_ptr        0x4               build/default/production/_ext/1472/tcp6_demo_app.o
dnsRes              0x4               build/default/production/_ext/1472/tcp6_demo_app.o
HTTPReplyDelay      0x4               build/default/production/_ext/1472/tcp6_demo_app.o
targetAddressIPv4   0x4               build/default/production/_ext/1472/ping_demo.o
TCPInBuffer         0x1000            build/default/production/_ext/1472/tcp6_demo_app.o
TCPInBufPtr         0x4               build/default/production/_ext/1472/tcp6_demo_app.o
mysrc               0x80              build/default/production/_ext/1472/tcp6_demo_app.o
pingTimer           0x4               build/default/production/_ext/1472/ping_demo.o
myResourceState     0x64              build/default/production/_ext/1472/tcp6_demo_app.o
serverIP            0x4               build/default/production/_ext/1472/tcp6_demo_app.o
i                   0x4               build/default/production/_ext/1472/tcp6_demo_app.o
mac_addr            0x6               build/default/production/_ext/1472/tcp6_demo_app.o
temp                0x20              build/default/production/_ext/1472/tcp6_demo_app.o
firstHopAddress     0x4               build/default/production/_ext/1472/ping_demo.o
lastBlock           0x40              build/default/production/_ext/101875047/hashes.o
clientTimer         0x4               build/default/production/_ext/1472/tcp6_demo_app.o
TCPReadByte         0x1               build/default/production/_ext/1472/tcp6_demo_app.o
remoteNode          0xa               build/default/production/_ext/427700826/tcpip_manager.o
targetHostName      0x4               build/default/production/_ext/1472/ping_demo.o
mac_addr_string     0x10              build/default/production/_ext/1472/tcp6_demo_app.o
j                   0x4               build/default/production/_ext/1472/tcp6_demo_app.o
TCPInBufferIndex    0x4               build/default/production/_ext/1472/tcp6_demo_app.o
targetMACAddr       0x6               build/default/production/_ext/1472/ping_demo.o
toggleLed           0x4               build/default/production/_ext/1472/tcp6_demo_app.o
OutString           0x200             build/default/production/_ext/1472/tcp6_demo_app.o
HTTPReplyLineCnt    0x4               build/default/production/_ext/1472/tcp6_demo_app.o
TCPIsPutReadyCnt    0x2               build/default/production/_ext/1472/tcp6_demo_app.o
TCPOutBuffer        0x200             build/default/production/_ext/1472/tcp6_demo_app.o
serverPort          0x2               build/default/production/_ext/1472/tcp6_demo_app.o
LCDText             0x21              build/default/production/_ext/792872985/lcd.o

Microchip PIC32 Memory-Usage Report

kseg0 Program-Memory Usage
section                    address  length [bytes]      (dec)  Description
-------                 ----------  -------------------------  -----------
.text.HTTPProcess       0x9d000020         0x17c4        6084   
.text._TcpHandleSeg     0x9d0017e4         0x1778        6008   
.text.vfprintf          0x9d002f5c         0x15a8        5544   
.text.DNSClientTask     0x9d004504         0x1144        4420   
.text.tcp6_demo_app_tas 0x9d005648          0xef4        3828   
.text.DHCPTask          0x9d00653c          0xa74        2676   
.text._TcpSend          0x9d006fb0          0xa40        2624   
.text.TCPAdjustFIFOSize 0x9d0079f0          0x974        2420   
.rodata                 0x9d008364          0x8f4        2292  Read-only const 
.text                   0x9d008c58          0x8ec        2284  App's exec code 
.text._vfprintf_cdnopsu 0x9d009544          0x8b8        2232   
.text.TCPTick           0x9d009dfc          0x890        2192   
.rodata                 0x9d00a68c          0x7d4        2004  Read-only const 
.text._DHCPReceive      0x9d00ae60          0x748        1864   
.text.NBNSTask          0x9d00b5a8          0x73c        1852   
.text.HTTPPrint         0x9d00bce4          0x6ac        1708   
.text.HTTPPostConfig    0x9d00c390          0x694        1684   
.text._DHCPSend         0x9d00ca24          0x5c8        1480   
.text.TCPFindArray      0x9d00cfec          0x578        1400   
.text.SHA1HashBlock     0x9d00d564          0x4fc        1276   
.text.SYS_Initialize    0x9d00da60          0x4f0        1264   
.text.TCPIP_ANNOUNCE_Se 0x9d00df50          0x490        1168   
.text._TCPIP_HEAP_Free  0x9d00e3e0          0x490        1168   
.text.TCPIP_STACK_Init  0x9d00e870          0x464        1124   
.text                   0x9d00ecd4          0x8a0        2208  App's exec code 
.rodata                 0x9d00f574          0x43c        1084  Read-only const 
.text.CommandHelp       0x9d00f9b0          0x428        1064   
.text.TCPOpen           0x9d00fdd8          0x420        1056   
.text.HTTPExecuteGet    0x9d0101f8          0x414        1044   
.text.HTTPMPFSUpload    0x9d01060c          0x410        1040   
.dinit                  0x9d010a1c          0x408        1032   
.text.ARPInitialize     0x9d010e24          0x3f4        1012   
.text._TcpFindMatchingS 0x9d011218          0x3e8        1000   
.text                   0x9d011600          0x3dc         988  App's exec code 
.text.MPFSSeek          0x9d0119dc          0x3ac         940   
.text.ENCX24J600_MACIni 0x9d011d88          0x3a0         928   
.text.FindMatchingSocke 0x9d012128          0x39c         924   
.text.TCPIP_Helper_Base 0x9d0124c4          0x394         916   
.rodata                 0x9d012858          0x38c         908  Read-only const 
.text._SYS_COMMAND_TASK 0x9d012be4          0x354         852   
.text.HTTPPostMD5       0x9d012f38          0x340         832   
.text.UDPOpen           0x9d013278          0x330         816   
.text.TCPIP_STACK_Bring 0x9d0135a8          0x32c         812   
.text.TCPIP_HELPER_Stri 0x9d0138d4          0x31c         796   
.text.HTTPInit          0x9d013bf0          0x318         792   
.text.ARPTask           0x9d013f08          0x310         784   
.text.TCPIP_IPV4_PutArr 0x9d014218          0x310         784   
.text.MPFSOpen          0x9d014528          0x30c         780   
.text.UDPInit           0x9d014834          0x300         768   
.text.tcp6_demo_app_ini 0x9d014b34          0x2d8         728   
.text.ProcessEscSequenc 0x9d014e0c          0x2c8         712   
.text.DoWrite           0x9d0150d4          0x2c4         708   
.text.HTTPReadTo        0x9d015398          0x2c4         708   
.text.ENCX24J600_MACGet 0x9d01565c          0x2c0         704   
.text.MD5HashBlock      0x9d01591c          0x2bc         700   
.text.TCPIP_STACK_Task  0x9d015bd8          0x2b8         696   
.text.main              0x9d015e90          0x2b8         696   
.text.ICMPProcess       0x9d016148          0x2ac         684   
.text.TCPPutArray       0x9d0163f4          0x2ac         684   
.text.MD5Calculate      0x9d0166a0          0x2a8         680   
.text.ParseCmdBuffer    0x9d016948          0x2a4         676   
.text.DRV_MEDIA_Open    0x9d016bec          0x294         660   
.rodata                 0x9d016e80          0x28c         652  Read-only const 
.text.MPFSGetArray      0x9d01710c          0x280         640   
.text.UDPProcessIPv4    0x9d01738c          0x278         632   
.text.SYS_FS_mount      0x9d017604          0x274         628   
.text.GetMaxSegSizeOpti 0x9d017878          0x274         628   
.text.XEEReadArray      0x9d017aec          0x268         616   
.text.TCPIP_IPV4_Calcul 0x9d017d54          0x268         616   
.text.HTTPSendFile      0x9d017fbc          0x264         612   
.text.TCPGetArray       0x9d018220          0x260         608   
.text.SYS_GENERATE_RAND 0x9d018480          0x25c         604   
.text.SYS_CLK_OscClockG 0x9d0186dc          0x258         600   
.text.TCPIP_IPV4_CopyTx 0x9d018934          0x250         592   
.text                   0x9d018b84          0x248         584  App's exec code 
.text.LoadDefaultConfig 0x9d018dcc          0x244         580   
.text.malloc            0x9d019010          0x240         576   
.text.LCD_UPDATE_OFFSET 0x9d019250          0x230         560   
.text.MPFSGet           0x9d019480          0x228         552   
.text.ARPEntryRemoveNet 0x9d0196a8          0x224         548   
.text.TCPIP_IPV4_GetDat 0x9d0198cc          0x224         548   
.text.__floatdisf       0x9d019af0          0x220         544   
.rodata                 0x9d019d10          0x21c         540  Read-only const 
.text.HTTPHeaderParseCo 0x9d019f2c          0x214         532   
.text.TCPInit           0x9d01a140          0x210         528   
.text.DHCPInit          0x9d01a350          0x204         516   
.text._TcpDisconnect    0x9d01a554          0x204         516   
.text.HTTPIncFile       0x9d01a758          0x200         512   
.text.UDPTask           0x9d01a958          0x200         512   
.rodata                 0x9d01ab58          0x1fc         508  Read-only const 
.text.SYS_USERIO_SetLED 0x9d01ad54          0x1f8         504   
.text.TCPIP_ANNOUNCE_Ta 0x9d01af4c          0x1f8         504   
.text.ARPProcess        0x9d01b144          0x1f0         496   
.text.TCPIP_IPV4_Flush  0x9d01b334          0x1ec         492   
.text.SYS_FS_ExtractFir 0x9d01b520          0x1e8         488   
.text.SYS_FS_initialize 0x9d01b708          0x1e8         488   
.text._TCPIP_HEAP_Mallo 0x9d01b8f0          0x1e0         480   
.rodata                 0x9d01bad0          0x1e0         480  Read-only const 
.text.StringToArgs      0x9d01bcb0          0x1dc         476   
.text.HTTPURLDecode     0x9d01be8c          0x1dc         476   
.text.TCPProcessIPv4    0x9d01c068          0x1dc         476   
.text.TCPIP_IPV4_IsTxPu 0x9d01c244          0x1d8         472   
.text.SYS_FS_chdir      0x9d01c41c          0x1d4         468   
.text.HTTPHeaderParseAu 0x9d01c5f0          0x1d4         468   
.text.UDPv4IsTxPutReady 0x9d01c7c4          0x1d0         464   
.text._TCPIsPutReady    0x9d01c994          0x1cc         460   
.text.UDPDeInit         0x9d01cb60          0x1cc         460   
.text.strtoul           0x9d01cd2c          0x1cc         460   
.text.SYS_USERIO_ReadIO 0x9d01cef8          0x1c8         456   
.text._TcpSocketSetIdle 0x9d01d0c0          0x1c8         456   
.text.ProcessTCPIPMacEv 0x9d01d288          0x1c4         452   
.text.HTTPPrint_ledSele 0x9d01d44c          0x1c4         452   
.text.TCPSetOptions     0x9d01d610          0x1b8         440   
.text.HTTPPrint_uploade 0x9d01d7c8          0x1b8         440   
.text._SystemTickIntHan 0x9d01d980          0x1b0         432   
.text.DisplayNodeMsg    0x9d01db30          0x1a0         416   
.text.HTTPPrint_led     0x9d01dcd0          0x1a0         416   
.text                   0x9d01de70          0x1a0         416  App's exec code 
.text._TcpCloseSocket   0x9d01e010          0x198         408   
.text.NBNSGetName       0x9d01e1a8          0x194         404   
.text._Sys_Ext1_Isr     0x9d01e33c          0x190         400   
.text._Sys_Ext3_Isr     0x9d01e4cc          0x190         400   
.text._Sys_CN_Isr       0x9d01e65c          0x190         400   
.text.TCPIP_HELPER_Stri 0x9d01e7ec          0x18c         396   
.text.DRV_MEDIA_Initial 0x9d01e978          0x188         392   
.text.UDPGetArray       0x9d01eb00          0x188         392   
.text.HTTPServer        0x9d01ec88          0x180         384   
.text.WriteReg          0x9d01ee08          0x180         384   
.text._OAHashFindBkt    0x9d01ef88          0x180         384   
.text.ARPIsResolved     0x9d01f108          0x178         376   
.text.TCPIP_IPV4_Alloca 0x9d01f280          0x178         376   
.text.TCPIP_HEAP_Create 0x9d01f3f8          0x178         376   
.text.HTTPPostLCD       0x9d01f570          0x178         376   
.text.SYS_FS_IsLegalDir 0x9d01f6e8          0x170         368   
.text.LCD_INIT          0x9d01f858          0x170         368   
.text._ARPProbeAddress  0x9d01f9c8          0x170         368   
.text.SpiChnOpen        0x9d01fb38          0x170         368   
.text.stricmppgm2ram    0x9d01fca8          0x16c         364   
.text.OAHashLookUpInser 0x9d01fe14          0x16c         364   
.text.UDPv4Flush        0x9d01ff80          0x16c         364   
.text                   0x9d0200ec          0x2d0         720  App's exec code 
.text.MPFSOpenID        0x9d0203bc          0x164         356   
.text.XEEIsBusy         0x9d020520          0x164         356   
.text.SYS_TICK_TimerDel 0x9d020684          0x160         352   
.text.USART_INIT        0x9d0207e4          0x160         352   
.text.DRV_SPI_TxRx      0x9d020944          0x160         352   
.text.DNSPutString      0x9d020aa4          0x160         352   
.text.ReadReg           0x9d020c04          0x160         352   
.text.TCPIP_IPV4_Transm 0x9d020d64          0x160         352   
.text.UDPBind           0x9d020ec4          0x160         352   
.text.encodeblock       0x9d021024          0x160         352   
.text.ARP_SendIfPkt     0x9d021184          0x15c         348   
.text.TCPIP_IPV4_GetHea 0x9d0212e0          0x15c         348   
.text.DRV_MEDIA_Read    0x9d02143c          0x158         344   
.text.HTTPPrint_config_ 0x9d021594          0x158         344   
.rodata                 0x9d0216ec          0x150         336  Read-only const 
.text._TCPIPStackIsLoca 0x9d02183c          0x150         336   
.text.scale             0x9d02198c          0x150         336   
.text._sbrk_init        0x9d021adc          0x14c         332   
.text._SYS_CMDIO_DELETE 0x9d021c28          0x148         328   
.text.ENCX24J600_MACCal 0x9d021d70          0x148         328   
.text.OAHashLookUp      0x9d021eb8          0x144         324   
.rodata                 0x9d021ffc          0x140         320  Read-only const 
.text.UDPSocketSetNet   0x9d02213c          0x140         320   
.text.ENCX24J600_SendSy 0x9d02227c          0x13c         316   
.text.BSP_Initialize    0x9d0223b8          0x138         312   
.text._ARPUpdateEntry   0x9d0224f0          0x138         312   
.text.TCPIP_IPV4_Queued 0x9d022628          0x138         312   
.text.UDPIsGetReady     0x9d022760          0x138         312   
.text.HTTPPrint_btn     0x9d022898          0x138         312   
.text._general_exceptio 0x9d0229d0          0x134         308   
.text.TCPIP_IPV4_Insert 0x9d022b04          0x134         308   
.text.uitoa             0x9d022c38          0x130         304   
.text.DRV_MEDIA_Write   0x9d022d68          0x130         304   
.text.UDPSetBcastIPV4Ad 0x9d022e98          0x130         304   
.text.realloc           0x9d022fc8          0x130         304   
.text.TCPIP_STACK_DeIni 0x9d0230f8          0x12c         300   
.text.DNSBeginUsage     0x9d023224          0x128         296   
.text.fputc             0x9d02334c          0x128         296   
.text.SYS_USERIO_Initia 0x9d023474          0x124         292   
.text.HTTPDeInit        0x9d023598          0x124         292   
.text._TCPSendWinIncUpd 0x9d0236bc          0x124         292   
.text.strtol            0x9d0237e0          0x124         292   
.text.TCPIP_IPV4_QueueP 0x9d023904          0x120         288   
.text.TCPOpenServer     0x9d023a24          0x120         288   
.text.UDPOpenServer     0x9d023b44          0x120         288   
.text                   0x9d023c64          0x120         288  App's exec code 
.text.fround            0x9d023d84          0x120         288   
.text.SHA1AddData       0x9d023ea4          0x11c         284   
.text.BFSReg            0x9d023fc0          0x11c         284   
.text.BFCReg            0x9d0240dc          0x11c         284   
.text.b64_encode        0x9d0241f8          0x11c         284   
.text.Execute3          0x9d024314          0x118         280   
.text.TCPIP_IPV4_Initia 0x9d02442c          0x118         280   
.text.SYS_FS_FSFromAbsP 0x9d024544          0x114         276   
.text.ENCX24J600_CalcIP 0x9d024658          0x114         276   
.text.Execute2          0x9d02476c          0x114         276   
.text.TCPIP_IPV4_PutHea 0x9d024880          0x114         276   
.text.DisplayIPValue    0x9d024994          0x114         276   
.text.MD5AddData        0x9d024aa8          0x110         272   
.text._flsbuf           0x9d024bb8          0x110         272   
.text._TcpSwapHeader    0x9d024cc8          0x10c         268   
.text.TCPIP_STACK_Bring 0x9d024dd4          0x108         264   
.text._DHCPClose        0x9d024edc          0x104         260   
.rodata                 0x9d024fe0          0x104         260  Read-only const 
.text.hexatob           0x9d0250e4          0x100         256   
.text.ToggleCRYPTEN     0x9d0251e4           0xfc         252   
.text.HTTPExecutePost   0x9d0252e0           0xfc         252   
.text.SYS_FS_IsAbsolute 0x9d0253dc           0xf8         248   
.text.ENCX24J600_MACFlu 0x9d0254d4           0xf8         248   
.text._TCPIPStackAddres 0x9d0255cc           0xf8         248   
.text.SingleListRemoveN 0x9d0256c4           0xf8         248   
.text.SYS_USERIO_Device 0x9d0257bc           0xf4         244   
.text.MPFSGetFilename   0x9d0258b0           0xf4         244   
.text.UDPSetSourceIPAdd 0x9d0259a4           0xf4         244   
.text.UDPSetDestination 0x9d025a98           0xf4         244   
.text._ARPAddCompleteEn 0x9d025b8c           0xf0         240   
.text.UDPDiscard        0x9d025c7c           0xf0         240   
.text.NBNSPutName       0x9d025d6c           0xec         236   
.text.TCPIsPutReady     0x9d025e58           0xec         236   
.text._TCPIP_HEAP_Callo 0x9d025f44           0xec         236   
.text.HTTPReadPostValue 0x9d026030           0xe8         232   
.text.DNSIsResolved     0x9d026118           0xe8         232   
.text.TCPIP_IPV4_PutUpp 0x9d026200           0xe8         232   
.text.UDPSetRxOffset    0x9d0262e8           0xe8         232   
.text.ProcessTCPIPTickE 0x9d0263d0           0xe8         232   
.rodata                 0x9d0264b8           0xe8         232  Read-only const 
.text.LCD_WRITE         0x9d0265a0           0xe4         228   
.text.ENCX24J600_MACPut 0x9d026684           0xe4         228   
.text.ReadMemoryWindow  0x9d026768           0xe4         228   
.text.ReadN             0x9d02684c           0xe4         228   
.text.WriteN            0x9d026930           0xe4         228   
.text.TCPIP_IPV4_ResetT 0x9d026a14           0xe4         228   
.text.TCPIP_IPV4_Alloca 0x9d026af8           0xe4         228   
.text.TCPDeInit         0x9d026bdc           0xe4         228   
.text.TCPIP_HEAP_Delete 0x9d026cc0           0xe4         228   
.text.SYS_TICK_TimerCre 0x9d026da4           0xe0         224   
.text._SYS_CMDIO_ADD    0x9d026e84           0xe0         224   
.text._ARPSetEntry      0x9d026f64           0xe0         224   
.text.ARPResolve        0x9d027044           0xe0         224   
.text.UDPPutArray       0x9d027124           0xe0         224   
.text._SYS_ERROR_PRINT  0x9d027204           0xdc         220   
.text.HTTPHeaderParseCo 0x9d0272e0           0xdc         220   
.text.ARPHashDeleteEntr 0x9d0273bc           0xdc         220   
.text.DHCPConnectionHan 0x9d027498           0xdc         220   
.text._TcpCleanup       0x9d027574           0xdc         220   
.text.TCPOpenClient     0x9d027650           0xdc         220   
.text.TcpAllocateEpheme 0x9d02772c           0xdc         220   
.text.UDPOpenClient     0x9d027808           0xdc         220   
.text.UdpAllocateEpheme 0x9d0278e4           0xdc         220   
.text.TCPIP_IPV4_GetPse 0x9d0279c0           0xd8         216   
.text._TCPIP_HEAP_Mallo 0x9d027a98           0xd8         216   
.text._SYS_RANDOM_INIT  0x9d027b70           0xd4         212   
.text.TCPIP_ANNOUNCE_In 0x9d027c44           0xd4         212   
.text._TcpAbort         0x9d027d18           0xd4         212   
.text.TCPClose          0x9d027dec           0xd4         212   
.text                   0x9d027ec0           0xd4         212  App's exec code 
.text.HTTPGetArg        0x9d027f94           0xd0         208   
.text._ARPDeleteResourc 0x9d028064           0xd0         208   
.text.fnv_32_hash       0x9d028134           0xd0         208   
.text._TcpSocketInitial 0x9d028204           0xd0         208   
.text.UDPSetOptions     0x9d0282d4           0xd0         208   
.text.general_exception 0x9d0283a4           0xd0         208   
.rodata                 0x9d028474            0x4           4  Read-only const 
.rodata                 0x9d028478           0xd0         208  Read-only const 
.text.DRV_MEDIA_WriteSe 0x9d028548           0xcc         204   
.text.HTTPSetMediaWrite 0x9d028614           0xcc         204   
.text.ENCX24J600_MACPow 0x9d0286e0           0xcc         204   
.text.WriteMemoryWindow 0x9d0287ac           0xcc         204   
.text.TCPIP_IPV4_SetPay 0x9d028878           0xcc         204   
.text.DNSRetry          0x9d028944           0xc8         200   
.text.DNSDiscardName    0x9d028a0c           0xc8         200   
.text.UDPClose          0x9d028ad4           0xc8         200   
.text.UDPSetTxOffset    0x9d028b9c           0xc8         200   
.text.InitNetConfig     0x9d028c64           0xc8         200   
.text.TCPIP_Helper_Form 0x9d028d2c           0xc8         200   
.text.HTTPPrintIP       0x9d028df4           0xc8         200   
.text.CmdAddHead        0x9d028ebc           0xc4         196   
.text.MPFSInit          0x9d028f80           0xc4         196   
.text._LoadFATRecord    0x9d029044           0xc4         196   
.text._DHCPEnable       0x9d029108           0xc4         196   
.text.SYS_TICK_Initiali 0x9d0291cc           0xc0         192   
.text._SYS_COMMAND_INIT 0x9d02928c           0xbc         188   
.text.XEEInit           0x9d029348           0xbc         188   
.text._ARPRemoveEntry   0x9d029404           0xbc         188   
.text.ENCX24_MACInitial 0x9d0294c0           0xbc         188   
.text.OAHashRemoveAll   0x9d02957c           0xbc         188   
.text.UDPDiscardNet     0x9d029638           0xbc         188   
.text.TCPIP_Helper_Stri 0x9d0296f4           0xbc         188   
.text._SYS_DEBUG_INIT   0x9d0297b0           0xb8         184   
.text._SYS_CONSOLE_INIT 0x9d029868           0xb8         184   
.text.Execute0          0x9d029920           0xb8         184   
.text.TCPv4AllocateTxPa 0x9d0299d8           0xb8         184   
.text._TCPIsGetReady    0x9d029a90           0xb8         184   
.text.UDPGetTxCount     0x9d029b48           0xb8         184   
.text.MPFSGetEndAddr    0x9d029c00           0xb4         180   
.text.Delay10us         0x9d029cb4           0xb4         180   
.text._TcpMac2RamCopy   0x9d029d68           0xb4         180   
.text.UDPv4AllocateTxPa 0x9d029e1c           0xb4         180   
.text.UDPIsTxPutReady   0x9d029ed0           0xb4         180   
.text._mon_putc         0x9d029f84           0xb4         180   
.text.CommandQuit       0x9d02a038           0xb0         176   
.text.CmdRemoveTail     0x9d02a0e8           0xb0         176   
.text.TCPIP_ANNOUNCE_De 0x9d02a198           0xb0         176   
.text._ARPRemoveCacheEn 0x9d02a248           0xb0         176   
.text._ARPNotifyClients 0x9d02a2f8           0xb0         176   
.text.ENCX24J600_MACGet 0x9d02a3a8           0xb0         176   
.text._Tcpv4AckFnc      0x9d02a458           0xb0         176   
.text._TCPIPStackSetNet 0x9d02a508           0xb0         176   
.text.MPFSGetFlags      0x9d02a5b8           0xac         172   
.text.MPFSGetSize       0x9d02a664           0xac         172   
.text.MPFSGetStartAddr  0x9d02a710           0xac         172   
.rodata                 0x9d02a7bc           0xac         172  Read-only const 
.text.TCPIsConnected    0x9d02a868           0xac         172   
.text.HTTPPrint_cookien 0x9d02a914           0xac         172   
.text._SYS_ERROR        0x9d02a9c0           0xa8         168   
.text.ARPDeinitialize   0x9d02aa68           0xa8         168   
.text.ENCX24J600_MACPow 0x9d02ab10           0xa8         168   
.text._TCPIPStackString 0x9d02abb8           0xa8         168   
.text                   0x9d02ac60           0xa8         168  App's exec code 
.text._Validate         0x9d02ad08           0xa4         164   
.text.XEEWriteArray     0x9d02adac           0xa4         164   
.text.DNSResolve        0x9d02ae50           0xa4         164   
.text.ReadPHYReg        0x9d02aef4           0xa4         164   
.text._ICMPAllocateTxPa 0x9d02af98           0xa4         164   
.text.TCPIP_IPV4_DeInit 0x9d02b03c           0xa4         164   
.text._TCPIPStackNetByA 0x9d02b0e0           0xa4         164   
.text.HTTPPrint_helloms 0x9d02b184           0xa4         164   
.text._sbrk             0x9d02b228           0xa4         164   
.text.USART_GETS        0x9d02b2cc           0xa0         160   
.text.XEEWrite          0x9d02b36c           0xa0         160   
.text._DHCPDiscard      0x9d02b40c           0xa0         160   
.text._DHCPNotifyClient 0x9d02b4ac           0xa0         160   
.text.ENCX24J600_MACDis 0x9d02b54c           0xa0         160   
.text._UdpSocketDcpt    0x9d02b5ec           0xa0         160   
.text.HTTPPrint_buildda 0x9d02b68c           0xa0         160   
.rodata                 0x9d02b72c           0xa0         160  Read-only const 
.text.strupr            0x9d02b7cc           0x9c         156   
.text.ANNOUNCE_Notify   0x9d02b868           0x9c         156   
.text.DHCPRegisterHandl 0x9d02b904           0x9c         156   
.text._TcpSocketKill    0x9d02b9a0           0x9c         156   
.text.TCPIsAvailablePor 0x9d02ba3c           0x9c         156   
.text.UdpIsAvailablePor 0x9d02bad8           0x9c         156   
.text._TCPIPStackMacIdT 0x9d02bb74           0x9c         156   
.text.SingleListRemoveH 0x9d02bc10           0x9c         156   
.text.HTTPPrint_ddns_st 0x9d02bcac           0x9c         156   
.text._SYS_DEBUG_OPEN   0x9d02bd48           0x98         152   
.text._SYS_ASSERT       0x9d02bde0           0x98         152   
.text._SYS_CONSOLE_OPEN 0x9d02be78           0x98         152   
.text.MPFSDeinit        0x9d02bf10           0x98         152   
.text.DelayMs           0x9d02bfa8           0x98         152   
.text                   0x9d02c040           0x98         152  App's exec code 
.text.HTTPHeaderParseLo 0x9d02c0d8           0x94         148   
.text.TCPWasReset       0x9d02c16c           0x94         148   
.text.TCP_PutArray      0x9d02c200           0x94         148   
.text.SingleListAddTail 0x9d02c294           0x94         148   
.text.USART_PRINT       0x9d02c328           0x90         144   
.text._HttpCleanup      0x9d02c3b8           0x90         144   
.text.DHCPIsBound       0x9d02c448           0x90         144   
.text.TCPIP_IPV4_FreePa 0x9d02c4d8           0x90         144   
.text.NBNSDeInit        0x9d02c568           0x90         144   
.text.TCPDiscard        0x9d02c5f8           0x90         144   
.text.TCP_SetPayload    0x9d02c688           0x90         144   
.text.atol              0x9d02c718           0x90         144   
.text.SYS_TICK_MsDelay  0x9d02c7a8           0x8c         140   
.text.SYS_TICK_UsDelay  0x9d02c834           0x8c         140   
.text.HTTPReadPostName  0x9d02c8c0           0x8c         140   
.text.SwapARPPacket     0x9d02c94c           0x8c         140   
.text.DNSClientInit     0x9d02c9d8           0x8c         140   
.text.WritePHYReg       0x9d02ca64           0x8c         140   
.text.SwapIPV4Header    0x9d02caf0           0x8c         140   
.text.UDPFlush          0x9d02cb7c           0x8c         140   
.text.UDPRemoteBind     0x9d02cc08           0x8c         140   
.text.HTTPNeedsAuth     0x9d02cc94           0x8c         140   
.text.HTTPPrint_status_ 0x9d02cd20           0x8c         140   
.text.HTTPPrint_status_ 0x9d02cdac           0x8c         140   
.text.write             0x9d02ce38           0x8c         140   
.text.SHA1Initialize    0x9d02cec4           0x88         136   
.text._SysGetCDevEntry  0x9d02cf4c           0x88         136   
.text.DHCPDeInit        0x9d02cfd4           0x88         136   
.text.TCP_IsTxPutReady  0x9d02d05c           0x88         136   
.text.TCP_PutHeader     0x9d02d0e4           0x88         136   
.text._TCPIPStackIpAddT 0x9d02d16c           0x88         136   
.text._TCPIPStackMACIdT 0x9d02d1f4           0x88         136   
.text.TCPIP_STACK_NetBc 0x9d02d27c           0x88         136   
.text.LFSRSeedRand      0x9d02d304           0x84         132   
.text._SYS_CONSOLE_PRIN 0x9d02d388           0x84         132   
.text.DRV_MEDIA_ReadSet 0x9d02d40c           0x84         132   
.text.ENCX24_MACPowerMo 0x9d02d490           0x84         132   
.text.OAHashInit        0x9d02d514           0x84         132   
.text._TCPIP_HEAP_Callo 0x9d02d598           0x84         132   
.text.TcpipStackFindMod 0x9d02d61c           0x84         132   
.text.TcpipStackFindMac 0x9d02d6a0           0x84         132   
.text.HTTPCheckAuth     0x9d02d724           0x84         132   
.text.atoi              0x9d02d7a8           0x84         132   
.text.TCPIP_IPV4_FlushD 0x9d02d82c           0x80         128   
.text.TCPDisconnect     0x9d02d8ac           0x80         128   
.text.TCP_IsTxReady     0x9d02d92c           0x80         128   
.text.TCP_CopyTxPacketS 0x9d02d9ac           0x80         128   
.text._Udpv4AckFnc      0x9d02da2c           0x80         128   
.text._SYS_CMDIO_GET_HA 0x9d02daac           0x7c         124   
.text.SYS_FS_setdefdir  0x9d02db28           0x7c         124   
.text.TCPFind           0x9d02dba4           0x7c         124   
.text.TCP_Flush         0x9d02dc20           0x7c         124   
.text._TCPIPStackAddres 0x9d02dc9c           0x7c         124   
.text.HTTPPrint_config_ 0x9d02dd18           0x7c         124   
.text.LFSRRand          0x9d02dd94           0x78         120   
.text.SYS_TICK_TimerSet 0x9d02de0c           0x78         120   
.text.DHCPDeRegisterHan 0x9d02de84           0x78         120   
.text.DNSClientDeInit   0x9d02defc           0x78         120   
.text.ENCX24J600_MACSet 0x9d02df74           0x78         120   
.text.SoftReset         0x9d02dfec           0x78         120   
.text.rand              0x9d02e064           0x78         120   
.text.strstr            0x9d02e0dc           0x78         120   
.text.MD5Initialize     0x9d02e154           0x74         116   
.text.SYS_RANDOM_ADD    0x9d02e1c8           0x74         116   
.text.CommandCleanup    0x9d02e23c           0x74         116   
.text.SYS_FS_IsLegalDir 0x9d02e2b0           0x74         116   
.text.TCPIP_IPV4_SetTxB 0x9d02e324           0x74         116   
.text.TCP_GetUpperLayer 0x9d02e398           0x74         116   
.text.TCP_IsPacketQueue 0x9d02e40c           0x74         116   
.text.TCP_ResetTransmit 0x9d02e480           0x74         116   
.text._TCPIP_HEAP_FreeD 0x9d02e4f4           0x74         116   
.text.UDPIsConnected    0x9d02e568           0x74         116   
.text.HTTPPrint_pot     0x9d02e5dc           0x74         116   
.text.HTTPPrint_config_ 0x9d02e650           0x74         116   
.text._sys_CONSOLE_PRIN 0x9d02e6c4           0x70         112   
.text._ARPDeleteCache   0x9d02e734           0x70         112   
.text.ENCX24_MACOpen    0x9d02e7a4           0x70         112   
.text.ENCX24_MACCheckLi 0x9d02e814           0x70         112   
.text.ICMPInitialize    0x9d02e884           0x70         112   
.text.TCPIP_IPV4_Single 0x9d02e8f4           0x70         112   
.text.NBNSInit          0x9d02e964           0x70         112   
.text.TCPPutString      0x9d02e9d4           0x70         112   
.text.TCPIPMacEventCB   0x9d02ea44           0x70         112   
.text.HTTPPrint_config_ 0x9d02eab4           0x70         112   
.text.HTTPPrint_config_ 0x9d02eb24           0x70         112   
.text.HTTPPrint_config_ 0x9d02eb94           0x70         112   
.text.HTTPPrint_config_ 0x9d02ec04           0x70         112   
.text.HTTPPrint_config_ 0x9d02ec74           0x70         112   
.text.CommandReset      0x9d02ece4           0x6c         108   
.text._ARPRefreshEntry  0x9d02ed50           0x6c         108   
.text.ENCX24_MACPutHead 0x9d02edbc           0x6c         108   
.text._TCPGetRxFIFOFree 0x9d02ee28           0x6c         108   
.text.TcpClientIpv4Remo 0x9d02ee94           0x6c         108   
.text.TCPIP_HEAP_FreeSi 0x9d02ef00           0x6c         108   
.rodata                 0x9d02ef6c           0x6c         108  Read-only const 
.text.TCPIP_STACK_NetGa 0x9d02efd8           0x6c         108   
.text.TCPIP_STACK_NetPr 0x9d02f044           0x6c         108   
.text.TCPIP_STACK_NetSe 0x9d02f0b0           0x6c         108   
.text.TCPIP_STACK_NetBI 0x9d02f11c           0x6c         108   
.text.TCPIP_Notificatio 0x9d02f188           0x6c         108   
.text.MPFSGetPosition   0x9d02f1f4           0x68         104   
.text.OAHashGetEntry    0x9d02f25c           0x68         104   
.text.TCPIP_IPV4_FreePa 0x9d02f2c4           0x68         104   
.text._TcpSocketBind    0x9d02f32c           0x68         104   
.text._TcpSocketChk     0x9d02f394           0x68         104   
.text._TcpFlush         0x9d02f3fc           0x68         104   
.text.TCPIsGetReady     0x9d02f464           0x68         104   
.text.TCPGetRxFIFOFree  0x9d02f4cc           0x68         104   
.text._UdpSocketBind    0x9d02f534           0x68         104   
.text.MACPutHeader      0x9d02f59c           0x68         104   
.text.TCPIP_STACK_NetNa 0x9d02f604           0x68         104   
.text.TCPIP_Notificatio 0x9d02f66c           0x68         104   
.rodata                 0x9d02f6d4           0x68         104  Read-only const 
.text.btohexa_high      0x9d02f73c           0x64         100   
.text.btohexa_low       0x9d02f7a0           0x64         100   
.text.MPFSClose         0x9d02f804           0x64         100   
.text.DRV_MEDIA_ReadByt 0x9d02f868           0x64         100   
.text.DHCPIsEnabled     0x9d02f8cc           0x64         100   
.text.TCPIP_IPV4_GetDat 0x9d02f930           0x64         100   
.text.TCPSocketGetNet   0x9d02f994           0x64         100   
.text._TCPIPStackIsNetL 0x9d02f9f8           0x64         100   
.text.TCPIP_Notificatio 0x9d02fa5c           0x64         100   
.text._sprintf_cdnopsux 0x9d02fac0           0x64         100   
.text.SYS_DRIVERS_Initi 0x9d02fb24           0x60          96   
.text.USART_PUTC        0x9d02fb84           0x60          96   
.text.HTTPReleaseMedia  0x9d02fbe4           0x60          96   
.text.ENCX24_MACDeiniti 0x9d02fc44           0x60          96   
.text.ICMPDeinitialize  0x9d02fca4           0x60          96   
.text.TCPIP_IPV4_SetRxB 0x9d02fd04           0x60          96   
.text.TCP_FreePacket    0x9d02fd64           0x60          96   
.text.MACCalcRxChecksum 0x9d02fdc4           0x60          96   
.rodata                 0x9d02fe24           0x60          96  Read-only const 
.text.HTTPPrint_reboota 0x9d02fe84           0x60          96   
.text.MPFSGetLong       0x9d02fee4           0x5c          92   
.text._DHCPCleanup      0x9d02ff40           0x5c          92   
.text.OAHashRemoveEntry 0x9d02ff9c           0x5c          92   
.text.TCPFlush          0x9d02fff8           0x5c          92   
.text.MACGetArray       0x9d030054           0x5c          92   
.text.MACPutArray       0x9d0300b0           0x5c          92   
.text._TCPIPStackNetAdd 0x9d03010c           0x5c          92   
.text._TCPIPStackNetMas 0x9d030168           0x5c          92   
.text._TCPIPStackNetMac 0x9d0301c4           0x5c          92   
.text.USART_OPEN        0x9d030220           0x58          88   
.text.USART_GETC        0x9d030278           0x58          88   
.text.LCD_ERASE         0x9d0302d0           0x58          88   
.text.WaitForDataByte   0x9d030328           0x58          88   
.text._XEEFlashInit     0x9d030380           0x58          88   
.text.ARPHashKeyHash    0x9d0303d8           0x58          88   
.text.ENCX24J600_MACSet 0x9d030430           0x58          88   
.text.ENCX24J600_MACSet 0x9d030488           0x58          88   
.text._TcpipHeapHandleT 0x9d0304e0           0x58          88   
.text.TCPIP_STACK_IxToN 0x9d030538           0x58          88   
.text._TCPIPStackIsNetU 0x9d030590           0x58          88   
.text.HTTPPrint_ddns_st 0x9d0305e8           0x58          88   
.text.HTTPPrint_smtps_e 0x9d030640           0x58          88   
.text.HTTPPrint_snmp_en 0x9d030698           0x58          88   
.text._SYS_CONSOLE_PUTC 0x9d0306f0           0x54          84   
.text._SYS_OUT_MESSAGE_ 0x9d030744           0x54          84   
.text.ENCX24_MACCalcRxC 0x9d030798           0x54          84   
.text._ICMPAckPacket    0x9d0307ec           0x54          84   
.text._TcpDiscardTx     0x9d030840           0x54          84   
.text.TCPPut            0x9d030894           0x54          84   
.text._UdpSocketInit    0x9d0308e8           0x54          84   
.text.UDPPut            0x9d03093c           0x54          84   
.text.MACGetHeader      0x9d030990           0x54          84   
.text.MACSetReadPtrInRx 0x9d0309e4           0x54          84   
.text.MACCalcIPBufferCh 0x9d030a38           0x54          84   
.text._TCPIPStackAddres 0x9d030a8c           0x54          84   
.text.HTTPPrint_version 0x9d030ae0           0x54          84   
.rodata                 0x9d030b34           0x54          84  Read-only const 
.text._vsnprintf_cdnops 0x9d030b88           0x54          84   
.text.vsnprintf         0x9d030bdc           0x54          84   
.text._SYS_CONSOLE_MESS 0x9d030c30           0x50          80   
.text._TCPIP_AnnounceCl 0x9d030c80           0x50          80   
.text.HTTPPrint_        0x9d030cd0           0x50          80   
.text.ARPHashKeyCompare 0x9d030d20           0x50          80   
.text._DNSReleaseSocket 0x9d030d70           0x50          80   
.text.strncpy           0x9d030dc0           0x50          80   
.text.DRV_SPI_Initializ 0x9d030e10           0x4c          76   
.text.ENCX24J600_MACPut 0x9d030e5c           0x4c          76   
.rodata                 0x9d030ea8           0x4c          76  Read-only const 
.text.ENCX24_MACPutArra 0x9d030ef4           0x4c          76   
.text.ENCX24_MACGetArra 0x9d030f40           0x4c          76   
.text.TCPGet            0x9d030f8c           0x4c          76   
.text.UDPGet            0x9d030fd8           0x4c          76   
.text.MACSetWritePtr    0x9d031024           0x4c          76   
.text.MACSetReadPtr     0x9d031070           0x4c          76   
.text.INTEnable         0x9d0310bc           0x4c          76   
.text                   0x9d031108           0x4c          76  App's exec code 
.text.SYS_CLK_Periphera 0x9d031154           0x48          72   
.text._SYS_CONSOLE_DATA 0x9d03119c           0x48          72   
.text._SYS_CONSOLE_GETC 0x9d0311e4           0x48          72   
.text._SYS_OUT_MESSAGE_ 0x9d03122c           0x48          72   
.rodata                 0x9d031274           0x48          72  Read-only const 
.text.HTTPCurConnection 0x9d0312bc           0x48          72   
.text.ARPHashKeyCopy    0x9d031304           0x48          72   
.text.DNSEndUsage       0x9d03134c           0x48          72   
.text.TCPIP_IPV4_SetSou 0x9d031394           0x48          72   
.text.TCPIP_STACK_NetAd 0x9d0313dc           0x48          72   
.text.TCPIP_STACK_NetMa 0x9d031424           0x48          72   
.text.TCPIP_STACK_NetMa 0x9d03146c           0x48          72   
.text._DefaultInterrupt 0x9d0314b4           0x48          72   
.text.sbrk              0x9d0314fc           0x48          72   
.text.SYS_CLK_ClockGet  0x9d031544           0x44          68   
.text._SYS_OUT_MESSAGE  0x9d031588           0x44          68   
.text._sys_CONSOLE_PUTC 0x9d0315cc           0x44          68   
.text.MPFSGetID         0x9d031610           0x44          68   
.text.USART_DATA_RDY    0x9d031654           0x44          68   
.text.ENCX24_MACGetHead 0x9d031698           0x44          68   
.text.ENCX24_MACSetRead 0x9d0316dc           0x44          68   
.text.ENCX24_MACCalcIPB 0x9d031720           0x44          68   
.text.TCPIP_IPV4_SetPac 0x9d031764           0x44          68   
.text.MACClose          0x9d0317a8           0x44          68   
.text.MACDiscardRx      0x9d0317ec           0x44          68   
.text.MACIsTxReady      0x9d031830           0x44          68   
.text.MACFlush          0x9d031874           0x44          68   
.text.MACCheckLink      0x9d0318b8           0x44          68   
.text.MACGetTxBaseAddr  0x9d0318fc           0x44          68   
.text.ProcessTCPIPMacGe 0x9d031940           0x44          68   
.text.TCPIP_STACK_NetHa 0x9d031984           0x44          68   
.text._TCPIPStackNetIx  0x9d0319c8           0x44          68   
.text._TCPIPStackSetGat 0x9d031a0c           0x44          68   
.text._TCPIPStackSetPri 0x9d031a50           0x44          68   
.text._TCPIPStackSetSec 0x9d031a94           0x44          68   
.text._TCPIPStackNetToM 0x9d031ad8           0x44          68   
.text.SingleListInit    0x9d031b1c           0x44          68   
.text.strncat           0x9d031b60           0x44          68   
.text.strncmp           0x9d031ba4           0x44          68   
.text                   0x9d031be8           0x44          68  App's exec code 
.text.XEEEndWrite       0x9d031c2c           0x40          64   
.text.HTTPCurConnection 0x9d031c6c           0x40          64   
.text.HTTPCurConnection 0x9d031cac           0x40          64   
.text.ENCX24J600_MACChe 0x9d031cec           0x40          64   
.text.ENCX24J600_MACIsT 0x9d031d2c           0x40          64   
.text.TCPIP_IPV4_Task   0x9d031d6c           0x40          64   
.text.UDPResetHeader    0x9d031dac           0x40          64   
.text.SpiChnDataRdy     0x9d031dec           0x40          64   
.text._sys_CONSOLE_MESS 0x9d031e2c           0x3c          60   
.text.DRV_MEDIA_WriteFl 0x9d031e68           0x3c          60   
.text.HTTPCurConnection 0x9d031ea4           0x3c          60   
.text.HTTPCurConnection 0x9d031ee0           0x3c          60   
.text._ARPDeleteClients 0x9d031f1c           0x3c          60   
.text.ARPTmoHandler     0x9d031f58           0x3c          60   
.text.ENCX24_MACSetWrit 0x9d031f94           0x3c          60   
.text.ENCX24_MACSetRead 0x9d031fd0           0x3c          60   
.text.TCPIP_IPV4_GetUpp 0x9d03200c           0x3c          60   
.text.TCPIP_IPV4_GetPay 0x9d032048           0x3c          60   
.rodata                 0x9d032084           0x3c          60  Read-only const 
.text.PORTSetPinsDigita 0x9d0320c0           0x3c          60   
.text.PORTSetPinsDigita 0x9d0320fc           0x3c          60   
.text                   0x9d032138           0x38          56  App's exec code 
.text.SYS_Tasks         0x9d032170           0x38          56   
.text._SYS_OUT_INIT     0x9d0321a8           0x38          56   
.text.DRV_MEDIA_Close   0x9d0321e0           0x38          56   
.text.ENCX24J600_MACGet 0x9d032218           0x38          56   
.text.ENCX24_MACClose   0x9d032250           0x38          56   
.text.ENCX24_MACGetRead 0x9d032288           0x38          56   
.text._OAHashProbeStep  0x9d0322c0           0x38          56   
.text.INTSetVectorPrior 0x9d0322f8           0x38          56   
.text.INTSetVectorSubPr 0x9d032330           0x38          56   
.text._sys_CONSOLE_DATA 0x9d032368           0x34          52   
.text._sys_CONSOLE_GETC 0x9d03239c           0x34          52   
.text.XEEBeginWrite     0x9d0323d0           0x34          52   
.text.DRV_MEDIA_ClientS 0x9d032404           0x34          52   
.text.HTTPCurConnection 0x9d032438           0x34          52   
.text.HTTPCurConnection 0x9d03246c           0x34          52   
.text.HTTPCurConnection 0x9d0324a0           0x34          52   
.text.HTTPCurConnection 0x9d0324d4           0x34          52   
.text.HTTPCurConnection 0x9d032508           0x34          52   
.text.ENCX24_MACIsTxRea 0x9d03253c           0x34          52   
.text.ENCX24_MACFlush   0x9d032570           0x34          52   
.text.ENCX24_MACDiscard 0x9d0325a4           0x34          52   
.text.TCPIP_IPV4_SetDes 0x9d0325d8           0x34          52   
.text.TCPIP_IPV4_GetDes 0x9d03260c           0x34          52   
.text.TCPIP_IPV4_GetSou 0x9d032640           0x34          52   
.text.ProcessTCPIPMacEr 0x9d032674           0x34          52   
.text.HTTPPrint_reboot  0x9d0326a8           0x34          52   
.text.INTEnableSystemMu 0x9d0326dc           0x34          52   
.text.SYS_USERIO_Tasks  0x9d032710           0x30          48   
.text.SYS_FS_mpfs2fs_In 0x9d032740           0x30          48   
.text.TCPIP_IPV4_TmoHan 0x9d032770           0x30          48   
.text._TcpTmoHandler    0x9d0327a0           0x30          48   
.text.TCPIP_STACK_TickH 0x9d0327d0           0x30          48   
.text.strcat            0x9d032800           0x30          48   
.text.SYS_WDT_Clear     0x9d032830           0x2c          44   
.text.TCPIP_ANNOUNCE_Ta 0x9d03285c           0x2c          44   
.text.ARPTaskPending    0x9d032888           0x2c          44   
.text.ENCX24_MACSetRXHa 0x9d0328b4           0x2c          44   
.text.TCPIP_IPV4_TaskPe 0x9d0328e0           0x2c          44   
.text.TCPTaskPending    0x9d03290c           0x2c          44   
.text.HTTPPrint_read_co 0x9d032938           0x2c          44   
.text.HTTPPrint_write_c 0x9d032964           0x2c          44   
.text.HTTPPrint_ddns_se 0x9d032990           0x2c          44   
.text.strchr            0x9d0329bc           0x2c          44   
.text._stub_sbd_memlayo 0x9d0329e8           0x2c          44   
.text.SYS_FS_GenError   0x9d032a14           0x28          40   
.rodata                 0x9d032a3c           0x28          40  Read-only const 
.text.ENCX24_MACGetTxBa 0x9d032a64           0x28          40   
.text.ZCLLEnable        0x9d032a8c           0x28          40   
.text.INTClearFlag      0x9d032ab4           0x28          40   
.text._ENCX24_Deinitial 0x9d032adc           0x24          36   
.text.TCPIP_STACK_GetDe 0x9d032b00           0x24          36   
.text.TCPIP_STACK_Netwo 0x9d032b24           0x24          36   
.text.HTTPPrint_lcdtext 0x9d032b48           0x24          36   
.text.HTTPPrint_ddns_us 0x9d032b6c           0x24          36   
.text.HTTPPrint_ddns_pa 0x9d032b90           0x24          36   
.text.HTTPPrint_ddns_ho 0x9d032bb4           0x24          36   
.text._snprintf_cdnopsu 0x9d032bd8           0x24          36   
.text.toupper           0x9d032bfc           0x24          36   
.rodata                 0x9d032c20           0x20          32  Read-only const 
.text.SpiChnReadC       0x9d032c40           0x20          32   
.text.SpiChnWriteC      0x9d032c60           0x20          32   
.text.SpiChnTxBuffEmpty 0x9d032c80           0x20          32   
.text.INTRestoreInterru 0x9d032ca0           0x1c          28   
.text.free              0x9d032cbc           0x1c          28   
.text.srand             0x9d032cd8           0x1c          28   
.text.SYS_Reboot        0x9d032cf4           0x18          24   
.text.CheKseg0CacheOn   0x9d032d0c           0x18          24   
.text                   0x9d032d24           0x18          24  App's exec code 
.rodata                 0x9d032d3c           0x34          52  Read-only const 
.text.OpenCoreTimer     0x9d032d70            0xc          12   
.text._bootstrap_except 0x9d032d7c            0xc          12   
.text.INTDisableInterru 0x9d032d88            0x8           8   
.text.INTEnableInterrup 0x9d032d90            0x8           8   
.text._on_reset         0x9d032d98            0x8           8   
.text._on_bootstrap     0x9d032da0            0x8           8   
.rodata                 0x9d032da8            0x8           8  Read-only const 
      Total kseg0_program_mem used  :     0x32d90      208272  39.7% of 0x80000

kseg0 Boot-Memory Usage
section                    address  length [bytes]      (dec)  Description
-------                 ----------  -------------------------  -----------
         Total kseg0_boot_mem used  :           0           0  <1% of 0x970

Exception-Memory Usage 
section                    address  length [bytes]      (dec)  Description
-------                 ----------  -------------------------  -----------
.app_excpt              0x9fc01180           0x10          16  General-Exception 
.vector_0               0x9fc01200            0x8           8  Interrupt Vector 0 
.vector_1               0x9fc01220            0x8           8  Interrupt Vector 1 
.vector_2               0x9fc01240            0x8           8  Interrupt Vector 2 
.vector_3               0x9fc01260            0x8           8  Interrupt Vector 3 
.vector_4               0x9fc01280            0x8           8  Interrupt Vector 4 
.vector_5               0x9fc012a0            0x8           8  Interrupt Vector 5 
.vector_6               0x9fc012c0            0x8           8  Interrupt Vector 6 
.vector_7               0x9fc012e0            0x8           8  Interrupt Vector 7 
.vector_8               0x9fc01300            0x8           8  Interrupt Vector 8 
.vector_9               0x9fc01320            0x8           8  Interrupt Vector 9 
.vector_10              0x9fc01340            0x8           8  Interrupt Vector 10 
.vector_11              0x9fc01360            0x8           8  Interrupt Vector 11 
.vector_12              0x9fc01380            0x8           8  Interrupt Vector 12 
.vector_13              0x9fc013a0            0x8           8  Interrupt Vector 13 
.vector_14              0x9fc013c0            0x8           8  Interrupt Vector 14 
.vector_15              0x9fc013e0            0x8           8  Interrupt Vector 15 
.vector_16              0x9fc01400            0x8           8  Interrupt Vector 16 
.vector_17              0x9fc01420            0x8           8  Interrupt Vector 17 
.vector_18              0x9fc01440            0x8           8  Interrupt Vector 18 
.vector_19              0x9fc01460            0x8           8  Interrupt Vector 19 
.vector_20              0x9fc01480            0x8           8  Interrupt Vector 20 
.vector_21              0x9fc014a0            0x8           8  Interrupt Vector 21 
.vector_22              0x9fc014c0            0x8           8  Interrupt Vector 22 
.vector_23              0x9fc014e0            0x8           8  Interrupt Vector 23 
.vector_24              0x9fc01500            0x8           8  Interrupt Vector 24 
.vector_25              0x9fc01520            0x8           8  Interrupt Vector 25 
.vector_26              0x9fc01540            0x8           8  Interrupt Vector 26 
.vector_27              0x9fc01560            0x8           8  Interrupt Vector 27 
.vector_28              0x9fc01580            0x8           8  Interrupt Vector 28 
.vector_29              0x9fc015a0            0x8           8  Interrupt Vector 29 
.vector_30              0x9fc015c0            0x8           8  Interrupt Vector 30 
.vector_31              0x9fc015e0            0x8           8  Interrupt Vector 31 
.vector_32              0x9fc01600            0x8           8  Interrupt Vector 32 
.vector_33              0x9fc01620            0x8           8  Interrupt Vector 33 
.vector_34              0x9fc01640            0x8           8  Interrupt Vector 34 
.vector_35              0x9fc01660            0x8           8  Interrupt Vector 35 
.vector_36              0x9fc01680            0x8           8  Interrupt Vector 36 
.vector_37              0x9fc016a0            0x8           8  Interrupt Vector 37 
.vector_38              0x9fc016c0            0x8           8  Interrupt Vector 38 
.vector_39              0x9fc016e0            0x8           8  Interrupt Vector 39 
.vector_40              0x9fc01700            0x8           8  Interrupt Vector 40 
.vector_41              0x9fc01720            0x8           8  Interrupt Vector 41 
.vector_42              0x9fc01740            0x8           8  Interrupt Vector 42 
.vector_43              0x9fc01760            0x8           8  Interrupt Vector 43 
.vector_44              0x9fc01780            0x8           8  Interrupt Vector 44 
.vector_45              0x9fc017a0            0x8           8  Interrupt Vector 45 
.vector_46              0x9fc017c0            0x8           8  Interrupt Vector 46 
.vector_47              0x9fc017e0            0x8           8  Interrupt Vector 47 
.vector_48              0x9fc01800            0x8           8  Interrupt Vector 48 
.vector_49              0x9fc01820            0x8           8  Interrupt Vector 49 
.vector_50              0x9fc01840            0x8           8  Interrupt Vector 50 
.vector_51              0x9fc01860            0x8           8  Interrupt Vector 51 
.vector_52              0x9fc01880            0x8           8  Interrupt Vector 52 
.vector_53              0x9fc018a0            0x8           8  Interrupt Vector 53 
.vector_54              0x9fc018c0            0x8           8  Interrupt Vector 54 
.vector_55              0x9fc018e0            0x8           8  Interrupt Vector 55 
.vector_56              0x9fc01900            0x8           8  Interrupt Vector 56 
.vector_57              0x9fc01920            0x8           8  Interrupt Vector 57 
.vector_58              0x9fc01940            0x8           8  Interrupt Vector 58 
.vector_59              0x9fc01960            0x8           8  Interrupt Vector 59 
.vector_60              0x9fc01980            0x8           8  Interrupt Vector 60 
.vector_61              0x9fc019a0            0x8           8  Interrupt Vector 61 
.vector_62              0x9fc019c0            0x8           8  Interrupt Vector 62 
.vector_63              0x9fc019e0            0x8           8  Interrupt Vector 63 
          Total exception_mem used  :       0x210         528  12.9% of 0x1000

kseg1 Boot-Memory Usage
section                    address  length [bytes]      (dec)  Description
-------                 ----------  -------------------------  -----------
.reset                  0xbfc00000          0x1f4         500  Reset handler 
.bev_excpt              0xbfc00380           0x10          16  BEV-Exception 
         Total kseg1_boot_mem used  :       0x204         516  44.2% of 0x490
        --------------------------------------------------------------------------
         Total Program Memory used  :     0x331a4      209316  39.3% of 0x81e00
        --------------------------------------------------------------------------


kseg1 Data-Memory Usage
section                    address  length [bytes]      (dec)  Description
-------                 ----------  -------------------------  -----------
.eh_frame               0xa0000000           0x30          48   
.sdata                  0xa0000030           0xe0         224  Small init data 
.sbss                   0xa0000110          0x38c         908  Small uninit data 
.bss                    0xa000049c         0x1adc        6876  Uninitialized data 
.bss                    0xa0001f78          0x458        1112  Uninitialized data 
.data                   0xa00023d0           0x44          68  Initialized data 
.bss                    0xa0002414           0x7c         124  Uninitialized data 
         Total kseg1_data_mem used  :      0x2490        9360  7.1% of 0x20000
        --------------------------------------------------------------------------
            Total Data Memory used  :      0x2490        9360  7.1% of 0x20000
        --------------------------------------------------------------------------


Dynamic Data-Memory Reservation
section                    address  length [bytes]      (dec)  Description
-------                 ----------  -------------------------  -----------
heap                    0xa0002498         0x6400       25600  Reserved for heap 
stack                   0xa00088b0        0x17748       96072  Reserved for stack 

        --------------------------------------------------------------------------

Discarded input sections

 .data          0x00000000        0x0 c:/program files (x86)/microchip/xc32/v1.21/bin/../lib/gcc/pic32mx/4.5.2/../../../../pic32mx/lib/size/crt0.o
 .bss           0x00000000        0x0 c:/program files (x86)/microchip/xc32/v1.21/bin/../lib/gcc/pic32mx/4.5.2/../../../../pic32mx/lib/size/crt0.o
 .pdr           0x00000000       0xa0 c:/program files (x86)/microchip/xc32/v1.21/bin/../lib/gcc/pic32mx/4.5.2/../../../../pic32mx/lib/size/crt0.o
 .text          0x00000000        0x0 build/default/production/_ext/1293749816/bsp.o
 .data          0x00000000        0x0 build/default/production/_ext/1293749816/bsp.o
 .bss           0x00000000        0x0 build/default/production/_ext/1293749816/bsp.o
 .reginfo       0x00000000       0x18 build/default/production/_ext/1293749816/bsp.o
 .pdr           0x00000000       0x20 build/default/production/_ext/1293749816/bsp.o
 .text          0x00000000        0x0 build/default/production/_ext/101875047/lfsr.o
 .data          0x00000000        0x0 build/default/production/_ext/101875047/lfsr.o
 .bss           0x00000000        0x0 build/default/production/_ext/101875047/lfsr.o
 .reginfo       0x00000000       0x18 build/default/production/_ext/101875047/lfsr.o
 .pdr           0x00000000       0x40 build/default/production/_ext/101875047/lfsr.o
 .text          0x00000000      0x400 build/default/production/_ext/101875047/big_int_helper_c32.o
 .data          0x00000000        0x0 build/default/production/_ext/101875047/big_int_helper_c32.o
 .bss           0x00000000       0x20 build/default/production/_ext/101875047/big_int_helper_c32.o
 .reginfo       0x00000000       0x18 build/default/production/_ext/101875047/big_int_helper_c32.o
 .pdr           0x00000000      0x100 build/default/production/_ext/101875047/big_int_helper_c32.o
 .text          0x00000000        0x0 build/default/production/_ext/101875047/big_int.o
 .data          0x00000000        0x0 build/default/production/_ext/101875047/big_int.o
 .bss           0x00000000        0x0 build/default/production/_ext/101875047/big_int.o
 .reginfo       0x00000000       0x18 build/default/production/_ext/101875047/big_int.o
 .pdr           0x00000000      0x1a0 build/default/production/_ext/101875047/big_int.o
 .text.BigInt   0x00000000       0x70 build/default/production/_ext/101875047/big_int.o
 .text.BigIntZero
                0x00000000       0x68 build/default/production/_ext/101875047/big_int.o
 .text.BigIntMod
                0x00000000      0x220 build/default/production/_ext/101875047/big_int.o
 .text.BigIntCompare
                0x00000000      0x16c build/default/production/_ext/101875047/big_int.o
 .text.BigIntMagnitudeDifference
                0x00000000       0x58 build/default/production/_ext/101875047/big_int.o
 .text.BigIntMagnitude
                0x00000000       0x50 build/default/production/_ext/101875047/big_int.o
 .text.BigIntMSB
                0x00000000       0xac build/default/production/_ext/101875047/big_int.o
 .text.BigIntMultiply
                0x00000000       0x94 build/default/production/_ext/101875047/big_int.o
 .text.BigIntSquare
                0x00000000       0x74 build/default/production/_ext/101875047/big_int.o
 .text.BigIntAdd
                0x00000000       0x74 build/default/production/_ext/101875047/big_int.o
 .text.BigIntSubtract
                0x00000000       0x74 build/default/production/_ext/101875047/big_int.o
 .text.BigIntCopy
                0x00000000       0x70 build/default/production/_ext/101875047/big_int.o
 .text.BigIntSwapEndianness
                0x00000000       0x9c build/default/production/_ext/101875047/big_int.o
 .text          0x00000000        0x0 build/default/production/_ext/101875047/hashes.o
 .data          0x00000000        0x0 build/default/production/_ext/101875047/hashes.o
 .bss           0x00000000        0x0 build/default/production/_ext/101875047/hashes.o
 .reginfo       0x00000000       0x18 build/default/production/_ext/101875047/hashes.o
 .pdr           0x00000000      0x120 build/default/production/_ext/101875047/hashes.o
 .text.HashAddData
                0x00000000       0x94 build/default/production/_ext/101875047/hashes.o
 .text.SHA1Calculate
                0x00000000      0x4b8 build/default/production/_ext/101875047/hashes.o
 .text          0x00000000        0x0 build/default/production/_ext/101875047/helpers.o
 .data          0x00000000        0x0 build/default/production/_ext/101875047/helpers.o
 .bss           0x00000000        0x0 build/default/production/_ext/101875047/helpers.o
 .reginfo       0x00000000       0x18 build/default/production/_ext/101875047/helpers.o
 .pdr           0x00000000      0x100 build/default/production/_ext/101875047/helpers.o
 .text.strnchr  0x00000000       0xb4 build/default/production/_ext/101875047/helpers.o
 .text.strncpy_m
                0x00000000      0x10c build/default/production/_ext/101875047/helpers.o
 .text          0x00000000        0x0 build/default/production/_ext/1472/berkeley_tcp_client_demo.o
 .data          0x00000000        0x0 build/default/production/_ext/1472/berkeley_tcp_client_demo.o
 .bss           0x00000000        0x0 build/default/production/_ext/1472/berkeley_tcp_client_demo.o
 .reginfo       0x00000000       0x18 build/default/production/_ext/1472/berkeley_tcp_client_demo.o
 .pdr           0x00000000        0x0 build/default/production/_ext/1472/berkeley_tcp_client_demo.o
 .text          0x00000000        0x0 build/default/production/_ext/1472/berkeley_tcp_server_demo.o
 .data          0x00000000        0x0 build/default/production/_ext/1472/berkeley_tcp_server_demo.o
 .bss           0x00000000        0x0 build/default/production/_ext/1472/berkeley_tcp_server_demo.o
 .reginfo       0x00000000       0x18 build/default/production/_ext/1472/berkeley_tcp_server_demo.o
 .pdr           0x00000000        0x0 build/default/production/_ext/1472/berkeley_tcp_server_demo.o
 .text          0x00000000        0x0 build/default/production/_ext/1472/berkeley_udp_client_demo.o
 .data          0x00000000        0x0 build/default/production/_ext/1472/berkeley_udp_client_demo.o
 .bss           0x00000000        0x0 build/default/production/_ext/1472/berkeley_udp_client_demo.o
 .reginfo       0x00000000       0x18 build/default/production/_ext/1472/berkeley_udp_client_demo.o
 .pdr           0x00000000        0x0 build/default/production/_ext/1472/berkeley_udp_client_demo.o
 .text          0x00000000        0x0 build/default/production/_ext/1472/generic_tcp_client.o
 .data          0x00000000        0x0 build/default/production/_ext/1472/generic_tcp_client.o
 .bss           0x00000000        0x0 build/default/production/_ext/1472/generic_tcp_client.o
 .reginfo       0x00000000       0x18 build/default/production/_ext/1472/generic_tcp_client.o
 .pdr           0x00000000        0x0 build/default/production/_ext/1472/generic_tcp_client.o
 .text          0x00000000        0x0 build/default/production/_ext/1472/generic_tcp_server.o
 .data          0x00000000        0x0 build/default/production/_ext/1472/generic_tcp_server.o
 .bss           0x00000000        0x0 build/default/production/_ext/1472/generic_tcp_server.o
 .reginfo       0x00000000       0x18 build/default/production/_ext/1472/generic_tcp_server.o
 .pdr           0x00000000        0x0 build/default/production/_ext/1472/generic_tcp_server.o
 .text          0x00000000        0x0 build/default/production/_ext/1472/ping_demo.o
 .data          0x00000000        0x0 build/default/production/_ext/1472/ping_demo.o
 .bss           0x00000000        0x0 build/default/production/_ext/1472/ping_demo.o
 .reginfo       0x00000000       0x18 build/default/production/_ext/1472/ping_demo.o
 .pdr           0x00000000       0x60 build/default/production/_ext/1472/ping_demo.o
 .sbss          0x00000000        0x8 build/default/production/_ext/1472/ping_demo.o
 .sdata         0x00000000        0x4 build/default/production/_ext/1472/ping_demo.o
 .text.Ping4    0x00000000       0x90 build/default/production/_ext/1472/ping_demo.o
 .text.PingDemoTask
                0x00000000       0x20 build/default/production/_ext/1472/ping_demo.o
 .rodata        0x00000000        0xc build/default/production/_ext/1472/ping_demo.o
 .text.PingProcessIPv4
                0x00000000      0x19c build/default/production/_ext/1472/ping_demo.o
 .text          0x00000000        0x0 build/default/production/_ext/1472/smtp_demo.o
 .data          0x00000000        0x0 build/default/production/_ext/1472/smtp_demo.o
 .bss           0x00000000        0x0 build/default/production/_ext/1472/smtp_demo.o
 .reginfo       0x00000000       0x18 build/default/production/_ext/1472/smtp_demo.o
 .pdr           0x00000000        0x0 build/default/production/_ext/1472/smtp_demo.o
 .text          0x00000000        0x0 build/default/production/_ext/365611741/system_services.o
 .data          0x00000000        0x0 build/default/production/_ext/365611741/system_services.o
 .bss           0x00000000        0x0 build/default/production/_ext/365611741/system_services.o
 .reginfo       0x00000000       0x18 build/default/production/_ext/365611741/system_services.o
 .pdr           0x00000000      0x420 build/default/production/_ext/365611741/system_services.o
 .text.SYS_RTCC_Initialize
                0x00000000       0xf4 build/default/production/_ext/365611741/system_services.o
 .text.SYS_RTCC_DateGet
                0x00000000       0x4c build/default/production/_ext/365611741/system_services.o
 .text.SYS_RTCC_TimeGet
                0x00000000       0x4c build/default/production/_ext/365611741/system_services.o
 .text.SYS_TICK_NsDelay
                0x00000000       0xa4 build/default/production/_ext/365611741/system_services.o
 .text.SYS_INT_SourceDisable
                0x00000000       0x5c build/default/production/_ext/365611741/system_services.o
 .text.SYS_INT_SourceEnable
                0x00000000       0x58 build/default/production/_ext/365611741/system_services.o
 .text.SYS_INT_SourceRestore
                0x00000000       0x70 build/default/production/_ext/365611741/system_services.o
 .text.SYS_INT_SourceStatusClear
                0x00000000       0x54 build/default/production/_ext/365611741/system_services.o
 .text.SYS_INT_PrioritySet
                0x00000000       0x5c build/default/production/_ext/365611741/system_services.o
 .text.SYS_INT_SubprioritySet
                0x00000000       0x5c build/default/production/_ext/365611741/system_services.o
 .text.SYS_INT_DynamicRegister
                0x00000000       0xbc build/default/production/_ext/365611741/system_services.o
 .text          0x00000000        0x0 build/default/production/_ext/365611741/system_debug.o
 .data          0x00000000        0x0 build/default/production/_ext/365611741/system_debug.o
 .bss           0x00000000        0x0 build/default/production/_ext/365611741/system_debug.o
 .reginfo       0x00000000       0x18 build/default/production/_ext/365611741/system_debug.o
 .pdr           0x00000000      0x2c0 build/default/production/_ext/365611741/system_debug.o
 .text.__sys_assert
                0x00000000       0x3c build/default/production/_ext/365611741/system_debug.o
 .text._SYS_PRINT
                0x00000000       0xcc build/default/production/_ext/365611741/system_debug.o
 .text._SYS_CONSOLE_GETLINE
                0x00000000       0x58 build/default/production/_ext/365611741/system_debug.o
 .text.SYS_OUT_GET_LCD_MESSAGE
                0x00000000       0x28 build/default/production/_ext/365611741/system_debug.o
 .text          0x00000000        0x0 build/default/production/_ext/365611741/system_random.o
 .data          0x00000000        0x0 build/default/production/_ext/365611741/system_random.o
 .reginfo       0x00000000       0x18 build/default/production/_ext/365611741/system_random.o
 .pdr           0x00000000       0xa0 build/default/production/_ext/365611741/system_random.o
 .text.SYS_RANDOM_GET
                0x00000000       0x84 build/default/production/_ext/365611741/system_random.o
 .text._SYS_RANDOM_DE_INIT
                0x00000000       0x20 build/default/production/_ext/365611741/system_random.o
 .text          0x00000000        0x0 build/default/production/_ext/365611741/system_command.o
 .data          0x00000000        0x0 build/default/production/_ext/365611741/system_command.o
 .reginfo       0x00000000       0x18 build/default/production/_ext/365611741/system_command.o
 .pdr           0x00000000      0x2a0 build/default/production/_ext/365611741/system_command.o
 .text._SYS_COMMAND_ADDGRP
                0x00000000      0x1b4 build/default/production/_ext/365611741/system_command.o
 .text          0x00000000        0x0 build/default/production/_ext/365611741/system_userio.o
 .data          0x00000000        0x0 build/default/production/_ext/365611741/system_userio.o
 .reginfo       0x00000000       0x18 build/default/production/_ext/365611741/system_userio.o
 .pdr           0x00000000      0x100 build/default/production/_ext/365611741/system_userio.o
 .text.SYS_USERIO_ButtonGetBitMap
                0x00000000       0x68 build/default/production/_ext/365611741/system_userio.o
 .text.SYS_USERIO_ButtonGet
                0x00000000      0x140 build/default/production/_ext/365611741/system_userio.o
 .text.SYS_USERIO_ButtonsTest
                0x00000000       0xa8 build/default/production/_ext/365611741/system_userio.o
 .text          0x00000000        0x0 build/default/production/_ext/97638081/sys_fs.o
 .data          0x00000000        0x0 build/default/production/_ext/97638081/sys_fs.o
 .reginfo       0x00000000       0x18 build/default/production/_ext/97638081/sys_fs.o
 .pdr           0x00000000      0x8a0 build/default/production/_ext/97638081/sys_fs.o
 .text.SYS_FS_mpfs2fs_Deinit
                0x00000000       0x30 build/default/production/_ext/97638081/sys_fs.o
 .text.SYS_FS_mpfs2fs_Open
                0x00000000       0x3c build/default/production/_ext/97638081/sys_fs.o
 .text.SYS_FS_mpfs2fs_OpenID
                0x00000000       0x40 build/default/production/_ext/97638081/sys_fs.o
 .text.SYS_FS_mpfs2fs_Close
                0x00000000       0x40 build/default/production/_ext/97638081/sys_fs.o
 .text.SYS_FS_mpfs2fs_Get
                0x00000000       0x48 build/default/production/_ext/97638081/sys_fs.o
 .text.SYS_FS_mpfs2fs_ArrayGet
                0x00000000       0x50 build/default/production/_ext/97638081/sys_fs.o
 .text.SYS_FS_mpfs2fs_LongGet
                0x00000000       0x48 build/default/production/_ext/97638081/sys_fs.o
 .text.SYS_FS_mpfs2fs_Seek
                0x00000000       0x50 build/default/production/_ext/97638081/sys_fs.o
 .text.SYS_FS_mpfs2fs_Format
                0x00000000       0x30 build/default/production/_ext/97638081/sys_fs.o
 .text.SYS_FS_mpfs2fs_ArrayPut
                0x00000000       0x50 build/default/production/_ext/97638081/sys_fs.o
 .text.SYS_FS_mpfs2fs_PutEnd
                0x00000000       0x50 build/default/production/_ext/97638081/sys_fs.o
 .text.SYS_FS_mpfs2fs_TimestampGet
                0x00000000       0x40 build/default/production/_ext/97638081/sys_fs.o
 .text.SYS_FS_mpfs2fs_MicrotimeGet
                0x00000000       0x40 build/default/production/_ext/97638081/sys_fs.o
 .text.SYS_FS_mpfs2fs_FlagsGet
                0x00000000       0x40 build/default/production/_ext/97638081/sys_fs.o
 .text.SYS_FS_mpfs2fs_SizeGet
                0x00000000       0x40 build/default/production/_ext/97638081/sys_fs.o
 .text.SYS_FS_mpfs2fs_BytesRemGet
                0x00000000       0x40 build/default/production/_ext/97638081/sys_fs.o
 .text.SYS_FS_mpfs2fs_StartAddrGet
                0x00000000       0x40 build/default/production/_ext/97638081/sys_fs.o
 .text.SYS_FS_mpfs2fs_EndAddrGet
                0x00000000       0x40 build/default/production/_ext/97638081/sys_fs.o
 .text.SYS_FS_mpfs2fs_FilenameGet
                0x00000000       0x58 build/default/production/_ext/97638081/sys_fs.o
 .text.SYS_FS_mpfs2fs_PositionGet
                0x00000000       0x40 build/default/production/_ext/97638081/sys_fs.o
 .text.SYS_FS_mpfs2fs_IDGet
                0x00000000       0x40 build/default/production/_ext/97638081/sys_fs.o
 .text.SYS_FS_IsLegalFileString
                0x00000000      0x144 build/default/production/_ext/97638081/sys_fs.o
 .text.SYS_FS_IsLegalFileChar
                0x00000000       0x7c build/default/production/_ext/97638081/sys_fs.o
 .text.SYS_FS_ExtractFilename
                0x00000000      0x104 build/default/production/_ext/97638081/sys_fs.o
 .text.SYS_FS_IsBadString
                0x00000000       0xd8 build/default/production/_ext/97638081/sys_fs.o
 .text.SYS_FS_ExtractPathname
                0x00000000      0x198 build/default/production/_ext/97638081/sys_fs.o
 .text.SYS_FS_createMBR
                0x00000000       0x64 build/default/production/_ext/97638081/sys_fs.o
 .text.SYS_FS_format
                0x00000000       0x6c build/default/production/_ext/97638081/sys_fs.o
 .text.SYS_FS_open
                0x00000000      0x374 build/default/production/_ext/97638081/sys_fs.o
 .text.SYS_FS_close
                0x00000000      0x198 build/default/production/_ext/97638081/sys_fs.o
 .text.SYS_FS_Loc2SysDesc
                0x00000000       0x74 build/default/production/_ext/97638081/sys_fs.o
 .text.SYS_FS_Sys2LocDesc
                0x00000000       0x90 build/default/production/_ext/97638081/sys_fs.o
 .text.SYS_FS_NextDescriptorGet
                0x00000000      0x150 build/default/production/_ext/97638081/sys_fs.o
 .text.SYS_FS_DescriptorIndexGet
                0x00000000      0x158 build/default/production/_ext/97638081/sys_fs.o
 .text.SYS_FS_DescriptorNameGet
                0x00000000      0x150 build/default/production/_ext/97638081/sys_fs.o
 .text.SYS_FS_fsize
                0x00000000       0xe0 build/default/production/_ext/97638081/sys_fs.o
 .text.SYS_FS_ftell
                0x00000000       0xe0 build/default/production/_ext/97638081/sys_fs.o
 .text.SYS_FS_fgetname
                0x00000000      0x11c build/default/production/_ext/97638081/sys_fs.o
 .text.SYS_FS_fstat
                0x00000000      0x114 build/default/production/_ext/97638081/sys_fs.o
 .text.SYS_FS_read
                0x00000000      0x18c build/default/production/_ext/97638081/sys_fs.o
 .text.SYS_FS_write
                0x00000000      0x134 build/default/production/_ext/97638081/sys_fs.o
 .text.SYS_FS_FSFromMountName
                0x00000000       0xc8 build/default/production/_ext/97638081/sys_fs.o
 .text.SYS_FS_FileTypeGet
                0x00000000       0xcc build/default/production/_ext/97638081/sys_fs.o
 .text.FS_MountRecGet
                0x00000000       0xd4 build/default/production/_ext/97638081/sys_fs.o
 .text.SYS_FS_fclose
                0x00000000       0x28 build/default/production/_ext/97638081/sys_fs.o
 .text.SYS_FS_fflush
                0x00000000       0x28 build/default/production/_ext/97638081/sys_fs.o
 .text.SYS_FS_fread
                0x00000000       0x34 build/default/production/_ext/97638081/sys_fs.o
 .text.SYS_FS_fwrite
                0x00000000       0x34 build/default/production/_ext/97638081/sys_fs.o
 .text.SYS_FS_remove
                0x00000000       0x28 build/default/production/_ext/97638081/sys_fs.o
 .text.SYS_FS_deinitialize
                0x00000000      0x128 build/default/production/_ext/97638081/sys_fs.o
 .text.SYS_FS_reinitialize
                0x00000000       0x58 build/default/production/_ext/97638081/sys_fs.o
 .text.SYS_FS_mkdir
                0x00000000       0xe0 build/default/production/_ext/97638081/sys_fs.o
 .text.SYS_FS_rmdir
                0x00000000       0xe8 build/default/production/_ext/97638081/sys_fs.o
 .text.SYS_FS_getcwd
                0x00000000       0x64 build/default/production/_ext/97638081/sys_fs.o
 .text.SYS_FS_lseek
                0x00000000      0x150 build/default/production/_ext/97638081/sys_fs.o
 .text.SYS_FS_unmount
                0x00000000       0x28 build/default/production/_ext/97638081/sys_fs.o
 .text.SYS_FS_error
                0x00000000       0x24 build/default/production/_ext/97638081/sys_fs.o
 .text.SYS_FS_clearerror
                0x00000000       0x24 build/default/production/_ext/97638081/sys_fs.o
 .text          0x00000000        0x0 build/default/production/_ext/97638081/mpfs2.o
 .data          0x00000000        0x0 build/default/production/_ext/97638081/mpfs2.o
 .reginfo       0x00000000       0x18 build/default/production/_ext/97638081/mpfs2.o
 .pdr           0x00000000      0x300 build/default/production/_ext/97638081/mpfs2.o
 .text.MPFSFormat
                0x00000000       0xdc build/default/production/_ext/97638081/mpfs2.o
 .text.MPFSPutArray
                0x00000000       0x68 build/default/production/_ext/97638081/mpfs2.o
 .text.MPFSPutEnd
                0x00000000       0x94 build/default/production/_ext/97638081/mpfs2.o
 .text.MPFSGetTimestamp
                0x00000000       0xac build/default/production/_ext/97638081/mpfs2.o
 .text.MPFSGetMicrotime
                0x00000000       0xac build/default/production/_ext/97638081/mpfs2.o
 .text.MPFSGetBytesRem
                0x00000000       0x94 build/default/production/_ext/97638081/mpfs2.o
 .text          0x00000000        0x0 build/default/production/_ext/792872985/usart.o
 .data          0x00000000        0x0 build/default/production/_ext/792872985/usart.o
 .bss           0x00000000        0x0 build/default/production/_ext/792872985/usart.o
 .reginfo       0x00000000       0x18 build/default/production/_ext/792872985/usart.o
 .pdr           0x00000000       0xe0 build/default/production/_ext/792872985/usart.o
 .text          0x00000000        0x0 build/default/production/_ext/792872985/lcd.o
 .data          0x00000000        0x0 build/default/production/_ext/792872985/lcd.o
 .bss           0x00000000        0x0 build/default/production/_ext/792872985/lcd.o
 .reginfo       0x00000000       0x18 build/default/production/_ext/792872985/lcd.o
 .pdr           0x00000000       0xc0 build/default/production/_ext/792872985/lcd.o
 .text          0x00000000        0x0 build/default/production/_ext/792872985/drv_spi.o
 .data          0x00000000        0x0 build/default/production/_ext/792872985/drv_spi.o
 .bss           0x00000000        0x0 build/default/production/_ext/792872985/drv_spi.o
 .reginfo       0x00000000       0x18 build/default/production/_ext/792872985/drv_spi.o
 .pdr           0x00000000       0x60 build/default/production/_ext/792872985/drv_spi.o
 .text          0x00000000        0x0 build/default/production/_ext/792872985/db_appio.o
 .data          0x00000000        0x0 build/default/production/_ext/792872985/db_appio.o
 .bss           0x00000000        0x0 build/default/production/_ext/792872985/db_appio.o
 .reginfo       0x00000000       0x18 build/default/production/_ext/792872985/db_appio.o
 .pdr           0x00000000        0x0 build/default/production/_ext/792872985/db_appio.o
 .text          0x00000000        0x0 build/default/production/_ext/792872985/spi_ram.o
 .data          0x00000000        0x0 build/default/production/_ext/792872985/spi_ram.o
 .bss           0x00000000        0x0 build/default/production/_ext/792872985/spi_ram.o
 .reginfo       0x00000000       0x18 build/default/production/_ext/792872985/spi_ram.o
 .pdr           0x00000000        0x0 build/default/production/_ext/792872985/spi_ram.o
 .text          0x00000000        0x0 build/default/production/_ext/792872985/spi_eeprom.o
 .data          0x00000000        0x0 build/default/production/_ext/792872985/spi_eeprom.o
 .bss           0x00000000        0x0 build/default/production/_ext/792872985/spi_eeprom.o
 .reginfo       0x00000000       0x18 build/default/production/_ext/792872985/spi_eeprom.o
 .pdr           0x00000000      0x160 build/default/production/_ext/792872985/spi_eeprom.o
 .text.XEEBeginRead
                0x00000000       0x34 build/default/production/_ext/792872985/spi_eeprom.o
 .text.XEERead  0x00000000       0x8c build/default/production/_ext/792872985/spi_eeprom.o
 .text.XEEEndRead
                0x00000000       0x24 build/default/production/_ext/792872985/spi_eeprom.o
 .text          0x00000000        0x0 build/default/production/_ext/792872985/spi_flash.o
 .data          0x00000000        0x0 build/default/production/_ext/792872985/spi_flash.o
 .bss           0x00000000        0x0 build/default/production/_ext/792872985/spi_flash.o
 .reginfo       0x00000000       0x18 build/default/production/_ext/792872985/spi_flash.o
 .pdr           0x00000000        0x0 build/default/production/_ext/792872985/spi_flash.o
 .text          0x00000000        0x0 build/default/production/_ext/792872985/drv_media.o
 .data          0x00000000        0x0 build/default/production/_ext/792872985/drv_media.o
 .bss           0x00000000        0x0 build/default/production/_ext/792872985/drv_media.o
 .reginfo       0x00000000       0x18 build/default/production/_ext/792872985/drv_media.o
 .pdr           0x00000000      0x1e0 build/default/production/_ext/792872985/drv_media.o
 .text.DRV_MEDIA_Deinitialize
                0x00000000       0x34 build/default/production/_ext/792872985/drv_media.o
 .text.DRV_MEDIA_ClientSizeGet
                0x00000000       0x40 build/default/production/_ext/792872985/drv_media.o
 .text.DRV_MEDIA_ClientRangeSet
                0x00000000       0xfc build/default/production/_ext/792872985/drv_media.o
 .text.DRV_MEDIA_WriteByte
                0x00000000       0xec build/default/production/_ext/792872985/drv_media.o
 .text          0x00000000        0x0 build/default/production/_ext/427700826/tcpip_announce.o
 .data          0x00000000        0x0 build/default/production/_ext/427700826/tcpip_announce.o
 .bss           0x00000000        0x0 build/default/production/_ext/427700826/tcpip_announce.o
 .reginfo       0x00000000       0x18 build/default/production/_ext/427700826/tcpip_announce.o
 .pdr           0x00000000       0xe0 build/default/production/_ext/427700826/tcpip_announce.o
 .text          0x00000000        0x0 build/default/production/_ext/427700826/http2.o
 .data          0x00000000        0x0 build/default/production/_ext/427700826/http2.o
 .bss           0x00000000        0x0 build/default/production/_ext/427700826/http2.o
 .reginfo       0x00000000       0x18 build/default/production/_ext/427700826/http2.o
 .pdr           0x00000000      0x4a0 build/default/production/_ext/427700826/http2.o
 .text.HTTPCurConnectionCallbackPosGet
                0x00000000       0x34 build/default/production/_ext/427700826/http2.o
 .text.HTTPCurConnectionByteCountSet
                0x00000000       0x3c build/default/production/_ext/427700826/http2.o
 .text.HTTPCurConnectionIsAuthorizedGet
                0x00000000       0x34 build/default/production/_ext/427700826/http2.o
 .text.HTTPCurConnectionIsAuthorizedSet
                0x00000000       0x40 build/default/production/_ext/427700826/http2.o
 .text.HTTPCurConnectionUserDataSet
                0x00000000       0x3c build/default/production/_ext/427700826/http2.o
 .text.HTTPCurConnectionUserDataGet
                0x00000000       0x34 build/default/production/_ext/427700826/http2.o
 .text          0x00000000        0x0 build/default/production/_ext/427700826/arcfour.o
 .data          0x00000000        0x0 build/default/production/_ext/427700826/arcfour.o
 .bss           0x00000000        0x0 build/default/production/_ext/427700826/arcfour.o
 .reginfo       0x00000000       0x18 build/default/production/_ext/427700826/arcfour.o
 .pdr           0x00000000        0x0 build/default/production/_ext/427700826/arcfour.o
 .text          0x00000000        0x0 build/default/production/_ext/427700826/arp.o
 .data          0x00000000        0x0 build/default/production/_ext/427700826/arp.o
 .bss           0x00000000        0x0 build/default/production/_ext/427700826/arp.o
 .reginfo       0x00000000       0x18 build/default/production/_ext/427700826/arp.o
 .pdr           0x00000000      0x480 build/default/production/_ext/427700826/arp.o
 .text.ARPRegisterHandler
                0x00000000       0x9c build/default/production/_ext/427700826/arp.o
 .text.ARPDeRegisterHandler
                0x00000000       0x78 build/default/production/_ext/427700826/arp.o
 .text.ARPProbe
                0x00000000       0x5c build/default/production/_ext/427700826/arp.o
 .text.ARPEntrySet
                0x00000000      0x24c build/default/production/_ext/427700826/arp.o
 .text.ARPEntryGet
                0x00000000       0x7c build/default/production/_ext/427700826/arp.o
 .text.ARPEntryRemove
                0x00000000       0xd0 build/default/production/_ext/427700826/arp.o
 .text.ARPEntryRemoveAll
                0x00000000       0x90 build/default/production/_ext/427700826/arp.o
 .text.ARPEntryQuery
                0x00000000      0x1a8 build/default/production/_ext/427700826/arp.o
 .text.ARPCacheGetEntriesNo
                0x00000000      0x15c build/default/production/_ext/427700826/arp.o
 .text.ARPCacheSetThreshold
                0x00000000       0xcc build/default/production/_ext/427700826/arp.o
 .text          0x00000000        0x0 build/default/production/_ext/427700826/berkeley_api.o
 .data          0x00000000        0x0 build/default/production/_ext/427700826/berkeley_api.o
 .bss           0x00000000        0x0 build/default/production/_ext/427700826/berkeley_api.o
 .reginfo       0x00000000       0x18 build/default/production/_ext/427700826/berkeley_api.o
 .pdr           0x00000000        0x0 build/default/production/_ext/427700826/berkeley_api.o
 .text          0x00000000        0x0 build/default/production/_ext/427700826/dhcp.o
 .data          0x00000000        0x0 build/default/production/_ext/427700826/dhcp.o
 .bss           0x00000000        0x0 build/default/production/_ext/427700826/dhcp.o
 .reginfo       0x00000000       0x18 build/default/production/_ext/427700826/dhcp.o
 .pdr           0x00000000      0x260 build/default/production/_ext/427700826/dhcp.o
 .text.DHCPDisable
                0x00000000       0x8c build/default/production/_ext/427700826/dhcp.o
 .text.DHCPEnable
                0x00000000       0xd8 build/default/production/_ext/427700826/dhcp.o
 .text.DHCPIsServerDetected
                0x00000000       0x90 build/default/production/_ext/427700826/dhcp.o
 .text.DHCPSetRequestTimeout
                0x00000000       0x2c build/default/production/_ext/427700826/dhcp.o
 .text          0x00000000        0x0 build/default/production/_ext/427700826/dhcps.o
 .data          0x00000000        0x0 build/default/production/_ext/427700826/dhcps.o
 .bss           0x00000000        0x0 build/default/production/_ext/427700826/dhcps.o
 .reginfo       0x00000000       0x18 build/default/production/_ext/427700826/dhcps.o
 .pdr           0x00000000       0x60 build/default/production/_ext/427700826/dhcps.o
 .text.DHCPServerDisable
                0x00000000       0x28 build/default/production/_ext/427700826/dhcps.o
 .text.DHCPServerEnable
                0x00000000       0x28 build/default/production/_ext/427700826/dhcps.o
 .text.DHCPServerIsEnabled
                0x00000000       0x28 build/default/production/_ext/427700826/dhcps.o
 .text          0x00000000        0x0 build/default/production/_ext/427700826/dns.o
 .data          0x00000000        0x0 build/default/production/_ext/427700826/dns.o
 .bss           0x00000000        0x0 build/default/production/_ext/427700826/dns.o
 .reginfo       0x00000000       0x18 build/default/production/_ext/427700826/dns.o
 .pdr           0x00000000      0x160 build/default/production/_ext/427700826/dns.o
 .text          0x00000000        0x0 build/default/production/_ext/427700826/dnss.o
 .data          0x00000000        0x0 build/default/production/_ext/427700826/dnss.o
 .bss           0x00000000        0x0 build/default/production/_ext/427700826/dnss.o
 .reginfo       0x00000000       0x18 build/default/production/_ext/427700826/dnss.o
 .pdr           0x00000000        0x0 build/default/production/_ext/427700826/dnss.o
 .text          0x00000000        0x0 build/default/production/_ext/427700826/dyn_dns.o
 .data          0x00000000        0x0 build/default/production/_ext/427700826/dyn_dns.o
 .bss           0x00000000        0x0 build/default/production/_ext/427700826/dyn_dns.o
 .reginfo       0x00000000       0x18 build/default/production/_ext/427700826/dyn_dns.o
 .pdr           0x00000000        0x0 build/default/production/_ext/427700826/dyn_dns.o
 .text          0x00000000        0x0 build/default/production/_ext/427700826/enc28_mac.o
 .data          0x00000000        0x0 build/default/production/_ext/427700826/enc28_mac.o
 .bss           0x00000000        0x0 build/default/production/_ext/427700826/enc28_mac.o
 .reginfo       0x00000000       0x18 build/default/production/_ext/427700826/enc28_mac.o
 .pdr           0x00000000        0x0 build/default/production/_ext/427700826/enc28_mac.o
 .text          0x00000000        0x0 build/default/production/_ext/427700826/enc28j60.o
 .data          0x00000000        0x0 build/default/production/_ext/427700826/enc28j60.o
 .bss           0x00000000        0x0 build/default/production/_ext/427700826/enc28j60.o
 .reginfo       0x00000000       0x18 build/default/production/_ext/427700826/enc28j60.o
 .pdr           0x00000000        0x0 build/default/production/_ext/427700826/enc28j60.o
 .text          0x00000000        0x0 build/default/production/_ext/427700826/encs24j600.o
 .data          0x00000000        0x0 build/default/production/_ext/427700826/encs24j600.o
 .bss           0x00000000        0x0 build/default/production/_ext/427700826/encs24j600.o
 .reginfo       0x00000000       0x18 build/default/production/_ext/427700826/encs24j600.o
 .pdr           0x00000000      0x460 build/default/production/_ext/427700826/encs24j600.o
 .text.ENCX24J600_MACMemCopyAsync
                0x00000000      0x17c build/default/production/_ext/427700826/encs24j600.o
 .text.ENCX24J600_SetCLKOUT
                0x00000000       0x98 build/default/production/_ext/427700826/encs24j600.o
 .text.ENCX24J600_GetCLKOUT
                0x00000000       0x4c build/default/production/_ext/427700826/encs24j600.o
 .text          0x00000000        0x0 build/default/production/_ext/427700826/encx24_mac.o
 .data          0x00000000        0x0 build/default/production/_ext/427700826/encx24_mac.o
 .bss           0x00000000        0x0 build/default/production/_ext/427700826/encx24_mac.o
 .reginfo       0x00000000       0x18 build/default/production/_ext/427700826/encx24_mac.o
 .pdr           0x00000000      0x2c0 build/default/production/_ext/427700826/encx24_mac.o
 .text          0x00000000        0x0 build/default/production/_ext/427700826/eth_pic32_ext_phy.o
 .data          0x00000000        0x0 build/default/production/_ext/427700826/eth_pic32_ext_phy.o
 .bss           0x00000000        0x0 build/default/production/_ext/427700826/eth_pic32_ext_phy.o
 .reginfo       0x00000000       0x18 build/default/production/_ext/427700826/eth_pic32_ext_phy.o
 .pdr           0x00000000        0x0 build/default/production/_ext/427700826/eth_pic32_ext_phy.o
 .text          0x00000000        0x0 build/default/production/_ext/427700826/eth_pic32_ext_phy_dp83848.o
 .data          0x00000000        0x0 build/default/production/_ext/427700826/eth_pic32_ext_phy_dp83848.o
 .bss           0x00000000        0x0 build/default/production/_ext/427700826/eth_pic32_ext_phy_dp83848.o
 .reginfo       0x00000000       0x18 build/default/production/_ext/427700826/eth_pic32_ext_phy_dp83848.o
 .pdr           0x00000000        0x0 build/default/production/_ext/427700826/eth_pic32_ext_phy_dp83848.o
 .text          0x00000000        0x0 build/default/production/_ext/427700826/eth_pic32_int_mac.o
 .data          0x00000000        0x0 build/default/production/_ext/427700826/eth_pic32_int_mac.o
 .bss           0x00000000        0x0 build/default/production/_ext/427700826/eth_pic32_int_mac.o
 .reginfo       0x00000000       0x18 build/default/production/_ext/427700826/eth_pic32_int_mac.o
 .pdr           0x00000000        0x0 build/default/production/_ext/427700826/eth_pic32_int_mac.o
 .text          0x00000000        0x0 build/default/production/_ext/427700826/ftp.o
 .data          0x00000000        0x0 build/default/production/_ext/427700826/ftp.o
 .bss           0x00000000        0x0 build/default/production/_ext/427700826/ftp.o
 .reginfo       0x00000000       0x18 build/default/production/_ext/427700826/ftp.o
 .pdr           0x00000000        0x0 build/default/production/_ext/427700826/ftp.o
 .text          0x00000000        0x0 build/default/production/_ext/427700826/hash_fnv.o
 .data          0x00000000        0x0 build/default/production/_ext/427700826/hash_fnv.o
 .bss           0x00000000        0x0 build/default/production/_ext/427700826/hash_fnv.o
 .reginfo       0x00000000       0x18 build/default/production/_ext/427700826/hash_fnv.o
 .pdr           0x00000000       0x40 build/default/production/_ext/427700826/hash_fnv.o
 .text.fnv_32a_hash
                0x00000000       0xd0 build/default/production/_ext/427700826/hash_fnv.o
 .text          0x00000000        0x0 build/default/production/_ext/427700826/hash_tbl.o
 .data          0x00000000        0x0 build/default/production/_ext/427700826/hash_tbl.o
 .bss           0x00000000        0x0 build/default/production/_ext/427700826/hash_tbl.o
 .reginfo       0x00000000       0x18 build/default/production/_ext/427700826/hash_tbl.o
 .pdr           0x00000000      0x100 build/default/production/_ext/427700826/hash_tbl.o
 .text          0x00000000        0x0 build/default/production/_ext/427700826/icmp.o
 .data          0x00000000        0x0 build/default/production/_ext/427700826/icmp.o
 .bss           0x00000000        0x0 build/default/production/_ext/427700826/icmp.o
 .reginfo       0x00000000       0x18 build/default/production/_ext/427700826/icmp.o
 .pdr           0x00000000       0xe0 build/default/production/_ext/427700826/icmp.o
 .text.ICMPRegisterCallback
                0x00000000       0x28 build/default/production/_ext/427700826/icmp.o
 .text.ICMPDeRegisterCallback
                0x00000000       0x28 build/default/production/_ext/427700826/icmp.o
 .text          0x00000000        0x0 build/default/production/_ext/427700826/icmpv6.o
 .data          0x00000000        0x0 build/default/production/_ext/427700826/icmpv6.o
 .bss           0x00000000        0x0 build/default/production/_ext/427700826/icmpv6.o
 .reginfo       0x00000000       0x18 build/default/production/_ext/427700826/icmpv6.o
 .pdr           0x00000000        0x0 build/default/production/_ext/427700826/icmpv6.o
 .text          0x00000000        0x0 build/default/production/_ext/427700826/ipv4.o
 .data          0x00000000        0x0 build/default/production/_ext/427700826/ipv4.o
 .bss           0x00000000        0x0 build/default/production/_ext/427700826/ipv4.o
 .reginfo       0x00000000       0x18 build/default/production/_ext/427700826/ipv4.o
 .pdr           0x00000000      0x4e0 build/default/production/_ext/427700826/ipv4.o
 .text.TCPIP_IPV4_Put
                0x00000000       0x5c build/default/production/_ext/427700826/ipv4.o
 .text          0x00000000        0x0 build/default/production/_ext/427700826/ipv6.o
 .data          0x00000000        0x0 build/default/production/_ext/427700826/ipv6.o
 .bss           0x00000000        0x0 build/default/production/_ext/427700826/ipv6.o
 .reginfo       0x00000000       0x18 build/default/production/_ext/427700826/ipv6.o
 .pdr           0x00000000        0x0 build/default/production/_ext/427700826/ipv6.o
 .text          0x00000000        0x0 build/default/production/_ext/427700826/mac_events_pic32.o
 .data          0x00000000        0x0 build/default/production/_ext/427700826/mac_events_pic32.o
 .bss           0x00000000        0x0 build/default/production/_ext/427700826/mac_events_pic32.o
 .reginfo       0x00000000       0x18 build/default/production/_ext/427700826/mac_events_pic32.o
 .pdr           0x00000000        0x0 build/default/production/_ext/427700826/mac_events_pic32.o
 .text          0x00000000        0x0 build/default/production/_ext/427700826/nbns.o
 .data          0x00000000        0x0 build/default/production/_ext/427700826/nbns.o
 .bss           0x00000000        0x0 build/default/production/_ext/427700826/nbns.o
 .reginfo       0x00000000       0x18 build/default/production/_ext/427700826/nbns.o
 .pdr           0x00000000       0xa0 build/default/production/_ext/427700826/nbns.o
 .text          0x00000000        0x0 build/default/production/_ext/427700826/ndp.o
 .data          0x00000000        0x0 build/default/production/_ext/427700826/ndp.o
 .bss           0x00000000        0x0 build/default/production/_ext/427700826/ndp.o
 .reginfo       0x00000000       0x18 build/default/production/_ext/427700826/ndp.o
 .pdr           0x00000000        0x0 build/default/production/_ext/427700826/ndp.o
 .text          0x00000000        0x0 build/default/production/_ext/427700826/tcpip_reboot.o
 .data          0x00000000        0x0 build/default/production/_ext/427700826/tcpip_reboot.o
 .bss           0x00000000        0x0 build/default/production/_ext/427700826/tcpip_reboot.o
 .reginfo       0x00000000       0x18 build/default/production/_ext/427700826/tcpip_reboot.o
 .pdr           0x00000000        0x0 build/default/production/_ext/427700826/tcpip_reboot.o
 .text          0x00000000        0x0 build/default/production/_ext/427700826/rsa.o
 .data          0x00000000        0x0 build/default/production/_ext/427700826/rsa.o
 .bss           0x00000000        0x0 build/default/production/_ext/427700826/rsa.o
 .reginfo       0x00000000       0x18 build/default/production/_ext/427700826/rsa.o
 .pdr           0x00000000        0x0 build/default/production/_ext/427700826/rsa.o
 .text          0x00000000        0x0 build/default/production/_ext/427700826/smtp.o
 .data          0x00000000        0x0 build/default/production/_ext/427700826/smtp.o
 .bss           0x00000000        0x0 build/default/production/_ext/427700826/smtp.o
 .reginfo       0x00000000       0x18 build/default/production/_ext/427700826/smtp.o
 .pdr           0x00000000        0x0 build/default/production/_ext/427700826/smtp.o
 .text          0x00000000        0x0 build/default/production/_ext/427700826/snmp.o
 .data          0x00000000        0x0 build/default/production/_ext/427700826/snmp.o
 .bss           0x00000000        0x0 build/default/production/_ext/427700826/snmp.o
 .reginfo       0x00000000       0x18 build/default/production/_ext/427700826/snmp.o
 .pdr           0x00000000        0x0 build/default/production/_ext/427700826/snmp.o
 .text          0x00000000        0x0 build/default/production/_ext/427700826/snmpv3.o
 .data          0x00000000        0x0 build/default/production/_ext/427700826/snmpv3.o
 .bss           0x00000000        0x0 build/default/production/_ext/427700826/snmpv3.o
 .reginfo       0x00000000       0x18 build/default/production/_ext/427700826/snmpv3.o
 .pdr           0x00000000        0x0 build/default/production/_ext/427700826/snmpv3.o
 .text          0x00000000        0x0 build/default/production/_ext/427700826/snmpv3_usm.o
 .data          0x00000000        0x0 build/default/production/_ext/427700826/snmpv3_usm.o
 .bss           0x00000000        0x0 build/default/production/_ext/427700826/snmpv3_usm.o
 .reginfo       0x00000000       0x18 build/default/production/_ext/427700826/snmpv3_usm.o
 .pdr           0x00000000        0x0 build/default/production/_ext/427700826/snmpv3_usm.o
 .text          0x00000000        0x0 build/default/production/_ext/427700826/sntp.o
 .data          0x00000000        0x0 build/default/production/_ext/427700826/sntp.o
 .bss           0x00000000        0x0 build/default/production/_ext/427700826/sntp.o
 .reginfo       0x00000000       0x18 build/default/production/_ext/427700826/sntp.o
 .pdr           0x00000000        0x0 build/default/production/_ext/427700826/sntp.o
 .text          0x00000000        0x0 build/default/production/_ext/427700826/ssl.o
 .data          0x00000000        0x0 build/default/production/_ext/427700826/ssl.o
 .bss           0x00000000        0x0 build/default/production/_ext/427700826/ssl.o
 .reginfo       0x00000000       0x18 build/default/production/_ext/427700826/ssl.o
 .pdr           0x00000000        0x0 build/default/production/_ext/427700826/ssl.o
 .text          0x00000000        0x0 build/default/production/_ext/427700826/tcp.o
 .data          0x00000000        0x0 build/default/production/_ext/427700826/tcp.o
 .bss           0x00000000        0x0 build/default/production/_ext/427700826/tcp.o
 .reginfo       0x00000000       0x18 build/default/production/_ext/427700826/tcp.o
 .pdr           0x00000000      0x9c0 build/default/production/_ext/427700826/tcp.o
 .text.TCPSetConnectionMSS
                0x00000000       0x44 build/default/production/_ext/427700826/tcp.o
 .text.TCPAbort
                0x00000000       0x6c build/default/production/_ext/427700826/tcp.o
 .text.TCPGetSocketInfo
                0x00000000       0xfc build/default/production/_ext/427700826/tcp.o
 .text.TCPSocketsNo
                0x00000000       0x24 build/default/production/_ext/427700826/tcp.o
 .text.TCPGetTxFIFOFull
                0x00000000       0xa4 build/default/production/_ext/427700826/tcp.o
 .text.TCPPeekArray
                0x00000000      0x1ac build/default/production/_ext/427700826/tcp.o
 .text.TCPPeek  0x00000000       0x60 build/default/production/_ext/427700826/tcp.o
 .text.TCPSocketSetNet
                0x00000000       0x80 build/default/production/_ext/427700826/tcp.o
 .text.TCPBind  0x00000000      0x1c4 build/default/production/_ext/427700826/tcp.o
 .text.TCPRemoteBind
                0x00000000       0x9c build/default/production/_ext/427700826/tcp.o
 .text.TCPGetOptions
                0x00000000      0x1b8 build/default/production/_ext/427700826/tcp.o
 .text.TCPSetDestinationIPAddress
                0x00000000       0xc4 build/default/production/_ext/427700826/tcp.o
 .text.TCPSetSourceIPAddress
                0x00000000       0xc4 build/default/production/_ext/427700826/tcp.o
 .text          0x00000000        0x0 build/default/production/_ext/427700826/tcpip_heap_alloc.o
 .data          0x00000000        0x0 build/default/production/_ext/427700826/tcpip_heap_alloc.o
 .bss           0x00000000        0x0 build/default/production/_ext/427700826/tcpip_heap_alloc.o
 .reginfo       0x00000000       0x18 build/default/production/_ext/427700826/tcpip_heap_alloc.o
 .pdr           0x00000000      0x200 build/default/production/_ext/427700826/tcpip_heap_alloc.o
 .text.TCPIP_HEAP_Size
                0x00000000       0x60 build/default/production/_ext/427700826/tcpip_heap_alloc.o
 .text.TCPIP_HEAP_MaxSize
                0x00000000       0xb0 build/default/production/_ext/427700826/tcpip_heap_alloc.o
 .text.TCPIP_HEAP_LastError
                0x00000000       0x6c build/default/production/_ext/427700826/tcpip_heap_alloc.o
 .text.TCPIP_HEAP_SetNoMemHandler
                0x00000000       0x5c build/default/production/_ext/427700826/tcpip_heap_alloc.o
 .text.TCPIP_HEAP_TraceGetEntry
                0x00000000       0x30 build/default/production/_ext/427700826/tcpip_heap_alloc.o
 .text.TCPIP_HEAP_TraceGetEntriesNo
                0x00000000       0x30 build/default/production/_ext/427700826/tcpip_heap_alloc.o
 .text          0x00000000        0x0 build/default/production/_ext/427700826/tcpip_storage.o
 .data          0x00000000        0x0 build/default/production/_ext/427700826/tcpip_storage.o
 .bss           0x00000000        0x0 build/default/production/_ext/427700826/tcpip_storage.o
 .reginfo       0x00000000       0x18 build/default/production/_ext/427700826/tcpip_storage.o
 .pdr           0x00000000        0x0 build/default/production/_ext/427700826/tcpip_storage.o
 .text          0x00000000        0x0 build/default/production/_ext/427700826/telnet.o
 .data          0x00000000        0x0 build/default/production/_ext/427700826/telnet.o
 .bss           0x00000000        0x0 build/default/production/_ext/427700826/telnet.o
 .reginfo       0x00000000       0x18 build/default/production/_ext/427700826/telnet.o
 .pdr           0x00000000        0x0 build/default/production/_ext/427700826/telnet.o
 .text          0x00000000        0x0 build/default/production/_ext/427700826/tftpc.o
 .data          0x00000000        0x0 build/default/production/_ext/427700826/tftpc.o
 .bss           0x00000000        0x0 build/default/production/_ext/427700826/tftpc.o
 .reginfo       0x00000000       0x18 build/default/production/_ext/427700826/tftpc.o
 .pdr           0x00000000        0x0 build/default/production/_ext/427700826/tftpc.o
 .text          0x00000000        0x0 build/default/production/_ext/427700826/udp.o
 .data          0x00000000        0x0 build/default/production/_ext/427700826/udp.o
 .bss           0x00000000        0x0 build/default/production/_ext/427700826/udp.o
 .reginfo       0x00000000       0x18 build/default/production/_ext/427700826/udp.o
 .pdr           0x00000000      0x560 build/default/production/_ext/427700826/udp.o
 .text.UDPGetSocketInfo
                0x00000000      0x100 build/default/production/_ext/427700826/udp.o
 .text.UDPPutString
                0x00000000       0xa0 build/default/production/_ext/427700826/udp.o
 .text.UDPSocketGetNet
                0x00000000       0x68 build/default/production/_ext/427700826/udp.o
 .text.UDPGetOptions
                0x00000000       0xdc build/default/production/_ext/427700826/udp.o
 .text          0x00000000        0x0 build/default/production/_ext/427700826/tcpip_mac_object.o
 .data          0x00000000        0x0 build/default/production/_ext/427700826/tcpip_mac_object.o
 .bss           0x00000000        0x0 build/default/production/_ext/427700826/tcpip_mac_object.o
 .reginfo       0x00000000       0x18 build/default/production/_ext/427700826/tcpip_mac_object.o
 .pdr           0x00000000      0x260 build/default/production/_ext/427700826/tcpip_mac_object.o
 .text.MACGetReadPtrInRx
                0x00000000       0x44 build/default/production/_ext/427700826/tcpip_mac_object.o
 .text.MACSetBaseReadPtr
                0x00000000       0x4c build/default/production/_ext/427700826/tcpip_mac_object.o
 .text.MACSetRXHashTableEntry
                0x00000000       0x54 build/default/production/_ext/427700826/tcpip_mac_object.o
 .text.MACPowerMode
                0x00000000       0x4c build/default/production/_ext/427700826/tcpip_mac_object.o
 .text          0x00000000        0x0 build/default/production/_ext/427700826/tcpip_manager.o
 .data          0x00000000        0x0 build/default/production/_ext/427700826/tcpip_manager.o
 .bss           0x00000000        0x0 build/default/production/_ext/427700826/tcpip_manager.o
 .reginfo       0x00000000       0x18 build/default/production/_ext/427700826/tcpip_manager.o
 .pdr           0x00000000      0x960 build/default/production/_ext/427700826/tcpip_manager.o
 .text.TCPIP_STACK_NetUp
                0x00000000      0x1c0 build/default/production/_ext/427700826/tcpip_manager.o
 .text.TCPIP_STACK_NetDown
                0x00000000      0x134 build/default/production/_ext/427700826/tcpip_manager.o
 .text.TCPIP_STACK_SetDefaultNet
                0x00000000       0x70 build/default/production/_ext/427700826/tcpip_manager.o
 .text._TCPIPStackIpAddFromNet
                0x00000000       0xec build/default/production/_ext/427700826/tcpip_manager.o
 .text._TCPIPStackMacToNet
                0x00000000       0x88 build/default/production/_ext/427700826/tcpip_manager.o
 .text._TCPIPStackMacToNetIx
                0x00000000       0x88 build/default/production/_ext/427700826/tcpip_manager.o
 .text.TCPIP_STACK_NetIx
                0x00000000       0x48 build/default/production/_ext/427700826/tcpip_manager.o
 .text.TCPIP_STACK_SetNetAddress
                0x00000000       0x80 build/default/production/_ext/427700826/tcpip_manager.o
 .text.TCPIP_STACK_SetNetGatewayAddress
                0x00000000       0x5c build/default/production/_ext/427700826/tcpip_manager.o
 .text.TCPIP_STACK_SetNetPriDNSAddress
                0x00000000       0x5c build/default/production/_ext/427700826/tcpip_manager.o
 .text.TCPIP_STACK_SetNetSecondDNSAddress
                0x00000000       0x5c build/default/production/_ext/427700826/tcpip_manager.o
 .text.TCPIP_STACK_SetNetMacAddress
                0x00000000       0x7c build/default/production/_ext/427700826/tcpip_manager.o
 .text.TCPIP_STACK_SetNetBIOSName
                0x00000000       0x8c build/default/production/_ext/427700826/tcpip_manager.o
 .text.TCPIP_STACK_SetLocalMasksType
                0x00000000       0x98 build/default/production/_ext/427700826/tcpip_manager.o
 .text.TCPIP_STACK_SetLocalMasks
                0x00000000       0x70 build/default/production/_ext/427700826/tcpip_manager.o
 .text.TCPIP_STACK_NetMACId
                0x00000000       0x44 build/default/production/_ext/427700826/tcpip_manager.o
 .text.TCPIP_STACK_ModuleGetConfig
                0x00000000       0x54 build/default/production/_ext/427700826/tcpip_manager.o
 .text.TCPIP_STACK_NetConfigGet
                0x00000000      0x10c build/default/production/_ext/427700826/tcpip_manager.o
 .text.NetConfigStringToBuffer
                0x00000000       0xf0 build/default/production/_ext/427700826/tcpip_manager.o
 .text.TCPIP_STACK_NetConfigSet
                0x00000000      0x4d8 build/default/production/_ext/427700826/tcpip_manager.o
 .text.TCPIP_STACK_IsNetUp
                0x00000000       0x48 build/default/production/_ext/427700826/tcpip_manager.o
 .text.TCPIP_STACK_IsNetLinked
                0x00000000       0x48 build/default/production/_ext/427700826/tcpip_manager.o
 .text._TCPIPStackAddressServiceCanStart
                0x00000000       0x54 build/default/production/_ext/427700826/tcpip_manager.o
 .text._TCPIPStackIsAddressOfNet
                0x00000000       0x74 build/default/production/_ext/427700826/tcpip_manager.o
 .text._TCPIPStackIsNetBcastAddress
                0x00000000       0x90 build/default/production/_ext/427700826/tcpip_manager.o
 .text._TCPIPStackIsBcastAddress
                0x00000000       0xb0 build/default/production/_ext/427700826/tcpip_manager.o
 .text._TCPIPStackNetMacId
                0x00000000       0x44 build/default/production/_ext/427700826/tcpip_manager.o
 .text          0x00000000        0x0 build/default/production/_ext/427700826/tcpip_helpers.o
 .data          0x00000000        0x0 build/default/production/_ext/427700826/tcpip_helpers.o
 .bss           0x00000000        0x0 build/default/production/_ext/427700826/tcpip_helpers.o
 .reginfo       0x00000000       0x18 build/default/production/_ext/427700826/tcpip_helpers.o
 .pdr           0x00000000      0x340 build/default/production/_ext/427700826/tcpip_helpers.o
 .text.TCPIP_HELPER_IPAddressToString
                0x00000000       0xec build/default/production/_ext/427700826/tcpip_helpers.o
 .text.TCPIP_HELPER_MACAddressToString
                0x00000000       0xf4 build/default/production/_ext/427700826/tcpip_helpers.o
 .text.TCPIP_HELPER_PowerModeToString
                0x00000000       0x58 build/default/production/_ext/427700826/tcpip_helpers.o
 .text.TCPIP_Helper_CalcMACBufferIPChecksum
                0x00000000      0x150 build/default/production/_ext/427700826/tcpip_helpers.o
 .text.TCPIP_Helper_FindCommonPrefix
                0x00000000      0x110 build/default/production/_ext/427700826/tcpip_helpers.o
 .text.SingleListAddHead
                0x00000000       0x74 build/default/production/_ext/427700826/tcpip_helpers.o
 .text.SingleListAddMid
                0x00000000       0x5c build/default/production/_ext/427700826/tcpip_helpers.o
 .text.SingleListRemoveNext
                0x00000000       0xb0 build/default/production/_ext/427700826/tcpip_helpers.o
 .text.SingleListAppendList
                0x00000000       0x64 build/default/production/_ext/427700826/tcpip_helpers.o
 .text.DoubleListInit
                0x00000000       0x44 build/default/production/_ext/427700826/tcpip_helpers.o
 .text.DoubleListAddHead
                0x00000000       0xbc build/default/production/_ext/427700826/tcpip_helpers.o
 .text.DoubleListAddTail
                0x00000000       0xbc build/default/production/_ext/427700826/tcpip_helpers.o
 .text.DoubleListAddMid
                0x00000000       0x78 build/default/production/_ext/427700826/tcpip_helpers.o
 .text.DoubleListRemoveHead
                0x00000000       0xa8 build/default/production/_ext/427700826/tcpip_helpers.o
 .text.DoubleListRemoveTail
                0x00000000       0xa8 build/default/production/_ext/427700826/tcpip_helpers.o
 .text.DoubleListRemoveMid
                0x00000000       0x64 build/default/production/_ext/427700826/tcpip_helpers.o
 .text.DoubleListRemoveNode
                0x00000000       0x90 build/default/production/_ext/427700826/tcpip_helpers.o
 .text          0x00000000        0x0 build/default/production/_ext/427700826/tcpip_commands.o
 .data          0x00000000        0x0 build/default/production/_ext/427700826/tcpip_commands.o
 .bss           0x00000000        0x0 build/default/production/_ext/427700826/tcpip_commands.o
 .reginfo       0x00000000       0x18 build/default/production/_ext/427700826/tcpip_commands.o
 .pdr           0x00000000        0x0 build/default/production/_ext/427700826/tcpip_commands.o
 .text          0x00000000        0x0 build/default/production/_ext/427700826/iperf.o
 .data          0x00000000        0x0 build/default/production/_ext/427700826/iperf.o
 .bss           0x00000000        0x0 build/default/production/_ext/427700826/iperf.o
 .reginfo       0x00000000       0x18 build/default/production/_ext/427700826/iperf.o
 .pdr           0x00000000        0x0 build/default/production/_ext/427700826/iperf.o
 .data          0x00000000        0x0 build/default/production/_ext/427700826/tcpip_helper_c32.o
 .bss           0x00000000        0x0 build/default/production/_ext/427700826/tcpip_helper_c32.o
 .reginfo       0x00000000       0x18 build/default/production/_ext/427700826/tcpip_helper_c32.o
 .pdr           0x00000000       0x60 build/default/production/_ext/427700826/tcpip_helper_c32.o
 .text          0x00000000        0x0 build/default/production/_ext/427700826/tcpip_notify.o
 .data          0x00000000        0x0 build/default/production/_ext/427700826/tcpip_notify.o
 .bss           0x00000000        0x0 build/default/production/_ext/427700826/tcpip_notify.o
 .reginfo       0x00000000       0x18 build/default/production/_ext/427700826/tcpip_notify.o
 .pdr           0x00000000       0x60 build/default/production/_ext/427700826/tcpip_notify.o
 .text          0x00000000        0x0 build/default/production/_ext/427700826/zero_conf_helper.o
 .data          0x00000000        0x0 build/default/production/_ext/427700826/zero_conf_helper.o
 .bss           0x00000000        0x0 build/default/production/_ext/427700826/zero_conf_helper.o
 .reginfo       0x00000000       0x18 build/default/production/_ext/427700826/zero_conf_helper.o
 .pdr           0x00000000        0x0 build/default/production/_ext/427700826/zero_conf_helper.o
 .text          0x00000000        0x0 build/default/production/_ext/427700826/zero_conf_link_local.o
 .data          0x00000000        0x0 build/default/production/_ext/427700826/zero_conf_link_local.o
 .bss           0x00000000        0x0 build/default/production/_ext/427700826/zero_conf_link_local.o
 .reginfo       0x00000000       0x18 build/default/production/_ext/427700826/zero_conf_link_local.o
 .pdr           0x00000000       0x60 build/default/production/_ext/427700826/zero_conf_link_local.o
 .text.ZCLLDisable
                0x00000000       0x28 build/default/production/_ext/427700826/zero_conf_link_local.o
 .text.ZCLLIsEnabled
                0x00000000       0x28 build/default/production/_ext/427700826/zero_conf_link_local.o
 .text          0x00000000        0x0 build/default/production/_ext/427700826/zero_conf_multicast_dns.o
 .data          0x00000000        0x0 build/default/production/_ext/427700826/zero_conf_multicast_dns.o
 .bss           0x00000000        0x0 build/default/production/_ext/427700826/zero_conf_multicast_dns.o
 .reginfo       0x00000000       0x18 build/default/production/_ext/427700826/zero_conf_multicast_dns.o
 .pdr           0x00000000        0x0 build/default/production/_ext/427700826/zero_conf_multicast_dns.o
 .text          0x00000000        0x0 build/default/production/_ext/334706090/wf_tx_power.o
 .data          0x00000000        0x0 build/default/production/_ext/334706090/wf_tx_power.o
 .bss           0x00000000        0x0 build/default/production/_ext/334706090/wf_tx_power.o
 .reginfo       0x00000000       0x18 build/default/production/_ext/334706090/wf_tx_power.o
 .pdr           0x00000000        0x0 build/default/production/_ext/334706090/wf_tx_power.o
 .text          0x00000000        0x0 build/default/production/_ext/334706090/wf_connect.o
 .data          0x00000000        0x0 build/default/production/_ext/334706090/wf_connect.o
 .bss           0x00000000        0x0 build/default/production/_ext/334706090/wf_connect.o
 .reginfo       0x00000000       0x18 build/default/production/_ext/334706090/wf_connect.o
 .pdr           0x00000000        0x0 build/default/production/_ext/334706090/wf_connect.o
 .text          0x00000000        0x0 build/default/production/_ext/334706090/wf_connection_algorithm.o
 .data          0x00000000        0x0 build/default/production/_ext/334706090/wf_connection_algorithm.o
 .bss           0x00000000        0x0 build/default/production/_ext/334706090/wf_connection_algorithm.o
 .reginfo       0x00000000       0x18 build/default/production/_ext/334706090/wf_connection_algorithm.o
 .pdr           0x00000000        0x0 build/default/production/_ext/334706090/wf_connection_algorithm.o
 .text          0x00000000        0x0 build/default/production/_ext/334706090/wf_connection_manager.o
 .data          0x00000000        0x0 build/default/production/_ext/334706090/wf_connection_manager.o
 .bss           0x00000000        0x0 build/default/production/_ext/334706090/wf_connection_manager.o
 .reginfo       0x00000000       0x18 build/default/production/_ext/334706090/wf_connection_manager.o
 .pdr           0x00000000        0x0 build/default/production/_ext/334706090/wf_connection_manager.o
 .text          0x00000000        0x0 build/default/production/_ext/334706090/wf_connection_profile.o
 .data          0x00000000        0x0 build/default/production/_ext/334706090/wf_connection_profile.o
 .bss           0x00000000        0x0 build/default/production/_ext/334706090/wf_connection_profile.o
 .reginfo       0x00000000       0x18 build/default/production/_ext/334706090/wf_connection_profile.o
 .pdr           0x00000000        0x0 build/default/production/_ext/334706090/wf_connection_profile.o
 .text          0x00000000        0x0 build/default/production/_ext/334706090/wf_easy_config.o
 .data          0x00000000        0x0 build/default/production/_ext/334706090/wf_easy_config.o
 .bss           0x00000000        0x0 build/default/production/_ext/334706090/wf_easy_config.o
 .reginfo       0x00000000       0x18 build/default/production/_ext/334706090/wf_easy_config.o
 .pdr           0x00000000        0x0 build/default/production/_ext/334706090/wf_easy_config.o
 .text          0x00000000        0x0 build/default/production/_ext/334706090/wf_eint.o
 .data          0x00000000        0x0 build/default/production/_ext/334706090/wf_eint.o
 .bss           0x00000000        0x0 build/default/production/_ext/334706090/wf_eint.o
 .reginfo       0x00000000       0x18 build/default/production/_ext/334706090/wf_eint.o
 .pdr           0x00000000       0x20 build/default/production/_ext/334706090/wf_eint.o
 .text.MCHP_Eint_EmptyFunc
                0x00000000       0x20 build/default/production/_ext/334706090/wf_eint.o
 .text          0x00000000        0x0 build/default/production/_ext/334706090/wf_event_handler.o
 .data          0x00000000        0x0 build/default/production/_ext/334706090/wf_event_handler.o
 .bss           0x00000000        0x0 build/default/production/_ext/334706090/wf_event_handler.o
 .reginfo       0x00000000       0x18 build/default/production/_ext/334706090/wf_event_handler.o
 .pdr           0x00000000        0x0 build/default/production/_ext/334706090/wf_event_handler.o
 .text          0x00000000        0x0 build/default/production/_ext/334706090/wf_init.o
 .data          0x00000000        0x0 build/default/production/_ext/334706090/wf_init.o
 .bss           0x00000000        0x0 build/default/production/_ext/334706090/wf_init.o
 .reginfo       0x00000000       0x18 build/default/production/_ext/334706090/wf_init.o
 .pdr           0x00000000        0x0 build/default/production/_ext/334706090/wf_init.o
 .text          0x00000000        0x0 build/default/production/_ext/334706090/wf_power_save.o
 .data          0x00000000        0x0 build/default/production/_ext/334706090/wf_power_save.o
 .bss           0x00000000        0x0 build/default/production/_ext/334706090/wf_power_save.o
 .reginfo       0x00000000       0x18 build/default/production/_ext/334706090/wf_power_save.o
 .pdr           0x00000000        0x0 build/default/production/_ext/334706090/wf_power_save.o
 .text          0x00000000        0x0 build/default/production/_ext/334706090/wf_scan.o
 .data          0x00000000        0x0 build/default/production/_ext/334706090/wf_scan.o
 .bss           0x00000000        0x0 build/default/production/_ext/334706090/wf_scan.o
 .reginfo       0x00000000       0x18 build/default/production/_ext/334706090/wf_scan.o
 .pdr           0x00000000        0x0 build/default/production/_ext/334706090/wf_scan.o
 .text          0x00000000        0x0 build/default/production/_ext/334706090/wf_spi.o
 .data          0x00000000        0x0 build/default/production/_ext/334706090/wf_spi.o
 .bss           0x00000000        0x0 build/default/production/_ext/334706090/wf_spi.o
 .reginfo       0x00000000       0x18 build/default/production/_ext/334706090/wf_spi.o
 .pdr           0x00000000       0x20 build/default/production/_ext/334706090/wf_spi.o
 .text.MCHP_Spi_EmptyFunc
                0x00000000       0x20 build/default/production/_ext/334706090/wf_spi.o
 .text          0x00000000        0x0 build/default/production/_ext/334706090/mrf24w_mac_pic32.o
 .data          0x00000000        0x0 build/default/production/_ext/334706090/mrf24w_mac_pic32.o
 .bss           0x00000000        0x0 build/default/production/_ext/334706090/mrf24w_mac_pic32.o
 .reginfo       0x00000000       0x18 build/default/production/_ext/334706090/mrf24w_mac_pic32.o
 .pdr           0x00000000        0x0 build/default/production/_ext/334706090/mrf24w_mac_pic32.o
 .text          0x00000000        0x0 build/default/production/_ext/334706090/mrf24w_events.o
 .data          0x00000000        0x0 build/default/production/_ext/334706090/mrf24w_events.o
 .bss           0x00000000        0x0 build/default/production/_ext/334706090/mrf24w_events.o
 .reginfo       0x00000000       0x18 build/default/production/_ext/334706090/mrf24w_events.o
 .pdr           0x00000000        0x0 build/default/production/_ext/334706090/mrf24w_events.o
 .text          0x00000000        0x0 build/default/production/_ext/334706090/wf_driver_com_24g.o
 .data          0x00000000        0x0 build/default/production/_ext/334706090/wf_driver_com_24g.o
 .bss           0x00000000        0x0 build/default/production/_ext/334706090/wf_driver_com_24g.o
 .reginfo       0x00000000       0x18 build/default/production/_ext/334706090/wf_driver_com_24g.o
 .pdr           0x00000000        0x0 build/default/production/_ext/334706090/wf_driver_com_24g.o
 .text          0x00000000        0x0 build/default/production/_ext/334706090/wf_driver_raw_24g.o
 .data          0x00000000        0x0 build/default/production/_ext/334706090/wf_driver_raw_24g.o
 .bss           0x00000000        0x0 build/default/production/_ext/334706090/wf_driver_raw_24g.o
 .reginfo       0x00000000       0x18 build/default/production/_ext/334706090/wf_driver_raw_24g.o
 .pdr           0x00000000        0x0 build/default/production/_ext/334706090/wf_driver_raw_24g.o
 .text          0x00000000        0x0 build/default/production/_ext/334706090/wf_mac_24g.o
 .data          0x00000000        0x0 build/default/production/_ext/334706090/wf_mac_24g.o
 .bss           0x00000000        0x0 build/default/production/_ext/334706090/wf_mac_24g.o
 .reginfo       0x00000000       0x18 build/default/production/_ext/334706090/wf_mac_24g.o
 .pdr           0x00000000        0x0 build/default/production/_ext/334706090/wf_mac_24g.o
 .text          0x00000000        0x0 build/default/production/_ext/334706090/wf_mgmt_msg_24g.o
 .data          0x00000000        0x0 build/default/production/_ext/334706090/wf_mgmt_msg_24g.o
 .bss           0x00000000        0x0 build/default/production/_ext/334706090/wf_mgmt_msg_24g.o
 .reginfo       0x00000000       0x18 build/default/production/_ext/334706090/wf_mgmt_msg_24g.o
 .pdr           0x00000000        0x0 build/default/production/_ext/334706090/wf_mgmt_msg_24g.o
 .text          0x00000000        0x0 build/default/production/_ext/334706090/wf_param_msg_24g.o
 .data          0x00000000        0x0 build/default/production/_ext/334706090/wf_param_msg_24g.o
 .bss           0x00000000        0x0 build/default/production/_ext/334706090/wf_param_msg_24g.o
 .reginfo       0x00000000       0x18 build/default/production/_ext/334706090/wf_param_msg_24g.o
 .pdr           0x00000000        0x0 build/default/production/_ext/334706090/wf_param_msg_24g.o
 .text          0x00000000        0x0 build/default/production/_ext/1472/main_demo.o
 .data          0x00000000        0x0 build/default/production/_ext/1472/main_demo.o
 .bss           0x00000000        0x0 build/default/production/_ext/1472/main_demo.o
 .reginfo       0x00000000       0x18 build/default/production/_ext/1472/main_demo.o
 .pdr           0x00000000       0x40 build/default/production/_ext/1472/main_demo.o
 .text          0x00000000        0x0 build/default/production/_ext/1472/custom_snmp_app.o
 .data          0x00000000        0x0 build/default/production/_ext/1472/custom_snmp_app.o
 .bss           0x00000000        0x0 build/default/production/_ext/1472/custom_snmp_app.o
 .reginfo       0x00000000       0x18 build/default/production/_ext/1472/custom_snmp_app.o
 .pdr           0x00000000        0x0 build/default/production/_ext/1472/custom_snmp_app.o
 .text          0x00000000        0x0 build/default/production/_ext/1472/custom_ssl_cert.o
 .data          0x00000000        0x0 build/default/production/_ext/1472/custom_ssl_cert.o
 .bss           0x00000000        0x0 build/default/production/_ext/1472/custom_ssl_cert.o
 .reginfo       0x00000000       0x18 build/default/production/_ext/1472/custom_ssl_cert.o
 .pdr           0x00000000        0x0 build/default/production/_ext/1472/custom_ssl_cert.o
 .text          0x00000000        0x0 build/default/production/_ext/1472/mpfs_img2.o
 .data          0x00000000        0x0 build/default/production/_ext/1472/mpfs_img2.o
 .bss           0x00000000        0x0 build/default/production/_ext/1472/mpfs_img2.o
 .reginfo       0x00000000       0x18 build/default/production/_ext/1472/mpfs_img2.o
 .pdr           0x00000000        0x0 build/default/production/_ext/1472/mpfs_img2.o
 .text          0x00000000        0x0 build/default/production/_ext/1472/wf_config.o
 .data          0x00000000        0x0 build/default/production/_ext/1472/wf_config.o
 .bss           0x00000000        0x0 build/default/production/_ext/1472/wf_config.o
 .reginfo       0x00000000       0x18 build/default/production/_ext/1472/wf_config.o
 .pdr           0x00000000        0x0 build/default/production/_ext/1472/wf_config.o
 .text          0x00000000        0x0 build/default/production/_ext/1472/custom_http_app.o
 .data          0x00000000        0x0 build/default/production/_ext/1472/custom_http_app.o
 .reginfo       0x00000000       0x18 build/default/production/_ext/1472/custom_http_app.o
 .pdr           0x00000000      0x500 build/default/production/_ext/1472/custom_http_app.o
 .text          0x00000000        0x0 build/default/production/_ext/1472/tcp6_demo_app.o
 .bss           0x00000000        0x0 build/default/production/_ext/1472/tcp6_demo_app.o
 .reginfo       0x00000000       0x18 build/default/production/_ext/1472/tcp6_demo_app.o
 .pdr           0x00000000       0x80 build/default/production/_ext/1472/tcp6_demo_app.o
 .text          0x00000000        0x0 c:/program files (x86)/microchip/xc32/v1.21/bin/../lib/gcc/pic32mx/4.5.2/../../../../pic32mx/lib/./proc/32MX795F512L\default_isr_vectors.o
 .data          0x00000000        0x0 c:/program files (x86)/microchip/xc32/v1.21/bin/../lib/gcc/pic32mx/4.5.2/../../../../pic32mx/lib/./proc/32MX795F512L\default_isr_vectors.o
 .bss           0x00000000        0x0 c:/program files (x86)/microchip/xc32/v1.21/bin/../lib/gcc/pic32mx/4.5.2/../../../../pic32mx/lib/./proc/32MX795F512L\default_isr_vectors.o
 .reginfo       0x00000000       0x18 c:/program files (x86)/microchip/xc32/v1.21/bin/../lib/gcc/pic32mx/4.5.2/../../../../pic32mx/lib/./proc/32MX795F512L\default_isr_vectors.o
 .pdr           0x00000000        0x0 c:/program files (x86)/microchip/xc32/v1.21/bin/../lib/gcc/pic32mx/4.5.2/../../../../pic32mx/lib/./proc/32MX795F512L\default_isr_vectors.o
 .discard       0x00000000      0x100 c:/program files (x86)/microchip/xc32/v1.21/bin/../lib/gcc/pic32mx/4.5.2/../../../../pic32mx/lib/./proc/32MX795F512L\default_isr_vectors.o
 .text          0x00000000        0x0 c:/program files (x86)/microchip/xc32/v1.21/bin/../lib/gcc/pic32mx/4.5.2/../../../../pic32mx/lib/./proc/32MX795F512L\processor.o
 .data          0x00000000        0x0 c:/program files (x86)/microchip/xc32/v1.21/bin/../lib/gcc/pic32mx/4.5.2/../../../../pic32mx/lib/./proc/32MX795F512L\processor.o
 .bss           0x00000000        0x0 c:/program files (x86)/microchip/xc32/v1.21/bin/../lib/gcc/pic32mx/4.5.2/../../../../pic32mx/lib/./proc/32MX795F512L\processor.o
 .reginfo       0x00000000       0x18 c:/program files (x86)/microchip/xc32/v1.21/bin/../lib/gcc/pic32mx/4.5.2/../../../../pic32mx/lib/./proc/32MX795F512L\processor.o
 .pdr           0x00000000        0x0 c:/program files (x86)/microchip/xc32/v1.21/bin/../lib/gcc/pic32mx/4.5.2/../../../../pic32mx/lib/./proc/32MX795F512L\processor.o
 .text          0x00000000        0x0 c:/program files (x86)/microchip/xc32/v1.21/bin/../lib/gcc/pic32mx/4.5.2/../../../../pic32mx/lib/size\libmchp_peripheral.a(open_core_timer_lib.o)
 .data          0x00000000        0x0 c:/program files (x86)/microchip/xc32/v1.21/bin/../lib/gcc/pic32mx/4.5.2/../../../../pic32mx/lib/size\libmchp_peripheral.a(open_core_timer_lib.o)
 .bss           0x00000000        0x0 c:/program files (x86)/microchip/xc32/v1.21/bin/../lib/gcc/pic32mx/4.5.2/../../../../pic32mx/lib/size\libmchp_peripheral.a(open_core_timer_lib.o)
 .reginfo       0x00000000       0x18 c:/program files (x86)/microchip/xc32/v1.21/bin/../lib/gcc/pic32mx/4.5.2/../../../../pic32mx/lib/size\libmchp_peripheral.a(open_core_timer_lib.o)
 .pdr           0x00000000       0x20 c:/program files (x86)/microchip/xc32/v1.21/bin/../lib/gcc/pic32mx/4.5.2/../../../../pic32mx/lib/size\libmchp_peripheral.a(open_core_timer_lib.o)
 .text          0x00000000        0x0 c:/program files (x86)/microchip/xc32/v1.21/bin/../lib/gcc/pic32mx/4.5.2/../../../../pic32mx/lib/size\libmchp_peripheral_32MX795F512L.a(soft_reset_lib.o)
 .data          0x00000000        0x0 c:/program files (x86)/microchip/xc32/v1.21/bin/../lib/gcc/pic32mx/4.5.2/../../../../pic32mx/lib/size\libmchp_peripheral_32MX795F512L.a(soft_reset_lib.o)
 .bss           0x00000000        0x0 c:/program files (x86)/microchip/xc32/v1.21/bin/../lib/gcc/pic32mx/4.5.2/../../../../pic32mx/lib/size\libmchp_peripheral_32MX795F512L.a(soft_reset_lib.o)
 .reginfo       0x00000000       0x18 c:/program files (x86)/microchip/xc32/v1.21/bin/../lib/gcc/pic32mx/4.5.2/../../../../pic32mx/lib/size\libmchp_peripheral_32MX795F512L.a(soft_reset_lib.o)
 .pdr           0x00000000       0x20 c:/program files (x86)/microchip/xc32/v1.21/bin/../lib/gcc/pic32mx/4.5.2/../../../../pic32mx/lib/size\libmchp_peripheral_32MX795F512L.a(soft_reset_lib.o)
 .text          0x00000000        0x0 c:/program files (x86)/microchip/xc32/v1.21/bin/../lib/gcc/pic32mx/4.5.2/../../../../pic32mx/lib/size\libmchp_peripheral_32MX795F512L.a(pcache.o)
 .data          0x00000000        0x0 c:/program files (x86)/microchip/xc32/v1.21/bin/../lib/gcc/pic32mx/4.5.2/../../../../pic32mx/lib/size\libmchp_peripheral_32MX795F512L.a(pcache.o)
 .bss           0x00000000        0x0 c:/program files (x86)/microchip/xc32/v1.21/bin/../lib/gcc/pic32mx/4.5.2/../../../../pic32mx/lib/size\libmchp_peripheral_32MX795F512L.a(pcache.o)
 .reginfo       0x00000000       0x18 c:/program files (x86)/microchip/xc32/v1.21/bin/../lib/gcc/pic32mx/4.5.2/../../../../pic32mx/lib/size\libmchp_peripheral_32MX795F512L.a(pcache.o)
 .pdr           0x00000000       0x40 c:/program files (x86)/microchip/xc32/v1.21/bin/../lib/gcc/pic32mx/4.5.2/../../../../pic32mx/lib/size\libmchp_peripheral_32MX795F512L.a(pcache.o)
 .text.CheKseg0CacheOff
                0x00000000       0x18 c:/program files (x86)/microchip/xc32/v1.21/bin/../lib/gcc/pic32mx/4.5.2/../../../../pic32mx/lib/size\libmchp_peripheral_32MX795F512L.a(pcache.o)
 .text          0x00000000        0x0 c:/program files (x86)/microchip/xc32/v1.21/bin/../lib/gcc/pic32mx/4.5.2/../../../../pic32mx/lib/size\libmchp_peripheral_32MX795F512L.a(int_disable_interrupts_lib.o)
 .data          0x00000000        0x0 c:/program files (x86)/microchip/xc32/v1.21/bin/../lib/gcc/pic32mx/4.5.2/../../../../pic32mx/lib/size\libmchp_peripheral_32MX795F512L.a(int_disable_interrupts_lib.o)
 .bss           0x00000000        0x0 c:/program files (x86)/microchip/xc32/v1.21/bin/../lib/gcc/pic32mx/4.5.2/../../../../pic32mx/lib/size\libmchp_peripheral_32MX795F512L.a(int_disable_interrupts_lib.o)
 .reginfo       0x00000000       0x18 c:/program files (x86)/microchip/xc32/v1.21/bin/../lib/gcc/pic32mx/4.5.2/../../../../pic32mx/lib/size\libmchp_peripheral_32MX795F512L.a(int_disable_interrupts_lib.o)
 .pdr           0x00000000       0x20 c:/program files (x86)/microchip/xc32/v1.21/bin/../lib/gcc/pic32mx/4.5.2/../../../../pic32mx/lib/size\libmchp_peripheral_32MX795F512L.a(int_disable_interrupts_lib.o)
 .text          0x00000000        0x0 c:/program files (x86)/microchip/xc32/v1.21/bin/../lib/gcc/pic32mx/4.5.2/../../../../pic32mx/lib/size\libmchp_peripheral_32MX795F512L.a(int_restore_interrupts_lib.o)
 .data          0x00000000        0x0 c:/program files (x86)/microchip/xc32/v1.21/bin/../lib/gcc/pic32mx/4.5.2/../../../../pic32mx/lib/size\libmchp_peripheral_32MX795F512L.a(int_restore_interrupts_lib.o)
 .bss           0x00000000        0x0 c:/program files (x86)/microchip/xc32/v1.21/bin/../lib/gcc/pic32mx/4.5.2/../../../../pic32mx/lib/size\libmchp_peripheral_32MX795F512L.a(int_restore_interrupts_lib.o)
 .reginfo       0x00000000       0x18 c:/program files (x86)/microchip/xc32/v1.21/bin/../lib/gcc/pic32mx/4.5.2/../../../../pic32mx/lib/size\libmchp_peripheral_32MX795F512L.a(int_restore_interrupts_lib.o)
 .pdr           0x00000000       0x20 c:/program files (x86)/microchip/xc32/v1.21/bin/../lib/gcc/pic32mx/4.5.2/../../../../pic32mx/lib/size\libmchp_peripheral_32MX795F512L.a(int_restore_interrupts_lib.o)
 .text          0x00000000        0x0 c:/program files (x86)/microchip/xc32/v1.21/bin/../lib/gcc/pic32mx/4.5.2/../../../../pic32mx/lib/size\libmchp_peripheral_32MX795F512L.a(int_enable_mv_int_lib.o)
 .data          0x00000000        0x0 c:/program files (x86)/microchip/xc32/v1.21/bin/../lib/gcc/pic32mx/4.5.2/../../../../pic32mx/lib/size\libmchp_peripheral_32MX795F512L.a(int_enable_mv_int_lib.o)
 .bss           0x00000000        0x0 c:/program files (x86)/microchip/xc32/v1.21/bin/../lib/gcc/pic32mx/4.5.2/../../../../pic32mx/lib/size\libmchp_peripheral_32MX795F512L.a(int_enable_mv_int_lib.o)
 .reginfo       0x00000000       0x18 c:/program files (x86)/microchip/xc32/v1.21/bin/../lib/gcc/pic32mx/4.5.2/../../../../pic32mx/lib/size\libmchp_peripheral_32MX795F512L.a(int_enable_mv_int_lib.o)
 .pdr           0x00000000       0x20 c:/program files (x86)/microchip/xc32/v1.21/bin/../lib/gcc/pic32mx/4.5.2/../../../../pic32mx/lib/size\libmchp_peripheral_32MX795F512L.a(int_enable_mv_int_lib.o)
 .text          0x00000000        0x0 c:/program files (x86)/microchip/xc32/v1.21/bin/../lib/gcc/pic32mx/4.5.2/../../../../pic32mx/lib/size\libmchp_peripheral_32MX795F512L.a(int_tbl_lib.o)
 .data          0x00000000        0x0 c:/program files (x86)/microchip/xc32/v1.21/bin/../lib/gcc/pic32mx/4.5.2/../../../../pic32mx/lib/size\libmchp_peripheral_32MX795F512L.a(int_tbl_lib.o)
 .bss           0x00000000        0x0 c:/program files (x86)/microchip/xc32/v1.21/bin/../lib/gcc/pic32mx/4.5.2/../../../../pic32mx/lib/size\libmchp_peripheral_32MX795F512L.a(int_tbl_lib.o)
 .reginfo       0x00000000       0x18 c:/program files (x86)/microchip/xc32/v1.21/bin/../lib/gcc/pic32mx/4.5.2/../../../../pic32mx/lib/size\libmchp_peripheral_32MX795F512L.a(int_tbl_lib.o)
 .pdr           0x00000000      0x120 c:/program files (x86)/microchip/xc32/v1.21/bin/../lib/gcc/pic32mx/4.5.2/../../../../pic32mx/lib/size\libmchp_peripheral_32MX795F512L.a(int_tbl_lib.o)
 .text.INTSetFlag
                0x00000000       0x28 c:/program files (x86)/microchip/xc32/v1.21/bin/../lib/gcc/pic32mx/4.5.2/../../../../pic32mx/lib/size\libmchp_peripheral_32MX795F512L.a(int_tbl_lib.o)
 .text.INTGetFlag
                0x00000000       0x28 c:/program files (x86)/microchip/xc32/v1.21/bin/../lib/gcc/pic32mx/4.5.2/../../../../pic32mx/lib/size\libmchp_peripheral_32MX795F512L.a(int_tbl_lib.o)
 .text.INTGetEnable
                0x00000000       0x28 c:/program files (x86)/microchip/xc32/v1.21/bin/../lib/gcc/pic32mx/4.5.2/../../../../pic32mx/lib/size\libmchp_peripheral_32MX795F512L.a(int_tbl_lib.o)
 .text.INTGetVectorPriority
                0x00000000       0x2c c:/program files (x86)/microchip/xc32/v1.21/bin/../lib/gcc/pic32mx/4.5.2/../../../../pic32mx/lib/size\libmchp_peripheral_32MX795F512L.a(int_tbl_lib.o)
 .text.INTGetVectorSubPriority
                0x00000000       0x2c c:/program files (x86)/microchip/xc32/v1.21/bin/../lib/gcc/pic32mx/4.5.2/../../../../pic32mx/lib/size\libmchp_peripheral_32MX795F512L.a(int_tbl_lib.o)
 .text          0x00000000        0x0 c:/program files (x86)/microchip/xc32/v1.21/bin/../lib/gcc/pic32mx/4.5.2/../../../../pic32mx/lib/size\libmchp_peripheral_32MX795F512L.a(rtcc_init_lib.o)
 .data          0x00000000        0x0 c:/program files (x86)/microchip/xc32/v1.21/bin/../lib/gcc/pic32mx/4.5.2/../../../../pic32mx/lib/size\libmchp_peripheral_32MX795F512L.a(rtcc_init_lib.o)
 .bss           0x00000000        0x0 c:/program files (x86)/microchip/xc32/v1.21/bin/../lib/gcc/pic32mx/4.5.2/../../../../pic32mx/lib/size\libmchp_peripheral_32MX795F512L.a(rtcc_init_lib.o)
 .reginfo       0x00000000       0x18 c:/program files (x86)/microchip/xc32/v1.21/bin/../lib/gcc/pic32mx/4.5.2/../../../../pic32mx/lib/size\libmchp_peripheral_32MX795F512L.a(rtcc_init_lib.o)
 .pdr           0x00000000       0x20 c:/program files (x86)/microchip/xc32/v1.21/bin/../lib/gcc/pic32mx/4.5.2/../../../../pic32mx/lib/size\libmchp_peripheral_32MX795F512L.a(rtcc_init_lib.o)
 .text.RtccInit
                0x00000000      0x170 c:/program files (x86)/microchip/xc32/v1.21/bin/../lib/gcc/pic32mx/4.5.2/../../../../pic32mx/lib/size\libmchp_peripheral_32MX795F512L.a(rtcc_init_lib.o)
 .text          0x00000000        0x0 c:/program files (x86)/microchip/xc32/v1.21/bin/../lib/gcc/pic32mx/4.5.2/../../../../pic32mx/lib/size\libmchp_peripheral_32MX795F512L.a(rtcc_open_lib.o)
 .data          0x00000000        0x0 c:/program files (x86)/microchip/xc32/v1.21/bin/../lib/gcc/pic32mx/4.5.2/../../../../pic32mx/lib/size\libmchp_peripheral_32MX795F512L.a(rtcc_open_lib.o)
 .bss           0x00000000        0x0 c:/program files (x86)/microchip/xc32/v1.21/bin/../lib/gcc/pic32mx/4.5.2/../../../../pic32mx/lib/size\libmchp_peripheral_32MX795F512L.a(rtcc_open_lib.o)
 .reginfo       0x00000000       0x18 c:/program files (x86)/microchip/xc32/v1.21/bin/../lib/gcc/pic32mx/4.5.2/../../../../pic32mx/lib/size\libmchp_peripheral_32MX795F512L.a(rtcc_open_lib.o)
 .pdr           0x00000000       0x20 c:/program files (x86)/microchip/xc32/v1.21/bin/../lib/gcc/pic32mx/4.5.2/../../../../pic32mx/lib/size\libmchp_peripheral_32MX795F512L.a(rtcc_open_lib.o)
 .text.RtccOpen
                0x00000000      0x1b0 c:/program files (x86)/microchip/xc32/v1.21/bin/../lib/gcc/pic32mx/4.5.2/../../../../pic32mx/lib/size\libmchp_peripheral_32MX795F512L.a(rtcc_open_lib.o)
 .text          0x00000000        0x0 c:/program files (x86)/microchip/xc32/v1.21/bin/../lib/gcc/pic32mx/4.5.2/../../../../pic32mx/lib/size\libmchp_peripheral_32MX795F512L.a(spi_chn_data_rdy_lib.o)
 .data          0x00000000        0x0 c:/program files (x86)/microchip/xc32/v1.21/bin/../lib/gcc/pic32mx/4.5.2/../../../../pic32mx/lib/size\libmchp_peripheral_32MX795F512L.a(spi_chn_data_rdy_lib.o)
 .bss           0x00000000        0x0 c:/program files (x86)/microchip/xc32/v1.21/bin/../lib/gcc/pic32mx/4.5.2/../../../../pic32mx/lib/size\libmchp_peripheral_32MX795F512L.a(spi_chn_data_rdy_lib.o)
 .reginfo       0x00000000       0x18 c:/program files (x86)/microchip/xc32/v1.21/bin/../lib/gcc/pic32mx/4.5.2/../../../../pic32mx/lib/size\libmchp_peripheral_32MX795F512L.a(spi_chn_data_rdy_lib.o)
 .pdr           0x00000000       0x20 c:/program files (x86)/microchip/xc32/v1.21/bin/../lib/gcc/pic32mx/4.5.2/../../../../pic32mx/lib/size\libmchp_peripheral_32MX795F512L.a(spi_chn_data_rdy_lib.o)
 .text          0x00000000        0x0 c:/program files (x86)/microchip/xc32/v1.21/bin/../lib/gcc/pic32mx/4.5.2/../../../../pic32mx/lib/size\libmchp_peripheral_32MX795F512L.a(spi_chn_getc_lib.o)
 .data          0x00000000        0x0 c:/program files (x86)/microchip/xc32/v1.21/bin/../lib/gcc/pic32mx/4.5.2/../../../../pic32mx/lib/size\libmchp_peripheral_32MX795F512L.a(spi_chn_getc_lib.o)
 .bss           0x00000000        0x0 c:/program files (x86)/microchip/xc32/v1.21/bin/../lib/gcc/pic32mx/4.5.2/../../../../pic32mx/lib/size\libmchp_peripheral_32MX795F512L.a(spi_chn_getc_lib.o)
 .reginfo       0x00000000       0x18 c:/program files (x86)/microchip/xc32/v1.21/bin/../lib/gcc/pic32mx/4.5.2/../../../../pic32mx/lib/size\libmchp_peripheral_32MX795F512L.a(spi_chn_getc_lib.o)
 .pdr           0x00000000       0x40 c:/program files (x86)/microchip/xc32/v1.21/bin/../lib/gcc/pic32mx/4.5.2/../../../../pic32mx/lib/size\libmchp_peripheral_32MX795F512L.a(spi_chn_getc_lib.o)
 .text.SpiChnGetC
                0x00000000       0x54 c:/program files (x86)/microchip/xc32/v1.21/bin/../lib/gcc/pic32mx/4.5.2/../../../../pic32mx/lib/size\libmchp_peripheral_32MX795F512L.a(spi_chn_getc_lib.o)
 .text          0x00000000        0x0 c:/program files (x86)/microchip/xc32/v1.21/bin/../lib/gcc/pic32mx/4.5.2/../../../../pic32mx/lib/size\libmchp_peripheral_32MX795F512L.a(spi_chn_open_lib.o)
 .data          0x00000000        0x0 c:/program files (x86)/microchip/xc32/v1.21/bin/../lib/gcc/pic32mx/4.5.2/../../../../pic32mx/lib/size\libmchp_peripheral_32MX795F512L.a(spi_chn_open_lib.o)
 .bss           0x00000000        0x0 c:/program files (x86)/microchip/xc32/v1.21/bin/../lib/gcc/pic32mx/4.5.2/../../../../pic32mx/lib/size\libmchp_peripheral_32MX795F512L.a(spi_chn_open_lib.o)
 .reginfo       0x00000000       0x18 c:/program files (x86)/microchip/xc32/v1.21/bin/../lib/gcc/pic32mx/4.5.2/../../../../pic32mx/lib/size\libmchp_peripheral_32MX795F512L.a(spi_chn_open_lib.o)
 .pdr           0x00000000       0x20 c:/program files (x86)/microchip/xc32/v1.21/bin/../lib/gcc/pic32mx/4.5.2/../../../../pic32mx/lib/size\libmchp_peripheral_32MX795F512L.a(spi_chn_open_lib.o)
 .text          0x00000000        0x0 c:/program files (x86)/microchip/xc32/v1.21/bin/../lib/gcc/pic32mx/4.5.2/../../../../pic32mx/lib/size\libmchp_peripheral_32MX795F512L.a(spi_chn_putc_lib.o)
 .data          0x00000000        0x0 c:/program files (x86)/microchip/xc32/v1.21/bin/../lib/gcc/pic32mx/4.5.2/../../../../pic32mx/lib/size\libmchp_peripheral_32MX795F512L.a(spi_chn_putc_lib.o)
 .bss           0x00000000        0x0 c:/program files (x86)/microchip/xc32/v1.21/bin/../lib/gcc/pic32mx/4.5.2/../../../../pic32mx/lib/size\libmchp_peripheral_32MX795F512L.a(spi_chn_putc_lib.o)
 .reginfo       0x00000000       0x18 c:/program files (x86)/microchip/xc32/v1.21/bin/../lib/gcc/pic32mx/4.5.2/../../../../pic32mx/lib/size\libmchp_peripheral_32MX795F512L.a(spi_chn_putc_lib.o)
 .pdr           0x00000000       0x60 c:/program files (x86)/microchip/xc32/v1.21/bin/../lib/gcc/pic32mx/4.5.2/../../../../pic32mx/lib/size\libmchp_peripheral_32MX795F512L.a(spi_chn_putc_lib.o)
 .text.SpiChnPutC
                0x00000000       0x54 c:/program files (x86)/microchip/xc32/v1.21/bin/../lib/gcc/pic32mx/4.5.2/../../../../pic32mx/lib/size\libmchp_peripheral_32MX795F512L.a(spi_chn_putc_lib.o)
 .text.SpiChnBuffer
                0x00000000       0x1c c:/program files (x86)/microchip/xc32/v1.21/bin/../lib/gcc/pic32mx/4.5.2/../../../../pic32mx/lib/size\libmchp_peripheral_32MX795F512L.a(spi_chn_putc_lib.o)
 .text          0x00000000        0x0 c:/program files (x86)/microchip/xc32/v1.21/bin/../lib/gcc/pic32mx/4.5.2/../../../../pic32mx/lib/size\libmchp_peripheral_32MX795F512L.a(spi_chn_tx_buff_empty_lib.o)
 .data          0x00000000        0x0 c:/program files (x86)/microchip/xc32/v1.21/bin/../lib/gcc/pic32mx/4.5.2/../../../../pic32mx/lib/size\libmchp_peripheral_32MX795F512L.a(spi_chn_tx_buff_empty_lib.o)
 .bss           0x00000000        0x0 c:/program files (x86)/microchip/xc32/v1.21/bin/../lib/gcc/pic32mx/4.5.2/../../../../pic32mx/lib/size\libmchp_peripheral_32MX795F512L.a(spi_chn_tx_buff_empty_lib.o)
 .reginfo       0x00000000       0x18 c:/program files (x86)/microchip/xc32/v1.21/bin/../lib/gcc/pic32mx/4.5.2/../../../../pic32mx/lib/size\libmchp_peripheral_32MX795F512L.a(spi_chn_tx_buff_empty_lib.o)
 .pdr           0x00000000       0x20 c:/program files (x86)/microchip/xc32/v1.21/bin/../lib/gcc/pic32mx/4.5.2/../../../../pic32mx/lib/size\libmchp_peripheral_32MX795F512L.a(spi_chn_tx_buff_empty_lib.o)
 .text          0x00000000        0x0 c:/program files (x86)/microchip/xc32/v1.21/bin/../lib/gcc/pic32mx/4.5.2/../../../../pic32mx/lib/size\libmchp_peripheral_32MX795F512L.a(spi_io_tbl_libp.o)
 .data          0x00000000        0x0 c:/program files (x86)/microchip/xc32/v1.21/bin/../lib/gcc/pic32mx/4.5.2/../../../../pic32mx/lib/size\libmchp_peripheral_32MX795F512L.a(spi_io_tbl_libp.o)
 .bss           0x00000000        0x0 c:/program files (x86)/microchip/xc32/v1.21/bin/../lib/gcc/pic32mx/4.5.2/../../../../pic32mx/lib/size\libmchp_peripheral_32MX795F512L.a(spi_io_tbl_libp.o)
 .reginfo       0x00000000       0x18 c:/program files (x86)/microchip/xc32/v1.21/bin/../lib/gcc/pic32mx/4.5.2/../../../../pic32mx/lib/size\libmchp_peripheral_32MX795F512L.a(spi_io_tbl_libp.o)
 .pdr           0x00000000        0x0 c:/program files (x86)/microchip/xc32/v1.21/bin/../lib/gcc/pic32mx/4.5.2/../../../../pic32mx/lib/size\libmchp_peripheral_32MX795F512L.a(spi_io_tbl_libp.o)
 .text          0x00000000        0x0 c:/program files (x86)/microchip/xc32/v1.21/bin/../lib/gcc/pic32mx/4.5.2/../../../../pic32mx/lib/size\libmchp_peripheral_32MX795F512L.a(spi_map_tbl_libp.o)
 .data          0x00000000        0x0 c:/program files (x86)/microchip/xc32/v1.21/bin/../lib/gcc/pic32mx/4.5.2/../../../../pic32mx/lib/size\libmchp_peripheral_32MX795F512L.a(spi_map_tbl_libp.o)
 .bss           0x00000000        0x0 c:/program files (x86)/microchip/xc32/v1.21/bin/../lib/gcc/pic32mx/4.5.2/../../../../pic32mx/lib/size\libmchp_peripheral_32MX795F512L.a(spi_map_tbl_libp.o)
 .reginfo       0x00000000       0x18 c:/program files (x86)/microchip/xc32/v1.21/bin/../lib/gcc/pic32mx/4.5.2/../../../../pic32mx/lib/size\libmchp_peripheral_32MX795F512L.a(spi_map_tbl_libp.o)
 .pdr           0x00000000        0x0 c:/program files (x86)/microchip/xc32/v1.21/bin/../lib/gcc/pic32mx/4.5.2/../../../../pic32mx/lib/size\libmchp_peripheral_32MX795F512L.a(spi_map_tbl_libp.o)
 .text          0x00000000        0x0 c:/program files (x86)/microchip/xc32/v1.21/bin/../lib/gcc/pic32mx/4.5.2/../../../../pic32mx/lib/size\libmchp_peripheral_32MX795F512L.a(port_set_pins_digital_in_lib.o)
 .data          0x00000000        0x0 c:/program files (x86)/microchip/xc32/v1.21/bin/../lib/gcc/pic32mx/4.5.2/../../../../pic32mx/lib/size\libmchp_peripheral_32MX795F512L.a(port_set_pins_digital_in_lib.o)
 .bss           0x00000000        0x0 c:/program files (x86)/microchip/xc32/v1.21/bin/../lib/gcc/pic32mx/4.5.2/../../../../pic32mx/lib/size\libmchp_peripheral_32MX795F512L.a(port_set_pins_digital_in_lib.o)
 .reginfo       0x00000000       0x18 c:/program files (x86)/microchip/xc32/v1.21/bin/../lib/gcc/pic32mx/4.5.2/../../../../pic32mx/lib/size\libmchp_peripheral_32MX795F512L.a(port_set_pins_digital_in_lib.o)
 .pdr           0x00000000       0x20 c:/program files (x86)/microchip/xc32/v1.21/bin/../lib/gcc/pic32mx/4.5.2/../../../../pic32mx/lib/size\libmchp_peripheral_32MX795F512L.a(port_set_pins_digital_in_lib.o)
 .text          0x00000000        0x0 c:/program files (x86)/microchip/xc32/v1.21/bin/../lib/gcc/pic32mx/4.5.2/../../../../pic32mx/lib/size\libmchp_peripheral_32MX795F512L.a(port_set_pins_digital_out_lib.o)
 .data          0x00000000        0x0 c:/program files (x86)/microchip/xc32/v1.21/bin/../lib/gcc/pic32mx/4.5.2/../../../../pic32mx/lib/size\libmchp_peripheral_32MX795F512L.a(port_set_pins_digital_out_lib.o)
 .bss           0x00000000        0x0 c:/program files (x86)/microchip/xc32/v1.21/bin/../lib/gcc/pic32mx/4.5.2/../../../../pic32mx/lib/size\libmchp_peripheral_32MX795F512L.a(port_set_pins_digital_out_lib.o)
 .reginfo       0x00000000       0x18 c:/program files (x86)/microchip/xc32/v1.21/bin/../lib/gcc/pic32mx/4.5.2/../../../../pic32mx/lib/size\libmchp_peripheral_32MX795F512L.a(port_set_pins_digital_out_lib.o)
 .pdr           0x00000000       0x20 c:/program files (x86)/microchip/xc32/v1.21/bin/../lib/gcc/pic32mx/4.5.2/../../../../pic32mx/lib/size\libmchp_peripheral_32MX795F512L.a(port_set_pins_digital_out_lib.o)
 .text          0x00000000        0x0 c:/program files (x86)/microchip/xc32/v1.21/bin/../lib/gcc/pic32mx/4.5.2/../../../../pic32mx/lib/size\libmchp_peripheral_32MX795F512L.a(_ports_tbl_libp.o)
 .data          0x00000000        0x0 c:/program files (x86)/microchip/xc32/v1.21/bin/../lib/gcc/pic32mx/4.5.2/../../../../pic32mx/lib/size\libmchp_peripheral_32MX795F512L.a(_ports_tbl_libp.o)
 .bss           0x00000000        0x0 c:/program files (x86)/microchip/xc32/v1.21/bin/../lib/gcc/pic32mx/4.5.2/../../../../pic32mx/lib/size\libmchp_peripheral_32MX795F512L.a(_ports_tbl_libp.o)
 .reginfo       0x00000000       0x18 c:/program files (x86)/microchip/xc32/v1.21/bin/../lib/gcc/pic32mx/4.5.2/../../../../pic32mx/lib/size\libmchp_peripheral_32MX795F512L.a(_ports_tbl_libp.o)
 .pdr           0x00000000        0x0 c:/program files (x86)/microchip/xc32/v1.21/bin/../lib/gcc/pic32mx/4.5.2/../../../../pic32mx/lib/size\libmchp_peripheral_32MX795F512L.a(_ports_tbl_libp.o)
 .text          0x00000000        0x0 c:/program files (x86)/microchip/xc32/v1.21/bin/../lib/gcc/pic32mx/4.5.2/../../../../pic32mx/lib/size\libmchp_peripheral_32MX795F512L.a(int_enable_interrupts_lib.o)
 .data          0x00000000        0x0 c:/program files (x86)/microchip/xc32/v1.21/bin/../lib/gcc/pic32mx/4.5.2/../../../../pic32mx/lib/size\libmchp_peripheral_32MX795F512L.a(int_enable_interrupts_lib.o)
 .bss           0x00000000        0x0 c:/program files (x86)/microchip/xc32/v1.21/bin/../lib/gcc/pic32mx/4.5.2/../../../../pic32mx/lib/size\libmchp_peripheral_32MX795F512L.a(int_enable_interrupts_lib.o)
 .reginfo       0x00000000       0x18 c:/program files (x86)/microchip/xc32/v1.21/bin/../lib/gcc/pic32mx/4.5.2/../../../../pic32mx/lib/size\libmchp_peripheral_32MX795F512L.a(int_enable_interrupts_lib.o)
 .pdr           0x00000000       0x20 c:/program files (x86)/microchip/xc32/v1.21/bin/../lib/gcc/pic32mx/4.5.2/../../../../pic32mx/lib/size\libmchp_peripheral_32MX795F512L.a(int_enable_interrupts_lib.o)
 .text          0x00000000        0x0 c:/program files (x86)/microchip/xc32/v1.21/bin/../lib/gcc/pic32mx/4.5.2/../../../../pic32mx/lib/size\libmchp_peripheral_32MX795F512L.a(_rtcc_wait_clock_off_lib.o)
 .data          0x00000000        0x0 c:/program files (x86)/microchip/xc32/v1.21/bin/../lib/gcc/pic32mx/4.5.2/../../../../pic32mx/lib/size\libmchp_peripheral_32MX795F512L.a(_rtcc_wait_clock_off_lib.o)
 .bss           0x00000000        0x0 c:/program files (x86)/microchip/xc32/v1.21/bin/../lib/gcc/pic32mx/4.5.2/../../../../pic32mx/lib/size\libmchp_peripheral_32MX795F512L.a(_rtcc_wait_clock_off_lib.o)
 .reginfo       0x00000000       0x18 c:/program files (x86)/microchip/xc32/v1.21/bin/../lib/gcc/pic32mx/4.5.2/../../../../pic32mx/lib/size\libmchp_peripheral_32MX795F512L.a(_rtcc_wait_clock_off_lib.o)
 .pdr           0x00000000       0x40 c:/program files (x86)/microchip/xc32/v1.21/bin/../lib/gcc/pic32mx/4.5.2/../../../../pic32mx/lib/size\libmchp_peripheral_32MX795F512L.a(_rtcc_wait_clock_off_lib.o)
 .text._RtccWaitClockOff
                0x00000000      0x104 c:/program files (x86)/microchip/xc32/v1.21/bin/../lib/gcc/pic32mx/4.5.2/../../../../pic32mx/lib/size\libmchp_peripheral_32MX795F512L.a(_rtcc_wait_clock_off_lib.o)
 .text._RtccSetClockWait
                0x00000000       0x14 c:/program files (x86)/microchip/xc32/v1.21/bin/../lib/gcc/pic32mx/4.5.2/../../../../pic32mx/lib/size\libmchp_peripheral_32MX795F512L.a(_rtcc_wait_clock_off_lib.o)
 .sdata         0x00000000        0x8 c:/program files (x86)/microchip/xc32/v1.21/bin/../lib/gcc/pic32mx/4.5.2/../../../../pic32mx/lib/size\libmchp_peripheral_32MX795F512L.a(_rtcc_wait_clock_off_lib.o)
 .text          0x00000000        0x0 c:/program files (x86)/microchip/xc32/v1.21/bin/../lib/gcc/pic32mx/4.5.2/../../../../pic32mx/lib/size\libmchp_peripheral_32MX795F512L.a(read_core_timer_lib.o)
 .data          0x00000000        0x0 c:/program files (x86)/microchip/xc32/v1.21/bin/../lib/gcc/pic32mx/4.5.2/../../../../pic32mx/lib/size\libmchp_peripheral_32MX795F512L.a(read_core_timer_lib.o)
 .bss           0x00000000        0x0 c:/program files (x86)/microchip/xc32/v1.21/bin/../lib/gcc/pic32mx/4.5.2/../../../../pic32mx/lib/size\libmchp_peripheral_32MX795F512L.a(read_core_timer_lib.o)
 .reginfo       0x00000000       0x18 c:/program files (x86)/microchip/xc32/v1.21/bin/../lib/gcc/pic32mx/4.5.2/../../../../pic32mx/lib/size\libmchp_peripheral_32MX795F512L.a(read_core_timer_lib.o)
 .pdr           0x00000000       0x20 c:/program files (x86)/microchip/xc32/v1.21/bin/../lib/gcc/pic32mx/4.5.2/../../../../pic32mx/lib/size\libmchp_peripheral_32MX795F512L.a(read_core_timer_lib.o)
 .text.ReadCoreTimer
                0x00000000        0x8 c:/program files (x86)/microchip/xc32/v1.21/bin/../lib/gcc/pic32mx/4.5.2/../../../../pic32mx/lib/size\libmchp_peripheral_32MX795F512L.a(read_core_timer_lib.o)
 .data          0x00000000        0x0 c:/program files (x86)/microchip/xc32/v1.21/bin/../lib/gcc/pic32mx/4.5.2/size\libgcc.a(_udivdi3.o)
 .bss           0x00000000        0x0 c:/program files (x86)/microchip/xc32/v1.21/bin/../lib/gcc/pic32mx/4.5.2/size\libgcc.a(_udivdi3.o)
 .reginfo       0x00000000       0x18 c:/program files (x86)/microchip/xc32/v1.21/bin/../lib/gcc/pic32mx/4.5.2/size\libgcc.a(_udivdi3.o)
 .pdr           0x00000000       0x20 c:/program files (x86)/microchip/xc32/v1.21/bin/../lib/gcc/pic32mx/4.5.2/size\libgcc.a(_udivdi3.o)
 .data          0x00000000        0x0 c:/program files (x86)/microchip/xc32/v1.21/bin/../lib/gcc/pic32mx/4.5.2/../../../../pic32mx/lib/size\libpic32.a(memcmp.o)
 .bss           0x00000000        0x0 c:/program files (x86)/microchip/xc32/v1.21/bin/../lib/gcc/pic32mx/4.5.2/../../../../pic32mx/lib/size\libpic32.a(memcmp.o)
 .reginfo       0x00000000       0x18 c:/program files (x86)/microchip/xc32/v1.21/bin/../lib/gcc/pic32mx/4.5.2/../../../../pic32mx/lib/size\libpic32.a(memcmp.o)
 .pdr           0x00000000       0x20 c:/program files (x86)/microchip/xc32/v1.21/bin/../lib/gcc/pic32mx/4.5.2/../../../../pic32mx/lib/size\libpic32.a(memcmp.o)
 .data          0x00000000        0x0 c:/program files (x86)/microchip/xc32/v1.21/bin/../lib/gcc/pic32mx/4.5.2/../../../../pic32mx/lib/size\libpic32.a(memcpy.o)
 .bss           0x00000000        0x0 c:/program files (x86)/microchip/xc32/v1.21/bin/../lib/gcc/pic32mx/4.5.2/../../../../pic32mx/lib/size\libpic32.a(memcpy.o)
 .reginfo       0x00000000       0x18 c:/program files (x86)/microchip/xc32/v1.21/bin/../lib/gcc/pic32mx/4.5.2/../../../../pic32mx/lib/size\libpic32.a(memcpy.o)
 .pdr           0x00000000       0x20 c:/program files (x86)/microchip/xc32/v1.21/bin/../lib/gcc/pic32mx/4.5.2/../../../../pic32mx/lib/size\libpic32.a(memcpy.o)
 .data          0x00000000        0x0 c:/program files (x86)/microchip/xc32/v1.21/bin/../lib/gcc/pic32mx/4.5.2/../../../../pic32mx/lib/size\libpic32.a(memset.o)
 .bss           0x00000000        0x0 c:/program files (x86)/microchip/xc32/v1.21/bin/../lib/gcc/pic32mx/4.5.2/../../../../pic32mx/lib/size\libpic32.a(memset.o)
 .reginfo       0x00000000       0x18 c:/program files (x86)/microchip/xc32/v1.21/bin/../lib/gcc/pic32mx/4.5.2/../../../../pic32mx/lib/size\libpic32.a(memset.o)
 .pdr           0x00000000       0x20 c:/program files (x86)/microchip/xc32/v1.21/bin/../lib/gcc/pic32mx/4.5.2/../../../../pic32mx/lib/size\libpic32.a(memset.o)
 .data          0x00000000        0x0 c:/program files (x86)/microchip/xc32/v1.21/bin/../lib/gcc/pic32mx/4.5.2/../../../../pic32mx/lib/size\libpic32.a(strcmp.o)
 .bss           0x00000000        0x0 c:/program files (x86)/microchip/xc32/v1.21/bin/../lib/gcc/pic32mx/4.5.2/../../../../pic32mx/lib/size\libpic32.a(strcmp.o)
 .reginfo       0x00000000       0x18 c:/program files (x86)/microchip/xc32/v1.21/bin/../lib/gcc/pic32mx/4.5.2/../../../../pic32mx/lib/size\libpic32.a(strcmp.o)
 .pdr           0x00000000       0x20 c:/program files (x86)/microchip/xc32/v1.21/bin/../lib/gcc/pic32mx/4.5.2/../../../../pic32mx/lib/size\libpic32.a(strcmp.o)
 .data          0x00000000        0x0 c:/program files (x86)/microchip/xc32/v1.21/bin/../lib/gcc/pic32mx/4.5.2/../../../../pic32mx/lib/size\libpic32.a(strcpy.o)
 .bss           0x00000000        0x0 c:/program files (x86)/microchip/xc32/v1.21/bin/../lib/gcc/pic32mx/4.5.2/../../../../pic32mx/lib/size\libpic32.a(strcpy.o)
 .reginfo       0x00000000       0x18 c:/program files (x86)/microchip/xc32/v1.21/bin/../lib/gcc/pic32mx/4.5.2/../../../../pic32mx/lib/size\libpic32.a(strcpy.o)
 .pdr           0x00000000       0x20 c:/program files (x86)/microchip/xc32/v1.21/bin/../lib/gcc/pic32mx/4.5.2/../../../../pic32mx/lib/size\libpic32.a(strcpy.o)
 .data          0x00000000        0x0 c:/program files (x86)/microchip/xc32/v1.21/bin/../lib/gcc/pic32mx/4.5.2/../../../../pic32mx/lib/size\libpic32.a(strlen.o)
 .bss           0x00000000        0x0 c:/program files (x86)/microchip/xc32/v1.21/bin/../lib/gcc/pic32mx/4.5.2/../../../../pic32mx/lib/size\libpic32.a(strlen.o)
 .reginfo       0x00000000       0x18 c:/program files (x86)/microchip/xc32/v1.21/bin/../lib/gcc/pic32mx/4.5.2/../../../../pic32mx/lib/size\libpic32.a(strlen.o)
 .pdr           0x00000000       0x20 c:/program files (x86)/microchip/xc32/v1.21/bin/../lib/gcc/pic32mx/4.5.2/../../../../pic32mx/lib/size\libpic32.a(strlen.o)
 .text          0x00000000        0x0 c:/program files (x86)/microchip/xc32/v1.21/bin/../lib/gcc/pic32mx/4.5.2/../../../../pic32mx/lib/size\libpic32.a(default-bootstrap-exception-handler.o)
 .data          0x00000000        0x0 c:/program files (x86)/microchip/xc32/v1.21/bin/../lib/gcc/pic32mx/4.5.2/../../../../pic32mx/lib/size\libpic32.a(default-bootstrap-exception-handler.o)
 .bss           0x00000000        0x0 c:/program files (x86)/microchip/xc32/v1.21/bin/../lib/gcc/pic32mx/4.5.2/../../../../pic32mx/lib/size\libpic32.a(default-bootstrap-exception-handler.o)
 .reginfo       0x00000000       0x18 c:/program files (x86)/microchip/xc32/v1.21/bin/../lib/gcc/pic32mx/4.5.2/../../../../pic32mx/lib/size\libpic32.a(default-bootstrap-exception-handler.o)
 .pdr           0x00000000       0x20 c:/program files (x86)/microchip/xc32/v1.21/bin/../lib/gcc/pic32mx/4.5.2/../../../../pic32mx/lib/size\libpic32.a(default-bootstrap-exception-handler.o)
 .text          0x00000000        0x0 c:/program files (x86)/microchip/xc32/v1.21/bin/../lib/gcc/pic32mx/4.5.2/../../../../pic32mx/lib/size\libpic32.a(default-on-reset.o)
 .data          0x00000000        0x0 c:/program files (x86)/microchip/xc32/v1.21/bin/../lib/gcc/pic32mx/4.5.2/../../../../pic32mx/lib/size\libpic32.a(default-on-reset.o)
 .bss           0x00000000        0x0 c:/program files (x86)/microchip/xc32/v1.21/bin/../lib/gcc/pic32mx/4.5.2/../../../../pic32mx/lib/size\libpic32.a(default-on-reset.o)
 .reginfo       0x00000000       0x18 c:/program files (x86)/microchip/xc32/v1.21/bin/../lib/gcc/pic32mx/4.5.2/../../../../pic32mx/lib/size\libpic32.a(default-on-reset.o)
 .pdr           0x00000000       0x20 c:/program files (x86)/microchip/xc32/v1.21/bin/../lib/gcc/pic32mx/4.5.2/../../../../pic32mx/lib/size\libpic32.a(default-on-reset.o)
 .text          0x00000000        0x0 c:/program files (x86)/microchip/xc32/v1.21/bin/../lib/gcc/pic32mx/4.5.2/../../../../pic32mx/lib/size\libpic32.a(default-on-bootstrap.o)
 .data          0x00000000        0x0 c:/program files (x86)/microchip/xc32/v1.21/bin/../lib/gcc/pic32mx/4.5.2/../../../../pic32mx/lib/size\libpic32.a(default-on-bootstrap.o)
 .bss           0x00000000        0x0 c:/program files (x86)/microchip/xc32/v1.21/bin/../lib/gcc/pic32mx/4.5.2/../../../../pic32mx/lib/size\libpic32.a(default-on-bootstrap.o)
 .reginfo       0x00000000       0x18 c:/program files (x86)/microchip/xc32/v1.21/bin/../lib/gcc/pic32mx/4.5.2/../../../../pic32mx/lib/size\libpic32.a(default-on-bootstrap.o)
 .pdr           0x00000000       0x20 c:/program files (x86)/microchip/xc32/v1.21/bin/../lib/gcc/pic32mx/4.5.2/../../../../pic32mx/lib/size\libpic32.a(default-on-bootstrap.o)
 .data          0x00000000        0x0 c:/program files (x86)/microchip/xc32/v1.21/bin/../lib/gcc/pic32mx/4.5.2/../../../../pic32mx/lib/size\libpic32.a(default-nmi-handler.o)
 .bss           0x00000000        0x0 c:/program files (x86)/microchip/xc32/v1.21/bin/../lib/gcc/pic32mx/4.5.2/../../../../pic32mx/lib/size\libpic32.a(default-nmi-handler.o)
 .reginfo       0x00000000       0x18 c:/program files (x86)/microchip/xc32/v1.21/bin/../lib/gcc/pic32mx/4.5.2/../../../../pic32mx/lib/size\libpic32.a(default-nmi-handler.o)
 .pdr           0x00000000       0x20 c:/program files (x86)/microchip/xc32/v1.21/bin/../lib/gcc/pic32mx/4.5.2/../../../../pic32mx/lib/size\libpic32.a(default-nmi-handler.o)
 .text          0x00000000        0x0 c:/program files (x86)/microchip/xc32/v1.21/bin/../lib/gcc/pic32mx/4.5.2/../../../../pic32mx/lib/size\libpic32.a(errno.o)
 .data          0x00000000        0x0 c:/program files (x86)/microchip/xc32/v1.21/bin/../lib/gcc/pic32mx/4.5.2/../../../../pic32mx/lib/size\libpic32.a(errno.o)
 .bss           0x00000000        0x0 c:/program files (x86)/microchip/xc32/v1.21/bin/../lib/gcc/pic32mx/4.5.2/../../../../pic32mx/lib/size\libpic32.a(errno.o)
 .reginfo       0x00000000       0x18 c:/program files (x86)/microchip/xc32/v1.21/bin/../lib/gcc/pic32mx/4.5.2/../../../../pic32mx/lib/size\libpic32.a(errno.o)
 .pdr           0x00000000        0x0 c:/program files (x86)/microchip/xc32/v1.21/bin/../lib/gcc/pic32mx/4.5.2/../../../../pic32mx/lib/size\libpic32.a(errno.o)
 .text          0x00000000        0x0 c:/program files (x86)/microchip/xc32/v1.21/bin/../lib/gcc/pic32mx/4.5.2/../../../../pic32mx/lib/size\libpic32.a(general-exception.o)
 .data          0x00000000        0x0 c:/program files (x86)/microchip/xc32/v1.21/bin/../lib/gcc/pic32mx/4.5.2/../../../../pic32mx/lib/size\libpic32.a(general-exception.o)
 .bss           0x00000000        0x0 c:/program files (x86)/microchip/xc32/v1.21/bin/../lib/gcc/pic32mx/4.5.2/../../../../pic32mx/lib/size\libpic32.a(general-exception.o)
 .reginfo       0x00000000       0x18 c:/program files (x86)/microchip/xc32/v1.21/bin/../lib/gcc/pic32mx/4.5.2/../../../../pic32mx/lib/size\libpic32.a(general-exception.o)
 .pdr           0x00000000       0x20 c:/program files (x86)/microchip/xc32/v1.21/bin/../lib/gcc/pic32mx/4.5.2/../../../../pic32mx/lib/size\libpic32.a(general-exception.o)
 .text          0x00000000        0x0 c:/program files (x86)/microchip/xc32/v1.21/bin/../lib/gcc/pic32mx/4.5.2/../../../../pic32mx/lib/size\libpic32.a(vector1.o)
 .data          0x00000000        0x0 c:/program files (x86)/microchip/xc32/v1.21/bin/../lib/gcc/pic32mx/4.5.2/../../../../pic32mx/lib/size\libpic32.a(vector1.o)
 .bss           0x00000000        0x0 c:/program files (x86)/microchip/xc32/v1.21/bin/../lib/gcc/pic32mx/4.5.2/../../../../pic32mx/lib/size\libpic32.a(vector1.o)
 .reginfo       0x00000000       0x18 c:/program files (x86)/microchip/xc32/v1.21/bin/../lib/gcc/pic32mx/4.5.2/../../../../pic32mx/lib/size\libpic32.a(vector1.o)
 .pdr           0x00000000       0x20 c:/program files (x86)/microchip/xc32/v1.21/bin/../lib/gcc/pic32mx/4.5.2/../../../../pic32mx/lib/size\libpic32.a(vector1.o)
 .text          0x00000000        0x0 c:/program files (x86)/microchip/xc32/v1.21/bin/../lib/gcc/pic32mx/4.5.2/../../../../pic32mx/lib/size\libpic32.a(vector2.o)
 .data          0x00000000        0x0 c:/program files (x86)/microchip/xc32/v1.21/bin/../lib/gcc/pic32mx/4.5.2/../../../../pic32mx/lib/size\libpic32.a(vector2.o)
 .bss           0x00000000        0x0 c:/program files (x86)/microchip/xc32/v1.21/bin/../lib/gcc/pic32mx/4.5.2/../../../../pic32mx/lib/size\libpic32.a(vector2.o)
 .reginfo       0x00000000       0x18 c:/program files (x86)/microchip/xc32/v1.21/bin/../lib/gcc/pic32mx/4.5.2/../../../../pic32mx/lib/size\libpic32.a(vector2.o)
 .pdr           0x00000000       0x20 c:/program files (x86)/microchip/xc32/v1.21/bin/../lib/gcc/pic32mx/4.5.2/../../../../pic32mx/lib/size\libpic32.a(vector2.o)
 .text          0x00000000        0x0 c:/program files (x86)/microchip/xc32/v1.21/bin/../lib/gcc/pic32mx/4.5.2/../../../../pic32mx/lib/size\libpic32.a(vector3.o)
 .data          0x00000000        0x0 c:/program files (x86)/microchip/xc32/v1.21/bin/../lib/gcc/pic32mx/4.5.2/../../../../pic32mx/lib/size\libpic32.a(vector3.o)
 .bss           0x00000000        0x0 c:/program files (x86)/microchip/xc32/v1.21/bin/../lib/gcc/pic32mx/4.5.2/../../../../pic32mx/lib/size\libpic32.a(vector3.o)
 .reginfo       0x00000000       0x18 c:/program files (x86)/microchip/xc32/v1.21/bin/../lib/gcc/pic32mx/4.5.2/../../../../pic32mx/lib/size\libpic32.a(vector3.o)
 .pdr           0x00000000       0x20 c:/program files (x86)/microchip/xc32/v1.21/bin/../lib/gcc/pic32mx/4.5.2/../../../../pic32mx/lib/size\libpic32.a(vector3.o)
 .text          0x00000000        0x0 c:/program files (x86)/microchip/xc32/v1.21/bin/../lib/gcc/pic32mx/4.5.2/../../../../pic32mx/lib/size\libpic32.a(vector4.o)
 .data          0x00000000        0x0 c:/program files (x86)/microchip/xc32/v1.21/bin/../lib/gcc/pic32mx/4.5.2/../../../../pic32mx/lib/size\libpic32.a(vector4.o)
 .bss           0x00000000        0x0 c:/program files (x86)/microchip/xc32/v1.21/bin/../lib/gcc/pic32mx/4.5.2/../../../../pic32mx/lib/size\libpic32.a(vector4.o)
 .reginfo       0x00000000       0x18 c:/program files (x86)/microchip/xc32/v1.21/bin/../lib/gcc/pic32mx/4.5.2/../../../../pic32mx/lib/size\libpic32.a(vector4.o)
 .pdr           0x00000000       0x20 c:/program files (x86)/microchip/xc32/v1.21/bin/../lib/gcc/pic32mx/4.5.2/../../../../pic32mx/lib/size\libpic32.a(vector4.o)
 .text          0x00000000        0x0 c:/program files (x86)/microchip/xc32/v1.21/bin/../lib/gcc/pic32mx/4.5.2/../../../../pic32mx/lib/size\libpic32.a(vector5.o)
 .data          0x00000000        0x0 c:/program files (x86)/microchip/xc32/v1.21/bin/../lib/gcc/pic32mx/4.5.2/../../../../pic32mx/lib/size\libpic32.a(vector5.o)
 .bss           0x00000000        0x0 c:/program files (x86)/microchip/xc32/v1.21/bin/../lib/gcc/pic32mx/4.5.2/../../../../pic32mx/lib/size\libpic32.a(vector5.o)
 .reginfo       0x00000000       0x18 c:/program files (x86)/microchip/xc32/v1.21/bin/../lib/gcc/pic32mx/4.5.2/../../../../pic32mx/lib/size\libpic32.a(vector5.o)
 .pdr           0x00000000       0x20 c:/program files (x86)/microchip/xc32/v1.21/bin/../lib/gcc/pic32mx/4.5.2/../../../../pic32mx/lib/size\libpic32.a(vector5.o)
 .text          0x00000000        0x0 c:/program files (x86)/microchip/xc32/v1.21/bin/../lib/gcc/pic32mx/4.5.2/../../../../pic32mx/lib/size\libpic32.a(vector6.o)
 .data          0x00000000        0x0 c:/program files (x86)/microchip/xc32/v1.21/bin/../lib/gcc/pic32mx/4.5.2/../../../../pic32mx/lib/size\libpic32.a(vector6.o)
 .bss           0x00000000        0x0 c:/program files (x86)/microchip/xc32/v1.21/bin/../lib/gcc/pic32mx/4.5.2/../../../../pic32mx/lib/size\libpic32.a(vector6.o)
 .reginfo       0x00000000       0x18 c:/program files (x86)/microchip/xc32/v1.21/bin/../lib/gcc/pic32mx/4.5.2/../../../../pic32mx/lib/size\libpic32.a(vector6.o)
 .pdr           0x00000000       0x20 c:/program files (x86)/microchip/xc32/v1.21/bin/../lib/gcc/pic32mx/4.5.2/../../../../pic32mx/lib/size\libpic32.a(vector6.o)
 .text          0x00000000        0x0 c:/program files (x86)/microchip/xc32/v1.21/bin/../lib/gcc/pic32mx/4.5.2/../../../../pic32mx/lib/size\libpic32.a(vector8.o)
 .data          0x00000000        0x0 c:/program files (x86)/microchip/xc32/v1.21/bin/../lib/gcc/pic32mx/4.5.2/../../../../pic32mx/lib/size\libpic32.a(vector8.o)
 .bss           0x00000000        0x0 c:/program files (x86)/microchip/xc32/v1.21/bin/../lib/gcc/pic32mx/4.5.2/../../../../pic32mx/lib/size\libpic32.a(vector8.o)
 .reginfo       0x00000000       0x18 c:/program files (x86)/microchip/xc32/v1.21/bin/../lib/gcc/pic32mx/4.5.2/../../../../pic32mx/lib/size\libpic32.a(vector8.o)
 .pdr           0x00000000       0x20 c:/program files (x86)/microchip/xc32/v1.21/bin/../lib/gcc/pic32mx/4.5.2/../../../../pic32mx/lib/size\libpic32.a(vector8.o)
 .text          0x00000000        0x0 c:/program files (x86)/microchip/xc32/v1.21/bin/../lib/gcc/pic32mx/4.5.2/../../../../pic32mx/lib/size\libpic32.a(vector9.o)
 .data          0x00000000        0x0 c:/program files (x86)/microchip/xc32/v1.21/bin/../lib/gcc/pic32mx/4.5.2/../../../../pic32mx/lib/size\libpic32.a(vector9.o)
 .bss           0x00000000        0x0 c:/program files (x86)/microchip/xc32/v1.21/bin/../lib/gcc/pic32mx/4.5.2/../../../../pic32mx/lib/size\libpic32.a(vector9.o)
 .reginfo       0x00000000       0x18 c:/program files (x86)/microchip/xc32/v1.21/bin/../lib/gcc/pic32mx/4.5.2/../../../../pic32mx/lib/size\libpic32.a(vector9.o)
 .pdr           0x00000000       0x20 c:/program files (x86)/microchip/xc32/v1.21/bin/../lib/gcc/pic32mx/4.5.2/../../../../pic32mx/lib/size\libpic32.a(vector9.o)
 .text          0x00000000        0x0 c:/program files (x86)/microchip/xc32/v1.21/bin/../lib/gcc/pic32mx/4.5.2/../../../../pic32mx/lib/size\libpic32.a(vector10.o)
 .data          0x00000000        0x0 c:/program files (x86)/microchip/xc32/v1.21/bin/../lib/gcc/pic32mx/4.5.2/../../../../pic32mx/lib/size\libpic32.a(vector10.o)
 .bss           0x00000000        0x0 c:/program files (x86)/microchip/xc32/v1.21/bin/../lib/gcc/pic32mx/4.5.2/../../../../pic32mx/lib/size\libpic32.a(vector10.o)
 .reginfo       0x00000000       0x18 c:/program files (x86)/microchip/xc32/v1.21/bin/../lib/gcc/pic32mx/4.5.2/../../../../pic32mx/lib/size\libpic32.a(vector10.o)
 .pdr           0x00000000       0x20 c:/program files (x86)/microchip/xc32/v1.21/bin/../lib/gcc/pic32mx/4.5.2/../../../../pic32mx/lib/size\libpic32.a(vector10.o)
 .text          0x00000000        0x0 c:/program files (x86)/microchip/xc32/v1.21/bin/../lib/gcc/pic32mx/4.5.2/../../../../pic32mx/lib/size\libpic32.a(vector11.o)
 .data          0x00000000        0x0 c:/program files (x86)/microchip/xc32/v1.21/bin/../lib/gcc/pic32mx/4.5.2/../../../../pic32mx/lib/size\libpic32.a(vector11.o)
 .bss           0x00000000        0x0 c:/program files (x86)/microchip/xc32/v1.21/bin/../lib/gcc/pic32mx/4.5.2/../../../../pic32mx/lib/size\libpic32.a(vector11.o)
 .reginfo       0x00000000       0x18 c:/program files (x86)/microchip/xc32/v1.21/bin/../lib/gcc/pic32mx/4.5.2/../../../../pic32mx/lib/size\libpic32.a(vector11.o)
 .pdr           0x00000000       0x20 c:/program files (x86)/microchip/xc32/v1.21/bin/../lib/gcc/pic32mx/4.5.2/../../../../pic32mx/lib/size\libpic32.a(vector11.o)
 .text          0x00000000        0x0 c:/program files (x86)/microchip/xc32/v1.21/bin/../lib/gcc/pic32mx/4.5.2/../../../../pic32mx/lib/size\libpic32.a(vector12.o)
 .data          0x00000000        0x0 c:/program files (x86)/microchip/xc32/v1.21/bin/../lib/gcc/pic32mx/4.5.2/../../../../pic32mx/lib/size\libpic32.a(vector12.o)
 .bss           0x00000000        0x0 c:/program files (x86)/microchip/xc32/v1.21/bin/../lib/gcc/pic32mx/4.5.2/../../../../pic32mx/lib/size\libpic32.a(vector12.o)
 .reginfo       0x00000000       0x18 c:/program files (x86)/microchip/xc32/v1.21/bin/../lib/gcc/pic32mx/4.5.2/../../../../pic32mx/lib/size\libpic32.a(vector12.o)
 .pdr           0x00000000       0x20 c:/program files (x86)/microchip/xc32/v1.21/bin/../lib/gcc/pic32mx/4.5.2/../../../../pic32mx/lib/size\libpic32.a(vector12.o)
 .text          0x00000000        0x0 c:/program files (x86)/microchip/xc32/v1.21/bin/../lib/gcc/pic32mx/4.5.2/../../../../pic32mx/lib/size\libpic32.a(vector13.o)
 .data          0x00000000        0x0 c:/program files (x86)/microchip/xc32/v1.21/bin/../lib/gcc/pic32mx/4.5.2/../../../../pic32mx/lib/size\libpic32.a(vector13.o)
 .bss           0x00000000        0x0 c:/program files (x86)/microchip/xc32/v1.21/bin/../lib/gcc/pic32mx/4.5.2/../../../../pic32mx/lib/size\libpic32.a(vector13.o)
 .reginfo       0x00000000       0x18 c:/program files (x86)/microchip/xc32/v1.21/bin/../lib/gcc/pic32mx/4.5.2/../../../../pic32mx/lib/size\libpic32.a(vector13.o)
 .pdr           0x00000000       0x20 c:/program files (x86)/microchip/xc32/v1.21/bin/../lib/gcc/pic32mx/4.5.2/../../../../pic32mx/lib/size\libpic32.a(vector13.o)
 .text          0x00000000        0x0 c:/program files (x86)/microchip/xc32/v1.21/bin/../lib/gcc/pic32mx/4.5.2/../../../../pic32mx/lib/size\libpic32.a(vector14.o)
 .data          0x00000000        0x0 c:/program files (x86)/microchip/xc32/v1.21/bin/../lib/gcc/pic32mx/4.5.2/../../../../pic32mx/lib/size\libpic32.a(vector14.o)
 .bss           0x00000000        0x0 c:/program files (x86)/microchip/xc32/v1.21/bin/../lib/gcc/pic32mx/4.5.2/../../../../pic32mx/lib/size\libpic32.a(vector14.o)
 .reginfo       0x00000000       0x18 c:/program files (x86)/microchip/xc32/v1.21/bin/../lib/gcc/pic32mx/4.5.2/../../../../pic32mx/lib/size\libpic32.a(vector14.o)
 .pdr           0x00000000       0x20 c:/program files (x86)/microchip/xc32/v1.21/bin/../lib/gcc/pic32mx/4.5.2/../../../../pic32mx/lib/size\libpic32.a(vector14.o)
 .text          0x00000000        0x0 c:/program files (x86)/microchip/xc32/v1.21/bin/../lib/gcc/pic32mx/4.5.2/../../../../pic32mx/lib/size\libpic32.a(vector16.o)
 .data          0x00000000        0x0 c:/program files (x86)/microchip/xc32/v1.21/bin/../lib/gcc/pic32mx/4.5.2/../../../../pic32mx/lib/size\libpic32.a(vector16.o)
 .bss           0x00000000        0x0 c:/program files (x86)/microchip/xc32/v1.21/bin/../lib/gcc/pic32mx/4.5.2/../../../../pic32mx/lib/size\libpic32.a(vector16.o)
 .reginfo       0x00000000       0x18 c:/program files (x86)/microchip/xc32/v1.21/bin/../lib/gcc/pic32mx/4.5.2/../../../../pic32mx/lib/size\libpic32.a(vector16.o)
 .pdr           0x00000000       0x20 c:/program files (x86)/microchip/xc32/v1.21/bin/../lib/gcc/pic32mx/4.5.2/../../../../pic32mx/lib/size\libpic32.a(vector16.o)
 .text          0x00000000        0x0 c:/program files (x86)/microchip/xc32/v1.21/bin/../lib/gcc/pic32mx/4.5.2/../../../../pic32mx/lib/size\libpic32.a(vector17.o)
 .data          0x00000000        0x0 c:/program files (x86)/microchip/xc32/v1.21/bin/../lib/gcc/pic32mx/4.5.2/../../../../pic32mx/lib/size\libpic32.a(vector17.o)
 .bss           0x00000000        0x0 c:/program files (x86)/microchip/xc32/v1.21/bin/../lib/gcc/pic32mx/4.5.2/../../../../pic32mx/lib/size\libpic32.a(vector17.o)
 .reginfo       0x00000000       0x18 c:/program files (x86)/microchip/xc32/v1.21/bin/../lib/gcc/pic32mx/4.5.2/../../../../pic32mx/lib/size\libpic32.a(vector17.o)
 .pdr           0x00000000       0x20 c:/program files (x86)/microchip/xc32/v1.21/bin/../lib/gcc/pic32mx/4.5.2/../../../../pic32mx/lib/size\libpic32.a(vector17.o)
 .text          0x00000000        0x0 c:/program files (x86)/microchip/xc32/v1.21/bin/../lib/gcc/pic32mx/4.5.2/../../../../pic32mx/lib/size\libpic32.a(vector18.o)
 .data          0x00000000        0x0 c:/program files (x86)/microchip/xc32/v1.21/bin/../lib/gcc/pic32mx/4.5.2/../../../../pic32mx/lib/size\libpic32.a(vector18.o)
 .bss           0x00000000        0x0 c:/program files (x86)/microchip/xc32/v1.21/bin/../lib/gcc/pic32mx/4.5.2/../../../../pic32mx/lib/size\libpic32.a(vector18.o)
 .reginfo       0x00000000       0x18 c:/program files (x86)/microchip/xc32/v1.21/bin/../lib/gcc/pic32mx/4.5.2/../../../../pic32mx/lib/size\libpic32.a(vector18.o)
 .pdr           0x00000000       0x20 c:/program files (x86)/microchip/xc32/v1.21/bin/../lib/gcc/pic32mx/4.5.2/../../../../pic32mx/lib/size\libpic32.a(vector18.o)
 .text          0x00000000        0x0 c:/program files (x86)/microchip/xc32/v1.21/bin/../lib/gcc/pic32mx/4.5.2/../../../../pic32mx/lib/size\libpic32.a(vector19.o)
 .data          0x00000000        0x0 c:/program files (x86)/microchip/xc32/v1.21/bin/../lib/gcc/pic32mx/4.5.2/../../../../pic32mx/lib/size\libpic32.a(vector19.o)
 .bss           0x00000000        0x0 c:/program files (x86)/microchip/xc32/v1.21/bin/../lib/gcc/pic32mx/4.5.2/../../../../pic32mx/lib/size\libpic32.a(vector19.o)
 .reginfo       0x00000000       0x18 c:/program files (x86)/microchip/xc32/v1.21/bin/../lib/gcc/pic32mx/4.5.2/../../../../pic32mx/lib/size\libpic32.a(vector19.o)
 .pdr           0x00000000       0x20 c:/program files (x86)/microchip/xc32/v1.21/bin/../lib/gcc/pic32mx/4.5.2/../../../../pic32mx/lib/size\libpic32.a(vector19.o)
 .text          0x00000000        0x0 c:/program files (x86)/microchip/xc32/v1.21/bin/../lib/gcc/pic32mx/4.5.2/../../../../pic32mx/lib/size\libpic32.a(vector20.o)
 .data          0x00000000        0x0 c:/program files (x86)/microchip/xc32/v1.21/bin/../lib/gcc/pic32mx/4.5.2/../../../../pic32mx/lib/size\libpic32.a(vector20.o)
 .bss           0x00000000        0x0 c:/program files (x86)/microchip/xc32/v1.21/bin/../lib/gcc/pic32mx/4.5.2/../../../../pic32mx/lib/size\libpic32.a(vector20.o)
 .reginfo       0x00000000       0x18 c:/program files (x86)/microchip/xc32/v1.21/bin/../lib/gcc/pic32mx/4.5.2/../../../../pic32mx/lib/size\libpic32.a(vector20.o)
 .pdr           0x00000000       0x20 c:/program files (x86)/microchip/xc32/v1.21/bin/../lib/gcc/pic32mx/4.5.2/../../../../pic32mx/lib/size\libpic32.a(vector20.o)
 .text          0x00000000        0x0 c:/program files (x86)/microchip/xc32/v1.21/bin/../lib/gcc/pic32mx/4.5.2/../../../../pic32mx/lib/size\libpic32.a(vector21.o)
 .data          0x00000000        0x0 c:/program files (x86)/microchip/xc32/v1.21/bin/../lib/gcc/pic32mx/4.5.2/../../../../pic32mx/lib/size\libpic32.a(vector21.o)
 .bss           0x00000000        0x0 c:/program files (x86)/microchip/xc32/v1.21/bin/../lib/gcc/pic32mx/4.5.2/../../../../pic32mx/lib/size\libpic32.a(vector21.o)
 .reginfo       0x00000000       0x18 c:/program files (x86)/microchip/xc32/v1.21/bin/../lib/gcc/pic32mx/4.5.2/../../../../pic32mx/lib/size\libpic32.a(vector21.o)
 .pdr           0x00000000       0x20 c:/program files (x86)/microchip/xc32/v1.21/bin/../lib/gcc/pic32mx/4.5.2/../../../../pic32mx/lib/size\libpic32.a(vector21.o)
 .text          0x00000000        0x0 c:/program files (x86)/microchip/xc32/v1.21/bin/../lib/gcc/pic32mx/4.5.2/../../../../pic32mx/lib/size\libpic32.a(vector22.o)
 .data          0x00000000        0x0 c:/program files (x86)/microchip/xc32/v1.21/bin/../lib/gcc/pic32mx/4.5.2/../../../../pic32mx/lib/size\libpic32.a(vector22.o)
 .bss           0x00000000        0x0 c:/program files (x86)/microchip/xc32/v1.21/bin/../lib/gcc/pic32mx/4.5.2/../../../../pic32mx/lib/size\libpic32.a(vector22.o)
 .reginfo       0x00000000       0x18 c:/program files (x86)/microchip/xc32/v1.21/bin/../lib/gcc/pic32mx/4.5.2/../../../../pic32mx/lib/size\libpic32.a(vector22.o)
 .pdr           0x00000000       0x20 c:/program files (x86)/microchip/xc32/v1.21/bin/../lib/gcc/pic32mx/4.5.2/../../../../pic32mx/lib/size\libpic32.a(vector22.o)
 .text          0x00000000        0x0 c:/program files (x86)/microchip/xc32/v1.21/bin/../lib/gcc/pic32mx/4.5.2/../../../../pic32mx/lib/size\libpic32.a(vector23.o)
 .data          0x00000000        0x0 c:/program files (x86)/microchip/xc32/v1.21/bin/../lib/gcc/pic32mx/4.5.2/../../../../pic32mx/lib/size\libpic32.a(vector23.o)
 .bss           0x00000000        0x0 c:/program files (x86)/microchip/xc32/v1.21/bin/../lib/gcc/pic32mx/4.5.2/../../../../pic32mx/lib/size\libpic32.a(vector23.o)
 .reginfo       0x00000000       0x18 c:/program files (x86)/microchip/xc32/v1.21/bin/../lib/gcc/pic32mx/4.5.2/../../../../pic32mx/lib/size\libpic32.a(vector23.o)
 .pdr           0x00000000       0x20 c:/program files (x86)/microchip/xc32/v1.21/bin/../lib/gcc/pic32mx/4.5.2/../../../../pic32mx/lib/size\libpic32.a(vector23.o)
 .text          0x00000000        0x0 c:/program files (x86)/microchip/xc32/v1.21/bin/../lib/gcc/pic32mx/4.5.2/../../../../pic32mx/lib/size\libpic32.a(vector24.o)
 .data          0x00000000        0x0 c:/program files (x86)/microchip/xc32/v1.21/bin/../lib/gcc/pic32mx/4.5.2/../../../../pic32mx/lib/size\libpic32.a(vector24.o)
 .bss           0x00000000        0x0 c:/program files (x86)/microchip/xc32/v1.21/bin/../lib/gcc/pic32mx/4.5.2/../../../../pic32mx/lib/size\libpic32.a(vector24.o)
 .reginfo       0x00000000       0x18 c:/program files (x86)/microchip/xc32/v1.21/bin/../lib/gcc/pic32mx/4.5.2/../../../../pic32mx/lib/size\libpic32.a(vector24.o)
 .pdr           0x00000000       0x20 c:/program files (x86)/microchip/xc32/v1.21/bin/../lib/gcc/pic32mx/4.5.2/../../../../pic32mx/lib/size\libpic32.a(vector24.o)
 .text          0x00000000        0x0 c:/program files (x86)/microchip/xc32/v1.21/bin/../lib/gcc/pic32mx/4.5.2/../../../../pic32mx/lib/size\libpic32.a(vector25.o)
 .data          0x00000000        0x0 c:/program files (x86)/microchip/xc32/v1.21/bin/../lib/gcc/pic32mx/4.5.2/../../../../pic32mx/lib/size\libpic32.a(vector25.o)
 .bss           0x00000000        0x0 c:/program files (x86)/microchip/xc32/v1.21/bin/../lib/gcc/pic32mx/4.5.2/../../../../pic32mx/lib/size\libpic32.a(vector25.o)
 .reginfo       0x00000000       0x18 c:/program files (x86)/microchip/xc32/v1.21/bin/../lib/gcc/pic32mx/4.5.2/../../../../pic32mx/lib/size\libpic32.a(vector25.o)
 .pdr           0x00000000       0x20 c:/program files (x86)/microchip/xc32/v1.21/bin/../lib/gcc/pic32mx/4.5.2/../../../../pic32mx/lib/size\libpic32.a(vector25.o)
 .text          0x00000000        0x0 c:/program files (x86)/microchip/xc32/v1.21/bin/../lib/gcc/pic32mx/4.5.2/../../../../pic32mx/lib/size\libpic32.a(vector27.o)
 .data          0x00000000        0x0 c:/program files (x86)/microchip/xc32/v1.21/bin/../lib/gcc/pic32mx/4.5.2/../../../../pic32mx/lib/size\libpic32.a(vector27.o)
 .bss           0x00000000        0x0 c:/program files (x86)/microchip/xc32/v1.21/bin/../lib/gcc/pic32mx/4.5.2/../../../../pic32mx/lib/size\libpic32.a(vector27.o)
 .reginfo       0x00000000       0x18 c:/program files (x86)/microchip/xc32/v1.21/bin/../lib/gcc/pic32mx/4.5.2/../../../../pic32mx/lib/size\libpic32.a(vector27.o)
 .pdr           0x00000000       0x20 c:/program files (x86)/microchip/xc32/v1.21/bin/../lib/gcc/pic32mx/4.5.2/../../../../pic32mx/lib/size\libpic32.a(vector27.o)
 .text          0x00000000        0x0 c:/program files (x86)/microchip/xc32/v1.21/bin/../lib/gcc/pic32mx/4.5.2/../../../../pic32mx/lib/size\libpic32.a(vector28.o)
 .data          0x00000000        0x0 c:/program files (x86)/microchip/xc32/v1.21/bin/../lib/gcc/pic32mx/4.5.2/../../../../pic32mx/lib/size\libpic32.a(vector28.o)
 .bss           0x00000000        0x0 c:/program files (x86)/microchip/xc32/v1.21/bin/../lib/gcc/pic32mx/4.5.2/../../../../pic32mx/lib/size\libpic32.a(vector28.o)
 .reginfo       0x00000000       0x18 c:/program files (x86)/microchip/xc32/v1.21/bin/../lib/gcc/pic32mx/4.5.2/../../../../pic32mx/lib/size\libpic32.a(vector28.o)
 .pdr           0x00000000       0x20 c:/program files (x86)/microchip/xc32/v1.21/bin/../lib/gcc/pic32mx/4.5.2/../../../../pic32mx/lib/size\libpic32.a(vector28.o)
 .text          0x00000000        0x0 c:/program files (x86)/microchip/xc32/v1.21/bin/../lib/gcc/pic32mx/4.5.2/../../../../pic32mx/lib/size\libpic32.a(vector29.o)
 .data          0x00000000        0x0 c:/program files (x86)/microchip/xc32/v1.21/bin/../lib/gcc/pic32mx/4.5.2/../../../../pic32mx/lib/size\libpic32.a(vector29.o)
 .bss           0x00000000        0x0 c:/program files (x86)/microchip/xc32/v1.21/bin/../lib/gcc/pic32mx/4.5.2/../../../../pic32mx/lib/size\libpic32.a(vector29.o)
 .reginfo       0x00000000       0x18 c:/program files (x86)/microchip/xc32/v1.21/bin/../lib/gcc/pic32mx/4.5.2/../../../../pic32mx/lib/size\libpic32.a(vector29.o)
 .pdr           0x00000000       0x20 c:/program files (x86)/microchip/xc32/v1.21/bin/../lib/gcc/pic32mx/4.5.2/../../../../pic32mx/lib/size\libpic32.a(vector29.o)
 .text          0x00000000        0x0 c:/program files (x86)/microchip/xc32/v1.21/bin/../lib/gcc/pic32mx/4.5.2/../../../../pic32mx/lib/size\libpic32.a(vector30.o)
 .data          0x00000000        0x0 c:/program files (x86)/microchip/xc32/v1.21/bin/../lib/gcc/pic32mx/4.5.2/../../../../pic32mx/lib/size\libpic32.a(vector30.o)
 .bss           0x00000000        0x0 c:/program files (x86)/microchip/xc32/v1.21/bin/../lib/gcc/pic32mx/4.5.2/../../../../pic32mx/lib/size\libpic32.a(vector30.o)
 .reginfo       0x00000000       0x18 c:/program files (x86)/microchip/xc32/v1.21/bin/../lib/gcc/pic32mx/4.5.2/../../../../pic32mx/lib/size\libpic32.a(vector30.o)
 .pdr           0x00000000       0x20 c:/program files (x86)/microchip/xc32/v1.21/bin/../lib/gcc/pic32mx/4.5.2/../../../../pic32mx/lib/size\libpic32.a(vector30.o)
 .text          0x00000000        0x0 c:/program files (x86)/microchip/xc32/v1.21/bin/../lib/gcc/pic32mx/4.5.2/../../../../pic32mx/lib/size\libpic32.a(vector31.o)
 .data          0x00000000        0x0 c:/program files (x86)/microchip/xc32/v1.21/bin/../lib/gcc/pic32mx/4.5.2/../../../../pic32mx/lib/size\libpic32.a(vector31.o)
 .bss           0x00000000        0x0 c:/program files (x86)/microchip/xc32/v1.21/bin/../lib/gcc/pic32mx/4.5.2/../../../../pic32mx/lib/size\libpic32.a(vector31.o)
 .reginfo       0x00000000       0x18 c:/program files (x86)/microchip/xc32/v1.21/bin/../lib/gcc/pic32mx/4.5.2/../../../../pic32mx/lib/size\libpic32.a(vector31.o)
 .pdr           0x00000000       0x20 c:/program files (x86)/microchip/xc32/v1.21/bin/../lib/gcc/pic32mx/4.5.2/../../../../pic32mx/lib/size\libpic32.a(vector31.o)
 .text          0x00000000        0x0 c:/program files (x86)/microchip/xc32/v1.21/bin/../lib/gcc/pic32mx/4.5.2/../../../../pic32mx/lib/size\libpic32.a(vector32.o)
 .data          0x00000000        0x0 c:/program files (x86)/microchip/xc32/v1.21/bin/../lib/gcc/pic32mx/4.5.2/../../../../pic32mx/lib/size\libpic32.a(vector32.o)
 .bss           0x00000000        0x0 c:/program files (x86)/microchip/xc32/v1.21/bin/../lib/gcc/pic32mx/4.5.2/../../../../pic32mx/lib/size\libpic32.a(vector32.o)
 .reginfo       0x00000000       0x18 c:/program files (x86)/microchip/xc32/v1.21/bin/../lib/gcc/pic32mx/4.5.2/../../../../pic32mx/lib/size\libpic32.a(vector32.o)
 .pdr           0x00000000       0x20 c:/program files (x86)/microchip/xc32/v1.21/bin/../lib/gcc/pic32mx/4.5.2/../../../../pic32mx/lib/size\libpic32.a(vector32.o)
 .text          0x00000000        0x0 c:/program files (x86)/microchip/xc32/v1.21/bin/../lib/gcc/pic32mx/4.5.2/../../../../pic32mx/lib/size\libpic32.a(vector33.o)
 .data          0x00000000        0x0 c:/program files (x86)/microchip/xc32/v1.21/bin/../lib/gcc/pic32mx/4.5.2/../../../../pic32mx/lib/size\libpic32.a(vector33.o)
 .bss           0x00000000        0x0 c:/program files (x86)/microchip/xc32/v1.21/bin/../lib/gcc/pic32mx/4.5.2/../../../../pic32mx/lib/size\libpic32.a(vector33.o)
 .reginfo       0x00000000       0x18 c:/program files (x86)/microchip/xc32/v1.21/bin/../lib/gcc/pic32mx/4.5.2/../../../../pic32mx/lib/size\libpic32.a(vector33.o)
 .pdr           0x00000000       0x20 c:/program files (x86)/microchip/xc32/v1.21/bin/../lib/gcc/pic32mx/4.5.2/../../../../pic32mx/lib/size\libpic32.a(vector33.o)
 .text          0x00000000        0x0 c:/program files (x86)/microchip/xc32/v1.21/bin/../lib/gcc/pic32mx/4.5.2/../../../../pic32mx/lib/size\libpic32.a(vector34.o)
 .data          0x00000000        0x0 c:/program files (x86)/microchip/xc32/v1.21/bin/../lib/gcc/pic32mx/4.5.2/../../../../pic32mx/lib/size\libpic32.a(vector34.o)
 .bss           0x00000000        0x0 c:/program files (x86)/microchip/xc32/v1.21/bin/../lib/gcc/pic32mx/4.5.2/../../../../pic32mx/lib/size\libpic32.a(vector34.o)
 .reginfo       0x00000000       0x18 c:/program files (x86)/microchip/xc32/v1.21/bin/../lib/gcc/pic32mx/4.5.2/../../../../pic32mx/lib/size\libpic32.a(vector34.o)
 .pdr           0x00000000       0x20 c:/program files (x86)/microchip/xc32/v1.21/bin/../lib/gcc/pic32mx/4.5.2/../../../../pic32mx/lib/size\libpic32.a(vector34.o)
 .text          0x00000000        0x0 c:/program files (x86)/microchip/xc32/v1.21/bin/../lib/gcc/pic32mx/4.5.2/../../../../pic32mx/lib/size\libpic32.a(vector35.o)
 .data          0x00000000        0x0 c:/program files (x86)/microchip/xc32/v1.21/bin/../lib/gcc/pic32mx/4.5.2/../../../../pic32mx/lib/size\libpic32.a(vector35.o)
 .bss           0x00000000        0x0 c:/program files (x86)/microchip/xc32/v1.21/bin/../lib/gcc/pic32mx/4.5.2/../../../../pic32mx/lib/size\libpic32.a(vector35.o)
 .reginfo       0x00000000       0x18 c:/program files (x86)/microchip/xc32/v1.21/bin/../lib/gcc/pic32mx/4.5.2/../../../../pic32mx/lib/size\libpic32.a(vector35.o)
 .pdr           0x00000000       0x20 c:/program files (x86)/microchip/xc32/v1.21/bin/../lib/gcc/pic32mx/4.5.2/../../../../pic32mx/lib/size\libpic32.a(vector35.o)
 .text          0x00000000        0x0 c:/program files (x86)/microchip/xc32/v1.21/bin/../lib/gcc/pic32mx/4.5.2/../../../../pic32mx/lib/size\libpic32.a(vector36.o)
 .data          0x00000000        0x0 c:/program files (x86)/microchip/xc32/v1.21/bin/../lib/gcc/pic32mx/4.5.2/../../../../pic32mx/lib/size\libpic32.a(vector36.o)
 .bss           0x00000000        0x0 c:/program files (x86)/microchip/xc32/v1.21/bin/../lib/gcc/pic32mx/4.5.2/../../../../pic32mx/lib/size\libpic32.a(vector36.o)
 .reginfo       0x00000000       0x18 c:/program files (x86)/microchip/xc32/v1.21/bin/../lib/gcc/pic32mx/4.5.2/../../../../pic32mx/lib/size\libpic32.a(vector36.o)
 .pdr           0x00000000       0x20 c:/program files (x86)/microchip/xc32/v1.21/bin/../lib/gcc/pic32mx/4.5.2/../../../../pic32mx/lib/size\libpic32.a(vector36.o)
 .text          0x00000000        0x0 c:/program files (x86)/microchip/xc32/v1.21/bin/../lib/gcc/pic32mx/4.5.2/../../../../pic32mx/lib/size\libpic32.a(vector37.o)
 .data          0x00000000        0x0 c:/program files (x86)/microchip/xc32/v1.21/bin/../lib/gcc/pic32mx/4.5.2/../../../../pic32mx/lib/size\libpic32.a(vector37.o)
 .bss           0x00000000        0x0 c:/program files (x86)/microchip/xc32/v1.21/bin/../lib/gcc/pic32mx/4.5.2/../../../../pic32mx/lib/size\libpic32.a(vector37.o)
 .reginfo       0x00000000       0x18 c:/program files (x86)/microchip/xc32/v1.21/bin/../lib/gcc/pic32mx/4.5.2/../../../../pic32mx/lib/size\libpic32.a(vector37.o)
 .pdr           0x00000000       0x20 c:/program files (x86)/microchip/xc32/v1.21/bin/../lib/gcc/pic32mx/4.5.2/../../../../pic32mx/lib/size\libpic32.a(vector37.o)
 .text          0x00000000        0x0 c:/program files (x86)/microchip/xc32/v1.21/bin/../lib/gcc/pic32mx/4.5.2/../../../../pic32mx/lib/size\libpic32.a(vector38.o)
 .data          0x00000000        0x0 c:/program files (x86)/microchip/xc32/v1.21/bin/../lib/gcc/pic32mx/4.5.2/../../../../pic32mx/lib/size\libpic32.a(vector38.o)
 .bss           0x00000000        0x0 c:/program files (x86)/microchip/xc32/v1.21/bin/../lib/gcc/pic32mx/4.5.2/../../../../pic32mx/lib/size\libpic32.a(vector38.o)
 .reginfo       0x00000000       0x18 c:/program files (x86)/microchip/xc32/v1.21/bin/../lib/gcc/pic32mx/4.5.2/../../../../pic32mx/lib/size\libpic32.a(vector38.o)
 .pdr           0x00000000       0x20 c:/program files (x86)/microchip/xc32/v1.21/bin/../lib/gcc/pic32mx/4.5.2/../../../../pic32mx/lib/size\libpic32.a(vector38.o)
 .text          0x00000000        0x0 c:/program files (x86)/microchip/xc32/v1.21/bin/../lib/gcc/pic32mx/4.5.2/../../../../pic32mx/lib/size\libpic32.a(vector39.o)
 .data          0x00000000        0x0 c:/program files (x86)/microchip/xc32/v1.21/bin/../lib/gcc/pic32mx/4.5.2/../../../../pic32mx/lib/size\libpic32.a(vector39.o)
 .bss           0x00000000        0x0 c:/program files (x86)/microchip/xc32/v1.21/bin/../lib/gcc/pic32mx/4.5.2/../../../../pic32mx/lib/size\libpic32.a(vector39.o)
 .reginfo       0x00000000       0x18 c:/program files (x86)/microchip/xc32/v1.21/bin/../lib/gcc/pic32mx/4.5.2/../../../../pic32mx/lib/size\libpic32.a(vector39.o)
 .pdr           0x00000000       0x20 c:/program files (x86)/microchip/xc32/v1.21/bin/../lib/gcc/pic32mx/4.5.2/../../../../pic32mx/lib/size\libpic32.a(vector39.o)
 .text          0x00000000        0x0 c:/program files (x86)/microchip/xc32/v1.21/bin/../lib/gcc/pic32mx/4.5.2/../../../../pic32mx/lib/size\libpic32.a(vector40.o)
 .data          0x00000000        0x0 c:/program files (x86)/microchip/xc32/v1.21/bin/../lib/gcc/pic32mx/4.5.2/../../../../pic32mx/lib/size\libpic32.a(vector40.o)
 .bss           0x00000000        0x0 c:/program files (x86)/microchip/xc32/v1.21/bin/../lib/gcc/pic32mx/4.5.2/../../../../pic32mx/lib/size\libpic32.a(vector40.o)
 .reginfo       0x00000000       0x18 c:/program files (x86)/microchip/xc32/v1.21/bin/../lib/gcc/pic32mx/4.5.2/../../../../pic32mx/lib/size\libpic32.a(vector40.o)
 .pdr           0x00000000       0x20 c:/program files (x86)/microchip/xc32/v1.21/bin/../lib/gcc/pic32mx/4.5.2/../../../../pic32mx/lib/size\libpic32.a(vector40.o)
 .text          0x00000000        0x0 c:/program files (x86)/microchip/xc32/v1.21/bin/../lib/gcc/pic32mx/4.5.2/../../../../pic32mx/lib/size\libpic32.a(vector41.o)
 .data          0x00000000        0x0 c:/program files (x86)/microchip/xc32/v1.21/bin/../lib/gcc/pic32mx/4.5.2/../../../../pic32mx/lib/size\libpic32.a(vector41.o)
 .bss           0x00000000        0x0 c:/program files (x86)/microchip/xc32/v1.21/bin/../lib/gcc/pic32mx/4.5.2/../../../../pic32mx/lib/size\libpic32.a(vector41.o)
 .reginfo       0x00000000       0x18 c:/program files (x86)/microchip/xc32/v1.21/bin/../lib/gcc/pic32mx/4.5.2/../../../../pic32mx/lib/size\libpic32.a(vector41.o)
 .pdr           0x00000000       0x20 c:/program files (x86)/microchip/xc32/v1.21/bin/../lib/gcc/pic32mx/4.5.2/../../../../pic32mx/lib/size\libpic32.a(vector41.o)
 .text          0x00000000        0x0 c:/program files (x86)/microchip/xc32/v1.21/bin/../lib/gcc/pic32mx/4.5.2/../../../../pic32mx/lib/size\libpic32.a(vector42.o)
 .data          0x00000000        0x0 c:/program files (x86)/microchip/xc32/v1.21/bin/../lib/gcc/pic32mx/4.5.2/../../../../pic32mx/lib/size\libpic32.a(vector42.o)
 .bss           0x00000000        0x0 c:/program files (x86)/microchip/xc32/v1.21/bin/../lib/gcc/pic32mx/4.5.2/../../../../pic32mx/lib/size\libpic32.a(vector42.o)
 .reginfo       0x00000000       0x18 c:/program files (x86)/microchip/xc32/v1.21/bin/../lib/gcc/pic32mx/4.5.2/../../../../pic32mx/lib/size\libpic32.a(vector42.o)
 .pdr           0x00000000       0x20 c:/program files (x86)/microchip/xc32/v1.21/bin/../lib/gcc/pic32mx/4.5.2/../../../../pic32mx/lib/size\libpic32.a(vector42.o)
 .text          0x00000000        0x0 c:/program files (x86)/microchip/xc32/v1.21/bin/../lib/gcc/pic32mx/4.5.2/../../../../pic32mx/lib/size\libpic32.a(vector43.o)
 .data          0x00000000        0x0 c:/program files (x86)/microchip/xc32/v1.21/bin/../lib/gcc/pic32mx/4.5.2/../../../../pic32mx/lib/size\libpic32.a(vector43.o)
 .bss           0x00000000        0x0 c:/program files (x86)/microchip/xc32/v1.21/bin/../lib/gcc/pic32mx/4.5.2/../../../../pic32mx/lib/size\libpic32.a(vector43.o)
 .reginfo       0x00000000       0x18 c:/program files (x86)/microchip/xc32/v1.21/bin/../lib/gcc/pic32mx/4.5.2/../../../../pic32mx/lib/size\libpic32.a(vector43.o)
 .pdr           0x00000000       0x20 c:/program files (x86)/microchip/xc32/v1.21/bin/../lib/gcc/pic32mx/4.5.2/../../../../pic32mx/lib/size\libpic32.a(vector43.o)
 .text          0x00000000        0x0 c:/program files (x86)/microchip/xc32/v1.21/bin/../lib/gcc/pic32mx/4.5.2/../../../../pic32mx/lib/size\libpic32.a(vector44.o)
 .data          0x00000000        0x0 c:/program files (x86)/microchip/xc32/v1.21/bin/../lib/gcc/pic32mx/4.5.2/../../../../pic32mx/lib/size\libpic32.a(vector44.o)
 .bss           0x00000000        0x0 c:/program files (x86)/microchip/xc32/v1.21/bin/../lib/gcc/pic32mx/4.5.2/../../../../pic32mx/lib/size\libpic32.a(vector44.o)
 .reginfo       0x00000000       0x18 c:/program files (x86)/microchip/xc32/v1.21/bin/../lib/gcc/pic32mx/4.5.2/../../../../pic32mx/lib/size\libpic32.a(vector44.o)
 .pdr           0x00000000       0x20 c:/program files (x86)/microchip/xc32/v1.21/bin/../lib/gcc/pic32mx/4.5.2/../../../../pic32mx/lib/size\libpic32.a(vector44.o)
 .text          0x00000000        0x0 c:/program files (x86)/microchip/xc32/v1.21/bin/../lib/gcc/pic32mx/4.5.2/../../../../pic32mx/lib/size\libpic32.a(vector45.o)
 .data          0x00000000        0x0 c:/program files (x86)/microchip/xc32/v1.21/bin/../lib/gcc/pic32mx/4.5.2/../../../../pic32mx/lib/size\libpic32.a(vector45.o)
 .bss           0x00000000        0x0 c:/program files (x86)/microchip/xc32/v1.21/bin/../lib/gcc/pic32mx/4.5.2/../../../../pic32mx/lib/size\libpic32.a(vector45.o)
 .reginfo       0x00000000       0x18 c:/program files (x86)/microchip/xc32/v1.21/bin/../lib/gcc/pic32mx/4.5.2/../../../../pic32mx/lib/size\libpic32.a(vector45.o)
 .pdr           0x00000000       0x20 c:/program files (x86)/microchip/xc32/v1.21/bin/../lib/gcc/pic32mx/4.5.2/../../../../pic32mx/lib/size\libpic32.a(vector45.o)
 .text          0x00000000        0x0 c:/program files (x86)/microchip/xc32/v1.21/bin/../lib/gcc/pic32mx/4.5.2/../../../../pic32mx/lib/size\libpic32.a(vector46.o)
 .data          0x00000000        0x0 c:/program files (x86)/microchip/xc32/v1.21/bin/../lib/gcc/pic32mx/4.5.2/../../../../pic32mx/lib/size\libpic32.a(vector46.o)
 .bss           0x00000000        0x0 c:/program files (x86)/microchip/xc32/v1.21/bin/../lib/gcc/pic32mx/4.5.2/../../../../pic32mx/lib/size\libpic32.a(vector46.o)
 .reginfo       0x00000000       0x18 c:/program files (x86)/microchip/xc32/v1.21/bin/../lib/gcc/pic32mx/4.5.2/../../../../pic32mx/lib/size\libpic32.a(vector46.o)
 .pdr           0x00000000       0x20 c:/program files (x86)/microchip/xc32/v1.21/bin/../lib/gcc/pic32mx/4.5.2/../../../../pic32mx/lib/size\libpic32.a(vector46.o)
 .text          0x00000000        0x0 c:/program files (x86)/microchip/xc32/v1.21/bin/../lib/gcc/pic32mx/4.5.2/../../../../pic32mx/lib/size\libpic32.a(vector47.o)
 .data          0x00000000        0x0 c:/program files (x86)/microchip/xc32/v1.21/bin/../lib/gcc/pic32mx/4.5.2/../../../../pic32mx/lib/size\libpic32.a(vector47.o)
 .bss           0x00000000        0x0 c:/program files (x86)/microchip/xc32/v1.21/bin/../lib/gcc/pic32mx/4.5.2/../../../../pic32mx/lib/size\libpic32.a(vector47.o)
 .reginfo       0x00000000       0x18 c:/program files (x86)/microchip/xc32/v1.21/bin/../lib/gcc/pic32mx/4.5.2/../../../../pic32mx/lib/size\libpic32.a(vector47.o)
 .pdr           0x00000000       0x20 c:/program files (x86)/microchip/xc32/v1.21/bin/../lib/gcc/pic32mx/4.5.2/../../../../pic32mx/lib/size\libpic32.a(vector47.o)
 .text          0x00000000        0x0 c:/program files (x86)/microchip/xc32/v1.21/bin/../lib/gcc/pic32mx/4.5.2/../../../../pic32mx/lib/size\libpic32.a(vector48.o)
 .data          0x00000000        0x0 c:/program files (x86)/microchip/xc32/v1.21/bin/../lib/gcc/pic32mx/4.5.2/../../../../pic32mx/lib/size\libpic32.a(vector48.o)
 .bss           0x00000000        0x0 c:/program files (x86)/microchip/xc32/v1.21/bin/../lib/gcc/pic32mx/4.5.2/../../../../pic32mx/lib/size\libpic32.a(vector48.o)
 .reginfo       0x00000000       0x18 c:/program files (x86)/microchip/xc32/v1.21/bin/../lib/gcc/pic32mx/4.5.2/../../../../pic32mx/lib/size\libpic32.a(vector48.o)
 .pdr           0x00000000       0x20 c:/program files (x86)/microchip/xc32/v1.21/bin/../lib/gcc/pic32mx/4.5.2/../../../../pic32mx/lib/size\libpic32.a(vector48.o)
 .text          0x00000000        0x0 c:/program files (x86)/microchip/xc32/v1.21/bin/../lib/gcc/pic32mx/4.5.2/../../../../pic32mx/lib/size\libpic32.a(vector49.o)
 .data          0x00000000        0x0 c:/program files (x86)/microchip/xc32/v1.21/bin/../lib/gcc/pic32mx/4.5.2/../../../../pic32mx/lib/size\libpic32.a(vector49.o)
 .bss           0x00000000        0x0 c:/program files (x86)/microchip/xc32/v1.21/bin/../lib/gcc/pic32mx/4.5.2/../../../../pic32mx/lib/size\libpic32.a(vector49.o)
 .reginfo       0x00000000       0x18 c:/program files (x86)/microchip/xc32/v1.21/bin/../lib/gcc/pic32mx/4.5.2/../../../../pic32mx/lib/size\libpic32.a(vector49.o)
 .pdr           0x00000000       0x20 c:/program files (x86)/microchip/xc32/v1.21/bin/../lib/gcc/pic32mx/4.5.2/../../../../pic32mx/lib/size\libpic32.a(vector49.o)
 .text          0x00000000        0x0 c:/program files (x86)/microchip/xc32/v1.21/bin/../lib/gcc/pic32mx/4.5.2/../../../../pic32mx/lib/size\libpic32.a(vector50.o)
 .data          0x00000000        0x0 c:/program files (x86)/microchip/xc32/v1.21/bin/../lib/gcc/pic32mx/4.5.2/../../../../pic32mx/lib/size\libpic32.a(vector50.o)
 .bss           0x00000000        0x0 c:/program files (x86)/microchip/xc32/v1.21/bin/../lib/gcc/pic32mx/4.5.2/../../../../pic32mx/lib/size\libpic32.a(vector50.o)
 .reginfo       0x00000000       0x18 c:/program files (x86)/microchip/xc32/v1.21/bin/../lib/gcc/pic32mx/4.5.2/../../../../pic32mx/lib/size\libpic32.a(vector50.o)
 .pdr           0x00000000       0x20 c:/program files (x86)/microchip/xc32/v1.21/bin/../lib/gcc/pic32mx/4.5.2/../../../../pic32mx/lib/size\libpic32.a(vector50.o)
 .text          0x00000000        0x0 c:/program files (x86)/microchip/xc32/v1.21/bin/../lib/gcc/pic32mx/4.5.2/../../../../pic32mx/lib/size\libpic32.a(vector51.o)
 .data          0x00000000        0x0 c:/program files (x86)/microchip/xc32/v1.21/bin/../lib/gcc/pic32mx/4.5.2/../../../../pic32mx/lib/size\libpic32.a(vector51.o)
 .bss           0x00000000        0x0 c:/program files (x86)/microchip/xc32/v1.21/bin/../lib/gcc/pic32mx/4.5.2/../../../../pic32mx/lib/size\libpic32.a(vector51.o)
 .reginfo       0x00000000       0x18 c:/program files (x86)/microchip/xc32/v1.21/bin/../lib/gcc/pic32mx/4.5.2/../../../../pic32mx/lib/size\libpic32.a(vector51.o)
 .pdr           0x00000000       0x20 c:/program files (x86)/microchip/xc32/v1.21/bin/../lib/gcc/pic32mx/4.5.2/../../../../pic32mx/lib/size\libpic32.a(vector51.o)
 .text          0x00000000        0x0 c:/program files (x86)/microchip/xc32/v1.21/bin/../lib/gcc/pic32mx/4.5.2/../../../../pic32mx/lib/size\libpic32.a(vector52.o)
 .data          0x00000000        0x0 c:/program files (x86)/microchip/xc32/v1.21/bin/../lib/gcc/pic32mx/4.5.2/../../../../pic32mx/lib/size\libpic32.a(vector52.o)
 .bss           0x00000000        0x0 c:/program files (x86)/microchip/xc32/v1.21/bin/../lib/gcc/pic32mx/4.5.2/../../../../pic32mx/lib/size\libpic32.a(vector52.o)
 .reginfo       0x00000000       0x18 c:/program files (x86)/microchip/xc32/v1.21/bin/../lib/gcc/pic32mx/4.5.2/../../../../pic32mx/lib/size\libpic32.a(vector52.o)
 .pdr           0x00000000       0x20 c:/program files (x86)/microchip/xc32/v1.21/bin/../lib/gcc/pic32mx/4.5.2/../../../../pic32mx/lib/size\libpic32.a(vector52.o)
 .text          0x00000000        0x0 c:/program files (x86)/microchip/xc32/v1.21/bin/../lib/gcc/pic32mx/4.5.2/../../../../pic32mx/lib/size\libpic32.a(vector53.o)
 .data          0x00000000        0x0 c:/program files (x86)/microchip/xc32/v1.21/bin/../lib/gcc/pic32mx/4.5.2/../../../../pic32mx/lib/size\libpic32.a(vector53.o)
 .bss           0x00000000        0x0 c:/program files (x86)/microchip/xc32/v1.21/bin/../lib/gcc/pic32mx/4.5.2/../../../../pic32mx/lib/size\libpic32.a(vector53.o)
 .reginfo       0x00000000       0x18 c:/program files (x86)/microchip/xc32/v1.21/bin/../lib/gcc/pic32mx/4.5.2/../../../../pic32mx/lib/size\libpic32.a(vector53.o)
 .pdr           0x00000000       0x20 c:/program files (x86)/microchip/xc32/v1.21/bin/../lib/gcc/pic32mx/4.5.2/../../../../pic32mx/lib/size\libpic32.a(vector53.o)
 .text          0x00000000        0x0 c:/program files (x86)/microchip/xc32/v1.21/bin/../lib/gcc/pic32mx/4.5.2/../../../../pic32mx/lib/size\libpic32.a(vector54.o)
 .data          0x00000000        0x0 c:/program files (x86)/microchip/xc32/v1.21/bin/../lib/gcc/pic32mx/4.5.2/../../../../pic32mx/lib/size\libpic32.a(vector54.o)
 .bss           0x00000000        0x0 c:/program files (x86)/microchip/xc32/v1.21/bin/../lib/gcc/pic32mx/4.5.2/../../../../pic32mx/lib/size\libpic32.a(vector54.o)
 .reginfo       0x00000000       0x18 c:/program files (x86)/microchip/xc32/v1.21/bin/../lib/gcc/pic32mx/4.5.2/../../../../pic32mx/lib/size\libpic32.a(vector54.o)
 .pdr           0x00000000       0x20 c:/program files (x86)/microchip/xc32/v1.21/bin/../lib/gcc/pic32mx/4.5.2/../../../../pic32mx/lib/size\libpic32.a(vector54.o)
 .text          0x00000000        0x0 c:/program files (x86)/microchip/xc32/v1.21/bin/../lib/gcc/pic32mx/4.5.2/../../../../pic32mx/lib/size\libpic32.a(vector55.o)
 .data          0x00000000        0x0 c:/program files (x86)/microchip/xc32/v1.21/bin/../lib/gcc/pic32mx/4.5.2/../../../../pic32mx/lib/size\libpic32.a(vector55.o)
 .bss           0x00000000        0x0 c:/program files (x86)/microchip/xc32/v1.21/bin/../lib/gcc/pic32mx/4.5.2/../../../../pic32mx/lib/size\libpic32.a(vector55.o)
 .reginfo       0x00000000       0x18 c:/program files (x86)/microchip/xc32/v1.21/bin/../lib/gcc/pic32mx/4.5.2/../../../../pic32mx/lib/size\libpic32.a(vector55.o)
 .pdr           0x00000000       0x20 c:/program files (x86)/microchip/xc32/v1.21/bin/../lib/gcc/pic32mx/4.5.2/../../../../pic32mx/lib/size\libpic32.a(vector55.o)
 .text          0x00000000        0x0 c:/program files (x86)/microchip/xc32/v1.21/bin/../lib/gcc/pic32mx/4.5.2/../../../../pic32mx/lib/size\libpic32.a(vector56.o)
 .data          0x00000000        0x0 c:/program files (x86)/microchip/xc32/v1.21/bin/../lib/gcc/pic32mx/4.5.2/../../../../pic32mx/lib/size\libpic32.a(vector56.o)
 .bss           0x00000000        0x0 c:/program files (x86)/microchip/xc32/v1.21/bin/../lib/gcc/pic32mx/4.5.2/../../../../pic32mx/lib/size\libpic32.a(vector56.o)
 .reginfo       0x00000000       0x18 c:/program files (x86)/microchip/xc32/v1.21/bin/../lib/gcc/pic32mx/4.5.2/../../../../pic32mx/lib/size\libpic32.a(vector56.o)
 .pdr           0x00000000       0x20 c:/program files (x86)/microchip/xc32/v1.21/bin/../lib/gcc/pic32mx/4.5.2/../../../../pic32mx/lib/size\libpic32.a(vector56.o)
 .text          0x00000000        0x0 c:/program files (x86)/microchip/xc32/v1.21/bin/../lib/gcc/pic32mx/4.5.2/../../../../pic32mx/lib/size\libpic32.a(vector57.o)
 .data          0x00000000        0x0 c:/program files (x86)/microchip/xc32/v1.21/bin/../lib/gcc/pic32mx/4.5.2/../../../../pic32mx/lib/size\libpic32.a(vector57.o)
 .bss           0x00000000        0x0 c:/program files (x86)/microchip/xc32/v1.21/bin/../lib/gcc/pic32mx/4.5.2/../../../../pic32mx/lib/size\libpic32.a(vector57.o)
 .reginfo       0x00000000       0x18 c:/program files (x86)/microchip/xc32/v1.21/bin/../lib/gcc/pic32mx/4.5.2/../../../../pic32mx/lib/size\libpic32.a(vector57.o)
 .pdr           0x00000000       0x20 c:/program files (x86)/microchip/xc32/v1.21/bin/../lib/gcc/pic32mx/4.5.2/../../../../pic32mx/lib/size\libpic32.a(vector57.o)
 .text          0x00000000        0x0 c:/program files (x86)/microchip/xc32/v1.21/bin/../lib/gcc/pic32mx/4.5.2/../../../../pic32mx/lib/size\libpic32.a(vector58.o)
 .data          0x00000000        0x0 c:/program files (x86)/microchip/xc32/v1.21/bin/../lib/gcc/pic32mx/4.5.2/../../../../pic32mx/lib/size\libpic32.a(vector58.o)
 .bss           0x00000000        0x0 c:/program files (x86)/microchip/xc32/v1.21/bin/../lib/gcc/pic32mx/4.5.2/../../../../pic32mx/lib/size\libpic32.a(vector58.o)
 .reginfo       0x00000000       0x18 c:/program files (x86)/microchip/xc32/v1.21/bin/../lib/gcc/pic32mx/4.5.2/../../../../pic32mx/lib/size\libpic32.a(vector58.o)
 .pdr           0x00000000       0x20 c:/program files (x86)/microchip/xc32/v1.21/bin/../lib/gcc/pic32mx/4.5.2/../../../../pic32mx/lib/size\libpic32.a(vector58.o)
 .text          0x00000000        0x0 c:/program files (x86)/microchip/xc32/v1.21/bin/../lib/gcc/pic32mx/4.5.2/../../../../pic32mx/lib/size\libpic32.a(vector59.o)
 .data          0x00000000        0x0 c:/program files (x86)/microchip/xc32/v1.21/bin/../lib/gcc/pic32mx/4.5.2/../../../../pic32mx/lib/size\libpic32.a(vector59.o)
 .bss           0x00000000        0x0 c:/program files (x86)/microchip/xc32/v1.21/bin/../lib/gcc/pic32mx/4.5.2/../../../../pic32mx/lib/size\libpic32.a(vector59.o)
 .reginfo       0x00000000       0x18 c:/program files (x86)/microchip/xc32/v1.21/bin/../lib/gcc/pic32mx/4.5.2/../../../../pic32mx/lib/size\libpic32.a(vector59.o)
 .pdr           0x00000000       0x20 c:/program files (x86)/microchip/xc32/v1.21/bin/../lib/gcc/pic32mx/4.5.2/../../../../pic32mx/lib/size\libpic32.a(vector59.o)
 .text          0x00000000        0x0 c:/program files (x86)/microchip/xc32/v1.21/bin/../lib/gcc/pic32mx/4.5.2/../../../../pic32mx/lib/size\libpic32.a(vector60.o)
 .data          0x00000000        0x0 c:/program files (x86)/microchip/xc32/v1.21/bin/../lib/gcc/pic32mx/4.5.2/../../../../pic32mx/lib/size\libpic32.a(vector60.o)
 .bss           0x00000000        0x0 c:/program files (x86)/microchip/xc32/v1.21/bin/../lib/gcc/pic32mx/4.5.2/../../../../pic32mx/lib/size\libpic32.a(vector60.o)
 .reginfo       0x00000000       0x18 c:/program files (x86)/microchip/xc32/v1.21/bin/../lib/gcc/pic32mx/4.5.2/../../../../pic32mx/lib/size\libpic32.a(vector60.o)
 .pdr           0x00000000       0x20 c:/program files (x86)/microchip/xc32/v1.21/bin/../lib/gcc/pic32mx/4.5.2/../../../../pic32mx/lib/size\libpic32.a(vector60.o)
 .text          0x00000000        0x0 c:/program files (x86)/microchip/xc32/v1.21/bin/../lib/gcc/pic32mx/4.5.2/../../../../pic32mx/lib/size\libpic32.a(vector61.o)
 .data          0x00000000        0x0 c:/program files (x86)/microchip/xc32/v1.21/bin/../lib/gcc/pic32mx/4.5.2/../../../../pic32mx/lib/size\libpic32.a(vector61.o)
 .bss           0x00000000        0x0 c:/program files (x86)/microchip/xc32/v1.21/bin/../lib/gcc/pic32mx/4.5.2/../../../../pic32mx/lib/size\libpic32.a(vector61.o)
 .reginfo       0x00000000       0x18 c:/program files (x86)/microchip/xc32/v1.21/bin/../lib/gcc/pic32mx/4.5.2/../../../../pic32mx/lib/size\libpic32.a(vector61.o)
 .pdr           0x00000000       0x20 c:/program files (x86)/microchip/xc32/v1.21/bin/../lib/gcc/pic32mx/4.5.2/../../../../pic32mx/lib/size\libpic32.a(vector61.o)
 .text          0x00000000        0x0 c:/program files (x86)/microchip/xc32/v1.21/bin/../lib/gcc/pic32mx/4.5.2/../../../../pic32mx/lib/size\libpic32.a(vector62.o)
 .data          0x00000000        0x0 c:/program files (x86)/microchip/xc32/v1.21/bin/../lib/gcc/pic32mx/4.5.2/../../../../pic32mx/lib/size\libpic32.a(vector62.o)
 .bss           0x00000000        0x0 c:/program files (x86)/microchip/xc32/v1.21/bin/../lib/gcc/pic32mx/4.5.2/../../../../pic32mx/lib/size\libpic32.a(vector62.o)
 .reginfo       0x00000000       0x18 c:/program files (x86)/microchip/xc32/v1.21/bin/../lib/gcc/pic32mx/4.5.2/../../../../pic32mx/lib/size\libpic32.a(vector62.o)
 .pdr           0x00000000       0x20 c:/program files (x86)/microchip/xc32/v1.21/bin/../lib/gcc/pic32mx/4.5.2/../../../../pic32mx/lib/size\libpic32.a(vector62.o)
 .text          0x00000000        0x0 c:/program files (x86)/microchip/xc32/v1.21/bin/../lib/gcc/pic32mx/4.5.2/../../../../pic32mx/lib/size\libpic32.a(vector63.o)
 .data          0x00000000        0x0 c:/program files (x86)/microchip/xc32/v1.21/bin/../lib/gcc/pic32mx/4.5.2/../../../../pic32mx/lib/size\libpic32.a(vector63.o)
 .bss           0x00000000        0x0 c:/program files (x86)/microchip/xc32/v1.21/bin/../lib/gcc/pic32mx/4.5.2/../../../../pic32mx/lib/size\libpic32.a(vector63.o)
 .reginfo       0x00000000       0x18 c:/program files (x86)/microchip/xc32/v1.21/bin/../lib/gcc/pic32mx/4.5.2/../../../../pic32mx/lib/size\libpic32.a(vector63.o)
 .pdr           0x00000000       0x20 c:/program files (x86)/microchip/xc32/v1.21/bin/../lib/gcc/pic32mx/4.5.2/../../../../pic32mx/lib/size\libpic32.a(vector63.o)
 .text          0x00000000        0x0 c:/program files (x86)/microchip/xc32/v1.21/bin/../lib/gcc/pic32mx/4.5.2/../../../../pic32mx/lib/size\libpic32.a(defaultinterrupt.o)
 .data          0x00000000        0x0 c:/program files (x86)/microchip/xc32/v1.21/bin/../lib/gcc/pic32mx/4.5.2/../../../../pic32mx/lib/size\libpic32.a(defaultinterrupt.o)
 .bss           0x00000000        0x0 c:/program files (x86)/microchip/xc32/v1.21/bin/../lib/gcc/pic32mx/4.5.2/../../../../pic32mx/lib/size\libpic32.a(defaultinterrupt.o)
 .reginfo       0x00000000       0x18 c:/program files (x86)/microchip/xc32/v1.21/bin/../lib/gcc/pic32mx/4.5.2/../../../../pic32mx/lib/size\libpic32.a(defaultinterrupt.o)
 .pdr           0x00000000       0x20 c:/program files (x86)/microchip/xc32/v1.21/bin/../lib/gcc/pic32mx/4.5.2/../../../../pic32mx/lib/size\libpic32.a(defaultinterrupt.o)
 .text          0x00000000        0x0 c:/program files (x86)/microchip/xc32/v1.21/bin/../lib/gcc/pic32mx/4.5.2/../../../../pic32mx/lib/size\libc.a(atoi.o)
 .data          0x00000000        0x0 c:/program files (x86)/microchip/xc32/v1.21/bin/../lib/gcc/pic32mx/4.5.2/../../../../pic32mx/lib/size\libc.a(atoi.o)
 .bss           0x00000000        0x0 c:/program files (x86)/microchip/xc32/v1.21/bin/../lib/gcc/pic32mx/4.5.2/../../../../pic32mx/lib/size\libc.a(atoi.o)
 .reginfo       0x00000000       0x18 c:/program files (x86)/microchip/xc32/v1.21/bin/../lib/gcc/pic32mx/4.5.2/../../../../pic32mx/lib/size\libc.a(atoi.o)
 .pdr           0x00000000       0x20 c:/program files (x86)/microchip/xc32/v1.21/bin/../lib/gcc/pic32mx/4.5.2/../../../../pic32mx/lib/size\libc.a(atoi.o)
 .text          0x00000000        0x0 c:/program files (x86)/microchip/xc32/v1.21/bin/../lib/gcc/pic32mx/4.5.2/../../../../pic32mx/lib/size\libc.a(atol.o)
 .data          0x00000000        0x0 c:/program files (x86)/microchip/xc32/v1.21/bin/../lib/gcc/pic32mx/4.5.2/../../../../pic32mx/lib/size\libc.a(atol.o)
 .bss           0x00000000        0x0 c:/program files (x86)/microchip/xc32/v1.21/bin/../lib/gcc/pic32mx/4.5.2/../../../../pic32mx/lib/size\libc.a(atol.o)
 .reginfo       0x00000000       0x18 c:/program files (x86)/microchip/xc32/v1.21/bin/../lib/gcc/pic32mx/4.5.2/../../../../pic32mx/lib/size\libc.a(atol.o)
 .pdr           0x00000000       0x20 c:/program files (x86)/microchip/xc32/v1.21/bin/../lib/gcc/pic32mx/4.5.2/../../../../pic32mx/lib/size\libc.a(atol.o)
 .text          0x00000000        0x0 c:/program files (x86)/microchip/xc32/v1.21/bin/../lib/gcc/pic32mx/4.5.2/../../../../pic32mx/lib/size\libc.a(ctype.o)
 .data          0x00000000        0x0 c:/program files (x86)/microchip/xc32/v1.21/bin/../lib/gcc/pic32mx/4.5.2/../../../../pic32mx/lib/size\libc.a(ctype.o)
 .bss           0x00000000        0x0 c:/program files (x86)/microchip/xc32/v1.21/bin/../lib/gcc/pic32mx/4.5.2/../../../../pic32mx/lib/size\libc.a(ctype.o)
 .reginfo       0x00000000       0x18 c:/program files (x86)/microchip/xc32/v1.21/bin/../lib/gcc/pic32mx/4.5.2/../../../../pic32mx/lib/size\libc.a(ctype.o)
 .pdr           0x00000000        0x0 c:/program files (x86)/microchip/xc32/v1.21/bin/../lib/gcc/pic32mx/4.5.2/../../../../pic32mx/lib/size\libc.a(ctype.o)
 .text          0x00000000        0x0 c:/program files (x86)/microchip/xc32/v1.21/bin/../lib/gcc/pic32mx/4.5.2/../../../../pic32mx/lib/size\libc.a(malloc.o)
 .data          0x00000000        0x0 c:/program files (x86)/microchip/xc32/v1.21/bin/../lib/gcc/pic32mx/4.5.2/../../../../pic32mx/lib/size\libc.a(malloc.o)
 .reginfo       0x00000000       0x18 c:/program files (x86)/microchip/xc32/v1.21/bin/../lib/gcc/pic32mx/4.5.2/../../../../pic32mx/lib/size\libc.a(malloc.o)
 .pdr           0x00000000       0x60 c:/program files (x86)/microchip/xc32/v1.21/bin/../lib/gcc/pic32mx/4.5.2/../../../../pic32mx/lib/size\libc.a(malloc.o)
 .text          0x00000000        0x0 c:/program files (x86)/microchip/xc32/v1.21/bin/../lib/gcc/pic32mx/4.5.2/../../../../pic32mx/lib/size\libc.a(rand.o)
 .data          0x00000000        0x0 c:/program files (x86)/microchip/xc32/v1.21/bin/../lib/gcc/pic32mx/4.5.2/../../../../pic32mx/lib/size\libc.a(rand.o)
 .reginfo       0x00000000       0x18 c:/program files (x86)/microchip/xc32/v1.21/bin/../lib/gcc/pic32mx/4.5.2/../../../../pic32mx/lib/size\libc.a(rand.o)
 .pdr           0x00000000       0x40 c:/program files (x86)/microchip/xc32/v1.21/bin/../lib/gcc/pic32mx/4.5.2/../../../../pic32mx/lib/size\libc.a(rand.o)
 .text          0x00000000        0x0 c:/program files (x86)/microchip/xc32/v1.21/bin/../lib/gcc/pic32mx/4.5.2/../../../../pic32mx/lib/size\libc.a(strcat.o)
 .data          0x00000000        0x0 c:/program files (x86)/microchip/xc32/v1.21/bin/../lib/gcc/pic32mx/4.5.2/../../../../pic32mx/lib/size\libc.a(strcat.o)
 .bss           0x00000000        0x0 c:/program files (x86)/microchip/xc32/v1.21/bin/../lib/gcc/pic32mx/4.5.2/../../../../pic32mx/lib/size\libc.a(strcat.o)
 .reginfo       0x00000000       0x18 c:/program files (x86)/microchip/xc32/v1.21/bin/../lib/gcc/pic32mx/4.5.2/../../../../pic32mx/lib/size\libc.a(strcat.o)
 .pdr           0x00000000       0x20 c:/program files (x86)/microchip/xc32/v1.21/bin/../lib/gcc/pic32mx/4.5.2/../../../../pic32mx/lib/size\libc.a(strcat.o)
 .text          0x00000000        0x0 c:/program files (x86)/microchip/xc32/v1.21/bin/../lib/gcc/pic32mx/4.5.2/../../../../pic32mx/lib/size\libc.a(strchr.o)
 .data          0x00000000        0x0 c:/program files (x86)/microchip/xc32/v1.21/bin/../lib/gcc/pic32mx/4.5.2/../../../../pic32mx/lib/size\libc.a(strchr.o)
 .bss           0x00000000        0x0 c:/program files (x86)/microchip/xc32/v1.21/bin/../lib/gcc/pic32mx/4.5.2/../../../../pic32mx/lib/size\libc.a(strchr.o)
 .reginfo       0x00000000       0x18 c:/program files (x86)/microchip/xc32/v1.21/bin/../lib/gcc/pic32mx/4.5.2/../../../../pic32mx/lib/size\libc.a(strchr.o)
 .pdr           0x00000000       0x20 c:/program files (x86)/microchip/xc32/v1.21/bin/../lib/gcc/pic32mx/4.5.2/../../../../pic32mx/lib/size\libc.a(strchr.o)
 .text          0x00000000        0x0 c:/program files (x86)/microchip/xc32/v1.21/bin/../lib/gcc/pic32mx/4.5.2/../../../../pic32mx/lib/size\libc.a(strncat.o)
 .data          0x00000000        0x0 c:/program files (x86)/microchip/xc32/v1.21/bin/../lib/gcc/pic32mx/4.5.2/../../../../pic32mx/lib/size\libc.a(strncat.o)
 .bss           0x00000000        0x0 c:/program files (x86)/microchip/xc32/v1.21/bin/../lib/gcc/pic32mx/4.5.2/../../../../pic32mx/lib/size\libc.a(strncat.o)
 .reginfo       0x00000000       0x18 c:/program files (x86)/microchip/xc32/v1.21/bin/../lib/gcc/pic32mx/4.5.2/../../../../pic32mx/lib/size\libc.a(strncat.o)
 .pdr           0x00000000       0x20 c:/program files (x86)/microchip/xc32/v1.21/bin/../lib/gcc/pic32mx/4.5.2/../../../../pic32mx/lib/size\libc.a(strncat.o)
 .text          0x00000000        0x0 c:/program files (x86)/microchip/xc32/v1.21/bin/../lib/gcc/pic32mx/4.5.2/../../../../pic32mx/lib/size\libc.a(strncmp.o)
 .data          0x00000000        0x0 c:/program files (x86)/microchip/xc32/v1.21/bin/../lib/gcc/pic32mx/4.5.2/../../../../pic32mx/lib/size\libc.a(strncmp.o)
 .bss           0x00000000        0x0 c:/program files (x86)/microchip/xc32/v1.21/bin/../lib/gcc/pic32mx/4.5.2/../../../../pic32mx/lib/size\libc.a(strncmp.o)
 .reginfo       0x00000000       0x18 c:/program files (x86)/microchip/xc32/v1.21/bin/../lib/gcc/pic32mx/4.5.2/../../../../pic32mx/lib/size\libc.a(strncmp.o)
 .pdr           0x00000000       0x20 c:/program files (x86)/microchip/xc32/v1.21/bin/../lib/gcc/pic32mx/4.5.2/../../../../pic32mx/lib/size\libc.a(strncmp.o)
 .text          0x00000000        0x0 c:/program files (x86)/microchip/xc32/v1.21/bin/../lib/gcc/pic32mx/4.5.2/../../../../pic32mx/lib/size\libc.a(strncpy.o)
 .data          0x00000000        0x0 c:/program files (x86)/microchip/xc32/v1.21/bin/../lib/gcc/pic32mx/4.5.2/../../../../pic32mx/lib/size\libc.a(strncpy.o)
 .bss           0x00000000        0x0 c:/program files (x86)/microchip/xc32/v1.21/bin/../lib/gcc/pic32mx/4.5.2/../../../../pic32mx/lib/size\libc.a(strncpy.o)
 .reginfo       0x00000000       0x18 c:/program files (x86)/microchip/xc32/v1.21/bin/../lib/gcc/pic32mx/4.5.2/../../../../pic32mx/lib/size\libc.a(strncpy.o)
 .pdr           0x00000000       0x20 c:/program files (x86)/microchip/xc32/v1.21/bin/../lib/gcc/pic32mx/4.5.2/../../../../pic32mx/lib/size\libc.a(strncpy.o)
 .text          0x00000000        0x0 c:/program files (x86)/microchip/xc32/v1.21/bin/../lib/gcc/pic32mx/4.5.2/../../../../pic32mx/lib/size\libc.a(strrchr.o)
 .data          0x00000000        0x0 c:/program files (x86)/microchip/xc32/v1.21/bin/../lib/gcc/pic32mx/4.5.2/../../../../pic32mx/lib/size\libc.a(strrchr.o)
 .bss           0x00000000        0x0 c:/program files (x86)/microchip/xc32/v1.21/bin/../lib/gcc/pic32mx/4.5.2/../../../../pic32mx/lib/size\libc.a(strrchr.o)
 .reginfo       0x00000000       0x18 c:/program files (x86)/microchip/xc32/v1.21/bin/../lib/gcc/pic32mx/4.5.2/../../../../pic32mx/lib/size\libc.a(strrchr.o)
 .pdr           0x00000000       0x20 c:/program files (x86)/microchip/xc32/v1.21/bin/../lib/gcc/pic32mx/4.5.2/../../../../pic32mx/lib/size\libc.a(strrchr.o)
 .text.strrchr  0x00000000       0x4c c:/program files (x86)/microchip/xc32/v1.21/bin/../lib/gcc/pic32mx/4.5.2/../../../../pic32mx/lib/size\libc.a(strrchr.o)
 .text          0x00000000        0x0 c:/program files (x86)/microchip/xc32/v1.21/bin/../lib/gcc/pic32mx/4.5.2/../../../../pic32mx/lib/size\libc.a(strstr.o)
 .data          0x00000000        0x0 c:/program files (x86)/microchip/xc32/v1.21/bin/../lib/gcc/pic32mx/4.5.2/../../../../pic32mx/lib/size\libc.a(strstr.o)
 .bss           0x00000000        0x0 c:/program files (x86)/microchip/xc32/v1.21/bin/../lib/gcc/pic32mx/4.5.2/../../../../pic32mx/lib/size\libc.a(strstr.o)
 .reginfo       0x00000000       0x18 c:/program files (x86)/microchip/xc32/v1.21/bin/../lib/gcc/pic32mx/4.5.2/../../../../pic32mx/lib/size\libc.a(strstr.o)
 .pdr           0x00000000       0x20 c:/program files (x86)/microchip/xc32/v1.21/bin/../lib/gcc/pic32mx/4.5.2/../../../../pic32mx/lib/size\libc.a(strstr.o)
 .text          0x00000000        0x0 c:/program files (x86)/microchip/xc32/v1.21/bin/../lib/gcc/pic32mx/4.5.2/../../../../pic32mx/lib/size\libc.a(strtol.o)
 .data          0x00000000        0x0 c:/program files (x86)/microchip/xc32/v1.21/bin/../lib/gcc/pic32mx/4.5.2/../../../../pic32mx/lib/size\libc.a(strtol.o)
 .bss           0x00000000        0x0 c:/program files (x86)/microchip/xc32/v1.21/bin/../lib/gcc/pic32mx/4.5.2/../../../../pic32mx/lib/size\libc.a(strtol.o)
 .reginfo       0x00000000       0x18 c:/program files (x86)/microchip/xc32/v1.21/bin/../lib/gcc/pic32mx/4.5.2/../../../../pic32mx/lib/size\libc.a(strtol.o)
 .pdr           0x00000000       0x40 c:/program files (x86)/microchip/xc32/v1.21/bin/../lib/gcc/pic32mx/4.5.2/../../../../pic32mx/lib/size\libc.a(strtol.o)
 .text          0x00000000        0x0 c:/program files (x86)/microchip/xc32/v1.21/bin/../lib/gcc/pic32mx/4.5.2/../../../../pic32mx/lib/size\libc.a(snprintf_cdnopsuxX.eo)
 .data          0x00000000        0x0 c:/program files (x86)/microchip/xc32/v1.21/bin/../lib/gcc/pic32mx/4.5.2/../../../../pic32mx/lib/size\libc.a(snprintf_cdnopsuxX.eo)
 .bss           0x00000000        0x0 c:/program files (x86)/microchip/xc32/v1.21/bin/../lib/gcc/pic32mx/4.5.2/../../../../pic32mx/lib/size\libc.a(snprintf_cdnopsuxX.eo)
 .reginfo       0x00000000       0x18 c:/program files (x86)/microchip/xc32/v1.21/bin/../lib/gcc/pic32mx/4.5.2/../../../../pic32mx/lib/size\libc.a(snprintf_cdnopsuxX.eo)
 .pdr           0x00000000       0x20 c:/program files (x86)/microchip/xc32/v1.21/bin/../lib/gcc/pic32mx/4.5.2/../../../../pic32mx/lib/size\libc.a(snprintf_cdnopsuxX.eo)
 .text          0x00000000        0x0 c:/program files (x86)/microchip/xc32/v1.21/bin/../lib/gcc/pic32mx/4.5.2/../../../../pic32mx/lib/size\libc.a(sprintf_cdnopsuxX.eo)
 .data          0x00000000        0x0 c:/program files (x86)/microchip/xc32/v1.21/bin/../lib/gcc/pic32mx/4.5.2/../../../../pic32mx/lib/size\libc.a(sprintf_cdnopsuxX.eo)
 .bss           0x00000000        0x0 c:/program files (x86)/microchip/xc32/v1.21/bin/../lib/gcc/pic32mx/4.5.2/../../../../pic32mx/lib/size\libc.a(sprintf_cdnopsuxX.eo)
 .reginfo       0x00000000       0x18 c:/program files (x86)/microchip/xc32/v1.21/bin/../lib/gcc/pic32mx/4.5.2/../../../../pic32mx/lib/size\libc.a(sprintf_cdnopsuxX.eo)
 .pdr           0x00000000       0x20 c:/program files (x86)/microchip/xc32/v1.21/bin/../lib/gcc/pic32mx/4.5.2/../../../../pic32mx/lib/size\libc.a(sprintf_cdnopsuxX.eo)
 .text          0x00000000        0x0 c:/program files (x86)/microchip/xc32/v1.21/bin/../lib/gcc/pic32mx/4.5.2/../../../../pic32mx/lib/size\libc.a(vsnprintf_cdnopsuxX.eo)
 .data          0x00000000        0x0 c:/program files (x86)/microchip/xc32/v1.21/bin/../lib/gcc/pic32mx/4.5.2/../../../../pic32mx/lib/size\libc.a(vsnprintf_cdnopsuxX.eo)
 .bss           0x00000000        0x0 c:/program files (x86)/microchip/xc32/v1.21/bin/../lib/gcc/pic32mx/4.5.2/../../../../pic32mx/lib/size\libc.a(vsnprintf_cdnopsuxX.eo)
 .reginfo       0x00000000       0x18 c:/program files (x86)/microchip/xc32/v1.21/bin/../lib/gcc/pic32mx/4.5.2/../../../../pic32mx/lib/size\libc.a(vsnprintf_cdnopsuxX.eo)
 .pdr           0x00000000       0x20 c:/program files (x86)/microchip/xc32/v1.21/bin/../lib/gcc/pic32mx/4.5.2/../../../../pic32mx/lib/size\libc.a(vsnprintf_cdnopsuxX.eo)
 .text          0x00000000        0x0 c:/program files (x86)/microchip/xc32/v1.21/bin/../lib/gcc/pic32mx/4.5.2/../../../../pic32mx/lib/size\libc.a(vsnprintf.o)
 .data          0x00000000        0x0 c:/program files (x86)/microchip/xc32/v1.21/bin/../lib/gcc/pic32mx/4.5.2/../../../../pic32mx/lib/size\libc.a(vsnprintf.o)
 .bss           0x00000000        0x0 c:/program files (x86)/microchip/xc32/v1.21/bin/../lib/gcc/pic32mx/4.5.2/../../../../pic32mx/lib/size\libc.a(vsnprintf.o)
 .reginfo       0x00000000       0x18 c:/program files (x86)/microchip/xc32/v1.21/bin/../lib/gcc/pic32mx/4.5.2/../../../../pic32mx/lib/size\libc.a(vsnprintf.o)
 .pdr           0x00000000       0x20 c:/program files (x86)/microchip/xc32/v1.21/bin/../lib/gcc/pic32mx/4.5.2/../../../../pic32mx/lib/size\libc.a(vsnprintf.o)
 .text          0x00000000        0x0 c:/program files (x86)/microchip/xc32/v1.21/bin/../lib/gcc/pic32mx/4.5.2/../../../../pic32mx/lib/size\libc.a(ctypef.o)
 .data          0x00000000        0x0 c:/program files (x86)/microchip/xc32/v1.21/bin/../lib/gcc/pic32mx/4.5.2/../../../../pic32mx/lib/size\libc.a(ctypef.o)
 .bss           0x00000000        0x0 c:/program files (x86)/microchip/xc32/v1.21/bin/../lib/gcc/pic32mx/4.5.2/../../../../pic32mx/lib/size\libc.a(ctypef.o)
 .reginfo       0x00000000       0x18 c:/program files (x86)/microchip/xc32/v1.21/bin/../lib/gcc/pic32mx/4.5.2/../../../../pic32mx/lib/size\libc.a(ctypef.o)
 .pdr           0x00000000      0x220 c:/program files (x86)/microchip/xc32/v1.21/bin/../lib/gcc/pic32mx/4.5.2/../../../../pic32mx/lib/size\libc.a(ctypef.o)
 .text.tolower  0x00000000       0x24 c:/program files (x86)/microchip/xc32/v1.21/bin/../lib/gcc/pic32mx/4.5.2/../../../../pic32mx/lib/size\libc.a(ctypef.o)
 .text.isalnum  0x00000000       0x18 c:/program files (x86)/microchip/xc32/v1.21/bin/../lib/gcc/pic32mx/4.5.2/../../../../pic32mx/lib/size\libc.a(ctypef.o)
 .text.isalpha  0x00000000       0x18 c:/program files (x86)/microchip/xc32/v1.21/bin/../lib/gcc/pic32mx/4.5.2/../../../../pic32mx/lib/size\libc.a(ctypef.o)
 .text.isascii  0x00000000        0x8 c:/program files (x86)/microchip/xc32/v1.21/bin/../lib/gcc/pic32mx/4.5.2/../../../../pic32mx/lib/size\libc.a(ctypef.o)
 .text.iscntrl  0x00000000       0x18 c:/program files (x86)/microchip/xc32/v1.21/bin/../lib/gcc/pic32mx/4.5.2/../../../../pic32mx/lib/size\libc.a(ctypef.o)
 .text.isdigit  0x00000000       0x18 c:/program files (x86)/microchip/xc32/v1.21/bin/../lib/gcc/pic32mx/4.5.2/../../../../pic32mx/lib/size\libc.a(ctypef.o)
 .text.isgraph  0x00000000       0x18 c:/program files (x86)/microchip/xc32/v1.21/bin/../lib/gcc/pic32mx/4.5.2/../../../../pic32mx/lib/size\libc.a(ctypef.o)
 .text.islower  0x00000000       0x18 c:/program files (x86)/microchip/xc32/v1.21/bin/../lib/gcc/pic32mx/4.5.2/../../../../pic32mx/lib/size\libc.a(ctypef.o)
 .text.isprint  0x00000000       0x18 c:/program files (x86)/microchip/xc32/v1.21/bin/../lib/gcc/pic32mx/4.5.2/../../../../pic32mx/lib/size\libc.a(ctypef.o)
 .text.ispunct  0x00000000       0x18 c:/program files (x86)/microchip/xc32/v1.21/bin/../lib/gcc/pic32mx/4.5.2/../../../../pic32mx/lib/size\libc.a(ctypef.o)
 .text.isspace  0x00000000       0x18 c:/program files (x86)/microchip/xc32/v1.21/bin/../lib/gcc/pic32mx/4.5.2/../../../../pic32mx/lib/size\libc.a(ctypef.o)
 .text.isupper  0x00000000       0x18 c:/program files (x86)/microchip/xc32/v1.21/bin/../lib/gcc/pic32mx/4.5.2/../../../../pic32mx/lib/size\libc.a(ctypef.o)
 .text.isxdigit
                0x00000000       0x18 c:/program files (x86)/microchip/xc32/v1.21/bin/../lib/gcc/pic32mx/4.5.2/../../../../pic32mx/lib/size\libc.a(ctypef.o)
 .text.toascii  0x00000000        0x8 c:/program files (x86)/microchip/xc32/v1.21/bin/../lib/gcc/pic32mx/4.5.2/../../../../pic32mx/lib/size\libc.a(ctypef.o)
 .text._tolower
                0x00000000        0x8 c:/program files (x86)/microchip/xc32/v1.21/bin/../lib/gcc/pic32mx/4.5.2/../../../../pic32mx/lib/size\libc.a(ctypef.o)
 .text._toupper
                0x00000000        0x8 c:/program files (x86)/microchip/xc32/v1.21/bin/../lib/gcc/pic32mx/4.5.2/../../../../pic32mx/lib/size\libc.a(ctypef.o)
 .text          0x00000000        0x0 c:/program files (x86)/microchip/xc32/v1.21/bin/../lib/gcc/pic32mx/4.5.2/../../../../pic32mx/lib/size\libc.a(doprnt_cdnopsuxX.eo)
 .data          0x00000000        0x0 c:/program files (x86)/microchip/xc32/v1.21/bin/../lib/gcc/pic32mx/4.5.2/../../../../pic32mx/lib/size\libc.a(doprnt_cdnopsuxX.eo)
 .bss           0x00000000        0x0 c:/program files (x86)/microchip/xc32/v1.21/bin/../lib/gcc/pic32mx/4.5.2/../../../../pic32mx/lib/size\libc.a(doprnt_cdnopsuxX.eo)
 .reginfo       0x00000000       0x18 c:/program files (x86)/microchip/xc32/v1.21/bin/../lib/gcc/pic32mx/4.5.2/../../../../pic32mx/lib/size\libc.a(doprnt_cdnopsuxX.eo)
 .pdr           0x00000000       0x20 c:/program files (x86)/microchip/xc32/v1.21/bin/../lib/gcc/pic32mx/4.5.2/../../../../pic32mx/lib/size\libc.a(doprnt_cdnopsuxX.eo)
 .text          0x00000000        0x0 c:/program files (x86)/microchip/xc32/v1.21/bin/../lib/gcc/pic32mx/4.5.2/../../../../pic32mx/lib/size\libc.a(doprnt.o)
 .data          0x00000000        0x0 c:/program files (x86)/microchip/xc32/v1.21/bin/../lib/gcc/pic32mx/4.5.2/../../../../pic32mx/lib/size\libc.a(doprnt.o)
 .bss           0x00000000        0x0 c:/program files (x86)/microchip/xc32/v1.21/bin/../lib/gcc/pic32mx/4.5.2/../../../../pic32mx/lib/size\libc.a(doprnt.o)
 .reginfo       0x00000000       0x18 c:/program files (x86)/microchip/xc32/v1.21/bin/../lib/gcc/pic32mx/4.5.2/../../../../pic32mx/lib/size\libc.a(doprnt.o)
 .pdr           0x00000000       0x60 c:/program files (x86)/microchip/xc32/v1.21/bin/../lib/gcc/pic32mx/4.5.2/../../../../pic32mx/lib/size\libc.a(doprnt.o)
 .text          0x00000000        0x0 c:/program files (x86)/microchip/xc32/v1.21/bin/../lib/gcc/pic32mx/4.5.2/../../../../pic32mx/lib/size\libc.a(_fputc_simple.o)
 .data          0x00000000        0x0 c:/program files (x86)/microchip/xc32/v1.21/bin/../lib/gcc/pic32mx/4.5.2/../../../../pic32mx/lib/size\libc.a(_fputc_simple.o)
 .bss           0x00000000        0x0 c:/program files (x86)/microchip/xc32/v1.21/bin/../lib/gcc/pic32mx/4.5.2/../../../../pic32mx/lib/size\libc.a(_fputc_simple.o)
 .reginfo       0x00000000       0x18 c:/program files (x86)/microchip/xc32/v1.21/bin/../lib/gcc/pic32mx/4.5.2/../../../../pic32mx/lib/size\libc.a(_fputc_simple.o)
 .pdr           0x00000000       0x20 c:/program files (x86)/microchip/xc32/v1.21/bin/../lib/gcc/pic32mx/4.5.2/../../../../pic32mx/lib/size\libc.a(_fputc_simple.o)
 .text          0x00000000        0x0 c:/program files (x86)/microchip/xc32/v1.21/bin/../lib/gcc/pic32mx/4.5.2/../../../../pic32mx/lib/size\libc.a(powersf.o)
 .data          0x00000000        0x0 c:/program files (x86)/microchip/xc32/v1.21/bin/../lib/gcc/pic32mx/4.5.2/../../../../pic32mx/lib/size\libc.a(powersf.o)
 .bss           0x00000000        0x0 c:/program files (x86)/microchip/xc32/v1.21/bin/../lib/gcc/pic32mx/4.5.2/../../../../pic32mx/lib/size\libc.a(powersf.o)
 .reginfo       0x00000000       0x18 c:/program files (x86)/microchip/xc32/v1.21/bin/../lib/gcc/pic32mx/4.5.2/../../../../pic32mx/lib/size\libc.a(powersf.o)
 .pdr           0x00000000        0x0 c:/program files (x86)/microchip/xc32/v1.21/bin/../lib/gcc/pic32mx/4.5.2/../../../../pic32mx/lib/size\libc.a(powersf.o)
 .text          0x00000000        0x0 c:/program files (x86)/microchip/xc32/v1.21/bin/../lib/gcc/pic32mx/4.5.2/../../../../pic32mx/lib/size\libc.a(_iob.o)
 .data          0x00000000       0xa0 c:/program files (x86)/microchip/xc32/v1.21/bin/../lib/gcc/pic32mx/4.5.2/../../../../pic32mx/lib/size\libc.a(_iob.o)
 .reginfo       0x00000000       0x18 c:/program files (x86)/microchip/xc32/v1.21/bin/../lib/gcc/pic32mx/4.5.2/../../../../pic32mx/lib/size\libc.a(_iob.o)
 .pdr           0x00000000        0x0 c:/program files (x86)/microchip/xc32/v1.21/bin/../lib/gcc/pic32mx/4.5.2/../../../../pic32mx/lib/size\libc.a(_iob.o)
 .sdata         0x00000000        0x4 c:/program files (x86)/microchip/xc32/v1.21/bin/../lib/gcc/pic32mx/4.5.2/../../../../pic32mx/lib/size\libc.a(_iob.o)
 .text          0x00000000        0x0 c:/program files (x86)/microchip/xc32/v1.21/bin/../lib/gcc/pic32mx/4.5.2/../../../../pic32mx/lib/size\libc.a(_flsbuf_simple.o)
 .data          0x00000000        0x0 c:/program files (x86)/microchip/xc32/v1.21/bin/../lib/gcc/pic32mx/4.5.2/../../../../pic32mx/lib/size\libc.a(_flsbuf_simple.o)
 .bss           0x00000000        0x0 c:/program files (x86)/microchip/xc32/v1.21/bin/../lib/gcc/pic32mx/4.5.2/../../../../pic32mx/lib/size\libc.a(_flsbuf_simple.o)
 .reginfo       0x00000000       0x18 c:/program files (x86)/microchip/xc32/v1.21/bin/../lib/gcc/pic32mx/4.5.2/../../../../pic32mx/lib/size\libc.a(_flsbuf_simple.o)
 .pdr           0x00000000       0x20 c:/program files (x86)/microchip/xc32/v1.21/bin/../lib/gcc/pic32mx/4.5.2/../../../../pic32mx/lib/size\libc.a(_flsbuf_simple.o)
 .text          0x00000000        0x0 c:/program files (x86)/microchip/xc32/v1.21/bin/../lib/gcc/pic32mx/4.5.2/../../../../pic32mx/lib/size\libpic32.a(sbrk.o)
 .data          0x00000000        0x0 c:/program files (x86)/microchip/xc32/v1.21/bin/../lib/gcc/pic32mx/4.5.2/../../../../pic32mx/lib/size\libpic32.a(sbrk.o)
 .reginfo       0x00000000       0x18 c:/program files (x86)/microchip/xc32/v1.21/bin/../lib/gcc/pic32mx/4.5.2/../../../../pic32mx/lib/size\libpic32.a(sbrk.o)
 .pdr           0x00000000       0xa0 c:/program files (x86)/microchip/xc32/v1.21/bin/../lib/gcc/pic32mx/4.5.2/../../../../pic32mx/lib/size\libpic32.a(sbrk.o)
 .text.getpagesize
                0x00000000        0x8 c:/program files (x86)/microchip/xc32/v1.21/bin/../lib/gcc/pic32mx/4.5.2/../../../../pic32mx/lib/size\libpic32.a(sbrk.o)
 .text          0x00000000        0x0 c:/program files (x86)/microchip/xc32/v1.21/bin/../lib/gcc/pic32mx/4.5.2/../../../../pic32mx/lib/size\libpic32.a(write.o)
 .data          0x00000000        0x0 c:/program files (x86)/microchip/xc32/v1.21/bin/../lib/gcc/pic32mx/4.5.2/../../../../pic32mx/lib/size\libpic32.a(write.o)
 .bss           0x00000000        0x0 c:/program files (x86)/microchip/xc32/v1.21/bin/../lib/gcc/pic32mx/4.5.2/../../../../pic32mx/lib/size\libpic32.a(write.o)
 .reginfo       0x00000000       0x18 c:/program files (x86)/microchip/xc32/v1.21/bin/../lib/gcc/pic32mx/4.5.2/../../../../pic32mx/lib/size\libpic32.a(write.o)
 .pdr           0x00000000       0x20 c:/program files (x86)/microchip/xc32/v1.21/bin/../lib/gcc/pic32mx/4.5.2/../../../../pic32mx/lib/size\libpic32.a(write.o)
 .text          0x00000000        0x0 c:/program files (x86)/microchip/xc32/v1.21/bin/../lib/gcc/pic32mx/4.5.2/../../../../pic32mx/lib/size\libpic32.a(_mon_putc.o)
 .data          0x00000000        0x0 c:/program files (x86)/microchip/xc32/v1.21/bin/../lib/gcc/pic32mx/4.5.2/../../../../pic32mx/lib/size\libpic32.a(_mon_putc.o)
 .bss           0x00000000        0x0 c:/program files (x86)/microchip/xc32/v1.21/bin/../lib/gcc/pic32mx/4.5.2/../../../../pic32mx/lib/size\libpic32.a(_mon_putc.o)
 .reginfo       0x00000000       0x18 c:/program files (x86)/microchip/xc32/v1.21/bin/../lib/gcc/pic32mx/4.5.2/../../../../pic32mx/lib/size\libpic32.a(_mon_putc.o)
 .pdr           0x00000000       0x20 c:/program files (x86)/microchip/xc32/v1.21/bin/../lib/gcc/pic32mx/4.5.2/../../../../pic32mx/lib/size\libpic32.a(_mon_putc.o)
 .text          0x00000000        0x0 c:/program files (x86)/microchip/xc32/v1.21/bin/../lib/gcc/pic32mx/4.5.2/../../../../pic32mx/lib/size\libpic32.a(xc32_uart.o)
 .data          0x00000000        0x0 c:/program files (x86)/microchip/xc32/v1.21/bin/../lib/gcc/pic32mx/4.5.2/../../../../pic32mx/lib/size\libpic32.a(xc32_uart.o)
 .bss           0x00000000        0x0 c:/program files (x86)/microchip/xc32/v1.21/bin/../lib/gcc/pic32mx/4.5.2/../../../../pic32mx/lib/size\libpic32.a(xc32_uart.o)
 .reginfo       0x00000000       0x18 c:/program files (x86)/microchip/xc32/v1.21/bin/../lib/gcc/pic32mx/4.5.2/../../../../pic32mx/lib/size\libpic32.a(xc32_uart.o)
 .pdr           0x00000000        0x0 c:/program files (x86)/microchip/xc32/v1.21/bin/../lib/gcc/pic32mx/4.5.2/../../../../pic32mx/lib/size\libpic32.a(xc32_uart.o)
 .data          0x00000000        0x0 c:/program files (x86)/microchip/xc32/v1.21/bin/../lib/gcc/pic32mx/4.5.2/../../../../pic32mx/lib/size\libm.a(fpmod32.o)
 .bss           0x00000000        0x0 c:/program files (x86)/microchip/xc32/v1.21/bin/../lib/gcc/pic32mx/4.5.2/../../../../pic32mx/lib/size\libm.a(fpmod32.o)
 .reginfo       0x00000000       0x18 c:/program files (x86)/microchip/xc32/v1.21/bin/../lib/gcc/pic32mx/4.5.2/../../../../pic32mx/lib/size\libm.a(fpmod32.o)
 .pdr           0x00000000        0x0 c:/program files (x86)/microchip/xc32/v1.21/bin/../lib/gcc/pic32mx/4.5.2/../../../../pic32mx/lib/size\libm.a(fpmod32.o)
 .data          0x00000000        0x0 c:/program files (x86)/microchip/xc32/v1.21/bin/../lib/gcc/pic32mx/4.5.2/../../../../pic32mx/lib/size\libm.a(fp32.o)
 .bss           0x00000000        0x0 c:/program files (x86)/microchip/xc32/v1.21/bin/../lib/gcc/pic32mx/4.5.2/../../../../pic32mx/lib/size\libm.a(fp32.o)
 .reginfo       0x00000000       0x18 c:/program files (x86)/microchip/xc32/v1.21/bin/../lib/gcc/pic32mx/4.5.2/../../../../pic32mx/lib/size\libm.a(fp32.o)
 .pdr           0x00000000        0x0 c:/program files (x86)/microchip/xc32/v1.21/bin/../lib/gcc/pic32mx/4.5.2/../../../../pic32mx/lib/size\libm.a(fp32.o)
 .text          0x00000000        0x0 c:/program files (x86)/microchip/xc32/v1.21/bin/../lib/gcc/pic32mx/4.5.2/../../../../pic32mx/lib/size\libe.a(_floatdisf.o)
 .data          0x00000000        0x0 c:/program files (x86)/microchip/xc32/v1.21/bin/../lib/gcc/pic32mx/4.5.2/../../../../pic32mx/lib/size\libe.a(_floatdisf.o)
 .bss           0x00000000        0x0 c:/program files (x86)/microchip/xc32/v1.21/bin/../lib/gcc/pic32mx/4.5.2/../../../../pic32mx/lib/size\libe.a(_floatdisf.o)
 .reginfo       0x00000000       0x18 c:/program files (x86)/microchip/xc32/v1.21/bin/../lib/gcc/pic32mx/4.5.2/../../../../pic32mx/lib/size\libe.a(_floatdisf.o)
 .pdr           0x00000000       0x20 c:/program files (x86)/microchip/xc32/v1.21/bin/../lib/gcc/pic32mx/4.5.2/../../../../pic32mx/lib/size\libe.a(_floatdisf.o)
 .data          0x00000000        0x0 c:/program files (x86)/microchip/xc32/v1.21/bin/../lib/gcc/pic32mx/4.5.2/size\libgcc.a(_lshrdi3.o)
 .bss           0x00000000        0x0 c:/program files (x86)/microchip/xc32/v1.21/bin/../lib/gcc/pic32mx/4.5.2/size\libgcc.a(_lshrdi3.o)
 .reginfo       0x00000000       0x18 c:/program files (x86)/microchip/xc32/v1.21/bin/../lib/gcc/pic32mx/4.5.2/size\libgcc.a(_lshrdi3.o)
 .pdr           0x00000000       0x20 c:/program files (x86)/microchip/xc32/v1.21/bin/../lib/gcc/pic32mx/4.5.2/size\libgcc.a(_lshrdi3.o)
 .data          0x00000000        0x0 c:/program files (x86)/microchip/xc32/v1.21/bin/../lib/gcc/pic32mx/4.5.2/size\libgcc.a(_floatundisf.o)
 .bss           0x00000000        0x0 c:/program files (x86)/microchip/xc32/v1.21/bin/../lib/gcc/pic32mx/4.5.2/size\libgcc.a(_floatundisf.o)
 .reginfo       0x00000000       0x18 c:/program files (x86)/microchip/xc32/v1.21/bin/../lib/gcc/pic32mx/4.5.2/size\libgcc.a(_floatundisf.o)
 .pdr           0x00000000       0x20 c:/program files (x86)/microchip/xc32/v1.21/bin/../lib/gcc/pic32mx/4.5.2/size\libgcc.a(_floatundisf.o)
 .data          0x00000000        0x0 c:/program files (x86)/microchip/xc32/v1.21/bin/../lib/gcc/pic32mx/4.5.2/size\libgcc.a(_umoddi3.o)
 .bss           0x00000000        0x0 c:/program files (x86)/microchip/xc32/v1.21/bin/../lib/gcc/pic32mx/4.5.2/size\libgcc.a(_umoddi3.o)
 .reginfo       0x00000000       0x18 c:/program files (x86)/microchip/xc32/v1.21/bin/../lib/gcc/pic32mx/4.5.2/size\libgcc.a(_umoddi3.o)
 .pdr           0x00000000       0x20 c:/program files (x86)/microchip/xc32/v1.21/bin/../lib/gcc/pic32mx/4.5.2/size\libgcc.a(_umoddi3.o)
 .data          0x00000000        0x0 c:/program files (x86)/microchip/xc32/v1.21/bin/../lib/gcc/pic32mx/4.5.2/size\libgcc.a(floatunsisf.o)
 .bss           0x00000000        0x0 c:/program files (x86)/microchip/xc32/v1.21/bin/../lib/gcc/pic32mx/4.5.2/size\libgcc.a(floatunsisf.o)
 .reginfo       0x00000000       0x18 c:/program files (x86)/microchip/xc32/v1.21/bin/../lib/gcc/pic32mx/4.5.2/size\libgcc.a(floatunsisf.o)
 .pdr           0x00000000       0x20 c:/program files (x86)/microchip/xc32/v1.21/bin/../lib/gcc/pic32mx/4.5.2/size\libgcc.a(floatunsisf.o)

Memory Configuration

Name             Origin             Length             Attributes
kseg0_program_mem 0x9d000000         0x00080000         xr
kseg0_boot_mem   0x9fc00490         0x00000970
exception_mem    0x9fc01000         0x00001000
kseg1_boot_mem   0xbfc00000         0x00000490
debug_exec_mem   0xbfc02000         0x00000ff0
config3          0xbfc02ff0         0x00000004
config2          0xbfc02ff4         0x00000004
config1          0xbfc02ff8         0x00000004
config0          0xbfc02ffc         0x00000004
kseg1_data_mem   0xa0000000         0x00020000         w !x
sfrs             0xbf800000         0x00100000
configsfrs       0xbfc02ff0         0x00000010
*default*        0x00000000         0xffffffff

Linker script and memory map

LOAD c:/program files (x86)/microchip/xc32/v1.21/bin/../lib/gcc/pic32mx/4.5.2/../../../../pic32mx/lib/size/crt0.o
LOAD build/default/production/_ext/1293749816/bsp.o
LOAD build/default/production/_ext/101875047/lfsr.o
LOAD build/default/production/_ext/101875047/big_int_helper_c32.o
LOAD build/default/production/_ext/101875047/big_int.o
LOAD build/default/production/_ext/101875047/hashes.o
LOAD build/default/production/_ext/101875047/helpers.o
LOAD build/default/production/_ext/1472/berkeley_tcp_client_demo.o
LOAD build/default/production/_ext/1472/berkeley_tcp_server_demo.o
LOAD build/default/production/_ext/1472/berkeley_udp_client_demo.o
LOAD build/default/production/_ext/1472/generic_tcp_client.o
LOAD build/default/production/_ext/1472/generic_tcp_server.o
LOAD build/default/production/_ext/1472/ping_demo.o
LOAD build/default/production/_ext/1472/smtp_demo.o
LOAD build/default/production/_ext/365611741/system_services.o
LOAD build/default/production/_ext/365611741/system_debug.o
LOAD build/default/production/_ext/365611741/system_random.o
LOAD build/default/production/_ext/365611741/system_command.o
LOAD build/default/production/_ext/365611741/system_userio.o
LOAD build/default/production/_ext/97638081/sys_fs.o
LOAD build/default/production/_ext/97638081/mpfs2.o
LOAD build/default/production/_ext/792872985/usart.o
LOAD build/default/production/_ext/792872985/lcd.o
LOAD build/default/production/_ext/792872985/drv_spi.o
LOAD build/default/production/_ext/792872985/db_appio.o
LOAD build/default/production/_ext/792872985/spi_ram.o
LOAD build/default/production/_ext/792872985/spi_eeprom.o
LOAD build/default/production/_ext/792872985/spi_flash.o
LOAD build/default/production/_ext/792872985/drv_media.o
LOAD build/default/production/_ext/427700826/tcpip_announce.o
LOAD build/default/production/_ext/427700826/http2.o
LOAD build/default/production/_ext/427700826/arcfour.o
LOAD build/default/production/_ext/427700826/arp.o
LOAD build/default/production/_ext/427700826/berkeley_api.o
LOAD build/default/production/_ext/427700826/dhcp.o
LOAD build/default/production/_ext/427700826/dhcps.o
LOAD build/default/production/_ext/427700826/dns.o
LOAD build/default/production/_ext/427700826/dnss.o
LOAD build/default/production/_ext/427700826/dyn_dns.o
LOAD build/default/production/_ext/427700826/enc28_mac.o
LOAD build/default/production/_ext/427700826/enc28j60.o
LOAD build/default/production/_ext/427700826/encs24j600.o
LOAD build/default/production/_ext/427700826/encx24_mac.o
LOAD build/default/production/_ext/427700826/eth_pic32_ext_phy.o
LOAD build/default/production/_ext/427700826/eth_pic32_ext_phy_dp83848.o
LOAD build/default/production/_ext/427700826/eth_pic32_int_mac.o
LOAD build/default/production/_ext/427700826/ftp.o
LOAD build/default/production/_ext/427700826/hash_fnv.o
LOAD build/default/production/_ext/427700826/hash_tbl.o
LOAD build/default/production/_ext/427700826/icmp.o
LOAD build/default/production/_ext/427700826/icmpv6.o
LOAD build/default/production/_ext/427700826/ipv4.o
LOAD build/default/production/_ext/427700826/ipv6.o
LOAD build/default/production/_ext/427700826/mac_events_pic32.o
LOAD build/default/production/_ext/427700826/nbns.o
LOAD build/default/production/_ext/427700826/ndp.o
LOAD build/default/production/_ext/427700826/tcpip_reboot.o
LOAD build/default/production/_ext/427700826/rsa.o
LOAD build/default/production/_ext/427700826/smtp.o
LOAD build/default/production/_ext/427700826/snmp.o
LOAD build/default/production/_ext/427700826/snmpv3.o
LOAD build/default/production/_ext/427700826/snmpv3_usm.o
LOAD build/default/production/_ext/427700826/sntp.o
LOAD build/default/production/_ext/427700826/ssl.o
LOAD build/default/production/_ext/427700826/tcp.o
LOAD build/default/production/_ext/427700826/tcpip_heap_alloc.o
LOAD build/default/production/_ext/427700826/tcpip_storage.o
LOAD build/default/production/_ext/427700826/telnet.o
LOAD build/default/production/_ext/427700826/tftpc.o
LOAD build/default/production/_ext/427700826/udp.o
LOAD build/default/production/_ext/427700826/tcpip_mac_object.o
LOAD build/default/production/_ext/427700826/tcpip_manager.o
LOAD build/default/production/_ext/427700826/tcpip_helpers.o
LOAD build/default/production/_ext/427700826/tcpip_commands.o
LOAD build/default/production/_ext/427700826/iperf.o
LOAD build/default/production/_ext/427700826/tcpip_helper_c32.o
LOAD build/default/production/_ext/427700826/tcpip_notify.o
LOAD build/default/production/_ext/427700826/zero_conf_helper.o
LOAD build/default/production/_ext/427700826/zero_conf_link_local.o
LOAD build/default/production/_ext/427700826/zero_conf_multicast_dns.o
LOAD build/default/production/_ext/334706090/wf_tx_power.o
LOAD build/default/production/_ext/334706090/wf_connect.o
LOAD build/default/production/_ext/334706090/wf_connection_algorithm.o
LOAD build/default/production/_ext/334706090/wf_connection_manager.o
LOAD build/default/production/_ext/334706090/wf_connection_profile.o
LOAD build/default/production/_ext/334706090/wf_easy_config.o
LOAD build/default/production/_ext/334706090/wf_eint.o
LOAD build/default/production/_ext/334706090/wf_event_handler.o
LOAD build/default/production/_ext/334706090/wf_init.o
LOAD build/default/production/_ext/334706090/wf_power_save.o
LOAD build/default/production/_ext/334706090/wf_scan.o
LOAD build/default/production/_ext/334706090/wf_spi.o
LOAD build/default/production/_ext/334706090/mrf24w_mac_pic32.o
LOAD build/default/production/_ext/334706090/mrf24w_events.o
LOAD build/default/production/_ext/334706090/wf_driver_com_24g.o
LOAD build/default/production/_ext/334706090/wf_driver_raw_24g.o
LOAD build/default/production/_ext/334706090/wf_mac_24g.o
LOAD build/default/production/_ext/334706090/wf_mgmt_msg_24g.o
LOAD build/default/production/_ext/334706090/wf_param_msg_24g.o
LOAD build/default/production/_ext/1472/main_demo.o
LOAD build/default/production/_ext/1472/custom_snmp_app.o
LOAD build/default/production/_ext/1472/custom_ssl_cert.o
LOAD build/default/production/_ext/1472/mpfs_img2.o
LOAD build/default/production/_ext/1472/wf_config.o
LOAD build/default/production/_ext/1472/custom_http_app.o
LOAD build/default/production/_ext/1472/tcp6_demo_app.o
                0x00000001                __MPLAB_BUILD = 0x1
                0x00006400                _min_heap_size = 0x6400
                0x00000800                _min_stack_size = 0x800
LOAD c:/program files (x86)/microchip/xc32/v1.21/bin/../lib/gcc/pic32mx/4.5.2/../../../../pic32mx/lib/./proc/32MX795F512L\default_isr_vectors.o
                0x00000400                PROVIDE (_min_stack_size, 0x400)
LOAD c:/program files (x86)/microchip/xc32/v1.21/bin/../lib/gcc/pic32mx/4.5.2/../../../../pic32mx/lib/./proc/32MX795F512L\processor.o
START GROUP
LOAD c:/program files (x86)/microchip/xc32/v1.21/bin/../lib/gcc/pic32mx/4.5.2/../../../../pic32mx/lib/size\libmchp_peripheral.a
END GROUP
START GROUP
LOAD c:/program files (x86)/microchip/xc32/v1.21/bin/../lib/gcc/pic32mx/4.5.2/../../../../pic32mx/lib/size\libmchp_peripheral_32MX795F512L.a
END GROUP
                0x00000001                PROVIDE (_vector_spacing, 0x1)
                0x9fc01000                _ebase_address = 0x9fc01000
                0xbfc00000                _RESET_ADDR = 0xbfc00000
                0xbfc00380                _BEV_EXCPT_ADDR = 0xbfc00380
                0xbfc00480                _DBG_EXCPT_ADDR = 0xbfc00480
                0xbfc02000                _DBG_CODE_ADDR = 0xbfc02000
                0x00000ff0                _DBG_CODE_SIZE = 0xff0
                0x9fc01180                _GEN_EXCPT_ADDR = (_ebase_address + 0x180)

.config_BFC02FF0
 *(.config_BFC02FF0)

.config_BFC02FF4
                0xbfc02ff4        0x4
 *(.config_BFC02FF4)
 .config_BFC02FF4
                0xbfc02ff4        0x4 build/default/production/_ext/1293749816/bsp.o

.config_BFC02FF8
                0xbfc02ff8        0x4
 *(.config_BFC02FF8)
 .config_BFC02FF8
                0xbfc02ff8        0x4 build/default/production/_ext/1293749816/bsp.o

.config_BFC02FFC
                0xbfc02ffc        0x4
 *(.config_BFC02FFC)
 .config_BFC02FFC
                0xbfc02ffc        0x4 build/default/production/_ext/1293749816/bsp.o
                0xbfc02000                PROVIDE (_DBG_CODE_ADDR, 0xbfc02000)
                0x00000ff0                PROVIDE (_DBG_CODE_SIZE, 0xff0)

.reset          0xbfc00000      0x1f4
 *(.reset)
 .reset         0xbfc00000       0x10 c:/program files (x86)/microchip/xc32/v1.21/bin/../lib/gcc/pic32mx/4.5.2/../../../../pic32mx/lib/size/crt0.o
                0xbfc00000                _reset
 *(.reset.startup)
 .reset.startup
                0xbfc00010      0x1e4 c:/program files (x86)/microchip/xc32/v1.21/bin/../lib/gcc/pic32mx/4.5.2/../../../../pic32mx/lib/size/crt0.o

.bev_excpt      0xbfc00380       0x10
 *(.bev_handler)
 .bev_handler   0xbfc00380       0x10 c:/program files (x86)/microchip/xc32/v1.21/bin/../lib/gcc/pic32mx/4.5.2/../../../../pic32mx/lib/size/crt0.o

.dbg_excpt      0xbfc00480        0x0
                0xbfc00480                . = (. + DEFINED (_DEBUGGER)?0x8:0x0)

.dbg_code       0xbfc02000        0x0
                0xbfc02000                . = (. + DEFINED (_DEBUGGER)?_DBG_CODE_SIZE:0x0)

.app_excpt      0x9fc01180       0x10
 *(.gen_handler)
 .gen_handler   0x9fc01180       0x10 c:/program files (x86)/microchip/xc32/v1.21/bin/../lib/gcc/pic32mx/4.5.2/../../../../pic32mx/lib/size/crt0.o

.vector_0       0x9fc01200        0x8
 *(.vector_0)
 .vector_0      0x9fc01200        0x8 build/default/production/_ext/365611741/system_services.o
                0x9fc01200                __vector_dispatch_0
                0x00000001                ASSERT (((_vector_spacing == 0x0) || (SIZEOF (.vector_0) <= (_vector_spacing << 0x5))), function at exception vector 0 too large)

.vector_1       0x9fc01220        0x8
 *(.vector_1)
 .vector_1      0x9fc01220        0x8 c:/program files (x86)/microchip/xc32/v1.21/bin/../lib/gcc/pic32mx/4.5.2/../../../../pic32mx/lib/size\libpic32.a(vector1.o)
                0x9fc01220                __vector_dispatch_1
                0x00000001                ASSERT (((_vector_spacing == 0x0) || (SIZEOF (.vector_1) <= (_vector_spacing << 0x5))), function at exception vector 1 too large)

.vector_2       0x9fc01240        0x8
 *(.vector_2)
 .vector_2      0x9fc01240        0x8 c:/program files (x86)/microchip/xc32/v1.21/bin/../lib/gcc/pic32mx/4.5.2/../../../../pic32mx/lib/size\libpic32.a(vector2.o)
                0x9fc01240                __vector_dispatch_2
                0x00000001                ASSERT (((_vector_spacing == 0x0) || (SIZEOF (.vector_2) <= (_vector_spacing << 0x5))), function at exception vector 2 too large)

.vector_3       0x9fc01260        0x8
 *(.vector_3)
 .vector_3      0x9fc01260        0x8 c:/program files (x86)/microchip/xc32/v1.21/bin/../lib/gcc/pic32mx/4.5.2/../../../../pic32mx/lib/size\libpic32.a(vector3.o)
                0x9fc01260                __vector_dispatch_3
                0x00000001                ASSERT (((_vector_spacing == 0x0) || (SIZEOF (.vector_3) <= (_vector_spacing << 0x5))), function at exception vector 3 too large)

.vector_4       0x9fc01280        0x8
 *(.vector_4)
 .vector_4      0x9fc01280        0x8 c:/program files (x86)/microchip/xc32/v1.21/bin/../lib/gcc/pic32mx/4.5.2/../../../../pic32mx/lib/size\libpic32.a(vector4.o)
                0x9fc01280                __vector_dispatch_4
                0x00000001                ASSERT (((_vector_spacing == 0x0) || (SIZEOF (.vector_4) <= (_vector_spacing << 0x5))), function at exception vector 4 too large)

.vector_5       0x9fc012a0        0x8
 *(.vector_5)
 .vector_5      0x9fc012a0        0x8 c:/program files (x86)/microchip/xc32/v1.21/bin/../lib/gcc/pic32mx/4.5.2/../../../../pic32mx/lib/size\libpic32.a(vector5.o)
                0x9fc012a0                __vector_dispatch_5
                0x00000001                ASSERT (((_vector_spacing == 0x0) || (SIZEOF (.vector_5) <= (_vector_spacing << 0x5))), function at exception vector 5 too large)

.vector_6       0x9fc012c0        0x8
 *(.vector_6)
 .vector_6      0x9fc012c0        0x8 c:/program files (x86)/microchip/xc32/v1.21/bin/../lib/gcc/pic32mx/4.5.2/../../../../pic32mx/lib/size\libpic32.a(vector6.o)
                0x9fc012c0                __vector_dispatch_6
                0x00000001                ASSERT (((_vector_spacing == 0x0) || (SIZEOF (.vector_6) <= (_vector_spacing << 0x5))), function at exception vector 6 too large)

.vector_7       0x9fc012e0        0x8
 *(.vector_7)
 .vector_7      0x9fc012e0        0x8 build/default/production/_ext/365611741/system_services.o
                0x9fc012e0                __vector_dispatch_7
                0x00000001                ASSERT (((_vector_spacing == 0x0) || (SIZEOF (.vector_7) <= (_vector_spacing << 0x5))), function at exception vector 7 too large)

.vector_8       0x9fc01300        0x8
 *(.vector_8)
 .vector_8      0x9fc01300        0x8 c:/program files (x86)/microchip/xc32/v1.21/bin/../lib/gcc/pic32mx/4.5.2/../../../../pic32mx/lib/size\libpic32.a(vector8.o)
                0x9fc01300                __vector_dispatch_8
                0x00000001                ASSERT (((_vector_spacing == 0x0) || (SIZEOF (.vector_8) <= (_vector_spacing << 0x5))), function at exception vector 8 too large)

.vector_9       0x9fc01320        0x8
 *(.vector_9)
 .vector_9      0x9fc01320        0x8 c:/program files (x86)/microchip/xc32/v1.21/bin/../lib/gcc/pic32mx/4.5.2/../../../../pic32mx/lib/size\libpic32.a(vector9.o)
                0x9fc01320                __vector_dispatch_9
                0x00000001                ASSERT (((_vector_spacing == 0x0) || (SIZEOF (.vector_9) <= (_vector_spacing << 0x5))), function at exception vector 9 too large)

.vector_10      0x9fc01340        0x8
 *(.vector_10)
 .vector_10     0x9fc01340        0x8 c:/program files (x86)/microchip/xc32/v1.21/bin/../lib/gcc/pic32mx/4.5.2/../../../../pic32mx/lib/size\libpic32.a(vector10.o)
                0x9fc01340                __vector_dispatch_10
                0x00000001                ASSERT (((_vector_spacing == 0x0) || (SIZEOF (.vector_10) <= (_vector_spacing << 0x5))), function at exception vector 10 too large)

.vector_11      0x9fc01360        0x8
 *(.vector_11)
 .vector_11     0x9fc01360        0x8 c:/program files (x86)/microchip/xc32/v1.21/bin/../lib/gcc/pic32mx/4.5.2/../../../../pic32mx/lib/size\libpic32.a(vector11.o)
                0x9fc01360                __vector_dispatch_11
                0x00000001                ASSERT (((_vector_spacing == 0x0) || (SIZEOF (.vector_11) <= (_vector_spacing << 0x5))), function at exception vector 11 too large)

.vector_12      0x9fc01380        0x8
 *(.vector_12)
 .vector_12     0x9fc01380        0x8 c:/program files (x86)/microchip/xc32/v1.21/bin/../lib/gcc/pic32mx/4.5.2/../../../../pic32mx/lib/size\libpic32.a(vector12.o)
                0x9fc01380                __vector_dispatch_12
                0x00000001                ASSERT (((_vector_spacing == 0x0) || (SIZEOF (.vector_12) <= (_vector_spacing << 0x5))), function at exception vector 12 too large)

.vector_13      0x9fc013a0        0x8
 *(.vector_13)
 .vector_13     0x9fc013a0        0x8 c:/program files (x86)/microchip/xc32/v1.21/bin/../lib/gcc/pic32mx/4.5.2/../../../../pic32mx/lib/size\libpic32.a(vector13.o)
                0x9fc013a0                __vector_dispatch_13
                0x00000001                ASSERT (((_vector_spacing == 0x0) || (SIZEOF (.vector_13) <= (_vector_spacing << 0x5))), function at exception vector 13 too large)

.vector_14      0x9fc013c0        0x8
 *(.vector_14)
 .vector_14     0x9fc013c0        0x8 c:/program files (x86)/microchip/xc32/v1.21/bin/../lib/gcc/pic32mx/4.5.2/../../../../pic32mx/lib/size\libpic32.a(vector14.o)
                0x9fc013c0                __vector_dispatch_14
                0x00000001                ASSERT (((_vector_spacing == 0x0) || (SIZEOF (.vector_14) <= (_vector_spacing << 0x5))), function at exception vector 14 too large)

.vector_15      0x9fc013e0        0x8
 *(.vector_15)
 .vector_15     0x9fc013e0        0x8 build/default/production/_ext/365611741/system_services.o
                0x9fc013e0                __vector_dispatch_15
                0x00000001                ASSERT (((_vector_spacing == 0x0) || (SIZEOF (.vector_15) <= (_vector_spacing << 0x5))), function at exception vector 15 too large)

.vector_16      0x9fc01400        0x8
 *(.vector_16)
 .vector_16     0x9fc01400        0x8 c:/program files (x86)/microchip/xc32/v1.21/bin/../lib/gcc/pic32mx/4.5.2/../../../../pic32mx/lib/size\libpic32.a(vector16.o)
                0x9fc01400                __vector_dispatch_16
                0x00000001                ASSERT (((_vector_spacing == 0x0) || (SIZEOF (.vector_16) <= (_vector_spacing << 0x5))), function at exception vector 16 too large)

.vector_17      0x9fc01420        0x8
 *(.vector_17)
 .vector_17     0x9fc01420        0x8 c:/program files (x86)/microchip/xc32/v1.21/bin/../lib/gcc/pic32mx/4.5.2/../../../../pic32mx/lib/size\libpic32.a(vector17.o)
                0x9fc01420                __vector_dispatch_17
                0x00000001                ASSERT (((_vector_spacing == 0x0) || (SIZEOF (.vector_17) <= (_vector_spacing << 0x5))), function at exception vector 17 too large)

.vector_18      0x9fc01440        0x8
 *(.vector_18)
 .vector_18     0x9fc01440        0x8 c:/program files (x86)/microchip/xc32/v1.21/bin/../lib/gcc/pic32mx/4.5.2/../../../../pic32mx/lib/size\libpic32.a(vector18.o)
                0x9fc01440                __vector_dispatch_18
                0x00000001                ASSERT (((_vector_spacing == 0x0) || (SIZEOF (.vector_18) <= (_vector_spacing << 0x5))), function at exception vector 18 too large)

.vector_19      0x9fc01460        0x8
 *(.vector_19)
 .vector_19     0x9fc01460        0x8 c:/program files (x86)/microchip/xc32/v1.21/bin/../lib/gcc/pic32mx/4.5.2/../../../../pic32mx/lib/size\libpic32.a(vector19.o)
                0x9fc01460                __vector_dispatch_19
                0x00000001                ASSERT (((_vector_spacing == 0x0) || (SIZEOF (.vector_19) <= (_vector_spacing << 0x5))), function at exception vector 19 too large)

.vector_20      0x9fc01480        0x8
 *(.vector_20)
 .vector_20     0x9fc01480        0x8 c:/program files (x86)/microchip/xc32/v1.21/bin/../lib/gcc/pic32mx/4.5.2/../../../../pic32mx/lib/size\libpic32.a(vector20.o)
                0x9fc01480                __vector_dispatch_20
                0x00000001                ASSERT (((_vector_spacing == 0x0) || (SIZEOF (.vector_20) <= (_vector_spacing << 0x5))), function at exception vector 20 too large)

.vector_21      0x9fc014a0        0x8
 *(.vector_21)
 .vector_21     0x9fc014a0        0x8 c:/program files (x86)/microchip/xc32/v1.21/bin/../lib/gcc/pic32mx/4.5.2/../../../../pic32mx/lib/size\libpic32.a(vector21.o)
                0x9fc014a0                __vector_dispatch_21
                0x00000001                ASSERT (((_vector_spacing == 0x0) || (SIZEOF (.vector_21) <= (_vector_spacing << 0x5))), function at exception vector 21 too large)

.vector_22      0x9fc014c0        0x8
 *(.vector_22)
 .vector_22     0x9fc014c0        0x8 c:/program files (x86)/microchip/xc32/v1.21/bin/../lib/gcc/pic32mx/4.5.2/../../../../pic32mx/lib/size\libpic32.a(vector22.o)
                0x9fc014c0                __vector_dispatch_22
                0x00000001                ASSERT (((_vector_spacing == 0x0) || (SIZEOF (.vector_22) <= (_vector_spacing << 0x5))), function at exception vector 22 too large)

.vector_23      0x9fc014e0        0x8
 *(.vector_23)
 .vector_23     0x9fc014e0        0x8 c:/program files (x86)/microchip/xc32/v1.21/bin/../lib/gcc/pic32mx/4.5.2/../../../../pic32mx/lib/size\libpic32.a(vector23.o)
                0x9fc014e0                __vector_dispatch_23
                0x00000001                ASSERT (((_vector_spacing == 0x0) || (SIZEOF (.vector_23) <= (_vector_spacing << 0x5))), function at exception vector 23 too large)

.vector_24      0x9fc01500        0x8
 *(.vector_24)
 .vector_24     0x9fc01500        0x8 c:/program files (x86)/microchip/xc32/v1.21/bin/../lib/gcc/pic32mx/4.5.2/../../../../pic32mx/lib/size\libpic32.a(vector24.o)
                0x9fc01500                __vector_dispatch_24
                0x00000001                ASSERT (((_vector_spacing == 0x0) || (SIZEOF (.vector_24) <= (_vector_spacing << 0x5))), function at exception vector 24 too large)

.vector_25      0x9fc01520        0x8
 *(.vector_25)
 .vector_25     0x9fc01520        0x8 c:/program files (x86)/microchip/xc32/v1.21/bin/../lib/gcc/pic32mx/4.5.2/../../../../pic32mx/lib/size\libpic32.a(vector25.o)
                0x9fc01520                __vector_dispatch_25
                0x00000001                ASSERT (((_vector_spacing == 0x0) || (SIZEOF (.vector_25) <= (_vector_spacing << 0x5))), function at exception vector 25 too large)

.vector_26      0x9fc01540        0x8
 *(.vector_26)
 .vector_26     0x9fc01540        0x8 build/default/production/_ext/365611741/system_services.o
                0x9fc01540                __vector_dispatch_26
                0x00000001                ASSERT (((_vector_spacing == 0x0) || (SIZEOF (.vector_26) <= (_vector_spacing << 0x5))), function at exception vector 26 too large)

.vector_27      0x9fc01560        0x8
 *(.vector_27)
 .vector_27     0x9fc01560        0x8 c:/program files (x86)/microchip/xc32/v1.21/bin/../lib/gcc/pic32mx/4.5.2/../../../../pic32mx/lib/size\libpic32.a(vector27.o)
                0x9fc01560                __vector_dispatch_27
                0x00000001                ASSERT (((_vector_spacing == 0x0) || (SIZEOF (.vector_27) <= (_vector_spacing << 0x5))), function at exception vector 27 too large)

.vector_28      0x9fc01580        0x8
 *(.vector_28)
 .vector_28     0x9fc01580        0x8 c:/program files (x86)/microchip/xc32/v1.21/bin/../lib/gcc/pic32mx/4.5.2/../../../../pic32mx/lib/size\libpic32.a(vector28.o)
                0x9fc01580                __vector_dispatch_28
                0x00000001                ASSERT (((_vector_spacing == 0x0) || (SIZEOF (.vector_28) <= (_vector_spacing << 0x5))), function at exception vector 28 too large)

.vector_29      0x9fc015a0        0x8
 *(.vector_29)
 .vector_29     0x9fc015a0        0x8 c:/program files (x86)/microchip/xc32/v1.21/bin/../lib/gcc/pic32mx/4.5.2/../../../../pic32mx/lib/size\libpic32.a(vector29.o)
                0x9fc015a0                __vector_dispatch_29
                0x00000001                ASSERT (((_vector_spacing == 0x0) || (SIZEOF (.vector_29) <= (_vector_spacing << 0x5))), function at exception vector 29 too large)

.vector_30      0x9fc015c0        0x8
 *(.vector_30)
 .vector_30     0x9fc015c0        0x8 c:/program files (x86)/microchip/xc32/v1.21/bin/../lib/gcc/pic32mx/4.5.2/../../../../pic32mx/lib/size\libpic32.a(vector30.o)
                0x9fc015c0                __vector_dispatch_30
                0x00000001                ASSERT (((_vector_spacing == 0x0) || (SIZEOF (.vector_30) <= (_vector_spacing << 0x5))), function at exception vector 30 too large)

.vector_31      0x9fc015e0        0x8
 *(.vector_31)
 .vector_31     0x9fc015e0        0x8 c:/program files (x86)/microchip/xc32/v1.21/bin/../lib/gcc/pic32mx/4.5.2/../../../../pic32mx/lib/size\libpic32.a(vector31.o)
                0x9fc015e0                __vector_dispatch_31
                0x00000001                ASSERT (((_vector_spacing == 0x0) || (SIZEOF (.vector_31) <= (_vector_spacing << 0x5))), function at exception vector 31 too large)

.vector_32      0x9fc01600        0x8
 *(.vector_32)
 .vector_32     0x9fc01600        0x8 c:/program files (x86)/microchip/xc32/v1.21/bin/../lib/gcc/pic32mx/4.5.2/../../../../pic32mx/lib/size\libpic32.a(vector32.o)
                0x9fc01600                __vector_dispatch_32
                0x00000001                ASSERT (((_vector_spacing == 0x0) || (SIZEOF (.vector_32) <= (_vector_spacing << 0x5))), function at exception vector 32 too large)

.vector_33      0x9fc01620        0x8
 *(.vector_33)
 .vector_33     0x9fc01620        0x8 c:/program files (x86)/microchip/xc32/v1.21/bin/../lib/gcc/pic32mx/4.5.2/../../../../pic32mx/lib/size\libpic32.a(vector33.o)
                0x9fc01620                __vector_dispatch_33
                0x00000001                ASSERT (((_vector_spacing == 0x0) || (SIZEOF (.vector_33) <= (_vector_spacing << 0x5))), function at exception vector 33 too large)

.vector_34      0x9fc01640        0x8
 *(.vector_34)
 .vector_34     0x9fc01640        0x8 c:/program files (x86)/microchip/xc32/v1.21/bin/../lib/gcc/pic32mx/4.5.2/../../../../pic32mx/lib/size\libpic32.a(vector34.o)
                0x9fc01640                __vector_dispatch_34
                0x00000001                ASSERT (((_vector_spacing == 0x0) || (SIZEOF (.vector_34) <= (_vector_spacing << 0x5))), function at exception vector 34 too large)

.vector_35      0x9fc01660        0x8
 *(.vector_35)
 .vector_35     0x9fc01660        0x8 c:/program files (x86)/microchip/xc32/v1.21/bin/../lib/gcc/pic32mx/4.5.2/../../../../pic32mx/lib/size\libpic32.a(vector35.o)
                0x9fc01660                __vector_dispatch_35
                0x00000001                ASSERT (((_vector_spacing == 0x0) || (SIZEOF (.vector_35) <= (_vector_spacing << 0x5))), function at exception vector 35 too large)

.vector_36      0x9fc01680        0x8
 *(.vector_36)
 .vector_36     0x9fc01680        0x8 c:/program files (x86)/microchip/xc32/v1.21/bin/../lib/gcc/pic32mx/4.5.2/../../../../pic32mx/lib/size\libpic32.a(vector36.o)
                0x9fc01680                __vector_dispatch_36
                0x00000001                ASSERT (((_vector_spacing == 0x0) || (SIZEOF (.vector_36) <= (_vector_spacing << 0x5))), function at exception vector 36 too large)

.vector_37      0x9fc016a0        0x8
 *(.vector_37)
 .vector_37     0x9fc016a0        0x8 c:/program files (x86)/microchip/xc32/v1.21/bin/../lib/gcc/pic32mx/4.5.2/../../../../pic32mx/lib/size\libpic32.a(vector37.o)
                0x9fc016a0                __vector_dispatch_37
                0x00000001                ASSERT (((_vector_spacing == 0x0) || (SIZEOF (.vector_37) <= (_vector_spacing << 0x5))), function at exception vector 37 too large)

.vector_38      0x9fc016c0        0x8
 *(.vector_38)
 .vector_38     0x9fc016c0        0x8 c:/program files (x86)/microchip/xc32/v1.21/bin/../lib/gcc/pic32mx/4.5.2/../../../../pic32mx/lib/size\libpic32.a(vector38.o)
                0x9fc016c0                __vector_dispatch_38
                0x00000001                ASSERT (((_vector_spacing == 0x0) || (SIZEOF (.vector_38) <= (_vector_spacing << 0x5))), function at exception vector 38 too large)

.vector_39      0x9fc016e0        0x8
 *(.vector_39)
 .vector_39     0x9fc016e0        0x8 c:/program files (x86)/microchip/xc32/v1.21/bin/../lib/gcc/pic32mx/4.5.2/../../../../pic32mx/lib/size\libpic32.a(vector39.o)
                0x9fc016e0                __vector_dispatch_39
                0x00000001                ASSERT (((_vector_spacing == 0x0) || (SIZEOF (.vector_39) <= (_vector_spacing << 0x5))), function at exception vector 39 too large)

.vector_40      0x9fc01700        0x8
 *(.vector_40)
 .vector_40     0x9fc01700        0x8 c:/program files (x86)/microchip/xc32/v1.21/bin/../lib/gcc/pic32mx/4.5.2/../../../../pic32mx/lib/size\libpic32.a(vector40.o)
                0x9fc01700                __vector_dispatch_40
                0x00000001                ASSERT (((_vector_spacing == 0x0) || (SIZEOF (.vector_40) <= (_vector_spacing << 0x5))), function at exception vector 40 too large)

.vector_41      0x9fc01720        0x8
 *(.vector_41)
 .vector_41     0x9fc01720        0x8 c:/program files (x86)/microchip/xc32/v1.21/bin/../lib/gcc/pic32mx/4.5.2/../../../../pic32mx/lib/size\libpic32.a(vector41.o)
                0x9fc01720                __vector_dispatch_41
                0x00000001                ASSERT (((_vector_spacing == 0x0) || (SIZEOF (.vector_41) <= (_vector_spacing << 0x5))), function at exception vector 41 too large)

.vector_42      0x9fc01740        0x8
 *(.vector_42)
 .vector_42     0x9fc01740        0x8 c:/program files (x86)/microchip/xc32/v1.21/bin/../lib/gcc/pic32mx/4.5.2/../../../../pic32mx/lib/size\libpic32.a(vector42.o)
                0x9fc01740                __vector_dispatch_42
                0x00000001                ASSERT (((_vector_spacing == 0x0) || (SIZEOF (.vector_42) <= (_vector_spacing << 0x5))), function at exception vector 42 too large)

.vector_43      0x9fc01760        0x8
 *(.vector_43)
 .vector_43     0x9fc01760        0x8 c:/program files (x86)/microchip/xc32/v1.21/bin/../lib/gcc/pic32mx/4.5.2/../../../../pic32mx/lib/size\libpic32.a(vector43.o)
                0x9fc01760                __vector_dispatch_43
                0x00000001                ASSERT (((_vector_spacing == 0x0) || (SIZEOF (.vector_43) <= (_vector_spacing << 0x5))), function at exception vector 43 too large)

.vector_44      0x9fc01780        0x8
 *(.vector_44)
 .vector_44     0x9fc01780        0x8 c:/program files (x86)/microchip/xc32/v1.21/bin/../lib/gcc/pic32mx/4.5.2/../../../../pic32mx/lib/size\libpic32.a(vector44.o)
                0x9fc01780                __vector_dispatch_44
                0x00000001                ASSERT (((_vector_spacing == 0x0) || (SIZEOF (.vector_44) <= (_vector_spacing << 0x5))), function at exception vector 44 too large)

.vector_45      0x9fc017a0        0x8
 *(.vector_45)
 .vector_45     0x9fc017a0        0x8 c:/program files (x86)/microchip/xc32/v1.21/bin/../lib/gcc/pic32mx/4.5.2/../../../../pic32mx/lib/size\libpic32.a(vector45.o)
                0x9fc017a0                __vector_dispatch_45
                0x00000001                ASSERT (((_vector_spacing == 0x0) || (SIZEOF (.vector_45) <= (_vector_spacing << 0x5))), function at exception vector 45 too large)

.vector_46      0x9fc017c0        0x8
 *(.vector_46)
 .vector_46     0x9fc017c0        0x8 c:/program files (x86)/microchip/xc32/v1.21/bin/../lib/gcc/pic32mx/4.5.2/../../../../pic32mx/lib/size\libpic32.a(vector46.o)
                0x9fc017c0                __vector_dispatch_46
                0x00000001                ASSERT (((_vector_spacing == 0x0) || (SIZEOF (.vector_46) <= (_vector_spacing << 0x5))), function at exception vector 46 too large)

.vector_47      0x9fc017e0        0x8
 *(.vector_47)
 .vector_47     0x9fc017e0        0x8 c:/program files (x86)/microchip/xc32/v1.21/bin/../lib/gcc/pic32mx/4.5.2/../../../../pic32mx/lib/size\libpic32.a(vector47.o)
                0x9fc017e0                __vector_dispatch_47
                0x00000001                ASSERT (((_vector_spacing == 0x0) || (SIZEOF (.vector_47) <= (_vector_spacing << 0x5))), function at exception vector 47 too large)

.vector_48      0x9fc01800        0x8
 *(.vector_48)
 .vector_48     0x9fc01800        0x8 c:/program files (x86)/microchip/xc32/v1.21/bin/../lib/gcc/pic32mx/4.5.2/../../../../pic32mx/lib/size\libpic32.a(vector48.o)
                0x9fc01800                __vector_dispatch_48
                0x00000001                ASSERT (((_vector_spacing == 0x0) || (SIZEOF (.vector_48) <= (_vector_spacing << 0x5))), function at exception vector 48 too large)

.vector_49      0x9fc01820        0x8
 *(.vector_49)
 .vector_49     0x9fc01820        0x8 c:/program files (x86)/microchip/xc32/v1.21/bin/../lib/gcc/pic32mx/4.5.2/../../../../pic32mx/lib/size\libpic32.a(vector49.o)
                0x9fc01820                __vector_dispatch_49
                0x00000001                ASSERT (((_vector_spacing == 0x0) || (SIZEOF (.vector_49) <= (_vector_spacing << 0x5))), function at exception vector 49 too large)

.vector_50      0x9fc01840        0x8
 *(.vector_50)
 .vector_50     0x9fc01840        0x8 c:/program files (x86)/microchip/xc32/v1.21/bin/../lib/gcc/pic32mx/4.5.2/../../../../pic32mx/lib/size\libpic32.a(vector50.o)
                0x9fc01840                __vector_dispatch_50
                0x00000001                ASSERT (((_vector_spacing == 0x0) || (SIZEOF (.vector_50) <= (_vector_spacing << 0x5))), function at exception vector 50 too large)

.vector_51      0x9fc01860        0x8
 *(.vector_51)
 .vector_51     0x9fc01860        0x8 c:/program files (x86)/microchip/xc32/v1.21/bin/../lib/gcc/pic32mx/4.5.2/../../../../pic32mx/lib/size\libpic32.a(vector51.o)
                0x9fc01860                __vector_dispatch_51
                0x00000001                ASSERT (((_vector_spacing == 0x0) || (SIZEOF (.vector_51) <= (_vector_spacing << 0x5))), function at exception vector 51 too large)

.vector_52      0x9fc01880        0x8
 *(.vector_52)
 .vector_52     0x9fc01880        0x8 c:/program files (x86)/microchip/xc32/v1.21/bin/../lib/gcc/pic32mx/4.5.2/../../../../pic32mx/lib/size\libpic32.a(vector52.o)
                0x9fc01880                __vector_dispatch_52
                0x00000001                ASSERT (((_vector_spacing == 0x0) || (SIZEOF (.vector_52) <= (_vector_spacing << 0x5))), function at exception vector 52 too large)

.vector_53      0x9fc018a0        0x8
 *(.vector_53)
 .vector_53     0x9fc018a0        0x8 c:/program files (x86)/microchip/xc32/v1.21/bin/../lib/gcc/pic32mx/4.5.2/../../../../pic32mx/lib/size\libpic32.a(vector53.o)
                0x9fc018a0                __vector_dispatch_53
                0x00000001                ASSERT (((_vector_spacing == 0x0) || (SIZEOF (.vector_53) <= (_vector_spacing << 0x5))), function at exception vector 53 too large)

.vector_54      0x9fc018c0        0x8
 *(.vector_54)
 .vector_54     0x9fc018c0        0x8 c:/program files (x86)/microchip/xc32/v1.21/bin/../lib/gcc/pic32mx/4.5.2/../../../../pic32mx/lib/size\libpic32.a(vector54.o)
                0x9fc018c0                __vector_dispatch_54
                0x00000001                ASSERT (((_vector_spacing == 0x0) || (SIZEOF (.vector_54) <= (_vector_spacing << 0x5))), function at exception vector 54 too large)

.vector_55      0x9fc018e0        0x8
 *(.vector_55)
 .vector_55     0x9fc018e0        0x8 c:/program files (x86)/microchip/xc32/v1.21/bin/../lib/gcc/pic32mx/4.5.2/../../../../pic32mx/lib/size\libpic32.a(vector55.o)
                0x9fc018e0                __vector_dispatch_55
                0x00000001                ASSERT (((_vector_spacing == 0x0) || (SIZEOF (.vector_55) <= (_vector_spacing << 0x5))), function at exception vector 55 too large)

.vector_56      0x9fc01900        0x8
 *(.vector_56)
 .vector_56     0x9fc01900        0x8 c:/program files (x86)/microchip/xc32/v1.21/bin/../lib/gcc/pic32mx/4.5.2/../../../../pic32mx/lib/size\libpic32.a(vector56.o)
                0x9fc01900                __vector_dispatch_56
                0x00000001                ASSERT (((_vector_spacing == 0x0) || (SIZEOF (.vector_56) <= (_vector_spacing << 0x5))), function at exception vector 56 too large)

.vector_57      0x9fc01920        0x8
 *(.vector_57)
 .vector_57     0x9fc01920        0x8 c:/program files (x86)/microchip/xc32/v1.21/bin/../lib/gcc/pic32mx/4.5.2/../../../../pic32mx/lib/size\libpic32.a(vector57.o)
                0x9fc01920                __vector_dispatch_57
                0x00000001                ASSERT (((_vector_spacing == 0x0) || (SIZEOF (.vector_57) <= (_vector_spacing << 0x5))), function at exception vector 57 too large)

.vector_58      0x9fc01940        0x8
 *(.vector_58)
 .vector_58     0x9fc01940        0x8 c:/program files (x86)/microchip/xc32/v1.21/bin/../lib/gcc/pic32mx/4.5.2/../../../../pic32mx/lib/size\libpic32.a(vector58.o)
                0x9fc01940                __vector_dispatch_58
                0x00000001                ASSERT (((_vector_spacing == 0x0) || (SIZEOF (.vector_58) <= (_vector_spacing << 0x5))), function at exception vector 58 too large)

.vector_59      0x9fc01960        0x8
 *(.vector_59)
 .vector_59     0x9fc01960        0x8 c:/program files (x86)/microchip/xc32/v1.21/bin/../lib/gcc/pic32mx/4.5.2/../../../../pic32mx/lib/size\libpic32.a(vector59.o)
                0x9fc01960                __vector_dispatch_59
                0x00000001                ASSERT (((_vector_spacing == 0x0) || (SIZEOF (.vector_59) <= (_vector_spacing << 0x5))), function at exception vector 59 too large)

.vector_60      0x9fc01980        0x8
 *(.vector_60)
 .vector_60     0x9fc01980        0x8 c:/program files (x86)/microchip/xc32/v1.21/bin/../lib/gcc/pic32mx/4.5.2/../../../../pic32mx/lib/size\libpic32.a(vector60.o)
                0x9fc01980                __vector_dispatch_60
                0x00000001                ASSERT (((_vector_spacing == 0x0) || (SIZEOF (.vector_60) <= (_vector_spacing << 0x5))), function at exception vector 60 too large)

.vector_61      0x9fc019a0        0x8
 *(.vector_61)
 .vector_61     0x9fc019a0        0x8 c:/program files (x86)/microchip/xc32/v1.21/bin/../lib/gcc/pic32mx/4.5.2/../../../../pic32mx/lib/size\libpic32.a(vector61.o)
                0x9fc019a0                __vector_dispatch_61
                0x00000001                ASSERT (((_vector_spacing == 0x0) || (SIZEOF (.vector_61) <= (_vector_spacing << 0x5))), function at exception vector 61 too large)

.vector_62      0x9fc019c0        0x8
 *(.vector_62)
 .vector_62     0x9fc019c0        0x8 c:/program files (x86)/microchip/xc32/v1.21/bin/../lib/gcc/pic32mx/4.5.2/../../../../pic32mx/lib/size\libpic32.a(vector62.o)
                0x9fc019c0                __vector_dispatch_62
                0x00000001                ASSERT (((_vector_spacing == 0x0) || (SIZEOF (.vector_62) <= (_vector_spacing << 0x5))), function at exception vector 62 too large)

.vector_63      0x9fc019e0        0x8
 *(.vector_63)
 .vector_63     0x9fc019e0        0x8 c:/program files (x86)/microchip/xc32/v1.21/bin/../lib/gcc/pic32mx/4.5.2/../../../../pic32mx/lib/size\libpic32.a(vector63.o)
                0x9fc019e0                __vector_dispatch_63
                0x00000001                ASSERT (((_vector_spacing == 0x0) || (SIZEOF (.vector_63) <= (_vector_spacing << 0x5))), function at exception vector 63 too large)

.startup
 *(.startup)

.text           0x9d000000        0x0
 *(.stub .gnu.linkonce.t.*)
 *(.text.*personality*)
 *(.mips16.fn.*)
 *(.mips16.call.*)
 *(.gnu.warning)
                0x9d000000                . = ALIGN (0x4)

.init           0x9d000000        0x0
 *crti.o(.init)
 *crtbegin.o(.init)
 *(EXCLUDE_FILE(*crtn.o *crtend?.o *crtend.o) .init)
 *crtend.o(.init)
 *crtn.o(.init)
                0x9d000000                . = ALIGN (0x4)

.fini           0x9d000000        0x0
 *(.fini)
                0x9d000000                . = ALIGN (0x4)

.preinit_array  0x9d000000        0x0
                0x9d000000                PROVIDE (__preinit_array_start, .)
 *(.preinit_array)
                0x9d000000                PROVIDE (__preinit_array_end, .)
                0x9d000000                . = ALIGN (0x4)

.init_array     0x9d000000        0x0
                0x9d000000                PROVIDE (__init_array_start, .)
 *(SORT(.init_array.*))
 *(.init_array)
                0x9d000000                PROVIDE (__init_array_end, .)
                0x9d000000                . = ALIGN (0x4)

.fini_array     0x9d000000        0x0
                0x9d000000                PROVIDE (__fini_array_start, .)
 *(SORT(.fini_array.*))
 *(.fini_array)
                0x9d000000                PROVIDE (__fini_array_end, .)
                0x9d000000                . = ALIGN (0x4)

.ctors          0x9d000000        0x0
 *crtbegin.o(.ctors)
 *crtbegin?.o(.ctors)
 *(EXCLUDE_FILE(*crtend?.o *crtend.o) .ctors)
 *(SORT(.ctors.*))
 *(.ctors)
                0x9d000000                . = ALIGN (0x4)

.dtors          0x9d000000        0x0
 *crtbegin.o(.dtors)
 *crtbegin?.o(.dtors)
 *(EXCLUDE_FILE(*crtend?.o *crtend.o) .dtors)
 *(SORT(.dtors.*))
 *(.dtors)
                0x9d000000                . = ALIGN (0x4)

.rodata         0x9d000000        0x0
 *(.gnu.linkonce.r.*)
 *(.rodata1)
                0x9d000000                . = ALIGN (0x4)

.sdata2         0x9fc00490        0x0
 *(.sdata2 .sdata2.* .gnu.linkonce.s2.*)
                0x9fc00490                . = ALIGN (0x4)

.sbss2          0x9fc00490        0x0
 *(.sbss2 .sbss2.* .gnu.linkonce.sb2.*)
                0x9fc00490                . = ALIGN (0x4)

.eh_frame_hdr
 *(.eh_frame_hdr)
                0x9fc00490                . = ALIGN (0x4)

.eh_frame
 *(.eh_frame)
                0x9fc00490                . = ALIGN (0x4)

.gcc_except_table
 *(.gcc_except_table .gcc_except_table.*)
                0x9fc00490                . = ALIGN (0x4)

.dbg_data       0xa0000000        0x0
                0xa0000000                . = (. + DEFINED (_DEBUGGER)?0x200:0x0)

.jcr            0xa0000000        0x0
 *(.jcr)
                0xa0000000                . = ALIGN (0x4)

.eh_frame       0xa0000000       0x30
 *(.eh_frame)
 .eh_frame      0xa0000000       0x20 c:/program files (x86)/microchip/xc32/v1.21/bin/../lib/gcc/pic32mx/4.5.2/size\libgcc.a(_udivdi3.o)
 .eh_frame      0xa0000020       0x10 c:/program files (x86)/microchip/xc32/v1.21/bin/../lib/gcc/pic32mx/4.5.2/size\libgcc.a(_umoddi3.o)
                0xa0000030                . = ALIGN (0x4)

.gcc_except_table
 *(.gcc_except_table .gcc_except_table.*)
                0xa0000030                . = ALIGN (0x4)

.persist        0xa0000030        0x0
                0xa0000030                _persist_begin = .
 *(.persist .persist.*)
 *(.pbss .pbss.*)
                0xa0000030                . = ALIGN (0x4)
                0xa0000030                _persist_end = .

.data           0xa0000030        0x0
 *(.gnu.linkonce.d.*)
 *(.data1)
                0xa0000030                . = ALIGN (0x4)
                0xa0000030                . = .
                0xa0008020                _gp = (ALIGN (0x10) + 0x7ff0)

.got            0xa0000030        0x0
 *(.got.plt)
 *(.got)
                0xa0000030                . = ALIGN (0x4)

.sdata          0xa0000030       0xe0
                0xa0000030                _sdata_begin = .
 *(.sdata .sdata.* .gnu.linkonce.s.*)
 .sdata         0xa0000030        0x4 build/default/production/_ext/101875047/lfsr.o
 .sdata         0xa0000034        0xc build/default/production/_ext/365611741/system_services.o
                0xa0000034                MEDIA_STORAGE_PARTITION_TABLE
 .sdata         0xa0000040       0x60 build/default/production/_ext/365611741/system_debug.o
 .sdata         0xa00000a0       0x1c build/default/production/_ext/792872985/usart.o
                0xa00000a0                _usart_cdev_obj
 .sdata         0xa00000bc       0x2c build/default/production/_ext/792872985/drv_media.o
 .sdata         0xa00000e8        0x8 build/default/production/_ext/427700826/arp.o
 .sdata         0xa00000f0        0x2 build/default/production/_ext/427700826/dns.o
 *fill*         0xa00000f2        0x2 00
 .sdata         0xa00000f4       0x10 build/default/production/_ext/427700826/encx24_mac.o
 .sdata         0xa0000104        0x4 build/default/production/_ext/427700826/tcpip_heap_alloc.o
 .sdata         0xa0000108        0x2 build/default/production/_ext/1472/tcp6_demo_app.o
                0xa0000108                mySocket
 *fill*         0xa000010a        0x2 00
 .sdata         0xa000010c        0x4 c:/program files (x86)/microchip/xc32/v1.21/bin/../lib/gcc/pic32mx/4.5.2/../../../../pic32mx/lib/size\libpic32.a(xc32_uart.o)
                0xa000010c                __XC_UART
                0xa0000110                . = ALIGN (0x4)
                0xa0000110                _sdata_end = .

.lit8
 *(.lit8)

.lit4
 *(.lit4)
                0xa0000110                . = ALIGN (0x4)
                0xa0000110                _data_end = .
                0xa0000110                _bss_begin = .

.sbss           0xa0000110      0x38c
                0xa0000110                _sbss_begin = .
 *(.dynsbss)
 *(.sbss .sbss.* .gnu.linkonce.sb.*)
 .sbss          0xa0000110       0x34 build/default/production/_ext/365611741/system_services.o
                0xa0000110                _SystemTickCount
                0xa0000114                _SystemTickResolution
 .sbss          0xa0000144        0x8 build/default/production/_ext/365611741/system_debug.o
 .sbss          0xa000014c       0x18 build/default/production/_ext/365611741/system_random.o
 .sbss          0xa0000164       0x5c build/default/production/_ext/365611741/system_command.o
 .sbss          0xa00001c0       0x30 build/default/production/_ext/365611741/system_userio.o
 .sbss          0xa00001f0       0x10 build/default/production/_ext/97638081/sys_fs.o
 .sbss          0xa0000200       0x24 build/default/production/_ext/97638081/mpfs2.o
 .sbss          0xa0000224       0x28 build/default/production/_ext/792872985/spi_eeprom.o
 .sbss          0xa000024c       0x34 build/default/production/_ext/792872985/drv_media.o
 .sbss          0xa0000280       0x1c build/default/production/_ext/427700826/tcpip_announce.o
 .sbss          0xa000029c       0x14 build/default/production/_ext/427700826/http2.o
 .sbss          0xa00002b0       0x3c build/default/production/_ext/427700826/arp.o
 .sbss          0xa00002ec       0x20 build/default/production/_ext/427700826/dhcp.o
 .sbss          0xa000030c       0x3c build/default/production/_ext/427700826/dns.o
 .sbss          0xa0000348       0x10 build/default/production/_ext/427700826/encs24j600.o
 .sbss          0xa0000358        0x8 build/default/production/_ext/427700826/icmp.o
 .sbss          0xa0000360       0x20 build/default/production/_ext/427700826/ipv4.o
                0xa0000370                ipv4QueuedPackets
 .sbss          0xa0000380        0xc build/default/production/_ext/427700826/nbns.o
 .sbss          0xa000038c       0x20 build/default/production/_ext/427700826/tcp.o
 .sbss          0xa00003ac       0x18 build/default/production/_ext/427700826/udp.o
                0xa00003ac                UDPSocketDcpt
 .sbss          0xa00003c4       0x3c build/default/production/_ext/427700826/tcpip_manager.o
 .sbss          0xa0000400        0x8 build/default/production/_ext/1472/main_demo.o
 .sbss          0xa0000408        0x2 build/default/production/_ext/1472/custom_http_app.o
 *fill*         0xa000040a        0x2 00
 .sbss          0xa000040c       0x10 build/default/production/_ext/1472/tcp6_demo_app.o
                0xa000040c                nAttempts
                0xa0000410                httpTransactionIndex
                0xa0000414                WaitDispatch2Timer
                0xa0000418                smMyDemoAppTasks
 .sbss          0xa000041c        0x4 c:/program files (x86)/microchip/xc32/v1.21/bin/../lib/gcc/pic32mx/4.5.2/../../../../pic32mx/lib/size\libpic32.a(errno.o)
                0xa000041c                errno
 .sbss          0xa0000420       0x10 c:/program files (x86)/microchip/xc32/v1.21/bin/../lib/gcc/pic32mx/4.5.2/../../../../pic32mx/lib/size\libc.a(malloc.o)
                0xa0000420                __allocp
                0xa0000424                __alloct
                0xa0000428                __allocx
 .sbss          0xa0000430        0x1 c:/program files (x86)/microchip/xc32/v1.21/bin/../lib/gcc/pic32mx/4.5.2/../../../../pic32mx/lib/size\libc.a(_iob.o)
                0xa0000430                _outdone
 *fill*         0xa0000431        0x3 00
 .sbss          0xa0000434        0x8 c:/program files (x86)/microchip/xc32/v1.21/bin/../lib/gcc/pic32mx/4.5.2/../../../../pic32mx/lib/size\libpic32.a(sbrk.o)
                0xa0000434                _minbrk
                0xa0000438                _maxbrk
 *(.scommon)
 .scommon       0xa000043c       0x1e build/default/production/_ext/1472/ping_demo.o
                0xa000043c                pNetIf
                0xa0000440                pingCount
                0xa0000444                targetAddressIPv4
                0xa0000448                pingTimer
                0xa000044c                firstHopAddress
                0xa0000450                targetHostName
                0xa0000454                targetMACAddr
 *fill*         0xa000045a        0x2 00
 .scommon       0xa000045c       0x40 build/default/production/_ext/1472/tcp6_demo_app.o
                0xa000045c                myNetHandle
                0xa0000460                mac_addr_ptr
                0xa0000464                dnsRes
                0xa0000468                HTTPReplyDelay
                0xa000046c                TCPInBufPtr
                0xa0000470                serverIP
                0xa0000474                i
                0xa0000478                mac_addr
                0xa0000480                clientTimer
                0xa0000484                TCPReadByte
                0xa0000488                j
                0xa000048c                TCPInBufferIndex
                0xa0000490                toggleLed
                0xa0000494                HTTPReplyLineCnt
                0xa0000498                TCPIsPutReadyCnt
                0xa000049a                serverPort
                0xa000049c                _sbss_end = .
                0xa000049c                . = ALIGN (0x4)

.bss            0xa000049c     0x1adc
 *(.dynbss)
 *(COMMON)
 COMMON         0xa000049c       0x40 build/default/production/_ext/101875047/hashes.o
                0xa000049c                lastBlock
 COMMON         0xa00004dc       0x21 build/default/production/_ext/792872985/lcd.o
                0xa00004dc                LCDText
 *fill*         0xa00004fd        0x3 00
 COMMON         0xa0000500        0xa build/default/production/_ext/427700826/tcpip_manager.o
                0xa0000500                remoteNode
 *fill*         0xa000050a        0x2 00
 COMMON         0xa000050c     0x1a6c build/default/production/_ext/1472/tcp6_demo_app.o
                0xa000050c                myb64
                0xa000058c                mySocketInfo
                0xa00005b4                httpTransaction
                0xa0000a64                TCPInBuffer
                0xa0001a64                mysrc
                0xa0001ae4                myResourceState
                0xa0001b48                temp
                0xa0001b68                mac_addr_string
                0xa0001b78                OutString
                0xa0001d78                TCPOutBuffer
                0xa0001f78                . = ALIGN ((. != 0x0)?0x4:0x1)
                0xa0001f78                . = ALIGN (0x4)
                0xa0001f78                _end = .
                0xa0001f78                _bss_end = .
                0x00020000                _bmxdudba_address = 0x20000
                0x00020000                _bmxdupba_address = 0x20000

/DISCARD/
 *(.pdr)
 *(.rel.dyn)
 *(.note.GNU-stack)
 *(.note.GNU-stack)
 *(.gnu_debuglink)
 *(.gnu.lto_*)
 *(.discard)

.gptab.sdata
 *(.gptab.data)
 *(.gptab.sdata)

.gptab.sbss
 *(.gptab.bss)
 *(.gptab.sbss)

.mdebug.abi32   0xa0001f78        0x0
 *(.mdebug.abi32)
 .mdebug.abi32  0xa0001f78        0x0 build/default/production/_ext/1293749816/bsp.o
 .mdebug.abi32  0xa0001f78        0x0 build/default/production/_ext/101875047/lfsr.o
 .mdebug.abi32  0xa0001f78        0x0 build/default/production/_ext/101875047/big_int.o
 .mdebug.abi32  0xa0001f78        0x0 build/default/production/_ext/101875047/hashes.o
 .mdebug.abi32  0xa0001f78        0x0 build/default/production/_ext/101875047/helpers.o
 .mdebug.abi32  0xa0001f78        0x0 build/default/production/_ext/1472/berkeley_tcp_client_demo.o
 .mdebug.abi32  0xa0001f78        0x0 build/default/production/_ext/1472/berkeley_tcp_server_demo.o
 .mdebug.abi32  0xa0001f78        0x0 build/default/production/_ext/1472/berkeley_udp_client_demo.o
 .mdebug.abi32  0xa0001f78        0x0 build/default/production/_ext/1472/generic_tcp_client.o
 .mdebug.abi32  0xa0001f78        0x0 build/default/production/_ext/1472/generic_tcp_server.o
 .mdebug.abi32  0xa0001f78        0x0 build/default/production/_ext/1472/ping_demo.o
 .mdebug.abi32  0xa0001f78        0x0 build/default/production/_ext/1472/smtp_demo.o
 .mdebug.abi32  0xa0001f78        0x0 build/default/production/_ext/365611741/system_services.o
 .mdebug.abi32  0xa0001f78        0x0 build/default/production/_ext/365611741/system_debug.o
 .mdebug.abi32  0xa0001f78        0x0 build/default/production/_ext/365611741/system_random.o
 .mdebug.abi32  0xa0001f78        0x0 build/default/production/_ext/365611741/system_command.o
 .mdebug.abi32  0xa0001f78        0x0 build/default/production/_ext/365611741/system_userio.o
 .mdebug.abi32  0xa0001f78        0x0 build/default/production/_ext/97638081/sys_fs.o
 .mdebug.abi32  0xa0001f78        0x0 build/default/production/_ext/97638081/mpfs2.o
 .mdebug.abi32  0xa0001f78        0x0 build/default/production/_ext/792872985/usart.o
 .mdebug.abi32  0xa0001f78        0x0 build/default/production/_ext/792872985/lcd.o
 .mdebug.abi32  0xa0001f78        0x0 build/default/production/_ext/792872985/drv_spi.o
 .mdebug.abi32  0xa0001f78        0x0 build/default/production/_ext/792872985/db_appio.o
 .mdebug.abi32  0xa0001f78        0x0 build/default/production/_ext/792872985/spi_ram.o
 .mdebug.abi32  0xa0001f78        0x0 build/default/production/_ext/792872985/spi_eeprom.o
 .mdebug.abi32  0xa0001f78        0x0 build/default/production/_ext/792872985/spi_flash.o
 .mdebug.abi32  0xa0001f78        0x0 build/default/production/_ext/792872985/drv_media.o
 .mdebug.abi32  0xa0001f78        0x0 build/default/production/_ext/427700826/tcpip_announce.o
 .mdebug.abi32  0xa0001f78        0x0 build/default/production/_ext/427700826/http2.o
 .mdebug.abi32  0xa0001f78        0x0 build/default/production/_ext/427700826/arcfour.o
 .mdebug.abi32  0xa0001f78        0x0 build/default/production/_ext/427700826/arp.o
 .mdebug.abi32  0xa0001f78        0x0 build/default/production/_ext/427700826/berkeley_api.o
 .mdebug.abi32  0xa0001f78        0x0 build/default/production/_ext/427700826/dhcp.o
 .mdebug.abi32  0xa0001f78        0x0 build/default/production/_ext/427700826/dhcps.o
 .mdebug.abi32  0xa0001f78        0x0 build/default/production/_ext/427700826/dns.o
 .mdebug.abi32  0xa0001f78        0x0 build/default/production/_ext/427700826/dnss.o
 .mdebug.abi32  0xa0001f78        0x0 build/default/production/_ext/427700826/dyn_dns.o
 .mdebug.abi32  0xa0001f78        0x0 build/default/production/_ext/427700826/enc28_mac.o
 .mdebug.abi32  0xa0001f78        0x0 build/default/production/_ext/427700826/enc28j60.o
 .mdebug.abi32  0xa0001f78        0x0 build/default/production/_ext/427700826/encs24j600.o
 .mdebug.abi32  0xa0001f78        0x0 build/default/production/_ext/427700826/encx24_mac.o
 .mdebug.abi32  0xa0001f78        0x0 build/default/production/_ext/427700826/eth_pic32_ext_phy.o
 .mdebug.abi32  0xa0001f78        0x0 build/default/production/_ext/427700826/eth_pic32_ext_phy_dp83848.o
 .mdebug.abi32  0xa0001f78        0x0 build/default/production/_ext/427700826/eth_pic32_int_mac.o
 .mdebug.abi32  0xa0001f78        0x0 build/default/production/_ext/427700826/ftp.o
 .mdebug.abi32  0xa0001f78        0x0 build/default/production/_ext/427700826/hash_fnv.o
 .mdebug.abi32  0xa0001f78        0x0 build/default/production/_ext/427700826/hash_tbl.o
 .mdebug.abi32  0xa0001f78        0x0 build/default/production/_ext/427700826/icmp.o
 .mdebug.abi32  0xa0001f78        0x0 build/default/production/_ext/427700826/icmpv6.o
 .mdebug.abi32  0xa0001f78        0x0 build/default/production/_ext/427700826/ipv4.o
 .mdebug.abi32  0xa0001f78        0x0 build/default/production/_ext/427700826/ipv6.o
 .mdebug.abi32  0xa0001f78        0x0 build/default/production/_ext/427700826/mac_events_pic32.o
 .mdebug.abi32  0xa0001f78        0x0 build/default/production/_ext/427700826/nbns.o
 .mdebug.abi32  0xa0001f78        0x0 build/default/production/_ext/427700826/ndp.o
 .mdebug.abi32  0xa0001f78        0x0 build/default/production/_ext/427700826/tcpip_reboot.o
 .mdebug.abi32  0xa0001f78        0x0 build/default/production/_ext/427700826/rsa.o
 .mdebug.abi32  0xa0001f78        0x0 build/default/production/_ext/427700826/smtp.o
 .mdebug.abi32  0xa0001f78        0x0 build/default/production/_ext/427700826/snmp.o
 .mdebug.abi32  0xa0001f78        0x0 build/default/production/_ext/427700826/snmpv3.o
 .mdebug.abi32  0xa0001f78        0x0 build/default/production/_ext/427700826/snmpv3_usm.o
 .mdebug.abi32  0xa0001f78        0x0 build/default/production/_ext/427700826/sntp.o
 .mdebug.abi32  0xa0001f78        0x0 build/default/production/_ext/427700826/ssl.o
 .mdebug.abi32  0xa0001f78        0x0 build/default/production/_ext/427700826/tcp.o
 .mdebug.abi32  0xa0001f78        0x0 build/default/production/_ext/427700826/tcpip_heap_alloc.o
 .mdebug.abi32  0xa0001f78        0x0 build/default/production/_ext/427700826/tcpip_storage.o
 .mdebug.abi32  0xa0001f78        0x0 build/default/production/_ext/427700826/telnet.o
 .mdebug.abi32  0xa0001f78        0x0 build/default/production/_ext/427700826/tftpc.o
 .mdebug.abi32  0xa0001f78        0x0 build/default/production/_ext/427700826/udp.o
 .mdebug.abi32  0xa0001f78        0x0 build/default/production/_ext/427700826/tcpip_mac_object.o
 .mdebug.abi32  0xa0001f78        0x0 build/default/production/_ext/427700826/tcpip_manager.o
 .mdebug.abi32  0xa0001f78        0x0 build/default/production/_ext/427700826/tcpip_helpers.o
 .mdebug.abi32  0xa0001f78        0x0 build/default/production/_ext/427700826/tcpip_commands.o
 .mdebug.abi32  0xa0001f78        0x0 build/default/production/_ext/427700826/iperf.o
 .mdebug.abi32  0xa0001f78        0x0 build/default/production/_ext/427700826/tcpip_notify.o
 .mdebug.abi32  0xa0001f78        0x0 build/default/production/_ext/427700826/zero_conf_helper.o
 .mdebug.abi32  0xa0001f78        0x0 build/default/production/_ext/427700826/zero_conf_link_local.o
 .mdebug.abi32  0xa0001f78        0x0 build/default/production/_ext/427700826/zero_conf_multicast_dns.o
 .mdebug.abi32  0xa0001f78        0x0 build/default/production/_ext/334706090/wf_tx_power.o
 .mdebug.abi32  0xa0001f78        0x0 build/default/production/_ext/334706090/wf_connect.o
 .mdebug.abi32  0xa0001f78        0x0 build/default/production/_ext/334706090/wf_connection_algorithm.o
 .mdebug.abi32  0xa0001f78        0x0 build/default/production/_ext/334706090/wf_connection_manager.o
 .mdebug.abi32  0xa0001f78        0x0 build/default/production/_ext/334706090/wf_connection_profile.o
 .mdebug.abi32  0xa0001f78        0x0 build/default/production/_ext/334706090/wf_easy_config.o
 .mdebug.abi32  0xa0001f78        0x0 build/default/production/_ext/334706090/wf_eint.o
 .mdebug.abi32  0xa0001f78        0x0 build/default/production/_ext/334706090/wf_event_handler.o
 .mdebug.abi32  0xa0001f78        0x0 build/default/production/_ext/334706090/wf_init.o
 .mdebug.abi32  0xa0001f78        0x0 build/default/production/_ext/334706090/wf_power_save.o
 .mdebug.abi32  0xa0001f78        0x0 build/default/production/_ext/334706090/wf_scan.o
 .mdebug.abi32  0xa0001f78        0x0 build/default/production/_ext/334706090/wf_spi.o
 .mdebug.abi32  0xa0001f78        0x0 build/default/production/_ext/334706090/mrf24w_mac_pic32.o
 .mdebug.abi32  0xa0001f78        0x0 build/default/production/_ext/334706090/mrf24w_events.o
 .mdebug.abi32  0xa0001f78        0x0 build/default/production/_ext/334706090/wf_driver_com_24g.o
 .mdebug.abi32  0xa0001f78        0x0 build/default/production/_ext/334706090/wf_driver_raw_24g.o
 .mdebug.abi32  0xa0001f78        0x0 build/default/production/_ext/334706090/wf_mac_24g.o
 .mdebug.abi32  0xa0001f78        0x0 build/default/production/_ext/334706090/wf_mgmt_msg_24g.o
 .mdebug.abi32  0xa0001f78        0x0 build/default/production/_ext/334706090/wf_param_msg_24g.o
 .mdebug.abi32  0xa0001f78        0x0 build/default/production/_ext/1472/main_demo.o
 .mdebug.abi32  0xa0001f78        0x0 build/default/production/_ext/1472/custom_snmp_app.o
 .mdebug.abi32  0xa0001f78        0x0 build/default/production/_ext/1472/custom_ssl_cert.o
 .mdebug.abi32  0xa0001f78        0x0 build/default/production/_ext/1472/mpfs_img2.o
 .mdebug.abi32  0xa0001f78        0x0 build/default/production/_ext/1472/wf_config.o
 .mdebug.abi32  0xa0001f78        0x0 build/default/production/_ext/1472/custom_http_app.o
 .mdebug.abi32  0xa0001f78        0x0 build/default/production/_ext/1472/tcp6_demo_app.o
 .mdebug.abi32  0xa0001f78        0x0 c:/program files (x86)/microchip/xc32/v1.21/bin/../lib/gcc/pic32mx/4.5.2/../../../../pic32mx/lib/size\libmchp_peripheral.a(open_core_timer_lib.o)
 .mdebug.abi32  0xa0001f78        0x0 c:/program files (x86)/microchip/xc32/v1.21/bin/../lib/gcc/pic32mx/4.5.2/../../../../pic32mx/lib/size\libmchp_peripheral_32MX795F512L.a(soft_reset_lib.o)
 .mdebug.abi32  0xa0001f78        0x0 c:/program files (x86)/microchip/xc32/v1.21/bin/../lib/gcc/pic32mx/4.5.2/../../../../pic32mx/lib/size\libmchp_peripheral_32MX795F512L.a(pcache.o)
 .mdebug.abi32  0xa0001f78        0x0 c:/program files (x86)/microchip/xc32/v1.21/bin/../lib/gcc/pic32mx/4.5.2/../../../../pic32mx/lib/size\libmchp_peripheral_32MX795F512L.a(int_disable_interrupts_lib.o)
 .mdebug.abi32  0xa0001f78        0x0 c:/program files (x86)/microchip/xc32/v1.21/bin/../lib/gcc/pic32mx/4.5.2/../../../../pic32mx/lib/size\libmchp_peripheral_32MX795F512L.a(int_restore_interrupts_lib.o)
 .mdebug.abi32  0xa0001f78        0x0 c:/program files (x86)/microchip/xc32/v1.21/bin/../lib/gcc/pic32mx/4.5.2/../../../../pic32mx/lib/size\libmchp_peripheral_32MX795F512L.a(int_enable_mv_int_lib.o)
 .mdebug.abi32  0xa0001f78        0x0 c:/program files (x86)/microchip/xc32/v1.21/bin/../lib/gcc/pic32mx/4.5.2/../../../../pic32mx/lib/size\libmchp_peripheral_32MX795F512L.a(int_tbl_lib.o)
 .mdebug.abi32  0xa0001f78        0x0 c:/program files (x86)/microchip/xc32/v1.21/bin/../lib/gcc/pic32mx/4.5.2/../../../../pic32mx/lib/size\libmchp_peripheral_32MX795F512L.a(rtcc_init_lib.o)
 .mdebug.abi32  0xa0001f78        0x0 c:/program files (x86)/microchip/xc32/v1.21/bin/../lib/gcc/pic32mx/4.5.2/../../../../pic32mx/lib/size\libmchp_peripheral_32MX795F512L.a(rtcc_open_lib.o)
 .mdebug.abi32  0xa0001f78        0x0 c:/program files (x86)/microchip/xc32/v1.21/bin/../lib/gcc/pic32mx/4.5.2/../../../../pic32mx/lib/size\libmchp_peripheral_32MX795F512L.a(spi_chn_data_rdy_lib.o)
 .mdebug.abi32  0xa0001f78        0x0 c:/program files (x86)/microchip/xc32/v1.21/bin/../lib/gcc/pic32mx/4.5.2/../../../../pic32mx/lib/size\libmchp_peripheral_32MX795F512L.a(spi_chn_getc_lib.o)
 .mdebug.abi32  0xa0001f78        0x0 c:/program files (x86)/microchip/xc32/v1.21/bin/../lib/gcc/pic32mx/4.5.2/../../../../pic32mx/lib/size\libmchp_peripheral_32MX795F512L.a(spi_chn_open_lib.o)
 .mdebug.abi32  0xa0001f78        0x0 c:/program files (x86)/microchip/xc32/v1.21/bin/../lib/gcc/pic32mx/4.5.2/../../../../pic32mx/lib/size\libmchp_peripheral_32MX795F512L.a(spi_chn_putc_lib.o)
 .mdebug.abi32  0xa0001f78        0x0 c:/program files (x86)/microchip/xc32/v1.21/bin/../lib/gcc/pic32mx/4.5.2/../../../../pic32mx/lib/size\libmchp_peripheral_32MX795F512L.a(spi_chn_tx_buff_empty_lib.o)
 .mdebug.abi32  0xa0001f78        0x0 c:/program files (x86)/microchip/xc32/v1.21/bin/../lib/gcc/pic32mx/4.5.2/../../../../pic32mx/lib/size\libmchp_peripheral_32MX795F512L.a(spi_io_tbl_libp.o)
 .mdebug.abi32  0xa0001f78        0x0 c:/program files (x86)/microchip/xc32/v1.21/bin/../lib/gcc/pic32mx/4.5.2/../../../../pic32mx/lib/size\libmchp_peripheral_32MX795F512L.a(spi_map_tbl_libp.o)
 .mdebug.abi32  0xa0001f78        0x0 c:/program files (x86)/microchip/xc32/v1.21/bin/../lib/gcc/pic32mx/4.5.2/../../../../pic32mx/lib/size\libmchp_peripheral_32MX795F512L.a(port_set_pins_digital_in_lib.o)
 .mdebug.abi32  0xa0001f78        0x0 c:/program files (x86)/microchip/xc32/v1.21/bin/../lib/gcc/pic32mx/4.5.2/../../../../pic32mx/lib/size\libmchp_peripheral_32MX795F512L.a(port_set_pins_digital_out_lib.o)
 .mdebug.abi32  0xa0001f78        0x0 c:/program files (x86)/microchip/xc32/v1.21/bin/../lib/gcc/pic32mx/4.5.2/../../../../pic32mx/lib/size\libmchp_peripheral_32MX795F512L.a(_ports_tbl_libp.o)
 .mdebug.abi32  0xa0001f78        0x0 c:/program files (x86)/microchip/xc32/v1.21/bin/../lib/gcc/pic32mx/4.5.2/../../../../pic32mx/lib/size\libmchp_peripheral_32MX795F512L.a(int_enable_interrupts_lib.o)
 .mdebug.abi32  0xa0001f78        0x0 c:/program files (x86)/microchip/xc32/v1.21/bin/../lib/gcc/pic32mx/4.5.2/../../../../pic32mx/lib/size\libmchp_peripheral_32MX795F512L.a(_rtcc_wait_clock_off_lib.o)
 .mdebug.abi32  0xa0001f78        0x0 c:/program files (x86)/microchip/xc32/v1.21/bin/../lib/gcc/pic32mx/4.5.2/../../../../pic32mx/lib/size\libmchp_peripheral_32MX795F512L.a(read_core_timer_lib.o)
 .mdebug.abi32  0xa0001f78        0x0 c:/program files (x86)/microchip/xc32/v1.21/bin/../lib/gcc/pic32mx/4.5.2/size\libgcc.a(_udivdi3.o)
 .mdebug.abi32  0xa0001f78        0x0 c:/program files (x86)/microchip/xc32/v1.21/bin/../lib/gcc/pic32mx/4.5.2/../../../../pic32mx/lib/size\libpic32.a(default-bootstrap-exception-handler.o)
 .mdebug.abi32  0xa0001f78        0x0 c:/program files (x86)/microchip/xc32/v1.21/bin/../lib/gcc/pic32mx/4.5.2/../../../../pic32mx/lib/size\libpic32.a(default-on-reset.o)
 .mdebug.abi32  0xa0001f78        0x0 c:/program files (x86)/microchip/xc32/v1.21/bin/../lib/gcc/pic32mx/4.5.2/../../../../pic32mx/lib/size\libpic32.a(default-on-bootstrap.o)
 .mdebug.abi32  0xa0001f78        0x0 c:/program files (x86)/microchip/xc32/v1.21/bin/../lib/gcc/pic32mx/4.5.2/../../../../pic32mx/lib/size\libpic32.a(errno.o)
 .mdebug.abi32  0xa0001f78        0x0 c:/program files (x86)/microchip/xc32/v1.21/bin/../lib/gcc/pic32mx/4.5.2/../../../../pic32mx/lib/size\libpic32.a(defaultinterrupt.o)
 .mdebug.abi32  0xa0001f78        0x0 c:/program files (x86)/microchip/xc32/v1.21/bin/../lib/gcc/pic32mx/4.5.2/../../../../pic32mx/lib/size\libc.a(atoi.o)
 .mdebug.abi32  0xa0001f78        0x0 c:/program files (x86)/microchip/xc32/v1.21/bin/../lib/gcc/pic32mx/4.5.2/../../../../pic32mx/lib/size\libc.a(atol.o)
 .mdebug.abi32  0xa0001f78        0x0 c:/program files (x86)/microchip/xc32/v1.21/bin/../lib/gcc/pic32mx/4.5.2/../../../../pic32mx/lib/size\libc.a(ctype.o)
 .mdebug.abi32  0xa0001f78        0x0 c:/program files (x86)/microchip/xc32/v1.21/bin/../lib/gcc/pic32mx/4.5.2/../../../../pic32mx/lib/size\libc.a(malloc.o)
 .mdebug.abi32  0xa0001f78        0x0 c:/program files (x86)/microchip/xc32/v1.21/bin/../lib/gcc/pic32mx/4.5.2/../../../../pic32mx/lib/size\libc.a(rand.o)
 .mdebug.abi32  0xa0001f78        0x0 c:/program files (x86)/microchip/xc32/v1.21/bin/../lib/gcc/pic32mx/4.5.2/../../../../pic32mx/lib/size\libc.a(strcat.o)
 .mdebug.abi32  0xa0001f78        0x0 c:/program files (x86)/microchip/xc32/v1.21/bin/../lib/gcc/pic32mx/4.5.2/../../../../pic32mx/lib/size\libc.a(strchr.o)
 .mdebug.abi32  0xa0001f78        0x0 c:/program files (x86)/microchip/xc32/v1.21/bin/../lib/gcc/pic32mx/4.5.2/../../../../pic32mx/lib/size\libc.a(strncat.o)
 .mdebug.abi32  0xa0001f78        0x0 c:/program files (x86)/microchip/xc32/v1.21/bin/../lib/gcc/pic32mx/4.5.2/../../../../pic32mx/lib/size\libc.a(strncmp.o)
 .mdebug.abi32  0xa0001f78        0x0 c:/program files (x86)/microchip/xc32/v1.21/bin/../lib/gcc/pic32mx/4.5.2/../../../../pic32mx/lib/size\libc.a(strncpy.o)
 .mdebug.abi32  0xa0001f78        0x0 c:/program files (x86)/microchip/xc32/v1.21/bin/../lib/gcc/pic32mx/4.5.2/../../../../pic32mx/lib/size\libc.a(strrchr.o)
 .mdebug.abi32  0xa0001f78        0x0 c:/program files (x86)/microchip/xc32/v1.21/bin/../lib/gcc/pic32mx/4.5.2/../../../../pic32mx/lib/size\libc.a(strstr.o)
 .mdebug.abi32  0xa0001f78        0x0 c:/program files (x86)/microchip/xc32/v1.21/bin/../lib/gcc/pic32mx/4.5.2/../../../../pic32mx/lib/size\libc.a(strtol.o)
 .mdebug.abi32  0xa0001f78        0x0 c:/program files (x86)/microchip/xc32/v1.21/bin/../lib/gcc/pic32mx/4.5.2/../../../../pic32mx/lib/size\libc.a(snprintf_cdnopsuxX.eo)
 .mdebug.abi32  0xa0001f78        0x0 c:/program files (x86)/microchip/xc32/v1.21/bin/../lib/gcc/pic32mx/4.5.2/../../../../pic32mx/lib/size\libc.a(sprintf_cdnopsuxX.eo)
 .mdebug.abi32  0xa0001f78        0x0 c:/program files (x86)/microchip/xc32/v1.21/bin/../lib/gcc/pic32mx/4.5.2/../../../../pic32mx/lib/size\libc.a(vsnprintf_cdnopsuxX.eo)
 .mdebug.abi32  0xa0001f78        0x0 c:/program files (x86)/microchip/xc32/v1.21/bin/../lib/gcc/pic32mx/4.5.2/../../../../pic32mx/lib/size\libc.a(vsnprintf.o)
 .mdebug.abi32  0xa0001f78        0x0 c:/program files (x86)/microchip/xc32/v1.21/bin/../lib/gcc/pic32mx/4.5.2/../../../../pic32mx/lib/size\libc.a(ctypef.o)
 .mdebug.abi32  0xa0001f78        0x0 c:/program files (x86)/microchip/xc32/v1.21/bin/../lib/gcc/pic32mx/4.5.2/../../../../pic32mx/lib/size\libc.a(doprnt_cdnopsuxX.eo)
 .mdebug.abi32  0xa0001f78        0x0 c:/program files (x86)/microchip/xc32/v1.21/bin/../lib/gcc/pic32mx/4.5.2/../../../../pic32mx/lib/size\libc.a(doprnt.o)
 .mdebug.abi32  0xa0001f78        0x0 c:/program files (x86)/microchip/xc32/v1.21/bin/../lib/gcc/pic32mx/4.5.2/../../../../pic32mx/lib/size\libc.a(_fputc_simple.o)
 .mdebug.abi32  0xa0001f78        0x0 c:/program files (x86)/microchip/xc32/v1.21/bin/../lib/gcc/pic32mx/4.5.2/../../../../pic32mx/lib/size\libc.a(powersf.o)
 .mdebug.abi32  0xa0001f78        0x0 c:/program files (x86)/microchip/xc32/v1.21/bin/../lib/gcc/pic32mx/4.5.2/../../../../pic32mx/lib/size\libc.a(_iob.o)
 .mdebug.abi32  0xa0001f78        0x0 c:/program files (x86)/microchip/xc32/v1.21/bin/../lib/gcc/pic32mx/4.5.2/../../../../pic32mx/lib/size\libc.a(_flsbuf_simple.o)
 .mdebug.abi32  0xa0001f78        0x0 c:/program files (x86)/microchip/xc32/v1.21/bin/../lib/gcc/pic32mx/4.5.2/../../../../pic32mx/lib/size\libpic32.a(sbrk.o)
 .mdebug.abi32  0xa0001f78        0x0 c:/program files (x86)/microchip/xc32/v1.21/bin/../lib/gcc/pic32mx/4.5.2/../../../../pic32mx/lib/size\libpic32.a(write.o)
 .mdebug.abi32  0xa0001f78        0x0 c:/program files (x86)/microchip/xc32/v1.21/bin/../lib/gcc/pic32mx/4.5.2/../../../../pic32mx/lib/size\libpic32.a(_mon_putc.o)
 .mdebug.abi32  0xa0001f78        0x0 c:/program files (x86)/microchip/xc32/v1.21/bin/../lib/gcc/pic32mx/4.5.2/../../../../pic32mx/lib/size\libpic32.a(xc32_uart.o)
 .mdebug.abi32  0xa0001f78        0x0 c:/program files (x86)/microchip/xc32/v1.21/bin/../lib/gcc/pic32mx/4.5.2/../../../../pic32mx/lib/size\libe.a(_floatdisf.o)
 .mdebug.abi32  0xa0001f78        0x0 c:/program files (x86)/microchip/xc32/v1.21/bin/../lib/gcc/pic32mx/4.5.2/size\libgcc.a(_lshrdi3.o)
 .mdebug.abi32  0xa0001f78        0x0 c:/program files (x86)/microchip/xc32/v1.21/bin/../lib/gcc/pic32mx/4.5.2/size\libgcc.a(_floatundisf.o)
 .mdebug.abi32  0xa0001f78        0x0 c:/program files (x86)/microchip/xc32/v1.21/bin/../lib/gcc/pic32mx/4.5.2/size\libgcc.a(_umoddi3.o)
 .mdebug.abi32  0xa0001f78        0x0 c:/program files (x86)/microchip/xc32/v1.21/bin/../lib/gcc/pic32mx/4.5.2/size\libgcc.a(floatunsisf.o)

.mdebug.abiN32
 *(.mdebug.abiN32)

.mdebug.abi64
 *(.mdebug.abi64)

.mdebug.abiO64
 *(.mdebug.abiO64)

.mdebug.eabi32
 *(.mdebug.eabi32)

.mdebug.eabi64
 *(.mdebug.eabi64)

.gcc_compiled_long32
 *(.gcc_compiled_long32)

.gcc_compiled_long64
 *(.gcc_compiled_long64)

.stab
 *(.stab)

.stabstr
 *(.stabstr)

.stab.excl
 *(.stab.excl)

.stab.exclstr
 *(.stab.exclstr)

.stab.index
 *(.stab.index)

.stab.indexstr
 *(.stab.indexstr)

.comment        0x00000000      0x2b5
 *(.comment)
 .comment       0x00000000       0x3c build/default/production/_ext/1293749816/bsp.o
                                 0x3d (size before relaxing)
 .comment       0x00000000       0x3d build/default/production/_ext/101875047/lfsr.o
 .comment       0x00000000       0x3d build/default/production/_ext/101875047/big_int.o
 .comment       0x00000000       0x3d build/default/production/_ext/101875047/hashes.o
 .comment       0x00000000       0x3d build/default/production/_ext/101875047/helpers.o
 .comment       0x00000000       0x3d build/default/production/_ext/1472/berkeley_tcp_client_demo.o
 .comment       0x00000000       0x3d build/default/production/_ext/1472/berkeley_tcp_server_demo.o
 .comment       0x00000000       0x3d build/default/production/_ext/1472/berkeley_udp_client_demo.o
 .comment       0x00000000       0x3d build/default/production/_ext/1472/generic_tcp_client.o
 .comment       0x00000000       0x3d build/default/production/_ext/1472/generic_tcp_server.o
 .comment       0x00000000       0x3d build/default/production/_ext/1472/ping_demo.o
 .comment       0x00000000       0x3d build/default/production/_ext/1472/smtp_demo.o
 .comment       0x00000000       0x3d build/default/production/_ext/365611741/system_services.o
 .comment       0x00000000       0x3d build/default/production/_ext/365611741/system_debug.o
 .comment       0x00000000       0x3d build/default/production/_ext/365611741/system_random.o
 .comment       0x00000000       0x3d build/default/production/_ext/365611741/system_command.o
 .comment       0x00000000       0x3d build/default/production/_ext/365611741/system_userio.o
 .comment       0x00000000       0x3d build/default/production/_ext/97638081/sys_fs.o
 .comment       0x00000000       0x3d build/default/production/_ext/97638081/mpfs2.o
 .comment       0x00000000       0x3d build/default/production/_ext/792872985/usart.o
 .comment       0x00000000       0x3d build/default/production/_ext/792872985/lcd.o
 .comment       0x00000000       0x3d build/default/production/_ext/792872985/drv_spi.o
 .comment       0x00000000       0x3d build/default/production/_ext/792872985/db_appio.o
 .comment       0x00000000       0x3d build/default/production/_ext/792872985/spi_ram.o
 .comment       0x00000000       0x3d build/default/production/_ext/792872985/spi_eeprom.o
 .comment       0x00000000       0x3d build/default/production/_ext/792872985/spi_flash.o
 .comment       0x00000000       0x3d build/default/production/_ext/792872985/drv_media.o
 .comment       0x00000000       0x3d build/default/production/_ext/427700826/tcpip_announce.o
 .comment       0x00000000       0x3d build/default/production/_ext/427700826/http2.o
 .comment       0x00000000       0x3d build/default/production/_ext/427700826/arcfour.o
 .comment       0x00000000       0x3d build/default/production/_ext/427700826/arp.o
 .comment       0x00000000       0x3d build/default/production/_ext/427700826/berkeley_api.o
 .comment       0x00000000       0x3d build/default/production/_ext/427700826/dhcp.o
 .comment       0x00000000       0x3d build/default/production/_ext/427700826/dhcps.o
 .comment       0x00000000       0x3d build/default/production/_ext/427700826/dns.o
 .comment       0x00000000       0x3d build/default/production/_ext/427700826/dnss.o
 .comment       0x00000000       0x3d build/default/production/_ext/427700826/dyn_dns.o
 .comment       0x00000000       0x3d build/default/production/_ext/427700826/enc28_mac.o
 .comment       0x00000000       0x3d build/default/production/_ext/427700826/enc28j60.o
 .comment       0x00000000       0x3d build/default/production/_ext/427700826/encs24j600.o
 .comment       0x00000000       0x3d build/default/production/_ext/427700826/encx24_mac.o
 .comment       0x00000000       0x3d build/default/production/_ext/427700826/eth_pic32_ext_phy.o
 .comment       0x00000000       0x3d build/default/production/_ext/427700826/eth_pic32_ext_phy_dp83848.o
 .comment       0x00000000       0x3d build/default/production/_ext/427700826/eth_pic32_int_mac.o
 .comment       0x00000000       0x3d build/default/production/_ext/427700826/ftp.o
 .comment       0x00000000       0x3d build/default/production/_ext/427700826/hash_fnv.o
 .comment       0x00000000       0x3d build/default/production/_ext/427700826/hash_tbl.o
 .comment       0x00000000       0x3d build/default/production/_ext/427700826/icmp.o
 .comment       0x00000000       0x3d build/default/production/_ext/427700826/icmpv6.o
 .comment       0x00000000       0x3d build/default/production/_ext/427700826/ipv4.o
 .comment       0x00000000       0x3d build/default/production/_ext/427700826/ipv6.o
 .comment       0x00000000       0x3d build/default/production/_ext/427700826/mac_events_pic32.o
 .comment       0x00000000       0x3d build/default/production/_ext/427700826/nbns.o
 .comment       0x00000000       0x3d build/default/production/_ext/427700826/ndp.o
 .comment       0x00000000       0x3d build/default/production/_ext/427700826/tcpip_reboot.o
 .comment       0x00000000       0x3d build/default/production/_ext/427700826/rsa.o
 .comment       0x00000000       0x3d build/default/production/_ext/427700826/smtp.o
 .comment       0x00000000       0x3d build/default/production/_ext/427700826/snmp.o
 .comment       0x00000000       0x3d build/default/production/_ext/427700826/snmpv3.o
 .comment       0x00000000       0x3d build/default/production/_ext/427700826/snmpv3_usm.o
 .comment       0x00000000       0x3d build/default/production/_ext/427700826/sntp.o
 .comment       0x00000000       0x3d build/default/production/_ext/427700826/ssl.o
 .comment       0x00000000       0x3d build/default/production/_ext/427700826/tcp.o
 .comment       0x00000000       0x3d build/default/production/_ext/427700826/tcpip_heap_alloc.o
 .comment       0x00000000       0x3d build/default/production/_ext/427700826/tcpip_storage.o
 .comment       0x00000000       0x3d build/default/production/_ext/427700826/telnet.o
 .comment       0x00000000       0x3d build/default/production/_ext/427700826/tftpc.o
 .comment       0x00000000       0x3d build/default/production/_ext/427700826/udp.o
 .comment       0x00000000       0x3d build/default/production/_ext/427700826/tcpip_mac_object.o
 .comment       0x00000000       0x3d build/default/production/_ext/427700826/tcpip_manager.o
 .comment       0x00000000       0x3d build/default/production/_ext/427700826/tcpip_helpers.o
 .comment       0x00000000       0x3d build/default/production/_ext/427700826/tcpip_commands.o
 .comment       0x00000000       0x3d build/default/production/_ext/427700826/iperf.o
 .comment       0x00000000       0x3d build/default/production/_ext/427700826/tcpip_notify.o
 .comment       0x00000000       0x3d build/default/production/_ext/427700826/zero_conf_helper.o
 .comment       0x00000000       0x3d build/default/production/_ext/427700826/zero_conf_link_local.o
 .comment       0x00000000       0x3d build/default/production/_ext/427700826/zero_conf_multicast_dns.o
 .comment       0x00000000       0x3d build/default/production/_ext/334706090/wf_tx_power.o
 .comment       0x00000000       0x3d build/default/production/_ext/334706090/wf_connect.o
 .comment       0x00000000       0x3d build/default/production/_ext/334706090/wf_connection_algorithm.o
 .comment       0x00000000       0x3d build/default/production/_ext/334706090/wf_connection_manager.o
 .comment       0x00000000       0x3d build/default/production/_ext/334706090/wf_connection_profile.o
 .comment       0x00000000       0x3d build/default/production/_ext/334706090/wf_easy_config.o
 .comment       0x00000000       0x3d build/default/production/_ext/334706090/wf_eint.o
 .comment       0x00000000       0x3d build/default/production/_ext/334706090/wf_event_handler.o
 .comment       0x00000000       0x3d build/default/production/_ext/334706090/wf_init.o
 .comment       0x00000000       0x3d build/default/production/_ext/334706090/wf_power_save.o
 .comment       0x00000000       0x3d build/default/production/_ext/334706090/wf_scan.o
 .comment       0x00000000       0x3d build/default/production/_ext/334706090/wf_spi.o
 .comment       0x00000000       0x3d build/default/production/_ext/334706090/mrf24w_mac_pic32.o
 .comment       0x00000000       0x3d build/default/production/_ext/334706090/mrf24w_events.o
 .comment       0x00000000       0x3d build/default/production/_ext/334706090/wf_driver_com_24g.o
 .comment       0x00000000       0x3d build/default/production/_ext/334706090/wf_driver_raw_24g.o
 .comment       0x00000000       0x3d build/default/production/_ext/334706090/wf_mac_24g.o
 .comment       0x00000000       0x3d build/default/production/_ext/334706090/wf_mgmt_msg_24g.o
 .comment       0x00000000       0x3d build/default/production/_ext/334706090/wf_param_msg_24g.o
 .comment       0x00000000       0x3d build/default/production/_ext/1472/main_demo.o
 .comment       0x00000000       0x3d build/default/production/_ext/1472/custom_snmp_app.o
 .comment       0x00000000       0x3d build/default/production/_ext/1472/custom_ssl_cert.o
 .comment       0x00000000       0x3d build/default/production/_ext/1472/mpfs_img2.o
 .comment       0x00000000       0x3d build/default/production/_ext/1472/wf_config.o
 .comment       0x00000000       0x3d build/default/production/_ext/1472/custom_http_app.o
 .comment       0x00000000       0x3d build/default/production/_ext/1472/tcp6_demo_app.o
 .comment       0x0000003c       0x3c c:/program files (x86)/microchip/xc32/v1.21/bin/../lib/gcc/pic32mx/4.5.2/../../../../pic32mx/lib/size\libmchp_peripheral.a(open_core_timer_lib.o)
                                 0x3d (size before relaxing)
 .comment       0x00000000       0x3d c:/program files (x86)/microchip/xc32/v1.21/bin/../lib/gcc/pic32mx/4.5.2/../../../../pic32mx/lib/size\libmchp_peripheral_32MX795F512L.a(soft_reset_lib.o)
 .comment       0x00000000       0x3d c:/program files (x86)/microchip/xc32/v1.21/bin/../lib/gcc/pic32mx/4.5.2/../../../../pic32mx/lib/size\libmchp_peripheral_32MX795F512L.a(pcache.o)
 .comment       0x00000000       0x3d c:/program files (x86)/microchip/xc32/v1.21/bin/../lib/gcc/pic32mx/4.5.2/../../../../pic32mx/lib/size\libmchp_peripheral_32MX795F512L.a(int_disable_interrupts_lib.o)
 .comment       0x00000000       0x3d c:/program files (x86)/microchip/xc32/v1.21/bin/../lib/gcc/pic32mx/4.5.2/../../../../pic32mx/lib/size\libmchp_peripheral_32MX795F512L.a(int_restore_interrupts_lib.o)
 .comment       0x00000000       0x3d c:/program files (x86)/microchip/xc32/v1.21/bin/../lib/gcc/pic32mx/4.5.2/../../../../pic32mx/lib/size\libmchp_peripheral_32MX795F512L.a(int_enable_mv_int_lib.o)
 .comment       0x00000000       0x3d c:/program files (x86)/microchip/xc32/v1.21/bin/../lib/gcc/pic32mx/4.5.2/../../../../pic32mx/lib/size\libmchp_peripheral_32MX795F512L.a(int_tbl_lib.o)
 .comment       0x00000000       0x3d c:/program files (x86)/microchip/xc32/v1.21/bin/../lib/gcc/pic32mx/4.5.2/../../../../pic32mx/lib/size\libmchp_peripheral_32MX795F512L.a(rtcc_init_lib.o)
 .comment       0x00000000       0x3d c:/program files (x86)/microchip/xc32/v1.21/bin/../lib/gcc/pic32mx/4.5.2/../../../../pic32mx/lib/size\libmchp_peripheral_32MX795F512L.a(rtcc_open_lib.o)
 .comment       0x00000000       0x3d c:/program files (x86)/microchip/xc32/v1.21/bin/../lib/gcc/pic32mx/4.5.2/../../../../pic32mx/lib/size\libmchp_peripheral_32MX795F512L.a(spi_chn_data_rdy_lib.o)
 .comment       0x00000000       0x3d c:/program files (x86)/microchip/xc32/v1.21/bin/../lib/gcc/pic32mx/4.5.2/../../../../pic32mx/lib/size\libmchp_peripheral_32MX795F512L.a(spi_chn_getc_lib.o)
 .comment       0x00000000       0x3d c:/program files (x86)/microchip/xc32/v1.21/bin/../lib/gcc/pic32mx/4.5.2/../../../../pic32mx/lib/size\libmchp_peripheral_32MX795F512L.a(spi_chn_open_lib.o)
 .comment       0x00000000       0x3d c:/program files (x86)/microchip/xc32/v1.21/bin/../lib/gcc/pic32mx/4.5.2/../../../../pic32mx/lib/size\libmchp_peripheral_32MX795F512L.a(spi_chn_putc_lib.o)
 .comment       0x00000000       0x3d c:/program files (x86)/microchip/xc32/v1.21/bin/../lib/gcc/pic32mx/4.5.2/../../../../pic32mx/lib/size\libmchp_peripheral_32MX795F512L.a(spi_chn_tx_buff_empty_lib.o)
 .comment       0x00000000       0x3d c:/program files (x86)/microchip/xc32/v1.21/bin/../lib/gcc/pic32mx/4.5.2/../../../../pic32mx/lib/size\libmchp_peripheral_32MX795F512L.a(spi_io_tbl_libp.o)
 .comment       0x00000000       0x3d c:/program files (x86)/microchip/xc32/v1.21/bin/../lib/gcc/pic32mx/4.5.2/../../../../pic32mx/lib/size\libmchp_peripheral_32MX795F512L.a(spi_map_tbl_libp.o)
 .comment       0x00000000       0x3d c:/program files (x86)/microchip/xc32/v1.21/bin/../lib/gcc/pic32mx/4.5.2/../../../../pic32mx/lib/size\libmchp_peripheral_32MX795F512L.a(port_set_pins_digital_in_lib.o)
 .comment       0x00000000       0x3d c:/program files (x86)/microchip/xc32/v1.21/bin/../lib/gcc/pic32mx/4.5.2/../../../../pic32mx/lib/size\libmchp_peripheral_32MX795F512L.a(port_set_pins_digital_out_lib.o)
 .comment       0x00000000       0x3d c:/program files (x86)/microchip/xc32/v1.21/bin/../lib/gcc/pic32mx/4.5.2/../../../../pic32mx/lib/size\libmchp_peripheral_32MX795F512L.a(_ports_tbl_libp.o)
 .comment       0x00000000       0x3d c:/program files (x86)/microchip/xc32/v1.21/bin/../lib/gcc/pic32mx/4.5.2/../../../../pic32mx/lib/size\libmchp_peripheral_32MX795F512L.a(int_enable_interrupts_lib.o)
 .comment       0x00000000       0x3d c:/program files (x86)/microchip/xc32/v1.21/bin/../lib/gcc/pic32mx/4.5.2/../../../../pic32mx/lib/size\libmchp_peripheral_32MX795F512L.a(_rtcc_wait_clock_off_lib.o)
 .comment       0x00000000       0x3d c:/program files (x86)/microchip/xc32/v1.21/bin/../lib/gcc/pic32mx/4.5.2/../../../../pic32mx/lib/size\libmchp_peripheral_32MX795F512L.a(read_core_timer_lib.o)
 .comment       0x00000000       0x3d c:/program files (x86)/microchip/xc32/v1.21/bin/../lib/gcc/pic32mx/4.5.2/size\libgcc.a(_udivdi3.o)
 .comment       0x00000078       0x18 c:/program files (x86)/microchip/xc32/v1.21/bin/../lib/gcc/pic32mx/4.5.2/../../../../pic32mx/lib/size\libpic32.a(memcmp.o)
                                 0x19 (size before relaxing)
 .comment       0x00000090       0x18 c:/program files (x86)/microchip/xc32/v1.21/bin/../lib/gcc/pic32mx/4.5.2/../../../../pic32mx/lib/size\libpic32.a(memset.o)
                                 0x19 (size before relaxing)
 .comment       0x000000a8       0x55 c:/program files (x86)/microchip/xc32/v1.21/bin/../lib/gcc/pic32mx/4.5.2/../../../../pic32mx/lib/size\libpic32.a(strcmp.o)
                                 0x56 (size before relaxing)
 .comment       0x000000fd       0x19 c:/program files (x86)/microchip/xc32/v1.21/bin/../lib/gcc/pic32mx/4.5.2/../../../../pic32mx/lib/size\libpic32.a(strcpy.o)
                                 0x1a (size before relaxing)
 .comment       0x00000116       0x19 c:/program files (x86)/microchip/xc32/v1.21/bin/../lib/gcc/pic32mx/4.5.2/../../../../pic32mx/lib/size\libpic32.a(strlen.o)
                                 0x1a (size before relaxing)
 .comment       0x00000000       0x3d c:/program files (x86)/microchip/xc32/v1.21/bin/../lib/gcc/pic32mx/4.5.2/../../../../pic32mx/lib/size\libpic32.a(default-bootstrap-exception-handler.o)
 .comment       0x00000000       0x3d c:/program files (x86)/microchip/xc32/v1.21/bin/../lib/gcc/pic32mx/4.5.2/../../../../pic32mx/lib/size\libpic32.a(default-on-reset.o)
 .comment       0x00000000       0x3d c:/program files (x86)/microchip/xc32/v1.21/bin/../lib/gcc/pic32mx/4.5.2/../../../../pic32mx/lib/size\libpic32.a(default-on-bootstrap.o)
 .comment       0x00000000       0x3d c:/program files (x86)/microchip/xc32/v1.21/bin/../lib/gcc/pic32mx/4.5.2/../../../../pic32mx/lib/size\libpic32.a(errno.o)
 .comment       0x00000000       0x3d c:/program files (x86)/microchip/xc32/v1.21/bin/../lib/gcc/pic32mx/4.5.2/../../../../pic32mx/lib/size\libpic32.a(defaultinterrupt.o)
 .comment       0x00000000       0x3d c:/program files (x86)/microchip/xc32/v1.21/bin/../lib/gcc/pic32mx/4.5.2/../../../../pic32mx/lib/size\libc.a(atoi.o)
 .comment       0x00000000       0x3d c:/program files (x86)/microchip/xc32/v1.21/bin/../lib/gcc/pic32mx/4.5.2/../../../../pic32mx/lib/size\libc.a(atol.o)
 .comment       0x0000012f       0x4e c:/program files (x86)/microchip/xc32/v1.21/bin/../lib/gcc/pic32mx/4.5.2/../../../../pic32mx/lib/size\libc.a(ctype.o)
                                 0x8b (size before relaxing)
 .comment       0x00000000       0x3d c:/program files (x86)/microchip/xc32/v1.21/bin/../lib/gcc/pic32mx/4.5.2/../../../../pic32mx/lib/size\libc.a(malloc.o)
 .comment       0x00000000       0x3d c:/program files (x86)/microchip/xc32/v1.21/bin/../lib/gcc/pic32mx/4.5.2/../../../../pic32mx/lib/size\libc.a(rand.o)
 .comment       0x00000000       0x3d c:/program files (x86)/microchip/xc32/v1.21/bin/../lib/gcc/pic32mx/4.5.2/../../../../pic32mx/lib/size\libc.a(strcat.o)
 .comment       0x00000000       0x3d c:/program files (x86)/microchip/xc32/v1.21/bin/../lib/gcc/pic32mx/4.5.2/../../../../pic32mx/lib/size\libc.a(strchr.o)
 .comment       0x00000000       0x3d c:/program files (x86)/microchip/xc32/v1.21/bin/../lib/gcc/pic32mx/4.5.2/../../../../pic32mx/lib/size\libc.a(strncat.o)
 .comment       0x00000000       0x3d c:/program files (x86)/microchip/xc32/v1.21/bin/../lib/gcc/pic32mx/4.5.2/../../../../pic32mx/lib/size\libc.a(strncmp.o)
 .comment       0x00000000       0x3d c:/program files (x86)/microchip/xc32/v1.21/bin/../lib/gcc/pic32mx/4.5.2/../../../../pic32mx/lib/size\libc.a(strncpy.o)
 .comment       0x00000000       0x3d c:/program files (x86)/microchip/xc32/v1.21/bin/../lib/gcc/pic32mx/4.5.2/../../../../pic32mx/lib/size\libc.a(strrchr.o)
 .comment       0x00000000       0x3d c:/program files (x86)/microchip/xc32/v1.21/bin/../lib/gcc/pic32mx/4.5.2/../../../../pic32mx/lib/size\libc.a(strstr.o)
 .comment       0x00000000       0x3d c:/program files (x86)/microchip/xc32/v1.21/bin/../lib/gcc/pic32mx/4.5.2/../../../../pic32mx/lib/size\libc.a(strtol.o)
 .comment       0x00000000       0x3d c:/program files (x86)/microchip/xc32/v1.21/bin/../lib/gcc/pic32mx/4.5.2/../../../../pic32mx/lib/size\libc.a(snprintf_cdnopsuxX.eo)
 .comment       0x00000000       0x3d c:/program files (x86)/microchip/xc32/v1.21/bin/../lib/gcc/pic32mx/4.5.2/../../../../pic32mx/lib/size\libc.a(sprintf_cdnopsuxX.eo)
 .comment       0x00000000       0x3d c:/program files (x86)/microchip/xc32/v1.21/bin/../lib/gcc/pic32mx/4.5.2/../../../../pic32mx/lib/size\libc.a(vsnprintf_cdnopsuxX.eo)
 .comment       0x00000000       0x3d c:/program files (x86)/microchip/xc32/v1.21/bin/../lib/gcc/pic32mx/4.5.2/../../../../pic32mx/lib/size\libc.a(vsnprintf.o)
 .comment       0x0000017d       0x4f c:/program files (x86)/microchip/xc32/v1.21/bin/../lib/gcc/pic32mx/4.5.2/../../../../pic32mx/lib/size\libc.a(ctypef.o)
                                 0x8c (size before relaxing)
 .comment       0x00000000       0x3d c:/program files (x86)/microchip/xc32/v1.21/bin/../lib/gcc/pic32mx/4.5.2/../../../../pic32mx/lib/size\libc.a(doprnt_cdnopsuxX.eo)
 .comment       0x00000000       0x3d c:/program files (x86)/microchip/xc32/v1.21/bin/../lib/gcc/pic32mx/4.5.2/../../../../pic32mx/lib/size\libc.a(doprnt.o)
 .comment       0x00000000       0x3d c:/program files (x86)/microchip/xc32/v1.21/bin/../lib/gcc/pic32mx/4.5.2/../../../../pic32mx/lib/size\libc.a(_fputc_simple.o)
 .comment       0x00000000       0x3d c:/program files (x86)/microchip/xc32/v1.21/bin/../lib/gcc/pic32mx/4.5.2/../../../../pic32mx/lib/size\libc.a(powersf.o)
 .comment       0x00000000       0x3d c:/program files (x86)/microchip/xc32/v1.21/bin/../lib/gcc/pic32mx/4.5.2/../../../../pic32mx/lib/size\libc.a(_iob.o)
 .comment       0x00000000       0x3d c:/program files (x86)/microchip/xc32/v1.21/bin/../lib/gcc/pic32mx/4.5.2/../../../../pic32mx/lib/size\libc.a(_flsbuf_simple.o)
 .comment       0x000001cc       0x4b c:/program files (x86)/microchip/xc32/v1.21/bin/../lib/gcc/pic32mx/4.5.2/../../../../pic32mx/lib/size\libpic32.a(sbrk.o)
                                 0x88 (size before relaxing)
 .comment       0x00000000       0x3d c:/program files (x86)/microchip/xc32/v1.21/bin/../lib/gcc/pic32mx/4.5.2/../../../../pic32mx/lib/size\libpic32.a(write.o)
 .comment       0x00000000       0x3d c:/program files (x86)/microchip/xc32/v1.21/bin/../lib/gcc/pic32mx/4.5.2/../../../../pic32mx/lib/size\libpic32.a(_mon_putc.o)
 .comment       0x00000000       0x3d c:/program files (x86)/microchip/xc32/v1.21/bin/../lib/gcc/pic32mx/4.5.2/../../../../pic32mx/lib/size\libpic32.a(xc32_uart.o)
 .comment       0x00000217       0x9e c:/program files (x86)/microchip/xc32/v1.21/bin/../lib/gcc/pic32mx/4.5.2/../../../../pic32mx/lib/size\libe.a(_floatdisf.o)
                                 0xdb (size before relaxing)
 .comment       0x00000000       0x3d c:/program files (x86)/microchip/xc32/v1.21/bin/../lib/gcc/pic32mx/4.5.2/size\libgcc.a(_lshrdi3.o)
 .comment       0x00000000       0x3d c:/program files (x86)/microchip/xc32/v1.21/bin/../lib/gcc/pic32mx/4.5.2/size\libgcc.a(_floatundisf.o)
 .comment       0x00000000       0x3d c:/program files (x86)/microchip/xc32/v1.21/bin/../lib/gcc/pic32mx/4.5.2/size\libgcc.a(_umoddi3.o)
 .comment       0x00000000       0x3d c:/program files (x86)/microchip/xc32/v1.21/bin/../lib/gcc/pic32mx/4.5.2/size\libgcc.a(floatunsisf.o)

.debug
 *(.debug)

.line
 *(.line)

.debug_srcinfo
 *(.debug_srcinfo)

.debug_sfnames
 *(.debug_sfnames)

.debug_aranges  0x00000000     0x2528
 *(.debug_aranges)
 .debug_aranges
                0x00000000       0x20 build/default/production/_ext/1293749816/bsp.o
 .debug_aranges
                0x00000020       0x28 build/default/production/_ext/101875047/lfsr.o
 .debug_aranges
                0x00000048       0x20 build/default/production/_ext/101875047/big_int_helper_c32.o
 .debug_aranges
                0x00000068       0x80 build/default/production/_ext/101875047/big_int.o
 .debug_aranges
                0x000000e8       0x60 build/default/production/_ext/101875047/hashes.o
 .debug_aranges
                0x00000148       0x58 build/default/production/_ext/101875047/helpers.o
 .debug_aranges
                0x000001a0       0x30 build/default/production/_ext/1472/ping_demo.o
 .debug_aranges
                0x000001d0      0x100 build/default/production/_ext/365611741/system_services.o
 .debug_aranges
                0x000002d0       0xc8 build/default/production/_ext/365611741/system_debug.o
 .debug_aranges
                0x00000398       0x40 build/default/production/_ext/365611741/system_random.o
 .debug_aranges
                0x000003d8       0xc0 build/default/production/_ext/365611741/system_command.o
 .debug_aranges
                0x00000498       0x58 build/default/production/_ext/365611741/system_userio.o
 .debug_aranges
                0x000004f0      0x240 build/default/production/_ext/97638081/sys_fs.o
 .debug_aranges
                0x00000730       0xd8 build/default/production/_ext/97638081/mpfs2.o
 .debug_aranges
                0x00000808       0x50 build/default/production/_ext/792872985/usart.o
 .debug_aranges
                0x00000858       0x48 build/default/production/_ext/792872985/lcd.o
 .debug_aranges
                0x000008a0       0x30 build/default/production/_ext/792872985/drv_spi.o
 .debug_aranges
                0x000008d0       0x70 build/default/production/_ext/792872985/spi_eeprom.o
 .debug_aranges
                0x00000940       0x90 build/default/production/_ext/792872985/drv_media.o
 .debug_aranges
                0x000009d0       0x50 build/default/production/_ext/427700826/tcpip_announce.o
 .debug_aranges
                0x00000a20      0x140 build/default/production/_ext/427700826/http2.o
 .debug_aranges
                0x00000b60      0x138 build/default/production/_ext/427700826/arp.o
 .debug_aranges
                0x00000c98       0xb0 build/default/production/_ext/427700826/dhcp.o
 .debug_aranges
                0x00000d48       0x30 build/default/production/_ext/427700826/dhcps.o
 .debug_aranges
                0x00000d78       0x70 build/default/production/_ext/427700826/dns.o
 .debug_aranges
                0x00000de8      0x130 build/default/production/_ext/427700826/encs24j600.o
 .debug_aranges
                0x00000f18       0xc8 build/default/production/_ext/427700826/encx24_mac.o
 .debug_aranges
                0x00000fe0       0x28 build/default/production/_ext/427700826/hash_fnv.o
 .debug_aranges
                0x00001008       0x58 build/default/production/_ext/427700826/hash_tbl.o
 .debug_aranges
                0x00001060       0x50 build/default/production/_ext/427700826/icmp.o
 .debug_aranges
                0x000010b0      0x150 build/default/production/_ext/427700826/ipv4.o
 .debug_aranges
                0x00001200       0x40 build/default/production/_ext/427700826/nbns.o
 .debug_aranges
                0x00001240      0x288 build/default/production/_ext/427700826/tcp.o
 .debug_aranges
                0x000014c8       0x98 build/default/production/_ext/427700826/tcpip_heap_alloc.o
 .debug_aranges
                0x00001560      0x170 build/default/production/_ext/427700826/udp.o
 .debug_aranges
                0x000016d0       0xb0 build/default/production/_ext/427700826/tcpip_mac_object.o
 .debug_aranges
                0x00001780      0x270 build/default/production/_ext/427700826/tcpip_manager.o
 .debug_aranges
                0x000019f0       0xe8 build/default/production/_ext/427700826/tcpip_helpers.o
 .debug_aranges
                0x00001ad8       0x20 build/default/production/_ext/427700826/tcpip_helper_c32.o
 .debug_aranges
                0x00001af8       0x30 build/default/production/_ext/427700826/tcpip_notify.o
 .debug_aranges
                0x00001b28       0x30 build/default/production/_ext/427700826/zero_conf_link_local.o
 .debug_aranges
                0x00001b58       0x20 build/default/production/_ext/334706090/wf_eint.o
 .debug_aranges
                0x00001b78       0x20 build/default/production/_ext/334706090/wf_spi.o
 .debug_aranges
                0x00001b98       0x28 build/default/production/_ext/1472/main_demo.o
 .debug_aranges
                0x00001bc0      0x158 build/default/production/_ext/1472/custom_http_app.o
 .debug_aranges
                0x00001d18       0x38 build/default/production/_ext/1472/tcp6_demo_app.o
 .debug_aranges
                0x00001d50       0x20 c:/program files (x86)/microchip/xc32/v1.21/bin/../lib/gcc/pic32mx/4.5.2/../../../../pic32mx/lib/size\libmchp_peripheral.a(open_core_timer_lib.o)
 .debug_aranges
                0x00001d70       0x20 c:/program files (x86)/microchip/xc32/v1.21/bin/../lib/gcc/pic32mx/4.5.2/../../../../pic32mx/lib/size\libmchp_peripheral_32MX795F512L.a(soft_reset_lib.o)
 .debug_aranges
                0x00001d90       0x28 c:/program files (x86)/microchip/xc32/v1.21/bin/../lib/gcc/pic32mx/4.5.2/../../../../pic32mx/lib/size\libmchp_peripheral_32MX795F512L.a(pcache.o)
 .debug_aranges
                0x00001db8       0x20 c:/program files (x86)/microchip/xc32/v1.21/bin/../lib/gcc/pic32mx/4.5.2/../../../../pic32mx/lib/size\libmchp_peripheral_32MX795F512L.a(int_disable_interrupts_lib.o)
 .debug_aranges
                0x00001dd8       0x20 c:/program files (x86)/microchip/xc32/v1.21/bin/../lib/gcc/pic32mx/4.5.2/../../../../pic32mx/lib/size\libmchp_peripheral_32MX795F512L.a(int_restore_interrupts_lib.o)
 .debug_aranges
                0x00001df8       0x20 c:/program files (x86)/microchip/xc32/v1.21/bin/../lib/gcc/pic32mx/4.5.2/../../../../pic32mx/lib/size\libmchp_peripheral_32MX795F512L.a(int_enable_mv_int_lib.o)
 .debug_aranges
                0x00001e18       0x60 c:/program files (x86)/microchip/xc32/v1.21/bin/../lib/gcc/pic32mx/4.5.2/../../../../pic32mx/lib/size\libmchp_peripheral_32MX795F512L.a(int_tbl_lib.o)
 .debug_aranges
                0x00001e78       0x20 c:/program files (x86)/microchip/xc32/v1.21/bin/../lib/gcc/pic32mx/4.5.2/../../../../pic32mx/lib/size\libmchp_peripheral_32MX795F512L.a(rtcc_init_lib.o)
 .debug_aranges
                0x00001e98       0x20 c:/program files (x86)/microchip/xc32/v1.21/bin/../lib/gcc/pic32mx/4.5.2/../../../../pic32mx/lib/size\libmchp_peripheral_32MX795F512L.a(rtcc_open_lib.o)
 .debug_aranges
                0x00001eb8       0x20 c:/program files (x86)/microchip/xc32/v1.21/bin/../lib/gcc/pic32mx/4.5.2/../../../../pic32mx/lib/size\libmchp_peripheral_32MX795F512L.a(spi_chn_data_rdy_lib.o)
 .debug_aranges
                0x00001ed8       0x28 c:/program files (x86)/microchip/xc32/v1.21/bin/../lib/gcc/pic32mx/4.5.2/../../../../pic32mx/lib/size\libmchp_peripheral_32MX795F512L.a(spi_chn_getc_lib.o)
 .debug_aranges
                0x00001f00       0x20 c:/program files (x86)/microchip/xc32/v1.21/bin/../lib/gcc/pic32mx/4.5.2/../../../../pic32mx/lib/size\libmchp_peripheral_32MX795F512L.a(spi_chn_open_lib.o)
 .debug_aranges
                0x00001f20       0x30 c:/program files (x86)/microchip/xc32/v1.21/bin/../lib/gcc/pic32mx/4.5.2/../../../../pic32mx/lib/size\libmchp_peripheral_32MX795F512L.a(spi_chn_putc_lib.o)
 .debug_aranges
                0x00001f50       0x20 c:/program files (x86)/microchip/xc32/v1.21/bin/../lib/gcc/pic32mx/4.5.2/../../../../pic32mx/lib/size\libmchp_peripheral_32MX795F512L.a(spi_chn_tx_buff_empty_lib.o)
 .debug_aranges
                0x00001f70       0x20 c:/program files (x86)/microchip/xc32/v1.21/bin/../lib/gcc/pic32mx/4.5.2/../../../../pic32mx/lib/size\libmchp_peripheral_32MX795F512L.a(port_set_pins_digital_in_lib.o)
 .debug_aranges
                0x00001f90       0x20 c:/program files (x86)/microchip/xc32/v1.21/bin/../lib/gcc/pic32mx/4.5.2/../../../../pic32mx/lib/size\libmchp_peripheral_32MX795F512L.a(port_set_pins_digital_out_lib.o)
 .debug_aranges
                0x00001fb0       0x20 c:/program files (x86)/microchip/xc32/v1.21/bin/../lib/gcc/pic32mx/4.5.2/../../../../pic32mx/lib/size\libmchp_peripheral_32MX795F512L.a(int_enable_interrupts_lib.o)
 .debug_aranges
                0x00001fd0       0x28 c:/program files (x86)/microchip/xc32/v1.21/bin/../lib/gcc/pic32mx/4.5.2/../../../../pic32mx/lib/size\libmchp_peripheral_32MX795F512L.a(_rtcc_wait_clock_off_lib.o)
 .debug_aranges
                0x00001ff8       0x20 c:/program files (x86)/microchip/xc32/v1.21/bin/../lib/gcc/pic32mx/4.5.2/../../../../pic32mx/lib/size\libmchp_peripheral_32MX795F512L.a(read_core_timer_lib.o)
 .debug_aranges
                0x00002018       0x20 c:/program files (x86)/microchip/xc32/v1.21/bin/../lib/gcc/pic32mx/4.5.2/size\libgcc.a(_udivdi3.o)
 .debug_aranges
                0x00002038       0x20 c:/program files (x86)/microchip/xc32/v1.21/bin/../lib/gcc/pic32mx/4.5.2/../../../../pic32mx/lib/size\libpic32.a(default-bootstrap-exception-handler.o)
 .debug_aranges
                0x00002058       0x20 c:/program files (x86)/microchip/xc32/v1.21/bin/../lib/gcc/pic32mx/4.5.2/../../../../pic32mx/lib/size\libpic32.a(default-on-reset.o)
 .debug_aranges
                0x00002078       0x20 c:/program files (x86)/microchip/xc32/v1.21/bin/../lib/gcc/pic32mx/4.5.2/../../../../pic32mx/lib/size\libpic32.a(default-on-bootstrap.o)
 .debug_aranges
                0x00002098       0x20 c:/program files (x86)/microchip/xc32/v1.21/bin/../lib/gcc/pic32mx/4.5.2/../../../../pic32mx/lib/size\libpic32.a(defaultinterrupt.o)
 .debug_aranges
                0x000020b8       0x20 c:/program files (x86)/microchip/xc32/v1.21/bin/../lib/gcc/pic32mx/4.5.2/../../../../pic32mx/lib/size\libc.a(atoi.o)
 .debug_aranges
                0x000020d8       0x20 c:/program files (x86)/microchip/xc32/v1.21/bin/../lib/gcc/pic32mx/4.5.2/../../../../pic32mx/lib/size\libc.a(atol.o)
 .debug_aranges
                0x000020f8       0x30 c:/program files (x86)/microchip/xc32/v1.21/bin/../lib/gcc/pic32mx/4.5.2/../../../../pic32mx/lib/size\libc.a(malloc.o)
 .debug_aranges
                0x00002128       0x28 c:/program files (x86)/microchip/xc32/v1.21/bin/../lib/gcc/pic32mx/4.5.2/../../../../pic32mx/lib/size\libc.a(rand.o)
 .debug_aranges
                0x00002150       0x20 c:/program files (x86)/microchip/xc32/v1.21/bin/../lib/gcc/pic32mx/4.5.2/../../../../pic32mx/lib/size\libc.a(strcat.o)
 .debug_aranges
                0x00002170       0x20 c:/program files (x86)/microchip/xc32/v1.21/bin/../lib/gcc/pic32mx/4.5.2/../../../../pic32mx/lib/size\libc.a(strchr.o)
 .debug_aranges
                0x00002190       0x20 c:/program files (x86)/microchip/xc32/v1.21/bin/../lib/gcc/pic32mx/4.5.2/../../../../pic32mx/lib/size\libc.a(strncat.o)
 .debug_aranges
                0x000021b0       0x20 c:/program files (x86)/microchip/xc32/v1.21/bin/../lib/gcc/pic32mx/4.5.2/../../../../pic32mx/lib/size\libc.a(strncmp.o)
 .debug_aranges
                0x000021d0       0x20 c:/program files (x86)/microchip/xc32/v1.21/bin/../lib/gcc/pic32mx/4.5.2/../../../../pic32mx/lib/size\libc.a(strncpy.o)
 .debug_aranges
                0x000021f0       0x20 c:/program files (x86)/microchip/xc32/v1.21/bin/../lib/gcc/pic32mx/4.5.2/../../../../pic32mx/lib/size\libc.a(strrchr.o)
 .debug_aranges
                0x00002210       0x20 c:/program files (x86)/microchip/xc32/v1.21/bin/../lib/gcc/pic32mx/4.5.2/../../../../pic32mx/lib/size\libc.a(strstr.o)
 .debug_aranges
                0x00002230       0x28 c:/program files (x86)/microchip/xc32/v1.21/bin/../lib/gcc/pic32mx/4.5.2/../../../../pic32mx/lib/size\libc.a(strtol.o)
 .debug_aranges
                0x00002258       0x20 c:/program files (x86)/microchip/xc32/v1.21/bin/../lib/gcc/pic32mx/4.5.2/../../../../pic32mx/lib/size\libc.a(snprintf_cdnopsuxX.eo)
 .debug_aranges
                0x00002278       0x20 c:/program files (x86)/microchip/xc32/v1.21/bin/../lib/gcc/pic32mx/4.5.2/../../../../pic32mx/lib/size\libc.a(sprintf_cdnopsuxX.eo)
 .debug_aranges
                0x00002298       0x20 c:/program files (x86)/microchip/xc32/v1.21/bin/../lib/gcc/pic32mx/4.5.2/../../../../pic32mx/lib/size\libc.a(vsnprintf_cdnopsuxX.eo)
 .debug_aranges
                0x000022b8       0x20 c:/program files (x86)/microchip/xc32/v1.21/bin/../lib/gcc/pic32mx/4.5.2/../../../../pic32mx/lib/size\libc.a(vsnprintf.o)
 .debug_aranges
                0x000022d8       0xa0 c:/program files (x86)/microchip/xc32/v1.21/bin/../lib/gcc/pic32mx/4.5.2/../../../../pic32mx/lib/size\libc.a(ctypef.o)
 .debug_aranges
                0x00002378       0x20 c:/program files (x86)/microchip/xc32/v1.21/bin/../lib/gcc/pic32mx/4.5.2/../../../../pic32mx/lib/size\libc.a(doprnt_cdnopsuxX.eo)
 .debug_aranges
                0x00002398       0x30 c:/program files (x86)/microchip/xc32/v1.21/bin/../lib/gcc/pic32mx/4.5.2/../../../../pic32mx/lib/size\libc.a(doprnt.o)
 .debug_aranges
                0x000023c8       0x20 c:/program files (x86)/microchip/xc32/v1.21/bin/../lib/gcc/pic32mx/4.5.2/../../../../pic32mx/lib/size\libc.a(_fputc_simple.o)
 .debug_aranges
                0x000023e8       0x20 c:/program files (x86)/microchip/xc32/v1.21/bin/../lib/gcc/pic32mx/4.5.2/../../../../pic32mx/lib/size\libc.a(_flsbuf_simple.o)
 .debug_aranges
                0x00002408       0x40 c:/program files (x86)/microchip/xc32/v1.21/bin/../lib/gcc/pic32mx/4.5.2/../../../../pic32mx/lib/size\libpic32.a(sbrk.o)
 .debug_aranges
                0x00002448       0x20 c:/program files (x86)/microchip/xc32/v1.21/bin/../lib/gcc/pic32mx/4.5.2/../../../../pic32mx/lib/size\libpic32.a(write.o)
 .debug_aranges
                0x00002468       0x20 c:/program files (x86)/microchip/xc32/v1.21/bin/../lib/gcc/pic32mx/4.5.2/../../../../pic32mx/lib/size\libpic32.a(_mon_putc.o)
 .debug_aranges
                0x00002488       0x20 c:/program files (x86)/microchip/xc32/v1.21/bin/../lib/gcc/pic32mx/4.5.2/../../../../pic32mx/lib/size\libe.a(_floatdisf.o)
 .debug_aranges
                0x000024a8       0x20 c:/program files (x86)/microchip/xc32/v1.21/bin/../lib/gcc/pic32mx/4.5.2/size\libgcc.a(_lshrdi3.o)
 .debug_aranges
                0x000024c8       0x20 c:/program files (x86)/microchip/xc32/v1.21/bin/../lib/gcc/pic32mx/4.5.2/size\libgcc.a(_floatundisf.o)
 .debug_aranges
                0x000024e8       0x20 c:/program files (x86)/microchip/xc32/v1.21/bin/../lib/gcc/pic32mx/4.5.2/size\libgcc.a(_umoddi3.o)
 .debug_aranges
                0x00002508       0x20 c:/program files (x86)/microchip/xc32/v1.21/bin/../lib/gcc/pic32mx/4.5.2/size\libgcc.a(floatunsisf.o)

.debug_pubnames
                0x00000000     0x4823
 *(.debug_pubnames)
 .debug_pubnames
                0x00000000       0x25 build/default/production/_ext/1293749816/bsp.o
 .debug_pubnames
                0x00000025       0x30 build/default/production/_ext/101875047/lfsr.o
 .debug_pubnames
                0x00000055       0xeb build/default/production/_ext/101875047/big_int.o
 .debug_pubnames
                0x00000140       0x97 build/default/production/_ext/101875047/hashes.o
 .debug_pubnames
                0x000001d7       0x81 build/default/production/_ext/101875047/helpers.o
 .debug_pubnames
                0x00000258       0xc4 build/default/production/_ext/1472/ping_demo.o
 .debug_pubnames
                0x0000031c      0x36a build/default/production/_ext/365611741/system_services.o
 .debug_pubnames
                0x00000686      0x1e1 build/default/production/_ext/365611741/system_debug.o
 .debug_pubnames
                0x00000867       0x83 build/default/production/_ext/365611741/system_random.o
 .debug_pubnames
                0x000008ea       0xab build/default/production/_ext/365611741/system_command.o
 .debug_pubnames
                0x00000995       0xc8 build/default/production/_ext/365611741/system_userio.o
 .debug_pubnames
                0x00000a5d      0x575 build/default/production/_ext/97638081/sys_fs.o
 .debug_pubnames
                0x00000fd2      0x17e build/default/production/_ext/97638081/mpfs2.o
 .debug_pubnames
                0x00001150       0x94 build/default/production/_ext/792872985/usart.o
 .debug_pubnames
                0x000011e4       0x77 build/default/production/_ext/792872985/lcd.o
 .debug_pubnames
                0x0000125b       0x3a build/default/production/_ext/792872985/drv_spi.o
 .debug_pubnames
                0x00001295       0xaa build/default/production/_ext/792872985/spi_eeprom.o
 .debug_pubnames
                0x0000133f      0x169 build/default/production/_ext/792872985/drv_media.o
 .debug_pubnames
                0x000014a8       0x93 build/default/production/_ext/427700826/tcpip_announce.o
 .debug_pubnames
                0x0000153b      0x2cc build/default/production/_ext/427700826/http2.o
 .debug_pubnames
                0x00001807      0x1ba build/default/production/_ext/427700826/arp.o
 .debug_pubnames
                0x000019c1       0xfb build/default/production/_ext/427700826/dhcp.o
 .debug_pubnames
                0x00001abc       0x55 build/default/production/_ext/427700826/dhcps.o
 .debug_pubnames
                0x00001b11       0x8d build/default/production/_ext/427700826/dns.o
 .debug_pubnames
                0x00001b9e      0x24c build/default/production/_ext/427700826/encs24j600.o
 .debug_pubnames
                0x00001dea       0x59 build/default/production/_ext/427700826/encx24_mac.o
 .debug_pubnames
                0x00001e43       0x33 build/default/production/_ext/427700826/hash_fnv.o
 .debug_pubnames
                0x00001e76       0x86 build/default/production/_ext/427700826/hash_tbl.o
 .debug_pubnames
                0x00001efc       0x7e build/default/production/_ext/427700826/icmp.o
 .debug_pubnames
                0x00001f7a      0x47f build/default/production/_ext/427700826/ipv4.o
 .debug_pubnames
                0x000023f9       0x3b build/default/production/_ext/427700826/nbns.o
 .debug_pubnames
                0x00002434      0x2b3 build/default/production/_ext/427700826/tcp.o
 .debug_pubnames
                0x000026e7      0x18c build/default/production/_ext/427700826/tcpip_heap_alloc.o
 .debug_pubnames
                0x00002873      0x25a build/default/production/_ext/427700826/udp.o
 .debug_pubnames
                0x00002acd      0x17b build/default/production/_ext/427700826/tcpip_mac_object.o
 .debug_pubnames
                0x00002c48      0x71e build/default/production/_ext/427700826/tcpip_manager.o
 .debug_pubnames
                0x00003366      0x2e1 build/default/production/_ext/427700826/tcpip_helpers.o
 .debug_pubnames
                0x00003647       0x69 build/default/production/_ext/427700826/tcpip_notify.o
 .debug_pubnames
                0x000036b0       0x43 build/default/production/_ext/427700826/zero_conf_link_local.o
 .debug_pubnames
                0x000036f3       0x2a build/default/production/_ext/334706090/wf_eint.o
 .debug_pubnames
                0x0000371d       0x29 build/default/production/_ext/334706090/wf_spi.o
 .debug_pubnames
                0x00003746      0x144 build/default/production/_ext/1472/main_demo.o
 .debug_pubnames
                0x0000388a      0x3a2 build/default/production/_ext/1472/custom_http_app.o
 .debug_pubnames
                0x00003c2c      0x298 build/default/production/_ext/1472/tcp6_demo_app.o
 .debug_pubnames
                0x00003ec4       0x24 c:/program files (x86)/microchip/xc32/v1.21/bin/../lib/gcc/pic32mx/4.5.2/../../../../pic32mx/lib/size\libmchp_peripheral.a(open_core_timer_lib.o)
 .debug_pubnames
                0x00003ee8       0x20 c:/program files (x86)/microchip/xc32/v1.21/bin/../lib/gcc/pic32mx/4.5.2/../../../../pic32mx/lib/size\libmchp_peripheral_32MX795F512L.a(soft_reset_lib.o)
 .debug_pubnames
                0x00003f08       0x3b c:/program files (x86)/microchip/xc32/v1.21/bin/../lib/gcc/pic32mx/4.5.2/../../../../pic32mx/lib/size\libmchp_peripheral_32MX795F512L.a(pcache.o)
 .debug_pubnames
                0x00003f43       0x2b c:/program files (x86)/microchip/xc32/v1.21/bin/../lib/gcc/pic32mx/4.5.2/../../../../pic32mx/lib/size\libmchp_peripheral_32MX795F512L.a(int_disable_interrupts_lib.o)
 .debug_pubnames
                0x00003f6e       0x2b c:/program files (x86)/microchip/xc32/v1.21/bin/../lib/gcc/pic32mx/4.5.2/../../../../pic32mx/lib/size\libmchp_peripheral_32MX795F512L.a(int_restore_interrupts_lib.o)
 .debug_pubnames
                0x00003f99       0x36 c:/program files (x86)/microchip/xc32/v1.21/bin/../lib/gcc/pic32mx/4.5.2/../../../../pic32mx/lib/size\libmchp_peripheral_32MX795F512L.a(int_enable_mv_int_lib.o)
 .debug_pubnames
                0x00003fcf       0xca c:/program files (x86)/microchip/xc32/v1.21/bin/../lib/gcc/pic32mx/4.5.2/../../../../pic32mx/lib/size\libmchp_peripheral_32MX795F512L.a(int_tbl_lib.o)
 .debug_pubnames
                0x00004099       0x1f c:/program files (x86)/microchip/xc32/v1.21/bin/../lib/gcc/pic32mx/4.5.2/../../../../pic32mx/lib/size\libmchp_peripheral_32MX795F512L.a(rtcc_init_lib.o)
 .debug_pubnames
                0x000040b8       0x1f c:/program files (x86)/microchip/xc32/v1.21/bin/../lib/gcc/pic32mx/4.5.2/../../../../pic32mx/lib/size\libmchp_peripheral_32MX795F512L.a(rtcc_open_lib.o)
 .debug_pubnames
                0x000040d7       0x24 c:/program files (x86)/microchip/xc32/v1.21/bin/../lib/gcc/pic32mx/4.5.2/../../../../pic32mx/lib/size\libmchp_peripheral_32MX795F512L.a(spi_chn_data_rdy_lib.o)
 .debug_pubnames
                0x000040fb       0x31 c:/program files (x86)/microchip/xc32/v1.21/bin/../lib/gcc/pic32mx/4.5.2/../../../../pic32mx/lib/size\libmchp_peripheral_32MX795F512L.a(spi_chn_getc_lib.o)
 .debug_pubnames
                0x0000412c       0x21 c:/program files (x86)/microchip/xc32/v1.21/bin/../lib/gcc/pic32mx/4.5.2/../../../../pic32mx/lib/size\libmchp_peripheral_32MX795F512L.a(spi_chn_open_lib.o)
 .debug_pubnames
                0x0000414d       0x43 c:/program files (x86)/microchip/xc32/v1.21/bin/../lib/gcc/pic32mx/4.5.2/../../../../pic32mx/lib/size\libmchp_peripheral_32MX795F512L.a(spi_chn_putc_lib.o)
 .debug_pubnames
                0x00004190       0x28 c:/program files (x86)/microchip/xc32/v1.21/bin/../lib/gcc/pic32mx/4.5.2/../../../../pic32mx/lib/size\libmchp_peripheral_32MX795F512L.a(spi_chn_tx_buff_empty_lib.o)
 .debug_pubnames
                0x000041b8       0x2b c:/program files (x86)/microchip/xc32/v1.21/bin/../lib/gcc/pic32mx/4.5.2/../../../../pic32mx/lib/size\libmchp_peripheral_32MX795F512L.a(port_set_pins_digital_in_lib.o)
 .debug_pubnames
                0x000041e3       0x2c c:/program files (x86)/microchip/xc32/v1.21/bin/../lib/gcc/pic32mx/4.5.2/../../../../pic32mx/lib/size\libmchp_peripheral_32MX795F512L.a(port_set_pins_digital_out_lib.o)
 .debug_pubnames
                0x0000420f       0x2a c:/program files (x86)/microchip/xc32/v1.21/bin/../lib/gcc/pic32mx/4.5.2/../../../../pic32mx/lib/size\libmchp_peripheral_32MX795F512L.a(int_enable_interrupts_lib.o)
 .debug_pubnames
                0x00004239       0x3e c:/program files (x86)/microchip/xc32/v1.21/bin/../lib/gcc/pic32mx/4.5.2/../../../../pic32mx/lib/size\libmchp_peripheral_32MX795F512L.a(_rtcc_wait_clock_off_lib.o)
 .debug_pubnames
                0x00004277       0x24 c:/program files (x86)/microchip/xc32/v1.21/bin/../lib/gcc/pic32mx/4.5.2/../../../../pic32mx/lib/size\libmchp_peripheral_32MX795F512L.a(read_core_timer_lib.o)
 .debug_pubnames
                0x0000429b       0x20 c:/program files (x86)/microchip/xc32/v1.21/bin/../lib/gcc/pic32mx/4.5.2/size\libgcc.a(_udivdi3.o)
 .debug_pubnames
                0x000042bb       0x33 c:/program files (x86)/microchip/xc32/v1.21/bin/../lib/gcc/pic32mx/4.5.2/../../../../pic32mx/lib/size\libpic32.a(default-bootstrap-exception-handler.o)
 .debug_pubnames
                0x000042ee       0x20 c:/program files (x86)/microchip/xc32/v1.21/bin/../lib/gcc/pic32mx/4.5.2/../../../../pic32mx/lib/size\libpic32.a(default-on-reset.o)
 .debug_pubnames
                0x0000430e       0x24 c:/program files (x86)/microchip/xc32/v1.21/bin/../lib/gcc/pic32mx/4.5.2/../../../../pic32mx/lib/size\libpic32.a(default-on-bootstrap.o)
 .debug_pubnames
                0x00004332       0x28 c:/program files (x86)/microchip/xc32/v1.21/bin/../lib/gcc/pic32mx/4.5.2/../../../../pic32mx/lib/size\libpic32.a(defaultinterrupt.o)
 .debug_pubnames
                0x0000435a       0x1b c:/program files (x86)/microchip/xc32/v1.21/bin/../lib/gcc/pic32mx/4.5.2/../../../../pic32mx/lib/size\libc.a(atoi.o)
 .debug_pubnames
                0x00004375       0x1b c:/program files (x86)/microchip/xc32/v1.21/bin/../lib/gcc/pic32mx/4.5.2/../../../../pic32mx/lib/size\libc.a(atol.o)
 .debug_pubnames
                0x00004390       0x32 c:/program files (x86)/microchip/xc32/v1.21/bin/../lib/gcc/pic32mx/4.5.2/../../../../pic32mx/lib/size\libc.a(malloc.o)
 .debug_pubnames
                0x000043c2       0x25 c:/program files (x86)/microchip/xc32/v1.21/bin/../lib/gcc/pic32mx/4.5.2/../../../../pic32mx/lib/size\libc.a(rand.o)
 .debug_pubnames
                0x000043e7       0x1d c:/program files (x86)/microchip/xc32/v1.21/bin/../lib/gcc/pic32mx/4.5.2/../../../../pic32mx/lib/size\libc.a(strcat.o)
 .debug_pubnames
                0x00004404       0x1d c:/program files (x86)/microchip/xc32/v1.21/bin/../lib/gcc/pic32mx/4.5.2/../../../../pic32mx/lib/size\libc.a(strchr.o)
 .debug_pubnames
                0x00004421       0x1e c:/program files (x86)/microchip/xc32/v1.21/bin/../lib/gcc/pic32mx/4.5.2/../../../../pic32mx/lib/size\libc.a(strncat.o)
 .debug_pubnames
                0x0000443f       0x1e c:/program files (x86)/microchip/xc32/v1.21/bin/../lib/gcc/pic32mx/4.5.2/../../../../pic32mx/lib/size\libc.a(strncmp.o)
 .debug_pubnames
                0x0000445d       0x1e c:/program files (x86)/microchip/xc32/v1.21/bin/../lib/gcc/pic32mx/4.5.2/../../../../pic32mx/lib/size\libc.a(strncpy.o)
 .debug_pubnames
                0x0000447b       0x1e c:/program files (x86)/microchip/xc32/v1.21/bin/../lib/gcc/pic32mx/4.5.2/../../../../pic32mx/lib/size\libc.a(strrchr.o)
 .debug_pubnames
                0x00004499       0x1d c:/program files (x86)/microchip/xc32/v1.21/bin/../lib/gcc/pic32mx/4.5.2/../../../../pic32mx/lib/size\libc.a(strstr.o)
 .debug_pubnames
                0x000044b6       0x29 c:/program files (x86)/microchip/xc32/v1.21/bin/../lib/gcc/pic32mx/4.5.2/../../../../pic32mx/lib/size\libc.a(strtol.o)
 .debug_pubnames
                0x000044df       0x2a c:/program files (x86)/microchip/xc32/v1.21/bin/../lib/gcc/pic32mx/4.5.2/../../../../pic32mx/lib/size\libc.a(snprintf_cdnopsuxX.eo)
 .debug_pubnames
                0x00004509       0x29 c:/program files (x86)/microchip/xc32/v1.21/bin/../lib/gcc/pic32mx/4.5.2/../../../../pic32mx/lib/size\libc.a(sprintf_cdnopsuxX.eo)
 .debug_pubnames
                0x00004532       0x2b c:/program files (x86)/microchip/xc32/v1.21/bin/../lib/gcc/pic32mx/4.5.2/../../../../pic32mx/lib/size\libc.a(vsnprintf_cdnopsuxX.eo)
 .debug_pubnames
                0x0000455d       0x20 c:/program files (x86)/microchip/xc32/v1.21/bin/../lib/gcc/pic32mx/4.5.2/../../../../pic32mx/lib/size\libc.a(vsnprintf.o)
 .debug_pubnames
                0x0000457d       0xe1 c:/program files (x86)/microchip/xc32/v1.21/bin/../lib/gcc/pic32mx/4.5.2/../../../../pic32mx/lib/size\libc.a(ctypef.o)
 .debug_pubnames
                0x0000465e       0x2a c:/program files (x86)/microchip/xc32/v1.21/bin/../lib/gcc/pic32mx/4.5.2/../../../../pic32mx/lib/size\libc.a(doprnt_cdnopsuxX.eo)
 .debug_pubnames
                0x00004688       0x1f c:/program files (x86)/microchip/xc32/v1.21/bin/../lib/gcc/pic32mx/4.5.2/../../../../pic32mx/lib/size\libc.a(doprnt.o)
 .debug_pubnames
                0x000046a7       0x1c c:/program files (x86)/microchip/xc32/v1.21/bin/../lib/gcc/pic32mx/4.5.2/../../../../pic32mx/lib/size\libc.a(_fputc_simple.o)
 .debug_pubnames
                0x000046c3       0x1e c:/program files (x86)/microchip/xc32/v1.21/bin/../lib/gcc/pic32mx/4.5.2/../../../../pic32mx/lib/size\libc.a(_flsbuf_simple.o)
 .debug_pubnames
                0x000046e1       0x5c c:/program files (x86)/microchip/xc32/v1.21/bin/../lib/gcc/pic32mx/4.5.2/../../../../pic32mx/lib/size\libpic32.a(sbrk.o)
 .debug_pubnames
                0x0000473d       0x1c c:/program files (x86)/microchip/xc32/v1.21/bin/../lib/gcc/pic32mx/4.5.2/../../../../pic32mx/lib/size\libpic32.a(write.o)
 .debug_pubnames
                0x00004759       0x20 c:/program files (x86)/microchip/xc32/v1.21/bin/../lib/gcc/pic32mx/4.5.2/../../../../pic32mx/lib/size\libpic32.a(_mon_putc.o)
 .debug_pubnames
                0x00004779       0x22 c:/program files (x86)/microchip/xc32/v1.21/bin/../lib/gcc/pic32mx/4.5.2/../../../../pic32mx/lib/size\libe.a(_floatdisf.o)
 .debug_pubnames
                0x0000479b       0x20 c:/program files (x86)/microchip/xc32/v1.21/bin/../lib/gcc/pic32mx/4.5.2/size\libgcc.a(_lshrdi3.o)
 .debug_pubnames
                0x000047bb       0x24 c:/program files (x86)/microchip/xc32/v1.21/bin/../lib/gcc/pic32mx/4.5.2/size\libgcc.a(_floatundisf.o)
 .debug_pubnames
                0x000047df       0x20 c:/program files (x86)/microchip/xc32/v1.21/bin/../lib/gcc/pic32mx/4.5.2/size\libgcc.a(_umoddi3.o)
 .debug_pubnames
                0x000047ff       0x24 c:/program files (x86)/microchip/xc32/v1.21/bin/../lib/gcc/pic32mx/4.5.2/size\libgcc.a(floatunsisf.o)

.debug_info     0x00000000    0xa03d1
 *(.debug_info .gnu.linkonce.wi.*)
 .debug_info    0x00000000     0x1a0c build/default/production/_ext/1293749816/bsp.o
 .debug_info    0x00001a0c      0x21b build/default/production/_ext/101875047/lfsr.o
 .debug_info    0x00001c27       0xb5 build/default/production/_ext/101875047/big_int_helper_c32.o
 .debug_info    0x00001cdc     0x1739 build/default/production/_ext/101875047/big_int.o
 .debug_info    0x00003415      0x824 build/default/production/_ext/101875047/hashes.o
 .debug_info    0x00003c39      0x50d build/default/production/_ext/101875047/helpers.o
 .debug_info    0x00004146        0x0 build/default/production/_ext/1472/berkeley_tcp_client_demo.o
 .debug_info    0x00004146        0x0 build/default/production/_ext/1472/berkeley_tcp_server_demo.o
 .debug_info    0x00004146        0x0 build/default/production/_ext/1472/berkeley_udp_client_demo.o
 .debug_info    0x00004146     0x11c8 build/default/production/_ext/1472/generic_tcp_client.o
 .debug_info    0x0000530e     0x11c8 build/default/production/_ext/1472/generic_tcp_server.o
 .debug_info    0x000064d6     0x1a63 build/default/production/_ext/1472/ping_demo.o
 .debug_info    0x00007f39        0x0 build/default/production/_ext/1472/smtp_demo.o
 .debug_info    0x00007f39     0x3449 build/default/production/_ext/365611741/system_services.o
 .debug_info    0x0000b382     0x1732 build/default/production/_ext/365611741/system_debug.o
 .debug_info    0x0000cab4     0x1c4c build/default/production/_ext/365611741/system_random.o
 .debug_info    0x0000e700     0x1a6c build/default/production/_ext/365611741/system_command.o
 .debug_info    0x0001016c     0x21c2 build/default/production/_ext/365611741/system_userio.o
 .debug_info    0x0001232e     0x2c2a build/default/production/_ext/97638081/sys_fs.o
 .debug_info    0x00014f58     0x1c9d build/default/production/_ext/97638081/mpfs2.o
 .debug_info    0x00016bf5     0x1668 build/default/production/_ext/792872985/usart.o
 .debug_info    0x0001825d     0x1b40 build/default/production/_ext/792872985/lcd.o
 .debug_info    0x00019d9d     0x168e build/default/production/_ext/792872985/drv_spi.o
 .debug_info    0x0001b42b        0x0 build/default/production/_ext/792872985/db_appio.o
 .debug_info    0x0001b42b     0x1185 build/default/production/_ext/792872985/spi_ram.o
 .debug_info    0x0001c5b0     0x1fdc build/default/production/_ext/792872985/spi_eeprom.o
 .debug_info    0x0001e58c     0x1187 build/default/production/_ext/792872985/spi_flash.o
 .debug_info    0x0001f713     0x22ef build/default/production/_ext/792872985/drv_media.o
 .debug_info    0x00021a02     0x224d build/default/production/_ext/427700826/tcpip_announce.o
 .debug_info    0x00023c4f     0x3e1e build/default/production/_ext/427700826/http2.o
 .debug_info    0x00027a6d     0x1386 build/default/production/_ext/427700826/arcfour.o
 .debug_info    0x00028df3     0x3c36 build/default/production/_ext/427700826/arp.o
 .debug_info    0x0002ca29     0x138b build/default/production/_ext/427700826/berkeley_api.o
 .debug_info    0x0002ddb4     0x3819 build/default/production/_ext/427700826/dhcp.o
 .debug_info    0x000315cd     0x1459 build/default/production/_ext/427700826/dhcps.o
 .debug_info    0x00032a26     0x28fe build/default/production/_ext/427700826/dns.o
 .debug_info    0x00035324     0x1383 build/default/production/_ext/427700826/dnss.o
 .debug_info    0x000366a7     0x1386 build/default/production/_ext/427700826/dyn_dns.o
 .debug_info    0x00037a2d     0x1388 build/default/production/_ext/427700826/enc28_mac.o
 .debug_info    0x00038db5     0x1387 build/default/production/_ext/427700826/enc28j60.o
 .debug_info    0x0003a13c     0x3dc9 build/default/production/_ext/427700826/encs24j600.o
 .debug_info    0x0003df05     0x2ad5 build/default/production/_ext/427700826/encx24_mac.o
 .debug_info    0x000409da     0x1390 build/default/production/_ext/427700826/eth_pic32_ext_phy.o
 .debug_info    0x00041d6a     0x1398 build/default/production/_ext/427700826/eth_pic32_ext_phy_dp83848.o
 .debug_info    0x00043102     0x1390 build/default/production/_ext/427700826/eth_pic32_int_mac.o
 .debug_info    0x00044492     0x1382 build/default/production/_ext/427700826/ftp.o
 .debug_info    0x00045814      0x277 build/default/production/_ext/427700826/hash_fnv.o
 .debug_info    0x00045a8b      0x795 build/default/production/_ext/427700826/hash_tbl.o
 .debug_info    0x00046220     0x26c6 build/default/production/_ext/427700826/icmp.o
 .debug_info    0x000488e6     0x1385 build/default/production/_ext/427700826/icmpv6.o
 .debug_info    0x00049c6b     0x3b8b build/default/production/_ext/427700826/ipv4.o
 .debug_info    0x0004d7f6     0x1383 build/default/production/_ext/427700826/ipv6.o
 .debug_info    0x0004eb79     0x138f build/default/production/_ext/427700826/mac_events_pic32.o
 .debug_info    0x0004ff08     0x26f4 build/default/production/_ext/427700826/nbns.o
 .debug_info    0x000525fc     0x1382 build/default/production/_ext/427700826/ndp.o
 .debug_info    0x0005397e     0x138b build/default/production/_ext/427700826/tcpip_reboot.o
 .debug_info    0x00054d09     0x1382 build/default/production/_ext/427700826/rsa.o
 .debug_info    0x0005608b     0x1383 build/default/production/_ext/427700826/smtp.o
 .debug_info    0x0005740e     0x1383 build/default/production/_ext/427700826/snmp.o
 .debug_info    0x00058791     0x1385 build/default/production/_ext/427700826/snmpv3.o
 .debug_info    0x00059b16     0x1389 build/default/production/_ext/427700826/snmpv3_usm.o
 .debug_info    0x0005ae9f     0x1383 build/default/production/_ext/427700826/sntp.o
 .debug_info    0x0005c222     0x1382 build/default/production/_ext/427700826/ssl.o
 .debug_info    0x0005d5a4     0x5802 build/default/production/_ext/427700826/tcp.o
 .debug_info    0x00062da6     0x1eeb build/default/production/_ext/427700826/tcpip_heap_alloc.o
 .debug_info    0x00064c91     0x138c build/default/production/_ext/427700826/tcpip_storage.o
 .debug_info    0x0006601d     0x1385 build/default/production/_ext/427700826/telnet.o
 .debug_info    0x000673a2     0x1384 build/default/production/_ext/427700826/tftpc.o
 .debug_info    0x00068726     0x419e build/default/production/_ext/427700826/udp.o
 .debug_info    0x0006c8c4     0x1d03 build/default/production/_ext/427700826/tcpip_mac_object.o
 .debug_info    0x0006e5c7     0x4ced build/default/production/_ext/427700826/tcpip_manager.o
 .debug_info    0x000732b4     0x2655 build/default/production/_ext/427700826/tcpip_helpers.o
 .debug_info    0x00075909     0x138d build/default/production/_ext/427700826/tcpip_commands.o
 .debug_info    0x00076c96     0x1384 build/default/production/_ext/427700826/iperf.o
 .debug_info    0x0007801a       0xb2 build/default/production/_ext/427700826/tcpip_helper_c32.o
 .debug_info    0x000780cc      0x38a build/default/production/_ext/427700826/tcpip_notify.o
 .debug_info    0x00078456     0x138f build/default/production/_ext/427700826/zero_conf_helper.o
 .debug_info    0x000797e5     0x1450 build/default/production/_ext/427700826/zero_conf_link_local.o
 .debug_info    0x0007ac35     0x1396 build/default/production/_ext/427700826/zero_conf_multicast_dns.o
 .debug_info    0x0007bfcb     0x138f build/default/production/_ext/334706090/wf_tx_power.o
 .debug_info    0x0007d35a     0x138e build/default/production/_ext/334706090/wf_connect.o
 .debug_info    0x0007e6e8     0x139b build/default/production/_ext/334706090/wf_connection_algorithm.o
 .debug_info    0x0007fa83     0x1399 build/default/production/_ext/334706090/wf_connection_manager.o
 .debug_info    0x00080e1c     0x1399 build/default/production/_ext/334706090/wf_connection_profile.o
 .debug_info    0x000821b5     0x1392 build/default/production/_ext/334706090/wf_easy_config.o
 .debug_info    0x00083547     0x13b3 build/default/production/_ext/334706090/wf_eint.o
 .debug_info    0x000848fa     0x1394 build/default/production/_ext/334706090/wf_event_handler.o
 .debug_info    0x00085c8e     0x138b build/default/production/_ext/334706090/wf_init.o
 .debug_info    0x00087019     0x1391 build/default/production/_ext/334706090/wf_power_save.o
 .debug_info    0x000883aa     0x138b build/default/production/_ext/334706090/wf_scan.o
 .debug_info    0x00089735     0x13b1 build/default/production/_ext/334706090/wf_spi.o
 .debug_info    0x0008aae6     0x1394 build/default/production/_ext/334706090/mrf24w_mac_pic32.o
 .debug_info    0x0008be7a     0x1391 build/default/production/_ext/334706090/mrf24w_events.o
 .debug_info    0x0008d20b     0x1395 build/default/production/_ext/334706090/wf_driver_com_24g.o
 .debug_info    0x0008e5a0     0x1395 build/default/production/_ext/334706090/wf_driver_raw_24g.o
 .debug_info    0x0008f935     0x138e build/default/production/_ext/334706090/wf_mac_24g.o
 .debug_info    0x00090cc3     0x1393 build/default/production/_ext/334706090/wf_mgmt_msg_24g.o
 .debug_info    0x00092056     0x1394 build/default/production/_ext/334706090/wf_param_msg_24g.o
 .debug_info    0x000933ea     0x22e1 build/default/production/_ext/1472/main_demo.o
 .debug_info    0x000956cb        0x0 build/default/production/_ext/1472/custom_snmp_app.o
 .debug_info    0x000956cb        0x0 build/default/production/_ext/1472/custom_ssl_cert.o
 .debug_info    0x000956cb     0x1168 build/default/production/_ext/1472/mpfs_img2.o
 .debug_info    0x00096833     0x1168 build/default/production/_ext/1472/wf_config.o
 .debug_info    0x0009799b     0x280d build/default/production/_ext/1472/custom_http_app.o
 .debug_info    0x0009a1a8     0x24b2 build/default/production/_ext/1472/tcp6_demo_app.o
 .debug_info    0x0009c65a       0xaa c:/program files (x86)/microchip/xc32/v1.21/bin/../lib/gcc/pic32mx/4.5.2/../../../../pic32mx/lib/size\libmchp_peripheral.a(open_core_timer_lib.o)
 .debug_info    0x0009c704       0xb2 c:/program files (x86)/microchip/xc32/v1.21/bin/../lib/gcc/pic32mx/4.5.2/../../../../pic32mx/lib/size\libmchp_peripheral_32MX795F512L.a(soft_reset_lib.o)
 .debug_info    0x0009c7b6       0xbf c:/program files (x86)/microchip/xc32/v1.21/bin/../lib/gcc/pic32mx/4.5.2/../../../../pic32mx/lib/size\libmchp_peripheral_32MX795F512L.a(pcache.o)
 .debug_info    0x0009c875       0xb6 c:/program files (x86)/microchip/xc32/v1.21/bin/../lib/gcc/pic32mx/4.5.2/../../../../pic32mx/lib/size\libmchp_peripheral_32MX795F512L.a(int_disable_interrupts_lib.o)
 .debug_info    0x0009c92b       0xb6 c:/program files (x86)/microchip/xc32/v1.21/bin/../lib/gcc/pic32mx/4.5.2/../../../../pic32mx/lib/size\libmchp_peripheral_32MX795F512L.a(int_restore_interrupts_lib.o)
 .debug_info    0x0009c9e1       0xbc c:/program files (x86)/microchip/xc32/v1.21/bin/../lib/gcc/pic32mx/4.5.2/../../../../pic32mx/lib/size\libmchp_peripheral_32MX795F512L.a(int_enable_mv_int_lib.o)
 .debug_info    0x0009ca9d      0x196 c:/program files (x86)/microchip/xc32/v1.21/bin/../lib/gcc/pic32mx/4.5.2/../../../../pic32mx/lib/size\libmchp_peripheral_32MX795F512L.a(int_tbl_lib.o)
 .debug_info    0x0009cc33      0x10c c:/program files (x86)/microchip/xc32/v1.21/bin/../lib/gcc/pic32mx/4.5.2/../../../../pic32mx/lib/size\libmchp_peripheral_32MX795F512L.a(rtcc_init_lib.o)
 .debug_info    0x0009cd3f      0x10c c:/program files (x86)/microchip/xc32/v1.21/bin/../lib/gcc/pic32mx/4.5.2/../../../../pic32mx/lib/size\libmchp_peripheral_32MX795F512L.a(rtcc_open_lib.o)
 .debug_info    0x0009ce4b       0xbc c:/program files (x86)/microchip/xc32/v1.21/bin/../lib/gcc/pic32mx/4.5.2/../../../../pic32mx/lib/size\libmchp_peripheral_32MX795F512L.a(spi_chn_data_rdy_lib.o)
 .debug_info    0x0009cf07       0xcf c:/program files (x86)/microchip/xc32/v1.21/bin/../lib/gcc/pic32mx/4.5.2/../../../../pic32mx/lib/size\libmchp_peripheral_32MX795F512L.a(spi_chn_getc_lib.o)
 .debug_info    0x0009cfd6       0xa2 c:/program files (x86)/microchip/xc32/v1.21/bin/../lib/gcc/pic32mx/4.5.2/../../../../pic32mx/lib/size\libmchp_peripheral_32MX795F512L.a(spi_chn_open_lib.o)
 .debug_info    0x0009d078       0xeb c:/program files (x86)/microchip/xc32/v1.21/bin/../lib/gcc/pic32mx/4.5.2/../../../../pic32mx/lib/size\libmchp_peripheral_32MX795F512L.a(spi_chn_putc_lib.o)
 .debug_info    0x0009d163       0xb2 c:/program files (x86)/microchip/xc32/v1.21/bin/../lib/gcc/pic32mx/4.5.2/../../../../pic32mx/lib/size\libmchp_peripheral_32MX795F512L.a(spi_chn_tx_buff_empty_lib.o)
 .debug_info    0x0009d215        0x0 c:/program files (x86)/microchip/xc32/v1.21/bin/../lib/gcc/pic32mx/4.5.2/../../../../pic32mx/lib/size\libmchp_peripheral_32MX795F512L.a(spi_io_tbl_libp.o)
 .debug_info    0x0009d215        0x0 c:/program files (x86)/microchip/xc32/v1.21/bin/../lib/gcc/pic32mx/4.5.2/../../../../pic32mx/lib/size\libmchp_peripheral_32MX795F512L.a(spi_map_tbl_libp.o)
 .debug_info    0x0009d215       0xba c:/program files (x86)/microchip/xc32/v1.21/bin/../lib/gcc/pic32mx/4.5.2/../../../../pic32mx/lib/size\libmchp_peripheral_32MX795F512L.a(port_set_pins_digital_in_lib.o)
 .debug_info    0x0009d2cf       0xbc c:/program files (x86)/microchip/xc32/v1.21/bin/../lib/gcc/pic32mx/4.5.2/../../../../pic32mx/lib/size\libmchp_peripheral_32MX795F512L.a(port_set_pins_digital_out_lib.o)
 .debug_info    0x0009d38b        0x0 c:/program files (x86)/microchip/xc32/v1.21/bin/../lib/gcc/pic32mx/4.5.2/../../../../pic32mx/lib/size\libmchp_peripheral_32MX795F512L.a(_ports_tbl_libp.o)
 .debug_info    0x0009d38b       0xb4 c:/program files (x86)/microchip/xc32/v1.21/bin/../lib/gcc/pic32mx/4.5.2/../../../../pic32mx/lib/size\libmchp_peripheral_32MX795F512L.a(int_enable_interrupts_lib.o)
 .debug_info    0x0009d43f       0xe7 c:/program files (x86)/microchip/xc32/v1.21/bin/../lib/gcc/pic32mx/4.5.2/../../../../pic32mx/lib/size\libmchp_peripheral_32MX795F512L.a(_rtcc_wait_clock_off_lib.o)
 .debug_info    0x0009d526       0xaa c:/program files (x86)/microchip/xc32/v1.21/bin/../lib/gcc/pic32mx/4.5.2/../../../../pic32mx/lib/size\libmchp_peripheral_32MX795F512L.a(read_core_timer_lib.o)
 .debug_info    0x0009d5d0      0x760 c:/program files (x86)/microchip/xc32/v1.21/bin/../lib/gcc/pic32mx/4.5.2/size\libgcc.a(_udivdi3.o)
 .debug_info    0x0009dd30       0xe8 c:/program files (x86)/microchip/xc32/v1.21/bin/../lib/gcc/pic32mx/4.5.2/../../../../pic32mx/lib/size\libpic32.a(default-bootstrap-exception-handler.o)
 .debug_info    0x0009de18       0xc2 c:/program files (x86)/microchip/xc32/v1.21/bin/../lib/gcc/pic32mx/4.5.2/../../../../pic32mx/lib/size\libpic32.a(default-on-reset.o)
 .debug_info    0x0009deda       0xca c:/program files (x86)/microchip/xc32/v1.21/bin/../lib/gcc/pic32mx/4.5.2/../../../../pic32mx/lib/size\libpic32.a(default-on-bootstrap.o)
 .debug_info    0x0009dfa4        0x0 c:/program files (x86)/microchip/xc32/v1.21/bin/../lib/gcc/pic32mx/4.5.2/../../../../pic32mx/lib/size\libpic32.a(errno.o)
 .debug_info    0x0009dfa4       0xdc c:/program files (x86)/microchip/xc32/v1.21/bin/../lib/gcc/pic32mx/4.5.2/../../../../pic32mx/lib/size\libpic32.a(defaultinterrupt.o)
 .debug_info    0x0009e080       0xb3 c:/program files (x86)/microchip/xc32/v1.21/bin/../lib/gcc/pic32mx/4.5.2/../../../../pic32mx/lib/size\libc.a(atoi.o)
 .debug_info    0x0009e133       0xb3 c:/program files (x86)/microchip/xc32/v1.21/bin/../lib/gcc/pic32mx/4.5.2/../../../../pic32mx/lib/size\libc.a(atol.o)
 .debug_info    0x0009e1e6        0x0 c:/program files (x86)/microchip/xc32/v1.21/bin/../lib/gcc/pic32mx/4.5.2/../../../../pic32mx/lib/size\libc.a(ctype.o)
 .debug_info    0x0009e1e6       0xe0 c:/program files (x86)/microchip/xc32/v1.21/bin/../lib/gcc/pic32mx/4.5.2/../../../../pic32mx/lib/size\libc.a(malloc.o)
 .debug_info    0x0009e2c6       0xc7 c:/program files (x86)/microchip/xc32/v1.21/bin/../lib/gcc/pic32mx/4.5.2/../../../../pic32mx/lib/size\libc.a(rand.o)
 .debug_info    0x0009e38d       0xb7 c:/program files (x86)/microchip/xc32/v1.21/bin/../lib/gcc/pic32mx/4.5.2/../../../../pic32mx/lib/size\libc.a(strcat.o)
 .debug_info    0x0009e444       0xb7 c:/program files (x86)/microchip/xc32/v1.21/bin/../lib/gcc/pic32mx/4.5.2/../../../../pic32mx/lib/size\libc.a(strchr.o)
 .debug_info    0x0009e4fb       0xb9 c:/program files (x86)/microchip/xc32/v1.21/bin/../lib/gcc/pic32mx/4.5.2/../../../../pic32mx/lib/size\libc.a(strncat.o)
 .debug_info    0x0009e5b4       0xb9 c:/program files (x86)/microchip/xc32/v1.21/bin/../lib/gcc/pic32mx/4.5.2/../../../../pic32mx/lib/size\libc.a(strncmp.o)
 .debug_info    0x0009e66d       0xb9 c:/program files (x86)/microchip/xc32/v1.21/bin/../lib/gcc/pic32mx/4.5.2/../../../../pic32mx/lib/size\libc.a(strncpy.o)
 .debug_info    0x0009e726       0xb9 c:/program files (x86)/microchip/xc32/v1.21/bin/../lib/gcc/pic32mx/4.5.2/../../../../pic32mx/lib/size\libc.a(strrchr.o)
 .debug_info    0x0009e7df       0xb7 c:/program files (x86)/microchip/xc32/v1.21/bin/../lib/gcc/pic32mx/4.5.2/../../../../pic32mx/lib/size\libc.a(strstr.o)
 .debug_info    0x0009e896       0xcd c:/program files (x86)/microchip/xc32/v1.21/bin/../lib/gcc/pic32mx/4.5.2/../../../../pic32mx/lib/size\libc.a(strtol.o)
 .debug_info    0x0009e963       0xc6 c:/program files (x86)/microchip/xc32/v1.21/bin/../lib/gcc/pic32mx/4.5.2/../../../../pic32mx/lib/size\libc.a(snprintf_cdnopsuxX.eo)
 .debug_info    0x0009ea29       0xc4 c:/program files (x86)/microchip/xc32/v1.21/bin/../lib/gcc/pic32mx/4.5.2/../../../../pic32mx/lib/size\libc.a(sprintf_cdnopsuxX.eo)
 .debug_info    0x0009eaed       0xc8 c:/program files (x86)/microchip/xc32/v1.21/bin/../lib/gcc/pic32mx/4.5.2/../../../../pic32mx/lib/size\libc.a(vsnprintf_cdnopsuxX.eo)
 .debug_info    0x0009ebb5       0xbd c:/program files (x86)/microchip/xc32/v1.21/bin/../lib/gcc/pic32mx/4.5.2/../../../../pic32mx/lib/size\libc.a(vsnprintf.o)
 .debug_info    0x0009ec72      0x21b c:/program files (x86)/microchip/xc32/v1.21/bin/../lib/gcc/pic32mx/4.5.2/../../../../pic32mx/lib/size\libc.a(ctypef.o)
 .debug_info    0x0009ee8d       0xc5 c:/program files (x86)/microchip/xc32/v1.21/bin/../lib/gcc/pic32mx/4.5.2/../../../../pic32mx/lib/size\libc.a(doprnt_cdnopsuxX.eo)
 .debug_info    0x0009ef52       0xe3 c:/program files (x86)/microchip/xc32/v1.21/bin/../lib/gcc/pic32mx/4.5.2/../../../../pic32mx/lib/size\libc.a(doprnt.o)
 .debug_info    0x0009f035       0xb5 c:/program files (x86)/microchip/xc32/v1.21/bin/../lib/gcc/pic32mx/4.5.2/../../../../pic32mx/lib/size\libc.a(_fputc_simple.o)
 .debug_info    0x0009f0ea        0x0 c:/program files (x86)/microchip/xc32/v1.21/bin/../lib/gcc/pic32mx/4.5.2/../../../../pic32mx/lib/size\libc.a(powersf.o)
 .debug_info    0x0009f0ea        0x0 c:/program files (x86)/microchip/xc32/v1.21/bin/../lib/gcc/pic32mx/4.5.2/../../../../pic32mx/lib/size\libc.a(_iob.o)
 .debug_info    0x0009f0ea       0xb8 c:/program files (x86)/microchip/xc32/v1.21/bin/../lib/gcc/pic32mx/4.5.2/../../../../pic32mx/lib/size\libc.a(_flsbuf_simple.o)
 .debug_info    0x0009f1a2      0x11b c:/program files (x86)/microchip/xc32/v1.21/bin/../lib/gcc/pic32mx/4.5.2/../../../../pic32mx/lib/size\libpic32.a(sbrk.o)
 .debug_info    0x0009f2bd       0xb3 c:/program files (x86)/microchip/xc32/v1.21/bin/../lib/gcc/pic32mx/4.5.2/../../../../pic32mx/lib/size\libpic32.a(write.o)
 .debug_info    0x0009f370       0xbb c:/program files (x86)/microchip/xc32/v1.21/bin/../lib/gcc/pic32mx/4.5.2/../../../../pic32mx/lib/size\libpic32.a(_mon_putc.o)
 .debug_info    0x0009f42b        0x0 c:/program files (x86)/microchip/xc32/v1.21/bin/../lib/gcc/pic32mx/4.5.2/../../../../pic32mx/lib/size\libpic32.a(xc32_uart.o)
 .debug_info    0x0009f42b       0xd1 c:/program files (x86)/microchip/xc32/v1.21/bin/../lib/gcc/pic32mx/4.5.2/../../../../pic32mx/lib/size\libe.a(_floatdisf.o)
 .debug_info    0x0009f4fc      0x326 c:/program files (x86)/microchip/xc32/v1.21/bin/../lib/gcc/pic32mx/4.5.2/size\libgcc.a(_lshrdi3.o)
 .debug_info    0x0009f822      0x2ad c:/program files (x86)/microchip/xc32/v1.21/bin/../lib/gcc/pic32mx/4.5.2/size\libgcc.a(_floatundisf.o)
 .debug_info    0x0009facf      0x79d c:/program files (x86)/microchip/xc32/v1.21/bin/../lib/gcc/pic32mx/4.5.2/size\libgcc.a(_umoddi3.o)
 .debug_info    0x000a026c      0x165 c:/program files (x86)/microchip/xc32/v1.21/bin/../lib/gcc/pic32mx/4.5.2/size\libgcc.a(floatunsisf.o)

.debug_abbrev   0x00000000     0xc845
 *(.debug_abbrev)
 .debug_abbrev  0x00000000      0x17d build/default/production/_ext/1293749816/bsp.o
 .debug_abbrev  0x0000017d       0x65 build/default/production/_ext/101875047/lfsr.o
 .debug_abbrev  0x000001e2       0x14 build/default/production/_ext/101875047/big_int_helper_c32.o
 .debug_abbrev  0x000001f6      0x218 build/default/production/_ext/101875047/big_int.o
 .debug_abbrev  0x0000040e      0x18e build/default/production/_ext/101875047/hashes.o
 .debug_abbrev  0x0000059c       0xfd build/default/production/_ext/101875047/helpers.o
 .debug_abbrev  0x00000699        0x1 build/default/production/_ext/1472/berkeley_tcp_client_demo.o
 .debug_abbrev  0x0000069a        0x1 build/default/production/_ext/1472/berkeley_tcp_server_demo.o
 .debug_abbrev  0x0000069b        0x1 build/default/production/_ext/1472/berkeley_udp_client_demo.o
 .debug_abbrev  0x0000069c      0x166 build/default/production/_ext/1472/generic_tcp_client.o
 .debug_abbrev  0x00000802      0x166 build/default/production/_ext/1472/generic_tcp_server.o
 .debug_abbrev  0x00000968      0x265 build/default/production/_ext/1472/ping_demo.o
 .debug_abbrev  0x00000bcd        0x1 build/default/production/_ext/1472/smtp_demo.o
 .debug_abbrev  0x00000bce      0x3f7 build/default/production/_ext/365611741/system_services.o
 .debug_abbrev  0x00000fc5      0x2dd build/default/production/_ext/365611741/system_debug.o
 .debug_abbrev  0x000012a2      0x230 build/default/production/_ext/365611741/system_random.o
 .debug_abbrev  0x000014d2      0x2a8 build/default/production/_ext/365611741/system_command.o
 .debug_abbrev  0x0000177a      0x26c build/default/production/_ext/365611741/system_userio.o
 .debug_abbrev  0x000019e6      0x329 build/default/production/_ext/97638081/sys_fs.o
 .debug_abbrev  0x00001d0f      0x27d build/default/production/_ext/97638081/mpfs2.o
 .debug_abbrev  0x00001f8c      0x218 build/default/production/_ext/792872985/usart.o
 .debug_abbrev  0x000021a4      0x201 build/default/production/_ext/792872985/lcd.o
 .debug_abbrev  0x000023a5      0x1e1 build/default/production/_ext/792872985/drv_spi.o
 .debug_abbrev  0x00002586        0x1 build/default/production/_ext/792872985/db_appio.o
 .debug_abbrev  0x00002587      0x166 build/default/production/_ext/792872985/spi_ram.o
 .debug_abbrev  0x000026ed      0x289 build/default/production/_ext/792872985/spi_eeprom.o
 .debug_abbrev  0x00002976      0x166 build/default/production/_ext/792872985/spi_flash.o
 .debug_abbrev  0x00002adc      0x288 build/default/production/_ext/792872985/drv_media.o
 .debug_abbrev  0x00002d64      0x35e build/default/production/_ext/427700826/tcpip_announce.o
 .debug_abbrev  0x000030c2      0x363 build/default/production/_ext/427700826/http2.o
 .debug_abbrev  0x00003425      0x18b build/default/production/_ext/427700826/arcfour.o
 .debug_abbrev  0x000035b0      0x3f8 build/default/production/_ext/427700826/arp.o
 .debug_abbrev  0x000039a8      0x18b build/default/production/_ext/427700826/berkeley_api.o
 .debug_abbrev  0x00003b33      0x3a3 build/default/production/_ext/427700826/dhcp.o
 .debug_abbrev  0x00003ed6      0x1ba build/default/production/_ext/427700826/dhcps.o
 .debug_abbrev  0x00004090      0x365 build/default/production/_ext/427700826/dns.o
 .debug_abbrev  0x000043f5      0x18b build/default/production/_ext/427700826/dnss.o
 .debug_abbrev  0x00004580      0x18b build/default/production/_ext/427700826/dyn_dns.o
 .debug_abbrev  0x0000470b      0x18b build/default/production/_ext/427700826/enc28_mac.o
 .debug_abbrev  0x00004896      0x18b build/default/production/_ext/427700826/enc28j60.o
 .debug_abbrev  0x00004a21      0x31d build/default/production/_ext/427700826/encs24j600.o
 .debug_abbrev  0x00004d3e      0x2d4 build/default/production/_ext/427700826/encx24_mac.o
 .debug_abbrev  0x00005012      0x18b build/default/production/_ext/427700826/eth_pic32_ext_phy.o
 .debug_abbrev  0x0000519d      0x18b build/default/production/_ext/427700826/eth_pic32_ext_phy_dp83848.o
 .debug_abbrev  0x00005328      0x18b build/default/production/_ext/427700826/eth_pic32_int_mac.o
 .debug_abbrev  0x000054b3      0x18b build/default/production/_ext/427700826/ftp.o
 .debug_abbrev  0x0000563e       0x8c build/default/production/_ext/427700826/hash_fnv.o
 .debug_abbrev  0x000056ca      0x1ca build/default/production/_ext/427700826/hash_tbl.o
 .debug_abbrev  0x00005894      0x2ff build/default/production/_ext/427700826/icmp.o
 .debug_abbrev  0x00005b93      0x18b build/default/production/_ext/427700826/icmpv6.o
 .debug_abbrev  0x00005d1e      0x3c7 build/default/production/_ext/427700826/ipv4.o
 .debug_abbrev  0x000060e5      0x18b build/default/production/_ext/427700826/ipv6.o
 .debug_abbrev  0x00006270      0x18b build/default/production/_ext/427700826/mac_events_pic32.o
 .debug_abbrev  0x000063fb      0x2c2 build/default/production/_ext/427700826/nbns.o
 .debug_abbrev  0x000066bd      0x18b build/default/production/_ext/427700826/ndp.o
 .debug_abbrev  0x00006848      0x18b build/default/production/_ext/427700826/tcpip_reboot.o
 .debug_abbrev  0x000069d3      0x18b build/default/production/_ext/427700826/rsa.o
 .debug_abbrev  0x00006b5e      0x18b build/default/production/_ext/427700826/smtp.o
 .debug_abbrev  0x00006ce9      0x18b build/default/production/_ext/427700826/snmp.o
 .debug_abbrev  0x00006e74      0x18b build/default/production/_ext/427700826/snmpv3.o
 .debug_abbrev  0x00006fff      0x18b build/default/production/_ext/427700826/snmpv3_usm.o
 .debug_abbrev  0x0000718a      0x18b build/default/production/_ext/427700826/sntp.o
 .debug_abbrev  0x00007315      0x18b build/default/production/_ext/427700826/ssl.o
 .debug_abbrev  0x000074a0      0x39d build/default/production/_ext/427700826/tcp.o
 .debug_abbrev  0x0000783d      0x295 build/default/production/_ext/427700826/tcpip_heap_alloc.o
 .debug_abbrev  0x00007ad2      0x18b build/default/production/_ext/427700826/tcpip_storage.o
 .debug_abbrev  0x00007c5d      0x18b build/default/production/_ext/427700826/telnet.o
 .debug_abbrev  0x00007de8      0x18b build/default/production/_ext/427700826/tftpc.o
 .debug_abbrev  0x00007f73      0x3ad build/default/production/_ext/427700826/udp.o
 .debug_abbrev  0x00008320      0x22e build/default/production/_ext/427700826/tcpip_mac_object.o
 .debug_abbrev  0x0000854e      0x3d7 build/default/production/_ext/427700826/tcpip_manager.o
 .debug_abbrev  0x00008925      0x28d build/default/production/_ext/427700826/tcpip_helpers.o
 .debug_abbrev  0x00008bb2      0x18b build/default/production/_ext/427700826/tcpip_commands.o
 .debug_abbrev  0x00008d3d      0x18b build/default/production/_ext/427700826/iperf.o
 .debug_abbrev  0x00008ec8       0x14 build/default/production/_ext/427700826/tcpip_helper_c32.o
 .debug_abbrev  0x00008edc       0xd9 build/default/production/_ext/427700826/tcpip_notify.o
 .debug_abbrev  0x00008fb5      0x18b build/default/production/_ext/427700826/zero_conf_helper.o
 .debug_abbrev  0x00009140      0x1ba build/default/production/_ext/427700826/zero_conf_link_local.o
 .debug_abbrev  0x000092fa      0x18b build/default/production/_ext/427700826/zero_conf_multicast_dns.o
 .debug_abbrev  0x00009485      0x18b build/default/production/_ext/334706090/wf_tx_power.o
 .debug_abbrev  0x00009610      0x18b build/default/production/_ext/334706090/wf_connect.o
 .debug_abbrev  0x0000979b      0x18b build/default/production/_ext/334706090/wf_connection_algorithm.o
 .debug_abbrev  0x00009926      0x18b build/default/production/_ext/334706090/wf_connection_manager.o
 .debug_abbrev  0x00009ab1      0x18b build/default/production/_ext/334706090/wf_connection_profile.o
 .debug_abbrev  0x00009c3c      0x18b build/default/production/_ext/334706090/wf_easy_config.o
 .debug_abbrev  0x00009dc7      0x1a2 build/default/production/_ext/334706090/wf_eint.o
 .debug_abbrev  0x00009f69      0x18b build/default/production/_ext/334706090/wf_event_handler.o
 .debug_abbrev  0x0000a0f4      0x18b build/default/production/_ext/334706090/wf_init.o
 .debug_abbrev  0x0000a27f      0x18b build/default/production/_ext/334706090/wf_power_save.o
 .debug_abbrev  0x0000a40a      0x18b build/default/production/_ext/334706090/wf_scan.o
 .debug_abbrev  0x0000a595      0x1a2 build/default/production/_ext/334706090/wf_spi.o
 .debug_abbrev  0x0000a737      0x18b build/default/production/_ext/334706090/mrf24w_mac_pic32.o
 .debug_abbrev  0x0000a8c2      0x18b build/default/production/_ext/334706090/mrf24w_events.o
 .debug_abbrev  0x0000aa4d      0x18b build/default/production/_ext/334706090/wf_driver_com_24g.o
 .debug_abbrev  0x0000abd8      0x18b build/default/production/_ext/334706090/wf_driver_raw_24g.o
 .debug_abbrev  0x0000ad63      0x18b build/default/production/_ext/334706090/wf_mac_24g.o
 .debug_abbrev  0x0000aeee      0x18b build/default/production/_ext/334706090/wf_mgmt_msg_24g.o
 .debug_abbrev  0x0000b079      0x18b build/default/production/_ext/334706090/wf_param_msg_24g.o
 .debug_abbrev  0x0000b204      0x263 build/default/production/_ext/1472/main_demo.o
 .debug_abbrev  0x0000b467        0x1 build/default/production/_ext/1472/custom_snmp_app.o
 .debug_abbrev  0x0000b468        0x1 build/default/production/_ext/1472/custom_ssl_cert.o
 .debug_abbrev  0x0000b469      0x166 build/default/production/_ext/1472/mpfs_img2.o
 .debug_abbrev  0x0000b5cf      0x166 build/default/production/_ext/1472/wf_config.o
 .debug_abbrev  0x0000b735      0x28b build/default/production/_ext/1472/custom_http_app.o
 .debug_abbrev  0x0000b9c0      0x283 build/default/production/_ext/1472/tcp6_demo_app.o
 .debug_abbrev  0x0000bc43       0x25 c:/program files (x86)/microchip/xc32/v1.21/bin/../lib/gcc/pic32mx/4.5.2/../../../../pic32mx/lib/size\libmchp_peripheral.a(open_core_timer_lib.o)
 .debug_abbrev  0x0000bc68       0x34 c:/program files (x86)/microchip/xc32/v1.21/bin/../lib/gcc/pic32mx/4.5.2/../../../../pic32mx/lib/size\libmchp_peripheral_32MX795F512L.a(soft_reset_lib.o)
 .debug_abbrev  0x0000bc9c       0x25 c:/program files (x86)/microchip/xc32/v1.21/bin/../lib/gcc/pic32mx/4.5.2/../../../../pic32mx/lib/size\libmchp_peripheral_32MX795F512L.a(pcache.o)
 .debug_abbrev  0x0000bcc1       0x25 c:/program files (x86)/microchip/xc32/v1.21/bin/../lib/gcc/pic32mx/4.5.2/../../../../pic32mx/lib/size\libmchp_peripheral_32MX795F512L.a(int_disable_interrupts_lib.o)
 .debug_abbrev  0x0000bce6       0x25 c:/program files (x86)/microchip/xc32/v1.21/bin/../lib/gcc/pic32mx/4.5.2/../../../../pic32mx/lib/size\libmchp_peripheral_32MX795F512L.a(int_restore_interrupts_lib.o)
 .debug_abbrev  0x0000bd0b       0x25 c:/program files (x86)/microchip/xc32/v1.21/bin/../lib/gcc/pic32mx/4.5.2/../../../../pic32mx/lib/size\libmchp_peripheral_32MX795F512L.a(int_enable_mv_int_lib.o)
 .debug_abbrev  0x0000bd30       0x25 c:/program files (x86)/microchip/xc32/v1.21/bin/../lib/gcc/pic32mx/4.5.2/../../../../pic32mx/lib/size\libmchp_peripheral_32MX795F512L.a(int_tbl_lib.o)
 .debug_abbrev  0x0000bd55       0x41 c:/program files (x86)/microchip/xc32/v1.21/bin/../lib/gcc/pic32mx/4.5.2/../../../../pic32mx/lib/size\libmchp_peripheral_32MX795F512L.a(rtcc_init_lib.o)
 .debug_abbrev  0x0000bd96       0x41 c:/program files (x86)/microchip/xc32/v1.21/bin/../lib/gcc/pic32mx/4.5.2/../../../../pic32mx/lib/size\libmchp_peripheral_32MX795F512L.a(rtcc_open_lib.o)
 .debug_abbrev  0x0000bdd7       0x34 c:/program files (x86)/microchip/xc32/v1.21/bin/../lib/gcc/pic32mx/4.5.2/../../../../pic32mx/lib/size\libmchp_peripheral_32MX795F512L.a(spi_chn_data_rdy_lib.o)
 .debug_abbrev  0x0000be0b       0x34 c:/program files (x86)/microchip/xc32/v1.21/bin/../lib/gcc/pic32mx/4.5.2/../../../../pic32mx/lib/size\libmchp_peripheral_32MX795F512L.a(spi_chn_getc_lib.o)
 .debug_abbrev  0x0000be3f       0x25 c:/program files (x86)/microchip/xc32/v1.21/bin/../lib/gcc/pic32mx/4.5.2/../../../../pic32mx/lib/size\libmchp_peripheral_32MX795F512L.a(spi_chn_open_lib.o)
 .debug_abbrev  0x0000be64       0x34 c:/program files (x86)/microchip/xc32/v1.21/bin/../lib/gcc/pic32mx/4.5.2/../../../../pic32mx/lib/size\libmchp_peripheral_32MX795F512L.a(spi_chn_putc_lib.o)
 .debug_abbrev  0x0000be98       0x25 c:/program files (x86)/microchip/xc32/v1.21/bin/../lib/gcc/pic32mx/4.5.2/../../../../pic32mx/lib/size\libmchp_peripheral_32MX795F512L.a(spi_chn_tx_buff_empty_lib.o)
 .debug_abbrev  0x0000bebd        0x1 c:/program files (x86)/microchip/xc32/v1.21/bin/../lib/gcc/pic32mx/4.5.2/../../../../pic32mx/lib/size\libmchp_peripheral_32MX795F512L.a(spi_io_tbl_libp.o)
 .debug_abbrev  0x0000bebe        0x1 c:/program files (x86)/microchip/xc32/v1.21/bin/../lib/gcc/pic32mx/4.5.2/../../../../pic32mx/lib/size\libmchp_peripheral_32MX795F512L.a(spi_map_tbl_libp.o)
 .debug_abbrev  0x0000bebf       0x25 c:/program files (x86)/microchip/xc32/v1.21/bin/../lib/gcc/pic32mx/4.5.2/../../../../pic32mx/lib/size\libmchp_peripheral_32MX795F512L.a(port_set_pins_digital_in_lib.o)
 .debug_abbrev  0x0000bee4       0x25 c:/program files (x86)/microchip/xc32/v1.21/bin/../lib/gcc/pic32mx/4.5.2/../../../../pic32mx/lib/size\libmchp_peripheral_32MX795F512L.a(port_set_pins_digital_out_lib.o)
 .debug_abbrev  0x0000bf09        0x1 c:/program files (x86)/microchip/xc32/v1.21/bin/../lib/gcc/pic32mx/4.5.2/../../../../pic32mx/lib/size\libmchp_peripheral_32MX795F512L.a(_ports_tbl_libp.o)
 .debug_abbrev  0x0000bf0a       0x25 c:/program files (x86)/microchip/xc32/v1.21/bin/../lib/gcc/pic32mx/4.5.2/../../../../pic32mx/lib/size\libmchp_peripheral_32MX795F512L.a(int_enable_interrupts_lib.o)
 .debug_abbrev  0x0000bf2f       0x34 c:/program files (x86)/microchip/xc32/v1.21/bin/../lib/gcc/pic32mx/4.5.2/../../../../pic32mx/lib/size\libmchp_peripheral_32MX795F512L.a(_rtcc_wait_clock_off_lib.o)
 .debug_abbrev  0x0000bf63       0x25 c:/program files (x86)/microchip/xc32/v1.21/bin/../lib/gcc/pic32mx/4.5.2/../../../../pic32mx/lib/size\libmchp_peripheral_32MX795F512L.a(read_core_timer_lib.o)
 .debug_abbrev  0x0000bf88      0x13d c:/program files (x86)/microchip/xc32/v1.21/bin/../lib/gcc/pic32mx/4.5.2/size\libgcc.a(_udivdi3.o)
 .debug_abbrev  0x0000c0c5       0x25 c:/program files (x86)/microchip/xc32/v1.21/bin/../lib/gcc/pic32mx/4.5.2/../../../../pic32mx/lib/size\libpic32.a(default-bootstrap-exception-handler.o)
 .debug_abbrev  0x0000c0ea       0x25 c:/program files (x86)/microchip/xc32/v1.21/bin/../lib/gcc/pic32mx/4.5.2/../../../../pic32mx/lib/size\libpic32.a(default-on-reset.o)
 .debug_abbrev  0x0000c10f       0x25 c:/program files (x86)/microchip/xc32/v1.21/bin/../lib/gcc/pic32mx/4.5.2/../../../../pic32mx/lib/size\libpic32.a(default-on-bootstrap.o)
 .debug_abbrev  0x0000c134        0x1 c:/program files (x86)/microchip/xc32/v1.21/bin/../lib/gcc/pic32mx/4.5.2/../../../../pic32mx/lib/size\libpic32.a(errno.o)
 .debug_abbrev  0x0000c135       0x25 c:/program files (x86)/microchip/xc32/v1.21/bin/../lib/gcc/pic32mx/4.5.2/../../../../pic32mx/lib/size\libpic32.a(defaultinterrupt.o)
 .debug_abbrev  0x0000c15a       0x25 c:/program files (x86)/microchip/xc32/v1.21/bin/../lib/gcc/pic32mx/4.5.2/../../../../pic32mx/lib/size\libc.a(atoi.o)
 .debug_abbrev  0x0000c17f       0x25 c:/program files (x86)/microchip/xc32/v1.21/bin/../lib/gcc/pic32mx/4.5.2/../../../../pic32mx/lib/size\libc.a(atol.o)
 .debug_abbrev  0x0000c1a4        0x1 c:/program files (x86)/microchip/xc32/v1.21/bin/../lib/gcc/pic32mx/4.5.2/../../../../pic32mx/lib/size\libc.a(ctype.o)
 .debug_abbrev  0x0000c1a5       0x25 c:/program files (x86)/microchip/xc32/v1.21/bin/../lib/gcc/pic32mx/4.5.2/../../../../pic32mx/lib/size\libc.a(malloc.o)
 .debug_abbrev  0x0000c1ca       0x25 c:/program files (x86)/microchip/xc32/v1.21/bin/../lib/gcc/pic32mx/4.5.2/../../../../pic32mx/lib/size\libc.a(rand.o)
 .debug_abbrev  0x0000c1ef       0x25 c:/program files (x86)/microchip/xc32/v1.21/bin/../lib/gcc/pic32mx/4.5.2/../../../../pic32mx/lib/size\libc.a(strcat.o)
 .debug_abbrev  0x0000c214       0x25 c:/program files (x86)/microchip/xc32/v1.21/bin/../lib/gcc/pic32mx/4.5.2/../../../../pic32mx/lib/size\libc.a(strchr.o)
 .debug_abbrev  0x0000c239       0x25 c:/program files (x86)/microchip/xc32/v1.21/bin/../lib/gcc/pic32mx/4.5.2/../../../../pic32mx/lib/size\libc.a(strncat.o)
 .debug_abbrev  0x0000c25e       0x25 c:/program files (x86)/microchip/xc32/v1.21/bin/../lib/gcc/pic32mx/4.5.2/../../../../pic32mx/lib/size\libc.a(strncmp.o)
 .debug_abbrev  0x0000c283       0x25 c:/program files (x86)/microchip/xc32/v1.21/bin/../lib/gcc/pic32mx/4.5.2/../../../../pic32mx/lib/size\libc.a(strncpy.o)
 .debug_abbrev  0x0000c2a8       0x25 c:/program files (x86)/microchip/xc32/v1.21/bin/../lib/gcc/pic32mx/4.5.2/../../../../pic32mx/lib/size\libc.a(strrchr.o)
 .debug_abbrev  0x0000c2cd       0x25 c:/program files (x86)/microchip/xc32/v1.21/bin/../lib/gcc/pic32mx/4.5.2/../../../../pic32mx/lib/size\libc.a(strstr.o)
 .debug_abbrev  0x0000c2f2       0x25 c:/program files (x86)/microchip/xc32/v1.21/bin/../lib/gcc/pic32mx/4.5.2/../../../../pic32mx/lib/size\libc.a(strtol.o)
 .debug_abbrev  0x0000c317       0x25 c:/program files (x86)/microchip/xc32/v1.21/bin/../lib/gcc/pic32mx/4.5.2/../../../../pic32mx/lib/size\libc.a(snprintf_cdnopsuxX.eo)
 .debug_abbrev  0x0000c33c       0x25 c:/program files (x86)/microchip/xc32/v1.21/bin/../lib/gcc/pic32mx/4.5.2/../../../../pic32mx/lib/size\libc.a(sprintf_cdnopsuxX.eo)
 .debug_abbrev  0x0000c361       0x25 c:/program files (x86)/microchip/xc32/v1.21/bin/../lib/gcc/pic32mx/4.5.2/../../../../pic32mx/lib/size\libc.a(vsnprintf_cdnopsuxX.eo)
 .debug_abbrev  0x0000c386       0x25 c:/program files (x86)/microchip/xc32/v1.21/bin/../lib/gcc/pic32mx/4.5.2/../../../../pic32mx/lib/size\libc.a(vsnprintf.o)
 .debug_abbrev  0x0000c3ab       0x25 c:/program files (x86)/microchip/xc32/v1.21/bin/../lib/gcc/pic32mx/4.5.2/../../../../pic32mx/lib/size\libc.a(ctypef.o)
 .debug_abbrev  0x0000c3d0       0x25 c:/program files (x86)/microchip/xc32/v1.21/bin/../lib/gcc/pic32mx/4.5.2/../../../../pic32mx/lib/size\libc.a(doprnt_cdnopsuxX.eo)
 .debug_abbrev  0x0000c3f5       0x36 c:/program files (x86)/microchip/xc32/v1.21/bin/../lib/gcc/pic32mx/4.5.2/../../../../pic32mx/lib/size\libc.a(doprnt.o)
 .debug_abbrev  0x0000c42b       0x25 c:/program files (x86)/microchip/xc32/v1.21/bin/../lib/gcc/pic32mx/4.5.2/../../../../pic32mx/lib/size\libc.a(_fputc_simple.o)
 .debug_abbrev  0x0000c450        0x1 c:/program files (x86)/microchip/xc32/v1.21/bin/../lib/gcc/pic32mx/4.5.2/../../../../pic32mx/lib/size\libc.a(powersf.o)
 .debug_abbrev  0x0000c451        0x1 c:/program files (x86)/microchip/xc32/v1.21/bin/../lib/gcc/pic32mx/4.5.2/../../../../pic32mx/lib/size\libc.a(_iob.o)
 .debug_abbrev  0x0000c452       0x25 c:/program files (x86)/microchip/xc32/v1.21/bin/../lib/gcc/pic32mx/4.5.2/../../../../pic32mx/lib/size\libc.a(_flsbuf_simple.o)
 .debug_abbrev  0x0000c477       0x38 c:/program files (x86)/microchip/xc32/v1.21/bin/../lib/gcc/pic32mx/4.5.2/../../../../pic32mx/lib/size\libpic32.a(sbrk.o)
 .debug_abbrev  0x0000c4af       0x25 c:/program files (x86)/microchip/xc32/v1.21/bin/../lib/gcc/pic32mx/4.5.2/../../../../pic32mx/lib/size\libpic32.a(write.o)
 .debug_abbrev  0x0000c4d4       0x25 c:/program files (x86)/microchip/xc32/v1.21/bin/../lib/gcc/pic32mx/4.5.2/../../../../pic32mx/lib/size\libpic32.a(_mon_putc.o)
 .debug_abbrev  0x0000c4f9        0x1 c:/program files (x86)/microchip/xc32/v1.21/bin/../lib/gcc/pic32mx/4.5.2/../../../../pic32mx/lib/size\libpic32.a(xc32_uart.o)
 .debug_abbrev  0x0000c4fa       0x32 c:/program files (x86)/microchip/xc32/v1.21/bin/../lib/gcc/pic32mx/4.5.2/../../../../pic32mx/lib/size\libe.a(_floatdisf.o)
 .debug_abbrev  0x0000c52c       0xe3 c:/program files (x86)/microchip/xc32/v1.21/bin/../lib/gcc/pic32mx/4.5.2/size\libgcc.a(_lshrdi3.o)
 .debug_abbrev  0x0000c60f       0x79 c:/program files (x86)/microchip/xc32/v1.21/bin/../lib/gcc/pic32mx/4.5.2/size\libgcc.a(_floatundisf.o)
 .debug_abbrev  0x0000c688      0x15c c:/program files (x86)/microchip/xc32/v1.21/bin/../lib/gcc/pic32mx/4.5.2/size\libgcc.a(_umoddi3.o)
 .debug_abbrev  0x0000c7e4       0x61 c:/program files (x86)/microchip/xc32/v1.21/bin/../lib/gcc/pic32mx/4.5.2/size\libgcc.a(floatunsisf.o)

.debug_line     0x00000000    0x179b4
 *(.debug_line)
 .debug_line    0x00000000      0x1de build/default/production/_ext/1293749816/bsp.o
 .debug_line    0x000001de       0xf0 build/default/production/_ext/101875047/lfsr.o
 .debug_line    0x000002ce      0x14f build/default/production/_ext/101875047/big_int_helper_c32.o
 .debug_line    0x0000041d      0x3eb build/default/production/_ext/101875047/big_int.o
 .debug_line    0x00000808      0x2e4 build/default/production/_ext/101875047/hashes.o
 .debug_line    0x00000aec      0x24e build/default/production/_ext/101875047/helpers.o
 .debug_line    0x00000d3a        0x0 build/default/production/_ext/1472/berkeley_tcp_client_demo.o
 .debug_line    0x00000d3a        0x0 build/default/production/_ext/1472/berkeley_tcp_server_demo.o
 .debug_line    0x00000d3a        0x0 build/default/production/_ext/1472/berkeley_udp_client_demo.o
 .debug_line    0x00000d3a      0x1c5 build/default/production/_ext/1472/generic_tcp_client.o
 .debug_line    0x00000eff      0x1c5 build/default/production/_ext/1472/generic_tcp_server.o
 .debug_line    0x000010c4      0x320 build/default/production/_ext/1472/ping_demo.o
 .debug_line    0x000013e4        0x0 build/default/production/_ext/1472/smtp_demo.o
 .debug_line    0x000013e4      0x70a build/default/production/_ext/365611741/system_services.o
 .debug_line    0x00001aee      0x45b build/default/production/_ext/365611741/system_debug.o
 .debug_line    0x00001f49      0x35d build/default/production/_ext/365611741/system_random.o
 .debug_line    0x000022a6      0x4ce build/default/production/_ext/365611741/system_command.o
 .debug_line    0x00002774      0x3be build/default/production/_ext/365611741/system_userio.o
 .debug_line    0x00002b32      0xa8d build/default/production/_ext/97638081/sys_fs.o
 .debug_line    0x000035bf      0x5c9 build/default/production/_ext/97638081/mpfs2.o
 .debug_line    0x00003b88      0x272 build/default/production/_ext/792872985/usart.o
 .debug_line    0x00003dfa      0x367 build/default/production/_ext/792872985/lcd.o
 .debug_line    0x00004161      0x2e9 build/default/production/_ext/792872985/drv_spi.o
 .debug_line    0x0000444a        0x0 build/default/production/_ext/792872985/db_appio.o
 .debug_line    0x0000444a      0x18e build/default/production/_ext/792872985/spi_ram.o
 .debug_line    0x000045d8      0x464 build/default/production/_ext/792872985/spi_eeprom.o
 .debug_line    0x00004a3c      0x18e build/default/production/_ext/792872985/spi_flash.o
 .debug_line    0x00004bca      0x4a8 build/default/production/_ext/792872985/drv_media.o
 .debug_line    0x00005072      0x488 build/default/production/_ext/427700826/tcpip_announce.o
 .debug_line    0x000054fa      0xbbe build/default/production/_ext/427700826/http2.o
 .debug_line    0x000060b8      0x230 build/default/production/_ext/427700826/arcfour.o
 .debug_line    0x000062e8      0x920 build/default/production/_ext/427700826/arp.o
 .debug_line    0x00006c08      0x230 build/default/production/_ext/427700826/berkeley_api.o
 .debug_line    0x00006e38      0x86e build/default/production/_ext/427700826/dhcp.o
 .debug_line    0x000076a6      0x29a build/default/production/_ext/427700826/dhcps.o
 .debug_line    0x00007940      0x653 build/default/production/_ext/427700826/dns.o
 .debug_line    0x00007f93      0x230 build/default/production/_ext/427700826/dnss.o
 .debug_line    0x000081c3      0x230 build/default/production/_ext/427700826/dyn_dns.o
 .debug_line    0x000083f3      0x230 build/default/production/_ext/427700826/enc28_mac.o
 .debug_line    0x00008623      0x230 build/default/production/_ext/427700826/enc28j60.o
 .debug_line    0x00008853      0x82d build/default/production/_ext/427700826/encs24j600.o
 .debug_line    0x00009080      0x4ee build/default/production/_ext/427700826/encx24_mac.o
 .debug_line    0x0000956e      0x230 build/default/production/_ext/427700826/eth_pic32_ext_phy.o
 .debug_line    0x0000979e      0x230 build/default/production/_ext/427700826/eth_pic32_ext_phy_dp83848.o
 .debug_line    0x000099ce      0x230 build/default/production/_ext/427700826/eth_pic32_int_mac.o
 .debug_line    0x00009bfe      0x230 build/default/production/_ext/427700826/ftp.o
 .debug_line    0x00009e2e      0x173 build/default/production/_ext/427700826/hash_fnv.o
 .debug_line    0x00009fa1      0x263 build/default/production/_ext/427700826/hash_tbl.o
 .debug_line    0x0000a204      0x402 build/default/production/_ext/427700826/icmp.o
 .debug_line    0x0000a606      0x230 build/default/production/_ext/427700826/icmpv6.o
 .debug_line    0x0000a836      0x89f build/default/production/_ext/427700826/ipv4.o
 .debug_line    0x0000b0d5      0x230 build/default/production/_ext/427700826/ipv6.o
 .debug_line    0x0000b305      0x230 build/default/production/_ext/427700826/mac_events_pic32.o
 .debug_line    0x0000b535      0x494 build/default/production/_ext/427700826/nbns.o
 .debug_line    0x0000b9c9      0x230 build/default/production/_ext/427700826/ndp.o
 .debug_line    0x0000bbf9      0x230 build/default/production/_ext/427700826/tcpip_reboot.o
 .debug_line    0x0000be29      0x230 build/default/production/_ext/427700826/rsa.o
 .debug_line    0x0000c059      0x230 build/default/production/_ext/427700826/smtp.o
 .debug_line    0x0000c289      0x230 build/default/production/_ext/427700826/snmp.o
 .debug_line    0x0000c4b9      0x230 build/default/production/_ext/427700826/snmpv3.o
 .debug_line    0x0000c6e9      0x230 build/default/production/_ext/427700826/snmpv3_usm.o
 .debug_line    0x0000c919      0x230 build/default/production/_ext/427700826/sntp.o
 .debug_line    0x0000cb49      0x230 build/default/production/_ext/427700826/ssl.o
 .debug_line    0x0000cd79     0x1428 build/default/production/_ext/427700826/tcp.o
 .debug_line    0x0000e1a1      0x536 build/default/production/_ext/427700826/tcpip_heap_alloc.o
 .debug_line    0x0000e6d7      0x230 build/default/production/_ext/427700826/tcpip_storage.o
 .debug_line    0x0000e907      0x230 build/default/production/_ext/427700826/telnet.o
 .debug_line    0x0000eb37      0x230 build/default/production/_ext/427700826/tftpc.o
 .debug_line    0x0000ed67      0xa18 build/default/production/_ext/427700826/udp.o
 .debug_line    0x0000f77f      0x47e build/default/production/_ext/427700826/tcpip_mac_object.o
 .debug_line    0x0000fbfd      0xdd5 build/default/production/_ext/427700826/tcpip_manager.o
 .debug_line    0x000109d2      0x691 build/default/production/_ext/427700826/tcpip_helpers.o
 .debug_line    0x00011063      0x230 build/default/production/_ext/427700826/tcpip_commands.o
 .debug_line    0x00011293      0x230 build/default/production/_ext/427700826/iperf.o
 .debug_line    0x000114c3       0xee build/default/production/_ext/427700826/tcpip_helper_c32.o
 .debug_line    0x000115b1      0x120 build/default/production/_ext/427700826/tcpip_notify.o
 .debug_line    0x000116d1      0x230 build/default/production/_ext/427700826/zero_conf_helper.o
 .debug_line    0x00011901      0x2a9 build/default/production/_ext/427700826/zero_conf_link_local.o
 .debug_line    0x00011baa      0x230 build/default/production/_ext/427700826/zero_conf_multicast_dns.o
 .debug_line    0x00011dda      0x230 build/default/production/_ext/334706090/wf_tx_power.o
 .debug_line    0x0001200a      0x230 build/default/production/_ext/334706090/wf_connect.o
 .debug_line    0x0001223a      0x230 build/default/production/_ext/334706090/wf_connection_algorithm.o
 .debug_line    0x0001246a      0x230 build/default/production/_ext/334706090/wf_connection_manager.o
 .debug_line    0x0001269a      0x230 build/default/production/_ext/334706090/wf_connection_profile.o
 .debug_line    0x000128ca      0x230 build/default/production/_ext/334706090/wf_easy_config.o
 .debug_line    0x00012afa      0x26c build/default/production/_ext/334706090/wf_eint.o
 .debug_line    0x00012d66      0x230 build/default/production/_ext/334706090/wf_event_handler.o
 .debug_line    0x00012f96      0x230 build/default/production/_ext/334706090/wf_init.o
 .debug_line    0x000131c6      0x230 build/default/production/_ext/334706090/wf_power_save.o
 .debug_line    0x000133f6      0x230 build/default/production/_ext/334706090/wf_scan.o
 .debug_line    0x00013626      0x26b build/default/production/_ext/334706090/wf_spi.o
 .debug_line    0x00013891      0x230 build/default/production/_ext/334706090/mrf24w_mac_pic32.o
 .debug_line    0x00013ac1      0x230 build/default/production/_ext/334706090/mrf24w_events.o
 .debug_line    0x00013cf1      0x230 build/default/production/_ext/334706090/wf_driver_com_24g.o
 .debug_line    0x00013f21      0x230 build/default/production/_ext/334706090/wf_driver_raw_24g.o
 .debug_line    0x00014151      0x230 build/default/production/_ext/334706090/wf_mac_24g.o
 .debug_line    0x00014381      0x230 build/default/production/_ext/334706090/wf_mgmt_msg_24g.o
 .debug_line    0x000145b1      0x230 build/default/production/_ext/334706090/wf_param_msg_24g.o
 .debug_line    0x000147e1      0x474 build/default/production/_ext/1472/main_demo.o
 .debug_line    0x00014c55        0x0 build/default/production/_ext/1472/custom_snmp_app.o
 .debug_line    0x00014c55        0x0 build/default/production/_ext/1472/custom_ssl_cert.o
 .debug_line    0x00014c55      0x18e build/default/production/_ext/1472/mpfs_img2.o
 .debug_line    0x00014de3      0x18e build/default/production/_ext/1472/wf_config.o
 .debug_line    0x00014f71      0x81c build/default/production/_ext/1472/custom_http_app.o
 .debug_line    0x0001578d      0x507 build/default/production/_ext/1472/tcp6_demo_app.o
 .debug_line    0x00015c94       0x6e c:/program files (x86)/microchip/xc32/v1.21/bin/../lib/gcc/pic32mx/4.5.2/../../../../pic32mx/lib/size\libmchp_peripheral.a(open_core_timer_lib.o)
 .debug_line    0x00015d02       0xbf c:/program files (x86)/microchip/xc32/v1.21/bin/../lib/gcc/pic32mx/4.5.2/../../../../pic32mx/lib/size\libmchp_peripheral_32MX795F512L.a(soft_reset_lib.o)
 .debug_line    0x00015dc1       0x62 c:/program files (x86)/microchip/xc32/v1.21/bin/../lib/gcc/pic32mx/4.5.2/../../../../pic32mx/lib/size\libmchp_peripheral_32MX795F512L.a(pcache.o)
 .debug_line    0x00015e23       0x73 c:/program files (x86)/microchip/xc32/v1.21/bin/../lib/gcc/pic32mx/4.5.2/../../../../pic32mx/lib/size\libmchp_peripheral_32MX795F512L.a(int_disable_interrupts_lib.o)
 .debug_line    0x00015e96       0x73 c:/program files (x86)/microchip/xc32/v1.21/bin/../lib/gcc/pic32mx/4.5.2/../../../../pic32mx/lib/size\libmchp_peripheral_32MX795F512L.a(int_restore_interrupts_lib.o)
 .debug_line    0x00015f09       0x6e c:/program files (x86)/microchip/xc32/v1.21/bin/../lib/gcc/pic32mx/4.5.2/../../../../pic32mx/lib/size\libmchp_peripheral_32MX795F512L.a(int_enable_mv_int_lib.o)
 .debug_line    0x00015f77       0x64 c:/program files (x86)/microchip/xc32/v1.21/bin/../lib/gcc/pic32mx/4.5.2/../../../../pic32mx/lib/size\libmchp_peripheral_32MX795F512L.a(int_tbl_lib.o)
 .debug_line    0x00015fdb       0xda c:/program files (x86)/microchip/xc32/v1.21/bin/../lib/gcc/pic32mx/4.5.2/../../../../pic32mx/lib/size\libmchp_peripheral_32MX795F512L.a(rtcc_init_lib.o)
 .debug_line    0x000160b5       0xda c:/program files (x86)/microchip/xc32/v1.21/bin/../lib/gcc/pic32mx/4.5.2/../../../../pic32mx/lib/size\libmchp_peripheral_32MX795F512L.a(rtcc_open_lib.o)
 .debug_line    0x0001618f       0x7f c:/program files (x86)/microchip/xc32/v1.21/bin/../lib/gcc/pic32mx/4.5.2/../../../../pic32mx/lib/size\libmchp_peripheral_32MX795F512L.a(spi_chn_data_rdy_lib.o)
 .debug_line    0x0001620e       0x7b c:/program files (x86)/microchip/xc32/v1.21/bin/../lib/gcc/pic32mx/4.5.2/../../../../pic32mx/lib/size\libmchp_peripheral_32MX795F512L.a(spi_chn_getc_lib.o)
 .debug_line    0x00016289       0x69 c:/program files (x86)/microchip/xc32/v1.21/bin/../lib/gcc/pic32mx/4.5.2/../../../../pic32mx/lib/size\libmchp_peripheral_32MX795F512L.a(spi_chn_open_lib.o)
 .debug_line    0x000162f2       0x7b c:/program files (x86)/microchip/xc32/v1.21/bin/../lib/gcc/pic32mx/4.5.2/../../../../pic32mx/lib/size\libmchp_peripheral_32MX795F512L.a(spi_chn_putc_lib.o)
 .debug_line    0x0001636d       0x72 c:/program files (x86)/microchip/xc32/v1.21/bin/../lib/gcc/pic32mx/4.5.2/../../../../pic32mx/lib/size\libmchp_peripheral_32MX795F512L.a(spi_chn_tx_buff_empty_lib.o)
 .debug_line    0x000163df        0x0 c:/program files (x86)/microchip/xc32/v1.21/bin/../lib/gcc/pic32mx/4.5.2/../../../../pic32mx/lib/size\libmchp_peripheral_32MX795F512L.a(spi_io_tbl_libp.o)
 .debug_line    0x000163df        0x0 c:/program files (x86)/microchip/xc32/v1.21/bin/../lib/gcc/pic32mx/4.5.2/../../../../pic32mx/lib/size\libmchp_peripheral_32MX795F512L.a(spi_map_tbl_libp.o)
 .debug_line    0x000163df       0x77 c:/program files (x86)/microchip/xc32/v1.21/bin/../lib/gcc/pic32mx/4.5.2/../../../../pic32mx/lib/size\libmchp_peripheral_32MX795F512L.a(port_set_pins_digital_in_lib.o)
 .debug_line    0x00016456       0x78 c:/program files (x86)/microchip/xc32/v1.21/bin/../lib/gcc/pic32mx/4.5.2/../../../../pic32mx/lib/size\libmchp_peripheral_32MX795F512L.a(port_set_pins_digital_out_lib.o)
 .debug_line    0x000164ce        0x0 c:/program files (x86)/microchip/xc32/v1.21/bin/../lib/gcc/pic32mx/4.5.2/../../../../pic32mx/lib/size\libmchp_peripheral_32MX795F512L.a(_ports_tbl_libp.o)
 .debug_line    0x000164ce       0x72 c:/program files (x86)/microchip/xc32/v1.21/bin/../lib/gcc/pic32mx/4.5.2/../../../../pic32mx/lib/size\libmchp_peripheral_32MX795F512L.a(int_enable_interrupts_lib.o)
 .debug_line    0x00016540       0xbd c:/program files (x86)/microchip/xc32/v1.21/bin/../lib/gcc/pic32mx/4.5.2/../../../../pic32mx/lib/size\libmchp_peripheral_32MX795F512L.a(_rtcc_wait_clock_off_lib.o)
 .debug_line    0x000165fd       0x6e c:/program files (x86)/microchip/xc32/v1.21/bin/../lib/gcc/pic32mx/4.5.2/../../../../pic32mx/lib/size\libmchp_peripheral_32MX795F512L.a(read_core_timer_lib.o)
 .debug_line    0x0001666b      0x119 c:/program files (x86)/microchip/xc32/v1.21/bin/../lib/gcc/pic32mx/4.5.2/size\libgcc.a(_udivdi3.o)
 .debug_line    0x00016784       0x9d c:/program files (x86)/microchip/xc32/v1.21/bin/../lib/gcc/pic32mx/4.5.2/../../../../pic32mx/lib/size\libpic32.a(default-bootstrap-exception-handler.o)
 .debug_line    0x00016821       0x8a c:/program files (x86)/microchip/xc32/v1.21/bin/../lib/gcc/pic32mx/4.5.2/../../../../pic32mx/lib/size\libpic32.a(default-on-reset.o)
 .debug_line    0x000168ab       0x8e c:/program files (x86)/microchip/xc32/v1.21/bin/../lib/gcc/pic32mx/4.5.2/../../../../pic32mx/lib/size\libpic32.a(default-on-bootstrap.o)
 .debug_line    0x00016939        0x0 c:/program files (x86)/microchip/xc32/v1.21/bin/../lib/gcc/pic32mx/4.5.2/../../../../pic32mx/lib/size\libpic32.a(errno.o)
 .debug_line    0x00016939       0x9c c:/program files (x86)/microchip/xc32/v1.21/bin/../lib/gcc/pic32mx/4.5.2/../../../../pic32mx/lib/size\libpic32.a(defaultinterrupt.o)
 .debug_line    0x000169d5       0x80 c:/program files (x86)/microchip/xc32/v1.21/bin/../lib/gcc/pic32mx/4.5.2/../../../../pic32mx/lib/size\libc.a(atoi.o)
 .debug_line    0x00016a55       0x80 c:/program files (x86)/microchip/xc32/v1.21/bin/../lib/gcc/pic32mx/4.5.2/../../../../pic32mx/lib/size\libc.a(atol.o)
 .debug_line    0x00016ad5        0x0 c:/program files (x86)/microchip/xc32/v1.21/bin/../lib/gcc/pic32mx/4.5.2/../../../../pic32mx/lib/size\libc.a(ctype.o)
 .debug_line    0x00016ad5       0x82 c:/program files (x86)/microchip/xc32/v1.21/bin/../lib/gcc/pic32mx/4.5.2/../../../../pic32mx/lib/size\libc.a(malloc.o)
 .debug_line    0x00016b57       0x80 c:/program files (x86)/microchip/xc32/v1.21/bin/../lib/gcc/pic32mx/4.5.2/../../../../pic32mx/lib/size\libc.a(rand.o)
 .debug_line    0x00016bd7       0x82 c:/program files (x86)/microchip/xc32/v1.21/bin/../lib/gcc/pic32mx/4.5.2/../../../../pic32mx/lib/size\libc.a(strcat.o)
 .debug_line    0x00016c59       0x82 c:/program files (x86)/microchip/xc32/v1.21/bin/../lib/gcc/pic32mx/4.5.2/../../../../pic32mx/lib/size\libc.a(strchr.o)
 .debug_line    0x00016cdb       0x83 c:/program files (x86)/microchip/xc32/v1.21/bin/../lib/gcc/pic32mx/4.5.2/../../../../pic32mx/lib/size\libc.a(strncat.o)
 .debug_line    0x00016d5e       0x83 c:/program files (x86)/microchip/xc32/v1.21/bin/../lib/gcc/pic32mx/4.5.2/../../../../pic32mx/lib/size\libc.a(strncmp.o)
 .debug_line    0x00016de1       0x83 c:/program files (x86)/microchip/xc32/v1.21/bin/../lib/gcc/pic32mx/4.5.2/../../../../pic32mx/lib/size\libc.a(strncpy.o)
 .debug_line    0x00016e64       0x83 c:/program files (x86)/microchip/xc32/v1.21/bin/../lib/gcc/pic32mx/4.5.2/../../../../pic32mx/lib/size\libc.a(strrchr.o)
 .debug_line    0x00016ee7       0x82 c:/program files (x86)/microchip/xc32/v1.21/bin/../lib/gcc/pic32mx/4.5.2/../../../../pic32mx/lib/size\libc.a(strstr.o)
 .debug_line    0x00016f69       0x82 c:/program files (x86)/microchip/xc32/v1.21/bin/../lib/gcc/pic32mx/4.5.2/../../../../pic32mx/lib/size\libc.a(strtol.o)
 .debug_line    0x00016feb       0x84 c:/program files (x86)/microchip/xc32/v1.21/bin/../lib/gcc/pic32mx/4.5.2/../../../../pic32mx/lib/size\libc.a(snprintf_cdnopsuxX.eo)
 .debug_line    0x0001706f       0x83 c:/program files (x86)/microchip/xc32/v1.21/bin/../lib/gcc/pic32mx/4.5.2/../../../../pic32mx/lib/size\libc.a(sprintf_cdnopsuxX.eo)
 .debug_line    0x000170f2       0x85 c:/program files (x86)/microchip/xc32/v1.21/bin/../lib/gcc/pic32mx/4.5.2/../../../../pic32mx/lib/size\libc.a(vsnprintf_cdnopsuxX.eo)
 .debug_line    0x00017177       0x85 c:/program files (x86)/microchip/xc32/v1.21/bin/../lib/gcc/pic32mx/4.5.2/../../../../pic32mx/lib/size\libc.a(vsnprintf.o)
 .debug_line    0x000171fc       0x82 c:/program files (x86)/microchip/xc32/v1.21/bin/../lib/gcc/pic32mx/4.5.2/../../../../pic32mx/lib/size\libc.a(ctypef.o)
 .debug_line    0x0001727e       0x82 c:/program files (x86)/microchip/xc32/v1.21/bin/../lib/gcc/pic32mx/4.5.2/../../../../pic32mx/lib/size\libc.a(doprnt_cdnopsuxX.eo)
 .debug_line    0x00017300       0x82 c:/program files (x86)/microchip/xc32/v1.21/bin/../lib/gcc/pic32mx/4.5.2/../../../../pic32mx/lib/size\libc.a(doprnt.o)
 .debug_line    0x00017382       0x81 c:/program files (x86)/microchip/xc32/v1.21/bin/../lib/gcc/pic32mx/4.5.2/../../../../pic32mx/lib/size\libc.a(_fputc_simple.o)
 .debug_line    0x00017403        0x0 c:/program files (x86)/microchip/xc32/v1.21/bin/../lib/gcc/pic32mx/4.5.2/../../../../pic32mx/lib/size\libc.a(powersf.o)
 .debug_line    0x00017403        0x0 c:/program files (x86)/microchip/xc32/v1.21/bin/../lib/gcc/pic32mx/4.5.2/../../../../pic32mx/lib/size\libc.a(_iob.o)
 .debug_line    0x00017403       0x82 c:/program files (x86)/microchip/xc32/v1.21/bin/../lib/gcc/pic32mx/4.5.2/../../../../pic32mx/lib/size\libc.a(_flsbuf_simple.o)
 .debug_line    0x00017485       0x7e c:/program files (x86)/microchip/xc32/v1.21/bin/../lib/gcc/pic32mx/4.5.2/../../../../pic32mx/lib/size\libpic32.a(sbrk.o)
 .debug_line    0x00017503       0x7f c:/program files (x86)/microchip/xc32/v1.21/bin/../lib/gcc/pic32mx/4.5.2/../../../../pic32mx/lib/size\libpic32.a(write.o)
 .debug_line    0x00017582       0x83 c:/program files (x86)/microchip/xc32/v1.21/bin/../lib/gcc/pic32mx/4.5.2/../../../../pic32mx/lib/size\libpic32.a(_mon_putc.o)
 .debug_line    0x00017605        0x0 c:/program files (x86)/microchip/xc32/v1.21/bin/../lib/gcc/pic32mx/4.5.2/../../../../pic32mx/lib/size\libpic32.a(xc32_uart.o)
 .debug_line    0x00017605       0x99 c:/program files (x86)/microchip/xc32/v1.21/bin/../lib/gcc/pic32mx/4.5.2/../../../../pic32mx/lib/size\libe.a(_floatdisf.o)
 .debug_line    0x0001769e       0xbe c:/program files (x86)/microchip/xc32/v1.21/bin/../lib/gcc/pic32mx/4.5.2/size\libgcc.a(_lshrdi3.o)
 .debug_line    0x0001775c       0xc9 c:/program files (x86)/microchip/xc32/v1.21/bin/../lib/gcc/pic32mx/4.5.2/size\libgcc.a(_floatundisf.o)
 .debug_line    0x00017825      0x11f c:/program files (x86)/microchip/xc32/v1.21/bin/../lib/gcc/pic32mx/4.5.2/size\libgcc.a(_umoddi3.o)
 .debug_line    0x00017944       0x70 c:/program files (x86)/microchip/xc32/v1.21/bin/../lib/gcc/pic32mx/4.5.2/size\libgcc.a(floatunsisf.o)

.debug_frame    0x00000000     0x664c
 *(.debug_frame)
 .debug_frame   0x00000000       0x2c build/default/production/_ext/1293749816/bsp.o
 .debug_frame   0x0000002c       0x48 build/default/production/_ext/101875047/lfsr.o
 .debug_frame   0x00000074      0x188 build/default/production/_ext/101875047/big_int.o
 .debug_frame   0x000001fc      0x10c build/default/production/_ext/101875047/hashes.o
 .debug_frame   0x00000308       0xf0 build/default/production/_ext/101875047/helpers.o
 .debug_frame   0x000003f8       0x64 build/default/production/_ext/1472/ping_demo.o
 .debug_frame   0x0000045c      0x3e8 build/default/production/_ext/365611741/system_services.o
 .debug_frame   0x00000844      0x278 build/default/production/_ext/365611741/system_debug.o
 .debug_frame   0x00000abc       0xa0 build/default/production/_ext/365611741/system_random.o
 .debug_frame   0x00000b5c      0x25c build/default/production/_ext/365611741/system_command.o
 .debug_frame   0x00000db8       0xf0 build/default/production/_ext/365611741/system_userio.o
 .debug_frame   0x00000ea8      0x7a8 build/default/production/_ext/97638081/sys_fs.o
 .debug_frame   0x00001650      0x2b8 build/default/production/_ext/97638081/mpfs2.o
 .debug_frame   0x00001908       0xd8 build/default/production/_ext/792872985/usart.o
 .debug_frame   0x000019e0       0xb8 build/default/production/_ext/792872985/lcd.o
 .debug_frame   0x00001a98       0x64 build/default/production/_ext/792872985/drv_spi.o
 .debug_frame   0x00001afc      0x144 build/default/production/_ext/792872985/spi_eeprom.o
 .debug_frame   0x00001c40      0x1b4 build/default/production/_ext/792872985/drv_media.o
 .debug_frame   0x00001df4       0xd8 build/default/production/_ext/427700826/tcpip_announce.o
 .debug_frame   0x00001ecc      0x434 build/default/production/_ext/427700826/http2.o
 .debug_frame   0x00002300      0x42c build/default/production/_ext/427700826/arp.o
 .debug_frame   0x0000272c      0x240 build/default/production/_ext/427700826/dhcp.o
 .debug_frame   0x0000296c       0x64 build/default/production/_ext/427700826/dhcps.o
 .debug_frame   0x000029d0      0x148 build/default/production/_ext/427700826/dns.o
 .debug_frame   0x00002b18      0x3e8 build/default/production/_ext/427700826/encs24j600.o
 .debug_frame   0x00002f00      0x278 build/default/production/_ext/427700826/encx24_mac.o
 .debug_frame   0x00003178       0x48 build/default/production/_ext/427700826/hash_fnv.o
 .debug_frame   0x000031c0       0xf0 build/default/production/_ext/427700826/hash_tbl.o
 .debug_frame   0x000032b0       0xd4 build/default/production/_ext/427700826/icmp.o
 .debug_frame   0x00003384      0x458 build/default/production/_ext/427700826/ipv4.o
 .debug_frame   0x000037dc       0x9c build/default/production/_ext/427700826/nbns.o
 .debug_frame   0x00003878      0x8ac build/default/production/_ext/427700826/tcp.o
 .debug_frame   0x00004124      0x1d0 build/default/production/_ext/427700826/tcpip_heap_alloc.o
 .debug_frame   0x000042f4      0x4e0 build/default/production/_ext/427700826/udp.o
 .debug_frame   0x000047d4      0x224 build/default/production/_ext/427700826/tcpip_mac_object.o
 .debug_frame   0x000049f8      0x844 build/default/production/_ext/427700826/tcpip_manager.o
 .debug_frame   0x0000523c      0x2e8 build/default/production/_ext/427700826/tcpip_helpers.o
 .debug_frame   0x00005524       0x64 build/default/production/_ext/427700826/tcpip_notify.o
 .debug_frame   0x00005588       0x64 build/default/production/_ext/427700826/zero_conf_link_local.o
 .debug_frame   0x000055ec       0x2c build/default/production/_ext/334706090/wf_eint.o
 .debug_frame   0x00005618       0x2c build/default/production/_ext/334706090/wf_spi.o
 .debug_frame   0x00005644       0x4c build/default/production/_ext/1472/main_demo.o
 .debug_frame   0x00005690      0x488 build/default/production/_ext/1472/custom_http_app.o
 .debug_frame   0x00005b18       0x84 build/default/production/_ext/1472/tcp6_demo_app.o
 .debug_frame   0x00005b9c       0x20 c:/program files (x86)/microchip/xc32/v1.21/bin/../lib/gcc/pic32mx/4.5.2/../../../../pic32mx/lib/size\libmchp_peripheral.a(open_core_timer_lib.o)
 .debug_frame   0x00005bbc       0x28 c:/program files (x86)/microchip/xc32/v1.21/bin/../lib/gcc/pic32mx/4.5.2/../../../../pic32mx/lib/size\libmchp_peripheral_32MX795F512L.a(soft_reset_lib.o)
 .debug_frame   0x00005be4       0x30 c:/program files (x86)/microchip/xc32/v1.21/bin/../lib/gcc/pic32mx/4.5.2/../../../../pic32mx/lib/size\libmchp_peripheral_32MX795F512L.a(pcache.o)
 .debug_frame   0x00005c14       0x20 c:/program files (x86)/microchip/xc32/v1.21/bin/../lib/gcc/pic32mx/4.5.2/../../../../pic32mx/lib/size\libmchp_peripheral_32MX795F512L.a(int_disable_interrupts_lib.o)
 .debug_frame   0x00005c34       0x20 c:/program files (x86)/microchip/xc32/v1.21/bin/../lib/gcc/pic32mx/4.5.2/../../../../pic32mx/lib/size\libmchp_peripheral_32MX795F512L.a(int_restore_interrupts_lib.o)
 .debug_frame   0x00005c54       0x28 c:/program files (x86)/microchip/xc32/v1.21/bin/../lib/gcc/pic32mx/4.5.2/../../../../pic32mx/lib/size\libmchp_peripheral_32MX795F512L.a(int_enable_mv_int_lib.o)
 .debug_frame   0x00005c7c       0xa0 c:/program files (x86)/microchip/xc32/v1.21/bin/../lib/gcc/pic32mx/4.5.2/../../../../pic32mx/lib/size\libmchp_peripheral_32MX795F512L.a(int_tbl_lib.o)
 .debug_frame   0x00005d1c       0x2c c:/program files (x86)/microchip/xc32/v1.21/bin/../lib/gcc/pic32mx/4.5.2/../../../../pic32mx/lib/size\libmchp_peripheral_32MX795F512L.a(rtcc_init_lib.o)
 .debug_frame   0x00005d48       0x34 c:/program files (x86)/microchip/xc32/v1.21/bin/../lib/gcc/pic32mx/4.5.2/../../../../pic32mx/lib/size\libmchp_peripheral_32MX795F512L.a(rtcc_open_lib.o)
 .debug_frame   0x00005d7c       0x20 c:/program files (x86)/microchip/xc32/v1.21/bin/../lib/gcc/pic32mx/4.5.2/../../../../pic32mx/lib/size\libmchp_peripheral_32MX795F512L.a(spi_chn_data_rdy_lib.o)
 .debug_frame   0x00005d9c       0x30 c:/program files (x86)/microchip/xc32/v1.21/bin/../lib/gcc/pic32mx/4.5.2/../../../../pic32mx/lib/size\libmchp_peripheral_32MX795F512L.a(spi_chn_getc_lib.o)
 .debug_frame   0x00005dcc       0x3c c:/program files (x86)/microchip/xc32/v1.21/bin/../lib/gcc/pic32mx/4.5.2/../../../../pic32mx/lib/size\libmchp_peripheral_32MX795F512L.a(spi_chn_open_lib.o)
 .debug_frame   0x00005e08       0x40 c:/program files (x86)/microchip/xc32/v1.21/bin/../lib/gcc/pic32mx/4.5.2/../../../../pic32mx/lib/size\libmchp_peripheral_32MX795F512L.a(spi_chn_putc_lib.o)
 .debug_frame   0x00005e48       0x20 c:/program files (x86)/microchip/xc32/v1.21/bin/../lib/gcc/pic32mx/4.5.2/../../../../pic32mx/lib/size\libmchp_peripheral_32MX795F512L.a(spi_chn_tx_buff_empty_lib.o)
 .debug_frame   0x00005e68       0x20 c:/program files (x86)/microchip/xc32/v1.21/bin/../lib/gcc/pic32mx/4.5.2/../../../../pic32mx/lib/size\libmchp_peripheral_32MX795F512L.a(port_set_pins_digital_in_lib.o)
 .debug_frame   0x00005e88       0x20 c:/program files (x86)/microchip/xc32/v1.21/bin/../lib/gcc/pic32mx/4.5.2/../../../../pic32mx/lib/size\libmchp_peripheral_32MX795F512L.a(port_set_pins_digital_out_lib.o)
 .debug_frame   0x00005ea8       0x20 c:/program files (x86)/microchip/xc32/v1.21/bin/../lib/gcc/pic32mx/4.5.2/../../../../pic32mx/lib/size\libmchp_peripheral_32MX795F512L.a(int_enable_interrupts_lib.o)
 .debug_frame   0x00005ec8       0x48 c:/program files (x86)/microchip/xc32/v1.21/bin/../lib/gcc/pic32mx/4.5.2/../../../../pic32mx/lib/size\libmchp_peripheral_32MX795F512L.a(_rtcc_wait_clock_off_lib.o)
 .debug_frame   0x00005f10       0x20 c:/program files (x86)/microchip/xc32/v1.21/bin/../lib/gcc/pic32mx/4.5.2/../../../../pic32mx/lib/size\libmchp_peripheral_32MX795F512L.a(read_core_timer_lib.o)
 .debug_frame   0x00005f30       0x20 c:/program files (x86)/microchip/xc32/v1.21/bin/../lib/gcc/pic32mx/4.5.2/size\libgcc.a(_udivdi3.o)
 .debug_frame   0x00005f50       0x20 c:/program files (x86)/microchip/xc32/v1.21/bin/../lib/gcc/pic32mx/4.5.2/../../../../pic32mx/lib/size\libpic32.a(default-bootstrap-exception-handler.o)
 .debug_frame   0x00005f70       0x20 c:/program files (x86)/microchip/xc32/v1.21/bin/../lib/gcc/pic32mx/4.5.2/../../../../pic32mx/lib/size\libpic32.a(default-on-reset.o)
 .debug_frame   0x00005f90       0x20 c:/program files (x86)/microchip/xc32/v1.21/bin/../lib/gcc/pic32mx/4.5.2/../../../../pic32mx/lib/size\libpic32.a(default-on-bootstrap.o)
 .debug_frame   0x00005fb0       0x20 c:/program files (x86)/microchip/xc32/v1.21/bin/../lib/gcc/pic32mx/4.5.2/../../../../pic32mx/lib/size\libpic32.a(defaultinterrupt.o)
 .debug_frame   0x00005fd0       0x20 c:/program files (x86)/microchip/xc32/v1.21/bin/../lib/gcc/pic32mx/4.5.2/../../../../pic32mx/lib/size\libc.a(atoi.o)
 .debug_frame   0x00005ff0       0x20 c:/program files (x86)/microchip/xc32/v1.21/bin/../lib/gcc/pic32mx/4.5.2/../../../../pic32mx/lib/size\libc.a(atol.o)
 .debug_frame   0x00006010       0x6c c:/program files (x86)/microchip/xc32/v1.21/bin/../lib/gcc/pic32mx/4.5.2/../../../../pic32mx/lib/size\libc.a(malloc.o)
 .debug_frame   0x0000607c       0x38 c:/program files (x86)/microchip/xc32/v1.21/bin/../lib/gcc/pic32mx/4.5.2/../../../../pic32mx/lib/size\libc.a(rand.o)
 .debug_frame   0x000060b4       0x20 c:/program files (x86)/microchip/xc32/v1.21/bin/../lib/gcc/pic32mx/4.5.2/../../../../pic32mx/lib/size\libc.a(strcat.o)
 .debug_frame   0x000060d4       0x20 c:/program files (x86)/microchip/xc32/v1.21/bin/../lib/gcc/pic32mx/4.5.2/../../../../pic32mx/lib/size\libc.a(strchr.o)
 .debug_frame   0x000060f4       0x20 c:/program files (x86)/microchip/xc32/v1.21/bin/../lib/gcc/pic32mx/4.5.2/../../../../pic32mx/lib/size\libc.a(strncat.o)
 .debug_frame   0x00006114       0x20 c:/program files (x86)/microchip/xc32/v1.21/bin/../lib/gcc/pic32mx/4.5.2/../../../../pic32mx/lib/size\libc.a(strncmp.o)
 .debug_frame   0x00006134       0x20 c:/program files (x86)/microchip/xc32/v1.21/bin/../lib/gcc/pic32mx/4.5.2/../../../../pic32mx/lib/size\libc.a(strncpy.o)
 .debug_frame   0x00006154       0x28 c:/program files (x86)/microchip/xc32/v1.21/bin/../lib/gcc/pic32mx/4.5.2/../../../../pic32mx/lib/size\libc.a(strrchr.o)
 .debug_frame   0x0000617c       0x2c c:/program files (x86)/microchip/xc32/v1.21/bin/../lib/gcc/pic32mx/4.5.2/../../../../pic32mx/lib/size\libc.a(strstr.o)
 .debug_frame   0x000061a8       0x58 c:/program files (x86)/microchip/xc32/v1.21/bin/../lib/gcc/pic32mx/4.5.2/../../../../pic32mx/lib/size\libc.a(strtol.o)
 .debug_frame   0x00006200       0x28 c:/program files (x86)/microchip/xc32/v1.21/bin/../lib/gcc/pic32mx/4.5.2/../../../../pic32mx/lib/size\libc.a(snprintf_cdnopsuxX.eo)
 .debug_frame   0x00006228       0x2c c:/program files (x86)/microchip/xc32/v1.21/bin/../lib/gcc/pic32mx/4.5.2/../../../../pic32mx/lib/size\libc.a(sprintf_cdnopsuxX.eo)
 .debug_frame   0x00006254       0x28 c:/program files (x86)/microchip/xc32/v1.21/bin/../lib/gcc/pic32mx/4.5.2/../../../../pic32mx/lib/size\libc.a(vsnprintf_cdnopsuxX.eo)
 .debug_frame   0x0000627c       0x28 c:/program files (x86)/microchip/xc32/v1.21/bin/../lib/gcc/pic32mx/4.5.2/../../../../pic32mx/lib/size\libc.a(vsnprintf.o)
 .debug_frame   0x000062a4      0x120 c:/program files (x86)/microchip/xc32/v1.21/bin/../lib/gcc/pic32mx/4.5.2/../../../../pic32mx/lib/size\libc.a(ctypef.o)
 .debug_frame   0x000063c4       0x38 c:/program files (x86)/microchip/xc32/v1.21/bin/../lib/gcc/pic32mx/4.5.2/../../../../pic32mx/lib/size\libc.a(doprnt_cdnopsuxX.eo)
 .debug_frame   0x000063fc       0x74 c:/program files (x86)/microchip/xc32/v1.21/bin/../lib/gcc/pic32mx/4.5.2/../../../../pic32mx/lib/size\libc.a(doprnt.o)
 .debug_frame   0x00006470       0x2c c:/program files (x86)/microchip/xc32/v1.21/bin/../lib/gcc/pic32mx/4.5.2/../../../../pic32mx/lib/size\libc.a(_fputc_simple.o)
 .debug_frame   0x0000649c       0x28 c:/program files (x86)/microchip/xc32/v1.21/bin/../lib/gcc/pic32mx/4.5.2/../../../../pic32mx/lib/size\libc.a(_flsbuf_simple.o)
 .debug_frame   0x000064c4       0x88 c:/program files (x86)/microchip/xc32/v1.21/bin/../lib/gcc/pic32mx/4.5.2/../../../../pic32mx/lib/size\libpic32.a(sbrk.o)
 .debug_frame   0x0000654c       0x2c c:/program files (x86)/microchip/xc32/v1.21/bin/../lib/gcc/pic32mx/4.5.2/../../../../pic32mx/lib/size\libpic32.a(write.o)
 .debug_frame   0x00006578       0x20 c:/program files (x86)/microchip/xc32/v1.21/bin/../lib/gcc/pic32mx/4.5.2/../../../../pic32mx/lib/size\libpic32.a(_mon_putc.o)
 .debug_frame   0x00006598       0x20 c:/program files (x86)/microchip/xc32/v1.21/bin/../lib/gcc/pic32mx/4.5.2/../../../../pic32mx/lib/size\libe.a(_floatdisf.o)
 .debug_frame   0x000065b8       0x20 c:/program files (x86)/microchip/xc32/v1.21/bin/../lib/gcc/pic32mx/4.5.2/size\libgcc.a(_lshrdi3.o)
 .debug_frame   0x000065d8       0x2c c:/program files (x86)/microchip/xc32/v1.21/bin/../lib/gcc/pic32mx/4.5.2/size\libgcc.a(_floatundisf.o)
 .debug_frame   0x00006604       0x20 c:/program files (x86)/microchip/xc32/v1.21/bin/../lib/gcc/pic32mx/4.5.2/size\libgcc.a(_umoddi3.o)
 .debug_frame   0x00006624       0x28 c:/program files (x86)/microchip/xc32/v1.21/bin/../lib/gcc/pic32mx/4.5.2/size\libgcc.a(floatunsisf.o)

.debug_str      0x00000000     0x8b9d
 *(.debug_str)
 .debug_str     0x00000000      0x175 build/default/production/_ext/1293749816/bsp.o
 .debug_str     0x00000175        0x0 build/default/production/_ext/101875047/lfsr.o
 .debug_str     0x00000175      0x12f build/default/production/_ext/101875047/big_int.o
 .debug_str     0x000002a4       0x1a build/default/production/_ext/101875047/hashes.o
 .debug_str     0x000002be        0x0 build/default/production/_ext/101875047/helpers.o
 .debug_str     0x000002be        0x0 build/default/production/_ext/1472/berkeley_tcp_client_demo.o
 .debug_str     0x000002be        0x0 build/default/production/_ext/1472/berkeley_tcp_server_demo.o
 .debug_str     0x000002be        0x0 build/default/production/_ext/1472/berkeley_udp_client_demo.o
 .debug_str     0x000002be      0x156 build/default/production/_ext/1472/generic_tcp_client.o
 .debug_str     0x00000414      0x156 build/default/production/_ext/1472/generic_tcp_server.o
 .debug_str     0x0000056a      0x18b build/default/production/_ext/1472/ping_demo.o
 .debug_str     0x000006f5        0x0 build/default/production/_ext/1472/smtp_demo.o
 .debug_str     0x000006f5      0x230 build/default/production/_ext/365611741/system_services.o
 .debug_str     0x00000925      0x15e build/default/production/_ext/365611741/system_debug.o
 .debug_str     0x00000a83      0x15f build/default/production/_ext/365611741/system_random.o
 .debug_str     0x00000be2      0x127 build/default/production/_ext/365611741/system_command.o
 .debug_str     0x00000d09      0x173 build/default/production/_ext/365611741/system_userio.o
 .debug_str     0x00000e7c      0x14f build/default/production/_ext/97638081/sys_fs.o
 .debug_str     0x00000fcb      0x135 build/default/production/_ext/97638081/mpfs2.o
 .debug_str     0x00001100      0x11a build/default/production/_ext/792872985/usart.o
 .debug_str     0x0000121a      0x17c build/default/production/_ext/792872985/lcd.o
 .debug_str     0x00001396      0x156 build/default/production/_ext/792872985/drv_spi.o
 .debug_str     0x000014ec        0x0 build/default/production/_ext/792872985/db_appio.o
 .debug_str     0x000014ec      0x12f build/default/production/_ext/792872985/spi_ram.o
 .debug_str     0x0000161b      0x1be build/default/production/_ext/792872985/spi_eeprom.o
 .debug_str     0x000017d9      0x12f build/default/production/_ext/792872985/spi_flash.o
 .debug_str     0x00001908      0x1c6 build/default/production/_ext/792872985/drv_media.o
 .debug_str     0x00001ace      0x196 build/default/production/_ext/427700826/tcpip_announce.o
 .debug_str     0x00001c64      0x1d1 build/default/production/_ext/427700826/http2.o
 .debug_str     0x00001e35      0x170 build/default/production/_ext/427700826/arcfour.o
 .debug_str     0x00001fa5      0x234 build/default/production/_ext/427700826/arp.o
 .debug_str     0x000021d9      0x170 build/default/production/_ext/427700826/berkeley_api.o
 .debug_str     0x00002349      0x1c6 build/default/production/_ext/427700826/dhcp.o
 .debug_str     0x0000250f      0x170 build/default/production/_ext/427700826/dhcps.o
 .debug_str     0x0000267f      0x18f build/default/production/_ext/427700826/dns.o
 .debug_str     0x0000280e      0x170 build/default/production/_ext/427700826/dnss.o
 .debug_str     0x0000297e      0x170 build/default/production/_ext/427700826/dyn_dns.o
 .debug_str     0x00002aee      0x170 build/default/production/_ext/427700826/enc28_mac.o
 .debug_str     0x00002c5e      0x170 build/default/production/_ext/427700826/enc28j60.o
 .debug_str     0x00002dce      0x21e build/default/production/_ext/427700826/encs24j600.o
 .debug_str     0x00002fec      0x194 build/default/production/_ext/427700826/encx24_mac.o
 .debug_str     0x00003180      0x170 build/default/production/_ext/427700826/eth_pic32_ext_phy.o
 .debug_str     0x000032f0      0x170 build/default/production/_ext/427700826/eth_pic32_ext_phy_dp83848.o
 .debug_str     0x00003460      0x170 build/default/production/_ext/427700826/eth_pic32_int_mac.o
 .debug_str     0x000035d0      0x170 build/default/production/_ext/427700826/ftp.o
 .debug_str     0x00003740        0x0 build/default/production/_ext/427700826/hash_fnv.o
 .debug_str     0x00003740        0xa build/default/production/_ext/427700826/hash_tbl.o
 .debug_str     0x0000374a      0x1a8 build/default/production/_ext/427700826/icmp.o
 .debug_str     0x000038f2      0x170 build/default/production/_ext/427700826/icmpv6.o
 .debug_str     0x00003a62      0x227 build/default/production/_ext/427700826/ipv4.o
 .debug_str     0x00003c89      0x170 build/default/production/_ext/427700826/ipv6.o
 .debug_str     0x00003df9      0x170 build/default/production/_ext/427700826/mac_events_pic32.o
 .debug_str     0x00003f69      0x1b1 build/default/production/_ext/427700826/nbns.o
 .debug_str     0x0000411a      0x170 build/default/production/_ext/427700826/ndp.o
 .debug_str     0x0000428a      0x170 build/default/production/_ext/427700826/tcpip_reboot.o
 .debug_str     0x000043fa      0x170 build/default/production/_ext/427700826/rsa.o
 .debug_str     0x0000456a      0x170 build/default/production/_ext/427700826/smtp.o
 .debug_str     0x000046da      0x170 build/default/production/_ext/427700826/snmp.o
 .debug_str     0x0000484a      0x170 build/default/production/_ext/427700826/snmpv3.o
 .debug_str     0x000049ba      0x170 build/default/production/_ext/427700826/snmpv3_usm.o
 .debug_str     0x00004b2a      0x170 build/default/production/_ext/427700826/sntp.o
 .debug_str     0x00004c9a      0x170 build/default/production/_ext/427700826/ssl.o
 .debug_str     0x00004e0a      0x26b build/default/production/_ext/427700826/tcp.o
 .debug_str     0x00005075      0x195 build/default/production/_ext/427700826/tcpip_heap_alloc.o
 .debug_str     0x0000520a      0x170 build/default/production/_ext/427700826/tcpip_storage.o
 .debug_str     0x0000537a      0x170 build/default/production/_ext/427700826/telnet.o
 .debug_str     0x000054ea      0x170 build/default/production/_ext/427700826/tftpc.o
 .debug_str     0x0000565a      0x247 build/default/production/_ext/427700826/udp.o
 .debug_str     0x000058a1      0x29a build/default/production/_ext/427700826/tcpip_mac_object.o
 .debug_str     0x00005b3b      0x32c build/default/production/_ext/427700826/tcpip_manager.o
 .debug_str     0x00005e67      0x181 build/default/production/_ext/427700826/tcpip_helpers.o
 .debug_str     0x00005fe8      0x170 build/default/production/_ext/427700826/tcpip_commands.o
 .debug_str     0x00006158      0x170 build/default/production/_ext/427700826/iperf.o
 .debug_str     0x000062c8        0xb build/default/production/_ext/427700826/tcpip_notify.o
 .debug_str     0x000062d3      0x170 build/default/production/_ext/427700826/zero_conf_helper.o
 .debug_str     0x00006443      0x170 build/default/production/_ext/427700826/zero_conf_link_local.o
 .debug_str     0x000065b3      0x170 build/default/production/_ext/427700826/zero_conf_multicast_dns.o
 .debug_str     0x00006723      0x170 build/default/production/_ext/334706090/wf_tx_power.o
 .debug_str     0x00006893      0x170 build/default/production/_ext/334706090/wf_connect.o
 .debug_str     0x00006a03      0x170 build/default/production/_ext/334706090/wf_connection_algorithm.o
 .debug_str     0x00006b73      0x170 build/default/production/_ext/334706090/wf_connection_manager.o
 .debug_str     0x00006ce3      0x170 build/default/production/_ext/334706090/wf_connection_profile.o
 .debug_str     0x00006e53      0x170 build/default/production/_ext/334706090/wf_easy_config.o
 .debug_str     0x00006fc3      0x170 build/default/production/_ext/334706090/wf_eint.o
 .debug_str     0x00007133      0x170 build/default/production/_ext/334706090/wf_event_handler.o
 .debug_str     0x000072a3      0x170 build/default/production/_ext/334706090/wf_init.o
 .debug_str     0x00007413      0x170 build/default/production/_ext/334706090/wf_power_save.o
 .debug_str     0x00007583      0x170 build/default/production/_ext/334706090/wf_scan.o
 .debug_str     0x000076f3      0x170 build/default/production/_ext/334706090/wf_spi.o
 .debug_str     0x00007863      0x170 build/default/production/_ext/334706090/mrf24w_mac_pic32.o
 .debug_str     0x000079d3      0x170 build/default/production/_ext/334706090/mrf24w_events.o
 .debug_str     0x00007b43      0x170 build/default/production/_ext/334706090/wf_driver_com_24g.o
 .debug_str     0x00007cb3      0x170 build/default/production/_ext/334706090/wf_driver_raw_24g.o
 .debug_str     0x00007e23      0x170 build/default/production/_ext/334706090/wf_mac_24g.o
 .debug_str     0x00007f93      0x170 build/default/production/_ext/334706090/wf_mgmt_msg_24g.o
 .debug_str     0x00008103      0x170 build/default/production/_ext/334706090/wf_param_msg_24g.o
 .debug_str     0x00008273      0x210 build/default/production/_ext/1472/main_demo.o
 .debug_str     0x00008483        0x0 build/default/production/_ext/1472/custom_snmp_app.o
 .debug_str     0x00008483        0x0 build/default/production/_ext/1472/custom_ssl_cert.o
 .debug_str     0x00008483      0x12f build/default/production/_ext/1472/mpfs_img2.o
 .debug_str     0x000085b2      0x12f build/default/production/_ext/1472/wf_config.o
 .debug_str     0x000086e1      0x1c3 build/default/production/_ext/1472/custom_http_app.o
 .debug_str     0x000088a4      0x2f9 build/default/production/_ext/1472/tcp6_demo_app.o
 .debug_str     0x00008b9d        0x0 c:/program files (x86)/microchip/xc32/v1.21/bin/../lib/gcc/pic32mx/4.5.2/../../../../pic32mx/lib/size\libmchp_peripheral.a(open_core_timer_lib.o)
 .debug_str     0x00008b9d        0x0 c:/program files (x86)/microchip/xc32/v1.21/bin/../lib/gcc/pic32mx/4.5.2/../../../../pic32mx/lib/size\libmchp_peripheral_32MX795F512L.a(soft_reset_lib.o)
 .debug_str     0x00008b9d        0x0 c:/program files (x86)/microchip/xc32/v1.21/bin/../lib/gcc/pic32mx/4.5.2/../../../../pic32mx/lib/size\libmchp_peripheral_32MX795F512L.a(pcache.o)
 .debug_str     0x00008b9d        0x0 c:/program files (x86)/microchip/xc32/v1.21/bin/../lib/gcc/pic32mx/4.5.2/../../../../pic32mx/lib/size\libmchp_peripheral_32MX795F512L.a(int_disable_interrupts_lib.o)
 .debug_str     0x00008b9d        0x0 c:/program files (x86)/microchip/xc32/v1.21/bin/../lib/gcc/pic32mx/4.5.2/../../../../pic32mx/lib/size\libmchp_peripheral_32MX795F512L.a(int_restore_interrupts_lib.o)
 .debug_str     0x00008b9d        0x0 c:/program files (x86)/microchip/xc32/v1.21/bin/../lib/gcc/pic32mx/4.5.2/../../../../pic32mx/lib/size\libmchp_peripheral_32MX795F512L.a(int_enable_mv_int_lib.o)
 .debug_str     0x00008b9d        0x0 c:/program files (x86)/microchip/xc32/v1.21/bin/../lib/gcc/pic32mx/4.5.2/../../../../pic32mx/lib/size\libmchp_peripheral_32MX795F512L.a(int_tbl_lib.o)
 .debug_str     0x00008b9d        0x0 c:/program files (x86)/microchip/xc32/v1.21/bin/../lib/gcc/pic32mx/4.5.2/../../../../pic32mx/lib/size\libmchp_peripheral_32MX795F512L.a(rtcc_init_lib.o)
 .debug_str     0x00008b9d        0x0 c:/program files (x86)/microchip/xc32/v1.21/bin/../lib/gcc/pic32mx/4.5.2/../../../../pic32mx/lib/size\libmchp_peripheral_32MX795F512L.a(rtcc_open_lib.o)
 .debug_str     0x00008b9d        0x0 c:/program files (x86)/microchip/xc32/v1.21/bin/../lib/gcc/pic32mx/4.5.2/../../../../pic32mx/lib/size\libmchp_peripheral_32MX795F512L.a(spi_chn_data_rdy_lib.o)
 .debug_str     0x00008b9d        0x0 c:/program files (x86)/microchip/xc32/v1.21/bin/../lib/gcc/pic32mx/4.5.2/../../../../pic32mx/lib/size\libmchp_peripheral_32MX795F512L.a(spi_chn_getc_lib.o)
 .debug_str     0x00008b9d        0x0 c:/program files (x86)/microchip/xc32/v1.21/bin/../lib/gcc/pic32mx/4.5.2/../../../../pic32mx/lib/size\libmchp_peripheral_32MX795F512L.a(spi_chn_open_lib.o)
 .debug_str     0x00008b9d        0x0 c:/program files (x86)/microchip/xc32/v1.21/bin/../lib/gcc/pic32mx/4.5.2/../../../../pic32mx/lib/size\libmchp_peripheral_32MX795F512L.a(spi_chn_putc_lib.o)
 .debug_str     0x00008b9d        0x0 c:/program files (x86)/microchip/xc32/v1.21/bin/../lib/gcc/pic32mx/4.5.2/../../../../pic32mx/lib/size\libmchp_peripheral_32MX795F512L.a(spi_chn_tx_buff_empty_lib.o)
 .debug_str     0x00008b9d        0x0 c:/program files (x86)/microchip/xc32/v1.21/bin/../lib/gcc/pic32mx/4.5.2/../../../../pic32mx/lib/size\libmchp_peripheral_32MX795F512L.a(spi_io_tbl_libp.o)
 .debug_str     0x00008b9d        0x0 c:/program files (x86)/microchip/xc32/v1.21/bin/../lib/gcc/pic32mx/4.5.2/../../../../pic32mx/lib/size\libmchp_peripheral_32MX795F512L.a(spi_map_tbl_libp.o)
 .debug_str     0x00008b9d        0x0 c:/program files (x86)/microchip/xc32/v1.21/bin/../lib/gcc/pic32mx/4.5.2/../../../../pic32mx/lib/size\libmchp_peripheral_32MX795F512L.a(port_set_pins_digital_in_lib.o)
 .debug_str     0x00008b9d        0x0 c:/program files (x86)/microchip/xc32/v1.21/bin/../lib/gcc/pic32mx/4.5.2/../../../../pic32mx/lib/size\libmchp_peripheral_32MX795F512L.a(port_set_pins_digital_out_lib.o)
 .debug_str     0x00008b9d        0x0 c:/program files (x86)/microchip/xc32/v1.21/bin/../lib/gcc/pic32mx/4.5.2/../../../../pic32mx/lib/size\libmchp_peripheral_32MX795F512L.a(_ports_tbl_libp.o)
 .debug_str     0x00008b9d        0x0 c:/program files (x86)/microchip/xc32/v1.21/bin/../lib/gcc/pic32mx/4.5.2/../../../../pic32mx/lib/size\libmchp_peripheral_32MX795F512L.a(int_enable_interrupts_lib.o)
 .debug_str     0x00008b9d        0x0 c:/program files (x86)/microchip/xc32/v1.21/bin/../lib/gcc/pic32mx/4.5.2/../../../../pic32mx/lib/size\libmchp_peripheral_32MX795F512L.a(_rtcc_wait_clock_off_lib.o)
 .debug_str     0x00008b9d        0x0 c:/program files (x86)/microchip/xc32/v1.21/bin/../lib/gcc/pic32mx/4.5.2/../../../../pic32mx/lib/size\libmchp_peripheral_32MX795F512L.a(read_core_timer_lib.o)
 .debug_str     0x00008b9d        0x0 c:/program files (x86)/microchip/xc32/v1.21/bin/../lib/gcc/pic32mx/4.5.2/size\libgcc.a(_udivdi3.o)
 .debug_str     0x00008b9d        0x0 c:/program files (x86)/microchip/xc32/v1.21/bin/../lib/gcc/pic32mx/4.5.2/../../../../pic32mx/lib/size\libpic32.a(default-bootstrap-exception-handler.o)
 .debug_str     0x00008b9d        0x0 c:/program files (x86)/microchip/xc32/v1.21/bin/../lib/gcc/pic32mx/4.5.2/../../../../pic32mx/lib/size\libpic32.a(default-on-reset.o)
 .debug_str     0x00008b9d        0x0 c:/program files (x86)/microchip/xc32/v1.21/bin/../lib/gcc/pic32mx/4.5.2/../../../../pic32mx/lib/size\libpic32.a(default-on-bootstrap.o)
 .debug_str     0x00008b9d        0x0 c:/program files (x86)/microchip/xc32/v1.21/bin/../lib/gcc/pic32mx/4.5.2/../../../../pic32mx/lib/size\libpic32.a(errno.o)
 .debug_str     0x00008b9d        0x0 c:/program files (x86)/microchip/xc32/v1.21/bin/../lib/gcc/pic32mx/4.5.2/../../../../pic32mx/lib/size\libpic32.a(defaultinterrupt.o)
 .debug_str     0x00008b9d        0x0 c:/program files (x86)/microchip/xc32/v1.21/bin/../lib/gcc/pic32mx/4.5.2/../../../../pic32mx/lib/size\libc.a(atoi.o)
 .debug_str     0x00008b9d        0x0 c:/program files (x86)/microchip/xc32/v1.21/bin/../lib/gcc/pic32mx/4.5.2/../../../../pic32mx/lib/size\libc.a(atol.o)
 .debug_str     0x00008b9d        0x0 c:/program files (x86)/microchip/xc32/v1.21/bin/../lib/gcc/pic32mx/4.5.2/../../../../pic32mx/lib/size\libc.a(ctype.o)
 .debug_str     0x00008b9d        0x0 c:/program files (x86)/microchip/xc32/v1.21/bin/../lib/gcc/pic32mx/4.5.2/../../../../pic32mx/lib/size\libc.a(malloc.o)
 .debug_str     0x00008b9d        0x0 c:/program files (x86)/microchip/xc32/v1.21/bin/../lib/gcc/pic32mx/4.5.2/../../../../pic32mx/lib/size\libc.a(rand.o)
 .debug_str     0x00008b9d        0x0 c:/program files (x86)/microchip/xc32/v1.21/bin/../lib/gcc/pic32mx/4.5.2/../../../../pic32mx/lib/size\libc.a(strcat.o)
 .debug_str     0x00008b9d        0x0 c:/program files (x86)/microchip/xc32/v1.21/bin/../lib/gcc/pic32mx/4.5.2/../../../../pic32mx/lib/size\libc.a(strchr.o)
 .debug_str     0x00008b9d        0x0 c:/program files (x86)/microchip/xc32/v1.21/bin/../lib/gcc/pic32mx/4.5.2/../../../../pic32mx/lib/size\libc.a(strncat.o)
 .debug_str     0x00008b9d        0x0 c:/program files (x86)/microchip/xc32/v1.21/bin/../lib/gcc/pic32mx/4.5.2/../../../../pic32mx/lib/size\libc.a(strncmp.o)
 .debug_str     0x00008b9d        0x0 c:/program files (x86)/microchip/xc32/v1.21/bin/../lib/gcc/pic32mx/4.5.2/../../../../pic32mx/lib/size\libc.a(strncpy.o)
 .debug_str     0x00008b9d        0x0 c:/program files (x86)/microchip/xc32/v1.21/bin/../lib/gcc/pic32mx/4.5.2/../../../../pic32mx/lib/size\libc.a(strrchr.o)
 .debug_str     0x00008b9d        0x0 c:/program files (x86)/microchip/xc32/v1.21/bin/../lib/gcc/pic32mx/4.5.2/../../../../pic32mx/lib/size\libc.a(strstr.o)
 .debug_str     0x00008b9d        0x0 c:/program files (x86)/microchip/xc32/v1.21/bin/../lib/gcc/pic32mx/4.5.2/../../../../pic32mx/lib/size\libc.a(strtol.o)
 .debug_str     0x00008b9d        0x0 c:/program files (x86)/microchip/xc32/v1.21/bin/../lib/gcc/pic32mx/4.5.2/../../../../pic32mx/lib/size\libc.a(snprintf_cdnopsuxX.eo)
 .debug_str     0x00008b9d        0x0 c:/program files (x86)/microchip/xc32/v1.21/bin/../lib/gcc/pic32mx/4.5.2/../../../../pic32mx/lib/size\libc.a(sprintf_cdnopsuxX.eo)
 .debug_str     0x00008b9d        0x0 c:/program files (x86)/microchip/xc32/v1.21/bin/../lib/gcc/pic32mx/4.5.2/../../../../pic32mx/lib/size\libc.a(vsnprintf_cdnopsuxX.eo)
 .debug_str     0x00008b9d        0x0 c:/program files (x86)/microchip/xc32/v1.21/bin/../lib/gcc/pic32mx/4.5.2/../../../../pic32mx/lib/size\libc.a(vsnprintf.o)
 .debug_str     0x00008b9d        0x0 c:/program files (x86)/microchip/xc32/v1.21/bin/../lib/gcc/pic32mx/4.5.2/../../../../pic32mx/lib/size\libc.a(ctypef.o)
 .debug_str     0x00008b9d        0x0 c:/program files (x86)/microchip/xc32/v1.21/bin/../lib/gcc/pic32mx/4.5.2/../../../../pic32mx/lib/size\libc.a(doprnt_cdnopsuxX.eo)
 .debug_str     0x00008b9d        0x0 c:/program files (x86)/microchip/xc32/v1.21/bin/../lib/gcc/pic32mx/4.5.2/../../../../pic32mx/lib/size\libc.a(doprnt.o)
 .debug_str     0x00008b9d        0x0 c:/program files (x86)/microchip/xc32/v1.21/bin/../lib/gcc/pic32mx/4.5.2/../../../../pic32mx/lib/size\libc.a(_fputc_simple.o)
 .debug_str     0x00008b9d        0x0 c:/program files (x86)/microchip/xc32/v1.21/bin/../lib/gcc/pic32mx/4.5.2/../../../../pic32mx/lib/size\libc.a(powersf.o)
 .debug_str     0x00008b9d        0x0 c:/program files (x86)/microchip/xc32/v1.21/bin/../lib/gcc/pic32mx/4.5.2/../../../../pic32mx/lib/size\libc.a(_iob.o)
 .debug_str     0x00008b9d        0x0 c:/program files (x86)/microchip/xc32/v1.21/bin/../lib/gcc/pic32mx/4.5.2/../../../../pic32mx/lib/size\libc.a(_flsbuf_simple.o)
 .debug_str     0x00008b9d        0x0 c:/program files (x86)/microchip/xc32/v1.21/bin/../lib/gcc/pic32mx/4.5.2/../../../../pic32mx/lib/size\libpic32.a(sbrk.o)
 .debug_str     0x00008b9d        0x0 c:/program files (x86)/microchip/xc32/v1.21/bin/../lib/gcc/pic32mx/4.5.2/../../../../pic32mx/lib/size\libpic32.a(write.o)
 .debug_str     0x00008b9d        0x0 c:/program files (x86)/microchip/xc32/v1.21/bin/../lib/gcc/pic32mx/4.5.2/../../../../pic32mx/lib/size\libpic32.a(_mon_putc.o)
 .debug_str     0x00008b9d        0x0 c:/program files (x86)/microchip/xc32/v1.21/bin/../lib/gcc/pic32mx/4.5.2/../../../../pic32mx/lib/size\libpic32.a(xc32_uart.o)
 .debug_str     0x00008b9d        0x0 c:/program files (x86)/microchip/xc32/v1.21/bin/../lib/gcc/pic32mx/4.5.2/../../../../pic32mx/lib/size\libe.a(_floatdisf.o)
 .debug_str     0x00008b9d        0x0 c:/program files (x86)/microchip/xc32/v1.21/bin/../lib/gcc/pic32mx/4.5.2/size\libgcc.a(_lshrdi3.o)
 .debug_str     0x00008b9d        0x0 c:/program files (x86)/microchip/xc32/v1.21/bin/../lib/gcc/pic32mx/4.5.2/size\libgcc.a(_floatundisf.o)
 .debug_str     0x00008b9d        0x0 c:/program files (x86)/microchip/xc32/v1.21/bin/../lib/gcc/pic32mx/4.5.2/size\libgcc.a(_umoddi3.o)
 .debug_str     0x00008b9d        0x0 c:/program files (x86)/microchip/xc32/v1.21/bin/../lib/gcc/pic32mx/4.5.2/size\libgcc.a(floatunsisf.o)

.debug_loc      0x00000000     0x166a
 *(.debug_loc)
 .debug_loc     0x00000000      0xa67 c:/program files (x86)/microchip/xc32/v1.21/bin/../lib/gcc/pic32mx/4.5.2/size\libgcc.a(_udivdi3.o)
 .debug_loc     0x00000a67       0x5f c:/program files (x86)/microchip/xc32/v1.21/bin/../lib/gcc/pic32mx/4.5.2/size\libgcc.a(_lshrdi3.o)
 .debug_loc     0x00000ac6       0xc9 c:/program files (x86)/microchip/xc32/v1.21/bin/../lib/gcc/pic32mx/4.5.2/size\libgcc.a(_floatundisf.o)
 .debug_loc     0x00000b8f      0xa73 c:/program files (x86)/microchip/xc32/v1.21/bin/../lib/gcc/pic32mx/4.5.2/size\libgcc.a(_umoddi3.o)
 .debug_loc     0x00001602       0x68 c:/program files (x86)/microchip/xc32/v1.21/bin/../lib/gcc/pic32mx/4.5.2/size\libgcc.a(floatunsisf.o)

.debug_macinfo
 *(.debug_macinfo)

.debug_weaknames
 *(.debug_weaknames)

.debug_funcnames
 *(.debug_funcnames)

.debug_typenames
 *(.debug_typenames)

.debug_varnames
 *(.debug_varnames)

.debug_pubtypes
                0x00000000     0x997b
 *(.debug_pubtypes)
 .debug_pubtypes
                0x00000000      0x143 build/default/production/_ext/1293749816/bsp.o
 .debug_pubtypes
                0x00000143       0x3e build/default/production/_ext/101875047/lfsr.o
 .debug_pubtypes
                0x00000181      0x13a build/default/production/_ext/101875047/big_int.o
 .debug_pubtypes
                0x000002bb       0x6d build/default/production/_ext/101875047/hashes.o
 .debug_pubtypes
                0x00000328       0x68 build/default/production/_ext/101875047/helpers.o
 .debug_pubtypes
                0x00000390       0xf4 build/default/production/_ext/1472/generic_tcp_client.o
 .debug_pubtypes
                0x00000484       0xf4 build/default/production/_ext/1472/generic_tcp_server.o
 .debug_pubtypes
                0x00000578      0x17a build/default/production/_ext/1472/ping_demo.o
 .debug_pubtypes
                0x000006f2      0x2a9 build/default/production/_ext/365611741/system_services.o
 .debug_pubtypes
                0x0000099b      0x1a8 build/default/production/_ext/365611741/system_debug.o
 .debug_pubtypes
                0x00000b43      0x14c build/default/production/_ext/365611741/system_random.o
 .debug_pubtypes
                0x00000c8f      0x1c6 build/default/production/_ext/365611741/system_command.o
 .debug_pubtypes
                0x00000e55      0x1fe build/default/production/_ext/365611741/system_userio.o
 .debug_pubtypes
                0x00001053      0x1ab build/default/production/_ext/97638081/sys_fs.o
 .debug_pubtypes
                0x000011fe      0x192 build/default/production/_ext/97638081/mpfs2.o
 .debug_pubtypes
                0x00001390      0x1a7 build/default/production/_ext/792872985/usart.o
 .debug_pubtypes
                0x00001537      0x174 build/default/production/_ext/792872985/lcd.o
 .debug_pubtypes
                0x000016ab      0x131 build/default/production/_ext/792872985/drv_spi.o
 .debug_pubtypes
                0x000017dc       0xe7 build/default/production/_ext/792872985/spi_ram.o
 .debug_pubtypes
                0x000018c3      0x17e build/default/production/_ext/792872985/spi_eeprom.o
 .debug_pubtypes
                0x00001a41       0xe7 build/default/production/_ext/792872985/spi_flash.o
 .debug_pubtypes
                0x00001b28      0x29a build/default/production/_ext/792872985/drv_media.o
 .debug_pubtypes
                0x00001dc2      0x2f6 build/default/production/_ext/427700826/tcpip_announce.o
 .debug_pubtypes
                0x000020b8      0x336 build/default/production/_ext/427700826/http2.o
 .debug_pubtypes
                0x000023ee      0x12c build/default/production/_ext/427700826/arcfour.o
 .debug_pubtypes
                0x0000251a      0x483 build/default/production/_ext/427700826/arp.o
 .debug_pubtypes
                0x0000299d      0x12c build/default/production/_ext/427700826/berkeley_api.o
 .debug_pubtypes
                0x00002ac9      0x392 build/default/production/_ext/427700826/dhcp.o
 .debug_pubtypes
                0x00002e5b      0x141 build/default/production/_ext/427700826/dhcps.o
 .debug_pubtypes
                0x00002f9c      0x312 build/default/production/_ext/427700826/dns.o
 .debug_pubtypes
                0x000032ae      0x12c build/default/production/_ext/427700826/dnss.o
 .debug_pubtypes
                0x000033da      0x12c build/default/production/_ext/427700826/dyn_dns.o
 .debug_pubtypes
                0x00003506      0x12c build/default/production/_ext/427700826/enc28_mac.o
 .debug_pubtypes
                0x00003632      0x12c build/default/production/_ext/427700826/enc28j60.o
 .debug_pubtypes
                0x0000375e      0x2ab build/default/production/_ext/427700826/encs24j600.o
 .debug_pubtypes
                0x00003a09      0x2ac build/default/production/_ext/427700826/encx24_mac.o
 .debug_pubtypes
                0x00003cb5      0x12c build/default/production/_ext/427700826/eth_pic32_ext_phy.o
 .debug_pubtypes
                0x00003de1      0x12c build/default/production/_ext/427700826/eth_pic32_ext_phy_dp83848.o
 .debug_pubtypes
                0x00003f0d      0x12c build/default/production/_ext/427700826/eth_pic32_int_mac.o
 .debug_pubtypes
                0x00004039      0x12c build/default/production/_ext/427700826/ftp.o
 .debug_pubtypes
                0x00004165       0x3a build/default/production/_ext/427700826/hash_fnv.o
 .debug_pubtypes
                0x0000419f       0xe1 build/default/production/_ext/427700826/hash_tbl.o
 .debug_pubtypes
                0x00004280      0x327 build/default/production/_ext/427700826/icmp.o
 .debug_pubtypes
                0x000045a7      0x12c build/default/production/_ext/427700826/icmpv6.o
 .debug_pubtypes
                0x000046d3      0x399 build/default/production/_ext/427700826/ipv4.o
 .debug_pubtypes
                0x00004a6c      0x12c build/default/production/_ext/427700826/ipv6.o
 .debug_pubtypes
                0x00004b98      0x12c build/default/production/_ext/427700826/mac_events_pic32.o
 .debug_pubtypes
                0x00004cc4      0x3be build/default/production/_ext/427700826/nbns.o
 .debug_pubtypes
                0x00005082      0x12c build/default/production/_ext/427700826/ndp.o
 .debug_pubtypes
                0x000051ae      0x12c build/default/production/_ext/427700826/tcpip_reboot.o
 .debug_pubtypes
                0x000052da      0x12c build/default/production/_ext/427700826/rsa.o
 .debug_pubtypes
                0x00005406      0x12c build/default/production/_ext/427700826/smtp.o
 .debug_pubtypes
                0x00005532      0x12c build/default/production/_ext/427700826/snmp.o
 .debug_pubtypes
                0x0000565e      0x12c build/default/production/_ext/427700826/snmpv3.o
 .debug_pubtypes
                0x0000578a      0x12c build/default/production/_ext/427700826/snmpv3_usm.o
 .debug_pubtypes
                0x000058b6      0x12c build/default/production/_ext/427700826/sntp.o
 .debug_pubtypes
                0x000059e2      0x12c build/default/production/_ext/427700826/ssl.o
 .debug_pubtypes
                0x00005b0e      0x468 build/default/production/_ext/427700826/tcp.o
 .debug_pubtypes
                0x00005f76      0x203 build/default/production/_ext/427700826/tcpip_heap_alloc.o
 .debug_pubtypes
                0x00006179      0x12c build/default/production/_ext/427700826/tcpip_storage.o
 .debug_pubtypes
                0x000062a5      0x12c build/default/production/_ext/427700826/telnet.o
 .debug_pubtypes
                0x000063d1      0x12c build/default/production/_ext/427700826/tftpc.o
 .debug_pubtypes
                0x000064fd      0x412 build/default/production/_ext/427700826/udp.o
 .debug_pubtypes
                0x0000690f      0x1e4 build/default/production/_ext/427700826/tcpip_mac_object.o
 .debug_pubtypes
                0x00006af3      0x508 build/default/production/_ext/427700826/tcpip_manager.o
 .debug_pubtypes
                0x00006ffb      0x262 build/default/production/_ext/427700826/tcpip_helpers.o
 .debug_pubtypes
                0x0000725d      0x12c build/default/production/_ext/427700826/tcpip_commands.o
 .debug_pubtypes
                0x00007389      0x12c build/default/production/_ext/427700826/iperf.o
 .debug_pubtypes
                0x000074b5       0x6c build/default/production/_ext/427700826/tcpip_notify.o
 .debug_pubtypes
                0x00007521      0x12c build/default/production/_ext/427700826/zero_conf_helper.o
 .debug_pubtypes
                0x0000764d      0x141 build/default/production/_ext/427700826/zero_conf_link_local.o
 .debug_pubtypes
                0x0000778e      0x12c build/default/production/_ext/427700826/zero_conf_multicast_dns.o
 .debug_pubtypes
                0x000078ba      0x12c build/default/production/_ext/334706090/wf_tx_power.o
 .debug_pubtypes
                0x000079e6      0x12c build/default/production/_ext/334706090/wf_connect.o
 .debug_pubtypes
                0x00007b12      0x12c build/default/production/_ext/334706090/wf_connection_algorithm.o
 .debug_pubtypes
                0x00007c3e      0x12c build/default/production/_ext/334706090/wf_connection_manager.o
 .debug_pubtypes
                0x00007d6a      0x12c build/default/production/_ext/334706090/wf_connection_profile.o
 .debug_pubtypes
                0x00007e96      0x12c build/default/production/_ext/334706090/wf_easy_config.o
 .debug_pubtypes
                0x00007fc2      0x12c build/default/production/_ext/334706090/wf_eint.o
 .debug_pubtypes
                0x000080ee      0x12c build/default/production/_ext/334706090/wf_event_handler.o
 .debug_pubtypes
                0x0000821a      0x12c build/default/production/_ext/334706090/wf_init.o
 .debug_pubtypes
                0x00008346      0x12c build/default/production/_ext/334706090/wf_power_save.o
 .debug_pubtypes
                0x00008472      0x12c build/default/production/_ext/334706090/wf_scan.o
 .debug_pubtypes
                0x0000859e      0x12c build/default/production/_ext/334706090/wf_spi.o
 .debug_pubtypes
                0x000086ca      0x12c build/default/production/_ext/334706090/mrf24w_mac_pic32.o
 .debug_pubtypes
                0x000087f6      0x12c build/default/production/_ext/334706090/mrf24w_events.o
 .debug_pubtypes
                0x00008922      0x12c build/default/production/_ext/334706090/wf_driver_com_24g.o
 .debug_pubtypes
                0x00008a4e      0x12c build/default/production/_ext/334706090/wf_driver_raw_24g.o
 .debug_pubtypes
                0x00008b7a      0x12c build/default/production/_ext/334706090/wf_mac_24g.o
 .debug_pubtypes
                0x00008ca6      0x12c build/default/production/_ext/334706090/wf_mgmt_msg_24g.o
 .debug_pubtypes
                0x00008dd2      0x12c build/default/production/_ext/334706090/wf_param_msg_24g.o
 .debug_pubtypes
                0x00008efe      0x2ea build/default/production/_ext/1472/main_demo.o
 .debug_pubtypes
                0x000091e8       0xe7 build/default/production/_ext/1472/mpfs_img2.o
 .debug_pubtypes
                0x000092cf       0xe7 build/default/production/_ext/1472/wf_config.o
 .debug_pubtypes
                0x000093b6      0x1e5 build/default/production/_ext/1472/custom_http_app.o
 .debug_pubtypes
                0x0000959b      0x258 build/default/production/_ext/1472/tcp6_demo_app.o
 .debug_pubtypes
                0x000097f3       0x59 c:/program files (x86)/microchip/xc32/v1.21/bin/../lib/gcc/pic32mx/4.5.2/size\libgcc.a(_udivdi3.o)
 .debug_pubtypes
                0x0000984c       0x62 c:/program files (x86)/microchip/xc32/v1.21/bin/../lib/gcc/pic32mx/4.5.2/size\libgcc.a(_lshrdi3.o)
 .debug_pubtypes
                0x000098ae       0x40 c:/program files (x86)/microchip/xc32/v1.21/bin/../lib/gcc/pic32mx/4.5.2/size\libgcc.a(_floatundisf.o)
 .debug_pubtypes
                0x000098ee       0x59 c:/program files (x86)/microchip/xc32/v1.21/bin/../lib/gcc/pic32mx/4.5.2/size\libgcc.a(_umoddi3.o)
 .debug_pubtypes
                0x00009947       0x34 c:/program files (x86)/microchip/xc32/v1.21/bin/../lib/gcc/pic32mx/4.5.2/size\libgcc.a(floatunsisf.o)

.debug_ranges   0x00000000     0x2088
 *(.debug_ranges)
 .debug_ranges  0x00000000       0x10 build/default/production/_ext/1293749816/bsp.o
 .debug_ranges  0x00000010       0x18 build/default/production/_ext/101875047/lfsr.o
 .debug_ranges  0x00000028       0x70 build/default/production/_ext/101875047/big_int.o
 .debug_ranges  0x00000098       0x50 build/default/production/_ext/101875047/hashes.o
 .debug_ranges  0x000000e8       0x48 build/default/production/_ext/101875047/helpers.o
 .debug_ranges  0x00000130       0x20 build/default/production/_ext/1472/ping_demo.o
 .debug_ranges  0x00000150      0x150 build/default/production/_ext/365611741/system_services.o
 .debug_ranges  0x000002a0       0xb8 build/default/production/_ext/365611741/system_debug.o
 .debug_ranges  0x00000358       0x30 build/default/production/_ext/365611741/system_random.o
 .debug_ranges  0x00000388       0xb0 build/default/production/_ext/365611741/system_command.o
 .debug_ranges  0x00000438       0x48 build/default/production/_ext/365611741/system_userio.o
 .debug_ranges  0x00000480      0x230 build/default/production/_ext/97638081/sys_fs.o
 .debug_ranges  0x000006b0       0xc8 build/default/production/_ext/97638081/mpfs2.o
 .debug_ranges  0x00000778       0x40 build/default/production/_ext/792872985/usart.o
 .debug_ranges  0x000007b8       0x38 build/default/production/_ext/792872985/lcd.o
 .debug_ranges  0x000007f0       0x20 build/default/production/_ext/792872985/drv_spi.o
 .debug_ranges  0x00000810       0x60 build/default/production/_ext/792872985/spi_eeprom.o
 .debug_ranges  0x00000870       0x80 build/default/production/_ext/792872985/drv_media.o
 .debug_ranges  0x000008f0       0x40 build/default/production/_ext/427700826/tcpip_announce.o
 .debug_ranges  0x00000930      0x130 build/default/production/_ext/427700826/http2.o
 .debug_ranges  0x00000a60      0x128 build/default/production/_ext/427700826/arp.o
 .debug_ranges  0x00000b88       0xa0 build/default/production/_ext/427700826/dhcp.o
 .debug_ranges  0x00000c28       0x20 build/default/production/_ext/427700826/dhcps.o
 .debug_ranges  0x00000c48       0x60 build/default/production/_ext/427700826/dns.o
 .debug_ranges  0x00000ca8      0x120 build/default/production/_ext/427700826/encs24j600.o
 .debug_ranges  0x00000dc8       0xb8 build/default/production/_ext/427700826/encx24_mac.o
 .debug_ranges  0x00000e80       0x18 build/default/production/_ext/427700826/hash_fnv.o
 .debug_ranges  0x00000e98       0x48 build/default/production/_ext/427700826/hash_tbl.o
 .debug_ranges  0x00000ee0       0x40 build/default/production/_ext/427700826/icmp.o
 .debug_ranges  0x00000f20      0x140 build/default/production/_ext/427700826/ipv4.o
 .debug_ranges  0x00001060       0x30 build/default/production/_ext/427700826/nbns.o
 .debug_ranges  0x00001090      0x290 build/default/production/_ext/427700826/tcp.o
 .debug_ranges  0x00001320       0x88 build/default/production/_ext/427700826/tcpip_heap_alloc.o
 .debug_ranges  0x000013a8      0x160 build/default/production/_ext/427700826/udp.o
 .debug_ranges  0x00001508       0xa0 build/default/production/_ext/427700826/tcpip_mac_object.o
 .debug_ranges  0x000015a8      0x260 build/default/production/_ext/427700826/tcpip_manager.o
 .debug_ranges  0x00001808       0xd8 build/default/production/_ext/427700826/tcpip_helpers.o
 .debug_ranges  0x000018e0       0x20 build/default/production/_ext/427700826/tcpip_notify.o
 .debug_ranges  0x00001900       0x20 build/default/production/_ext/427700826/zero_conf_link_local.o
 .debug_ranges  0x00001920       0x10 build/default/production/_ext/334706090/wf_eint.o
 .debug_ranges  0x00001930       0x10 build/default/production/_ext/334706090/wf_spi.o
 .debug_ranges  0x00001940       0x18 build/default/production/_ext/1472/main_demo.o
 .debug_ranges  0x00001958      0x148 build/default/production/_ext/1472/custom_http_app.o
 .debug_ranges  0x00001aa0       0x28 build/default/production/_ext/1472/tcp6_demo_app.o
 .debug_ranges  0x00001ac8       0x10 c:/program files (x86)/microchip/xc32/v1.21/bin/../lib/gcc/pic32mx/4.5.2/../../../../pic32mx/lib/size\libmchp_peripheral.a(open_core_timer_lib.o)
 .debug_ranges  0x00001ad8       0x10 c:/program files (x86)/microchip/xc32/v1.21/bin/../lib/gcc/pic32mx/4.5.2/../../../../pic32mx/lib/size\libmchp_peripheral_32MX795F512L.a(soft_reset_lib.o)
 .debug_ranges  0x00001ae8       0x18 c:/program files (x86)/microchip/xc32/v1.21/bin/../lib/gcc/pic32mx/4.5.2/../../../../pic32mx/lib/size\libmchp_peripheral_32MX795F512L.a(pcache.o)
 .debug_ranges  0x00001b00       0x10 c:/program files (x86)/microchip/xc32/v1.21/bin/../lib/gcc/pic32mx/4.5.2/../../../../pic32mx/lib/size\libmchp_peripheral_32MX795F512L.a(int_disable_interrupts_lib.o)
 .debug_ranges  0x00001b10       0x10 c:/program files (x86)/microchip/xc32/v1.21/bin/../lib/gcc/pic32mx/4.5.2/../../../../pic32mx/lib/size\libmchp_peripheral_32MX795F512L.a(int_restore_interrupts_lib.o)
 .debug_ranges  0x00001b20       0x10 c:/program files (x86)/microchip/xc32/v1.21/bin/../lib/gcc/pic32mx/4.5.2/../../../../pic32mx/lib/size\libmchp_peripheral_32MX795F512L.a(int_enable_mv_int_lib.o)
 .debug_ranges  0x00001b30       0x50 c:/program files (x86)/microchip/xc32/v1.21/bin/../lib/gcc/pic32mx/4.5.2/../../../../pic32mx/lib/size\libmchp_peripheral_32MX795F512L.a(int_tbl_lib.o)
 .debug_ranges  0x00001b80       0x10 c:/program files (x86)/microchip/xc32/v1.21/bin/../lib/gcc/pic32mx/4.5.2/../../../../pic32mx/lib/size\libmchp_peripheral_32MX795F512L.a(rtcc_init_lib.o)
 .debug_ranges  0x00001b90       0x10 c:/program files (x86)/microchip/xc32/v1.21/bin/../lib/gcc/pic32mx/4.5.2/../../../../pic32mx/lib/size\libmchp_peripheral_32MX795F512L.a(rtcc_open_lib.o)
 .debug_ranges  0x00001ba0       0x10 c:/program files (x86)/microchip/xc32/v1.21/bin/../lib/gcc/pic32mx/4.5.2/../../../../pic32mx/lib/size\libmchp_peripheral_32MX795F512L.a(spi_chn_data_rdy_lib.o)
 .debug_ranges  0x00001bb0       0x18 c:/program files (x86)/microchip/xc32/v1.21/bin/../lib/gcc/pic32mx/4.5.2/../../../../pic32mx/lib/size\libmchp_peripheral_32MX795F512L.a(spi_chn_getc_lib.o)
 .debug_ranges  0x00001bc8       0x10 c:/program files (x86)/microchip/xc32/v1.21/bin/../lib/gcc/pic32mx/4.5.2/../../../../pic32mx/lib/size\libmchp_peripheral_32MX795F512L.a(spi_chn_open_lib.o)
 .debug_ranges  0x00001bd8       0x20 c:/program files (x86)/microchip/xc32/v1.21/bin/../lib/gcc/pic32mx/4.5.2/../../../../pic32mx/lib/size\libmchp_peripheral_32MX795F512L.a(spi_chn_putc_lib.o)
 .debug_ranges  0x00001bf8       0x10 c:/program files (x86)/microchip/xc32/v1.21/bin/../lib/gcc/pic32mx/4.5.2/../../../../pic32mx/lib/size\libmchp_peripheral_32MX795F512L.a(spi_chn_tx_buff_empty_lib.o)
 .debug_ranges  0x00001c08       0x10 c:/program files (x86)/microchip/xc32/v1.21/bin/../lib/gcc/pic32mx/4.5.2/../../../../pic32mx/lib/size\libmchp_peripheral_32MX795F512L.a(port_set_pins_digital_in_lib.o)
 .debug_ranges  0x00001c18       0x10 c:/program files (x86)/microchip/xc32/v1.21/bin/../lib/gcc/pic32mx/4.5.2/../../../../pic32mx/lib/size\libmchp_peripheral_32MX795F512L.a(port_set_pins_digital_out_lib.o)
 .debug_ranges  0x00001c28       0x10 c:/program files (x86)/microchip/xc32/v1.21/bin/../lib/gcc/pic32mx/4.5.2/../../../../pic32mx/lib/size\libmchp_peripheral_32MX795F512L.a(int_enable_interrupts_lib.o)
 .debug_ranges  0x00001c38       0x18 c:/program files (x86)/microchip/xc32/v1.21/bin/../lib/gcc/pic32mx/4.5.2/../../../../pic32mx/lib/size\libmchp_peripheral_32MX795F512L.a(_rtcc_wait_clock_off_lib.o)
 .debug_ranges  0x00001c50       0x10 c:/program files (x86)/microchip/xc32/v1.21/bin/../lib/gcc/pic32mx/4.5.2/../../../../pic32mx/lib/size\libmchp_peripheral_32MX795F512L.a(read_core_timer_lib.o)
 .debug_ranges  0x00001c60       0xc0 c:/program files (x86)/microchip/xc32/v1.21/bin/../lib/gcc/pic32mx/4.5.2/size\libgcc.a(_udivdi3.o)
 .debug_ranges  0x00001d20       0x10 c:/program files (x86)/microchip/xc32/v1.21/bin/../lib/gcc/pic32mx/4.5.2/../../../../pic32mx/lib/size\libpic32.a(default-bootstrap-exception-handler.o)
 .debug_ranges  0x00001d30       0x10 c:/program files (x86)/microchip/xc32/v1.21/bin/../lib/gcc/pic32mx/4.5.2/../../../../pic32mx/lib/size\libpic32.a(default-on-reset.o)
 .debug_ranges  0x00001d40       0x10 c:/program files (x86)/microchip/xc32/v1.21/bin/../lib/gcc/pic32mx/4.5.2/../../../../pic32mx/lib/size\libpic32.a(default-on-bootstrap.o)
 .debug_ranges  0x00001d50       0x10 c:/program files (x86)/microchip/xc32/v1.21/bin/../lib/gcc/pic32mx/4.5.2/../../../../pic32mx/lib/size\libpic32.a(defaultinterrupt.o)
 .debug_ranges  0x00001d60       0x10 c:/program files (x86)/microchip/xc32/v1.21/bin/../lib/gcc/pic32mx/4.5.2/../../../../pic32mx/lib/size\libc.a(atoi.o)
 .debug_ranges  0x00001d70       0x10 c:/program files (x86)/microchip/xc32/v1.21/bin/../lib/gcc/pic32mx/4.5.2/../../../../pic32mx/lib/size\libc.a(atol.o)
 .debug_ranges  0x00001d80       0x20 c:/program files (x86)/microchip/xc32/v1.21/bin/../lib/gcc/pic32mx/4.5.2/../../../../pic32mx/lib/size\libc.a(malloc.o)
 .debug_ranges  0x00001da0       0x18 c:/program files (x86)/microchip/xc32/v1.21/bin/../lib/gcc/pic32mx/4.5.2/../../../../pic32mx/lib/size\libc.a(rand.o)
 .debug_ranges  0x00001db8       0x10 c:/program files (x86)/microchip/xc32/v1.21/bin/../lib/gcc/pic32mx/4.5.2/../../../../pic32mx/lib/size\libc.a(strcat.o)
 .debug_ranges  0x00001dc8       0x10 c:/program files (x86)/microchip/xc32/v1.21/bin/../lib/gcc/pic32mx/4.5.2/../../../../pic32mx/lib/size\libc.a(strchr.o)
 .debug_ranges  0x00001dd8       0x10 c:/program files (x86)/microchip/xc32/v1.21/bin/../lib/gcc/pic32mx/4.5.2/../../../../pic32mx/lib/size\libc.a(strncat.o)
 .debug_ranges  0x00001de8       0x10 c:/program files (x86)/microchip/xc32/v1.21/bin/../lib/gcc/pic32mx/4.5.2/../../../../pic32mx/lib/size\libc.a(strncmp.o)
 .debug_ranges  0x00001df8       0x10 c:/program files (x86)/microchip/xc32/v1.21/bin/../lib/gcc/pic32mx/4.5.2/../../../../pic32mx/lib/size\libc.a(strncpy.o)
 .debug_ranges  0x00001e08       0x10 c:/program files (x86)/microchip/xc32/v1.21/bin/../lib/gcc/pic32mx/4.5.2/../../../../pic32mx/lib/size\libc.a(strrchr.o)
 .debug_ranges  0x00001e18       0x10 c:/program files (x86)/microchip/xc32/v1.21/bin/../lib/gcc/pic32mx/4.5.2/../../../../pic32mx/lib/size\libc.a(strstr.o)
 .debug_ranges  0x00001e28       0x18 c:/program files (x86)/microchip/xc32/v1.21/bin/../lib/gcc/pic32mx/4.5.2/../../../../pic32mx/lib/size\libc.a(strtol.o)
 .debug_ranges  0x00001e40       0x10 c:/program files (x86)/microchip/xc32/v1.21/bin/../lib/gcc/pic32mx/4.5.2/../../../../pic32mx/lib/size\libc.a(snprintf_cdnopsuxX.eo)
 .debug_ranges  0x00001e50       0x10 c:/program files (x86)/microchip/xc32/v1.21/bin/../lib/gcc/pic32mx/4.5.2/../../../../pic32mx/lib/size\libc.a(sprintf_cdnopsuxX.eo)
 .debug_ranges  0x00001e60       0x10 c:/program files (x86)/microchip/xc32/v1.21/bin/../lib/gcc/pic32mx/4.5.2/../../../../pic32mx/lib/size\libc.a(vsnprintf_cdnopsuxX.eo)
 .debug_ranges  0x00001e70       0x10 c:/program files (x86)/microchip/xc32/v1.21/bin/../lib/gcc/pic32mx/4.5.2/../../../../pic32mx/lib/size\libc.a(vsnprintf.o)
 .debug_ranges  0x00001e80       0x90 c:/program files (x86)/microchip/xc32/v1.21/bin/../lib/gcc/pic32mx/4.5.2/../../../../pic32mx/lib/size\libc.a(ctypef.o)
 .debug_ranges  0x00001f10       0x10 c:/program files (x86)/microchip/xc32/v1.21/bin/../lib/gcc/pic32mx/4.5.2/../../../../pic32mx/lib/size\libc.a(doprnt_cdnopsuxX.eo)
 .debug_ranges  0x00001f20       0x20 c:/program files (x86)/microchip/xc32/v1.21/bin/../lib/gcc/pic32mx/4.5.2/../../../../pic32mx/lib/size\libc.a(doprnt.o)
 .debug_ranges  0x00001f40       0x10 c:/program files (x86)/microchip/xc32/v1.21/bin/../lib/gcc/pic32mx/4.5.2/../../../../pic32mx/lib/size\libc.a(_fputc_simple.o)
 .debug_ranges  0x00001f50       0x10 c:/program files (x86)/microchip/xc32/v1.21/bin/../lib/gcc/pic32mx/4.5.2/../../../../pic32mx/lib/size\libc.a(_flsbuf_simple.o)
 .debug_ranges  0x00001f60       0x30 c:/program files (x86)/microchip/xc32/v1.21/bin/../lib/gcc/pic32mx/4.5.2/../../../../pic32mx/lib/size\libpic32.a(sbrk.o)
 .debug_ranges  0x00001f90       0x10 c:/program files (x86)/microchip/xc32/v1.21/bin/../lib/gcc/pic32mx/4.5.2/../../../../pic32mx/lib/size\libpic32.a(write.o)
 .debug_ranges  0x00001fa0       0x10 c:/program files (x86)/microchip/xc32/v1.21/bin/../lib/gcc/pic32mx/4.5.2/../../../../pic32mx/lib/size\libpic32.a(_mon_putc.o)
 .debug_ranges  0x00001fb0       0x10 c:/program files (x86)/microchip/xc32/v1.21/bin/../lib/gcc/pic32mx/4.5.2/../../../../pic32mx/lib/size\libe.a(_floatdisf.o)
 .debug_ranges  0x00001fc0       0xc8 c:/program files (x86)/microchip/xc32/v1.21/bin/../lib/gcc/pic32mx/4.5.2/size\libgcc.a(_umoddi3.o)

.gnu.attributes
                0x00000000       0x10
 *(.gnu.attributes)
 .gnu.attributes
                0x00000000       0x10 build/default/production/_ext/1293749816/bsp.o
 .gnu.attributes
                0x00000010       0x10 build/default/production/_ext/101875047/lfsr.o
 .gnu.attributes
                0x00000020       0x10 build/default/production/_ext/101875047/big_int.o
 .gnu.attributes
                0x00000030       0x10 build/default/production/_ext/101875047/hashes.o
 .gnu.attributes
                0x00000040       0x10 build/default/production/_ext/101875047/helpers.o
 .gnu.attributes
                0x00000050       0x10 build/default/production/_ext/1472/berkeley_tcp_client_demo.o
 .gnu.attributes
                0x00000060       0x10 build/default/production/_ext/1472/berkeley_tcp_server_demo.o
 .gnu.attributes
                0x00000070       0x10 build/default/production/_ext/1472/berkeley_udp_client_demo.o
 .gnu.attributes
                0x00000080       0x10 build/default/production/_ext/1472/generic_tcp_client.o
 .gnu.attributes
                0x00000090       0x10 build/default/production/_ext/1472/generic_tcp_server.o
 .gnu.attributes
                0x000000a0       0x10 build/default/production/_ext/1472/ping_demo.o
 .gnu.attributes
                0x000000b0       0x10 build/default/production/_ext/1472/smtp_demo.o
 .gnu.attributes
                0x000000c0       0x10 build/default/production/_ext/365611741/system_services.o
 .gnu.attributes
                0x000000d0       0x10 build/default/production/_ext/365611741/system_debug.o
 .gnu.attributes
                0x000000e0       0x10 build/default/production/_ext/365611741/system_random.o
 .gnu.attributes
                0x000000f0       0x10 build/default/production/_ext/365611741/system_command.o
 .gnu.attributes
                0x00000100       0x10 build/default/production/_ext/365611741/system_userio.o
 .gnu.attributes
                0x00000110       0x10 build/default/production/_ext/97638081/sys_fs.o
 .gnu.attributes
                0x00000120       0x10 build/default/production/_ext/97638081/mpfs2.o
 .gnu.attributes
                0x00000130       0x10 build/default/production/_ext/792872985/usart.o
 .gnu.attributes
                0x00000140       0x10 build/default/production/_ext/792872985/lcd.o
 .gnu.attributes
                0x00000150       0x10 build/default/production/_ext/792872985/drv_spi.o
 .gnu.attributes
                0x00000160       0x10 build/default/production/_ext/792872985/db_appio.o
 .gnu.attributes
                0x00000170       0x10 build/default/production/_ext/792872985/spi_ram.o
 .gnu.attributes
                0x00000180       0x10 build/default/production/_ext/792872985/spi_eeprom.o
 .gnu.attributes
                0x00000190       0x10 build/default/production/_ext/792872985/spi_flash.o
 .gnu.attributes
                0x000001a0       0x10 build/default/production/_ext/792872985/drv_media.o
 .gnu.attributes
                0x000001b0       0x10 build/default/production/_ext/427700826/tcpip_announce.o
 .gnu.attributes
                0x000001c0       0x10 build/default/production/_ext/427700826/http2.o
 .gnu.attributes
                0x000001d0       0x10 build/default/production/_ext/427700826/arcfour.o
 .gnu.attributes
                0x000001e0       0x10 build/default/production/_ext/427700826/arp.o
 .gnu.attributes
                0x000001f0       0x10 build/default/production/_ext/427700826/berkeley_api.o
 .gnu.attributes
                0x00000200       0x10 build/default/production/_ext/427700826/dhcp.o
 .gnu.attributes
                0x00000210       0x10 build/default/production/_ext/427700826/dhcps.o
 .gnu.attributes
                0x00000220       0x10 build/default/production/_ext/427700826/dns.o
 .gnu.attributes
                0x00000230       0x10 build/default/production/_ext/427700826/dnss.o
 .gnu.attributes
                0x00000240       0x10 build/default/production/_ext/427700826/dyn_dns.o
 .gnu.attributes
                0x00000250       0x10 build/default/production/_ext/427700826/enc28_mac.o
 .gnu.attributes
                0x00000260       0x10 build/default/production/_ext/427700826/enc28j60.o
 .gnu.attributes
                0x00000270       0x10 build/default/production/_ext/427700826/encs24j600.o
 .gnu.attributes
                0x00000280       0x10 build/default/production/_ext/427700826/encx24_mac.o
 .gnu.attributes
                0x00000290       0x10 build/default/production/_ext/427700826/eth_pic32_ext_phy.o
 .gnu.attributes
                0x000002a0       0x10 build/default/production/_ext/427700826/eth_pic32_ext_phy_dp83848.o
 .gnu.attributes
                0x000002b0       0x10 build/default/production/_ext/427700826/eth_pic32_int_mac.o
 .gnu.attributes
                0x000002c0       0x10 build/default/production/_ext/427700826/ftp.o
 .gnu.attributes
                0x000002d0       0x10 build/default/production/_ext/427700826/hash_fnv.o
 .gnu.attributes
                0x000002e0       0x10 build/default/production/_ext/427700826/hash_tbl.o
 .gnu.attributes
                0x000002f0       0x10 build/default/production/_ext/427700826/icmp.o
 .gnu.attributes
                0x00000300       0x10 build/default/production/_ext/427700826/icmpv6.o
 .gnu.attributes
                0x00000310       0x10 build/default/production/_ext/427700826/ipv4.o
 .gnu.attributes
                0x00000320       0x10 build/default/production/_ext/427700826/ipv6.o
 .gnu.attributes
                0x00000330       0x10 build/default/production/_ext/427700826/mac_events_pic32.o
 .gnu.attributes
                0x00000340       0x10 build/default/production/_ext/427700826/nbns.o
 .gnu.attributes
                0x00000350       0x10 build/default/production/_ext/427700826/ndp.o
 .gnu.attributes
                0x00000360       0x10 build/default/production/_ext/427700826/tcpip_reboot.o
 .gnu.attributes
                0x00000370       0x10 build/default/production/_ext/427700826/rsa.o
 .gnu.attributes
                0x00000380       0x10 build/default/production/_ext/427700826/smtp.o
 .gnu.attributes
                0x00000390       0x10 build/default/production/_ext/427700826/snmp.o
 .gnu.attributes
                0x000003a0       0x10 build/default/production/_ext/427700826/snmpv3.o
 .gnu.attributes
                0x000003b0       0x10 build/default/production/_ext/427700826/snmpv3_usm.o
 .gnu.attributes
                0x000003c0       0x10 build/default/production/_ext/427700826/sntp.o
 .gnu.attributes
                0x000003d0       0x10 build/default/production/_ext/427700826/ssl.o
 .gnu.attributes
                0x000003e0       0x10 build/default/production/_ext/427700826/tcp.o
 .gnu.attributes
                0x000003f0       0x10 build/default/production/_ext/427700826/tcpip_heap_alloc.o
 .gnu.attributes
                0x00000400       0x10 build/default/production/_ext/427700826/tcpip_storage.o
 .gnu.attributes
                0x00000410       0x10 build/default/production/_ext/427700826/telnet.o
 .gnu.attributes
                0x00000420       0x10 build/default/production/_ext/427700826/tftpc.o
 .gnu.attributes
                0x00000430       0x10 build/default/production/_ext/427700826/udp.o
 .gnu.attributes
                0x00000440       0x10 build/default/production/_ext/427700826/tcpip_mac_object.o
 .gnu.attributes
                0x00000450       0x10 build/default/production/_ext/427700826/tcpip_manager.o
 .gnu.attributes
                0x00000460       0x10 build/default/production/_ext/427700826/tcpip_helpers.o
 .gnu.attributes
                0x00000470       0x10 build/default/production/_ext/427700826/tcpip_commands.o
 .gnu.attributes
                0x00000480       0x10 build/default/production/_ext/427700826/iperf.o
 .gnu.attributes
                0x00000490       0x10 build/default/production/_ext/427700826/tcpip_notify.o
 .gnu.attributes
                0x000004a0       0x10 build/default/production/_ext/427700826/zero_conf_helper.o
 .gnu.attributes
                0x000004b0       0x10 build/default/production/_ext/427700826/zero_conf_link_local.o
 .gnu.attributes
                0x000004c0       0x10 build/default/production/_ext/427700826/zero_conf_multicast_dns.o
 .gnu.attributes
                0x000004d0       0x10 build/default/production/_ext/334706090/wf_tx_power.o
 .gnu.attributes
                0x000004e0       0x10 build/default/production/_ext/334706090/wf_connect.o
 .gnu.attributes
                0x000004f0       0x10 build/default/production/_ext/334706090/wf_connection_algorithm.o
 .gnu.attributes
                0x00000500       0x10 build/default/production/_ext/334706090/wf_connection_manager.o
 .gnu.attributes
                0x00000510       0x10 build/default/production/_ext/334706090/wf_connection_profile.o
 .gnu.attributes
                0x00000520       0x10 build/default/production/_ext/334706090/wf_easy_config.o
 .gnu.attributes
                0x00000530       0x10 build/default/production/_ext/334706090/wf_eint.o
 .gnu.attributes
                0x00000540       0x10 build/default/production/_ext/334706090/wf_event_handler.o
 .gnu.attributes
                0x00000550       0x10 build/default/production/_ext/334706090/wf_init.o
 .gnu.attributes
                0x00000560       0x10 build/default/production/_ext/334706090/wf_power_save.o
 .gnu.attributes
                0x00000570       0x10 build/default/production/_ext/334706090/wf_scan.o
 .gnu.attributes
                0x00000580       0x10 build/default/production/_ext/334706090/wf_spi.o
 .gnu.attributes
                0x00000590       0x10 build/default/production/_ext/334706090/mrf24w_mac_pic32.o
 .gnu.attributes
                0x000005a0       0x10 build/default/production/_ext/334706090/mrf24w_events.o
 .gnu.attributes
                0x000005b0       0x10 build/default/production/_ext/334706090/wf_driver_com_24g.o
 .gnu.attributes
                0x000005c0       0x10 build/default/production/_ext/334706090/wf_driver_raw_24g.o
 .gnu.attributes
                0x000005d0       0x10 build/default/production/_ext/334706090/wf_mac_24g.o
 .gnu.attributes
                0x000005e0       0x10 build/default/production/_ext/334706090/wf_mgmt_msg_24g.o
 .gnu.attributes
                0x000005f0       0x10 build/default/production/_ext/334706090/wf_param_msg_24g.o
 .gnu.attributes
                0x00000600       0x10 build/default/production/_ext/1472/main_demo.o
 .gnu.attributes
                0x00000610       0x10 build/default/production/_ext/1472/custom_snmp_app.o
 .gnu.attributes
                0x00000620       0x10 build/default/production/_ext/1472/custom_ssl_cert.o
 .gnu.attributes
                0x00000630       0x10 build/default/production/_ext/1472/mpfs_img2.o
 .gnu.attributes
                0x00000640       0x10 build/default/production/_ext/1472/wf_config.o
 .gnu.attributes
                0x00000650       0x10 build/default/production/_ext/1472/custom_http_app.o
 .gnu.attributes
                0x00000660       0x10 build/default/production/_ext/1472/tcp6_demo_app.o
 .gnu.attributes
                0x00000670       0x10 c:/program files (x86)/microchip/xc32/v1.21/bin/../lib/gcc/pic32mx/4.5.2/../../../../pic32mx/lib/size\libmchp_peripheral.a(open_core_timer_lib.o)
 .gnu.attributes
                0x00000680       0x10 c:/program files (x86)/microchip/xc32/v1.21/bin/../lib/gcc/pic32mx/4.5.2/../../../../pic32mx/lib/size\libmchp_peripheral_32MX795F512L.a(soft_reset_lib.o)
 .gnu.attributes
                0x00000690       0x10 c:/program files (x86)/microchip/xc32/v1.21/bin/../lib/gcc/pic32mx/4.5.2/../../../../pic32mx/lib/size\libmchp_peripheral_32MX795F512L.a(pcache.o)
 .gnu.attributes
                0x000006a0       0x10 c:/program files (x86)/microchip/xc32/v1.21/bin/../lib/gcc/pic32mx/4.5.2/../../../../pic32mx/lib/size\libmchp_peripheral_32MX795F512L.a(int_disable_interrupts_lib.o)
 .gnu.attributes
                0x000006b0       0x10 c:/program files (x86)/microchip/xc32/v1.21/bin/../lib/gcc/pic32mx/4.5.2/../../../../pic32mx/lib/size\libmchp_peripheral_32MX795F512L.a(int_restore_interrupts_lib.o)
 .gnu.attributes
                0x000006c0       0x10 c:/program files (x86)/microchip/xc32/v1.21/bin/../lib/gcc/pic32mx/4.5.2/../../../../pic32mx/lib/size\libmchp_peripheral_32MX795F512L.a(int_enable_mv_int_lib.o)
 .gnu.attributes
                0x000006d0       0x10 c:/program files (x86)/microchip/xc32/v1.21/bin/../lib/gcc/pic32mx/4.5.2/../../../../pic32mx/lib/size\libmchp_peripheral_32MX795F512L.a(int_tbl_lib.o)
 .gnu.attributes
                0x000006e0       0x10 c:/program files (x86)/microchip/xc32/v1.21/bin/../lib/gcc/pic32mx/4.5.2/../../../../pic32mx/lib/size\libmchp_peripheral_32MX795F512L.a(rtcc_init_lib.o)
 .gnu.attributes
                0x000006f0       0x10 c:/program files (x86)/microchip/xc32/v1.21/bin/../lib/gcc/pic32mx/4.5.2/../../../../pic32mx/lib/size\libmchp_peripheral_32MX795F512L.a(rtcc_open_lib.o)
 .gnu.attributes
                0x00000700       0x10 c:/program files (x86)/microchip/xc32/v1.21/bin/../lib/gcc/pic32mx/4.5.2/../../../../pic32mx/lib/size\libmchp_peripheral_32MX795F512L.a(spi_chn_data_rdy_lib.o)
 .gnu.attributes
                0x00000710       0x10 c:/program files (x86)/microchip/xc32/v1.21/bin/../lib/gcc/pic32mx/4.5.2/../../../../pic32mx/lib/size\libmchp_peripheral_32MX795F512L.a(spi_chn_getc_lib.o)
 .gnu.attributes
                0x00000720       0x10 c:/program files (x86)/microchip/xc32/v1.21/bin/../lib/gcc/pic32mx/4.5.2/../../../../pic32mx/lib/size\libmchp_peripheral_32MX795F512L.a(spi_chn_open_lib.o)
 .gnu.attributes
                0x00000730       0x10 c:/program files (x86)/microchip/xc32/v1.21/bin/../lib/gcc/pic32mx/4.5.2/../../../../pic32mx/lib/size\libmchp_peripheral_32MX795F512L.a(spi_chn_putc_lib.o)
 .gnu.attributes
                0x00000740       0x10 c:/program files (x86)/microchip/xc32/v1.21/bin/../lib/gcc/pic32mx/4.5.2/../../../../pic32mx/lib/size\libmchp_peripheral_32MX795F512L.a(spi_chn_tx_buff_empty_lib.o)
 .gnu.attributes
                0x00000750       0x10 c:/program files (x86)/microchip/xc32/v1.21/bin/../lib/gcc/pic32mx/4.5.2/../../../../pic32mx/lib/size\libmchp_peripheral_32MX795F512L.a(spi_io_tbl_libp.o)
 .gnu.attributes
                0x00000760       0x10 c:/program files (x86)/microchip/xc32/v1.21/bin/../lib/gcc/pic32mx/4.5.2/../../../../pic32mx/lib/size\libmchp_peripheral_32MX795F512L.a(spi_map_tbl_libp.o)
 .gnu.attributes
                0x00000770       0x10 c:/program files (x86)/microchip/xc32/v1.21/bin/../lib/gcc/pic32mx/4.5.2/../../../../pic32mx/lib/size\libmchp_peripheral_32MX795F512L.a(port_set_pins_digital_in_lib.o)
 .gnu.attributes
                0x00000780       0x10 c:/program files (x86)/microchip/xc32/v1.21/bin/../lib/gcc/pic32mx/4.5.2/../../../../pic32mx/lib/size\libmchp_peripheral_32MX795F512L.a(port_set_pins_digital_out_lib.o)
 .gnu.attributes
                0x00000790       0x10 c:/program files (x86)/microchip/xc32/v1.21/bin/../lib/gcc/pic32mx/4.5.2/../../../../pic32mx/lib/size\libmchp_peripheral_32MX795F512L.a(_ports_tbl_libp.o)
 .gnu.attributes
                0x000007a0       0x10 c:/program files (x86)/microchip/xc32/v1.21/bin/../lib/gcc/pic32mx/4.5.2/../../../../pic32mx/lib/size\libmchp_peripheral_32MX795F512L.a(int_enable_interrupts_lib.o)
 .gnu.attributes
                0x000007b0       0x10 c:/program files (x86)/microchip/xc32/v1.21/bin/../lib/gcc/pic32mx/4.5.2/../../../../pic32mx/lib/size\libmchp_peripheral_32MX795F512L.a(_rtcc_wait_clock_off_lib.o)
 .gnu.attributes
                0x000007c0       0x10 c:/program files (x86)/microchip/xc32/v1.21/bin/../lib/gcc/pic32mx/4.5.2/../../../../pic32mx/lib/size\libmchp_peripheral_32MX795F512L.a(read_core_timer_lib.o)
 .gnu.attributes
                0x000007d0       0x10 c:/program files (x86)/microchip/xc32/v1.21/bin/../lib/gcc/pic32mx/4.5.2/size\libgcc.a(_udivdi3.o)
 .gnu.attributes
                0x000007e0       0x10 c:/program files (x86)/microchip/xc32/v1.21/bin/../lib/gcc/pic32mx/4.5.2/../../../../pic32mx/lib/size\libpic32.a(default-bootstrap-exception-handler.o)
 .gnu.attributes
                0x000007f0       0x10 c:/program files (x86)/microchip/xc32/v1.21/bin/../lib/gcc/pic32mx/4.5.2/../../../../pic32mx/lib/size\libpic32.a(default-on-reset.o)
 .gnu.attributes
                0x00000800       0x10 c:/program files (x86)/microchip/xc32/v1.21/bin/../lib/gcc/pic32mx/4.5.2/../../../../pic32mx/lib/size\libpic32.a(default-on-bootstrap.o)
 .gnu.attributes
                0x00000810       0x10 c:/program files (x86)/microchip/xc32/v1.21/bin/../lib/gcc/pic32mx/4.5.2/../../../../pic32mx/lib/size\libpic32.a(errno.o)
 .gnu.attributes
                0x00000820       0x10 c:/program files (x86)/microchip/xc32/v1.21/bin/../lib/gcc/pic32mx/4.5.2/../../../../pic32mx/lib/size\libpic32.a(defaultinterrupt.o)
 .gnu.attributes
                0x00000830       0x10 c:/program files (x86)/microchip/xc32/v1.21/bin/../lib/gcc/pic32mx/4.5.2/../../../../pic32mx/lib/size\libc.a(atoi.o)
 .gnu.attributes
                0x00000840       0x10 c:/program files (x86)/microchip/xc32/v1.21/bin/../lib/gcc/pic32mx/4.5.2/../../../../pic32mx/lib/size\libc.a(atol.o)
 .gnu.attributes
                0x00000850       0x10 c:/program files (x86)/microchip/xc32/v1.21/bin/../lib/gcc/pic32mx/4.5.2/../../../../pic32mx/lib/size\libc.a(ctype.o)
 .gnu.attributes
                0x00000860       0x10 c:/program files (x86)/microchip/xc32/v1.21/bin/../lib/gcc/pic32mx/4.5.2/../../../../pic32mx/lib/size\libc.a(malloc.o)
 .gnu.attributes
                0x00000870       0x10 c:/program files (x86)/microchip/xc32/v1.21/bin/../lib/gcc/pic32mx/4.5.2/../../../../pic32mx/lib/size\libc.a(rand.o)
 .gnu.attributes
                0x00000880       0x10 c:/program files (x86)/microchip/xc32/v1.21/bin/../lib/gcc/pic32mx/4.5.2/../../../../pic32mx/lib/size\libc.a(strcat.o)
 .gnu.attributes
                0x00000890       0x10 c:/program files (x86)/microchip/xc32/v1.21/bin/../lib/gcc/pic32mx/4.5.2/../../../../pic32mx/lib/size\libc.a(strchr.o)
 .gnu.attributes
                0x000008a0       0x10 c:/program files (x86)/microchip/xc32/v1.21/bin/../lib/gcc/pic32mx/4.5.2/../../../../pic32mx/lib/size\libc.a(strncat.o)
 .gnu.attributes
                0x000008b0       0x10 c:/program files (x86)/microchip/xc32/v1.21/bin/../lib/gcc/pic32mx/4.5.2/../../../../pic32mx/lib/size\libc.a(strncmp.o)
 .gnu.attributes
                0x000008c0       0x10 c:/program files (x86)/microchip/xc32/v1.21/bin/../lib/gcc/pic32mx/4.5.2/../../../../pic32mx/lib/size\libc.a(strncpy.o)
 .gnu.attributes
                0x000008d0       0x10 c:/program files (x86)/microchip/xc32/v1.21/bin/../lib/gcc/pic32mx/4.5.2/../../../../pic32mx/lib/size\libc.a(strrchr.o)
 .gnu.attributes
                0x000008e0       0x10 c:/program files (x86)/microchip/xc32/v1.21/bin/../lib/gcc/pic32mx/4.5.2/../../../../pic32mx/lib/size\libc.a(strstr.o)
 .gnu.attributes
                0x000008f0       0x10 c:/program files (x86)/microchip/xc32/v1.21/bin/../lib/gcc/pic32mx/4.5.2/../../../../pic32mx/lib/size\libc.a(strtol.o)
 .gnu.attributes
                0x00000900       0x10 c:/program files (x86)/microchip/xc32/v1.21/bin/../lib/gcc/pic32mx/4.5.2/../../../../pic32mx/lib/size\libc.a(snprintf_cdnopsuxX.eo)
 .gnu.attributes
                0x00000910       0x10 c:/program files (x86)/microchip/xc32/v1.21/bin/../lib/gcc/pic32mx/4.5.2/../../../../pic32mx/lib/size\libc.a(sprintf_cdnopsuxX.eo)
 .gnu.attributes
                0x00000920       0x10 c:/program files (x86)/microchip/xc32/v1.21/bin/../lib/gcc/pic32mx/4.5.2/../../../../pic32mx/lib/size\libc.a(vsnprintf_cdnopsuxX.eo)
 .gnu.attributes
                0x00000930       0x10 c:/program files (x86)/microchip/xc32/v1.21/bin/../lib/gcc/pic32mx/4.5.2/../../../../pic32mx/lib/size\libc.a(vsnprintf.o)
 .gnu.attributes
                0x00000940       0x10 c:/program files (x86)/microchip/xc32/v1.21/bin/../lib/gcc/pic32mx/4.5.2/../../../../pic32mx/lib/size\libc.a(ctypef.o)
 .gnu.attributes
                0x00000950       0x10 c:/program files (x86)/microchip/xc32/v1.21/bin/../lib/gcc/pic32mx/4.5.2/../../../../pic32mx/lib/size\libc.a(doprnt_cdnopsuxX.eo)
 .gnu.attributes
                0x00000960       0x10 c:/program files (x86)/microchip/xc32/v1.21/bin/../lib/gcc/pic32mx/4.5.2/../../../../pic32mx/lib/size\libc.a(doprnt.o)
 .gnu.attributes
                0x00000970       0x10 c:/program files (x86)/microchip/xc32/v1.21/bin/../lib/gcc/pic32mx/4.5.2/../../../../pic32mx/lib/size\libc.a(_fputc_simple.o)
 .gnu.attributes
                0x00000980       0x10 c:/program files (x86)/microchip/xc32/v1.21/bin/../lib/gcc/pic32mx/4.5.2/../../../../pic32mx/lib/size\libc.a(powersf.o)
 .gnu.attributes
                0x00000990       0x10 c:/program files (x86)/microchip/xc32/v1.21/bin/../lib/gcc/pic32mx/4.5.2/../../../../pic32mx/lib/size\libc.a(_iob.o)
 .gnu.attributes
                0x000009a0       0x10 c:/program files (x86)/microchip/xc32/v1.21/bin/../lib/gcc/pic32mx/4.5.2/../../../../pic32mx/lib/size\libc.a(_flsbuf_simple.o)
 .gnu.attributes
                0x000009b0       0x10 c:/program files (x86)/microchip/xc32/v1.21/bin/../lib/gcc/pic32mx/4.5.2/../../../../pic32mx/lib/size\libpic32.a(sbrk.o)
 .gnu.attributes
                0x000009c0       0x10 c:/program files (x86)/microchip/xc32/v1.21/bin/../lib/gcc/pic32mx/4.5.2/../../../../pic32mx/lib/size\libpic32.a(write.o)
 .gnu.attributes
                0x000009d0       0x10 c:/program files (x86)/microchip/xc32/v1.21/bin/../lib/gcc/pic32mx/4.5.2/../../../../pic32mx/lib/size\libpic32.a(_mon_putc.o)
 .gnu.attributes
                0x000009e0       0x10 c:/program files (x86)/microchip/xc32/v1.21/bin/../lib/gcc/pic32mx/4.5.2/../../../../pic32mx/lib/size\libpic32.a(xc32_uart.o)
 .gnu.attributes
                0x000009f0       0x10 c:/program files (x86)/microchip/xc32/v1.21/bin/../lib/gcc/pic32mx/4.5.2/../../../../pic32mx/lib/size\libe.a(_floatdisf.o)
 .gnu.attributes
                0x00000a00       0x10 c:/program files (x86)/microchip/xc32/v1.21/bin/../lib/gcc/pic32mx/4.5.2/size\libgcc.a(_lshrdi3.o)
 .gnu.attributes
                0x00000a10       0x10 c:/program files (x86)/microchip/xc32/v1.21/bin/../lib/gcc/pic32mx/4.5.2/size\libgcc.a(_floatundisf.o)
 .gnu.attributes
                0x00000a20       0x10 c:/program files (x86)/microchip/xc32/v1.21/bin/../lib/gcc/pic32mx/4.5.2/size\libgcc.a(_umoddi3.o)
 .gnu.attributes
                0x00000a30       0x10 c:/program files (x86)/microchip/xc32/v1.21/bin/../lib/gcc/pic32mx/4.5.2/size\libgcc.a(floatunsisf.o)
LOAD c:/program files (x86)/microchip/xc32/v1.21/bin/../lib/gcc/pic32mx/4.5.2/size\libgcc.a
START GROUP
LOAD c:/program files (x86)/microchip/xc32/v1.21/bin/../lib/gcc/pic32mx/4.5.2/../../../../pic32mx/lib/size\libpic32.a
LOAD c:/program files (x86)/microchip/xc32/v1.21/bin/../lib/gcc/pic32mx/4.5.2/../../../../pic32mx/lib/size\libdebug.a
LOAD c:/program files (x86)/microchip/xc32/v1.21/bin/../lib/gcc/pic32mx/4.5.2/../../../../pic32mx/lib/size\libm.a
LOAD c:/program files (x86)/microchip/xc32/v1.21/bin/../lib/gcc/pic32mx/4.5.2/../../../../pic32mx/lib/size\libe.a
LOAD c:/program files (x86)/microchip/xc32/v1.21/bin/../lib/gcc/pic32mx/4.5.2/../../../../pic32mx/lib/size\libdsp.a
LOAD c:/program files (x86)/microchip/xc32/v1.21/bin/../lib/gcc/pic32mx/4.5.2/size\libgcc.a
LOAD c:/program files (x86)/microchip/xc32/v1.21/bin/../lib/gcc/pic32mx/4.5.2/../../../../pic32mx/lib/size\libpic32.a
LOAD c:/program files (x86)/microchip/xc32/v1.21/bin/../lib/gcc/pic32mx/4.5.2/../../../../pic32mx/lib/size\libc.a
LOAD c:/program files (x86)/microchip/xc32/v1.21/bin/../lib/gcc/pic32mx/4.5.2/../../../../pic32mx/lib/size\libpic32.a
END GROUP
LOAD c:/program files (x86)/microchip/xc32/v1.21/bin/../lib/gcc/pic32mx/4.5.2/size\libgcc.a
OUTPUT(dist/default/production/tcp6_demo_app.X.production.elf elf32-tradlittlemips)
LOAD stack
LOAD data_init

.reginfo        0x9d000000       0x18
 .reginfo       0x9d000000       0x18 c:/program files (x86)/microchip/xc32/v1.21/bin/../lib/gcc/pic32mx/4.5.2/../../../../pic32mx/lib/size/crt0.o

.stack          0xa00088b0      0x800
 .stack         0xa00088b0      0x800 stack

.bss            0xa0001f78      0x458
 .bss           0xa0001f78      0x210 build/default/production/_ext/97638081/sys_fs.o
 .bss           0xa0002188       0xd8 build/default/production/_ext/97638081/mpfs2.o
 .bss           0xa0002260       0x68 build/default/production/_ext/365611741/system_command.o
 .bss           0xa00022c8       0x5c build/default/production/_ext/365611741/system_random.o
 .bss           0xa0002324       0x5c build/default/production/_ext/1472/custom_http_app.o
 .bss           0xa0002380       0x50 build/default/production/_ext/365611741/system_userio.o

.data           0xa00023d0       0x44
 .data          0xa00023d0       0x44 build/default/production/_ext/1472/tcp6_demo_app.o
                0xa00023d0                b64

.bss            0xa0002414       0x7c
 .bss           0xa0002414       0x40 c:/program files (x86)/microchip/xc32/v1.21/bin/../lib/gcc/pic32mx/4.5.2/../../../../pic32mx/lib/size\libc.a(_iob.o)
                0xa0002414                _sibuf
                0xa0002434                _sobuf
 .bss           0xa0002454       0x1c c:/program files (x86)/microchip/xc32/v1.21/bin/../lib/gcc/pic32mx/4.5.2/../../../../pic32mx/lib/size\libpic32.a(sbrk.o)
 .bss           0xa0002470       0x10 c:/program files (x86)/microchip/xc32/v1.21/bin/../lib/gcc/pic32mx/4.5.2/../../../../pic32mx/lib/size\libc.a(malloc.o)
                0xa0002470                __allocs
 .bss           0xa0002480       0x10 c:/program files (x86)/microchip/xc32/v1.21/bin/../lib/gcc/pic32mx/4.5.2/../../../../pic32mx/lib/size\libc.a(rand.o)

.text.HTTPProcess
                0x9d000020     0x17c4
 .text.HTTPProcess
                0x9d000020     0x17c4 build/default/production/_ext/427700826/http2.o

.text._TcpHandleSeg
                0x9d0017e4     0x1778
 .text._TcpHandleSeg
                0x9d0017e4     0x1778 build/default/production/_ext/427700826/tcp.o

.text.vfprintf  0x9d002f5c     0x15a8
 .text.vfprintf
                0x9d002f5c     0x15a8 c:/program files (x86)/microchip/xc32/v1.21/bin/../lib/gcc/pic32mx/4.5.2/../../../../pic32mx/lib/size\libc.a(doprnt.o)
                0x9d002f5c                vfprintf

.text.DNSClientTask
                0x9d004504     0x1144
 .text.DNSClientTask
                0x9d004504     0x1144 build/default/production/_ext/427700826/dns.o
                0x9d004504                DNSClientTask

.text.tcp6_demo_app_tasks
                0x9d005648      0xef4
 .text.tcp6_demo_app_tasks
                0x9d005648      0xef4 build/default/production/_ext/1472/tcp6_demo_app.o
                0x9d005648                tcp6_demo_app_tasks

.text.DHCPTask  0x9d00653c      0xa74
 .text.DHCPTask
                0x9d00653c      0xa74 build/default/production/_ext/427700826/dhcp.o
                0x9d00653c                DHCPTask

.text._TcpSend  0x9d006fb0      0xa40
 .text._TcpSend
                0x9d006fb0      0xa40 build/default/production/_ext/427700826/tcp.o

.text.TCPAdjustFIFOSize
                0x9d0079f0      0x974
 .text.TCPAdjustFIFOSize
                0x9d0079f0      0x974 build/default/production/_ext/427700826/tcp.o
                0x9d0079f0                TCPAdjustFIFOSize

.rodata         0x9d008364      0x8f4
 .rodata        0x9d008364      0x8f4 build/default/production/_ext/427700826/http2.o

.text           0x9d008c58      0x8ec
 .text          0x9d008c58      0x8ec c:/program files (x86)/microchip/xc32/v1.21/bin/../lib/gcc/pic32mx/4.5.2/../../../../pic32mx/lib/size\libm.a(fp32.o)
                0x9d008c58                __subsf3
                0x9d008c58                fpsub
                0x9d008c60                fpadd
                0x9d008c60                __addsf3
                0x9d008ecc                fpmul
                0x9d008ecc                __mulsf3
                0x9d009084                fpdiv
                0x9d009084                __divsf3
                0x9d0092b0                litofp
                0x9d0092b0                sitofp
                0x9d0092b0                __floatsisf
                0x9d00930c                uitofp
                0x9d00930c                ultofp
                0x9d009358                fptosi
                0x9d009358                fptoli
                0x9d009358                __fixsfsi
                0x9d0093d0                __fixunssfsi
                0x9d0093d0                fptoul
                0x9d0093d0                fptoui
                0x9d009444                __eqsf2
                0x9d009444                __nesf2
                0x9d009444                __lesf2
                0x9d009444                __ltsf2
                0x9d009444                fpcmp
                0x9d009444                __gtsf2
                0x9d009444                __gesf2
                0x9d0094d8                fpfabs
                0x9d0094d8                fabsf
                0x9d0094e8                __negsf2
                0x9d0094f8                fpnan
                0x9d0094f8                nanf

.text._vfprintf_cdnopsuxX
                0x9d009544      0x8b8
 .text._vfprintf_cdnopsuxX
                0x9d009544      0x8b8 c:/program files (x86)/microchip/xc32/v1.21/bin/../lib/gcc/pic32mx/4.5.2/../../../../pic32mx/lib/size\libc.a(doprnt_cdnopsuxX.eo)
                0x9d009544                _vfprintf_cdnopuxX
                0x9d009544                _vfprintf_cdnopsuxX

.text.TCPTick   0x9d009dfc      0x890
 .text.TCPTick  0x9d009dfc      0x890 build/default/production/_ext/427700826/tcp.o
                0x9d009dfc                TCPTick

.rodata         0x9d00a68c      0x7d4
 .rodata        0x9d00a68c      0x7d4 c:/program files (x86)/microchip/xc32/v1.21/bin/../lib/gcc/pic32mx/4.5.2/../../../../pic32mx/lib/size\libmchp_peripheral_32MX795F512L.a(int_tbl_lib.o)
                0x9d00a68c                __IntSrcTbl
                0x9d00aba8                __IntVectorTbl

.text._DHCPReceive
                0x9d00ae60      0x748
 .text._DHCPReceive
                0x9d00ae60      0x748 build/default/production/_ext/427700826/dhcp.o

.text.NBNSTask  0x9d00b5a8      0x73c
 .text.NBNSTask
                0x9d00b5a8      0x73c build/default/production/_ext/427700826/nbns.o
                0x9d00b5a8                NBNSTask

.text.HTTPPrint
                0x9d00bce4      0x6ac
 .text.HTTPPrint
                0x9d00bce4      0x6ac build/default/production/_ext/427700826/http2.o
                0x9d00bce4                HTTPPrint

.text.HTTPPostConfig
                0x9d00c390      0x694
 .text.HTTPPostConfig
                0x9d00c390      0x694 build/default/production/_ext/1472/custom_http_app.o

.text._DHCPSend
                0x9d00ca24      0x5c8
 .text._DHCPSend
                0x9d00ca24      0x5c8 build/default/production/_ext/427700826/dhcp.o

.text.TCPFindArray
                0x9d00cfec      0x578
 .text.TCPFindArray
                0x9d00cfec      0x578 build/default/production/_ext/427700826/tcp.o
                0x9d00cfec                TCPFindArray

.text.SHA1HashBlock
                0x9d00d564      0x4fc
 .text.SHA1HashBlock
                0x9d00d564      0x4fc build/default/production/_ext/101875047/hashes.o

.text.SYS_Initialize
                0x9d00da60      0x4f0
 .text.SYS_Initialize
                0x9d00da60      0x4f0 build/default/production/_ext/365611741/system_services.o
                0x9d00da60                SYS_Initialize

.text.TCPIP_ANNOUNCE_Send
                0x9d00df50      0x490
 .text.TCPIP_ANNOUNCE_Send
                0x9d00df50      0x490 build/default/production/_ext/427700826/tcpip_announce.o
                0x9d00df50                TCPIP_ANNOUNCE_Send

.text._TCPIP_HEAP_Free
                0x9d00e3e0      0x490
 .text._TCPIP_HEAP_Free
                0x9d00e3e0      0x490 build/default/production/_ext/427700826/tcpip_heap_alloc.o
                0x9d00e3e0                _TCPIP_HEAP_Free

.text.TCPIP_STACK_Init
                0x9d00e870      0x464
 .text.TCPIP_STACK_Init
                0x9d00e870      0x464 build/default/production/_ext/427700826/tcpip_manager.o
                0x9d00e870                TCPIP_STACK_Init

.text           0x9d00ecd4      0x8a0
 .text          0x9d00ecd4      0x460 c:/program files (x86)/microchip/xc32/v1.21/bin/../lib/gcc/pic32mx/4.5.2/size\libgcc.a(_umoddi3.o)
                0x9d00ecd4                __umoddi3
 .text          0x9d00f134      0x440 c:/program files (x86)/microchip/xc32/v1.21/bin/../lib/gcc/pic32mx/4.5.2/size\libgcc.a(_udivdi3.o)
                0x9d00f134                __udivdi3

.rodata         0x9d00f574      0x43c
 .rodata        0x9d00f574      0x43c build/default/production/_ext/1472/tcp6_demo_app.o
                0x9d00f574                Version
                0x9d00f578                CompileDate
                0x9d00f584                CompileTime
                0x9d00f694                HTTP_TRANSACTION_LIST

.text.CommandHelp
                0x9d00f9b0      0x428
 .text.CommandHelp
                0x9d00f9b0      0x428 build/default/production/_ext/365611741/system_command.o

.text.TCPOpen   0x9d00fdd8      0x420
 .text.TCPOpen  0x9d00fdd8      0x420 build/default/production/_ext/427700826/tcp.o

.text.HTTPExecuteGet
                0x9d0101f8      0x414
 .text.HTTPExecuteGet
                0x9d0101f8      0x414 build/default/production/_ext/1472/custom_http_app.o
                0x9d0101f8                HTTPExecuteGet

.text.HTTPMPFSUpload
                0x9d01060c      0x410
 .text.HTTPMPFSUpload
                0x9d01060c      0x410 build/default/production/_ext/427700826/http2.o

.dinit          0x9d010a1c      0x408
 .dinit         0x9d010a1c      0x408 data_init

.text.ARPInitialize
                0x9d010e24      0x3f4
 .text.ARPInitialize
                0x9d010e24      0x3f4 build/default/production/_ext/427700826/arp.o
                0x9d010e24                ARPInitialize

.text._TcpFindMatchingSocket
                0x9d011218      0x3e8
 .text._TcpFindMatchingSocket
                0x9d011218      0x3e8 build/default/production/_ext/427700826/tcp.o

.text           0x9d011600      0x3dc
 .text          0x9d011600      0x3dc c:/program files (x86)/microchip/xc32/v1.21/bin/../lib/gcc/pic32mx/4.5.2/../../../../pic32mx/lib/size\libm.a(fpmod32.o)
                0x9d011600                fmodf
                0x9d011600                fpfmod
                0x9d011744                frexpf
                0x9d011744                fpfrexp
                0x9d0117c8                __mchp_ldexpf
                0x9d0117c8                fpldexp
                0x9d01190c                fpmodf
                0x9d01190c                modff

.text.MPFSSeek  0x9d0119dc      0x3ac
 .text.MPFSSeek
                0x9d0119dc      0x3ac build/default/production/_ext/97638081/mpfs2.o
                0x9d0119dc                MPFSSeek

.text.ENCX24J600_MACInit
                0x9d011d88      0x3a0
 .text.ENCX24J600_MACInit
                0x9d011d88      0x3a0 build/default/production/_ext/427700826/encs24j600.o
                0x9d011d88                ENCX24J600_MACInit

.text.FindMatchingSocket
                0x9d012128      0x39c
 .text.FindMatchingSocket
                0x9d012128      0x39c build/default/production/_ext/427700826/udp.o

.text.TCPIP_Helper_Base64Decode
                0x9d0124c4      0x394
 .text.TCPIP_Helper_Base64Decode
                0x9d0124c4      0x394 build/default/production/_ext/427700826/tcpip_helpers.o
                0x9d0124c4                TCPIP_Helper_Base64Decode

.rodata         0x9d012858      0x38c
 .rodata        0x9d012858      0x38c build/default/production/_ext/427700826/tcpip_manager.o

.text._SYS_COMMAND_TASK
                0x9d012be4      0x354
 .text._SYS_COMMAND_TASK
                0x9d012be4      0x354 build/default/production/_ext/365611741/system_command.o
                0x9d012be4                _SYS_COMMAND_TASK

.text.HTTPPostMD5
                0x9d012f38      0x340
 .text.HTTPPostMD5
                0x9d012f38      0x340 build/default/production/_ext/1472/custom_http_app.o

.text.UDPOpen   0x9d013278      0x330
 .text.UDPOpen  0x9d013278      0x330 build/default/production/_ext/427700826/udp.o

.text.TCPIP_STACK_BringNetUp
                0x9d0135a8      0x32c
 .text.TCPIP_STACK_BringNetUp
                0x9d0135a8      0x32c build/default/production/_ext/427700826/tcpip_manager.o

.text.TCPIP_HELPER_StringToIPAddress
                0x9d0138d4      0x31c
 .text.TCPIP_HELPER_StringToIPAddress
                0x9d0138d4      0x31c build/default/production/_ext/427700826/tcpip_helpers.o
                0x9d0138d4                TCPIP_HELPER_StringToIPAddress

.text.HTTPInit  0x9d013bf0      0x318
 .text.HTTPInit
                0x9d013bf0      0x318 build/default/production/_ext/427700826/http2.o
                0x9d013bf0                HTTPInit

.text.ARPTask   0x9d013f08      0x310
 .text.ARPTask  0x9d013f08      0x310 build/default/production/_ext/427700826/arp.o
                0x9d013f08                ARPTask

.text.TCPIP_IPV4_PutArrayHelper
                0x9d014218      0x310
 .text.TCPIP_IPV4_PutArrayHelper
                0x9d014218      0x310 build/default/production/_ext/427700826/ipv4.o
                0x9d014218                TCPIP_IPV4_PutArrayHelper

.text.MPFSOpen  0x9d014528      0x30c
 .text.MPFSOpen
                0x9d014528      0x30c build/default/production/_ext/97638081/mpfs2.o
                0x9d014528                MPFSOpen

.text.UDPInit   0x9d014834      0x300
 .text.UDPInit  0x9d014834      0x300 build/default/production/_ext/427700826/udp.o
                0x9d014834                UDPInit

.text.tcp6_demo_app_init
                0x9d014b34      0x2d8
 .text.tcp6_demo_app_init
                0x9d014b34      0x2d8 build/default/production/_ext/1472/tcp6_demo_app.o
                0x9d014b34                tcp6_demo_app_init

.text.ProcessEscSequence
                0x9d014e0c      0x2c8
 .text.ProcessEscSequence
                0x9d014e0c      0x2c8 build/default/production/_ext/365611741/system_command.o

.text.DoWrite   0x9d0150d4      0x2c4
 .text.DoWrite  0x9d0150d4      0x2c4 build/default/production/_ext/792872985/spi_eeprom.o

.text.HTTPReadTo
                0x9d015398      0x2c4
 .text.HTTPReadTo
                0x9d015398      0x2c4 build/default/production/_ext/427700826/http2.o

.text.ENCX24J600_MACGetHeader
                0x9d01565c      0x2c0
 .text.ENCX24J600_MACGetHeader
                0x9d01565c      0x2c0 build/default/production/_ext/427700826/encs24j600.o
                0x9d01565c                ENCX24J600_MACGetHeader

.text.MD5HashBlock
                0x9d01591c      0x2bc
 .text.MD5HashBlock
                0x9d01591c      0x2bc build/default/production/_ext/101875047/hashes.o

.text.TCPIP_STACK_Task
                0x9d015bd8      0x2b8
 .text.TCPIP_STACK_Task
                0x9d015bd8      0x2b8 build/default/production/_ext/427700826/tcpip_manager.o
                0x9d015bd8                TCPIP_STACK_Task

.text.main      0x9d015e90      0x2b8
 .text.main     0x9d015e90      0x2b8 build/default/production/_ext/1472/main_demo.o
                0x9d015e90                main

.text.ICMPProcess
                0x9d016148      0x2ac
 .text.ICMPProcess
                0x9d016148      0x2ac build/default/production/_ext/427700826/icmp.o
                0x9d016148                ICMPProcess

.text.TCPPutArray
                0x9d0163f4      0x2ac
 .text.TCPPutArray
                0x9d0163f4      0x2ac build/default/production/_ext/427700826/tcp.o
                0x9d0163f4                TCPPutArray

.text.MD5Calculate
                0x9d0166a0      0x2a8
 .text.MD5Calculate
                0x9d0166a0      0x2a8 build/default/production/_ext/101875047/hashes.o
                0x9d0166a0                MD5Calculate

.text.ParseCmdBuffer
                0x9d016948      0x2a4
 .text.ParseCmdBuffer
                0x9d016948      0x2a4 build/default/production/_ext/365611741/system_command.o

.text.DRV_MEDIA_Open
                0x9d016bec      0x294
 .text.DRV_MEDIA_Open
                0x9d016bec      0x294 build/default/production/_ext/792872985/drv_media.o
                0x9d016bec                DRV_MEDIA_Open

.rodata         0x9d016e80      0x28c
 .rodata        0x9d016e80      0x28c build/default/production/_ext/365611741/system_command.o
                0x9d016e90                sysConsoleApi

.text.MPFSGetArray
                0x9d01710c      0x280
 .text.MPFSGetArray
                0x9d01710c      0x280 build/default/production/_ext/97638081/mpfs2.o
                0x9d01710c                MPFSGetArray

.text.UDPProcessIPv4
                0x9d01738c      0x278
 .text.UDPProcessIPv4
                0x9d01738c      0x278 build/default/production/_ext/427700826/udp.o
                0x9d01738c                UDPProcessIPv4

.text.SYS_FS_mount
                0x9d017604      0x274
 .text.SYS_FS_mount
                0x9d017604      0x274 build/default/production/_ext/97638081/sys_fs.o
                0x9d017604                SYS_FS_mount

.text.GetMaxSegSizeOption
                0x9d017878      0x274
 .text.GetMaxSegSizeOption
                0x9d017878      0x274 build/default/production/_ext/427700826/tcp.o

.text.XEEReadArray
                0x9d017aec      0x268
 .text.XEEReadArray
                0x9d017aec      0x268 build/default/production/_ext/792872985/spi_eeprom.o
                0x9d017aec                XEEReadArray

.text.TCPIP_IPV4_CalculatePayloadChecksum
                0x9d017d54      0x268
 .text.TCPIP_IPV4_CalculatePayloadChecksum
                0x9d017d54      0x268 build/default/production/_ext/427700826/ipv4.o
                0x9d017d54                TCPIP_IPV4_CalculatePayloadChecksum

.text.HTTPSendFile
                0x9d017fbc      0x264
 .text.HTTPSendFile
                0x9d017fbc      0x264 build/default/production/_ext/427700826/http2.o

.text.TCPGetArray
                0x9d018220      0x260
 .text.TCPGetArray
                0x9d018220      0x260 build/default/production/_ext/427700826/tcp.o
                0x9d018220                TCPGetArray

.text.SYS_GENERATE_RANDOM_DWORD
                0x9d018480      0x25c
 .text.SYS_GENERATE_RANDOM_DWORD
                0x9d018480      0x25c build/default/production/_ext/365611741/system_random.o
                0x9d018480                SYS_GENERATE_RANDOM_DWORD

.text.SYS_CLK_OscClockGet
                0x9d0186dc      0x258
 .text.SYS_CLK_OscClockGet
                0x9d0186dc      0x258 build/default/production/_ext/365611741/system_services.o
                0x9d0186dc                SYS_CLK_OscClockGet

.text.TCPIP_IPV4_CopyTxPacketStruct
                0x9d018934      0x250
 .text.TCPIP_IPV4_CopyTxPacketStruct
                0x9d018934      0x250 build/default/production/_ext/427700826/ipv4.o
                0x9d018934                TCPIP_IPV4_CopyTxPacketStruct

.text           0x9d018b84      0x248
 .text          0x9d018b84      0x248 build/default/production/_ext/427700826/tcpip_helper_c32.o
                0x9d018b84                TCPIP_HELPER_htonl
                0x9d018b90                TCPIP_HELPER_htons
                0x9d018b9c                TCPIP_Helper_CalcIPChecksum

.text.LoadDefaultConfig
                0x9d018dcc      0x244
 .text.LoadDefaultConfig
                0x9d018dcc      0x244 build/default/production/_ext/427700826/tcpip_manager.o

.text.malloc    0x9d019010      0x240
 .text.malloc   0x9d019010      0x240 c:/program files (x86)/microchip/xc32/v1.21/bin/../lib/gcc/pic32mx/4.5.2/../../../../pic32mx/lib/size\libc.a(malloc.o)
                0x9d019010                malloc

.text.LCD_UPDATE_OFFSET
                0x9d019250      0x230
 .text.LCD_UPDATE_OFFSET
                0x9d019250      0x230 build/default/production/_ext/792872985/lcd.o
                0x9d019250                LCD_UPDATE_OFFSET

.text.MPFSGet   0x9d019480      0x228
 .text.MPFSGet  0x9d019480      0x228 build/default/production/_ext/97638081/mpfs2.o
                0x9d019480                MPFSGet

.text.ARPEntryRemoveNet
                0x9d0196a8      0x224
 .text.ARPEntryRemoveNet
                0x9d0196a8      0x224 build/default/production/_ext/427700826/arp.o
                0x9d0196a8                ARPEntryRemoveNet

.text.TCPIP_IPV4_GetDataSegmentByType
                0x9d0198cc      0x224
 .text.TCPIP_IPV4_GetDataSegmentByType
                0x9d0198cc      0x224 build/default/production/_ext/427700826/ipv4.o
                0x9d0198cc                TCPIP_IPV4_GetDataSegmentByType

.text.__floatdisf
                0x9d019af0      0x220
 .text.__floatdisf
                0x9d019af0      0x220 c:/program files (x86)/microchip/xc32/v1.21/bin/../lib/gcc/pic32mx/4.5.2/../../../../pic32mx/lib/size\libe.a(_floatdisf.o)
                0x9d019af0                __floatdisf

.rodata         0x9d019d10      0x21c
 .rodata        0x9d019d10      0x21c build/default/production/_ext/365611741/system_services.o
                0x9d019d20                MEDIA_STORAGE_TCPIP_STORAGE_PARTITION
                0x9d019d34                MEDIA_STORAGE_MPFS_IMAGE_PARTITION
                0x9d019d48                MEDIA_STORAGE_CONFIGURATION

.text.HTTPHeaderParseCookie
                0x9d019f2c      0x214
 .text.HTTPHeaderParseCookie
                0x9d019f2c      0x214 build/default/production/_ext/427700826/http2.o

.text.TCPInit   0x9d01a140      0x210
 .text.TCPInit  0x9d01a140      0x210 build/default/production/_ext/427700826/tcp.o
                0x9d01a140                TCPInit

.text.DHCPInit  0x9d01a350      0x204
 .text.DHCPInit
                0x9d01a350      0x204 build/default/production/_ext/427700826/dhcp.o
                0x9d01a350                DHCPInit

.text._TcpDisconnect
                0x9d01a554      0x204
 .text._TcpDisconnect
                0x9d01a554      0x204 build/default/production/_ext/427700826/tcp.o

.text.HTTPIncFile
                0x9d01a758      0x200
 .text.HTTPIncFile
                0x9d01a758      0x200 build/default/production/_ext/427700826/http2.o
                0x9d01a758                HTTPIncFile

.text.UDPTask   0x9d01a958      0x200
 .text.UDPTask  0x9d01a958      0x200 build/default/production/_ext/427700826/udp.o
                0x9d01a958                UDPTask

.rodata         0x9d01ab58      0x1fc
 .rodata        0x9d01ab58      0x1fc build/default/production/_ext/1472/main_demo.o
                0x9d01ab58                arpConfigData
                0x9d01ab78                dhcpConfigData
                0x9d01ab88                httpConfigData
                0x9d01ab94                macPIC32INTConfigData
                0x9d01aba4                mac97J60ConfigData
                0x9d01aba4                tcpConfigData
                0x9d01aba4                macMRF24WConfigData
                0x9d01aba4                macENCJ600ConfigData
                0x9d01aba4                macENCJ60ConfigData
                0x9d01abac                udpConfigData
                0x9d01ac18                TCPIP_HOSTS_CONFIGURATION
                0x9d01ac40                TCPIP_STACK_MODULE_CONFIG_TBL

.text.SYS_USERIO_SetLED
                0x9d01ad54      0x1f8
 .text.SYS_USERIO_SetLED
                0x9d01ad54      0x1f8 build/default/production/_ext/365611741/system_userio.o
                0x9d01ad54                SYS_USERIO_SetLED

.text.TCPIP_ANNOUNCE_Task
                0x9d01af4c      0x1f8
 .text.TCPIP_ANNOUNCE_Task
                0x9d01af4c      0x1f8 build/default/production/_ext/427700826/tcpip_announce.o
                0x9d01af4c                TCPIP_ANNOUNCE_Task

.text.ARPProcess
                0x9d01b144      0x1f0
 .text.ARPProcess
                0x9d01b144      0x1f0 build/default/production/_ext/427700826/arp.o
                0x9d01b144                ARPProcess

.text.TCPIP_IPV4_Flush
                0x9d01b334      0x1ec
 .text.TCPIP_IPV4_Flush
                0x9d01b334      0x1ec build/default/production/_ext/427700826/ipv4.o
                0x9d01b334                TCPIP_IPV4_Flush

.text.SYS_FS_ExtractFirstFilename
                0x9d01b520      0x1e8
 .text.SYS_FS_ExtractFirstFilename
                0x9d01b520      0x1e8 build/default/production/_ext/97638081/sys_fs.o

.text.SYS_FS_initialize
                0x9d01b708      0x1e8
 .text.SYS_FS_initialize
                0x9d01b708      0x1e8 build/default/production/_ext/97638081/sys_fs.o
                0x9d01b708                SYS_FS_initialize

.text._TCPIP_HEAP_Malloc
                0x9d01b8f0      0x1e0
 .text._TCPIP_HEAP_Malloc
                0x9d01b8f0      0x1e0 build/default/production/_ext/427700826/tcpip_heap_alloc.o
                0x9d01b8f0                _TCPIP_HEAP_Malloc

.rodata         0x9d01bad0      0x1e0
 .rodata        0x9d01bad0      0x1e0 build/default/production/_ext/1472/custom_http_app.o
                0x9d01bbfc                HTML_UP_ARROW
                0x9d01bc00                HTML_DOWN_ARROW

.text.StringToArgs
                0x9d01bcb0      0x1dc
 .text.StringToArgs
                0x9d01bcb0      0x1dc build/default/production/_ext/365611741/system_command.o

.text.HTTPURLDecode
                0x9d01be8c      0x1dc
 .text.HTTPURLDecode
                0x9d01be8c      0x1dc build/default/production/_ext/427700826/http2.o
                0x9d01be8c                HTTPURLDecode

.text.TCPProcessIPv4
                0x9d01c068      0x1dc
 .text.TCPProcessIPv4
                0x9d01c068      0x1dc build/default/production/_ext/427700826/tcp.o
                0x9d01c068                TCPProcessIPv4

.text.TCPIP_IPV4_IsTxPutReady
                0x9d01c244      0x1d8
 .text.TCPIP_IPV4_IsTxPutReady
                0x9d01c244      0x1d8 build/default/production/_ext/427700826/ipv4.o
                0x9d01c244                TCPIP_IPV4_IsTxPutReady

.text.SYS_FS_chdir
                0x9d01c41c      0x1d4
 .text.SYS_FS_chdir
                0x9d01c41c      0x1d4 build/default/production/_ext/97638081/sys_fs.o
                0x9d01c41c                SYS_FS_chdir

.text.HTTPHeaderParseAuthorization
                0x9d01c5f0      0x1d4
 .text.HTTPHeaderParseAuthorization
                0x9d01c5f0      0x1d4 build/default/production/_ext/427700826/http2.o

.text.UDPv4IsTxPutReady
                0x9d01c7c4      0x1d0
 .text.UDPv4IsTxPutReady
                0x9d01c7c4      0x1d0 build/default/production/_ext/427700826/udp.o

.text._TCPIsPutReady
                0x9d01c994      0x1cc
 .text._TCPIsPutReady
                0x9d01c994      0x1cc build/default/production/_ext/427700826/tcp.o

.text.UDPDeInit
                0x9d01cb60      0x1cc
 .text.UDPDeInit
                0x9d01cb60      0x1cc build/default/production/_ext/427700826/udp.o
                0x9d01cb60                UDPDeInit

.text.strtoul   0x9d01cd2c      0x1cc
 .text.strtoul  0x9d01cd2c      0x1cc c:/program files (x86)/microchip/xc32/v1.21/bin/../lib/gcc/pic32mx/4.5.2/../../../../pic32mx/lib/size\libc.a(strtol.o)
                0x9d01cd2c                strtoul

.text.SYS_USERIO_ReadIO
                0x9d01cef8      0x1c8
 .text.SYS_USERIO_ReadIO
                0x9d01cef8      0x1c8 build/default/production/_ext/365611741/system_userio.o

.text._TcpSocketSetIdleState
                0x9d01d0c0      0x1c8
 .text._TcpSocketSetIdleState
                0x9d01d0c0      0x1c8 build/default/production/_ext/427700826/tcp.o

.text.ProcessTCPIPMacEvents
                0x9d01d288      0x1c4
 .text.ProcessTCPIPMacEvents
                0x9d01d288      0x1c4 build/default/production/_ext/427700826/tcpip_manager.o

.text.HTTPPrint_ledSelected
                0x9d01d44c      0x1c4
 .text.HTTPPrint_ledSelected
                0x9d01d44c      0x1c4 build/default/production/_ext/1472/custom_http_app.o
                0x9d01d44c                HTTPPrint_ledSelected

.text.TCPSetOptions
                0x9d01d610      0x1b8
 .text.TCPSetOptions
                0x9d01d610      0x1b8 build/default/production/_ext/427700826/tcp.o
                0x9d01d610                TCPSetOptions

.text.HTTPPrint_uploadedmd5
                0x9d01d7c8      0x1b8
 .text.HTTPPrint_uploadedmd5
                0x9d01d7c8      0x1b8 build/default/production/_ext/1472/custom_http_app.o
                0x9d01d7c8                HTTPPrint_uploadedmd5

.text._SystemTickIntHandler
                0x9d01d980      0x1b0
 .text._SystemTickIntHandler
                0x9d01d980      0x1b0 build/default/production/_ext/365611741/system_services.o
                0x9d01d980                _SystemTickIntHandler

.text.DisplayNodeMsg
                0x9d01db30      0x1a0
 .text.DisplayNodeMsg
                0x9d01db30      0x1a0 build/default/production/_ext/365611741/system_command.o

.text.HTTPPrint_led
                0x9d01dcd0      0x1a0
 .text.HTTPPrint_led
                0x9d01dcd0      0x1a0 build/default/production/_ext/1472/custom_http_app.o
                0x9d01dcd0                HTTPPrint_led

.text           0x9d01de70      0x1a0
 .text          0x9d01de70      0x1a0 c:/program files (x86)/microchip/xc32/v1.21/bin/../lib/gcc/pic32mx/4.5.2/../../../../pic32mx/lib/size\libpic32.a(strcpy.o)
                0x9d01de70                strcpy

.text._TcpCloseSocket
                0x9d01e010      0x198
 .text._TcpCloseSocket
                0x9d01e010      0x198 build/default/production/_ext/427700826/tcp.o

.text.NBNSGetName
                0x9d01e1a8      0x194
 .text.NBNSGetName
                0x9d01e1a8      0x194 build/default/production/_ext/427700826/nbns.o

.text._Sys_Ext1_Isr
                0x9d01e33c      0x190
 .text._Sys_Ext1_Isr
                0x9d01e33c      0x190 build/default/production/_ext/365611741/system_services.o
                0x9d01e33c                _Sys_Ext1_Isr

.text._Sys_Ext3_Isr
                0x9d01e4cc      0x190
 .text._Sys_Ext3_Isr
                0x9d01e4cc      0x190 build/default/production/_ext/365611741/system_services.o
                0x9d01e4cc                _Sys_Ext3_Isr

.text._Sys_CN_Isr
                0x9d01e65c      0x190
 .text._Sys_CN_Isr
                0x9d01e65c      0x190 build/default/production/_ext/365611741/system_services.o
                0x9d01e65c                _Sys_CN_Isr

.text.TCPIP_HELPER_StringToMACAddress
                0x9d01e7ec      0x18c
 .text.TCPIP_HELPER_StringToMACAddress
                0x9d01e7ec      0x18c build/default/production/_ext/427700826/tcpip_helpers.o
                0x9d01e7ec                TCPIP_HELPER_StringToMACAddress

.text.DRV_MEDIA_Initialize
                0x9d01e978      0x188
 .text.DRV_MEDIA_Initialize
                0x9d01e978      0x188 build/default/production/_ext/792872985/drv_media.o
                0x9d01e978                DRV_MEDIA_Initialize

.text.UDPGetArray
                0x9d01eb00      0x188
 .text.UDPGetArray
                0x9d01eb00      0x188 build/default/production/_ext/427700826/udp.o
                0x9d01eb00                UDPGetArray

.text.HTTPServer
                0x9d01ec88      0x180
 .text.HTTPServer
                0x9d01ec88      0x180 build/default/production/_ext/427700826/http2.o
                0x9d01ec88                HTTPServer

.text.WriteReg  0x9d01ee08      0x180
 .text.WriteReg
                0x9d01ee08      0x180 build/default/production/_ext/427700826/encs24j600.o

.text._OAHashFindBkt
                0x9d01ef88      0x180
 .text._OAHashFindBkt
                0x9d01ef88      0x180 build/default/production/_ext/427700826/hash_tbl.o

.text.ARPIsResolved
                0x9d01f108      0x178
 .text.ARPIsResolved
                0x9d01f108      0x178 build/default/production/_ext/427700826/arp.o
                0x9d01f108                ARPIsResolved

.text.TCPIP_IPV4_AllocateTxPacket
                0x9d01f280      0x178
 .text.TCPIP_IPV4_AllocateTxPacket
                0x9d01f280      0x178 build/default/production/_ext/427700826/ipv4.o
                0x9d01f280                TCPIP_IPV4_AllocateTxPacket

.text.TCPIP_HEAP_Create
                0x9d01f3f8      0x178
 .text.TCPIP_HEAP_Create
                0x9d01f3f8      0x178 build/default/production/_ext/427700826/tcpip_heap_alloc.o
                0x9d01f3f8                TCPIP_HEAP_Create

.text.HTTPPostLCD
                0x9d01f570      0x178
 .text.HTTPPostLCD
                0x9d01f570      0x178 build/default/production/_ext/1472/custom_http_app.o

.text.SYS_FS_IsLegalDirString
                0x9d01f6e8      0x170
 .text.SYS_FS_IsLegalDirString
                0x9d01f6e8      0x170 build/default/production/_ext/97638081/sys_fs.o
                0x9d01f6e8                SYS_FS_IsLegalDirString

.text.LCD_INIT  0x9d01f858      0x170
 .text.LCD_INIT
                0x9d01f858      0x170 build/default/production/_ext/792872985/lcd.o
                0x9d01f858                LCD_INIT

.text._ARPProbeAddress
                0x9d01f9c8      0x170
 .text._ARPProbeAddress
                0x9d01f9c8      0x170 build/default/production/_ext/427700826/arp.o

.text.SpiChnOpen
                0x9d01fb38      0x170
 .text.SpiChnOpen
                0x9d01fb38      0x170 c:/program files (x86)/microchip/xc32/v1.21/bin/../lib/gcc/pic32mx/4.5.2/../../../../pic32mx/lib/size\libmchp_peripheral_32MX795F512L.a(spi_chn_open_lib.o)
                0x9d01fb38                SpiChnOpen

.text.stricmppgm2ram
                0x9d01fca8      0x16c
 .text.stricmppgm2ram
                0x9d01fca8      0x16c build/default/production/_ext/101875047/helpers.o
                0x9d01fca8                stricmppgm2ram

.text.OAHashLookUpInsert
                0x9d01fe14      0x16c
 .text.OAHashLookUpInsert
                0x9d01fe14      0x16c build/default/production/_ext/427700826/hash_tbl.o
                0x9d01fe14                OAHashLookUpInsert

.text.UDPv4Flush
                0x9d01ff80      0x16c
 .text.UDPv4Flush
                0x9d01ff80      0x16c build/default/production/_ext/427700826/udp.o

.text           0x9d0200ec      0x2d0
 .text          0x9d0200ec      0x168 c:/program files (x86)/microchip/xc32/v1.21/bin/../lib/gcc/pic32mx/4.5.2/../../../../pic32mx/lib/size\libpic32.a(memcpy.o)
                0x9d0200ec                memcpy
 .text          0x9d020254      0x168 c:/program files (x86)/microchip/xc32/v1.21/bin/../lib/gcc/pic32mx/4.5.2/../../../../pic32mx/lib/size\libpic32.a(strlen.o)
                0x9d020254                strlen

.text.MPFSOpenID
                0x9d0203bc      0x164
 .text.MPFSOpenID
                0x9d0203bc      0x164 build/default/production/_ext/97638081/mpfs2.o
                0x9d0203bc                MPFSOpenID

.text.XEEIsBusy
                0x9d020520      0x164
 .text.XEEIsBusy
                0x9d020520      0x164 build/default/production/_ext/792872985/spi_eeprom.o
                0x9d020520                XEEIsBusy

.text.SYS_TICK_TimerDelete
                0x9d020684      0x160
 .text.SYS_TICK_TimerDelete
                0x9d020684      0x160 build/default/production/_ext/365611741/system_services.o
                0x9d020684                SYS_TICK_TimerDelete

.text.USART_INIT
                0x9d0207e4      0x160
 .text.USART_INIT
                0x9d0207e4      0x160 build/default/production/_ext/792872985/usart.o
                0x9d0207e4                USART_INIT

.text.DRV_SPI_TxRx
                0x9d020944      0x160
 .text.DRV_SPI_TxRx
                0x9d020944      0x160 build/default/production/_ext/792872985/drv_spi.o
                0x9d020944                DRV_SPI_TxRx

.text.DNSPutString
                0x9d020aa4      0x160
 .text.DNSPutString
                0x9d020aa4      0x160 build/default/production/_ext/427700826/dns.o

.text.ReadReg   0x9d020c04      0x160
 .text.ReadReg  0x9d020c04      0x160 build/default/production/_ext/427700826/encs24j600.o

.text.TCPIP_IPV4_TransmitPacket
                0x9d020d64      0x160
 .text.TCPIP_IPV4_TransmitPacket
                0x9d020d64      0x160 build/default/production/_ext/427700826/ipv4.o
                0x9d020d64                TCPIP_IPV4_TransmitPacket

.text.UDPBind   0x9d020ec4      0x160
 .text.UDPBind  0x9d020ec4      0x160 build/default/production/_ext/427700826/udp.o
                0x9d020ec4                UDPBind

.text.encodeblock
                0x9d021024      0x160
 .text.encodeblock
                0x9d021024      0x160 build/default/production/_ext/1472/tcp6_demo_app.o
                0x9d021024                encodeblock

.text.ARP_SendIfPkt
                0x9d021184      0x15c
 .text.ARP_SendIfPkt
                0x9d021184      0x15c build/default/production/_ext/427700826/arp.o

.text.TCPIP_IPV4_GetHeader
                0x9d0212e0      0x15c
 .text.TCPIP_IPV4_GetHeader
                0x9d0212e0      0x15c build/default/production/_ext/427700826/ipv4.o
                0x9d0212e0                TCPIP_IPV4_GetHeader

.text.DRV_MEDIA_Read
                0x9d02143c      0x158
 .text.DRV_MEDIA_Read
                0x9d02143c      0x158 build/default/production/_ext/792872985/drv_media.o
                0x9d02143c                DRV_MEDIA_Read

.text.HTTPPrint_config_mac
                0x9d021594      0x158
 .text.HTTPPrint_config_mac
                0x9d021594      0x158 build/default/production/_ext/1472/custom_http_app.o
                0x9d021594                HTTPPrint_config_mac

.rodata         0x9d0216ec      0x150
 .rodata        0x9d0216ec      0x150 build/default/production/_ext/365611741/system_debug.o

.text._TCPIPStackIsLocalNetwork
                0x9d02183c      0x150
 .text._TCPIPStackIsLocalNetwork
                0x9d02183c      0x150 build/default/production/_ext/427700826/tcpip_manager.o
                0x9d02183c                _TCPIPStackIsLocalNetwork

.text.scale     0x9d02198c      0x150
 .text.scale    0x9d02198c      0x150 c:/program files (x86)/microchip/xc32/v1.21/bin/../lib/gcc/pic32mx/4.5.2/../../../../pic32mx/lib/size\libc.a(doprnt.o)

.text._sbrk_init
                0x9d021adc      0x14c
 .text._sbrk_init
                0x9d021adc      0x14c c:/program files (x86)/microchip/xc32/v1.21/bin/../lib/gcc/pic32mx/4.5.2/../../../../pic32mx/lib/size\libpic32.a(sbrk.o)
                0x9d021adc                _sbrk_init

.text._SYS_CMDIO_DELETE
                0x9d021c28      0x148
 .text._SYS_CMDIO_DELETE
                0x9d021c28      0x148 build/default/production/_ext/365611741/system_command.o
                0x9d021c28                _SYS_CMDIO_DELETE

.text.ENCX24J600_MACCalcRxChecksum
                0x9d021d70      0x148
 .text.ENCX24J600_MACCalcRxChecksum
                0x9d021d70      0x148 build/default/production/_ext/427700826/encs24j600.o
                0x9d021d70                ENCX24J600_MACCalcRxChecksum

.text.OAHashLookUp
                0x9d021eb8      0x144
 .text.OAHashLookUp
                0x9d021eb8      0x144 build/default/production/_ext/427700826/hash_tbl.o
                0x9d021eb8                OAHashLookUp

.rodata         0x9d021ffc      0x140
 .rodata        0x9d021ffc      0x140 build/default/production/_ext/101875047/hashes.o

.text.UDPSocketSetNet
                0x9d02213c      0x140
 .text.UDPSocketSetNet
                0x9d02213c      0x140 build/default/production/_ext/427700826/udp.o
                0x9d02213c                UDPSocketSetNet

.text.ENCX24J600_SendSystemReset
                0x9d02227c      0x13c
 .text.ENCX24J600_SendSystemReset
                0x9d02227c      0x13c build/default/production/_ext/427700826/encs24j600.o

.text.BSP_Initialize
                0x9d0223b8      0x138
 .text.BSP_Initialize
                0x9d0223b8      0x138 build/default/production/_ext/1293749816/bsp.o
                0x9d0223b8                BSP_Initialize

.text._ARPUpdateEntry
                0x9d0224f0      0x138
 .text._ARPUpdateEntry
                0x9d0224f0      0x138 build/default/production/_ext/427700826/arp.o

.text.TCPIP_IPV4_QueuedPacketTransmitTask
                0x9d022628      0x138
 .text.TCPIP_IPV4_QueuedPacketTransmitTask
                0x9d022628      0x138 build/default/production/_ext/427700826/ipv4.o

.text.UDPIsGetReady
                0x9d022760      0x138
 .text.UDPIsGetReady
                0x9d022760      0x138 build/default/production/_ext/427700826/udp.o
                0x9d022760                UDPIsGetReady

.text.HTTPPrint_btn
                0x9d022898      0x138
 .text.HTTPPrint_btn
                0x9d022898      0x138 build/default/production/_ext/1472/custom_http_app.o
                0x9d022898                HTTPPrint_btn

.text._general_exception_handler
                0x9d0229d0      0x134
 .text._general_exception_handler
                0x9d0229d0      0x134 build/default/production/_ext/365611741/system_debug.o
                0x9d0229d0                _general_exception_handler

.text.TCPIP_IPV4_InsertIPPacketSegment
                0x9d022b04      0x134
 .text.TCPIP_IPV4_InsertIPPacketSegment
                0x9d022b04      0x134 build/default/production/_ext/427700826/ipv4.o
                0x9d022b04                TCPIP_IPV4_InsertIPPacketSegment

.text.uitoa     0x9d022c38      0x130
 .text.uitoa    0x9d022c38      0x130 build/default/production/_ext/101875047/helpers.o
                0x9d022c38                uitoa

.text.DRV_MEDIA_Write
                0x9d022d68      0x130
 .text.DRV_MEDIA_Write
                0x9d022d68      0x130 build/default/production/_ext/792872985/drv_media.o
                0x9d022d68                DRV_MEDIA_Write

.text.UDPSetBcastIPV4Address
                0x9d022e98      0x130
 .text.UDPSetBcastIPV4Address
                0x9d022e98      0x130 build/default/production/_ext/427700826/udp.o
                0x9d022e98                UDPSetBcastIPV4Address

.text.realloc   0x9d022fc8      0x130
 .text.realloc  0x9d022fc8      0x130 c:/program files (x86)/microchip/xc32/v1.21/bin/../lib/gcc/pic32mx/4.5.2/../../../../pic32mx/lib/size\libc.a(malloc.o)
                0x9d022fc8                realloc

.text.TCPIP_STACK_DeInit
                0x9d0230f8      0x12c
 .text.TCPIP_STACK_DeInit
                0x9d0230f8      0x12c build/default/production/_ext/427700826/tcpip_manager.o
                0x9d0230f8                TCPIP_STACK_DeInit

.text.DNSBeginUsage
                0x9d023224      0x128
 .text.DNSBeginUsage
                0x9d023224      0x128 build/default/production/_ext/427700826/dns.o
                0x9d023224                DNSBeginUsage

.text.fputc     0x9d02334c      0x128
 .text.fputc    0x9d02334c      0x128 c:/program files (x86)/microchip/xc32/v1.21/bin/../lib/gcc/pic32mx/4.5.2/../../../../pic32mx/lib/size\libc.a(_fputc_simple.o)
                0x9d02334c                fputc

.text.SYS_USERIO_Initialize
                0x9d023474      0x124
 .text.SYS_USERIO_Initialize
                0x9d023474      0x124 build/default/production/_ext/365611741/system_userio.o
                0x9d023474                SYS_USERIO_Initialize

.text.HTTPDeInit
                0x9d023598      0x124
 .text.HTTPDeInit
                0x9d023598      0x124 build/default/production/_ext/427700826/http2.o
                0x9d023598                HTTPDeInit

.text._TCPSendWinIncUpdate
                0x9d0236bc      0x124
 .text._TCPSendWinIncUpdate
                0x9d0236bc      0x124 build/default/production/_ext/427700826/tcp.o

.text.strtol    0x9d0237e0      0x124
 .text.strtol   0x9d0237e0      0x124 c:/program files (x86)/microchip/xc32/v1.21/bin/../lib/gcc/pic32mx/4.5.2/../../../../pic32mx/lib/size\libc.a(strtol.o)
                0x9d0237e0                strtol

.text.TCPIP_IPV4_QueuePacket
                0x9d023904      0x120
 .text.TCPIP_IPV4_QueuePacket
                0x9d023904      0x120 build/default/production/_ext/427700826/ipv4.o

.text.TCPOpenServer
                0x9d023a24      0x120
 .text.TCPOpenServer
                0x9d023a24      0x120 build/default/production/_ext/427700826/tcp.o
                0x9d023a24                TCPOpenServer

.text.UDPOpenServer
                0x9d023b44      0x120
 .text.UDPOpenServer
                0x9d023b44      0x120 build/default/production/_ext/427700826/udp.o
                0x9d023b44                UDPOpenServer

.text           0x9d023c64      0x120
 .text          0x9d023c64      0x120 c:/program files (x86)/microchip/xc32/v1.21/bin/../lib/gcc/pic32mx/4.5.2/../../../../pic32mx/lib/size\libpic32.a(strcmp.o)
                0x9d023c64                strcmp

.text.fround    0x9d023d84      0x120
 .text.fround   0x9d023d84      0x120 c:/program files (x86)/microchip/xc32/v1.21/bin/../lib/gcc/pic32mx/4.5.2/../../../../pic32mx/lib/size\libc.a(doprnt.o)

.text.SHA1AddData
                0x9d023ea4      0x11c
 .text.SHA1AddData
                0x9d023ea4      0x11c build/default/production/_ext/101875047/hashes.o
                0x9d023ea4                SHA1AddData

.text.BFSReg    0x9d023fc0      0x11c
 .text.BFSReg   0x9d023fc0      0x11c build/default/production/_ext/427700826/encs24j600.o

.text.BFCReg    0x9d0240dc      0x11c
 .text.BFCReg   0x9d0240dc      0x11c build/default/production/_ext/427700826/encs24j600.o

.text.b64_encode
                0x9d0241f8      0x11c
 .text.b64_encode
                0x9d0241f8      0x11c build/default/production/_ext/1472/tcp6_demo_app.o
                0x9d0241f8                b64_encode

.text.Execute3  0x9d024314      0x118
 .text.Execute3
                0x9d024314      0x118 build/default/production/_ext/427700826/encs24j600.o

.text.TCPIP_IPV4_Initialize
                0x9d02442c      0x118
 .text.TCPIP_IPV4_Initialize
                0x9d02442c      0x118 build/default/production/_ext/427700826/ipv4.o
                0x9d02442c                TCPIP_IPV4_Initialize

.text.SYS_FS_FSFromAbsPath
                0x9d024544      0x114
 .text.SYS_FS_FSFromAbsPath
                0x9d024544      0x114 build/default/production/_ext/97638081/sys_fs.o

.text.ENCX24J600_CalcIPBufferChecksum
                0x9d024658      0x114
 .text.ENCX24J600_CalcIPBufferChecksum
                0x9d024658      0x114 build/default/production/_ext/427700826/encs24j600.o
                0x9d024658                ENCX24J600_CalcIPBufferChecksum

.text.Execute2  0x9d02476c      0x114
 .text.Execute2
                0x9d02476c      0x114 build/default/production/_ext/427700826/encs24j600.o

.text.TCPIP_IPV4_PutHeader
                0x9d024880      0x114
 .text.TCPIP_IPV4_PutHeader
                0x9d024880      0x114 build/default/production/_ext/427700826/ipv4.o
                0x9d024880                TCPIP_IPV4_PutHeader

.text.DisplayIPValue
                0x9d024994      0x114
 .text.DisplayIPValue
                0x9d024994      0x114 build/default/production/_ext/1472/main_demo.o
                0x9d024994                DisplayIPValue

.text.MD5AddData
                0x9d024aa8      0x110
 .text.MD5AddData
                0x9d024aa8      0x110 build/default/production/_ext/101875047/hashes.o
                0x9d024aa8                MD5AddData

.text._flsbuf   0x9d024bb8      0x110
 .text._flsbuf  0x9d024bb8      0x110 c:/program files (x86)/microchip/xc32/v1.21/bin/../lib/gcc/pic32mx/4.5.2/../../../../pic32mx/lib/size\libc.a(_flsbuf_simple.o)
                0x9d024bb8                _flsbuf

.text._TcpSwapHeader
                0x9d024cc8      0x10c
 .text._TcpSwapHeader
                0x9d024cc8      0x10c build/default/production/_ext/427700826/tcp.o

.text.TCPIP_STACK_BringNetDown
                0x9d024dd4      0x108
 .text.TCPIP_STACK_BringNetDown
                0x9d024dd4      0x108 build/default/production/_ext/427700826/tcpip_manager.o

.text._DHCPClose
                0x9d024edc      0x104
 .text._DHCPClose
                0x9d024edc      0x104 build/default/production/_ext/427700826/dhcp.o

.rodata         0x9d024fe0      0x104
 .rodata        0x9d024fe0      0x104 c:/program files (x86)/microchip/xc32/v1.21/bin/../lib/gcc/pic32mx/4.5.2/../../../../pic32mx/lib/size\libc.a(ctype.o)
                0x9d024fe0                _ctype

.text.hexatob   0x9d0250e4      0x100
 .text.hexatob  0x9d0250e4      0x100 build/default/production/_ext/101875047/helpers.o
                0x9d0250e4                hexatob

.text.ToggleCRYPTEN
                0x9d0251e4       0xfc
 .text.ToggleCRYPTEN
                0x9d0251e4       0xfc build/default/production/_ext/427700826/encs24j600.o

.text.HTTPExecutePost
                0x9d0252e0       0xfc
 .text.HTTPExecutePost
                0x9d0252e0       0xfc build/default/production/_ext/1472/custom_http_app.o
                0x9d0252e0                HTTPExecutePost

.text.SYS_FS_IsAbsolutePath
                0x9d0253dc       0xf8
 .text.SYS_FS_IsAbsolutePath
                0x9d0253dc       0xf8 build/default/production/_ext/97638081/sys_fs.o

.text.ENCX24J600_MACFlush
                0x9d0254d4       0xf8
 .text.ENCX24J600_MACFlush
                0x9d0254d4       0xf8 build/default/production/_ext/427700826/encs24j600.o
                0x9d0254d4                ENCX24J600_MACFlush

.text._TCPIPStackAddressServiceEvent
                0x9d0255cc       0xf8
 .text._TCPIPStackAddressServiceEvent
                0x9d0255cc       0xf8 build/default/production/_ext/427700826/tcpip_manager.o
                0x9d0255cc                _TCPIPStackAddressServiceEvent

.text.SingleListRemoveNode
                0x9d0256c4       0xf8
 .text.SingleListRemoveNode
                0x9d0256c4       0xf8 build/default/production/_ext/427700826/tcpip_helpers.o
                0x9d0256c4                SingleListRemoveNode

.text.SYS_USERIO_DeviceDebounce
                0x9d0257bc       0xf4
 .text.SYS_USERIO_DeviceDebounce
                0x9d0257bc       0xf4 build/default/production/_ext/365611741/system_userio.o
                0x9d0257bc                SYS_USERIO_DeviceDebounce

.text.MPFSGetFilename
                0x9d0258b0       0xf4
 .text.MPFSGetFilename
                0x9d0258b0       0xf4 build/default/production/_ext/97638081/mpfs2.o
                0x9d0258b0                MPFSGetFilename

.text.UDPSetSourceIPAddress
                0x9d0259a4       0xf4
 .text.UDPSetSourceIPAddress
                0x9d0259a4       0xf4 build/default/production/_ext/427700826/udp.o
                0x9d0259a4                UDPSetSourceIPAddress

.text.UDPSetDestinationIPAddress
                0x9d025a98       0xf4
 .text.UDPSetDestinationIPAddress
                0x9d025a98       0xf4 build/default/production/_ext/427700826/udp.o
                0x9d025a98                UDPSetDestinationIPAddress

.text._ARPAddCompleteEntry
                0x9d025b8c       0xf0
 .text._ARPAddCompleteEntry
                0x9d025b8c       0xf0 build/default/production/_ext/427700826/arp.o

.text.UDPDiscard
                0x9d025c7c       0xf0
 .text.UDPDiscard
                0x9d025c7c       0xf0 build/default/production/_ext/427700826/udp.o
                0x9d025c7c                UDPDiscard

.text.NBNSPutName
                0x9d025d6c       0xec
 .text.NBNSPutName
                0x9d025d6c       0xec build/default/production/_ext/427700826/nbns.o

.text.TCPIsPutReady
                0x9d025e58       0xec
 .text.TCPIsPutReady
                0x9d025e58       0xec build/default/production/_ext/427700826/tcp.o
                0x9d025e58                TCPIsPutReady

.text._TCPIP_HEAP_CallocDebug
                0x9d025f44       0xec
 .text._TCPIP_HEAP_CallocDebug
                0x9d025f44       0xec build/default/production/_ext/427700826/tcpip_heap_alloc.o
                0x9d025f44                _TCPIP_HEAP_CallocDebug

.text.HTTPReadPostValue
                0x9d026030       0xe8
 .text.HTTPReadPostValue
                0x9d026030       0xe8 build/default/production/_ext/427700826/http2.o
                0x9d026030                HTTPReadPostValue

.text.DNSIsResolved
                0x9d026118       0xe8
 .text.DNSIsResolved
                0x9d026118       0xe8 build/default/production/_ext/427700826/dns.o
                0x9d026118                DNSIsResolved

.text.TCPIP_IPV4_PutUpperLayerHeader
                0x9d026200       0xe8
 .text.TCPIP_IPV4_PutUpperLayerHeader
                0x9d026200       0xe8 build/default/production/_ext/427700826/ipv4.o
                0x9d026200                TCPIP_IPV4_PutUpperLayerHeader

.text.UDPSetRxOffset
                0x9d0262e8       0xe8
 .text.UDPSetRxOffset
                0x9d0262e8       0xe8 build/default/production/_ext/427700826/udp.o
                0x9d0262e8                UDPSetRxOffset

.text.ProcessTCPIPTickEvent
                0x9d0263d0       0xe8
 .text.ProcessTCPIPTickEvent
                0x9d0263d0       0xe8 build/default/production/_ext/427700826/tcpip_manager.o

.rodata         0x9d0264b8       0xe8
 .rodata        0x9d0264b8       0xe8 c:/program files (x86)/microchip/xc32/v1.21/bin/../lib/gcc/pic32mx/4.5.2/../../../../pic32mx/lib/size\libc.a(doprnt.o)

.text.LCD_WRITE
                0x9d0265a0       0xe4
 .text.LCD_WRITE
                0x9d0265a0       0xe4 build/default/production/_ext/792872985/lcd.o
                0x9d0265a0                LCD_WRITE

.text.ENCX24J600_MACPutHeader
                0x9d026684       0xe4
 .text.ENCX24J600_MACPutHeader
                0x9d026684       0xe4 build/default/production/_ext/427700826/encs24j600.o
                0x9d026684                ENCX24J600_MACPutHeader

.text.ReadMemoryWindow
                0x9d026768       0xe4
 .text.ReadMemoryWindow
                0x9d026768       0xe4 build/default/production/_ext/427700826/encs24j600.o

.text.ReadN     0x9d02684c       0xe4
 .text.ReadN    0x9d02684c       0xe4 build/default/production/_ext/427700826/encs24j600.o

.text.WriteN    0x9d026930       0xe4
 .text.WriteN   0x9d026930       0xe4 build/default/production/_ext/427700826/encs24j600.o

.text.TCPIP_IPV4_ResetTransmitPacketState
                0x9d026a14       0xe4
 .text.TCPIP_IPV4_ResetTransmitPacketState
                0x9d026a14       0xe4 build/default/production/_ext/427700826/ipv4.o
                0x9d026a14                TCPIP_IPV4_ResetTransmitPacketState

.text.TCPIP_IPV4_AllocateDataSegmentHeader
                0x9d026af8       0xe4
 .text.TCPIP_IPV4_AllocateDataSegmentHeader
                0x9d026af8       0xe4 build/default/production/_ext/427700826/ipv4.o
                0x9d026af8                TCPIP_IPV4_AllocateDataSegmentHeader

.text.TCPDeInit
                0x9d026bdc       0xe4
 .text.TCPDeInit
                0x9d026bdc       0xe4 build/default/production/_ext/427700826/tcp.o
                0x9d026bdc                TCPDeInit

.text.TCPIP_HEAP_Delete
                0x9d026cc0       0xe4
 .text.TCPIP_HEAP_Delete
                0x9d026cc0       0xe4 build/default/production/_ext/427700826/tcpip_heap_alloc.o
                0x9d026cc0                TCPIP_HEAP_Delete

.text.SYS_TICK_TimerCreate
                0x9d026da4       0xe0
 .text.SYS_TICK_TimerCreate
                0x9d026da4       0xe0 build/default/production/_ext/365611741/system_services.o
                0x9d026da4                SYS_TICK_TimerCreate

.text._SYS_CMDIO_ADD
                0x9d026e84       0xe0
 .text._SYS_CMDIO_ADD
                0x9d026e84       0xe0 build/default/production/_ext/365611741/system_command.o
                0x9d026e84                _SYS_CMDIO_ADD

.text._ARPSetEntry
                0x9d026f64       0xe0
 .text._ARPSetEntry
                0x9d026f64       0xe0 build/default/production/_ext/427700826/arp.o

.text.ARPResolve
                0x9d027044       0xe0
 .text.ARPResolve
                0x9d027044       0xe0 build/default/production/_ext/427700826/arp.o
                0x9d027044                ARPResolve

.text.UDPPutArray
                0x9d027124       0xe0
 .text.UDPPutArray
                0x9d027124       0xe0 build/default/production/_ext/427700826/udp.o
                0x9d027124                UDPPutArray

.text._SYS_ERROR_PRINT
                0x9d027204       0xdc
 .text._SYS_ERROR_PRINT
                0x9d027204       0xdc build/default/production/_ext/365611741/system_debug.o
                0x9d027204                _SYS_ERROR_PRINT

.text.HTTPHeaderParseContentLength
                0x9d0272e0       0xdc
 .text.HTTPHeaderParseContentLength
                0x9d0272e0       0xdc build/default/production/_ext/427700826/http2.o

.text.ARPHashDeleteEntry
                0x9d0273bc       0xdc
 .text.ARPHashDeleteEntry
                0x9d0273bc       0xdc build/default/production/_ext/427700826/arp.o
                0x9d0273bc                ARPHashDeleteEntry

.text.DHCPConnectionHandler
                0x9d027498       0xdc
 .text.DHCPConnectionHandler
                0x9d027498       0xdc build/default/production/_ext/427700826/dhcp.o
                0x9d027498                DHCPConnectionHandler

.text._TcpCleanup
                0x9d027574       0xdc
 .text._TcpCleanup
                0x9d027574       0xdc build/default/production/_ext/427700826/tcp.o

.text.TCPOpenClient
                0x9d027650       0xdc
 .text.TCPOpenClient
                0x9d027650       0xdc build/default/production/_ext/427700826/tcp.o
                0x9d027650                TCPOpenClient

.text.TcpAllocateEphemeralPort
                0x9d02772c       0xdc
 .text.TcpAllocateEphemeralPort
                0x9d02772c       0xdc build/default/production/_ext/427700826/tcp.o

.text.UDPOpenClient
                0x9d027808       0xdc
 .text.UDPOpenClient
                0x9d027808       0xdc build/default/production/_ext/427700826/udp.o
                0x9d027808                UDPOpenClient

.text.UdpAllocateEphemeralPort
                0x9d0278e4       0xdc
 .text.UdpAllocateEphemeralPort
                0x9d0278e4       0xdc build/default/production/_ext/427700826/udp.o

.text.TCPIP_IPV4_GetPseudoHeaderChecksum
                0x9d0279c0       0xd8
 .text.TCPIP_IPV4_GetPseudoHeaderChecksum
                0x9d0279c0       0xd8 build/default/production/_ext/427700826/ipv4.o
                0x9d0279c0                TCPIP_IPV4_GetPseudoHeaderChecksum

.text._TCPIP_HEAP_MallocDebug
                0x9d027a98       0xd8
 .text._TCPIP_HEAP_MallocDebug
                0x9d027a98       0xd8 build/default/production/_ext/427700826/tcpip_heap_alloc.o
                0x9d027a98                _TCPIP_HEAP_MallocDebug

.text._SYS_RANDOM_INIT
                0x9d027b70       0xd4
 .text._SYS_RANDOM_INIT
                0x9d027b70       0xd4 build/default/production/_ext/365611741/system_random.o
                0x9d027b70                _SYS_RANDOM_INIT

.text.TCPIP_ANNOUNCE_Init
                0x9d027c44       0xd4
 .text.TCPIP_ANNOUNCE_Init
                0x9d027c44       0xd4 build/default/production/_ext/427700826/tcpip_announce.o
                0x9d027c44                TCPIP_ANNOUNCE_Init

.text._TcpAbort
                0x9d027d18       0xd4
 .text._TcpAbort
                0x9d027d18       0xd4 build/default/production/_ext/427700826/tcp.o

.text.TCPClose  0x9d027dec       0xd4
 .text.TCPClose
                0x9d027dec       0xd4 build/default/production/_ext/427700826/tcp.o
                0x9d027dec                TCPClose

.text           0x9d027ec0       0xd4
 .text          0x9d027ec0       0xd4 c:/program files (x86)/microchip/xc32/v1.21/bin/../lib/gcc/pic32mx/4.5.2/size\libgcc.a(_floatundisf.o)
                0x9d027ec0                __floatundisf

.text.HTTPGetArg
                0x9d027f94       0xd0
 .text.HTTPGetArg
                0x9d027f94       0xd0 build/default/production/_ext/427700826/http2.o
                0x9d027f94                HTTPGetArg

.text._ARPDeleteResources
                0x9d028064       0xd0
 .text._ARPDeleteResources
                0x9d028064       0xd0 build/default/production/_ext/427700826/arp.o

.text.fnv_32_hash
                0x9d028134       0xd0
 .text.fnv_32_hash
                0x9d028134       0xd0 build/default/production/_ext/427700826/hash_fnv.o
                0x9d028134                fnv_32_hash

.text._TcpSocketInitialize
                0x9d028204       0xd0
 .text._TcpSocketInitialize
                0x9d028204       0xd0 build/default/production/_ext/427700826/tcp.o

.text.UDPSetOptions
                0x9d0282d4       0xd0
 .text.UDPSetOptions
                0x9d0282d4       0xd0 build/default/production/_ext/427700826/udp.o
                0x9d0282d4                UDPSetOptions

.text.general_exception
                0x9d0283a4       0xd0
 .text.general_exception
                0x9d0283a4       0xd0 c:/program files (x86)/microchip/xc32/v1.21/bin/../lib/gcc/pic32mx/4.5.2/../../../../pic32mx/lib/size\libpic32.a(general-exception.o)
                0x9d0283a4                _general_exception_context

.rodata         0x9d028478       0xd0
 .rodata        0x9d028478       0xd0 c:/program files (x86)/microchip/xc32/v1.21/bin/../lib/gcc/pic32mx/4.5.2/../../../../pic32mx/lib/size\libc.a(doprnt_cdnopsuxX.eo)

.text.DRV_MEDIA_WriteSetOffset
                0x9d028548       0xcc
 .text.DRV_MEDIA_WriteSetOffset
                0x9d028548       0xcc build/default/production/_ext/792872985/drv_media.o
                0x9d028548                DRV_MEDIA_WriteSetOffset

.text.HTTPSetMediaWriteHeader
                0x9d028614       0xcc
 .text.HTTPSetMediaWriteHeader
                0x9d028614       0xcc build/default/production/_ext/427700826/http2.o

.text.ENCX24J600_MACPowerDown
                0x9d0286e0       0xcc
 .text.ENCX24J600_MACPowerDown
                0x9d0286e0       0xcc build/default/production/_ext/427700826/encs24j600.o
                0x9d0286e0                ENCX24J600_MACPowerDown

.text.WriteMemoryWindow
                0x9d0287ac       0xcc
 .text.WriteMemoryWindow
                0x9d0287ac       0xcc build/default/production/_ext/427700826/encs24j600.o

.text.TCPIP_IPV4_SetPayload
                0x9d028878       0xcc
 .text.TCPIP_IPV4_SetPayload
                0x9d028878       0xcc build/default/production/_ext/427700826/ipv4.o
                0x9d028878                TCPIP_IPV4_SetPayload

.text.DNSRetry  0x9d028944       0xc8
 .text.DNSRetry
                0x9d028944       0xc8 build/default/production/_ext/427700826/dns.o

.text.DNSDiscardName
                0x9d028a0c       0xc8
 .text.DNSDiscardName
                0x9d028a0c       0xc8 build/default/production/_ext/427700826/dns.o

.text.UDPClose  0x9d028ad4       0xc8
 .text.UDPClose
                0x9d028ad4       0xc8 build/default/production/_ext/427700826/udp.o
                0x9d028ad4                UDPClose

.text.UDPSetTxOffset
                0x9d028b9c       0xc8
 .text.UDPSetTxOffset
                0x9d028b9c       0xc8 build/default/production/_ext/427700826/udp.o
                0x9d028b9c                UDPSetTxOffset

.text.InitNetConfig
                0x9d028c64       0xc8
 .text.InitNetConfig
                0x9d028c64       0xc8 build/default/production/_ext/427700826/tcpip_manager.o

.text.TCPIP_Helper_FormatNetBIOSName
                0x9d028d2c       0xc8
 .text.TCPIP_Helper_FormatNetBIOSName
                0x9d028d2c       0xc8 build/default/production/_ext/427700826/tcpip_helpers.o
                0x9d028d2c                TCPIP_Helper_FormatNetBIOSName

.text.HTTPPrintIP
                0x9d028df4       0xc8
 .text.HTTPPrintIP
                0x9d028df4       0xc8 build/default/production/_ext/1472/custom_http_app.o
                0x9d028df4                HTTPPrintIP

.text.CmdAddHead
                0x9d028ebc       0xc4
 .text.CmdAddHead
                0x9d028ebc       0xc4 build/default/production/_ext/365611741/system_command.o

.text.MPFSInit  0x9d028f80       0xc4
 .text.MPFSInit
                0x9d028f80       0xc4 build/default/production/_ext/97638081/mpfs2.o
                0x9d028f80                MPFSInit

.text._LoadFATRecord
                0x9d029044       0xc4
 .text._LoadFATRecord
                0x9d029044       0xc4 build/default/production/_ext/97638081/mpfs2.o

.text._DHCPEnable
                0x9d029108       0xc4
 .text._DHCPEnable
                0x9d029108       0xc4 build/default/production/_ext/427700826/dhcp.o

.text.SYS_TICK_Initialize
                0x9d0291cc       0xc0
 .text.SYS_TICK_Initialize
                0x9d0291cc       0xc0 build/default/production/_ext/365611741/system_services.o
                0x9d0291cc                SYS_TICK_Initialize

.text._SYS_COMMAND_INIT
                0x9d02928c       0xbc
 .text._SYS_COMMAND_INIT
                0x9d02928c       0xbc build/default/production/_ext/365611741/system_command.o
                0x9d02928c                _SYS_COMMAND_INIT

.text.XEEInit   0x9d029348       0xbc
 .text.XEEInit  0x9d029348       0xbc build/default/production/_ext/792872985/spi_eeprom.o
                0x9d029348                XEEInit

.text._ARPRemoveEntry
                0x9d029404       0xbc
 .text._ARPRemoveEntry
                0x9d029404       0xbc build/default/production/_ext/427700826/arp.o

.text.ENCX24_MACInitialize
                0x9d0294c0       0xbc
 .text.ENCX24_MACInitialize
                0x9d0294c0       0xbc build/default/production/_ext/427700826/encx24_mac.o
                0x9d0294c0                ENCX24_MACInitialize

.text.OAHashRemoveAll
                0x9d02957c       0xbc
 .text.OAHashRemoveAll
                0x9d02957c       0xbc build/default/production/_ext/427700826/hash_tbl.o
                0x9d02957c                OAHashRemoveAll

.text.UDPDiscardNet
                0x9d029638       0xbc
 .text.UDPDiscardNet
                0x9d029638       0xbc build/default/production/_ext/427700826/udp.o
                0x9d029638                UDPDiscardNet

.text.TCPIP_Helper_StringToPowerMode
                0x9d0296f4       0xbc
 .text.TCPIP_Helper_StringToPowerMode
                0x9d0296f4       0xbc build/default/production/_ext/427700826/tcpip_helpers.o
                0x9d0296f4                TCPIP_Helper_StringToPowerMode

.text._SYS_DEBUG_INIT
                0x9d0297b0       0xb8
 .text._SYS_DEBUG_INIT
                0x9d0297b0       0xb8 build/default/production/_ext/365611741/system_debug.o
                0x9d0297b0                _SYS_DEBUG_INIT

.text._SYS_CONSOLE_INIT
                0x9d029868       0xb8
 .text._SYS_CONSOLE_INIT
                0x9d029868       0xb8 build/default/production/_ext/365611741/system_debug.o
                0x9d029868                _SYS_CONSOLE_INIT

.text.Execute0  0x9d029920       0xb8
 .text.Execute0
                0x9d029920       0xb8 build/default/production/_ext/427700826/encs24j600.o

.text.TCPv4AllocateTxPacketStruct
                0x9d0299d8       0xb8
 .text.TCPv4AllocateTxPacketStruct
                0x9d0299d8       0xb8 build/default/production/_ext/427700826/tcp.o

.text._TCPIsGetReady
                0x9d029a90       0xb8
 .text._TCPIsGetReady
                0x9d029a90       0xb8 build/default/production/_ext/427700826/tcp.o

.text.UDPGetTxCount
                0x9d029b48       0xb8
 .text.UDPGetTxCount
                0x9d029b48       0xb8 build/default/production/_ext/427700826/udp.o
                0x9d029b48                UDPGetTxCount

.text.MPFSGetEndAddr
                0x9d029c00       0xb4
 .text.MPFSGetEndAddr
                0x9d029c00       0xb4 build/default/production/_ext/97638081/mpfs2.o
                0x9d029c00                MPFSGetEndAddr

.text.Delay10us
                0x9d029cb4       0xb4
 .text.Delay10us
                0x9d029cb4       0xb4 build/default/production/_ext/792872985/lcd.o
                0x9d029cb4                Delay10us

.text._TcpMac2RamCopy
                0x9d029d68       0xb4
 .text._TcpMac2RamCopy
                0x9d029d68       0xb4 build/default/production/_ext/427700826/tcp.o

.text.UDPv4AllocateTxPacketStruct
                0x9d029e1c       0xb4
 .text.UDPv4AllocateTxPacketStruct
                0x9d029e1c       0xb4 build/default/production/_ext/427700826/udp.o

.text.UDPIsTxPutReady
                0x9d029ed0       0xb4
 .text.UDPIsTxPutReady
                0x9d029ed0       0xb4 build/default/production/_ext/427700826/udp.o
                0x9d029ed0                UDPIsTxPutReady

.text._mon_putc
                0x9d029f84       0xb4
 .text._mon_putc
                0x9d029f84       0xb4 c:/program files (x86)/microchip/xc32/v1.21/bin/../lib/gcc/pic32mx/4.5.2/../../../../pic32mx/lib/size\libpic32.a(_mon_putc.o)
                0x9d029f84                _mon_putc

.text.CommandQuit
                0x9d02a038       0xb0
 .text.CommandQuit
                0x9d02a038       0xb0 build/default/production/_ext/365611741/system_command.o

.text.CmdRemoveTail
                0x9d02a0e8       0xb0
 .text.CmdRemoveTail
                0x9d02a0e8       0xb0 build/default/production/_ext/365611741/system_command.o

.text.TCPIP_ANNOUNCE_DeInit
                0x9d02a198       0xb0
 .text.TCPIP_ANNOUNCE_DeInit
                0x9d02a198       0xb0 build/default/production/_ext/427700826/tcpip_announce.o
                0x9d02a198                TCPIP_ANNOUNCE_DeInit

.text._ARPRemoveCacheEntries
                0x9d02a248       0xb0
 .text._ARPRemoveCacheEntries
                0x9d02a248       0xb0 build/default/production/_ext/427700826/arp.o

.text._ARPNotifyClients
                0x9d02a2f8       0xb0
 .text._ARPNotifyClients
                0x9d02a2f8       0xb0 build/default/production/_ext/427700826/arp.o

.text.ENCX24J600_MACGetArray
                0x9d02a3a8       0xb0
 .text.ENCX24J600_MACGetArray
                0x9d02a3a8       0xb0 build/default/production/_ext/427700826/encs24j600.o
                0x9d02a3a8                ENCX24J600_MACGetArray

.text._Tcpv4AckFnc
                0x9d02a458       0xb0
 .text._Tcpv4AckFnc
                0x9d02a458       0xb0 build/default/production/_ext/427700826/tcp.o

.text._TCPIPStackSetNetAddress
                0x9d02a508       0xb0
 .text._TCPIPStackSetNetAddress
                0x9d02a508       0xb0 build/default/production/_ext/427700826/tcpip_manager.o
                0x9d02a508                _TCPIPStackSetNetAddress

.text.MPFSGetFlags
                0x9d02a5b8       0xac
 .text.MPFSGetFlags
                0x9d02a5b8       0xac build/default/production/_ext/97638081/mpfs2.o
                0x9d02a5b8                MPFSGetFlags

.text.MPFSGetSize
                0x9d02a664       0xac
 .text.MPFSGetSize
                0x9d02a664       0xac build/default/production/_ext/97638081/mpfs2.o
                0x9d02a664                MPFSGetSize

.text.MPFSGetStartAddr
                0x9d02a710       0xac
 .text.MPFSGetStartAddr
                0x9d02a710       0xac build/default/production/_ext/97638081/mpfs2.o
                0x9d02a710                MPFSGetStartAddr

.rodata         0x9d02a7bc       0xac
 .rodata        0x9d02a7bc       0xac build/default/production/_ext/427700826/tcp.o

.text.TCPIsConnected
                0x9d02a868       0xac
 .text.TCPIsConnected
                0x9d02a868       0xac build/default/production/_ext/427700826/tcp.o
                0x9d02a868                TCPIsConnected

.text.HTTPPrint_cookiename
                0x9d02a914       0xac
 .text.HTTPPrint_cookiename
                0x9d02a914       0xac build/default/production/_ext/1472/custom_http_app.o
                0x9d02a914                HTTPPrint_cookiename

.text._SYS_ERROR
                0x9d02a9c0       0xa8
 .text._SYS_ERROR
                0x9d02a9c0       0xa8 build/default/production/_ext/365611741/system_debug.o
                0x9d02a9c0                _SYS_ERROR

.text.ARPDeinitialize
                0x9d02aa68       0xa8
 .text.ARPDeinitialize
                0x9d02aa68       0xa8 build/default/production/_ext/427700826/arp.o
                0x9d02aa68                ARPDeinitialize

.text.ENCX24J600_MACPowerUp
                0x9d02ab10       0xa8
 .text.ENCX24J600_MACPowerUp
                0x9d02ab10       0xa8 build/default/production/_ext/427700826/encs24j600.o
                0x9d02ab10                ENCX24J600_MACPowerUp

.text._TCPIPStackStringToMACId
                0x9d02abb8       0xa8
 .text._TCPIPStackStringToMACId
                0x9d02abb8       0xa8 build/default/production/_ext/427700826/tcpip_manager.o
                0x9d02abb8                _TCPIPStackStringToMACId

.text           0x9d02ac60       0xa8
 .text          0x9d02ac60       0xa8 c:/program files (x86)/microchip/xc32/v1.21/bin/../lib/gcc/pic32mx/4.5.2/../../../../pic32mx/lib/size\libpic32.a(memset.o)
                0x9d02ac60                memset

.text._Validate
                0x9d02ad08       0xa4
 .text._Validate
                0x9d02ad08       0xa4 build/default/production/_ext/97638081/mpfs2.o

.text.XEEWriteArray
                0x9d02adac       0xa4
 .text.XEEWriteArray
                0x9d02adac       0xa4 build/default/production/_ext/792872985/spi_eeprom.o
                0x9d02adac                XEEWriteArray

.text.DNSResolve
                0x9d02ae50       0xa4
 .text.DNSResolve
                0x9d02ae50       0xa4 build/default/production/_ext/427700826/dns.o
                0x9d02ae50                DNSResolve

.text.ReadPHYReg
                0x9d02aef4       0xa4
 .text.ReadPHYReg
                0x9d02aef4       0xa4 build/default/production/_ext/427700826/encs24j600.o

.text._ICMPAllocateTxPacketStruct
                0x9d02af98       0xa4
 .text._ICMPAllocateTxPacketStruct
                0x9d02af98       0xa4 build/default/production/_ext/427700826/icmp.o

.text.TCPIP_IPV4_DeInitialize
                0x9d02b03c       0xa4
 .text.TCPIP_IPV4_DeInitialize
                0x9d02b03c       0xa4 build/default/production/_ext/427700826/ipv4.o
                0x9d02b03c                TCPIP_IPV4_DeInitialize

.text._TCPIPStackNetByAddress
                0x9d02b0e0       0xa4
 .text._TCPIPStackNetByAddress
                0x9d02b0e0       0xa4 build/default/production/_ext/427700826/tcpip_manager.o
                0x9d02b0e0                _TCPIPStackNetByAddress

.text.HTTPPrint_hellomsg
                0x9d02b184       0xa4
 .text.HTTPPrint_hellomsg
                0x9d02b184       0xa4 build/default/production/_ext/1472/custom_http_app.o
                0x9d02b184                HTTPPrint_hellomsg

.text._sbrk     0x9d02b228       0xa4
 .text._sbrk    0x9d02b228       0xa4 c:/program files (x86)/microchip/xc32/v1.21/bin/../lib/gcc/pic32mx/4.5.2/../../../../pic32mx/lib/size\libpic32.a(sbrk.o)
                0x9d02b228                _sbrk

.text.USART_GETS
                0x9d02b2cc       0xa0
 .text.USART_GETS
                0x9d02b2cc       0xa0 build/default/production/_ext/792872985/usart.o
                0x9d02b2cc                USART_GETS

.text.XEEWrite  0x9d02b36c       0xa0
 .text.XEEWrite
                0x9d02b36c       0xa0 build/default/production/_ext/792872985/spi_eeprom.o
                0x9d02b36c                XEEWrite

.text._DHCPDiscard
                0x9d02b40c       0xa0
 .text._DHCPDiscard
                0x9d02b40c       0xa0 build/default/production/_ext/427700826/dhcp.o

.text._DHCPNotifyClients
                0x9d02b4ac       0xa0
 .text._DHCPNotifyClients
                0x9d02b4ac       0xa0 build/default/production/_ext/427700826/dhcp.o

.text.ENCX24J600_MACDiscardRx
                0x9d02b54c       0xa0
 .text.ENCX24J600_MACDiscardRx
                0x9d02b54c       0xa0 build/default/production/_ext/427700826/encs24j600.o
                0x9d02b54c                ENCX24J600_MACDiscardRx

.text._UdpSocketDcpt
                0x9d02b5ec       0xa0
 .text._UdpSocketDcpt
                0x9d02b5ec       0xa0 build/default/production/_ext/427700826/udp.o

.text.HTTPPrint_builddate
                0x9d02b68c       0xa0
 .text.HTTPPrint_builddate
                0x9d02b68c       0xa0 build/default/production/_ext/1472/custom_http_app.o
                0x9d02b68c                HTTPPrint_builddate

.rodata         0x9d02b72c       0xa0
 .rodata        0x9d02b72c       0xa0 c:/program files (x86)/microchip/xc32/v1.21/bin/../lib/gcc/pic32mx/4.5.2/../../../../pic32mx/lib/size\libmchp_peripheral_32MX795F512L.a(spi_io_tbl_libp.o)
                0x9d02b72c                _SpiIoTbl

.text.strupr    0x9d02b7cc       0x9c
 .text.strupr   0x9d02b7cc       0x9c build/default/production/_ext/101875047/helpers.o
                0x9d02b7cc                strupr

.text.ANNOUNCE_Notify
                0x9d02b868       0x9c
 .text.ANNOUNCE_Notify
                0x9d02b868       0x9c build/default/production/_ext/427700826/tcpip_announce.o

.text.DHCPRegisterHandler
                0x9d02b904       0x9c
 .text.DHCPRegisterHandler
                0x9d02b904       0x9c build/default/production/_ext/427700826/dhcp.o
                0x9d02b904                DHCPRegisterHandler

.text._TcpSocketKill
                0x9d02b9a0       0x9c
 .text._TcpSocketKill
                0x9d02b9a0       0x9c build/default/production/_ext/427700826/tcp.o

.text.TCPIsAvailablePort
                0x9d02ba3c       0x9c
 .text.TCPIsAvailablePort
                0x9d02ba3c       0x9c build/default/production/_ext/427700826/tcp.o

.text.UdpIsAvailablePort
                0x9d02bad8       0x9c
 .text.UdpIsAvailablePort
                0x9d02bad8       0x9c build/default/production/_ext/427700826/udp.o

.text._TCPIPStackMacIdToNet
                0x9d02bb74       0x9c
 .text._TCPIPStackMacIdToNet
                0x9d02bb74       0x9c build/default/production/_ext/427700826/tcpip_manager.o
                0x9d02bb74                _TCPIPStackMacIdToNet

.text.SingleListRemoveHead
                0x9d02bc10       0x9c
 .text.SingleListRemoveHead
                0x9d02bc10       0x9c build/default/production/_ext/427700826/tcpip_helpers.o
                0x9d02bc10                SingleListRemoveHead

.text.HTTPPrint_ddns_status_msg
                0x9d02bcac       0x9c
 .text.HTTPPrint_ddns_status_msg
                0x9d02bcac       0x9c build/default/production/_ext/1472/custom_http_app.o
                0x9d02bcac                HTTPPrint_ddns_status_msg

.text._SYS_DEBUG_OPEN
                0x9d02bd48       0x98
 .text._SYS_DEBUG_OPEN
                0x9d02bd48       0x98 build/default/production/_ext/365611741/system_debug.o
                0x9d02bd48                _SYS_DEBUG_OPEN

.text._SYS_ASSERT
                0x9d02bde0       0x98
 .text._SYS_ASSERT
                0x9d02bde0       0x98 build/default/production/_ext/365611741/system_debug.o
                0x9d02bde0                _SYS_ASSERT

.text._SYS_CONSOLE_OPEN
                0x9d02be78       0x98
 .text._SYS_CONSOLE_OPEN
                0x9d02be78       0x98 build/default/production/_ext/365611741/system_debug.o
                0x9d02be78                _SYS_CONSOLE_OPEN

.text.MPFSDeinit
                0x9d02bf10       0x98
 .text.MPFSDeinit
                0x9d02bf10       0x98 build/default/production/_ext/97638081/mpfs2.o
                0x9d02bf10                MPFSDeinit

.text.DelayMs   0x9d02bfa8       0x98
 .text.DelayMs  0x9d02bfa8       0x98 build/default/production/_ext/792872985/lcd.o
                0x9d02bfa8                DelayMs

.text           0x9d02c040       0x98
 .text          0x9d02c040       0x98 c:/program files (x86)/microchip/xc32/v1.21/bin/../lib/gcc/pic32mx/4.5.2/../../../../pic32mx/lib/size\libpic32.a(memcmp.o)
                0x9d02c040                memcmp

.text.HTTPHeaderParseLookup
                0x9d02c0d8       0x94
 .text.HTTPHeaderParseLookup
                0x9d02c0d8       0x94 build/default/production/_ext/427700826/http2.o

.text.TCPWasReset
                0x9d02c16c       0x94
 .text.TCPWasReset
                0x9d02c16c       0x94 build/default/production/_ext/427700826/tcp.o
                0x9d02c16c                TCPWasReset

.text.TCP_PutArray
                0x9d02c200       0x94
 .text.TCP_PutArray
                0x9d02c200       0x94 build/default/production/_ext/427700826/tcp.o

.text.SingleListAddTail
                0x9d02c294       0x94
 .text.SingleListAddTail
                0x9d02c294       0x94 build/default/production/_ext/427700826/tcpip_helpers.o
                0x9d02c294                SingleListAddTail

.text.USART_PRINT
                0x9d02c328       0x90
 .text.USART_PRINT
                0x9d02c328       0x90 build/default/production/_ext/792872985/usart.o
                0x9d02c328                USART_PRINT

.text._HttpCleanup
                0x9d02c3b8       0x90
 .text._HttpCleanup
                0x9d02c3b8       0x90 build/default/production/_ext/427700826/http2.o

.text.DHCPIsBound
                0x9d02c448       0x90
 .text.DHCPIsBound
                0x9d02c448       0x90 build/default/production/_ext/427700826/dhcp.o
                0x9d02c448                DHCPIsBound

.text.TCPIP_IPV4_FreePacketData
                0x9d02c4d8       0x90
 .text.TCPIP_IPV4_FreePacketData
                0x9d02c4d8       0x90 build/default/production/_ext/427700826/ipv4.o
                0x9d02c4d8                TCPIP_IPV4_FreePacketData

.text.NBNSDeInit
                0x9d02c568       0x90
 .text.NBNSDeInit
                0x9d02c568       0x90 build/default/production/_ext/427700826/nbns.o
                0x9d02c568                NBNSDeInit

.text.TCPDiscard
                0x9d02c5f8       0x90
 .text.TCPDiscard
                0x9d02c5f8       0x90 build/default/production/_ext/427700826/tcp.o
                0x9d02c5f8                TCPDiscard

.text.TCP_SetPayload
                0x9d02c688       0x90
 .text.TCP_SetPayload
                0x9d02c688       0x90 build/default/production/_ext/427700826/tcp.o

.text.atol      0x9d02c718       0x90
 .text.atol     0x9d02c718       0x90 c:/program files (x86)/microchip/xc32/v1.21/bin/../lib/gcc/pic32mx/4.5.2/../../../../pic32mx/lib/size\libc.a(atol.o)
                0x9d02c718                atol

.text.SYS_TICK_MsDelay
                0x9d02c7a8       0x8c
 .text.SYS_TICK_MsDelay
                0x9d02c7a8       0x8c build/default/production/_ext/365611741/system_services.o
                0x9d02c7a8                SYS_TICK_MsDelay

.text.SYS_TICK_UsDelay
                0x9d02c834       0x8c
 .text.SYS_TICK_UsDelay
                0x9d02c834       0x8c build/default/production/_ext/365611741/system_services.o
                0x9d02c834                SYS_TICK_UsDelay

.text.HTTPReadPostName
                0x9d02c8c0       0x8c
 .text.HTTPReadPostName
                0x9d02c8c0       0x8c build/default/production/_ext/427700826/http2.o
                0x9d02c8c0                HTTPReadPostName

.text.SwapARPPacket
                0x9d02c94c       0x8c
 .text.SwapARPPacket
                0x9d02c94c       0x8c build/default/production/_ext/427700826/arp.o

.text.DNSClientInit
                0x9d02c9d8       0x8c
 .text.DNSClientInit
                0x9d02c9d8       0x8c build/default/production/_ext/427700826/dns.o
                0x9d02c9d8                DNSClientInit

.text.WritePHYReg
                0x9d02ca64       0x8c
 .text.WritePHYReg
                0x9d02ca64       0x8c build/default/production/_ext/427700826/encs24j600.o

.text.SwapIPV4Header
                0x9d02caf0       0x8c
 .text.SwapIPV4Header
                0x9d02caf0       0x8c build/default/production/_ext/427700826/ipv4.o

.text.UDPFlush  0x9d02cb7c       0x8c
 .text.UDPFlush
                0x9d02cb7c       0x8c build/default/production/_ext/427700826/udp.o
                0x9d02cb7c                UDPFlush

.text.UDPRemoteBind
                0x9d02cc08       0x8c
 .text.UDPRemoteBind
                0x9d02cc08       0x8c build/default/production/_ext/427700826/udp.o
                0x9d02cc08                UDPRemoteBind

.text.HTTPNeedsAuth
                0x9d02cc94       0x8c
 .text.HTTPNeedsAuth
                0x9d02cc94       0x8c build/default/production/_ext/1472/custom_http_app.o
                0x9d02cc94                HTTPNeedsAuth

.text.HTTPPrint_status_ok
                0x9d02cd20       0x8c
 .text.HTTPPrint_status_ok
                0x9d02cd20       0x8c build/default/production/_ext/1472/custom_http_app.o
                0x9d02cd20                HTTPPrint_status_ok

.text.HTTPPrint_status_fail
                0x9d02cdac       0x8c
 .text.HTTPPrint_status_fail
                0x9d02cdac       0x8c build/default/production/_ext/1472/custom_http_app.o
                0x9d02cdac                HTTPPrint_status_fail

.text.write     0x9d02ce38       0x8c
 .text.write    0x9d02ce38       0x8c c:/program files (x86)/microchip/xc32/v1.21/bin/../lib/gcc/pic32mx/4.5.2/../../../../pic32mx/lib/size\libpic32.a(write.o)
                0x9d02ce38                write

.text.SHA1Initialize
                0x9d02cec4       0x88
 .text.SHA1Initialize
                0x9d02cec4       0x88 build/default/production/_ext/101875047/hashes.o
                0x9d02cec4                SHA1Initialize

.text._SysGetCDevEntry
                0x9d02cf4c       0x88
 .text._SysGetCDevEntry
                0x9d02cf4c       0x88 build/default/production/_ext/365611741/system_debug.o

.text.DHCPDeInit
                0x9d02cfd4       0x88
 .text.DHCPDeInit
                0x9d02cfd4       0x88 build/default/production/_ext/427700826/dhcp.o
                0x9d02cfd4                DHCPDeInit

.text.TCP_IsTxPutReady
                0x9d02d05c       0x88
 .text.TCP_IsTxPutReady
                0x9d02d05c       0x88 build/default/production/_ext/427700826/tcp.o

.text.TCP_PutHeader
                0x9d02d0e4       0x88
 .text.TCP_PutHeader
                0x9d02d0e4       0x88 build/default/production/_ext/427700826/tcp.o

.text._TCPIPStackIpAddToNet
                0x9d02d16c       0x88
 .text._TCPIPStackIpAddToNet
                0x9d02d16c       0x88 build/default/production/_ext/427700826/tcpip_manager.o
                0x9d02d16c                _TCPIPStackIpAddToNet

.text._TCPIPStackMACIdToString
                0x9d02d1f4       0x88
 .text._TCPIPStackMACIdToString
                0x9d02d1f4       0x88 build/default/production/_ext/427700826/tcpip_manager.o
                0x9d02d1f4                _TCPIPStackMACIdToString

.text.TCPIP_STACK_NetBcastAddress
                0x9d02d27c       0x88
 .text.TCPIP_STACK_NetBcastAddress
                0x9d02d27c       0x88 build/default/production/_ext/427700826/tcpip_manager.o
                0x9d02d27c                TCPIP_STACK_NetBcastAddress

.text.LFSRSeedRand
                0x9d02d304       0x84
 .text.LFSRSeedRand
                0x9d02d304       0x84 build/default/production/_ext/101875047/lfsr.o
                0x9d02d304                LFSRSeedRand

.text._SYS_CONSOLE_PRINT
                0x9d02d388       0x84
 .text._SYS_CONSOLE_PRINT
                0x9d02d388       0x84 build/default/production/_ext/365611741/system_debug.o
                0x9d02d388                _SYS_CONSOLE_PRINT

.text.DRV_MEDIA_ReadSetOffset
                0x9d02d40c       0x84
 .text.DRV_MEDIA_ReadSetOffset
                0x9d02d40c       0x84 build/default/production/_ext/792872985/drv_media.o
                0x9d02d40c                DRV_MEDIA_ReadSetOffset

.text.ENCX24_MACPowerMode
                0x9d02d490       0x84
 .text.ENCX24_MACPowerMode
                0x9d02d490       0x84 build/default/production/_ext/427700826/encx24_mac.o

.text.OAHashInit
                0x9d02d514       0x84
 .text.OAHashInit
                0x9d02d514       0x84 build/default/production/_ext/427700826/hash_tbl.o
                0x9d02d514                OAHashInit

.text._TCPIP_HEAP_Calloc
                0x9d02d598       0x84
 .text._TCPIP_HEAP_Calloc
                0x9d02d598       0x84 build/default/production/_ext/427700826/tcpip_heap_alloc.o
                0x9d02d598                _TCPIP_HEAP_Calloc

.text.TcpipStackFindModuleData
                0x9d02d61c       0x84
 .text.TcpipStackFindModuleData
                0x9d02d61c       0x84 build/default/production/_ext/427700826/tcpip_manager.o

.text.TcpipStackFindMacModule
                0x9d02d6a0       0x84
 .text.TcpipStackFindMacModule
                0x9d02d6a0       0x84 build/default/production/_ext/427700826/tcpip_manager.o

.text.HTTPCheckAuth
                0x9d02d724       0x84
 .text.HTTPCheckAuth
                0x9d02d724       0x84 build/default/production/_ext/1472/custom_http_app.o
                0x9d02d724                HTTPCheckAuth

.text.atoi      0x9d02d7a8       0x84
 .text.atoi     0x9d02d7a8       0x84 c:/program files (x86)/microchip/xc32/v1.21/bin/../lib/gcc/pic32mx/4.5.2/../../../../pic32mx/lib/size\libc.a(atoi.o)
                0x9d02d7a8                atoi

.text.TCPIP_IPV4_FlushDataSegments
                0x9d02d82c       0x80
 .text.TCPIP_IPV4_FlushDataSegments
                0x9d02d82c       0x80 build/default/production/_ext/427700826/ipv4.o
                0x9d02d82c                TCPIP_IPV4_FlushDataSegments

.text.TCPDisconnect
                0x9d02d8ac       0x80
 .text.TCPDisconnect
                0x9d02d8ac       0x80 build/default/production/_ext/427700826/tcp.o
                0x9d02d8ac                TCPDisconnect

.text.TCP_IsTxReady
                0x9d02d92c       0x80
 .text.TCP_IsTxReady
                0x9d02d92c       0x80 build/default/production/_ext/427700826/tcp.o

.text.TCP_CopyTxPacketStruct
                0x9d02d9ac       0x80
 .text.TCP_CopyTxPacketStruct
                0x9d02d9ac       0x80 build/default/production/_ext/427700826/tcp.o

.text._Udpv4AckFnc
                0x9d02da2c       0x80
 .text._Udpv4AckFnc
                0x9d02da2c       0x80 build/default/production/_ext/427700826/udp.o

.text._SYS_CMDIO_GET_HANDLE
                0x9d02daac       0x7c
 .text._SYS_CMDIO_GET_HANDLE
                0x9d02daac       0x7c build/default/production/_ext/365611741/system_command.o
                0x9d02daac                _SYS_CMDIO_GET_HANDLE

.text.SYS_FS_setdefdir
                0x9d02db28       0x7c
 .text.SYS_FS_setdefdir
                0x9d02db28       0x7c build/default/production/_ext/97638081/sys_fs.o
                0x9d02db28                SYS_FS_setdefdir

.text.TCPFind   0x9d02dba4       0x7c
 .text.TCPFind  0x9d02dba4       0x7c build/default/production/_ext/427700826/tcp.o
                0x9d02dba4                TCPFind

.text.TCP_Flush
                0x9d02dc20       0x7c
 .text.TCP_Flush
                0x9d02dc20       0x7c build/default/production/_ext/427700826/tcp.o

.text._TCPIPStackAddressServiceSelect
                0x9d02dc9c       0x7c
 .text._TCPIPStackAddressServiceSelect
                0x9d02dc9c       0x7c build/default/production/_ext/427700826/tcpip_manager.o
                0x9d02dc9c                _TCPIPStackAddressServiceSelect

.text.HTTPPrint_config_dhcpchecked
                0x9d02dd18       0x7c
 .text.HTTPPrint_config_dhcpchecked
                0x9d02dd18       0x7c build/default/production/_ext/1472/custom_http_app.o
                0x9d02dd18                HTTPPrint_config_dhcpchecked

.text.LFSRRand  0x9d02dd94       0x78
 .text.LFSRRand
                0x9d02dd94       0x78 build/default/production/_ext/101875047/lfsr.o
                0x9d02dd94                LFSRRand

.text.SYS_TICK_TimerSetRate
                0x9d02de0c       0x78
 .text.SYS_TICK_TimerSetRate
                0x9d02de0c       0x78 build/default/production/_ext/365611741/system_services.o
                0x9d02de0c                SYS_TICK_TimerSetRate

.text.DHCPDeRegisterHandler
                0x9d02de84       0x78
 .text.DHCPDeRegisterHandler
                0x9d02de84       0x78 build/default/production/_ext/427700826/dhcp.o
                0x9d02de84                DHCPDeRegisterHandler

.text.DNSClientDeInit
                0x9d02defc       0x78
 .text.DNSClientDeInit
                0x9d02defc       0x78 build/default/production/_ext/427700826/dns.o
                0x9d02defc                DNSClientDeInit

.text.ENCX24J600_MACSetReadPtrInRx
                0x9d02df74       0x78
 .text.ENCX24J600_MACSetReadPtrInRx
                0x9d02df74       0x78 build/default/production/_ext/427700826/encs24j600.o
                0x9d02df74                ENCX24J600_MACSetReadPtrInRx

.text.SoftReset
                0x9d02dfec       0x78
 .text.SoftReset
                0x9d02dfec       0x78 c:/program files (x86)/microchip/xc32/v1.21/bin/../lib/gcc/pic32mx/4.5.2/../../../../pic32mx/lib/size\libmchp_peripheral_32MX795F512L.a(soft_reset_lib.o)
                0x9d02dfec                SoftReset

.text.rand      0x9d02e064       0x78
 .text.rand     0x9d02e064       0x78 c:/program files (x86)/microchip/xc32/v1.21/bin/../lib/gcc/pic32mx/4.5.2/../../../../pic32mx/lib/size\libc.a(rand.o)
                0x9d02e064                rand

.text.strstr    0x9d02e0dc       0x78
 .text.strstr   0x9d02e0dc       0x78 c:/program files (x86)/microchip/xc32/v1.21/bin/../lib/gcc/pic32mx/4.5.2/../../../../pic32mx/lib/size\libc.a(strstr.o)
                0x9d02e0dc                strstr

.text.MD5Initialize
                0x9d02e154       0x74
 .text.MD5Initialize
                0x9d02e154       0x74 build/default/production/_ext/101875047/hashes.o
                0x9d02e154                MD5Initialize

.text.SYS_RANDOM_ADD
                0x9d02e1c8       0x74
 .text.SYS_RANDOM_ADD
                0x9d02e1c8       0x74 build/default/production/_ext/365611741/system_random.o
                0x9d02e1c8                SYS_RANDOM_ADD

.text.CommandCleanup
                0x9d02e23c       0x74
 .text.CommandCleanup
                0x9d02e23c       0x74 build/default/production/_ext/365611741/system_command.o

.text.SYS_FS_IsLegalDirChar
                0x9d02e2b0       0x74
 .text.SYS_FS_IsLegalDirChar
                0x9d02e2b0       0x74 build/default/production/_ext/97638081/sys_fs.o
                0x9d02e2b0                SYS_FS_IsLegalDirChar

.text.TCPIP_IPV4_SetTxBuffer
                0x9d02e324       0x74
 .text.TCPIP_IPV4_SetTxBuffer
                0x9d02e324       0x74 build/default/production/_ext/427700826/ipv4.o
                0x9d02e324                TCPIP_IPV4_SetTxBuffer

.text.TCP_GetUpperLayerHeaderPtr
                0x9d02e398       0x74
 .text.TCP_GetUpperLayerHeaderPtr
                0x9d02e398       0x74 build/default/production/_ext/427700826/tcp.o

.text.TCP_IsPacketQueued
                0x9d02e40c       0x74
 .text.TCP_IsPacketQueued
                0x9d02e40c       0x74 build/default/production/_ext/427700826/tcp.o

.text.TCP_ResetTransmitPacketState
                0x9d02e480       0x74
 .text.TCP_ResetTransmitPacketState
                0x9d02e480       0x74 build/default/production/_ext/427700826/tcp.o

.text._TCPIP_HEAP_FreeDebug
                0x9d02e4f4       0x74
 .text._TCPIP_HEAP_FreeDebug
                0x9d02e4f4       0x74 build/default/production/_ext/427700826/tcpip_heap_alloc.o
                0x9d02e4f4                _TCPIP_HEAP_FreeDebug

.text.UDPIsConnected
                0x9d02e568       0x74
 .text.UDPIsConnected
                0x9d02e568       0x74 build/default/production/_ext/427700826/udp.o
                0x9d02e568                UDPIsConnected

.text.HTTPPrint_pot
                0x9d02e5dc       0x74
 .text.HTTPPrint_pot
                0x9d02e5dc       0x74 build/default/production/_ext/1472/custom_http_app.o
                0x9d02e5dc                HTTPPrint_pot

.text.HTTPPrint_config_hostname
                0x9d02e650       0x74
 .text.HTTPPrint_config_hostname
                0x9d02e650       0x74 build/default/production/_ext/1472/custom_http_app.o
                0x9d02e650                HTTPPrint_config_hostname

.text._sys_CONSOLE_PRINT
                0x9d02e6c4       0x70
 .text._sys_CONSOLE_PRINT
                0x9d02e6c4       0x70 build/default/production/_ext/365611741/system_command.o

.text._ARPDeleteCache
                0x9d02e734       0x70
 .text._ARPDeleteCache
                0x9d02e734       0x70 build/default/production/_ext/427700826/arp.o

.text.ENCX24_MACOpen
                0x9d02e7a4       0x70
 .text.ENCX24_MACOpen
                0x9d02e7a4       0x70 build/default/production/_ext/427700826/encx24_mac.o
                0x9d02e7a4                ENCX24_MACOpen

.text.ENCX24_MACCheckLink
                0x9d02e814       0x70
 .text.ENCX24_MACCheckLink
                0x9d02e814       0x70 build/default/production/_ext/427700826/encx24_mac.o

.text.ICMPInitialize
                0x9d02e884       0x70
 .text.ICMPInitialize
                0x9d02e884       0x70 build/default/production/_ext/427700826/icmp.o
                0x9d02e884                ICMPInitialize

.text.TCPIP_IPV4_SingleListFree
                0x9d02e8f4       0x70
 .text.TCPIP_IPV4_SingleListFree
                0x9d02e8f4       0x70 build/default/production/_ext/427700826/ipv4.o
                0x9d02e8f4                TCPIP_IPV4_SingleListFree

.text.NBNSInit  0x9d02e964       0x70
 .text.NBNSInit
                0x9d02e964       0x70 build/default/production/_ext/427700826/nbns.o
                0x9d02e964                NBNSInit

.text.TCPPutString
                0x9d02e9d4       0x70
 .text.TCPPutString
                0x9d02e9d4       0x70 build/default/production/_ext/427700826/tcp.o
                0x9d02e9d4                TCPPutString

.text.TCPIPMacEventCB
                0x9d02ea44       0x70
 .text.TCPIPMacEventCB
                0x9d02ea44       0x70 build/default/production/_ext/427700826/tcpip_manager.o

.text.HTTPPrint_config_ip
                0x9d02eab4       0x70
 .text.HTTPPrint_config_ip
                0x9d02eab4       0x70 build/default/production/_ext/1472/custom_http_app.o
                0x9d02eab4                HTTPPrint_config_ip

.text.HTTPPrint_config_gw
                0x9d02eb24       0x70
 .text.HTTPPrint_config_gw
                0x9d02eb24       0x70 build/default/production/_ext/1472/custom_http_app.o
                0x9d02eb24                HTTPPrint_config_gw

.text.HTTPPrint_config_subnet
                0x9d02eb94       0x70
 .text.HTTPPrint_config_subnet
                0x9d02eb94       0x70 build/default/production/_ext/1472/custom_http_app.o
                0x9d02eb94                HTTPPrint_config_subnet

.text.HTTPPrint_config_dns1
                0x9d02ec04       0x70
 .text.HTTPPrint_config_dns1
                0x9d02ec04       0x70 build/default/production/_ext/1472/custom_http_app.o
                0x9d02ec04                HTTPPrint_config_dns1

.text.HTTPPrint_config_dns2
                0x9d02ec74       0x70
 .text.HTTPPrint_config_dns2
                0x9d02ec74       0x70 build/default/production/_ext/1472/custom_http_app.o
                0x9d02ec74                HTTPPrint_config_dns2

.text.CommandReset
                0x9d02ece4       0x6c
 .text.CommandReset
                0x9d02ece4       0x6c build/default/production/_ext/365611741/system_command.o

.text._ARPRefreshEntry
                0x9d02ed50       0x6c
 .text._ARPRefreshEntry
                0x9d02ed50       0x6c build/default/production/_ext/427700826/arp.o

.text.ENCX24_MACPutHeader
                0x9d02edbc       0x6c
 .text.ENCX24_MACPutHeader
                0x9d02edbc       0x6c build/default/production/_ext/427700826/encx24_mac.o

.text._TCPGetRxFIFOFree
                0x9d02ee28       0x6c
 .text._TCPGetRxFIFOFree
                0x9d02ee28       0x6c build/default/production/_ext/427700826/tcp.o

.text.TcpClientIpv4RemoteHash
                0x9d02ee94       0x6c
 .text.TcpClientIpv4RemoteHash
                0x9d02ee94       0x6c build/default/production/_ext/427700826/tcp.o

.text.TCPIP_HEAP_FreeSize
                0x9d02ef00       0x6c
 .text.TCPIP_HEAP_FreeSize
                0x9d02ef00       0x6c build/default/production/_ext/427700826/tcpip_heap_alloc.o
                0x9d02ef00                TCPIP_HEAP_FreeSize

.rodata         0x9d02ef6c       0x6c
 .rodata        0x9d02ef6c       0x6c build/default/production/_ext/427700826/udp.o

.text.TCPIP_STACK_NetGatewayAddress
                0x9d02efd8       0x6c
 .text.TCPIP_STACK_NetGatewayAddress
                0x9d02efd8       0x6c build/default/production/_ext/427700826/tcpip_manager.o
                0x9d02efd8                TCPIP_STACK_NetGatewayAddress

.text.TCPIP_STACK_NetPriDNSAddress
                0x9d02f044       0x6c
 .text.TCPIP_STACK_NetPriDNSAddress
                0x9d02f044       0x6c build/default/production/_ext/427700826/tcpip_manager.o
                0x9d02f044                TCPIP_STACK_NetPriDNSAddress

.text.TCPIP_STACK_NetSecondDNSAddress
                0x9d02f0b0       0x6c
 .text.TCPIP_STACK_NetSecondDNSAddress
                0x9d02f0b0       0x6c build/default/production/_ext/427700826/tcpip_manager.o
                0x9d02f0b0                TCPIP_STACK_NetSecondDNSAddress

.text.TCPIP_STACK_NetBIOSName
                0x9d02f11c       0x6c
 .text.TCPIP_STACK_NetBIOSName
                0x9d02f11c       0x6c build/default/production/_ext/427700826/tcpip_manager.o
                0x9d02f11c                TCPIP_STACK_NetBIOSName

.text.TCPIP_NotificationRemove
                0x9d02f188       0x6c
 .text.TCPIP_NotificationRemove
                0x9d02f188       0x6c build/default/production/_ext/427700826/tcpip_notify.o
                0x9d02f188                TCPIP_NotificationRemove

.text.MPFSGetPosition
                0x9d02f1f4       0x68
 .text.MPFSGetPosition
                0x9d02f1f4       0x68 build/default/production/_ext/97638081/mpfs2.o
                0x9d02f1f4                MPFSGetPosition

.text.OAHashGetEntry
                0x9d02f25c       0x68
 .text.OAHashGetEntry
                0x9d02f25c       0x68 build/default/production/_ext/427700826/hash_tbl.o
                0x9d02f25c                OAHashGetEntry

.text.TCPIP_IPV4_FreePacket
                0x9d02f2c4       0x68
 .text.TCPIP_IPV4_FreePacket
                0x9d02f2c4       0x68 build/default/production/_ext/427700826/ipv4.o
                0x9d02f2c4                TCPIP_IPV4_FreePacket

.text._TcpSocketBind
                0x9d02f32c       0x68
 .text._TcpSocketBind
                0x9d02f32c       0x68 build/default/production/_ext/427700826/tcp.o

.text._TcpSocketChk
                0x9d02f394       0x68
 .text._TcpSocketChk
                0x9d02f394       0x68 build/default/production/_ext/427700826/tcp.o

.text._TcpFlush
                0x9d02f3fc       0x68
 .text._TcpFlush
                0x9d02f3fc       0x68 build/default/production/_ext/427700826/tcp.o

.text.TCPIsGetReady
                0x9d02f464       0x68
 .text.TCPIsGetReady
                0x9d02f464       0x68 build/default/production/_ext/427700826/tcp.o
                0x9d02f464                TCPIsGetReady

.text.TCPGetRxFIFOFree
                0x9d02f4cc       0x68
 .text.TCPGetRxFIFOFree
                0x9d02f4cc       0x68 build/default/production/_ext/427700826/tcp.o
                0x9d02f4cc                TCPGetRxFIFOFree

.text._UdpSocketBind
                0x9d02f534       0x68
 .text._UdpSocketBind
                0x9d02f534       0x68 build/default/production/_ext/427700826/udp.o

.text.MACPutHeader
                0x9d02f59c       0x68
 .text.MACPutHeader
                0x9d02f59c       0x68 build/default/production/_ext/427700826/tcpip_mac_object.o
                0x9d02f59c                MACPutHeader

.text.TCPIP_STACK_NetName
                0x9d02f604       0x68
 .text.TCPIP_STACK_NetName
                0x9d02f604       0x68 build/default/production/_ext/427700826/tcpip_manager.o
                0x9d02f604                TCPIP_STACK_NetName

.text.TCPIP_NotificationAdd
                0x9d02f66c       0x68
 .text.TCPIP_NotificationAdd
                0x9d02f66c       0x68 build/default/production/_ext/427700826/tcpip_notify.o
                0x9d02f66c                TCPIP_NotificationAdd

.rodata         0x9d02f6d4       0x68
 .rodata        0x9d02f6d4       0x68 c:/program files (x86)/microchip/xc32/v1.21/bin/../lib/gcc/pic32mx/4.5.2/../../../../pic32mx/lib/size\libc.a(powersf.o)
                0x9d02f6d4                _powers_f
                0x9d02f708                _npowers_f

.text.btohexa_high
                0x9d02f73c       0x64
 .text.btohexa_high
                0x9d02f73c       0x64 build/default/production/_ext/101875047/helpers.o
                0x9d02f73c                btohexa_high

.text.btohexa_low
                0x9d02f7a0       0x64
 .text.btohexa_low
                0x9d02f7a0       0x64 build/default/production/_ext/101875047/helpers.o
                0x9d02f7a0                btohexa_low

.text.MPFSClose
                0x9d02f804       0x64
 .text.MPFSClose
                0x9d02f804       0x64 build/default/production/_ext/97638081/mpfs2.o
                0x9d02f804                MPFSClose

.text.DRV_MEDIA_ReadByte
                0x9d02f868       0x64
 .text.DRV_MEDIA_ReadByte
                0x9d02f868       0x64 build/default/production/_ext/792872985/drv_media.o
                0x9d02f868                DRV_MEDIA_ReadByte

.text.DHCPIsEnabled
                0x9d02f8cc       0x64
 .text.DHCPIsEnabled
                0x9d02f8cc       0x64 build/default/production/_ext/427700826/dhcp.o
                0x9d02f8cc                DHCPIsEnabled

.text.TCPIP_IPV4_GetDataSegmentContentsByType
                0x9d02f930       0x64
 .text.TCPIP_IPV4_GetDataSegmentContentsByType
                0x9d02f930       0x64 build/default/production/_ext/427700826/ipv4.o
                0x9d02f930                TCPIP_IPV4_GetDataSegmentContentsByType

.text.TCPSocketGetNet
                0x9d02f994       0x64
 .text.TCPSocketGetNet
                0x9d02f994       0x64 build/default/production/_ext/427700826/tcp.o
                0x9d02f994                TCPSocketGetNet

.text._TCPIPStackIsNetLinked
                0x9d02f9f8       0x64
 .text._TCPIPStackIsNetLinked
                0x9d02f9f8       0x64 build/default/production/_ext/427700826/tcpip_manager.o
                0x9d02f9f8                _TCPIPStackIsNetLinked

.text.TCPIP_NotificationRemoveAll
                0x9d02fa5c       0x64
 .text.TCPIP_NotificationRemoveAll
                0x9d02fa5c       0x64 build/default/production/_ext/427700826/tcpip_notify.o
                0x9d02fa5c                TCPIP_NotificationRemoveAll

.text._sprintf_cdnopsuxX
                0x9d02fac0       0x64
 .text._sprintf_cdnopsuxX
                0x9d02fac0       0x64 c:/program files (x86)/microchip/xc32/v1.21/bin/../lib/gcc/pic32mx/4.5.2/../../../../pic32mx/lib/size\libc.a(sprintf_cdnopsuxX.eo)
                0x9d02fac0                _sprintf_cdnopuxX
                0x9d02fac0                _sprintf_cdnopsuxX

.text.SYS_DRIVERS_Initialize
                0x9d02fb24       0x60
 .text.SYS_DRIVERS_Initialize
                0x9d02fb24       0x60 build/default/production/_ext/365611741/system_services.o
                0x9d02fb24                SYS_DRIVERS_Initialize

.text.USART_PUTC
                0x9d02fb84       0x60
 .text.USART_PUTC
                0x9d02fb84       0x60 build/default/production/_ext/792872985/usart.o
                0x9d02fb84                USART_PUTC

.text.HTTPReleaseMedia
                0x9d02fbe4       0x60
 .text.HTTPReleaseMedia
                0x9d02fbe4       0x60 build/default/production/_ext/427700826/http2.o

.text.ENCX24_MACDeinitialize
                0x9d02fc44       0x60
 .text.ENCX24_MACDeinitialize
                0x9d02fc44       0x60 build/default/production/_ext/427700826/encx24_mac.o
                0x9d02fc44                ENCX24_MACDeinitialize

.text.ICMPDeinitialize
                0x9d02fca4       0x60
 .text.ICMPDeinitialize
                0x9d02fca4       0x60 build/default/production/_ext/427700826/icmp.o
                0x9d02fca4                ICMPDeinitialize

.text.TCPIP_IPV4_SetRxBuffer
                0x9d02fd04       0x60
 .text.TCPIP_IPV4_SetRxBuffer
                0x9d02fd04       0x60 build/default/production/_ext/427700826/ipv4.o
                0x9d02fd04                TCPIP_IPV4_SetRxBuffer

.text.TCP_FreePacket
                0x9d02fd64       0x60
 .text.TCP_FreePacket
                0x9d02fd64       0x60 build/default/production/_ext/427700826/tcp.o

.text.MACCalcRxChecksum
                0x9d02fdc4       0x60
 .text.MACCalcRxChecksum
                0x9d02fdc4       0x60 build/default/production/_ext/427700826/tcpip_mac_object.o
                0x9d02fdc4                MACCalcRxChecksum

.rodata         0x9d02fe24       0x60
 .rodata        0x9d02fe24       0x60 build/default/production/_ext/427700826/tcpip_helpers.o

.text.HTTPPrint_rebootaddr
                0x9d02fe84       0x60
 .text.HTTPPrint_rebootaddr
                0x9d02fe84       0x60 build/default/production/_ext/1472/custom_http_app.o
                0x9d02fe84                HTTPPrint_rebootaddr

.text.MPFSGetLong
                0x9d02fee4       0x5c
 .text.MPFSGetLong
                0x9d02fee4       0x5c build/default/production/_ext/97638081/mpfs2.o
                0x9d02fee4                MPFSGetLong

.text._DHCPCleanup
                0x9d02ff40       0x5c
 .text._DHCPCleanup
                0x9d02ff40       0x5c build/default/production/_ext/427700826/dhcp.o

.text.OAHashRemoveEntry
                0x9d02ff9c       0x5c
 .text.OAHashRemoveEntry
                0x9d02ff9c       0x5c build/default/production/_ext/427700826/hash_tbl.o
                0x9d02ff9c                OAHashRemoveEntry

.text.TCPFlush  0x9d02fff8       0x5c
 .text.TCPFlush
                0x9d02fff8       0x5c build/default/production/_ext/427700826/tcp.o
                0x9d02fff8                TCPFlush

.text.MACGetArray
                0x9d030054       0x5c
 .text.MACGetArray
                0x9d030054       0x5c build/default/production/_ext/427700826/tcpip_mac_object.o
                0x9d030054                MACGetArray

.text.MACPutArray
                0x9d0300b0       0x5c
 .text.MACPutArray
                0x9d0300b0       0x5c build/default/production/_ext/427700826/tcpip_mac_object.o
                0x9d0300b0                MACPutArray

.text._TCPIPStackNetAddress
                0x9d03010c       0x5c
 .text._TCPIPStackNetAddress
                0x9d03010c       0x5c build/default/production/_ext/427700826/tcpip_manager.o
                0x9d03010c                _TCPIPStackNetAddress

.text._TCPIPStackNetMask
                0x9d030168       0x5c
 .text._TCPIPStackNetMask
                0x9d030168       0x5c build/default/production/_ext/427700826/tcpip_manager.o
                0x9d030168                _TCPIPStackNetMask

.text._TCPIPStackNetMacAddress
                0x9d0301c4       0x5c
 .text._TCPIPStackNetMacAddress
                0x9d0301c4       0x5c build/default/production/_ext/427700826/tcpip_manager.o
                0x9d0301c4                _TCPIPStackNetMacAddress

.text.USART_OPEN
                0x9d030220       0x58
 .text.USART_OPEN
                0x9d030220       0x58 build/default/production/_ext/792872985/usart.o
                0x9d030220                USART_OPEN

.text.USART_GETC
                0x9d030278       0x58
 .text.USART_GETC
                0x9d030278       0x58 build/default/production/_ext/792872985/usart.o
                0x9d030278                USART_GETC

.text.LCD_ERASE
                0x9d0302d0       0x58
 .text.LCD_ERASE
                0x9d0302d0       0x58 build/default/production/_ext/792872985/lcd.o
                0x9d0302d0                LCD_ERASE

.text.WaitForDataByte
                0x9d030328       0x58
 .text.WaitForDataByte
                0x9d030328       0x58 build/default/production/_ext/792872985/drv_spi.o

.text._XEEFlashInit
                0x9d030380       0x58
 .text._XEEFlashInit
                0x9d030380       0x58 build/default/production/_ext/792872985/drv_media.o

.text.ARPHashKeyHash
                0x9d0303d8       0x58
 .text.ARPHashKeyHash
                0x9d0303d8       0x58 build/default/production/_ext/427700826/arp.o
                0x9d0303d8                ARPHashKeyHash

.text.ENCX24J600_MACSetWritePtr
                0x9d030430       0x58
 .text.ENCX24J600_MACSetWritePtr
                0x9d030430       0x58 build/default/production/_ext/427700826/encs24j600.o
                0x9d030430                ENCX24J600_MACSetWritePtr

.text.ENCX24J600_MACSetReadPtr
                0x9d030488       0x58
 .text.ENCX24J600_MACSetReadPtr
                0x9d030488       0x58 build/default/production/_ext/427700826/encs24j600.o
                0x9d030488                ENCX24J600_MACSetReadPtr

.text._TcpipHeapHandleToDcpt
                0x9d0304e0       0x58
 .text._TcpipHeapHandleToDcpt
                0x9d0304e0       0x58 build/default/production/_ext/427700826/tcpip_heap_alloc.o

.text.TCPIP_STACK_IxToNet
                0x9d030538       0x58
 .text.TCPIP_STACK_IxToNet
                0x9d030538       0x58 build/default/production/_ext/427700826/tcpip_manager.o
                0x9d030538                TCPIP_STACK_IxToNet

.text._TCPIPStackIsNetUp
                0x9d030590       0x58
 .text._TCPIPStackIsNetUp
                0x9d030590       0x58 build/default/production/_ext/427700826/tcpip_manager.o
                0x9d030590                _TCPIPStackIsNetUp

.text.HTTPPrint_ddns_status
                0x9d0305e8       0x58
 .text.HTTPPrint_ddns_status
                0x9d0305e8       0x58 build/default/production/_ext/1472/custom_http_app.o
                0x9d0305e8                HTTPPrint_ddns_status

.text.HTTPPrint_smtps_en
                0x9d030640       0x58
 .text.HTTPPrint_smtps_en
                0x9d030640       0x58 build/default/production/_ext/1472/custom_http_app.o
                0x9d030640                HTTPPrint_smtps_en

.text.HTTPPrint_snmp_en
                0x9d030698       0x58
 .text.HTTPPrint_snmp_en
                0x9d030698       0x58 build/default/production/_ext/1472/custom_http_app.o
                0x9d030698                HTTPPrint_snmp_en

.text._SYS_CONSOLE_PUTC
                0x9d0306f0       0x54
 .text._SYS_CONSOLE_PUTC
                0x9d0306f0       0x54 build/default/production/_ext/365611741/system_debug.o
                0x9d0306f0                _SYS_CONSOLE_PUTC

.text._SYS_OUT_MESSAGE_OFFSET
                0x9d030744       0x54
 .text._SYS_OUT_MESSAGE_OFFSET
                0x9d030744       0x54 build/default/production/_ext/365611741/system_debug.o
                0x9d030744                _SYS_OUT_MESSAGE_OFFSET

.text.ENCX24_MACCalcRxChecksum
                0x9d030798       0x54
 .text.ENCX24_MACCalcRxChecksum
                0x9d030798       0x54 build/default/production/_ext/427700826/encx24_mac.o

.text._ICMPAckPacket
                0x9d0307ec       0x54
 .text._ICMPAckPacket
                0x9d0307ec       0x54 build/default/production/_ext/427700826/icmp.o

.text._TcpDiscardTx
                0x9d030840       0x54
 .text._TcpDiscardTx
                0x9d030840       0x54 build/default/production/_ext/427700826/tcp.o

.text.TCPPut    0x9d030894       0x54
 .text.TCPPut   0x9d030894       0x54 build/default/production/_ext/427700826/tcp.o
                0x9d030894                TCPPut

.text._UdpSocketInit
                0x9d0308e8       0x54
 .text._UdpSocketInit
                0x9d0308e8       0x54 build/default/production/_ext/427700826/udp.o

.text.UDPPut    0x9d03093c       0x54
 .text.UDPPut   0x9d03093c       0x54 build/default/production/_ext/427700826/udp.o
                0x9d03093c                UDPPut

.text.MACGetHeader
                0x9d030990       0x54
 .text.MACGetHeader
                0x9d030990       0x54 build/default/production/_ext/427700826/tcpip_mac_object.o
                0x9d030990                MACGetHeader

.text.MACSetReadPtrInRx
                0x9d0309e4       0x54
 .text.MACSetReadPtrInRx
                0x9d0309e4       0x54 build/default/production/_ext/427700826/tcpip_mac_object.o
                0x9d0309e4                MACSetReadPtrInRx

.text.MACCalcIPBufferChecksum
                0x9d030a38       0x54
 .text.MACCalcIPBufferChecksum
                0x9d030a38       0x54 build/default/production/_ext/427700826/tcpip_mac_object.o
                0x9d030a38                MACCalcIPBufferChecksum

.text._TCPIPStackAddressServiceSetDefault
                0x9d030a8c       0x54
 .text._TCPIPStackAddressServiceSetDefault
                0x9d030a8c       0x54 build/default/production/_ext/427700826/tcpip_manager.o
                0x9d030a8c                _TCPIPStackAddressServiceSetDefault

.text.HTTPPrint_version
                0x9d030ae0       0x54
 .text.HTTPPrint_version
                0x9d030ae0       0x54 build/default/production/_ext/1472/custom_http_app.o
                0x9d030ae0                HTTPPrint_version

.rodata         0x9d030b34       0x54
 .rodata        0x9d030b34       0x54 c:/program files (x86)/microchip/xc32/v1.21/bin/../lib/gcc/pic32mx/4.5.2/../../../../pic32mx/lib/size\libmchp_peripheral_32MX795F512L.a(_ports_tbl_libp.o)
                0x9d030b34                PortRegTbl

.text._vsnprintf_cdnopsuxX
                0x9d030b88       0x54
 .text._vsnprintf_cdnopsuxX
                0x9d030b88       0x54 c:/program files (x86)/microchip/xc32/v1.21/bin/../lib/gcc/pic32mx/4.5.2/../../../../pic32mx/lib/size\libc.a(vsnprintf_cdnopsuxX.eo)
                0x9d030b88                _vsnprintf_cdnopsuxX

.text.vsnprintf
                0x9d030bdc       0x54
 .text.vsnprintf
                0x9d030bdc       0x54 c:/program files (x86)/microchip/xc32/v1.21/bin/../lib/gcc/pic32mx/4.5.2/../../../../pic32mx/lib/size\libc.a(vsnprintf.o)
                0x9d030bdc                vsnprintf

.text._SYS_CONSOLE_MESSAGE
                0x9d030c30       0x50
 .text._SYS_CONSOLE_MESSAGE
                0x9d030c30       0x50 build/default/production/_ext/365611741/system_debug.o
                0x9d030c30                _SYS_CONSOLE_MESSAGE

.text._TCPIP_AnnounceCleanup
                0x9d030c80       0x50
 .text._TCPIP_AnnounceCleanup
                0x9d030c80       0x50 build/default/production/_ext/427700826/tcpip_announce.o

.text.HTTPPrint_
                0x9d030cd0       0x50
 .text.HTTPPrint_
                0x9d030cd0       0x50 build/default/production/_ext/427700826/http2.o
                0x9d030cd0                HTTPPrint_

.text.ARPHashKeyCompare
                0x9d030d20       0x50
 .text.ARPHashKeyCompare
                0x9d030d20       0x50 build/default/production/_ext/427700826/arp.o
                0x9d030d20                ARPHashKeyCompare

.text._DNSReleaseSocket
                0x9d030d70       0x50
 .text._DNSReleaseSocket
                0x9d030d70       0x50 build/default/production/_ext/427700826/dns.o

.text.strncpy   0x9d030dc0       0x50
 .text.strncpy  0x9d030dc0       0x50 c:/program files (x86)/microchip/xc32/v1.21/bin/../lib/gcc/pic32mx/4.5.2/../../../../pic32mx/lib/size\libc.a(strncpy.o)
                0x9d030dc0                strncpy

.text.DRV_SPI_Initialize
                0x9d030e10       0x4c
 .text.DRV_SPI_Initialize
                0x9d030e10       0x4c build/default/production/_ext/792872985/drv_spi.o
                0x9d030e10                DRV_SPI_Initialize

.text.ENCX24J600_MACPutArray
                0x9d030e5c       0x4c
 .text.ENCX24J600_MACPutArray
                0x9d030e5c       0x4c build/default/production/_ext/427700826/encs24j600.o
                0x9d030e5c                ENCX24J600_MACPutArray

.rodata         0x9d030ea8       0x4c
 .rodata        0x9d030ea8       0x4c build/default/production/_ext/427700826/encx24_mac.o

.text.ENCX24_MACPutArray
                0x9d030ef4       0x4c
 .text.ENCX24_MACPutArray
                0x9d030ef4       0x4c build/default/production/_ext/427700826/encx24_mac.o

.text.ENCX24_MACGetArray
                0x9d030f40       0x4c
 .text.ENCX24_MACGetArray
                0x9d030f40       0x4c build/default/production/_ext/427700826/encx24_mac.o

.text.TCPGet    0x9d030f8c       0x4c
 .text.TCPGet   0x9d030f8c       0x4c build/default/production/_ext/427700826/tcp.o
                0x9d030f8c                TCPGet

.text.UDPGet    0x9d030fd8       0x4c
 .text.UDPGet   0x9d030fd8       0x4c build/default/production/_ext/427700826/udp.o
                0x9d030fd8                UDPGet

.text.MACSetWritePtr
                0x9d031024       0x4c
 .text.MACSetWritePtr
                0x9d031024       0x4c build/default/production/_ext/427700826/tcpip_mac_object.o
                0x9d031024                MACSetWritePtr

.text.MACSetReadPtr
                0x9d031070       0x4c
 .text.MACSetReadPtr
                0x9d031070       0x4c build/default/production/_ext/427700826/tcpip_mac_object.o
                0x9d031070                MACSetReadPtr

.text.INTEnable
                0x9d0310bc       0x4c
 .text.INTEnable
                0x9d0310bc       0x4c c:/program files (x86)/microchip/xc32/v1.21/bin/../lib/gcc/pic32mx/4.5.2/../../../../pic32mx/lib/size\libmchp_peripheral_32MX795F512L.a(int_tbl_lib.o)
                0x9d0310bc                INTEnable

.text           0x9d031108       0x4c
 .text          0x9d031108       0x4c c:/program files (x86)/microchip/xc32/v1.21/bin/../lib/gcc/pic32mx/4.5.2/size\libgcc.a(floatunsisf.o)
                0x9d031108                __floatunsisf

.text.SYS_CLK_PeripheralClockGet
                0x9d031154       0x48
 .text.SYS_CLK_PeripheralClockGet
                0x9d031154       0x48 build/default/production/_ext/365611741/system_services.o
                0x9d031154                SYS_CLK_PeripheralClockGet

.text._SYS_CONSOLE_DATA_RDY
                0x9d03119c       0x48
 .text._SYS_CONSOLE_DATA_RDY
                0x9d03119c       0x48 build/default/production/_ext/365611741/system_debug.o
                0x9d03119c                _SYS_CONSOLE_DATA_RDY

.text._SYS_CONSOLE_GETC
                0x9d0311e4       0x48
 .text._SYS_CONSOLE_GETC
                0x9d0311e4       0x48 build/default/production/_ext/365611741/system_debug.o
                0x9d0311e4                _SYS_CONSOLE_GETC

.text._SYS_OUT_MESSAGE_LINE
                0x9d03122c       0x48
 .text._SYS_OUT_MESSAGE_LINE
                0x9d03122c       0x48 build/default/production/_ext/365611741/system_debug.o
                0x9d03122c                _SYS_OUT_MESSAGE_LINE

.rodata         0x9d031274       0x48
 .rodata        0x9d031274       0x48 build/default/production/_ext/97638081/sys_fs.o

.text.HTTPCurConnectionByteCountDec
                0x9d0312bc       0x48
 .text.HTTPCurConnectionByteCountDec
                0x9d0312bc       0x48 build/default/production/_ext/427700826/http2.o
                0x9d0312bc                HTTPCurConnectionByteCountDec

.text.ARPHashKeyCopy
                0x9d031304       0x48
 .text.ARPHashKeyCopy
                0x9d031304       0x48 build/default/production/_ext/427700826/arp.o
                0x9d031304                ARPHashKeyCopy

.text.DNSEndUsage
                0x9d03134c       0x48
 .text.DNSEndUsage
                0x9d03134c       0x48 build/default/production/_ext/427700826/dns.o
                0x9d03134c                DNSEndUsage

.text.TCPIP_IPV4_SetSourceAddress
                0x9d031394       0x48
 .text.TCPIP_IPV4_SetSourceAddress
                0x9d031394       0x48 build/default/production/_ext/427700826/ipv4.o
                0x9d031394                TCPIP_IPV4_SetSourceAddress

.text.TCPIP_STACK_NetAddress
                0x9d0313dc       0x48
 .text.TCPIP_STACK_NetAddress
                0x9d0313dc       0x48 build/default/production/_ext/427700826/tcpip_manager.o
                0x9d0313dc                TCPIP_STACK_NetAddress

.text.TCPIP_STACK_NetMask
                0x9d031424       0x48
 .text.TCPIP_STACK_NetMask
                0x9d031424       0x48 build/default/production/_ext/427700826/tcpip_manager.o
                0x9d031424                TCPIP_STACK_NetMask

.text.TCPIP_STACK_NetMacAddress
                0x9d03146c       0x48
 .text.TCPIP_STACK_NetMacAddress
                0x9d03146c       0x48 build/default/production/_ext/427700826/tcpip_manager.o
                0x9d03146c                TCPIP_STACK_NetMacAddress

.text._DefaultInterrupt
                0x9d0314b4       0x48
 .text._DefaultInterrupt
                0x9d0314b4       0x48 c:/program files (x86)/microchip/xc32/v1.21/bin/../lib/gcc/pic32mx/4.5.2/../../../../pic32mx/lib/size\libpic32.a(defaultinterrupt.o)
                0x9d0314b4                _DefaultInterrupt

.text.sbrk      0x9d0314fc       0x48
 .text.sbrk     0x9d0314fc       0x48 c:/program files (x86)/microchip/xc32/v1.21/bin/../lib/gcc/pic32mx/4.5.2/../../../../pic32mx/lib/size\libpic32.a(sbrk.o)
                0x9d0314fc                sbrk

.text.SYS_CLK_ClockGet
                0x9d031544       0x44
 .text.SYS_CLK_ClockGet
                0x9d031544       0x44 build/default/production/_ext/365611741/system_services.o
                0x9d031544                SYS_CLK_ClockGet

.text._SYS_OUT_MESSAGE
                0x9d031588       0x44
 .text._SYS_OUT_MESSAGE
                0x9d031588       0x44 build/default/production/_ext/365611741/system_debug.o
                0x9d031588                _SYS_OUT_MESSAGE

.text._sys_CONSOLE_PUTC
                0x9d0315cc       0x44
 .text._sys_CONSOLE_PUTC
                0x9d0315cc       0x44 build/default/production/_ext/365611741/system_command.o

.text.MPFSGetID
                0x9d031610       0x44
 .text.MPFSGetID
                0x9d031610       0x44 build/default/production/_ext/97638081/mpfs2.o
                0x9d031610                MPFSGetID

.text.USART_DATA_RDY
                0x9d031654       0x44
 .text.USART_DATA_RDY
                0x9d031654       0x44 build/default/production/_ext/792872985/usart.o
                0x9d031654                USART_DATA_RDY

.text.ENCX24_MACGetHeader
                0x9d031698       0x44
 .text.ENCX24_MACGetHeader
                0x9d031698       0x44 build/default/production/_ext/427700826/encx24_mac.o

.text.ENCX24_MACSetReadPtrInRx
                0x9d0316dc       0x44
 .text.ENCX24_MACSetReadPtrInRx
                0x9d0316dc       0x44 build/default/production/_ext/427700826/encx24_mac.o

.text.ENCX24_MACCalcIPBufferChecksum
                0x9d031720       0x44
 .text.ENCX24_MACCalcIPBufferChecksum
                0x9d031720       0x44 build/default/production/_ext/427700826/encx24_mac.o

.text.TCPIP_IPV4_SetPacketIPProtocol
                0x9d031764       0x44
 .text.TCPIP_IPV4_SetPacketIPProtocol
                0x9d031764       0x44 build/default/production/_ext/427700826/ipv4.o
                0x9d031764                TCPIP_IPV4_SetPacketIPProtocol

.text.MACClose  0x9d0317a8       0x44
 .text.MACClose
                0x9d0317a8       0x44 build/default/production/_ext/427700826/tcpip_mac_object.o
                0x9d0317a8                MACClose

.text.MACDiscardRx
                0x9d0317ec       0x44
 .text.MACDiscardRx
                0x9d0317ec       0x44 build/default/production/_ext/427700826/tcpip_mac_object.o
                0x9d0317ec                MACDiscardRx

.text.MACIsTxReady
                0x9d031830       0x44
 .text.MACIsTxReady
                0x9d031830       0x44 build/default/production/_ext/427700826/tcpip_mac_object.o
                0x9d031830                MACIsTxReady

.text.MACFlush  0x9d031874       0x44
 .text.MACFlush
                0x9d031874       0x44 build/default/production/_ext/427700826/tcpip_mac_object.o
                0x9d031874                MACFlush

.text.MACCheckLink
                0x9d0318b8       0x44
 .text.MACCheckLink
                0x9d0318b8       0x44 build/default/production/_ext/427700826/tcpip_mac_object.o
                0x9d0318b8                MACCheckLink

.text.MACGetTxBaseAddr
                0x9d0318fc       0x44
 .text.MACGetTxBaseAddr
                0x9d0318fc       0x44 build/default/production/_ext/427700826/tcpip_mac_object.o
                0x9d0318fc                MACGetTxBaseAddr

.text.ProcessTCPIPMacGeneric
                0x9d031940       0x44
 .text.ProcessTCPIPMacGeneric
                0x9d031940       0x44 build/default/production/_ext/427700826/tcpip_manager.o

.text.TCPIP_STACK_NetHandle
                0x9d031984       0x44
 .text.TCPIP_STACK_NetHandle
                0x9d031984       0x44 build/default/production/_ext/427700826/tcpip_manager.o
                0x9d031984                TCPIP_STACK_NetHandle

.text._TCPIPStackNetIx
                0x9d0319c8       0x44
 .text._TCPIPStackNetIx
                0x9d0319c8       0x44 build/default/production/_ext/427700826/tcpip_manager.o
                0x9d0319c8                _TCPIPStackNetIx

.text._TCPIPStackSetGatewayAddress
                0x9d031a0c       0x44
 .text._TCPIPStackSetGatewayAddress
                0x9d031a0c       0x44 build/default/production/_ext/427700826/tcpip_manager.o
                0x9d031a0c                _TCPIPStackSetGatewayAddress

.text._TCPIPStackSetPriDNSAddress
                0x9d031a50       0x44
 .text._TCPIPStackSetPriDNSAddress
                0x9d031a50       0x44 build/default/production/_ext/427700826/tcpip_manager.o
                0x9d031a50                _TCPIPStackSetPriDNSAddress

.text._TCPIPStackSetSecondDNSAddress
                0x9d031a94       0x44
 .text._TCPIPStackSetSecondDNSAddress
                0x9d031a94       0x44 build/default/production/_ext/427700826/tcpip_manager.o
                0x9d031a94                _TCPIPStackSetSecondDNSAddress

.text._TCPIPStackNetToMac
                0x9d031ad8       0x44
 .text._TCPIPStackNetToMac
                0x9d031ad8       0x44 build/default/production/_ext/427700826/tcpip_manager.o
                0x9d031ad8                _TCPIPStackNetToMac

.text.SingleListInit
                0x9d031b1c       0x44
 .text.SingleListInit
                0x9d031b1c       0x44 build/default/production/_ext/427700826/tcpip_helpers.o
                0x9d031b1c                SingleListInit

.text.strncat   0x9d031b60       0x44
 .text.strncat  0x9d031b60       0x44 c:/program files (x86)/microchip/xc32/v1.21/bin/../lib/gcc/pic32mx/4.5.2/../../../../pic32mx/lib/size\libc.a(strncat.o)
                0x9d031b60                strncat

.text.strncmp   0x9d031ba4       0x44
 .text.strncmp  0x9d031ba4       0x44 c:/program files (x86)/microchip/xc32/v1.21/bin/../lib/gcc/pic32mx/4.5.2/../../../../pic32mx/lib/size\libc.a(strncmp.o)
                0x9d031ba4                strncmp

.text           0x9d031be8       0x44
 .text          0x9d031be8       0x44 c:/program files (x86)/microchip/xc32/v1.21/bin/../lib/gcc/pic32mx/4.5.2/size\libgcc.a(_lshrdi3.o)
                0x9d031be8                __lshrdi3

.text.XEEEndWrite
                0x9d031c2c       0x40
 .text.XEEEndWrite
                0x9d031c2c       0x40 build/default/production/_ext/792872985/spi_eeprom.o
                0x9d031c2c                XEEEndWrite

.text.HTTPCurConnectionPostSmSet
                0x9d031c6c       0x40
 .text.HTTPCurConnectionPostSmSet
                0x9d031c6c       0x40 build/default/production/_ext/427700826/http2.o
                0x9d031c6c                HTTPCurConnectionPostSmSet

.text.HTTPCurConnectionHasArgsSet
                0x9d031cac       0x40
 .text.HTTPCurConnectionHasArgsSet
                0x9d031cac       0x40 build/default/production/_ext/427700826/http2.o
                0x9d031cac                HTTPCurConnectionHasArgsSet

.text.ENCX24J600_MACCheckLink
                0x9d031cec       0x40
 .text.ENCX24J600_MACCheckLink
                0x9d031cec       0x40 build/default/production/_ext/427700826/encs24j600.o
                0x9d031cec                ENCX24J600_MACCheckLink

.text.ENCX24J600_MACIsTxReady
                0x9d031d2c       0x40
 .text.ENCX24J600_MACIsTxReady
                0x9d031d2c       0x40 build/default/production/_ext/427700826/encs24j600.o
                0x9d031d2c                ENCX24J600_MACIsTxReady

.text.TCPIP_IPV4_Task
                0x9d031d6c       0x40
 .text.TCPIP_IPV4_Task
                0x9d031d6c       0x40 build/default/production/_ext/427700826/ipv4.o
                0x9d031d6c                TCPIP_IPV4_Task

.text.UDPResetHeader
                0x9d031dac       0x40
 .text.UDPResetHeader
                0x9d031dac       0x40 build/default/production/_ext/427700826/udp.o
                0x9d031dac                UDPResetHeader

.text.SpiChnDataRdy
                0x9d031dec       0x40
 .text.SpiChnDataRdy
                0x9d031dec       0x40 c:/program files (x86)/microchip/xc32/v1.21/bin/../lib/gcc/pic32mx/4.5.2/../../../../pic32mx/lib/size\libmchp_peripheral_32MX795F512L.a(spi_chn_data_rdy_lib.o)
                0x9d031dec                SpiChnDataRdy

.text._sys_CONSOLE_MESSAGE
                0x9d031e2c       0x3c
 .text._sys_CONSOLE_MESSAGE
                0x9d031e2c       0x3c build/default/production/_ext/365611741/system_command.o

.text.DRV_MEDIA_WriteFlush
                0x9d031e68       0x3c
 .text.DRV_MEDIA_WriteFlush
                0x9d031e68       0x3c build/default/production/_ext/792872985/drv_media.o
                0x9d031e68                DRV_MEDIA_WriteFlush

.text.HTTPCurConnectionCallbackPosSet
                0x9d031ea4       0x3c
 .text.HTTPCurConnectionCallbackPosSet
                0x9d031ea4       0x3c build/default/production/_ext/427700826/http2.o
                0x9d031ea4                HTTPCurConnectionCallbackPosSet

.text.HTTPCurConnectionStatusSet
                0x9d031ee0       0x3c
 .text.HTTPCurConnectionStatusSet
                0x9d031ee0       0x3c build/default/production/_ext/427700826/http2.o
                0x9d031ee0                HTTPCurConnectionStatusSet

.text._ARPDeleteClients
                0x9d031f1c       0x3c
 .text._ARPDeleteClients
                0x9d031f1c       0x3c build/default/production/_ext/427700826/arp.o

.text.ARPTmoHandler
                0x9d031f58       0x3c
 .text.ARPTmoHandler
                0x9d031f58       0x3c build/default/production/_ext/427700826/arp.o

.text.ENCX24_MACSetWritePtr
                0x9d031f94       0x3c
 .text.ENCX24_MACSetWritePtr
                0x9d031f94       0x3c build/default/production/_ext/427700826/encx24_mac.o

.text.ENCX24_MACSetReadPtr
                0x9d031fd0       0x3c
 .text.ENCX24_MACSetReadPtr
                0x9d031fd0       0x3c build/default/production/_ext/427700826/encx24_mac.o

.text.TCPIP_IPV4_GetUpperLayerHeaderPtr
                0x9d03200c       0x3c
 .text.TCPIP_IPV4_GetUpperLayerHeaderPtr
                0x9d03200c       0x3c build/default/production/_ext/427700826/ipv4.o
                0x9d03200c                TCPIP_IPV4_GetUpperLayerHeaderPtr

.text.TCPIP_IPV4_GetPayloadLength
                0x9d032048       0x3c
 .text.TCPIP_IPV4_GetPayloadLength
                0x9d032048       0x3c build/default/production/_ext/427700826/ipv4.o
                0x9d032048                TCPIP_IPV4_GetPayloadLength

.rodata         0x9d032084       0x3c
 .rodata        0x9d032084       0x3c build/default/production/_ext/427700826/tcpip_heap_alloc.o

.text.PORTSetPinsDigitalIn
                0x9d0320c0       0x3c
 .text.PORTSetPinsDigitalIn
                0x9d0320c0       0x3c c:/program files (x86)/microchip/xc32/v1.21/bin/../lib/gcc/pic32mx/4.5.2/../../../../pic32mx/lib/size\libmchp_peripheral_32MX795F512L.a(port_set_pins_digital_in_lib.o)
                0x9d0320c0                PORTSetPinsDigitalIn

.text.PORTSetPinsDigitalOut
                0x9d0320fc       0x3c
 .text.PORTSetPinsDigitalOut
                0x9d0320fc       0x3c c:/program files (x86)/microchip/xc32/v1.21/bin/../lib/gcc/pic32mx/4.5.2/../../../../pic32mx/lib/size\libmchp_peripheral_32MX795F512L.a(port_set_pins_digital_out_lib.o)
                0x9d0320fc                PORTSetPinsDigitalOut

.text           0x9d032138       0x38
 .text          0x9d032138       0x38 c:/program files (x86)/microchip/xc32/v1.21/bin/../lib/gcc/pic32mx/4.5.2/../../../../pic32mx/lib/size/crt0.o
                0x9d032164                __crt0_exit

.text.SYS_Tasks
                0x9d032170       0x38
 .text.SYS_Tasks
                0x9d032170       0x38 build/default/production/_ext/365611741/system_services.o
                0x9d032170                SYS_Tasks

.text._SYS_OUT_INIT
                0x9d0321a8       0x38
 .text._SYS_OUT_INIT
                0x9d0321a8       0x38 build/default/production/_ext/365611741/system_debug.o
                0x9d0321a8                _SYS_OUT_INIT

.text.DRV_MEDIA_Close
                0x9d0321e0       0x38
 .text.DRV_MEDIA_Close
                0x9d0321e0       0x38 build/default/production/_ext/792872985/drv_media.o
                0x9d0321e0                DRV_MEDIA_Close

.text.ENCX24J600_MACGetReadPtrInRx
                0x9d032218       0x38
 .text.ENCX24J600_MACGetReadPtrInRx
                0x9d032218       0x38 build/default/production/_ext/427700826/encs24j600.o
                0x9d032218                ENCX24J600_MACGetReadPtrInRx

.text.ENCX24_MACClose
                0x9d032250       0x38
 .text.ENCX24_MACClose
                0x9d032250       0x38 build/default/production/_ext/427700826/encx24_mac.o

.text.ENCX24_MACGetReadPtrInRx
                0x9d032288       0x38
 .text.ENCX24_MACGetReadPtrInRx
                0x9d032288       0x38 build/default/production/_ext/427700826/encx24_mac.o

.text._OAHashProbeStep
                0x9d0322c0       0x38
 .text._OAHashProbeStep
                0x9d0322c0       0x38 build/default/production/_ext/427700826/hash_tbl.o

.text.INTSetVectorPriority
                0x9d0322f8       0x38
 .text.INTSetVectorPriority
                0x9d0322f8       0x38 c:/program files (x86)/microchip/xc32/v1.21/bin/../lib/gcc/pic32mx/4.5.2/../../../../pic32mx/lib/size\libmchp_peripheral_32MX795F512L.a(int_tbl_lib.o)
                0x9d0322f8                INTSetVectorPriority

.text.INTSetVectorSubPriority
                0x9d032330       0x38
 .text.INTSetVectorSubPriority
                0x9d032330       0x38 c:/program files (x86)/microchip/xc32/v1.21/bin/../lib/gcc/pic32mx/4.5.2/../../../../pic32mx/lib/size\libmchp_peripheral_32MX795F512L.a(int_tbl_lib.o)
                0x9d032330                INTSetVectorSubPriority

.text._sys_CONSOLE_DATA_RDY
                0x9d032368       0x34
 .text._sys_CONSOLE_DATA_RDY
                0x9d032368       0x34 build/default/production/_ext/365611741/system_command.o

.text._sys_CONSOLE_GETC
                0x9d03239c       0x34
 .text._sys_CONSOLE_GETC
                0x9d03239c       0x34 build/default/production/_ext/365611741/system_command.o

.text.XEEBeginWrite
                0x9d0323d0       0x34
 .text.XEEBeginWrite
                0x9d0323d0       0x34 build/default/production/_ext/792872985/spi_eeprom.o
                0x9d0323d0                XEEBeginWrite

.text.DRV_MEDIA_ClientStatus
                0x9d032404       0x34
 .text.DRV_MEDIA_ClientStatus
                0x9d032404       0x34 build/default/production/_ext/792872985/drv_media.o
                0x9d032404                DRV_MEDIA_ClientStatus

.text.HTTPCurConnectionFileGet
                0x9d032438       0x34
 .text.HTTPCurConnectionFileGet
                0x9d032438       0x34 build/default/production/_ext/427700826/http2.o
                0x9d032438                HTTPCurConnectionFileGet

.text.HTTPCurConnectionPostSmGet
                0x9d03246c       0x34
 .text.HTTPCurConnectionPostSmGet
                0x9d03246c       0x34 build/default/production/_ext/427700826/http2.o
                0x9d03246c                HTTPCurConnectionPostSmGet

.text.HTTPCurConnectionDataBufferGet
                0x9d0324a0       0x34
 .text.HTTPCurConnectionDataBufferGet
                0x9d0324a0       0x34 build/default/production/_ext/427700826/http2.o
                0x9d0324a0                HTTPCurConnectionDataBufferGet

.text.HTTPCurConnectionByteCountGet
                0x9d0324d4       0x34
 .text.HTTPCurConnectionByteCountGet
                0x9d0324d4       0x34 build/default/production/_ext/427700826/http2.o
                0x9d0324d4                HTTPCurConnectionByteCountGet

.text.HTTPCurConnectionSocketGet
                0x9d032508       0x34
 .text.HTTPCurConnectionSocketGet
                0x9d032508       0x34 build/default/production/_ext/427700826/http2.o
                0x9d032508                HTTPCurConnectionSocketGet

.text.ENCX24_MACIsTxReady
                0x9d03253c       0x34
 .text.ENCX24_MACIsTxReady
                0x9d03253c       0x34 build/default/production/_ext/427700826/encx24_mac.o

.text.ENCX24_MACFlush
                0x9d032570       0x34
 .text.ENCX24_MACFlush
                0x9d032570       0x34 build/default/production/_ext/427700826/encx24_mac.o

.text.ENCX24_MACDiscardRx
                0x9d0325a4       0x34
 .text.ENCX24_MACDiscardRx
                0x9d0325a4       0x34 build/default/production/_ext/427700826/encx24_mac.o

.text.TCPIP_IPV4_SetDestAddress
                0x9d0325d8       0x34
 .text.TCPIP_IPV4_SetDestAddress
                0x9d0325d8       0x34 build/default/production/_ext/427700826/ipv4.o
                0x9d0325d8                TCPIP_IPV4_SetDestAddress

.text.TCPIP_IPV4_GetDestAddress
                0x9d03260c       0x34
 .text.TCPIP_IPV4_GetDestAddress
                0x9d03260c       0x34 build/default/production/_ext/427700826/ipv4.o
                0x9d03260c                TCPIP_IPV4_GetDestAddress

.text.TCPIP_IPV4_GetSourceAddress
                0x9d032640       0x34
 .text.TCPIP_IPV4_GetSourceAddress
                0x9d032640       0x34 build/default/production/_ext/427700826/ipv4.o
                0x9d032640                TCPIP_IPV4_GetSourceAddress

.text.ProcessTCPIPMacErrorEvents
                0x9d032674       0x34
 .text.ProcessTCPIPMacErrorEvents
                0x9d032674       0x34 build/default/production/_ext/427700826/tcpip_manager.o

.text.HTTPPrint_reboot
                0x9d0326a8       0x34
 .text.HTTPPrint_reboot
                0x9d0326a8       0x34 build/default/production/_ext/1472/custom_http_app.o
                0x9d0326a8                HTTPPrint_reboot

.text.INTEnableSystemMultiVectoredInt
                0x9d0326dc       0x34
 .text.INTEnableSystemMultiVectoredInt
                0x9d0326dc       0x34 c:/program files (x86)/microchip/xc32/v1.21/bin/../lib/gcc/pic32mx/4.5.2/../../../../pic32mx/lib/size\libmchp_peripheral_32MX795F512L.a(int_enable_mv_int_lib.o)
                0x9d0326dc                INTEnableSystemMultiVectoredInt

.text.SYS_USERIO_Tasks
                0x9d032710       0x30
 .text.SYS_USERIO_Tasks
                0x9d032710       0x30 build/default/production/_ext/365611741/system_userio.o
                0x9d032710                SYS_USERIO_Tasks

.text.SYS_FS_mpfs2fs_Init
                0x9d032740       0x30
 .text.SYS_FS_mpfs2fs_Init
                0x9d032740       0x30 build/default/production/_ext/97638081/sys_fs.o
                0x9d032740                SYS_FS_mpfs2fs_Init

.text.TCPIP_IPV4_TmoHandler
                0x9d032770       0x30
 .text.TCPIP_IPV4_TmoHandler
                0x9d032770       0x30 build/default/production/_ext/427700826/ipv4.o
                0x9d032770                TCPIP_IPV4_TmoHandler

.text._TcpTmoHandler
                0x9d0327a0       0x30
 .text._TcpTmoHandler
                0x9d0327a0       0x30 build/default/production/_ext/427700826/tcp.o

.text.TCPIP_STACK_TickHandler
                0x9d0327d0       0x30
 .text.TCPIP_STACK_TickHandler
                0x9d0327d0       0x30 build/default/production/_ext/427700826/tcpip_manager.o

.text.strcat    0x9d032800       0x30
 .text.strcat   0x9d032800       0x30 c:/program files (x86)/microchip/xc32/v1.21/bin/../lib/gcc/pic32mx/4.5.2/../../../../pic32mx/lib/size\libc.a(strcat.o)
                0x9d032800                strcat

.text.SYS_WDT_Clear
                0x9d032830       0x2c
 .text.SYS_WDT_Clear
                0x9d032830       0x2c build/default/production/_ext/365611741/system_services.o
                0x9d032830                SYS_WDT_Clear

.text.TCPIP_ANNOUNCE_TaskPending
                0x9d03285c       0x2c
 .text.TCPIP_ANNOUNCE_TaskPending
                0x9d03285c       0x2c build/default/production/_ext/427700826/tcpip_announce.o
                0x9d03285c                TCPIP_ANNOUNCE_TaskPending

.text.ARPTaskPending
                0x9d032888       0x2c
 .text.ARPTaskPending
                0x9d032888       0x2c build/default/production/_ext/427700826/arp.o
                0x9d032888                ARPTaskPending

.text.ENCX24_MACSetRXHashTableEntry
                0x9d0328b4       0x2c
 .text.ENCX24_MACSetRXHashTableEntry
                0x9d0328b4       0x2c build/default/production/_ext/427700826/encx24_mac.o

.text.TCPIP_IPV4_TaskPending
                0x9d0328e0       0x2c
 .text.TCPIP_IPV4_TaskPending
                0x9d0328e0       0x2c build/default/production/_ext/427700826/ipv4.o
                0x9d0328e0                TCPIP_IPV4_TaskPending

.text.TCPTaskPending
                0x9d03290c       0x2c
 .text.TCPTaskPending
                0x9d03290c       0x2c build/default/production/_ext/427700826/tcp.o
                0x9d03290c                TCPTaskPending

.text.HTTPPrint_read_comm
                0x9d032938       0x2c
 .text.HTTPPrint_read_comm
                0x9d032938       0x2c build/default/production/_ext/1472/custom_http_app.o
                0x9d032938                HTTPPrint_read_comm

.text.HTTPPrint_write_comm
                0x9d032964       0x2c
 .text.HTTPPrint_write_comm
                0x9d032964       0x2c build/default/production/_ext/1472/custom_http_app.o
                0x9d032964                HTTPPrint_write_comm

.text.HTTPPrint_ddns_service
                0x9d032990       0x2c
 .text.HTTPPrint_ddns_service
                0x9d032990       0x2c build/default/production/_ext/1472/custom_http_app.o
                0x9d032990                HTTPPrint_ddns_service

.text.strchr    0x9d0329bc       0x2c
 .text.strchr   0x9d0329bc       0x2c c:/program files (x86)/microchip/xc32/v1.21/bin/../lib/gcc/pic32mx/4.5.2/../../../../pic32mx/lib/size\libc.a(strchr.o)
                0x9d0329bc                strchr

.text._stub_sbd_memlayout
                0x9d0329e8       0x2c
 .text._stub_sbd_memlayout
                0x9d0329e8       0x2c c:/program files (x86)/microchip/xc32/v1.21/bin/../lib/gcc/pic32mx/4.5.2/../../../../pic32mx/lib/size\libpic32.a(sbrk.o)
                0x9d0329e8                _stub_sbd_memlayout
                0x9d0329e8                _sbd_memlayout

.text.SYS_FS_GenError
                0x9d032a14       0x28
 .text.SYS_FS_GenError
                0x9d032a14       0x28 build/default/production/_ext/97638081/sys_fs.o

.rodata         0x9d032a3c       0x28
 .rodata        0x9d032a3c       0x28 build/default/production/_ext/792872985/usart.o

.text.ENCX24_MACGetTxBaseAddr
                0x9d032a64       0x28
 .text.ENCX24_MACGetTxBaseAddr
                0x9d032a64       0x28 build/default/production/_ext/427700826/encx24_mac.o

.text.ZCLLEnable
                0x9d032a8c       0x28
 .text.ZCLLEnable
                0x9d032a8c       0x28 build/default/production/_ext/427700826/zero_conf_link_local.o
                0x9d032a8c                ZCLLEnable

.text.INTClearFlag
                0x9d032ab4       0x28
 .text.INTClearFlag
                0x9d032ab4       0x28 c:/program files (x86)/microchip/xc32/v1.21/bin/../lib/gcc/pic32mx/4.5.2/../../../../pic32mx/lib/size\libmchp_peripheral_32MX795F512L.a(int_tbl_lib.o)
                0x9d032ab4                INTClearFlag

.text._ENCX24_Deinitialize
                0x9d032adc       0x24
 .text._ENCX24_Deinitialize
                0x9d032adc       0x24 build/default/production/_ext/427700826/encx24_mac.o

.text.TCPIP_STACK_GetDefaultNet
                0x9d032b00       0x24
 .text.TCPIP_STACK_GetDefaultNet
                0x9d032b00       0x24 build/default/production/_ext/427700826/tcpip_manager.o
                0x9d032b00                TCPIP_STACK_GetDefaultNet

.text.TCPIP_STACK_NetworksNo
                0x9d032b24       0x24
 .text.TCPIP_STACK_NetworksNo
                0x9d032b24       0x24 build/default/production/_ext/427700826/tcpip_manager.o
                0x9d032b24                TCPIP_STACK_NetworksNo

.text.HTTPPrint_lcdtext
                0x9d032b48       0x24
 .text.HTTPPrint_lcdtext
                0x9d032b48       0x24 build/default/production/_ext/1472/custom_http_app.o
                0x9d032b48                HTTPPrint_lcdtext

.text.HTTPPrint_ddns_user
                0x9d032b6c       0x24
 .text.HTTPPrint_ddns_user
                0x9d032b6c       0x24 build/default/production/_ext/1472/custom_http_app.o
                0x9d032b6c                HTTPPrint_ddns_user

.text.HTTPPrint_ddns_pass
                0x9d032b90       0x24
 .text.HTTPPrint_ddns_pass
                0x9d032b90       0x24 build/default/production/_ext/1472/custom_http_app.o
                0x9d032b90                HTTPPrint_ddns_pass

.text.HTTPPrint_ddns_host
                0x9d032bb4       0x24
 .text.HTTPPrint_ddns_host
                0x9d032bb4       0x24 build/default/production/_ext/1472/custom_http_app.o
                0x9d032bb4                HTTPPrint_ddns_host

.text._snprintf_cdnopsuxX
                0x9d032bd8       0x24
 .text._snprintf_cdnopsuxX
                0x9d032bd8       0x24 c:/program files (x86)/microchip/xc32/v1.21/bin/../lib/gcc/pic32mx/4.5.2/../../../../pic32mx/lib/size\libc.a(snprintf_cdnopsuxX.eo)
                0x9d032bd8                _snprintf_cdnopsuxX

.text.toupper   0x9d032bfc       0x24
 .text.toupper  0x9d032bfc       0x24 c:/program files (x86)/microchip/xc32/v1.21/bin/../lib/gcc/pic32mx/4.5.2/../../../../pic32mx/lib/size\libc.a(ctypef.o)
                0x9d032bfc                toupper

.rodata         0x9d032c20       0x20
 .rodata        0x9d032c20       0x20 build/default/production/_ext/427700826/arp.o

.text.SpiChnReadC
                0x9d032c40       0x20
 .text.SpiChnReadC
                0x9d032c40       0x20 c:/program files (x86)/microchip/xc32/v1.21/bin/../lib/gcc/pic32mx/4.5.2/../../../../pic32mx/lib/size\libmchp_peripheral_32MX795F512L.a(spi_chn_getc_lib.o)
                0x9d032c40                SpiChnReadC

.text.SpiChnWriteC
                0x9d032c60       0x20
 .text.SpiChnWriteC
                0x9d032c60       0x20 c:/program files (x86)/microchip/xc32/v1.21/bin/../lib/gcc/pic32mx/4.5.2/../../../../pic32mx/lib/size\libmchp_peripheral_32MX795F512L.a(spi_chn_putc_lib.o)
                0x9d032c60                SpiChnWriteC

.text.SpiChnTxBuffEmpty
                0x9d032c80       0x20
 .text.SpiChnTxBuffEmpty
                0x9d032c80       0x20 c:/program files (x86)/microchip/xc32/v1.21/bin/../lib/gcc/pic32mx/4.5.2/../../../../pic32mx/lib/size\libmchp_peripheral_32MX795F512L.a(spi_chn_tx_buff_empty_lib.o)
                0x9d032c80                SpiChnTxBuffEmpty

.text.INTRestoreInterrupts
                0x9d032ca0       0x1c
 .text.INTRestoreInterrupts
                0x9d032ca0       0x1c c:/program files (x86)/microchip/xc32/v1.21/bin/../lib/gcc/pic32mx/4.5.2/../../../../pic32mx/lib/size\libmchp_peripheral_32MX795F512L.a(int_restore_interrupts_lib.o)
                0x9d032ca0                INTRestoreInterrupts

.text.free      0x9d032cbc       0x1c
 .text.free     0x9d032cbc       0x1c c:/program files (x86)/microchip/xc32/v1.21/bin/../lib/gcc/pic32mx/4.5.2/../../../../pic32mx/lib/size\libc.a(malloc.o)
                0x9d032cbc                free

.text.srand     0x9d032cd8       0x1c
 .text.srand    0x9d032cd8       0x1c c:/program files (x86)/microchip/xc32/v1.21/bin/../lib/gcc/pic32mx/4.5.2/../../../../pic32mx/lib/size\libc.a(rand.o)
                0x9d032cd8                srand

.text.SYS_Reboot
                0x9d032cf4       0x18
 .text.SYS_Reboot
                0x9d032cf4       0x18 build/default/production/_ext/365611741/system_services.o
                0x9d032cf4                SYS_Reboot

.text.CheKseg0CacheOn
                0x9d032d0c       0x18
 .text.CheKseg0CacheOn
                0x9d032d0c       0x18 c:/program files (x86)/microchip/xc32/v1.21/bin/../lib/gcc/pic32mx/4.5.2/../../../../pic32mx/lib/size\libmchp_peripheral_32MX795F512L.a(pcache.o)
                0x9d032d0c                CheKseg0CacheOn

.text           0x9d032d24       0x18
 .text          0x9d032d24       0x18 c:/program files (x86)/microchip/xc32/v1.21/bin/../lib/gcc/pic32mx/4.5.2/../../../../pic32mx/lib/size\libpic32.a(default-nmi-handler.o)
                0x9d032d24                _nmi_handler

.rodata         0x9d032d3c       0x34
 .rodata        0x9d032d3c       0x14 c:/program files (x86)/microchip/xc32/v1.21/bin/../lib/gcc/pic32mx/4.5.2/../../../../pic32mx/lib/size\libmchp_peripheral_32MX795F512L.a(spi_map_tbl_libp.o)
                0x9d032d3c                _SpiMapTbl
 .rodata        0x9d032d50       0x10 build/default/production/_ext/97638081/mpfs2.o
 .rodata        0x9d032d60       0x10 build/default/production/_ext/427700826/dhcp.o

.text.OpenCoreTimer
                0x9d032d70        0xc
 .text.OpenCoreTimer
                0x9d032d70        0xc c:/program files (x86)/microchip/xc32/v1.21/bin/../lib/gcc/pic32mx/4.5.2/../../../../pic32mx/lib/size\libmchp_peripheral.a(open_core_timer_lib.o)
                0x9d032d70                OpenCoreTimer

.text._bootstrap_exception_handler
                0x9d032d7c        0xc
 .text._bootstrap_exception_handler
                0x9d032d7c        0xc c:/program files (x86)/microchip/xc32/v1.21/bin/../lib/gcc/pic32mx/4.5.2/../../../../pic32mx/lib/size\libpic32.a(default-bootstrap-exception-handler.o)
                0x9d032d7c                _bootstrap_exception_handler

.text.INTDisableInterrupts
                0x9d032d88        0x8
 .text.INTDisableInterrupts
                0x9d032d88        0x8 c:/program files (x86)/microchip/xc32/v1.21/bin/../lib/gcc/pic32mx/4.5.2/../../../../pic32mx/lib/size\libmchp_peripheral_32MX795F512L.a(int_disable_interrupts_lib.o)
                0x9d032d88                INTDisableInterrupts

.text.INTEnableInterrupts
                0x9d032d90        0x8
 .text.INTEnableInterrupts
                0x9d032d90        0x8 c:/program files (x86)/microchip/xc32/v1.21/bin/../lib/gcc/pic32mx/4.5.2/../../../../pic32mx/lib/size\libmchp_peripheral_32MX795F512L.a(int_enable_interrupts_lib.o)
                0x9d032d90                INTEnableInterrupts

.text._on_reset
                0x9d032d98        0x8
 .text._on_reset
                0x9d032d98        0x8 c:/program files (x86)/microchip/xc32/v1.21/bin/../lib/gcc/pic32mx/4.5.2/../../../../pic32mx/lib/size\libpic32.a(default-on-reset.o)
                0x9d032d98                _on_reset

.text._on_bootstrap
                0x9d032da0        0x8
 .text._on_bootstrap
                0x9d032da0        0x8 c:/program files (x86)/microchip/xc32/v1.21/bin/../lib/gcc/pic32mx/4.5.2/../../../../pic32mx/lib/size\libpic32.a(default-on-bootstrap.o)
                0x9d032da0                _on_bootstrap

.rodata         0x9d032da8        0x8
 .rodata        0x9d032da8        0x8 c:/program files (x86)/microchip/xc32/v1.21/bin/../lib/gcc/pic32mx/4.5.2/size\libgcc.a(_floatundisf.o)

.rodata         0x9d028474        0x4
 .rodata        0x9d028474        0x4 build/default/production/_ext/427700826/tcpip_announce.o
